 luafar3

 Timestamp is 61f9eaf9 (Wed Feb  2 02:22:49 2022)

 Preferred load address is 0000000180000000

 Start         Length     Name                   Class
 0001:00000000 000545b0H .text$mn                CODE
 0001:000545b0 00000040H .text$mn$00             CODE
 0001:000545f0 00000520H .text$x                 CODE
 0002:00000000 00000740H .idata$5                DATA
 0002:00000740 00000028H .00cfg                  DATA
 0002:00000768 00000008H .CRT$XCA                DATA
 0002:00000770 00000008H .CRT$XCZ                DATA
 0002:00000778 00000008H .CRT$XIA                DATA
 0002:00000780 00000018H .CRT$XIC                DATA
 0002:00000798 00000008H .CRT$XIZ                DATA
 0002:000007a0 00000008H .CRT$XPA                DATA
 0002:000007a8 00000018H .CRT$XPX                DATA
 0002:000007c0 00000008H .CRT$XPXA               DATA
 0002:000007c8 00000008H .CRT$XPZ                DATA
 0002:000007d0 00000008H .CRT$XTA                DATA
 0002:000007d8 00000008H .CRT$XTZ                DATA
 0002:000007e0 00000000H .gehcont$y              DATA
 0002:000007e0 00000000H .gfids$y                DATA
 0002:000007e0 000173a0H .rdata                  DATA
 0002:00017b80 00000000H .rdata$CastGuardVftablesA DATA
 0002:00017b80 00000000H .rdata$CastGuardVftablesC DATA
 0002:00017b80 00000000H .rdata$r                DATA
 0002:00017b80 00000020H .rdata$voltmd           DATA
 0002:00017ba0 000002f8H .rdata$zzzdbg           DATA
 0002:00017e98 00000008H .rtc$IAA                DATA
 0002:00017ea0 00000008H .rtc$IZZ                DATA
 0002:00017ea8 00000008H .rtc$TAA                DATA
 0002:00017eb0 00000008H .rtc$TZZ                DATA
 0002:00017eb8 000049f8H .xdata                  DATA
 0002:0001c8b0 00000000H .xdata$x                DATA
 0002:0001c8b0 0000049cH .edata                  DATA
 0002:0001cd4c 00000078H .idata$2                DATA
 0002:0001cdc4 00000014H .idata$3                DATA
 0002:0001cdd8 00000740H .idata$4                DATA
 0002:0001d518 00000ffcH .idata$6                DATA
 0003:00000000 0000bba0H .data                   DATA
 0003:0000bba0 00000000H .data$r                 DATA
 0003:0000bba0 00000000H .data$rs                DATA
 0003:0000bba0 00001250H .bss                    DATA
 0004:00000000 00004584H .pdata                  DATA
 0005:00000000 000000fcH _RDATA                  DATA
 0006:00000000 00000060H .rsrc$01                DATA
 0006:00000060 00000320H .rsrc$02                DATA

  Address         Publics by Value              Rva+Base               Lib:Object

 0000:00000000       __arm64x_redirection_metadata 0000000000000000     <absolute>
 0000:00000000       __guard_longjmp_table      0000000000000000     <absolute>
 0000:00000000       __x64_code_ranges_to_entry_points 0000000000000000     <absolute>
 0000:00000000       __guard_iat_count          0000000000000000     <absolute>
 0000:00000000       __guard_longjmp_count      0000000000000000     <absolute>
 0000:00000000       __dynamic_value_reloc_table 0000000000000000     <absolute>
 0000:00000000       __guard_fids_count         0000000000000000     <absolute>
 0000:00000000       __hybrid_auxiliary_iat     0000000000000000     <absolute>
 0000:00000000       __hybrid_auxiliary_iat_copy 0000000000000000     <absolute>
 0000:00000000       __arm64x_extra_rfe_table   0000000000000000     <absolute>
 0000:00000000       ___safe_se_handler_table   0000000000000000     <absolute>
 0000:00000000       __guard_iat_table          0000000000000000     <absolute>
 0000:00000000       __hybrid_code_map          0000000000000000     <absolute>
 0000:00000000       __arm64x_extra_rfe_table_size 0000000000000000     <absolute>
 0000:00000000       __AbsoluteZero             0000000000000000     <absolute>
 0000:00000000       ___safe_se_handler_count   0000000000000000     <absolute>
 0000:00000000       __guard_check_icall_a64n_fptr 0000000000000000     <absolute>
 0000:00000000       __guard_fids_table         0000000000000000     <absolute>
 0000:00000000       __x64_code_ranges_to_entry_points_count 0000000000000000     <absolute>
 0000:00000000       __guard_eh_cont_count      0000000000000000     <absolute>
 0000:00000000       __arm64x_redirection_metadata_count 0000000000000000     <absolute>
 0000:00000000       __enclave_config           0000000000000000     <absolute>
 0000:00000000       __guard_eh_cont_table      0000000000000000     <absolute>
 0000:00000000       __arm64x_native_entrypoint 0000000000000000     <absolute>
 0000:00000000       __hybrid_code_map_count    0000000000000000     <absolute>
 0000:00000100       __guard_flags              0000000000000100     <absolute>
 0000:00000000       __ImageBase                0000000180000000     <linker-defined>
 0001:00000000       __local_stdio_printf_options 0000000180001000 f i bit64.obj
 0001:00000010       sprintf                    0000000180001010 f i bit64.obj
 0001:00000070       bit64_pushuserdata         0000000180001070 f   bit64.obj
 0001:000000d0       bit64_push                 00000001800010d0 f   bit64.obj
 0001:00000160       bit64_getvalue             0000000180001160 f   bit64.obj
 0001:00000210       check64                    0000000180001210 f   bit64.obj
 0001:00000ee0       luaopen_bit64              0000000180001ee0 f   bit64.obj
 0001:00000f50       traceback                  0000000180001f50 f   exported.obj
 0001:00001010       GetExportFunction          0000000180002010 f   exported.obj
 0001:000010c0       pcall_msg                  00000001800020c0 f   exported.obj
 0001:00001290       PushPluginObject           0000000180002290 f   exported.obj
 0001:000012f0       PushPluginPair             00000001800022f0 f   exported.obj
 0001:00001370       _AddStringToCollector      0000000180002370 f   exported.obj
 0001:000014b0       AddBufToCollector          00000001800024b0 f   exported.obj
 0001:00001530       CreateStringsArray         0000000180002530 f   exported.obj
 0001:00001640       FarPanelItemFreeCallback   0000000180002640 f   exported.obj
 0001:00001670       FillPluginPanelItem        0000000180002670 f   exported.obj
 0001:00001e70       LF_GetFindData             0000000180002e70 f   exported.obj
 0001:00002090       LF_FreeFindData            0000000180003090 f   exported.obj
 0001:00002110       UpdateFileSelection        0000000180003110 f   exported.obj
 0001:000022f0       LF_GetFiles                00000001800032f0 f   exported.obj
 0001:00002520       RunDefaultScript           0000000180003520 f   exported.obj
 0001:00002820       LF_RunDefaultScript        0000000180003820 f   exported.obj
 0001:00002a40       LF_Analyse                 0000000180003a40 f   exported.obj
 0001:00002b10       LF_CloseAnalyse            0000000180003b10 f   exported.obj
 0001:00002b20       LF_GetOpenPanelInfo        0000000180003b20 f   exported.obj
 0001:00003710       PushFarMacroValue          0000000180004710 f   exported.obj
 0001:00003950       PackMacroValues            0000000180004950 f   exported.obj
 0001:00003cf0       LF_Open                    0000000180004cf0 f   exported.obj
 0001:00004340       LF_ClosePanel              0000000180005340 f   exported.obj
 0001:000043b0       LF_Compare                 00000001800053b0 f   exported.obj
 0001:00004460       LF_Configure               0000000180005460 f   exported.obj
 0001:000044f0       LF_DeleteFiles             00000001800054f0 f   exported.obj
 0001:000045a0       LF_MakeDirectory           00000001800055a0 f   exported.obj
 0001:000046a0       LF_ProcessPanelEvent       00000001800056a0 f   exported.obj
 0001:00004840       LF_ProcessHostFile         0000000180005840 f   exported.obj
 0001:00004930       LF_ProcessPanelInput       0000000180005930 f   exported.obj
 0001:000049c0       LF_PutFiles                00000001800059c0 f   exported.obj
 0001:00004b90       LF_SetDirectory            0000000180005b90 f   exported.obj
 0001:00004d20       LF_SetFindList             0000000180005d20 f   exported.obj
 0001:00004db0       LF_ExitFAR                 0000000180005db0 f   exported.obj
 0001:00004e50       getPluginMenuItems         0000000180005e50 f   exported.obj
 0001:00004f20       LF_GetPluginInfo           0000000180005f20 f   exported.obj
 0001:000050c0       LF_ProcessEditorInput      00000001800060c0 f   exported.obj
 0001:00005140       LF_ProcessEditorEvent      0000000180006140 f   exported.obj
 0001:00005460       LF_ProcessViewerEvent      0000000180006460 f   exported.obj
 0001:00005510       LF_ProcessDialogEvent      0000000180006510 f   exported.obj
 0001:00005850       LF_ProcessSynchroEvent     0000000180006850 f   exported.obj
 0001:00005a50       LF_GetContentFields        0000000180006a50 f   exported.obj
 0001:00005c10       LF_GetContentData          0000000180006c10 f   exported.obj
 0001:00005fc0       LF_FreeContentData         0000000180006fc0 f   exported.obj
 0001:00006010       LF_GetGlobalInfo           0000000180007010 f   exported.obj
 0001:000064e0       LF_ProcessConsoleInput     00000001800074e0 f   exported.obj
 0001:000066e0       LF_LoadFile                00000001800076e0 f   lflua.obj
 0001:00006a10       luaB_loadfileW             0000000180007a10 f   lflua.obj
 0001:00006b40       luaB_dofileW               0000000180007b40 f   lflua.obj
 0001:00006c70       LF_Gsub                    0000000180007c70 f   lflua.obj
 0001:00006dc0       method_gc                  0000000180007dc0 f   lregex.obj
 0001:00006e40       method_tostring            0000000180007e40 f   lregex.obj
 0001:00006eb0       check_regex_pattern        0000000180007eb0 f   lregex.obj
 0001:00006f80       push_far_regex             0000000180007f80 f   lregex.obj
 0001:00007030       _regex_gmatch_closure      0000000180008030 f   lregex.obj
 0001:000071b0       regex_gmatch_closure       00000001800081b0 f   lregex.obj
 0001:000071c0       regex_gmatch_closureW      00000001800081c0 f   lregex.obj
 0001:000071d0       _Gmatch                    00000001800081d0 f   lregex.obj
 0001:000073a0       func_Gmatch                00000001800083a0 f   lregex.obj
 0001:000073b0       func_GmatchW               00000001800083b0 f   lregex.obj
 0001:000073c0       rx_find_match              00000001800083c0 f   lregex.obj
 0001:000078e0       method_bracketscount       00000001800088e0 f   lregex.obj
 0001:00007960       rx_gsub                    0000000180008960 f   lregex.obj
 0001:00008550       func_New                   0000000180009550 f   lregex.obj
 0001:000085a0       method_find                00000001800095a0 f   lregex.obj
 0001:000085b0       func_find                  00000001800095b0 f   lregex.obj
 0001:000085c0       method_findW               00000001800095c0 f   lregex.obj
 0001:000085d0       func_findW                 00000001800095d0 f   lregex.obj
 0001:000085e0       method_match               00000001800095e0 f   lregex.obj
 0001:000085f0       func_match                 00000001800095f0 f   lregex.obj
 0001:00008600       method_matchW              0000000180009600 f   lregex.obj
 0001:000087f0       func_matchW                00000001800097f0 f   lregex.obj
 0001:000089d0       method_exec                00000001800099d0 f   lregex.obj
 0001:000089e0       func_exec                  00000001800099e0 f   lregex.obj
 0001:000089f0       method_execW               00000001800099f0 f   lregex.obj
 0001:00008a10       func_execW                 0000000180009a10 f   lregex.obj
 0001:00008a30       method_gsub                0000000180009a30 f   lregex.obj
 0001:00008a40       func_gsub                  0000000180009a40 f   lregex.obj
 0001:00008a50       method_gsubW               0000000180009a50 f   lregex.obj
 0001:00008a60       func_gsubW                 0000000180009a60 f   lregex.obj
 0001:00008a70       luaopen_regex              0000000180009a70 f   lregex.obj
 0001:00008e30       Open_Luamacro              0000000180009e30 f   luamacro.obj
 0001:00009410       far_MacroCallFar           000000018000a410 f   luamacro.obj
 0001:00009660       far_FarMacroCallToLua      000000018000a660 f   luamacro.obj
 0001:000097b0       uc_len                     000000018000a7b0 f   lusercontrol.obj
 0001:00009c30       luaopen_usercontrol        000000018000ac30 f   lusercontrol.obj
 0001:00009c80       CreateRegKey               000000018000ac80 f   reg.obj
 0001:00009ce0       fprintf                    000000018000ace0 f i service.obj
 0001:00009d30       DllMain                    000000018000ad30 f   service.obj
 0001:0000a060       GetFlagCombination         000000018000b060 f   service.obj
 0001:0000a340       OptFlags                   000000018000b340 f   service.obj
 0001:0000a4f0       ConvertLuaValue            000000018000b4f0 f   service.obj
 0001:0000aa60       StoreTempString            000000018000ba60 f   service.obj
 0001:0000ad70       PushPanelItem              000000018000bd70 f   service.obj
 0001:0000b480       PushPanelItems             000000018000c480 f   service.obj
 0001:0000e250       GetFarColor                000000018000f250 f   service.obj
 0001:0000e450       PushFarColor               000000018000f450 f   service.obj
 0001:0000ed50       PushInputRecord            000000018000fd50 f   service.obj
 0001:0000f180       FillInputRecord            0000000180010180 f   service.obj
 0001:000108a0       LF_Message                 00000001800118a0 f   service.obj
 0001:00010df0       LF_Error                   0000000180011df0 f   service.obj
 0001:00013880       CreateList                 0000000180014880 f   service.obj
 0001:00014ad0       NewDialogData              0000000180015ad0 f   service.obj
 0001:00014ba0       DialogHandleEqual          0000000180015ba0 f   service.obj
 0001:000165e0       PushDNParams               00000001800175e0 f   service.obj
 0001:000169c0       ProcessDNResult            00000001800179c0 f   service.obj
 0001:00016c90       LF_DlgProc                 0000000180017c90 f   service.obj
 0001:0001c9a0       MacroAddCallback           000000018001d9a0 f   service.obj
 0001:0001d360       pushFileTime               000000018001e360 f   service.obj
 0001:0001f0e0       TimerCallback              00000001800200e0 f   service.obj
 0001:00022180       LF_RunLuafarInit           0000000180023180 f   service.obj
 0001:00022290       _guard_check_icall_nop     0000000180023290 f   LIBCMT:guard_support.obj
 0001:00022290       LF_ProcessEnvVars          0000000180023290 f   service.obj
 0001:000222a0       LF_InitLuaState1           00000001800232a0 f   service.obj
 0001:00022570       LF_InitLuaState2           0000000180023570 f   service.obj
 0001:00022650       LF_MacroCallback           0000000180023650 f   service.obj
 0001:00022660       LF_DoFile                  0000000180023660 f   service.obj
 0001:000227f0       LF_GetLuafarAPI            00000001800237f0 f   service.obj
 0001:00022840       luaopen_luafar3            0000000180023840 f   service.obj
 0001:00022a60       _snwprintf                 0000000180023a60 f i slnunico.obj
 0001:00023520       luaopen_unicode            0000000180024520 f   slnunico.obj
 0001:00028ef0       luaopen_utf8               0000000180029ef0 f   lutf8lib.obj
 0001:000291c0       __local_stdio_scanf_options 000000018002a1c0 f i uliolib51.obj
 0001:000291d0       fscanf                     000000018002a1d0 f i uliolib51.obj
 0001:0002b030       luaopen_uio                000000018002c030 f   uliolib51.obj
 0001:0002c8b0       luaopen_upackage           000000018002d8b0 f   uloadlib51.obj
 0001:0002cb50       pusherrorcode              000000018002db50 f   ustring.obj
 0001:0002ccb0       SysErrorReturn             000000018002dcb0 f   ustring.obj
 0001:0002ccf0       PutIntToArray              000000018002dcf0 f   ustring.obj
 0001:0002cd40       PutIntToTable              000000018002dd40 f   ustring.obj
 0001:0002cd80       PutNumToTable              000000018002dd80 f   ustring.obj
 0001:0002cdc0       PutBoolToTable             000000018002ddc0 f   ustring.obj
 0001:0002ce00       PutStrToTable              000000018002de00 f   ustring.obj
 0001:0002ce40       PutStrToArray              000000018002de40 f   ustring.obj
 0001:0002ce80       PutWStrToTable             000000018002de80 f   ustring.obj
 0001:0002cec0       PutWStrToArray             000000018002dec0 f   ustring.obj
 0001:0002cf20       PutLStrToTable             000000018002df20 f   ustring.obj
 0001:0002cf60       GetOptNumFromTable         000000018002df60 f   ustring.obj
 0001:0002cfc0       GetOptIntFromTable         000000018002dfc0 f   ustring.obj
 0001:0002d020       GetOptIntFromArray         000000018002e020 f   ustring.obj
 0001:0002d090       GetBoolFromTable           000000018002e090 f   ustring.obj
 0001:0002d0e0       GetOptBoolFromTable        000000018002e0e0 f   ustring.obj
 0001:0002d140       check_utf8_string          000000018002e140 f   ustring.obj
 0001:0002d250       utf8_to_utf16              000000018002e250 f   ustring.obj
 0001:0002d370       opt_utf8_string            000000018002e370 f   ustring.obj
 0001:0002d3c0       push_multibyte_string      000000018002e3c0 f   ustring.obj
 0001:0002d4d0       push_utf8_string           000000018002e4d0 f   ustring.obj
 0001:0002d500       ustring_WideCharToMultiByte 000000018002e500 f   ustring.obj
 0001:0002d690       ustring_MultiByteToWideChar 000000018002e690 f   ustring.obj
 0001:0002d830       ustring_OemToUtf8          000000018002e830 f   ustring.obj
 0001:0002d940       ustring_Utf8ToOem          000000018002e940 f   ustring.obj
 0001:0002dae0       ustring_Utf16ToUtf8        000000018002eae0 f   ustring.obj
 0001:0002db30       ustring_Utf8ToUtf16        000000018002eb30 f   ustring.obj
 0001:0002dc10       ustring_GetACP             000000018002ec10 f   ustring.obj
 0001:0002dc40       ustring_GetOEMCP           000000018002ec40 f   ustring.obj
 0001:0002dc70       ustring_GetConsoleCP       000000018002ec70 f   ustring.obj
 0001:0002dca0       ustring_SetConsoleCP       000000018002eca0 f   ustring.obj
 0001:0002dd10       ustring_GetConsoleOutputCP 000000018002ed10 f   ustring.obj
 0001:0002dd40       ustring_SetConsoleOutputCP 000000018002ed40 f   ustring.obj
 0001:0002ddb0       EnumCodePagesProc          000000018002edb0 f   ustring.obj
 0001:0002ded0       ustring_EnumSystemCodePages 000000018002eed0 f   ustring.obj
 0001:0002df60       ustring_GetCPInfo          000000018002ef60 f   ustring.obj
 0001:0002e230       ustring_GetLogicalDriveStrings 000000018002f230 f   ustring.obj
 0001:0002e3e0       ustring_GetDriveType       000000018002f3e0 f   ustring.obj
 0001:0002e570       ustring_Uuid               000000018002f570 f   ustring.obj
 0001:0002e640       ustring_SearchPath         000000018002f640 f   ustring.obj
 0001:0002ea80       ustring_GlobalMemoryStatus 000000018002fa80 f   ustring.obj
 0001:0002ed40       ustring_Sleep              000000018002fd40 f   ustring.obj
 0001:0002ed70       PushAttrString             000000018002fd70 f   ustring.obj
 0001:0002ee80       DecodeAttributes           000000018002fe80 f   ustring.obj
 0001:0002ef80       SetAttrWords               000000018002ff80 f   ustring.obj
 0001:0002f160       ustring_SetFileAttr        0000000180030160 f   ustring.obj
 0001:0002f2a0       ustring_GetFileAttr        00000001800302a0 f   ustring.obj
 0001:0002f3c0       ustring_SHGetFolderPath    00000001800303c0 f   ustring.obj
 0001:0002f520       push_utf16_string          0000000180030520 f   ustring.obj
 0001:0002f550       ustring_sub                0000000180030550 f   ustring.obj
 0001:0002f610       ustring_len                0000000180030610 f   ustring.obj
 0001:0002f650       check_utf16_string         0000000180030650 f   ustring.obj
 0001:0002f680       opt_utf16_string           0000000180030680 f   ustring.obj
 0001:0002f990       ustring_GetCurrentDir      0000000180030990 f   ustring.obj
 0001:0002fbe0       ustring_SetCurrentDir      0000000180030be0 f   ustring.obj
 0001:0002fd00       ustring_GetKeyState        0000000180030d00 f   ustring.obj
 0001:0002fd60       luaopen_ustring            0000000180030d60 f   ustring.obj
 0001:0002fdc0       GetIntFromArray            0000000180030dc0 f   util.obj
 0001:0002fe90       GetFileTimeFromTable       0000000180030e90 f   util.obj
 0001:0002ffa0       PutFileTimeToTable         0000000180030fa0 f   util.obj
 0001:00033e60       win_WriteConsole           0000000180034e60 f   win.obj
 0001:000340b0       win_IsWinVersion           00000001800350b0 f   win.obj
 0001:00034e60       luaopen_win                0000000180035e60 f   win.obj
 0001:00034eea       luaopen_table              0000000180035eea f   lua51:lua51.dll
 0001:00034ef0       luaopen_base               0000000180035ef0 f   lua51:lua51.dll
 0001:00034ef6       luaopen_os                 0000000180035ef6 f   lua51:lua51.dll
 0001:00034efc       luaopen_string             0000000180035efc f   lua51:lua51.dll
 0001:00034f02       luaopen_math               0000000180035f02 f   lua51:lua51.dll
 0001:00034f08       luaopen_debug              0000000180035f08 f   lua51:lua51.dll
 0001:00034f20       __security_check_cookie    0000000180035f20 f   LIBCMT:amdsecgs.obj
 0001:00034f40       __raise_securityfailure    0000000180035f40 f   LIBCMT:gs_report.obj
 0001:00034f74       __report_gsfailure         0000000180035f74 f   LIBCMT:gs_report.obj
 0001:00035048       __report_rangecheckfailure 0000000180036048 f   LIBCMT:gs_report.obj
 0001:0003505c       __report_securityfailure   000000018003605c f   LIBCMT:gs_report.obj
 0001:000354fc       _DllMainCRTStartup         00000001800364fc f   LIBCMT:dll_dllmain.obj
 0001:0003553c       __security_init_cookie     000000018003653c f   LIBCMT:gs_support.obj
 0001:000355e8       ?__scrt_initialize_type_info@@YAXXZ 00000001800365e8 f   LIBCMT:tncleanup.obj
 0001:000355f8       ?__scrt_uninitialize_type_info@@YAXXZ 00000001800365f8 f   LIBCMT:tncleanup.obj
 0001:00035604       __scrt_initialize_default_local_stdio_options 0000000180036604 f   LIBCMT:default_local_stdio_options.obj
 0001:00035620       __scrt_acquire_startup_lock 0000000180036620 f   LIBCMT:utility.obj
 0001:0003565c       __scrt_dllmain_after_initialize_c 000000018003665c f   LIBCMT:utility.obj
 0001:00035690       __scrt_dllmain_before_initialize_c 0000000180036690 f   LIBCMT:utility.obj
 0001:000356a8       __scrt_dllmain_crt_thread_attach 00000001800366a8 f   LIBCMT:utility.obj
 0001:000356d0       __scrt_dllmain_crt_thread_detach 00000001800366d0 f   LIBCMT:utility.obj
 0001:000356e8       __scrt_dllmain_exception_filter 00000001800366e8 f   LIBCMT:utility.obj
 0001:00035748       __scrt_dllmain_uninitialize_c 0000000180036748 f   LIBCMT:utility.obj
 0001:00035778       __scrt_dllmain_uninitialize_critical 0000000180036778 f   LIBCMT:utility.obj
 0001:0003578c       __scrt_initialize_crt      000000018003678c f   LIBCMT:utility.obj
 0001:000357d8       __scrt_initialize_onexit_tables 00000001800367d8 f   LIBCMT:utility.obj
 0001:00035864       __scrt_is_nonwritable_in_current_image 0000000180036864 f   LIBCMT:utility.obj
 0001:000358fc       __scrt_release_startup_lock 00000001800368fc f   LIBCMT:utility.obj
 0001:00035920       __scrt_uninitialize_crt    0000000180036920 f   LIBCMT:utility.obj
 0001:0003594c       __scrt_get_dyn_tls_init_callback 000000018003694c f   LIBCMT:dyn_tls_init.obj
 0001:00035954       __crt_debugger_hook        0000000180036954 f   LIBCMT:utility_desktop.obj
 0001:0003595c       __scrt_fastfail            000000018003695c f   LIBCMT:utility_desktop.obj
 0001:00035aa8       _RTC_Initialize            0000000180036aa8 f   LIBCMT:initsect.obj
 0001:00035ae4       _RTC_Terminate             0000000180036ae4 f   LIBCMT:initsect.obj
 0001:00035b20       __isa_available_init       0000000180036b20 f   LIBCMT:cpu_disp.obj
 0001:00035cc4       _get_startup_argv_mode     0000000180036cc4 f   LIBCMT:argv_mode.obj
 0001:00035ccc       __scrt_is_ucrt_dll_in_use  0000000180036ccc f   LIBCMT:ucrt_detection.obj
 0001:00035ce0       wcsrchr                    0000000180036ce0 f   libvcruntime:wcsrchr.obj
 0001:00035d90       wcsstr                     0000000180036d90 f   libvcruntime:wcsstr.obj
 0001:00035fa8       wcschr                     0000000180036fa8 f   libvcruntime:wcschr.obj
 0001:00036024       strchr                     0000000180037024 f   libvcruntime:strchr.obj
 0001:000360a4       strrchr                    00000001800370a4 f   libvcruntime:strrchr.obj
 0001:000361d0       __C_specific_handler       00000001800371d0 f   libvcruntime:riscchandler.obj
 0001:000363dc       __std_type_info_destroy_list 00000001800373dc f   libvcruntime:std_type_info.obj
 0001:00036408       __vcrt_initialize          0000000180037408 f   libvcruntime:initialization.obj
 0001:00036430       __vcrt_thread_attach       0000000180037430 f   libvcruntime:initialization.obj
 0001:00036444       __vcrt_thread_detach       0000000180037444 f   libvcruntime:initialization.obj
 0001:00036458       __vcrt_uninitialize        0000000180037458 f   libvcruntime:initialization.obj
 0001:00036474       __vcrt_uninitialize_critical 0000000180037474 f   libvcruntime:initialization.obj
 0001:00036484       __DestructExceptionObject  0000000180037484 f   libvcruntime:ehhelpers.obj
 0001:000364f4       ?_CallMemberFunction0@@YAXQEAX0@Z 00000001800374f4 f i libvcruntime:ehhelpers.obj
 0001:00036510       memset_repmovs             0000000180037510 f   libvcruntime:memset.obj
 0001:00036530       memset                     0000000180037530 f   libvcruntime:memset.obj
 0001:000366d0       _NLG_Notify                00000001800376d0 f   libvcruntime:notify.obj
 0001:000366f0       __NLG_Dispatch2            00000001800376f0 f   libvcruntime:notify.obj
 0001:00036700       __NLG_Return2              0000000180037700 f   libvcruntime:notify.obj
 0001:00036704       __except_validate_context_record 0000000180037704 f   libvcruntime:jbcxrval.obj
 0001:0003673c       __vcrt_freefls             000000018003773c f   libvcruntime:per_thread_data.obj
 0001:0003675c       __vcrt_freeptd             000000018003775c f   libvcruntime:per_thread_data.obj
 0001:000367ac       __vcrt_getptd              00000001800377ac f   libvcruntime:per_thread_data.obj
 0001:000367c8       __vcrt_getptd_noexit       00000001800377c8 f   libvcruntime:per_thread_data.obj
 0001:00036888       __vcrt_initialize_ptd      0000000180037888 f   libvcruntime:per_thread_data.obj
 0001:000368d0       __vcrt_uninitialize_ptd    00000001800378d0 f   libvcruntime:per_thread_data.obj
 0001:000368f4       __vcrt_initialize_locks    00000001800378f4 f   libvcruntime:locks.obj
 0001:00036928       __vcrt_uninitialize_locks  0000000180037928 f   libvcruntime:locks.obj
 0001:00036970       memcpy_repmovs             0000000180037970 f   libvcruntime:memcpy.obj
 0001:00036990       memcpy                     0000000180037990 f   libvcruntime:memcpy.obj
 0001:00036990       memmove                    0000000180037990 f   libvcruntime:memcpy.obj
 0001:00037158       __vcrt_FlsAlloc            0000000180038158 f   libvcruntime:winapi_downlevel.obj
 0001:000371a0       __vcrt_FlsFree             00000001800381a0 f   libvcruntime:winapi_downlevel.obj
 0001:000371e8       __vcrt_FlsGetValue         00000001800381e8 f   libvcruntime:winapi_downlevel.obj
 0001:00037230       __vcrt_FlsSetValue         0000000180038230 f   libvcruntime:winapi_downlevel.obj
 0001:00037284       __vcrt_InitializeCriticalSectionEx 0000000180038284 f   libvcruntime:winapi_downlevel.obj
 0001:00037300       _CallSettingFrame          0000000180038300 f   libvcruntime:handlers.obj
 0001:00037350       _CallSettingFrame_LookupContinuationIndex 0000000180038350 f   libvcruntime:handlers.obj
 0001:00037380       _CallSettingFrame_NotifyContinuationAddr 0000000180038380 f   libvcruntime:handlers.obj
 0001:000373b0       _CallSettingFrameEncoded   00000001800383b0 f   libvcruntime:handlers.obj
 0001:000377d8       ??$ensure_buffer_is_big_enough@D@formatting_buffer@__crt_stdio_output@@QEAA_N_K@Z 00000001800387d8 f i libucrt:output.obj
 0001:00037880       ??$ensure_buffer_is_big_enough@_W@formatting_buffer@__crt_stdio_output@@QEAA_N_K@Z 0000000180038880 f i libucrt:output.obj
 0001:0003792c       ??$is_wide_character_specifier@_W@__crt_stdio_output@@YA_N_K_WW4length_modifier@0@@Z 000000018003892c f i libucrt:output.obj
 0001:0003796c       ??$type_case_integer_parse_into_buffer@I@?$output_processor@DV?$stream_output_adapter@D@__crt_stdio_output@@V?$standard_base@DV?$stream_output_adapter@D@__crt_stdio_output@@@2@@__crt_stdio_output@@AEAAXII_N@Z 000000018003896c f i libucrt:output.obj
 0001:0003796c       ??$type_case_integer_parse_into_buffer@I@?$output_processor@DV?$string_output_adapter@D@__crt_stdio_output@@V?$standard_base@DV?$string_output_adapter@D@__crt_stdio_output@@@2@@__crt_stdio_output@@AEAAXII_N@Z 000000018003896c f i libucrt:output.obj
 0001:000379f4       ??$type_case_integer_parse_into_buffer@I@?$output_processor@_WV?$string_output_adapter@_W@__crt_stdio_output@@V?$standard_base@_WV?$string_output_adapter@_W@__crt_stdio_output@@@2@@__crt_stdio_output@@AEAAXII_N@Z 00000001800389f4 f i libucrt:output.obj
 0001:00037a98       ??$type_case_integer_parse_into_buffer@_K@?$output_processor@DV?$stream_output_adapter@D@__crt_stdio_output@@V?$standard_base@DV?$stream_output_adapter@D@__crt_stdio_output@@@2@@__crt_stdio_output@@AEAAX_KI_N@Z 0000000180038a98 f i libucrt:output.obj
 0001:00037a98       ??$type_case_integer_parse_into_buffer@_K@?$output_processor@DV?$string_output_adapter@D@__crt_stdio_output@@V?$standard_base@DV?$string_output_adapter@D@__crt_stdio_output@@@2@@__crt_stdio_output@@AEAAX_KI_N@Z 0000000180038a98 f i libucrt:output.obj
 0001:00037b28       ??$type_case_integer_parse_into_buffer@_K@?$output_processor@_WV?$string_output_adapter@_W@__crt_stdio_output@@V?$standard_base@_WV?$string_output_adapter@_W@__crt_stdio_output@@@2@@__crt_stdio_output@@AEAAX_KI_N@Z 0000000180038b28 f i libucrt:output.obj
 0001:00037bcc       ??$write_multiple_characters@V?$stream_output_adapter@D@__crt_stdio_output@@D@__crt_stdio_output@@YAXAEBV?$stream_output_adapter@D@0@DHQEAH@Z 0000000180038bcc f i libucrt:output.obj
 0001:00037c58       ??$write_multiple_characters@V?$string_output_adapter@D@__crt_stdio_output@@D@__crt_stdio_output@@YAXAEBV?$string_output_adapter@D@0@DHQEAH@Z 0000000180038c58 f i libucrt:output.obj
 0001:00037cd0       ??$write_multiple_characters@V?$string_output_adapter@_W@__crt_stdio_output@@D@__crt_stdio_output@@YAXAEBV?$string_output_adapter@_W@0@DHQEAH@Z 0000000180038cd0 f i libucrt:output.obj
 0001:00037d4c       ??0_LocaleUpdate@@QEAA@QEAU__crt_locale_pointers@@@Z 0000000180038d4c f i libucrt:output.obj
 0001:00037f18       ?crop_zeroes@__crt_stdio_output@@YAXPEADQEAU__crt_locale_pointers@@@Z 0000000180038f18 f i libucrt:output.obj
 0001:00037f84       ?parse_int_from_format_string@?$output_processor@DV?$stream_output_adapter@D@__crt_stdio_output@@V?$standard_base@DV?$stream_output_adapter@D@__crt_stdio_output@@@2@@__crt_stdio_output@@AEAA_NQEAH@Z 0000000180038f84 f i libucrt:output.obj
 0001:00037f84       ?parse_int_from_format_string@?$output_processor@DV?$string_output_adapter@D@__crt_stdio_output@@V?$standard_base@DV?$string_output_adapter@D@__crt_stdio_output@@@2@@__crt_stdio_output@@AEAA_NQEAH@Z 0000000180038f84 f i libucrt:output.obj
 0001:00038028       ?parse_int_from_format_string@?$output_processor@_WV?$string_output_adapter@_W@__crt_stdio_output@@V?$standard_base@_WV?$string_output_adapter@_W@__crt_stdio_output@@@2@@__crt_stdio_output@@AEAA_NQEAH@Z 0000000180039028 f i libucrt:output.obj
 0001:000380cc       ?process@?$output_processor@DV?$stream_output_adapter@D@__crt_stdio_output@@V?$standard_base@DV?$stream_output_adapter@D@__crt_stdio_output@@@2@@__crt_stdio_output@@QEAAHXZ 00000001800390cc f i libucrt:output.obj
 0001:000382e4       ?process@?$output_processor@DV?$string_output_adapter@D@__crt_stdio_output@@V?$standard_base@DV?$string_output_adapter@D@__crt_stdio_output@@@2@@__crt_stdio_output@@QEAAHXZ 00000001800392e4 f i libucrt:output.obj
 0001:000384f0       ?process@?$output_processor@_WV?$string_output_adapter@_W@__crt_stdio_output@@V?$standard_base@_WV?$string_output_adapter@_W@__crt_stdio_output@@@2@@__crt_stdio_output@@QEAAHXZ 00000001800394f0 f i libucrt:output.obj
 0001:0003876c       ?state_case_normal@?$output_processor@DV?$stream_output_adapter@D@__crt_stdio_output@@V?$standard_base@DV?$stream_output_adapter@D@__crt_stdio_output@@@2@@__crt_stdio_output@@AEAA_NXZ 000000018003976c f i libucrt:output.obj
 0001:000387dc       ?state_case_normal@?$output_processor@DV?$string_output_adapter@D@__crt_stdio_output@@V?$standard_base@DV?$string_output_adapter@D@__crt_stdio_output@@@2@@__crt_stdio_output@@AEAA_NXZ 00000001800397dc f i libucrt:output.obj
 0001:00038850       ?state_case_normal_tchar@?$output_processor@DV?$stream_output_adapter@D@__crt_stdio_output@@V?$standard_base@DV?$stream_output_adapter@D@__crt_stdio_output@@@2@@__crt_stdio_output@@AEAA_ND@Z 0000000180039850 f i libucrt:output.obj
 0001:000388f4       ?state_case_normal_tchar@?$output_processor@DV?$string_output_adapter@D@__crt_stdio_output@@V?$standard_base@DV?$string_output_adapter@D@__crt_stdio_output@@@2@@__crt_stdio_output@@AEAA_ND@Z 00000001800398f4 f i libucrt:output.obj
 0001:0003899c       ?state_case_size@?$output_processor@DV?$stream_output_adapter@D@__crt_stdio_output@@V?$standard_base@DV?$stream_output_adapter@D@__crt_stdio_output@@@2@@__crt_stdio_output@@AEAA_NXZ 000000018003999c f i libucrt:output.obj
 0001:00038b10       ?state_case_size@?$output_processor@DV?$string_output_adapter@D@__crt_stdio_output@@V?$standard_base@DV?$string_output_adapter@D@__crt_stdio_output@@@2@@__crt_stdio_output@@AEAA_NXZ 0000000180039b10 f i libucrt:output.obj
 0001:00038c84       ?state_case_size@?$output_processor@_WV?$string_output_adapter@_W@__crt_stdio_output@@V?$standard_base@_WV?$string_output_adapter@_W@__crt_stdio_output@@@2@@__crt_stdio_output@@AEAA_NXZ 0000000180039c84 f i libucrt:output.obj
 0001:00038e1c       ?state_case_type@?$output_processor@DV?$stream_output_adapter@D@__crt_stdio_output@@V?$standard_base@DV?$stream_output_adapter@D@__crt_stdio_output@@@2@@__crt_stdio_output@@AEAA_NXZ 0000000180039e1c f i libucrt:output.obj
 0001:000390a0       ?state_case_type@?$output_processor@DV?$string_output_adapter@D@__crt_stdio_output@@V?$standard_base@DV?$string_output_adapter@D@__crt_stdio_output@@@2@@__crt_stdio_output@@AEAA_NXZ 000000018003a0a0 f i libucrt:output.obj
 0001:00039308       ?state_case_type@?$output_processor@_WV?$string_output_adapter@_W@__crt_stdio_output@@V?$standard_base@_WV?$string_output_adapter@_W@__crt_stdio_output@@@2@@__crt_stdio_output@@AEAA_NXZ 000000018003a308 f i libucrt:output.obj
 0001:000395d4       ?type_case_Z@?$output_processor@DV?$stream_output_adapter@D@__crt_stdio_output@@V?$standard_base@DV?$stream_output_adapter@D@__crt_stdio_output@@@2@@__crt_stdio_output@@AEAA_NXZ 000000018003a5d4 f i libucrt:output.obj
 0001:000395d4       ?type_case_Z@?$output_processor@DV?$string_output_adapter@D@__crt_stdio_output@@V?$standard_base@DV?$string_output_adapter@D@__crt_stdio_output@@@2@@__crt_stdio_output@@AEAA_NXZ 000000018003a5d4 f i libucrt:output.obj
 0001:00039648       ?type_case_Z@?$output_processor@_WV?$string_output_adapter@_W@__crt_stdio_output@@V?$standard_base@_WV?$string_output_adapter@_W@__crt_stdio_output@@@2@@__crt_stdio_output@@AEAA_NXZ 000000018003a648 f i libucrt:output.obj
 0001:000396c4       ?type_case_a@?$output_processor@DV?$string_output_adapter@D@__crt_stdio_output@@V?$standard_base@DV?$string_output_adapter@D@__crt_stdio_output@@@2@@__crt_stdio_output@@AEAA_NXZ 000000018003a6c4 f i libucrt:output.obj
 0001:000396c4       ?type_case_a@?$output_processor@DV?$stream_output_adapter@D@__crt_stdio_output@@V?$standard_base@DV?$stream_output_adapter@D@__crt_stdio_output@@@2@@__crt_stdio_output@@AEAA_NXZ 000000018003a6c4 f i libucrt:output.obj
 0001:000398dc       ?type_case_a@?$output_processor@_WV?$string_output_adapter@_W@__crt_stdio_output@@V?$standard_base@_WV?$string_output_adapter@_W@__crt_stdio_output@@@2@@__crt_stdio_output@@AEAA_NXZ 000000018003a8dc f i libucrt:output.obj
 0001:00039b18       ?type_case_c_tchar@?$output_processor@DV?$stream_output_adapter@D@__crt_stdio_output@@V?$standard_base@DV?$stream_output_adapter@D@__crt_stdio_output@@@2@@__crt_stdio_output@@AEAA_ND@Z 000000018003ab18 f i libucrt:output.obj
 0001:00039b18       ?type_case_c_tchar@?$output_processor@DV?$string_output_adapter@D@__crt_stdio_output@@V?$standard_base@DV?$string_output_adapter@D@__crt_stdio_output@@@2@@__crt_stdio_output@@AEAA_ND@Z 000000018003ab18 f i libucrt:output.obj
 0001:00039bd4       ?type_case_c_tchar@?$output_processor@_WV?$string_output_adapter@_W@__crt_stdio_output@@V?$standard_base@_WV?$string_output_adapter@_W@__crt_stdio_output@@@2@@__crt_stdio_output@@AEAA_N_W@Z 000000018003abd4 f i libucrt:output.obj
 0001:00039c7c       ?type_case_integer@?$output_processor@DV?$string_output_adapter@D@__crt_stdio_output@@V?$standard_base@DV?$string_output_adapter@D@__crt_stdio_output@@@2@@__crt_stdio_output@@AEAA_NI_N@Z 000000018003ac7c f i libucrt:output.obj
 0001:00039c7c       ?type_case_integer@?$output_processor@DV?$stream_output_adapter@D@__crt_stdio_output@@V?$standard_base@DV?$stream_output_adapter@D@__crt_stdio_output@@@2@@__crt_stdio_output@@AEAA_NI_N@Z 000000018003ac7c f i libucrt:output.obj
 0001:00039e44       ?type_case_integer@?$output_processor@_WV?$string_output_adapter@_W@__crt_stdio_output@@V?$standard_base@_WV?$string_output_adapter@_W@__crt_stdio_output@@@2@@__crt_stdio_output@@AEAA_NI_N@Z 000000018003ae44 f i libucrt:output.obj
 0001:0003a010       ?type_case_n@?$output_processor@DV?$string_output_adapter@D@__crt_stdio_output@@V?$standard_base@DV?$string_output_adapter@D@__crt_stdio_output@@@2@@__crt_stdio_output@@AEAA_NXZ 000000018003b010 f i libucrt:output.obj
 0001:0003a010       ?type_case_n@?$output_processor@DV?$stream_output_adapter@D@__crt_stdio_output@@V?$standard_base@DV?$stream_output_adapter@D@__crt_stdio_output@@@2@@__crt_stdio_output@@AEAA_NXZ 000000018003b010 f i libucrt:output.obj
 0001:0003a010       ?type_case_n@?$output_processor@_WV?$string_output_adapter@_W@__crt_stdio_output@@V?$standard_base@_WV?$string_output_adapter@_W@__crt_stdio_output@@@2@@__crt_stdio_output@@AEAA_NXZ 000000018003b010 f i libucrt:output.obj
 0001:0003a0ec       ?type_case_s@?$output_processor@DV?$stream_output_adapter@D@__crt_stdio_output@@V?$standard_base@DV?$stream_output_adapter@D@__crt_stdio_output@@@2@@__crt_stdio_output@@AEAA_NXZ 000000018003b0ec f i libucrt:output.obj
 0001:0003a0ec       ?type_case_s@?$output_processor@DV?$string_output_adapter@D@__crt_stdio_output@@V?$standard_base@DV?$string_output_adapter@D@__crt_stdio_output@@@2@@__crt_stdio_output@@AEAA_NXZ 000000018003b0ec f i libucrt:output.obj
 0001:0003a184       ?type_case_s@?$output_processor@_WV?$string_output_adapter@_W@__crt_stdio_output@@V?$standard_base@_WV?$string_output_adapter@_W@__crt_stdio_output@@@2@@__crt_stdio_output@@AEAA_NXZ 000000018003b184 f i libucrt:output.obj
 0001:0003a24c       ?validate_stream_is_ansi_if_required@?$__acrt_stdio_char_traits@D@@SA_NQEAU_iobuf@@@Z 000000018003b24c f i libucrt:output.obj
 0001:0003a2e8       ?write_stored_string_tchar@?$output_processor@DV?$stream_output_adapter@D@__crt_stdio_output@@V?$standard_base@DV?$stream_output_adapter@D@__crt_stdio_output@@@2@@__crt_stdio_output@@AEAA_ND@Z 000000018003b2e8 f i libucrt:output.obj
 0001:0003a40c       ?write_stored_string_tchar@?$output_processor@DV?$string_output_adapter@D@__crt_stdio_output@@V?$standard_base@DV?$string_output_adapter@D@__crt_stdio_output@@@2@@__crt_stdio_output@@AEAA_ND@Z 000000018003b40c f i libucrt:output.obj
 0001:0003a4e4       ?write_stored_string_tchar@?$output_processor@_WV?$string_output_adapter@_W@__crt_stdio_output@@V?$standard_base@_WV?$string_output_adapter@_W@__crt_stdio_output@@@2@@__crt_stdio_output@@AEAA_N_W@Z 000000018003b4e4 f i libucrt:output.obj
 0001:0003a5d0       ?write_string@?$string_output_adapter@D@__crt_stdio_output@@QEBAXQEBDHQEAHAEAV__crt_deferred_errno_cache@@@Z 000000018003b5d0 f i libucrt:output.obj
 0001:0003a674       ?write_string@?$string_output_adapter@_W@__crt_stdio_output@@QEBAXQEB_WHQEAHAEAV__crt_deferred_errno_cache@@@Z 000000018003b674 f i libucrt:output.obj
 0001:0003a71c       ?write_string_impl@?$output_adapter_common@DV?$stream_output_adapter@D@__crt_stdio_output@@@__crt_stdio_output@@IEBAXQEBDHQEAHAEAV__crt_deferred_errno_cache@@@Z 000000018003b71c f i libucrt:output.obj
 0001:0003a814       __stdio_common_vfprintf    000000018003b814 f   libucrt:output.obj
 0001:0003a8a0       __stdio_common_vsprintf    000000018003b8a0 f   libucrt:output.obj
 0001:0003a8a8       __stdio_common_vswprintf   000000018003b8a8 f   libucrt:output.obj
 0001:0003a8b0       _fclose_nolock             000000018003b8b0 f   libucrt:fclose.obj
 0001:0003a934       fclose                     000000018003b934 f   libucrt:fclose.obj
 0001:0003a998       wcsdup                     000000018003b998 f   libucrt:wcsdup.obj
 0001:0003a998       _wcsdup                    000000018003b998 f   libucrt:wcsdup.obj
 0001:0003aa1c       _clearfp                   000000018003ba1c f   libucrt:ieee.obj
 0001:0003aa8c       _control87                 000000018003ba8c f   libucrt:ieee.obj
 0001:0003ae20       _wfopen                    000000018003be20 f   libucrt:fopen.obj
 0001:0003ae2c       free                       000000018003be2c f   libucrt:free.obj
 0001:0003ae40       malloc                     000000018003be40 f   libucrt:malloc.obj
 0001:0003ae48       feof                       000000018003be48 f   libucrt:feoferr.obj
 0001:0003ae74       ferror                     000000018003be74 f   libucrt:feoferr.obj
 0001:0003aea0       __acrt_initialize_stdio    000000018003bea0 f   libucrt:_file.obj
 0001:0003afc0       __acrt_iob_func            000000018003bfc0 f   libucrt:_file.obj
 0001:0003afd4       __acrt_uninitialize_stdio  000000018003bfd4 f   libucrt:_file.obj
 0001:0003b030       _lock_file                 000000018003c030 f   libucrt:_file.obj
 0001:0003b03c       _unlock_file               000000018003c03c f   libucrt:_file.obj
 0001:0003b048       _fgetc_nolock              000000018003c048 f   libucrt:fgetc.obj
 0001:0003b08c       _getc_nolock               000000018003c08c f   libucrt:fgetc.obj
 0001:0003b094       fgetc                      000000018003c094 f   libucrt:fgetc.obj
 0001:0003b19c       getc                       000000018003c19c f   libucrt:fgetc.obj
 0001:0003b2a4       _wfreopen                  000000018003c2a4 f   libucrt:freopen.obj
 0001:0003b2d4       rewind                     000000018003c2d4 f   libucrt:rewind.obj
 0001:0003b398       __acrt_errno_from_os_error 000000018003c398 f   libucrt:errno.obj
 0001:0003b3e0       __acrt_errno_map_os_error  000000018003c3e0 f   libucrt:errno.obj
 0001:0003b430       __doserrno                 000000018003c430 f   libucrt:errno.obj
 0001:0003b450       _errno                     000000018003c450 f   libucrt:errno.obj
 0001:0003b470       _ungetc_nolock             000000018003c470 f   libucrt:ungetc.obj
 0001:0003b598       ungetc                     000000018003c598 f   libucrt:ungetc.obj
 0001:0003b5f0       _fread_nolock_s            000000018003c5f0 f   libucrt:fread.obj
 0001:0003b880       fread                      000000018003c880 f   libucrt:fread.obj
 0001:0003b8a0       fread_s                    000000018003c8a0 f   libucrt:fread.obj
 0001:0003b948       strerror                   000000018003c948 f   libucrt:strerror.obj
 0001:0003b9f0       __ascii_wcsicmp            000000018003c9f0 f   libucrt:wcsicmp.obj
 0001:0003ba30       _wcsicmp                   000000018003ca30 f   libucrt:wcsicmp.obj
 0001:0003ba78       _wcsicmp_l                 000000018003ca78 f   libucrt:wcsicmp.obj
 0001:0003bba0       iswctype                   000000018003cba0 f   libucrt:iswctype.obj
 0001:0003bc10       wcsncpy                    000000018003cc10 f   libucrt:wcsncpy.obj
 0001:0003bc70       strncmp                    000000018003cc70 f   libucrt:strncmp.obj
 0001:0003bcf0       _ischartype_l              000000018003ccf0 f i libucrt:_ctype.obj
 0001:0003bd68       isdigit                    000000018003cd68 f i libucrt:_ctype.obj
 0001:0003bdd4       isspace                    000000018003cdd4 f i libucrt:_ctype.obj
 0001:0003be50       strncpy                    000000018003ce50 f   libucrt:strncpy.obj
 0001:0003c060       strpbrk                    000000018003d060 f   libucrt:strpbrk.obj
 0001:0003cb4c       _pclose                    000000018003db4c f   libucrt:popen.obj
 0001:0003cc24       _wpopen                    000000018003dc24 f   libucrt:popen.obj
 0001:0003ce48       __acrt_stdio_flush_nolock  000000018003de48 f   libucrt:fflush.obj
 0001:0003cec4       _fflush_nolock             000000018003dec4 f   libucrt:fflush.obj
 0001:0003cf10       _flushall                  000000018003df10 f   libucrt:fflush.obj
 0001:0003cf18       fflush                     000000018003df18 f   libucrt:fflush.obj
 0001:0003cf80       clearerr                   000000018003df80 f   libucrt:clearerr.obj
 0001:0003cf88       clearerr_s                 000000018003df88 f   libucrt:clearerr.obj
 0001:0003d0fc       fgets                      000000018003e0fc f   libucrt:fgets.obj
 0001:0003d4b4       __acrt_stdio_free_tmpfile_name_buffers_nolock 000000018003e4b4 f   libucrt:tmpfile.obj
 0001:0003d53c       tmpfile                    000000018003e53c f   libucrt:tmpfile.obj
 0001:0003d604       _fwrite_nolock             000000018003e604 f   libucrt:fwrite.obj
 0001:0003d7b0       fwrite                     000000018003e7b0 f   libucrt:fwrite.obj
 0001:0003d954       setvbuf                    000000018003e954 f   libucrt:setvbuf.obj
 0001:0003da30       ??$is_overflow_condition@_K@__crt_strtox@@YA_NI_K@Z 000000018003ea30 f i libucrt:input.obj
 0001:0003da60       ??$parse_floating_point@V?$input_adapter_character_source@V?$stream_input_adapter@D@__crt_stdio_input@@@__crt_strtox@@M@__crt_strtox@@YA?AW4SLD_STATUS@@QEAU__crt_locale_pointers@@V?$input_adapter_character_source@V?$stream_input_adapter@D@__crt_stdio_input@@@0@QEAM@Z 000000018003ea60 f i libucrt:input.obj
 0001:0003db08       ??$parse_floating_point@V?$input_adapter_character_source@V?$stream_input_adapter@D@__crt_stdio_input@@@__crt_strtox@@N@__crt_strtox@@YA?AW4SLD_STATUS@@QEAU__crt_locale_pointers@@V?$input_adapter_character_source@V?$stream_input_adapter@D@__crt_stdio_input@@@0@QEAN@Z 000000018003eb08 f i libucrt:input.obj
 0001:0003dbb0       ??$parse_floating_point_from_source@V?$input_adapter_character_source@V?$stream_input_adapter@D@__crt_stdio_input@@@__crt_strtox@@@__crt_strtox@@YA?AW4floating_point_parse_result@0@QEAU__crt_locale_pointers@@AEAV?$input_adapter_character_source@V?$stream_input_adapter@D@__crt_stdio_input@@@0@AEAUfloating_point_string@0@@Z 000000018003ebb0 f i libucrt:input.obj
 0001:0003e418       ??$parse_floating_point_possible_infinity@DV?$input_adapter_character_source@V?$stream_input_adapter@D@__crt_stdio_input@@@__crt_strtox@@_K@__crt_strtox@@YA?AW4floating_point_parse_result@0@AEADAEAV?$input_adapter_character_source@V?$stream_input_adapter@D@__crt_stdio_input@@@0@_K@Z 000000018003f418 f i libucrt:input.obj
 0001:0003e688       ??$parse_floating_point_possible_nan@DV?$input_adapter_character_source@V?$stream_input_adapter@D@__crt_stdio_input@@@__crt_strtox@@_K@__crt_strtox@@YA?AW4floating_point_parse_result@0@AEADAEAV?$input_adapter_character_source@V?$stream_input_adapter@D@__crt_stdio_input@@@0@_K@Z 000000018003f688 f i libucrt:input.obj
 0001:0003e924       ??$parse_floating_point_possible_nan_is_ind@DV?$input_adapter_character_source@V?$stream_input_adapter@D@__crt_stdio_input@@@__crt_strtox@@@__crt_strtox@@YA_NAEADAEAV?$input_adapter_character_source@V?$stream_input_adapter@D@__crt_stdio_input@@@0@@Z 000000018003f924 f i libucrt:input.obj
 0001:0003e9bc       ??$parse_floating_point_possible_nan_is_snan@DV?$input_adapter_character_source@V?$stream_input_adapter@D@__crt_stdio_input@@@__crt_strtox@@@__crt_strtox@@YA_NAEADAEAV?$input_adapter_character_source@V?$stream_input_adapter@D@__crt_stdio_input@@@0@@Z 000000018003f9bc f i libucrt:input.obj
 0001:0003ea54       ??$parse_floating_point_write_result@M@__crt_strtox@@YA?AW4SLD_STATUS@@W4floating_point_parse_result@0@AEBUfloating_point_string@0@QEAM@Z 000000018003fa54 f i libucrt:input.obj
 0001:0003ebc4       ??$parse_floating_point_write_result@N@__crt_strtox@@YA?AW4SLD_STATUS@@W4floating_point_parse_result@0@AEBUfloating_point_string@0@QEAN@Z 000000018003fbc4 f i libucrt:input.obj
 0001:0003eda4       ??$parse_integer@_KV?$input_adapter_character_source@V?$stream_input_adapter@D@__crt_stdio_input@@@__crt_strtox@@@__crt_strtox@@YA_KQEAU__crt_locale_pointers@@V?$input_adapter_character_source@V?$stream_input_adapter@D@__crt_stdio_input@@@0@H_N@Z 000000018003fda4 f i libucrt:input.obj
 0001:0003f210       ??$process_floating_point_specifier_t@M@?$input_processor@DV?$stream_input_adapter@D@__crt_stdio_input@@@__crt_stdio_input@@AEAA_NXZ 0000000180040210 f i libucrt:input.obj
 0001:0003f2b0       ??$process_floating_point_specifier_t@N@?$input_processor@DV?$stream_input_adapter@D@__crt_stdio_input@@@__crt_stdio_input@@AEAA_NXZ 00000001800402b0 f i libucrt:input.obj
 0001:0003f350       ??$process_string_specifier_tchar@D@?$input_processor@DV?$stream_input_adapter@D@__crt_stdio_input@@@__crt_stdio_input@@AEAA_NW4conversion_mode@1@D@Z 0000000180040350 f i libucrt:input.obj
 0001:0003f4ec       ??$process_string_specifier_tchar@_W@?$input_processor@DV?$stream_input_adapter@D@__crt_stdio_input@@@__crt_stdio_input@@AEAA_NW4conversion_mode@1@_W@Z 00000001800404ec f i libucrt:input.obj
 0001:0003f6c0       ??$skip_whitespace@Vstream_input_adapter@__crt_stdio_input@@D@__crt_stdio_input@@YAHAEAV?$stream_input_adapter@D@0@QEAU__crt_locale_pointers@@@Z 00000001800406c0 f i libucrt:input.obj
 0001:0003f87c       ?advance@?$format_string_parser@D@__crt_stdio_input@@QEAA_NXZ 000000018004087c f i libucrt:input.obj
 0001:0003fa44       ?as_double@floating_point_value@__crt_strtox@@QEBAAEANXZ 0000000180040a44 f i libucrt:input.obj
 0001:0003fa80       ?as_float@floating_point_value@__crt_strtox@@QEBAAEAMXZ 0000000180040a80 f i libucrt:input.obj
 0001:0003fabc       ?assemble_floating_point_value@__crt_strtox@@YA?AW4SLD_STATUS@@_KH_N1AEBVfloating_point_value@1@@Z 0000000180040abc f i libucrt:input.obj
 0001:0003fe64       ?assemble_floating_point_value_from_big_integer@__crt_strtox@@YA?AW4SLD_STATUS@@AEBUbig_integer@1@I_N1AEBVfloating_point_value@1@@Z 0000000180040e64 f i libucrt:input.obj
 0001:0003ffc8       ?convert_decimal_string_to_floating_type_common@__crt_strtox@@YA?AW4SLD_STATUS@@AEBUfloating_point_string@1@AEBVfloating_point_value@1@@Z 0000000180040fc8 f i libucrt:input.obj
 0001:00041d4c       ?convert_hexadecimal_string_to_floating_type_common@__crt_strtox@@YA?AW4SLD_STATUS@@AEBUfloating_point_string@1@AEBVfloating_point_value@1@@Z 0000000180042d4c f i libucrt:input.obj
 0001:00041e00       ?divide@__crt_strtox@@YA_KAEAUbig_integer@1@AEBU21@@Z 0000000180042e00 f i libucrt:input.obj
 0001:0004222c       ?length@?$format_string_parser@D@__crt_stdio_input@@QEBA_KXZ 000000018004322c f i libucrt:input.obj
 0001:000422c8       ?process@?$input_processor@DV?$stream_input_adapter@D@__crt_stdio_input@@@__crt_stdio_input@@QEAAHXZ 00000001800432c8 f i libucrt:input.obj
 0001:00042388       ?process_conversion_specifier@?$input_processor@DV?$stream_input_adapter@D@__crt_stdio_input@@@__crt_stdio_input@@AEAA_NXZ 0000000180043388 f i libucrt:input.obj
 0001:000424a4       ?process_floating_point_specifier@?$input_processor@DV?$stream_input_adapter@D@__crt_stdio_input@@@__crt_stdio_input@@AEAA_NXZ 00000001800434a4 f i libucrt:input.obj
 0001:00042508       ?process_integer_specifier@?$input_processor@DV?$stream_input_adapter@D@__crt_stdio_input@@@__crt_stdio_input@@AEAA_NI_N@Z 0000000180043508 f i libucrt:input.obj
 0001:000425b4       ?process_literal_character_tchar@?$input_processor@DV?$stream_input_adapter@D@__crt_stdio_input@@@__crt_stdio_input@@AEAA_ND@Z 00000001800435b4 f i libucrt:input.obj
 0001:00042628       ?process_state@?$input_processor@DV?$stream_input_adapter@D@__crt_stdio_input@@@__crt_stdio_input@@AEAA_NXZ 0000000180043628 f i libucrt:input.obj
 0001:000426e4       ?process_string_specifier@?$input_processor@DV?$stream_input_adapter@D@__crt_stdio_input@@@__crt_stdio_input@@AEAA_NW4conversion_mode@2@@Z 00000001800436e4 f i libucrt:input.obj
 0001:00042764       ?scan_conversion_specifier@?$format_string_parser@D@__crt_stdio_input@@AEAA_NXZ 0000000180043764 f i libucrt:input.obj
 0001:00042908       ?scan_optional_field_width@?$format_string_parser@D@__crt_stdio_input@@AEAA_NXZ 0000000180043908 f i libucrt:input.obj
 0001:000429b0       ?scan_optional_length_modifier@?$format_string_parser@D@__crt_stdio_input@@AEAAXXZ 00000001800439b0 f i libucrt:input.obj
 0001:00042ae8       ?scan_scanset_range@?$format_string_parser@D@__crt_stdio_input@@AEAA_NXZ 0000000180043ae8 f i libucrt:input.obj
 0001:00042c9c       ?write_character@?$input_processor@DV?$stream_input_adapter@D@__crt_stdio_input@@@__crt_stdio_input@@AEAA_NQEFA_W_KAEAPEFA_WAEA_KD@Z 0000000180043c9c f i libucrt:input.obj
 0001:00042d30       ?write_integer@?$input_processor@DV?$stream_input_adapter@D@__crt_stdio_input@@@__crt_stdio_input@@AEAA_N_K@Z 0000000180043d30 f i libucrt:input.obj
 0001:00042da4       __stdio_common_vfscanf     0000000180043da4 f   libucrt:input.obj
 0001:00043388       _ftelli64                  0000000180044388 f   libucrt:ftell.obj
 0001:00043390       _ftelli64_nolock           0000000180044390 f   libucrt:ftell.obj
 0001:000435a0       _fseeki64                  00000001800445a0 f   libucrt:fseek.obj
 0001:00043794       _wdupenv_s                 0000000180044794 f   libucrt:getenv.obj
 0001:000437b4       _wgetenv                   00000001800447b4 f   libucrt:getenv.obj
 0001:000437bc       _wsystem                   00000001800447bc f   libucrt:system.obj
 0001:000438f4       wcscmp                     00000001800448f4 f   libucrt:wcscmp.obj
 0001:0004392c       _initterm                  000000018004492c f   libucrt:initterm.obj
 0001:00043990       _initterm_e                0000000180044990 f   libucrt:initterm.obj
 0001:000439d0       _seh_filter_dll            00000001800449d0 f   libucrt:exception_filter.obj
 0001:000439e4       _seh_filter_exe            00000001800449e4 f   libucrt:exception_filter.obj
 0001:00043dd4       __acrt_initialize_thread_local_exit_callback 0000000180044dd4 f   libucrt:exit.obj
 0001:00043ddc       _cexit                     0000000180044ddc f   libucrt:exit.obj
 0001:00043dec       _exit                      0000000180044dec f   libucrt:exit.obj
 0001:00043df8       _is_c_termination_complete 0000000180044df8 f   libucrt:exit.obj
 0001:00043fc4       __acrt_allocate_buffer_for_argv 0000000180044fc4 f   libucrt:argv_parsing.obj
 0001:00044024       _configure_narrow_argv     0000000180045024 f   libucrt:argv_parsing.obj
 0001:000445cc       __dcrt_get_or_create_wide_environment_nolock 00000001800455cc f   libucrt:environment_initialization.obj
 0001:00044608       __dcrt_uninitialize_environments_nolock 0000000180045608 f   libucrt:environment_initialization.obj
 0001:00044640       _initialize_narrow_environment 0000000180045640 f   libucrt:environment_initialization.obj
 0001:0004479c       _execute_onexit_table      000000018004579c f   libucrt:onexit.obj
 0001:000447d8       _initialize_onexit_table   00000001800457d8 f   libucrt:onexit.obj
 0001:00044838       __acrt_uninitialize_command_line 0000000180045838 f   libucrt:argv_data.obj
 0001:00044930       __acrt_initialize          0000000180045930 f   libucrt:initialization.obj
 0001:00044944       __acrt_thread_attach       0000000180045944 f   libucrt:initialization.obj
 0001:00044958       __acrt_thread_detach       0000000180045958 f   libucrt:initialization.obj
 0001:00044968       __acrt_uninitialize        0000000180045968 f   libucrt:initialization.obj
 0001:000449a0       __acrt_uninitialize_critical 00000001800459a0 f   libucrt:initialization.obj
 0001:000449b0       terminate                  00000001800459b0 f   libucrt:terminate.obj
 0001:00044bd4       strupr                     0000000180045bd4 f   libucrt:strupr.obj
 0001:00044bd4       _strupr                    0000000180045bd4 f   libucrt:strupr.obj
 0001:00044c34       _strupr_s_l                0000000180045c34 f   libucrt:strupr.obj
 0001:00044c80       __ascii_stricmp            0000000180045c80 f   libucrt:stricmp.obj
 0001:00044cbc       _stricmp                   0000000180045cbc f   libucrt:stricmp.obj
 0001:00044cbc       stricmp                    0000000180045cbc f   libucrt:stricmp.obj
 0001:00044d04       _stricmp_l                 0000000180045d04 f   libucrt:stricmp.obj
 0001:00044d8c       strcpy_s                   0000000180045d8c f   libucrt:strcpy_s.obj
 0001:00044dec       abort                      0000000180045dec f   libucrt:abort.obj
 0001:00044e44       ??$parse_integer@KV?$c_string_character_source@D@__crt_strtox@@@__crt_strtox@@YAKQEAU__crt_locale_pointers@@V?$c_string_character_source@D@0@H_N@Z 0000000180045e44 f i libucrt:atox.obj
 0001:0004514c       ??$parse_integer@KV?$c_string_character_source@_W@__crt_strtox@@@__crt_strtox@@YAKQEAU__crt_locale_pointers@@V?$c_string_character_source@_W@0@H_N@Z 000000018004614c f i libucrt:atox.obj
 0001:000457f4       ??$parse_integer@_KV?$c_string_character_source@D@__crt_strtox@@@__crt_strtox@@YA_KQEAU__crt_locale_pointers@@V?$c_string_character_source@D@0@H_N@Z 00000001800467f4 f i libucrt:atox.obj
 0001:00045ae4       calloc                     0000000180046ae4 f   libucrt:calloc.obj
 0001:00045aec       wcsncmp                    0000000180046aec f   libucrt:wcsncmp.obj
 0001:00045b18       __acrt_call_reportfault    0000000180046b18 f   libucrt:invalid_parameter.obj
 0001:00045c74       __acrt_initialize_invalid_parameter_handler 0000000180046c74 f   libucrt:invalid_parameter.obj
 0001:00045c7c       _invalid_parameter         0000000180046c7c f   libucrt:invalid_parameter.obj
 0001:00045d2c       _invalid_parameter_noinfo  0000000180046d2c f   libucrt:invalid_parameter.obj
 0001:00045d4c       _invoke_watson             0000000180046d4c f   libucrt:invalid_parameter.obj
 0001:00045d94       _free_base                 0000000180046d94 f   libucrt:free_base.obj
 0001:00045dd4       _malloc_base               0000000180046dd4 f   libucrt:malloc_base.obj
 0001:00045e34       strtol                     0000000180046e34 f   libucrt:strtox.obj
 0001:00045e60       strtoull                   0000000180046e60 f   libucrt:strtox.obj
 0001:00045e8c       wcstol                     0000000180046e8c f   libucrt:strtox.obj
 0001:00045eb8       _mbtowc_l                  0000000180046eb8 f   libucrt:mbtowc.obj
 0001:00046038       mbtowc                     0000000180047038 f   libucrt:mbtowc.obj
 0001:00046040       _wctomb_s_l                0000000180047040 f   libucrt:wctomb.obj
 0001:000461dc       wctomb_s                   00000001800471dc f   libucrt:wctomb.obj
 0001:000461f0       strnlen                    00000001800471f0 f   libucrt:strnlen.obj
 0001:00046340       wcsnlen                    0000000180047340 f   libucrt:strnlen.obj
 0001:00046890       __acrt_freeptd             0000000180047890 f   libucrt:per_thread_data.obj
 0001:000468d4       __acrt_getptd              00000001800478d4 f   libucrt:per_thread_data.obj
 0001:000469a8       __acrt_getptd_head         00000001800479a8 f   libucrt:per_thread_data.obj
 0001:00046a50       __acrt_getptd_noexit       0000000180047a50 f   libucrt:per_thread_data.obj
 0001:00046b1c       __acrt_initialize_ptd      0000000180047b1c f   libucrt:per_thread_data.obj
 0001:00046b58       __acrt_uninitialize_ptd    0000000180047b58 f   libucrt:per_thread_data.obj
 0001:00046b7c       __acrt_update_locale_info  0000000180047b7c f   libucrt:locale_update.obj
 0001:00046bb0       __acrt_update_multibyte_info 0000000180047bb0 f   libucrt:locale_update.obj
 0001:0004747c       __acrt_fp_format           000000018004847c f   libucrt:cvt.obj
 0001:00047780       _fileno                    0000000180048780 f   libucrt:fileno.obj
 0001:000477a8       _fputc_nolock              00000001800487a8 f   libucrt:fputc.obj
 0001:000477c0       _get_printf_count_output   00000001800487c0 f   libucrt:printf_count_output.obj
 0001:000477d8       __acrt_stdio_begin_temporary_buffering_nolock 00000001800487d8 f   libucrt:_sftbuf.obj
 0001:000478a8       __acrt_stdio_end_temporary_buffering_nolock 00000001800488a8 f   libucrt:_sftbuf.obj
 0001:00047954       __acrt_set_locale_changed  0000000180048954 f   libucrt:wsetlocale.obj
 0001:00047960       __acrt_uninitialize_locale 0000000180048960 f   libucrt:wsetlocale.obj
 0001:00047b8c       __acrt_initialize_lowio    0000000180048b8c f   libucrt:ioinit.obj
 0001:00047bc8       __acrt_uninitialize_lowio  0000000180048bc8 f   libucrt:ioinit.obj
 0001:00047c7c       _close                     0000000180048c7c f   libucrt:close.obj
 0001:00047d20       _close_nolock              0000000180048d20 f   libucrt:close.obj
 0001:00047de0       ?__acrt_stdio_allocate_stream@@YA?AV__crt_stdio_stream@@XZ 0000000180048de0 f   libucrt:stream.obj
 0001:00047e38       ?__acrt_stdio_free_stream@@YAXV__crt_stdio_stream@@@Z 0000000180048e38 f   libucrt:stream.obj
 0001:00047f40       __acrt_stdio_free_buffer_nolock 0000000180048f40 f   libucrt:_freebuf.obj
 0001:00047f80       wcscpy_s                   0000000180048f80 f   libucrt:wcscpy_s.obj
 0001:00048000       _get_fpsr                  0000000180049000 f   libucrt:fpsr.obj
 0001:00048010       _set_fpsr                  0000000180049010 f   libucrt:fpsr.obj
 0001:0004801a       _fclrf                     000000018004901a f   libucrt:fpsr.obj
 0001:0004802e       _frnd                      000000018004902e f   libucrt:fpsr.obj
 0001:00048050       ??$__acrt_stdio_parse_mode@_W@@YA?AU__acrt_stdio_stream_mode@@QEB_W@Z 0000000180049050 f i libucrt:openfile.obj
 0001:00048350       _wopenfile                 0000000180049350 f   libucrt:openfile.obj
 0001:000483ec       _calloc_base               00000001800493ec f   libucrt:calloc_base.obj
 0001:0004863c       __acrt_AppPolicyGetProcessTerminationMethodInternal 000000018004963c f   libucrt:winapi_thunks.obj
 0001:0004868c       __acrt_AreFileApisANSI     000000018004968c f   libucrt:winapi_thunks.obj
 0001:000486c8       __acrt_CompareStringEx     00000001800496c8 f   libucrt:winapi_thunks.obj
 0001:000487a4       __acrt_FlsAlloc            00000001800497a4 f   libucrt:winapi_thunks.obj
 0001:000487ec       __acrt_FlsFree             00000001800497ec f   libucrt:winapi_thunks.obj
 0001:00048834       __acrt_FlsGetValue         0000000180049834 f   libucrt:winapi_thunks.obj
 0001:0004887c       __acrt_FlsSetValue         000000018004987c f   libucrt:winapi_thunks.obj
 0001:000488d0       __acrt_InitializeCriticalSectionEx 00000001800498d0 f   libucrt:winapi_thunks.obj
 0001:00048934       __acrt_LCMapStringEx       0000000180049934 f   libucrt:winapi_thunks.obj
 0001:00048a10       __acrt_LocaleNameToLCID    0000000180049a10 f   libucrt:winapi_thunks.obj
 0001:00048a60       __acrt_initialize_winapi_thunks 0000000180049a60 f   libucrt:winapi_thunks.obj
 0001:00048a94       __acrt_uninitialize_winapi_thunks 0000000180049a94 f   libucrt:winapi_thunks.obj
 0001:00048ad8       _fcloseall                 0000000180049ad8 f   libucrt:closeall.obj
 0001:00048b8c       __acrt_stdio_refill_and_read_narrow_nolock 0000000180049b8c f   libucrt:_filbuf.obj
 0001:00049064       _lseek                     000000018004a064 f   libucrt:lseek.obj
 0001:0004906c       _lseeki64                  000000018004a06c f   libucrt:lseek.obj
 0001:00049074       _lseeki64_nolock           000000018004a074 f   libucrt:lseek.obj
 0001:0004907c       __acrt_stdio_allocate_buffer_nolock 000000018004a07c f   libucrt:_getbuf.obj
 0001:000496bc       _read                      000000018004a6bc f   libucrt:read.obj
 0001:000497d8       _read_nolock               000000018004a7d8 f   libucrt:read.obj
 0001:00049c30       __sys_errlist              000000018004ac30 f   libucrt:syserr.obj
 0001:00049c38       __sys_nerr                 000000018004ac38 f   libucrt:syserr.obj
 0001:00049c40       strncpy_s                  000000018004ac40 f   libucrt:strncpy_s.obj
 0001:00049d14       _towlower_l                000000018004ad14 f   libucrt:towlower.obj
 0001:00049dd0       __pctype_func              000000018004add0 f   libucrt:ctype.obj
 0001:00049e00       __acrt_GetStringTypeW      000000018004ae00 f   libucrt:getstringtypew.obj
 0001:00049e08       _isctype_l                 000000018004ae08 f   libucrt:isctype.obj
 0001:00049f10       _recalloc_base             000000018004af10 f   libucrt:recalloc.obj
 0001:00049fa8       wcscat_s                   000000018004afa8 f   libucrt:wcscat_s.obj
 0001:0004a028       _cwait                     000000018004b028 f   libucrt:wait.obj
 0001:0004a0e0       __acrt_wgetpath            000000018004b0e0 f   libucrt:getpath.obj
 0001:0004a1d4       ??$__acrt_mbs_to_wcs_cp@U__crt_win32_buffer_internal_dynamic_resizing@@@@YAHQEBDAEAV?$__crt_win32_buffer@_WU__crt_win32_buffer_internal_dynamic_resizing@@@@I@Z 000000018004b1d4 f i libucrt:createprocessa.obj
 0001:0004a34c       __acrt_initialize_locks    000000018004b34c f   libucrt:locks.obj
 0001:0004a394       __acrt_lock                000000018004b394 f   libucrt:locks.obj
 0001:0004a3b0       __acrt_uninitialize_locks  000000018004b3b0 f   libucrt:locks.obj
 0001:0004a3e8       __acrt_unlock              000000018004b3e8 f   libucrt:locks.obj
 0001:0004a404       _waccess_s                 000000018004b404 f   libucrt:waccess.obj
 0001:0004a4b0       _pipe                      000000018004b4b0 f   libucrt:pipe.obj
 0001:0004a840       _wfdopen                   000000018004b840 f   libucrt:fdopen.obj
 0001:0004a8d4       _commit                    000000018004b8d4 f   libucrt:commit.obj
 0001:0004b1c8       _write                     000000018004c1c8 f   libucrt:write.obj
 0001:0004b2b4       _write_nolock              000000018004c2b4 f   libucrt:write.obj
 0001:0004b6c4       _ui64toa_s                 000000018004c6c4 f   libucrt:xtoa.obj
 0001:0004b6d8       _strdup                    000000018004c6d8 f   libucrt:strdup.obj
 0001:0004b750       __acrt_GetTempPathA        000000018004c750 f   libucrt:gettemppath.obj
 0001:0004bee4       _sopen_nolock              000000018004cee4 f   libucrt:open.obj
 0001:0004bffc       _sopen_s                   000000018004cffc f   libucrt:open.obj
 0001:0004c030       _wsopen_nolock             000000018004d030 f   libucrt:open.obj
 0001:0004c418       _wsopen_s                  000000018004d418 f   libucrt:open.obj
 0001:0004c44c       __acrt_uninitialize_tmpfile 000000018004d44c f   libucrt:rmtmp.obj
 0001:0004c460       _rmtmp                     000000018004d460 f   libucrt:rmtmp.obj
 0001:0004c654       __acrt_stdio_flush_and_write_narrow_nolock 000000018004d654 f   libucrt:_flsbuf.obj
 0001:0004c740       fegetround                 000000018004d740 f   libucrt:fegetround.obj
 0001:0004c754       _wcsnicoll                 000000018004d754 f   libucrt:wcsnicol.obj
 0001:0004c7a4       _wcsnicoll_l               000000018004d7a4 f   libucrt:wcsnicol.obj
 0001:0004cfd8       _wspawnve                  000000018004dfd8 f   libucrt:spawnv.obj
 0001:0004d308       _wspawnvpe                 000000018004e308 f   libucrt:spawnvp.obj
 0001:0004d310       __acrt_get_process_end_policy 000000018004e310 f   libucrt:win_policies.obj
 0001:0004d360       ??$__acrt_wcs_to_mbs_cp@U__crt_win32_buffer_internal_dynamic_resizing@@@@YAHQEB_WAEAV?$__crt_win32_buffer@DU__crt_win32_buffer_internal_dynamic_resizing@@@@I@Z 000000018004e360 f i libucrt:argv_wildcards.obj
 0001:0004db90       __acrt_expand_narrow_argv_wildcards 000000018004eb90 f   libucrt:argv_wildcards.obj
 0001:0004db98       ??$__acrt_wcs_to_mbs_cp@U__crt_win32_buffer_no_resizing@@@@YAHQEB_WAEAV?$__crt_win32_buffer@DU__crt_win32_buffer_no_resizing@@@@I@Z 000000018004eb98 f i libucrt:getmodulefilenamea.obj
 0001:0004dcac       __acrt_GetModuleFileNameA  000000018004ecac f   libucrt:getmodulefilenamea.obj
 0001:0004e4f8       __acrt_initialize_multibyte 000000018004f4f8 f   libucrt:mbctype.obj
 0001:0004e558       __acrt_update_thread_multibyte_data 000000018004f558 f   libucrt:mbctype.obj
 0001:0004e574       _setmbcp_nolock            000000018004f574 f   libucrt:mbctype.obj
 0001:0004e8a8       _ismbblead                 000000018004f8a8 f   libucrt:ismbbyte.obj
 0001:0004e8bc       __acrt_initialize_command_line 000000018004f8bc f   libucrt:argv_data.obj
 0001:0004e8e4       __acrt_MultiByteToWideChar 000000018004f8e4 f   libucrt:multibytetowidechar.obj
 0001:0004e940       __acrt_WideCharToMultiByte 000000018004f940 f   libucrt:widechartomultibyte.obj
 0001:0004e9d8       __dcrt_get_narrow_environment_from_os 000000018004f9d8 f   libucrt:get_environment_from_os.obj
 0001:0004eadc       __dcrt_get_wide_environment_from_os 000000018004fadc f   libucrt:get_environment_from_os.obj
 0001:0004ef90       __dcrt_set_variable_in_wide_environment_nolock 000000018004ff90 f   libucrt:setenv.obj
 0001:0004ef98       __acrt_initialize_heap     000000018004ff98 f   libucrt:heap_handle.obj
 0001:0004efb4       __acrt_uninitialize_heap   000000018004ffb4 f   libucrt:heap_handle.obj
 0001:0004efc0       __acrt_execute_initializers 000000018004ffc0 f   libucrt:shared_initialization.obj
 0001:0004f040       __acrt_execute_uninitializers 0000000180050040 f   libucrt:shared_initialization.obj
 0001:0004f07c       __acrt_initialize_new_handler 000000018005007c f   libucrt:new_handler.obj
 0001:0004f084       _callnewh                  0000000180050084 f   libucrt:new_handler.obj
 0001:0004f0b4       _query_new_handler         00000001800500b4 f   libucrt:new_handler.obj
 0001:0004f130       __acrt_get_sigabrt_handler 0000000180050130 f   libucrt:signal.obj
 0001:0004f160       __acrt_initialize_signal_handlers 0000000180050160 f   libucrt:signal.obj
 0001:0004f180       raise                      0000000180050180 f   libucrt:signal.obj
 0001:0004f3ec       __acrt_has_user_matherr    00000001800503ec f   libucrt:matherr.obj
 0001:0004f40c       __acrt_initialize_user_matherr 000000018005040c f   libucrt:matherr.obj
 0001:0004f414       __acrt_invoke_user_matherr 0000000180050414 f   libucrt:matherr.obj
 0001:0004f75c       __acrt_LCMapStringA        000000018005075c f   libucrt:lcmapstringa.obj
 0001:0004f7f4       _query_new_mode            00000001800507f4 f   libucrt:new_mode.obj
 0001:0004f7fc       _isleadbyte_l              00000001800507fc f i libucrt:_wctype.obj
 0001:0004f848       ?__mbrtowc_utf8@__crt_mbstring@@YA_KPEA_WPEBD_KPEAU_Mbstatet@@@Z 0000000180050848 f   libucrt:mbrtowc.obj
 0001:0004f884       ?__mbsrtowcs_utf8@__crt_mbstring@@YA_KPEA_WPEAPEBD_KPEAU_Mbstatet@@@Z 0000000180050884 f   libucrt:mbrtowc.obj
 0001:0004f9fc       ?__c32rtomb_utf8@__crt_mbstring@@YA_KPEAD_UPEAU_Mbstatet@@@Z 00000001800509fc f   libucrt:c32rtomb.obj
 0001:0004fab0       __acrt_add_locale_ref      0000000180050ab0 f   libucrt:locale_refcounting.obj
 0001:0004fb3c       __acrt_free_locale         0000000180050b3c f   libucrt:locale_refcounting.obj
 0001:0004fcb4       __acrt_locale_add_lc_time_reference 0000000180050cb4 f   libucrt:locale_refcounting.obj
 0001:0004fcdc       __acrt_locale_free_lc_time_if_unreferenced 0000000180050cdc f   libucrt:locale_refcounting.obj
 0001:0004fd14       __acrt_locale_release_lc_time_reference 0000000180050d14 f   libucrt:locale_refcounting.obj
 0001:0004fd3c       __acrt_release_locale_ref  0000000180050d3c f   libucrt:locale_refcounting.obj
 0001:0004fde4       __acrt_update_thread_locale_data 0000000180050de4 f   libucrt:locale_refcounting.obj
 0001:0004fe50       _updatetlocinfoEx_nolock   0000000180050e50 f   libucrt:locale_refcounting.obj
 0001:0004feb8       __acrt_fp_strflt_to_string 0000000180050eb8 f   libucrt:_fptostr.obj
 0001:0004ff9c       __acrt_fltout              0000000180050f9c f   libucrt:cfout.obj
 0001:000511d0       _isatty                    00000001800521d0 f   libucrt:isatty.obj
 0001:00051230       __acrt_locale_free_monetary 0000000180052230 f   libucrt:initmon.obj
 0001:0005133c       __acrt_locale_free_numeric 000000018005233c f   libucrt:initnum.obj
 0001:00051400       __acrt_locale_free_time    0000000180052400 f   libucrt:inittime.obj
 0001:00051508       __acrt_GetStringTypeA      0000000180052508 f   libucrt:getstringtypea.obj
 0001:00051698       __acrt_lowio_create_handle_array 0000000180052698 f   libucrt:osfinfo.obj
 0001:00051740       __acrt_lowio_destroy_handle_array 0000000180052740 f   libucrt:osfinfo.obj
 0001:00051790       __acrt_lowio_ensure_fh_exists 0000000180052790 f   libucrt:osfinfo.obj
 0001:00051838       __acrt_lowio_lock_fh       0000000180052838 f   libucrt:osfinfo.obj
 0001:00051860       __acrt_lowio_set_os_handle 0000000180052860 f   libucrt:osfinfo.obj
 0001:00051920       __acrt_lowio_unlock_fh     0000000180052920 f   libucrt:osfinfo.obj
 0001:00051948       _alloc_osfhnd              0000000180052948 f   libucrt:osfinfo.obj
 0001:00051a88       _free_osfhnd               0000000180052a88 f   libucrt:osfinfo.obj
 0001:00051b44       _get_osfhandle             0000000180052b44 f   libucrt:osfinfo.obj
 0001:00051bbc       __ascii_wcsnicmp           0000000180052bbc f   libucrt:wcsnicmp.obj
 0001:00051c08       _wcsnicmp                  0000000180052c08 f   libucrt:wcsnicmp.obj
 0001:00051c50       _wcsnicmp_l                0000000180052c50 f   libucrt:wcsnicmp.obj
 0001:00051da0       __acrt_DownlevelLocaleNameToLCID 0000000180052da0 f   libucrt:lcidtoname_downlevel.obj
 0001:00051e50       __acrt_LCMapStringW        0000000180052e50 f   libucrt:lcmapstringw.obj
 0001:00051ed8       _msize_base                0000000180052ed8 f   libucrt:msize.obj
 0001:00051f14       _realloc_base              0000000180052f14 f   libucrt:realloc_base.obj
 0001:00051f90       _get_fmode                 0000000180052f90 f   libucrt:setmode.obj
 0001:00051fc0       _setmode_nolock            0000000180052fc0 f   libucrt:setmode.obj
 0001:000520a0       _putwch_nolock             00000001800530a0 f   libucrt:putwch.obj
 0001:000520dc       _chsize_nolock             00000001800530dc f   libucrt:chsize.obj
 0001:00052248       __acrt_fenv_get_common_round_control 0000000180053248 f   libucrt:_fenvutils.obj
 0001:00052254       __acrt_fenv_get_control    0000000180053254 f   libucrt:_fenvutils.obj
 0001:00052348       __acrt_fenv_get_status     0000000180053348 f   libucrt:_fenvutils.obj
 0001:0005239c       __acrt_fenv_set_control    000000018005339c f   libucrt:_fenvutils.obj
 0001:000524e4       __acrt_fenv_set_status     00000001800534e4 f   libucrt:_fenvutils.obj
 0001:00052568       __acrt_CompareStringW      0000000180053568 f   libucrt:comparestringw.obj
 0001:00052948       __acrt_pack_wide_command_line_and_environment 0000000180053948 f   libucrt:cenvarg.obj
 0001:00052ad0       qsort                      0000000180053ad0 f   libucrt:qsort.obj
 0001:00052e80       _mbsdec                    0000000180053e80 f   libucrt:mbsdec.obj
 0001:00052e88       _mbsdec_l                  0000000180053e88 f   libucrt:mbsdec.obj
 0001:00052f34       __strncnt                  0000000180053f34 f   libucrt:strncnt.obj
 0001:00052f4c       ?__mbrtoc32_utf8@__crt_mbstring@@YA_KPEA_UPEBD_KPEAU_Mbstatet@@@Z 0000000180053f4c f   libucrt:mbrtoc32.obj
 0001:00053128       fegetenv                   0000000180054128 f   libucrt:fegetenv.obj
 0001:00053148       fesetenv                   0000000180054148 f   libucrt:fesetenv.obj
 0001:00053194       feholdexcept               0000000180054194 f   libucrt:feholdexcept.obj
 0001:000531e4       ceil                       00000001800541e4 f   libucrt:ceil.obj
 0001:000532b0       log10                      00000001800542b0 f   libucrt:log10.obj
 0001:0005385c       _query_app_type            000000018005485c f   libucrt:report_runtime_error.obj
 0001:00053864       __dcrt_lowio_ensure_console_output_initialized 0000000180054864 f   libucrt:initcon.obj
 0001:000538b8       __dcrt_terminate_console_output 00000001800548b8 f   libucrt:initcon.obj
 0001:000538d4       __dcrt_write_console       00000001800548d4 f   libucrt:initcon.obj
 0001:00053ab8       _handle_error              0000000180054ab8 f   libucrt:libm_error.obj
 0001:00053be0       _handle_nan                0000000180054be0 f   libucrt:libm_error.obj
 0001:00053c00       __acrt_initialize_fma3     0000000180054c00 f   libucrt:fma3_available.obj
 0001:00053c70       _log10_special             0000000180054c70 f   libucrt:log_special.obj
 0001:00053d28       _raise_exc                 0000000180054d28 f   libucrt:fpexcept.obj
 0001:00053d50       _raise_exc_ex              0000000180054d50 f   libucrt:fpexcept.obj
 0001:00054060       _set_errno_from_matherr    0000000180055060 f   libucrt:fpexcept.obj
 0001:00054090       _clrfp                     0000000180055090 f   libucrt:fpctrl.obj
 0001:000540b0       _ctrlfp                    00000001800550b0 f   libucrt:fpctrl.obj
 0001:0005412c       _set_statfp                000000018005512c f   libucrt:fpctrl.obj
 0001:0005414c       _statfp                    000000018005514c f   libucrt:fpctrl.obj
 0001:00054160       _FindPESection             0000000180055160 f   LIBCMT:pesect.obj
 0001:000541b0       _IsNonwritableInCurrentImage 00000001800551b0 f   LIBCMT:pesect.obj
 0001:00054200       _ValidateImageBase         0000000180055200 f   LIBCMT:pesect.obj
 0001:00054230       __GSHandlerCheck           0000000180055230 f   LIBCMT:gshandler.obj
 0001:00054250       __GSHandlerCheckCommon     0000000180055250 f   LIBCMT:gshandler.obj
 0001:000542ac       __GSHandlerCheck_SEH       00000001800552ac f   LIBCMT:gshandlerseh.obj
 0001:00054350       __chkstk                   0000000180055350 f   LIBCMT:chkstk.obj
 0001:00054350       _alloca_probe              0000000180055350 f   LIBCMT:chkstk.obj
 0001:000543a0       _local_unwind              00000001800553a0 f   libvcruntime:jmpuwind.obj
 0001:000543e0       memcmp                     00000001800553e0 f   libvcruntime:memcmp.obj
 0001:000544c0       memchr                     00000001800554c0 f   libvcruntime:memchr.obj
 0001:00054540       strcmp                     0000000180055540 f   libucrt:strcmp.obj
 0001:000545c0       _guard_dispatch_icall_nop  00000001800555c0 f   LIBCMT:guard_dispatch.obj
 0001:000545e0       _guard_xfg_dispatch_icall_nop 00000001800555e0 f   LIBCMT:guard_xfg_dispatch.obj
 0002:00000000       __imp_RegDeleteKeyW        0000000180056000     advapi32:ADVAPI32.dll
 0002:00000008       __imp_RegEnumKeyExW        0000000180056008     advapi32:ADVAPI32.dll
 0002:00000010       __imp_RegDeleteValueW      0000000180056010     advapi32:ADVAPI32.dll
 0002:00000018       __imp_RegEnumValueW        0000000180056018     advapi32:ADVAPI32.dll
 0002:00000020       __imp_RegCloseKey          0000000180056020     advapi32:ADVAPI32.dll
 0002:00000028       __imp_RegCreateKeyExW      0000000180056028     advapi32:ADVAPI32.dll
 0002:00000030       __imp_RegSetValueExW       0000000180056030     advapi32:ADVAPI32.dll
 0002:00000038       __imp_RegOpenKeyExW        0000000180056038     advapi32:ADVAPI32.dll
 0002:00000040       __imp_RegQueryValueExW     0000000180056040     advapi32:ADVAPI32.dll
 0002:00000048       \177ADVAPI32_NULL_THUNK_DATA 0000000180056048     advapi32:ADVAPI32.dll
 0002:00000050       __imp_DeleteTimerQueueTimer 0000000180056050     kernel32:KERNEL32.dll
 0002:00000058       __imp_CreateTimerQueue     0000000180056058     kernel32:KERNEL32.dll
 0002:00000060       __imp_GetModuleFileNameW   0000000180056060     kernel32:KERNEL32.dll
 0002:00000068       __imp_LoadLibraryW         0000000180056068     kernel32:KERNEL32.dll
 0002:00000070       __imp_FreeLibrary          0000000180056070     kernel32:KERNEL32.dll
 0002:00000078       __imp_GetCPInfoExW         0000000180056078     kernel32:KERNEL32.dll
 0002:00000080       __imp_GetOEMCP             0000000180056080     kernel32:KERNEL32.dll
 0002:00000088       __imp_SearchPathW          0000000180056088     kernel32:KERNEL32.dll
 0002:00000090       __imp_GetConsoleOutputCP   0000000180056090     kernel32:KERNEL32.dll
 0002:00000098       __imp_SetConsoleMode       0000000180056098     kernel32:KERNEL32.dll
 0002:000000a0       __imp_GetConsoleCP         00000001800560a0     kernel32:KERNEL32.dll
 0002:000000a8       __imp_EnumSystemCodePagesW 00000001800560a8     kernel32:KERNEL32.dll
 0002:000000b0       __imp_GetACP               00000001800560b0     kernel32:KERNEL32.dll
 0002:000000b8       __imp_SetFileAttributesW   00000001800560b8     kernel32:KERNEL32.dll
 0002:000000c0       __imp_GetLogicalDriveStringsW 00000001800560c0     kernel32:KERNEL32.dll
 0002:000000c8       __imp_MultiByteToWideChar  00000001800560c8     kernel32:KERNEL32.dll
 0002:000000d0       __imp_Sleep                00000001800560d0     kernel32:KERNEL32.dll
 0002:000000d8       __imp_GetConsoleMode       00000001800560d8     kernel32:KERNEL32.dll
 0002:000000e0       __imp_FormatMessageW       00000001800560e0     kernel32:KERNEL32.dll
 0002:000000e8       __imp_GetLastError         00000001800560e8     kernel32:KERNEL32.dll
 0002:000000f0       __imp_OutputDebugStringW   00000001800560f0     kernel32:KERNEL32.dll
 0002:000000f8       __imp_GetCurrentDirectoryW 00000001800560f8     kernel32:KERNEL32.dll
 0002:00000100       __imp_SetCurrentDirectoryW 0000000180056100     kernel32:KERNEL32.dll
 0002:00000108       __imp_SetConsoleCP         0000000180056108     kernel32:KERNEL32.dll
 0002:00000110       __imp_GlobalMemoryStatusEx 0000000180056110     kernel32:KERNEL32.dll
 0002:00000118       __imp_GetModuleHandleW     0000000180056118     kernel32:KERNEL32.dll
 0002:00000120       __imp_SetConsoleOutputCP   0000000180056120     kernel32:KERNEL32.dll
 0002:00000128       __imp_GetDriveTypeW        0000000180056128     kernel32:KERNEL32.dll
 0002:00000130       __imp_CreateDirectoryW     0000000180056130     kernel32:KERNEL32.dll
 0002:00000138       __imp_FindFirstFileW       0000000180056138     kernel32:KERNEL32.dll
 0002:00000140       __imp_CompareStringW       0000000180056140     kernel32:KERNEL32.dll
 0002:00000148       __imp_RemoveDirectoryW     0000000180056148     kernel32:KERNEL32.dll
 0002:00000150       __imp_SetFileTime          0000000180056150     kernel32:KERNEL32.dll
 0002:00000158       __imp_SetEnvironmentVariableW 0000000180056158     kernel32:KERNEL32.dll
 0002:00000160       __imp_FindClose            0000000180056160     kernel32:KERNEL32.dll
 0002:00000168       __imp_CreateFileW          0000000180056168     kernel32:KERNEL32.dll
 0002:00000170       __imp_ReadConsoleInputW    0000000180056170     kernel32:KERNEL32.dll
 0002:00000178       __imp_FileTimeToSystemTime 0000000180056178     kernel32:KERNEL32.dll
 0002:00000180       __imp_DeleteFileW          0000000180056180     kernel32:KERNEL32.dll
 0002:00000188       __imp_CloseHandle          0000000180056188     kernel32:KERNEL32.dll
 0002:00000190       __imp_FileTimeToLocalFileTime 0000000180056190     kernel32:KERNEL32.dll
 0002:00000198       __imp_PeekConsoleInputW    0000000180056198     kernel32:KERNEL32.dll
 0002:000001a0       __imp_WriteConsoleW        00000001800561a0     kernel32:KERNEL32.dll
 0002:000001a8       __imp_MoveFileExW          00000001800561a8     kernel32:KERNEL32.dll
 0002:000001b0       __imp_VerSetConditionMask  00000001800561b0     kernel32:KERNEL32.dll
 0002:000001b8       __imp_SystemTimeToFileTime 00000001800561b8     kernel32:KERNEL32.dll
 0002:000001c0       __imp_CopyFileW            00000001800561c0     kernel32:KERNEL32.dll
 0002:000001c8       __imp_VerifyVersionInfoW   00000001800561c8     kernel32:KERNEL32.dll
 0002:000001d0       __imp_GetSystemTimeAsFileTime 00000001800561d0     kernel32:KERNEL32.dll
 0002:000001d8       __imp_GetFileTime          00000001800561d8     kernel32:KERNEL32.dll
 0002:000001e0       __imp_SetEndOfFile         00000001800561e0     kernel32:KERNEL32.dll
 0002:000001e8       __imp_GetProcAddress       00000001800561e8     kernel32:KERNEL32.dll
 0002:000001f0       __imp_ChangeTimerQueueTimer 00000001800561f0     kernel32:KERNEL32.dll
 0002:000001f8       __imp_GetModuleHandleA     00000001800561f8     kernel32:KERNEL32.dll
 0002:00000200       __imp_GetFileAttributesW   0000000180056200     kernel32:KERNEL32.dll
 0002:00000208       __imp_GetEnvironmentVariableW 0000000180056208     kernel32:KERNEL32.dll
 0002:00000210       __imp_GetStdHandle         0000000180056210     kernel32:KERNEL32.dll
 0002:00000218       __imp_GetConsoleScreenBufferInfo 0000000180056218     kernel32:KERNEL32.dll
 0002:00000220       __imp_CreateTimerQueueTimer 0000000180056220     kernel32:KERNEL32.dll
 0002:00000228       __imp_WideCharToMultiByte  0000000180056228     kernel32:KERNEL32.dll
 0002:00000230       __imp_DeleteTimerQueueEx   0000000180056230     kernel32:KERNEL32.dll
 0002:00000238       __imp_HeapReAlloc          0000000180056238     kernel32:KERNEL32.dll
 0002:00000240       __imp_HeapSize             0000000180056240     kernel32:KERNEL32.dll
 0002:00000248       __imp_SetStdHandle         0000000180056248     kernel32:KERNEL32.dll
 0002:00000250       __imp_GetProcessHeap       0000000180056250     kernel32:KERNEL32.dll
 0002:00000258       __imp_FreeEnvironmentStringsW 0000000180056258     kernel32:KERNEL32.dll
 0002:00000260       __imp_GetEnvironmentStringsW 0000000180056260     kernel32:KERNEL32.dll
 0002:00000268       __imp_GetCommandLineW      0000000180056268     kernel32:KERNEL32.dll
 0002:00000270       __imp_GetCommandLineA      0000000180056270     kernel32:KERNEL32.dll
 0002:00000278       __imp_GetCPInfo            0000000180056278     kernel32:KERNEL32.dll
 0002:00000280       __imp_IsValidCodePage      0000000180056280     kernel32:KERNEL32.dll
 0002:00000288       __imp_FindNextFileW        0000000180056288     kernel32:KERNEL32.dll
 0002:00000290       __imp_FindFirstFileExW     0000000180056290     kernel32:KERNEL32.dll
 0002:00000298       __imp_GetFileSizeEx        0000000180056298     kernel32:KERNEL32.dll
 0002:000002a0       __imp_WriteFile            00000001800562a0     kernel32:KERNEL32.dll
 0002:000002a8       __imp_FlushFileBuffers     00000001800562a8     kernel32:KERNEL32.dll
 0002:000002b0       __imp_CreatePipe           00000001800562b0     kernel32:KERNEL32.dll
 0002:000002b8       __imp_GetFileAttributesExW 00000001800562b8     kernel32:KERNEL32.dll
 0002:000002c0       __imp_GetExitCodeProcess   00000001800562c0     kernel32:KERNEL32.dll
 0002:000002c8       __imp_WaitForSingleObject  00000001800562c8     kernel32:KERNEL32.dll
 0002:000002d0       __imp_GetStringTypeW       00000001800562d0     kernel32:KERNEL32.dll
 0002:000002d8       __imp_ReadConsoleW         00000001800562d8     kernel32:KERNEL32.dll
 0002:000002e0       __imp_SetFilePointerEx     00000001800562e0     kernel32:KERNEL32.dll
 0002:000002e8       __imp_LCMapStringW         00000001800562e8     kernel32:KERNEL32.dll
 0002:000002f0       __imp_GetFileType          00000001800562f0     kernel32:KERNEL32.dll
 0002:000002f8       __imp_HeapAlloc            00000001800562f8     kernel32:KERNEL32.dll
 0002:00000300       __imp_HeapFree             0000000180056300     kernel32:KERNEL32.dll
 0002:00000308       __imp_GetModuleHandleExW   0000000180056308     kernel32:KERNEL32.dll
 0002:00000310       __imp_ExitProcess          0000000180056310     kernel32:KERNEL32.dll
 0002:00000318       __imp_ReadFile             0000000180056318     kernel32:KERNEL32.dll
 0002:00000320       __imp_GetTempPathW         0000000180056320     kernel32:KERNEL32.dll
 0002:00000328       __imp_CreateProcessW       0000000180056328     kernel32:KERNEL32.dll
 0002:00000330       __imp_DuplicateHandle      0000000180056330     kernel32:KERNEL32.dll
 0002:00000338       __imp_RaiseException       0000000180056338     kernel32:KERNEL32.dll
 0002:00000340       __imp_LoadLibraryExW       0000000180056340     kernel32:KERNEL32.dll
 0002:00000348       __imp_TlsFree              0000000180056348     kernel32:KERNEL32.dll
 0002:00000350       __imp_TlsSetValue          0000000180056350     kernel32:KERNEL32.dll
 0002:00000358       __imp_TlsGetValue          0000000180056358     kernel32:KERNEL32.dll
 0002:00000360       __imp_TlsAlloc             0000000180056360     kernel32:KERNEL32.dll
 0002:00000368       __imp_InitializeCriticalSectionAndSpinCount 0000000180056368     kernel32:KERNEL32.dll
 0002:00000370       __imp_DeleteCriticalSection 0000000180056370     kernel32:KERNEL32.dll
 0002:00000378       __imp_RtlUnwind            0000000180056378     kernel32:KERNEL32.dll
 0002:00000380       __imp_LeaveCriticalSection 0000000180056380     kernel32:KERNEL32.dll
 0002:00000388       __imp_EnterCriticalSection 0000000180056388     kernel32:KERNEL32.dll
 0002:00000390       __imp_SetLastError         0000000180056390     kernel32:KERNEL32.dll
 0002:00000398       __imp_InterlockedFlushSList 0000000180056398     kernel32:KERNEL32.dll
 0002:000003a0       __imp_RtlUnwindEx          00000001800563a0     kernel32:KERNEL32.dll
 0002:000003a8       __imp_GetStartupInfoW      00000001800563a8     kernel32:KERNEL32.dll
 0002:000003b0       __imp_IsDebuggerPresent    00000001800563b0     kernel32:KERNEL32.dll
 0002:000003b8       __imp_InitializeSListHead  00000001800563b8     kernel32:KERNEL32.dll
 0002:000003c0       __imp_GetCurrentThreadId   00000001800563c0     kernel32:KERNEL32.dll
 0002:000003c8       __imp_GetCurrentProcessId  00000001800563c8     kernel32:KERNEL32.dll
 0002:000003d0       __imp_QueryPerformanceCounter 00000001800563d0     kernel32:KERNEL32.dll
 0002:000003d8       __imp_IsProcessorFeaturePresent 00000001800563d8     kernel32:KERNEL32.dll
 0002:000003e0       __imp_TerminateProcess     00000001800563e0     kernel32:KERNEL32.dll
 0002:000003e8       __imp_GetCurrentProcess    00000001800563e8     kernel32:KERNEL32.dll
 0002:000003f0       __imp_SetUnhandledExceptionFilter 00000001800563f0     kernel32:KERNEL32.dll
 0002:000003f8       __imp_UnhandledExceptionFilter 00000001800563f8     kernel32:KERNEL32.dll
 0002:00000400       __imp_RtlVirtualUnwind     0000000180056400     kernel32:KERNEL32.dll
 0002:00000408       __imp_RtlLookupFunctionEntry 0000000180056408     kernel32:KERNEL32.dll
 0002:00000410       __imp_RtlCaptureContext    0000000180056410     kernel32:KERNEL32.dll
 0002:00000418       \177KERNEL32_NULL_THUNK_DATA 0000000180056418     kernel32:KERNEL32.dll
 0002:00000420       __imp_UuidCreate           0000000180056420     rpcrt4:RPCRT4.dll
 0002:00000428       __imp_UuidToStringA        0000000180056428     rpcrt4:RPCRT4.dll
 0002:00000430       __imp_RpcStringFreeA       0000000180056430     rpcrt4:RPCRT4.dll
 0002:00000438       __imp_UuidFromStringA      0000000180056438     rpcrt4:RPCRT4.dll
 0002:00000440       \177RPCRT4_NULL_THUNK_DATA 0000000180056440     rpcrt4:RPCRT4.dll
 0002:00000448       __imp_SHGetFolderPathW     0000000180056448     shell32:SHELL32.dll
 0002:00000450       __imp_ShellExecuteW        0000000180056450     shell32:SHELL32.dll
 0002:00000458       \177SHELL32_NULL_THUNK_DATA 0000000180056458     shell32:SHELL32.dll
 0002:00000460       __imp_GetKeyState          0000000180056460     user32:USER32.dll
 0002:00000468       \177USER32_NULL_THUNK_DATA 0000000180056468     user32:USER32.dll
 0002:00000470       __imp_luaL_optnumber       0000000180056470     lua51:lua51.dll
 0002:00000478       __imp_luaopen_string       0000000180056478     lua51:lua51.dll
 0002:00000480       __imp_luaopen_math         0000000180056480     lua51:lua51.dll
 0002:00000488       __imp_luaL_checknumber     0000000180056488     lua51:lua51.dll
 0002:00000490       __imp_luaL_typerror        0000000180056490     lua51:lua51.dll
 0002:00000498       __imp_lua_setfenv          0000000180056498     lua51:lua51.dll
 0002:000004a0       __imp_luaopen_debug        00000001800564a0     lua51:lua51.dll
 0002:000004a8       __imp_lua_setallocf        00000001800564a8     lua51:lua51.dll
 0002:000004b0       __imp_lua_dump             00000001800564b0     lua51:lua51.dll
 0002:000004b8       __imp_luaL_prepbuffer      00000001800564b8     lua51:lua51.dll
 0002:000004c0       __imp_luaL_checkstack      00000001800564c0     lua51:lua51.dll
 0002:000004c8       __imp_lua_typename         00000001800564c8     lua51:lua51.dll
 0002:000004d0       __imp_lua_tocfunction      00000001800564d0     lua51:lua51.dll
 0002:000004d8       __imp_luaL_checkoption     00000001800564d8     lua51:lua51.dll
 0002:000004e0       __imp_lua_iscfunction      00000001800564e0     lua51:lua51.dll
 0002:000004e8       __imp_luaL_gsub            00000001800564e8     lua51:lua51.dll
 0002:000004f0       __imp_lua_isuserdata       00000001800564f0     lua51:lua51.dll
 0002:000004f8       __imp_luaopen_os           00000001800564f8     lua51:lua51.dll
 0002:00000500       __imp_lua_getinfo          0000000180056500     lua51:lua51.dll
 0002:00000508       __imp_luaL_optlstring      0000000180056508     lua51:lua51.dll
 0002:00000510       __imp_lua_checkstack       0000000180056510     lua51:lua51.dll
 0002:00000518       __imp_luaL_optinteger      0000000180056518     lua51:lua51.dll
 0002:00000520       __imp_luaL_checkudata      0000000180056520     lua51:lua51.dll
 0002:00000528       __imp_luaL_addvalue        0000000180056528     lua51:lua51.dll
 0002:00000530       __imp_luaL_error           0000000180056530     lua51:lua51.dll
 0002:00000538       __imp_luaL_checklstring    0000000180056538     lua51:lua51.dll
 0002:00000540       __imp_luaL_buffinit        0000000180056540     lua51:lua51.dll
 0002:00000548       __imp_luaL_addlstring      0000000180056548     lua51:lua51.dll
 0002:00000550       __imp_lua_load             0000000180056550     lua51:lua51.dll
 0002:00000558       __imp_lua_error            0000000180056558     lua51:lua51.dll
 0002:00000560       __imp_lua_pushfstring      0000000180056560     lua51:lua51.dll
 0002:00000568       __imp_lua_concat           0000000180056568     lua51:lua51.dll
 0002:00000570       __imp_luaL_pushresult      0000000180056570     lua51:lua51.dll
 0002:00000578       __imp_luaL_loadstring      0000000180056578     lua51:lua51.dll
 0002:00000580       __imp_lua_insert           0000000180056580     lua51:lua51.dll
 0002:00000588       __imp_lua_rawseti          0000000180056588     lua51:lua51.dll
 0002:00000590       __imp_lua_toboolean        0000000180056590     lua51:lua51.dll
 0002:00000598       __imp_lua_pcall            0000000180056598     lua51:lua51.dll
 0002:000005a0       __imp_lua_next             00000001800565a0     lua51:lua51.dll
 0002:000005a8       __imp_lua_rawget           00000001800565a8     lua51:lua51.dll
 0002:000005b0       __imp_luaL_unref           00000001800565b0     lua51:lua51.dll
 0002:000005b8       __imp_lua_remove           00000001800565b8     lua51:lua51.dll
 0002:000005c0       __imp_lua_rawgeti          00000001800565c0     lua51:lua51.dll
 0002:000005c8       __imp_lua_objlen           00000001800565c8     lua51:lua51.dll
 0002:000005d0       __imp_lua_topointer        00000001800565d0     lua51:lua51.dll
 0002:000005d8       __imp_lua_isstring         00000001800565d8     lua51:lua51.dll
 0002:000005e0       __imp_lua_tointeger        00000001800565e0     lua51:lua51.dll
 0002:000005e8       __imp_lua_createtable      00000001800565e8     lua51:lua51.dll
 0002:000005f0       __imp_luaL_ref             00000001800565f0     lua51:lua51.dll
 0002:000005f8       __imp_lua_gettable         00000001800565f8     lua51:lua51.dll
 0002:00000600       __imp_lua_pushlightuserdata 0000000180056600     lua51:lua51.dll
 0002:00000608       __imp_lua_pushlstring      0000000180056608     lua51:lua51.dll
 0002:00000610       __imp_lua_isnumber         0000000180056610     lua51:lua51.dll
 0002:00000618       __imp_lua_pushinteger      0000000180056618     lua51:lua51.dll
 0002:00000620       __imp_lua_pushnil          0000000180056620     lua51:lua51.dll
 0002:00000628       __imp_lua_replace          0000000180056628     lua51:lua51.dll
 0002:00000630       __imp_luaL_argerror        0000000180056630     lua51:lua51.dll
 0002:00000638       __imp_lua_pushvalue        0000000180056638     lua51:lua51.dll
 0002:00000640       __imp_luaL_newmetatable    0000000180056640     lua51:lua51.dll
 0002:00000648       __imp_lua_settop           0000000180056648     lua51:lua51.dll
 0002:00000650       __imp_lua_setmetatable     0000000180056650     lua51:lua51.dll
 0002:00000658       __imp_luaL_register        0000000180056658     lua51:lua51.dll
 0002:00000660       __imp_lua_getfield         0000000180056660     lua51:lua51.dll
 0002:00000668       __imp_lua_gettop           0000000180056668     lua51:lua51.dll
 0002:00000670       __imp_lua_pushnumber       0000000180056670     lua51:lua51.dll
 0002:00000678       __imp_lua_pushstring       0000000180056678     lua51:lua51.dll
 0002:00000680       __imp_lua_touserdata       0000000180056680     lua51:lua51.dll
 0002:00000688       __imp_lua_call             0000000180056688     lua51:lua51.dll
 0002:00000690       __imp_lua_tolstring        0000000180056690     lua51:lua51.dll
 0002:00000698       __imp_lua_pushboolean      0000000180056698     lua51:lua51.dll
 0002:000006a0       __imp_lua_tonumber         00000001800566a0     lua51:lua51.dll
 0002:000006a8       __imp_lua_newuserdata      00000001800566a8     lua51:lua51.dll
 0002:000006b0       __imp_luaL_checkinteger    00000001800566b0     lua51:lua51.dll
 0002:000006b8       __imp_lua_setfield         00000001800566b8     lua51:lua51.dll
 0002:000006c0       __imp_lua_type             00000001800566c0     lua51:lua51.dll
 0002:000006c8       __imp_lua_rawequal         00000001800566c8     lua51:lua51.dll
 0002:000006d0       __imp_lua_getmetatable     00000001800566d0     lua51:lua51.dll
 0002:000006d8       __imp_lua_pushcclosure     00000001800566d8     lua51:lua51.dll
 0002:000006e0       __imp_luaopen_base         00000001800566e0     lua51:lua51.dll
 0002:000006e8       __imp_lua_getfenv          00000001800566e8     lua51:lua51.dll
 0002:000006f0       __imp_lua_settable         00000001800566f0     lua51:lua51.dll
 0002:000006f8       __imp_luaL_checkany        00000001800566f8     lua51:lua51.dll
 0002:00000700       __imp_lua_getallocf        0000000180056700     lua51:lua51.dll
 0002:00000708       __imp_luaL_findtable       0000000180056708     lua51:lua51.dll
 0002:00000710       __imp_luaopen_table        0000000180056710     lua51:lua51.dll
 0002:00000718       __imp_luaL_checktype       0000000180056718     lua51:lua51.dll
 0002:00000720       __imp_lua_rawset           0000000180056720     lua51:lua51.dll
 0002:00000728       __imp_lua_getstack         0000000180056728     lua51:lua51.dll
 0002:00000730       __imp_lua_gc               0000000180056730     lua51:lua51.dll
 0002:00000738       \177lua51_NULL_THUNK_DATA  0000000180056738     lua51:lua51.dll
 0002:00000740       __guard_check_icall_fptr   0000000180056740     LIBCMT:guard_support.obj
 0002:00000748       __guard_xfg_check_icall_fptr 0000000180056748     LIBCMT:guard_support.obj
 0002:00000750       __guard_dispatch_icall_fptr 0000000180056750     LIBCMT:guard_support.obj
 0002:00000758       __guard_xfg_dispatch_icall_fptr 0000000180056758     LIBCMT:guard_support.obj
 0002:00000760       __guard_xfg_table_dispatch_icall_fptr 0000000180056760     LIBCMT:guard_support.obj
 0002:00000768       __xc_a                     0000000180056768     LIBCMT:initializers.obj
 0002:00000770       __xc_z                     0000000180056770     LIBCMT:initializers.obj
 0002:00000778       __xi_a                     0000000180056778     LIBCMT:initializers.obj
 0002:00000780       __acrt_stdio_initializer   0000000180056780     libucrt:stdio_initializer.obj
 0002:00000788       __acrt_multibyte_initializer 0000000180056788     libucrt:multibyte_initializer.obj
 0002:00000790       __acrt_tran_fma3_initializer 0000000180056790     libucrt:fma3_initializer.obj
 0002:00000798       __xi_z                     0000000180056798     LIBCMT:initializers.obj
 0002:000007a0       __xp_a                     00000001800567a0     LIBCMT:initializers.obj
 0002:000007a8       __acrt_locale_terminator   00000001800567a8     libucrt:locale_initializer.obj
 0002:000007b0       __acrt_tmpfile_terminator  00000001800567b0     libucrt:tmpfile_initializer.obj
 0002:000007b8       __dcrt_console_output_terminator 00000001800567b8     libucrt:console_output_initializer.obj
 0002:000007c0       __acrt_stdio_terminator    00000001800567c0     libucrt:stdio_initializer.obj
 0002:000007c8       __xp_z                     00000001800567c8     LIBCMT:initializers.obj
 0002:000007d0       __xt_a                     00000001800567d0     LIBCMT:initializers.obj
 0002:000007d8       __xt_z                     00000001800567d8     LIBCMT:initializers.obj
 0002:000007f0       _pRawDllMain               00000001800567f0     LIBCMT:dll_dllmain.obj
 0002:000007f0       _pDefaultRawDllMain        00000001800567f0     LIBCMT:dll_dllmain.obj
 0002:000007f8       _pDestructExceptionObject  00000001800567f8     libvcruntime:ehhelpers.obj
 0002:00000f00       ??_C@_08EHJDFFNH@__based?$CI@ 0000000180056f00     libvcruntime:undname.obj
 0002:00000f10       ??_C@_07KOLFKCDI@__cdecl@  0000000180056f10     libvcruntime:undname.obj
 0002:00000f18       ??_C@_08GHMPAG@__pascal@   0000000180056f18     libvcruntime:undname.obj
 0002:00000f28       ??_C@_09IFJBGAPI@__stdcall@ 0000000180056f28     libvcruntime:undname.obj
 0002:00000f38       ??_C@_0L@NPHFGOKO@__thiscall@ 0000000180056f38     libvcruntime:undname.obj
 0002:00000f48       ??_C@_0L@JMKHOMEK@__fastcall@ 0000000180056f48     libvcruntime:undname.obj
 0002:00000f58       ??_C@_0N@BCKKPABJ@__vectorcall@ 0000000180056f58     libvcruntime:undname.obj
 0002:00000f68       ??_C@_09HIJEGCPM@__clrcall@ 0000000180056f68     libvcruntime:undname.obj
 0002:00000f74       ??_C@_06GHPCKEAG@__eabi@   0000000180056f74     libvcruntime:undname.obj
 0002:00000f80       ??_C@_09IOPIDJLG@__swift_1@ 0000000180056f80     libvcruntime:undname.obj
 0002:00000f90       ??_C@_09KFNFGKHF@__swift_2@ 0000000180056f90     libvcruntime:undname.obj
 0002:00000fa0       ??_C@_07JOMMBBKO@__ptr64@  0000000180056fa0     libvcruntime:undname.obj
 0002:00000fa8       ??_C@_0L@PILCLIHE@__restrict@ 0000000180056fa8     libvcruntime:undname.obj
 0002:00000fb8       ??_C@_0M@GFIIJFMG@__unaligned@ 0000000180056fb8     libvcruntime:undname.obj
 0002:00000fc8       ??_C@_09DHDLOLLB@restrict?$CI@ 0000000180056fc8     libvcruntime:undname.obj
 0002:00000fd4       ??_C@_04NIHEBCM@?5new@     0000000180056fd4     libvcruntime:undname.obj
 0002:00000fe0       ??_C@_07FPCDHGMM@?5delete@ 0000000180056fe0     libvcruntime:undname.obj
 0002:00000fe8       ??_C@_01NEMOKFLO@?$DN@     0000000180056fe8     libvcruntime:undname.obj
 0002:00000fec       ??_C@_02GPIOPFAK@?$DO?$DO@ 0000000180056fec     libvcruntime:undname.obj
 0002:00000ff0       ??_C@_02FODMEDOG@?$DM?$DM@ 0000000180056ff0     libvcruntime:undname.obj
 0002:00000ff4       ??_C@_01DCLJPIOD@?$CB@     0000000180056ff4     libvcruntime:undname.obj
 0002:00000ff8       ??_C@_02EGOFBIJA@?$DN?$DN@ 0000000180056ff8     libvcruntime:undname.obj
 0002:00000ffc       ??_C@_02FDNJECIE@?$CB?$DN@ 0000000180056ffc     libvcruntime:undname.obj
 0002:00001000       ??_C@_02GPECMEKF@?$FL?$FN@ 0000000180057000     libvcruntime:undname.obj
 0002:00001008       ??_C@_08LHJFAFGD@operator@ 0000000180057008     libvcruntime:undname.obj
 0002:00001014       ??_C@_02HBOOOICD@?9?$DO@   0000000180057014     libvcruntime:undname.obj
 0002:00001018       ??_C@_01NBENCBCI@?$CK@     0000000180057018     libvcruntime:undname.obj
 0002:0000101c       ??_C@_02ECNGHCIF@?$CL?$CL@ 000000018005701c     libvcruntime:undname.obj
 0002:00001020       ??_C@_02BAABKJLB@?9?9@     0000000180057020     libvcruntime:undname.obj
 0002:00001024       ??_C@_01JOAMLHOP@?9@       0000000180057024     libvcruntime:undname.obj
 0002:00001028       ??_C@_01MIFGBAGJ@?$CL@     0000000180057028     libvcruntime:undname.obj
 0002:0000102c       ??_C@_01HNPIGOCE@?$CG@     000000018005702c     libvcruntime:undname.obj
 0002:00001030       ??_C@_03MNHNFDLC@?9?$DO?$CK@ 0000000180057030     libvcruntime:undname.obj
 0002:00001034       ??_C@_01FGNFDNOH@?$CF@     0000000180057034     libvcruntime:undname.obj
 0002:00001038       ??_C@_01MNNFJEPP@?$DM@     0000000180057038     libvcruntime:undname.obj
 0002:0000103c       ??_C@_02EHCHHCKH@?$DM?$DN@ 000000018005703c     libvcruntime:undname.obj
 0002:00001040       ??_C@_01PPODPGHN@?$DO@     0000000180057040     libvcruntime:undname.obj
 0002:00001044       ??_C@_02EEKDKGMJ@?$DO?$DN@ 0000000180057044     libvcruntime:undname.obj
 0002:00001048       ??_C@_01IHBHIGKO@?0@       0000000180057048     libvcruntime:undname.obj
 0002:0000104c       ??_C@_02HCKGKOFO@?$CI?$CJ@ 000000018005704c     libvcruntime:undname.obj
 0002:00001050       ??_C@_01PJKLJHI@?$HO@      0000000180057050     libvcruntime:undname.obj
 0002:00001054       ??_C@_01JKBOJNNK@?$FO@     0000000180057054     libvcruntime:undname.obj
 0002:00001058       ??_C@_01DNKMNLPK@?$HM@     0000000180057058     libvcruntime:undname.obj
 0002:0000105c       ??_C@_02PPKAJPJL@?$CG?$CG@ 000000018005705c     libvcruntime:undname.obj
 0002:00001060       ??_C@_02NONPIBCD@?$HM?$HM@ 0000000180057060     libvcruntime:undname.obj
 0002:00001064       ??_C@_02FPIMKNGF@?$CK?$DN@ 0000000180057064     libvcruntime:undname.obj
 0002:00001068       ??_C@_02FOEOMHFC@?$CL?$DN@ 0000000180057068     libvcruntime:undname.obj
 0002:0000106c       ??_C@_02FKMDLLOA@?9?$DN@   000000018005706c     libvcruntime:undname.obj
 0002:00001070       ??_C@_02FJEHGPIO@?1?$DN@   0000000180057070     libvcruntime:undname.obj
 0002:00001074       ??_C@_02FENAOKFI@?$CF?$DN@ 0000000180057074     libvcruntime:undname.obj
 0002:00001078       ??_C@_03IKFCCPFF@?$DO?$DO?$DN@ 0000000180057078     libvcruntime:undname.obj
 0002:0000107c       ??_C@_03CDNPDDLA@?$DM?$DM?$DN@ 000000018005707c     libvcruntime:undname.obj
 0002:00001080       ??_C@_02FGJGFEAB@?$CG?$DN@ 0000000180057080     libvcruntime:undname.obj
 0002:00001084       ??_C@_02DHLNPPGH@?$HM?$DN@ 0000000180057084     libvcruntime:undname.obj
 0002:00001088       ??_C@_02MHEGNOJ@?$FO?$DN@  0000000180057088     libvcruntime:undname.obj
 0002:00001090       ??_C@_09IFPLHPGF@?$GAvftable?8@ 0000000180057090     libvcruntime:undname.obj
 0002:000010a0       ??_C@_09BLBHBJP@?$GAvbtable?8@ 00000001800570a0     libvcruntime:undname.obj
 0002:000010b0       ??_C@_07FEEIOKP@?$GAvcall?8@ 00000001800570b0     libvcruntime:undname.obj
 0002:000010b8       ??_C@_08LLFFHHDJ@?$GAtypeof?8@ 00000001800570b8     libvcruntime:undname.obj
 0002:000010c8       ??_C@_0BF@KDPPACIK@?$GAlocal?5static?5guard?8@ 00000001800570c8     libvcruntime:undname.obj
 0002:000010e0       ??_C@_08OBABFOLI@?$GAstring?8@ 00000001800570e0     libvcruntime:undname.obj
 0002:000010f0       ??_C@_0BD@JDLKDPAB@?$GAvbase?5destructor?8@ 00000001800570f0     libvcruntime:undname.obj
 0002:00001108       ??_C@_0BN@DEGPLNFK@?$GAvector?5deleting?5destructor?8@ 0000000180057108     libvcruntime:undname.obj
 0002:00001128       ??_C@_0BO@OBMKPJIG@?$GAdefault?5constructor?5closure?8@ 0000000180057128     libvcruntime:undname.obj
 0002:00001148       ??_C@_0BN@IMDCHIKM@?$GAscalar?5deleting?5destructor?8@ 0000000180057148     libvcruntime:undname.obj
 0002:00001168       ??_C@_0BO@PFGOCPJJ@?$GAvector?5constructor?5iterator?8@ 0000000180057168     libvcruntime:undname.obj
 0002:00001188       ??_C@_0BN@LFPFMEDL@?$GAvector?5destructor?5iterator?8@ 0000000180057188     libvcruntime:undname.obj
 0002:000011a8       ??_C@_0CE@IKBNEHA@?$GAvector?5vbase?5constructor?5itera@ 00000001800571a8     libvcruntime:undname.obj
 0002:000011d0       ??_C@_0BL@NILFHHPC@?$GAvirtual?5displacement?5map?8@ 00000001800571d0     libvcruntime:undname.obj
 0002:000011f0       ??_C@_0CB@JONCMFFK@?$GAeh?5vector?5constructor?5iterator@ 00000001800571f0     libvcruntime:undname.obj
 0002:00001218       ??_C@_0CA@GCEOPDGL@?$GAeh?5vector?5destructor?5iterator?8@ 0000000180057218     libvcruntime:undname.obj
 0002:00001238       ??_C@_0CH@OOJPLCPH@?$GAeh?5vector?5vbase?5constructor?5it@ 0000000180057238     libvcruntime:undname.obj
 0002:00001260       ??_C@_0BL@LLKPOHJI@?$GAcopy?5constructor?5closure?8@ 0000000180057260     libvcruntime:undname.obj
 0002:00001280       ??_C@_0BA@KBCDOMBN@?$GAudt?5returning?8@ 0000000180057280     libvcruntime:undname.obj
 0002:00001290       ??_C@_03KLGMFNMG@?$GAEH@   0000000180057290     libvcruntime:undname.obj
 0002:00001294       ??_C@_05KHLCHHI@?$GARTTI@  0000000180057294     libvcruntime:undname.obj
 0002:000012a0       ??_C@_0BA@KKLDJDLB@?$GAlocal?5vftable?8@ 00000001800572a0     libvcruntime:undname.obj
 0002:000012b0       ??_C@_0CE@IIHCMGGL@?$GAlocal?5vftable?5constructor?5clos@ 00000001800572b0     libvcruntime:undname.obj
 0002:000012d4       ??_C@_06FHBGPFGH@?5new?$FL?$FN@ 00000001800572d4     libvcruntime:undname.obj
 0002:000012e0       ??_C@_09LBNFPBCA@?5delete?$FL?$FN@ 00000001800572e0     libvcruntime:undname.obj
 0002:000012f0       ??_C@_0P@HJKNJFNN@?$GAomni?5callsig?8@ 00000001800572f0     libvcruntime:undname.obj
 0002:00001300       ??_C@_0BL@CNOONJFP@?$GAplacement?5delete?5closure?8@ 0000000180057300     libvcruntime:undname.obj
 0002:00001320       ??_C@_0BN@CKNJLHMB@?$GAplacement?5delete?$FL?$FN?5closure?8@ 0000000180057320     libvcruntime:undname.obj
 0002:00001340       ??_C@_0CG@CFDHKGGD@?$GAmanaged?5vector?5constructor?5ite@ 0000000180057340     libvcruntime:undname.obj
 0002:00001368       ??_C@_0CF@IMGKMJNO@?$GAmanaged?5vector?5destructor?5iter@ 0000000180057368     libvcruntime:undname.obj
 0002:00001390       ??_C@_0CG@HLDDJMAG@?$GAeh?5vector?5copy?5constructor?5ite@ 0000000180057390     libvcruntime:undname.obj
 0002:000013b8       ??_C@_0CM@FCBBDIGB@?$GAeh?5vector?5vbase?5copy?5construct@ 00000001800573b8     libvcruntime:undname.obj
 0002:000013e8       ??_C@_0BL@CLIPGLGB@?$GAdynamic?5initializer?5for?5?8@ 00000001800573e8     libvcruntime:undname.obj
 0002:00001408       ??_C@_0CB@PDBIFEP@?$GAdynamic?5atexit?5destructor?5for?5@ 0000000180057408     libvcruntime:undname.obj
 0002:00001430       ??_C@_0CD@CGAJBKEJ@?$GAvector?5copy?5constructor?5iterat@ 0000000180057430     libvcruntime:undname.obj
 0002:00001458       ??_C@_0CJ@GJELGAMM@?$GAvector?5vbase?5copy?5constructor?5@ 0000000180057458     libvcruntime:undname.obj
 0002:00001488       ??_C@_0CL@FGIJHLCE@?$GAmanaged?5vector?5copy?5constructo@ 0000000180057488     libvcruntime:undname.obj
 0002:000014b8       ??_C@_0BM@PMGGMLDN@?$GAlocal?5static?5thread?5guard?8@ 00000001800574b8     libvcruntime:undname.obj
 0002:000014d8       ??_C@_0N@BDNMDMOL@operator?5?$CC?$CC?5@ 00000001800574d8     libvcruntime:undname.obj
 0002:000014e8       ??_C@_0BC@GGEBGALA@operator?5co_await@ 00000001800574e8     libvcruntime:undname.obj
 0002:00001500       ??_C@_0M@GAAIMMOH@operator?$DM?$DN?$DO@ 0000000180057500     libvcruntime:undname.obj
 0002:00001510       ??_C@_0BC@DAFEJGAK@?5Type?5Descriptor?8@ 0000000180057510     libvcruntime:undname.obj
 0002:00001528       ??_C@_0BM@LDKODKLH@?5Base?5Class?5Descriptor?5at?5?$CI@ 0000000180057528     libvcruntime:undname.obj
 0002:00001548       ??_C@_0BD@LGICGFMM@?5Base?5Class?5Array?8@ 0000000180057548     libvcruntime:undname.obj
 0002:00001560       ??_C@_0BN@MECKDCOJ@?5Class?5Hierarchy?5Descriptor?8@ 0000000180057560     libvcruntime:undname.obj
 0002:00001580       ??_C@_0BK@CFCOFLF@?5Complete?5Object?5Locator?8@ 0000000180057580     libvcruntime:undname.obj
 0002:000015a0       ??_C@_0BG@JNJLAMPM@?$GAanonymous?5namespace?8@ 00000001800575a0     libvcruntime:undname.obj
 0002:000015d0       ??_C@_1DM@KHCHBNEB@?$AAa?$AAp?$AAi?$AA?9?$AAm?$AAs?$AA?9?$AAw?$AAi?$AAn?$AA?9?$AAc?$AAo?$AAr?$AAe@ 00000001800575d0     libvcruntime:winapi_downlevel.obj
 0002:00001610       ??_C@_1DK@LPPGFMPP@?$AAa?$AAp?$AAi?$AA?9?$AAm?$AAs?$AA?9?$AAw?$AAi?$AAn?$AA?9?$AAc?$AAo?$AAr?$AAe@ 0000000180057610     libvcruntime:winapi_downlevel.obj
 0002:00001650       ??_C@_1BC@GDMECMAK@?$AAk?$AAe?$AAr?$AAn?$AAe?$AAl?$AA3?$AA2@ 0000000180057650     libvcruntime:winapi_downlevel.obj
 0002:00001668       ??_C@_1BA@PFFKHIOG@?$AAa?$AAp?$AAi?$AA?9?$AAm?$AAs?$AA?9@ 0000000180057668     libvcruntime:winapi_downlevel.obj
 0002:00001680       ??_C@_08KNHFBNJ@FlsAlloc@  0000000180057680     libvcruntime:winapi_downlevel.obj
 0002:00001698       ??_C@_07PEJMOBNF@FlsFree@  0000000180057698     libvcruntime:winapi_downlevel.obj
 0002:000016a8       ??_C@_0M@GDNOONDI@FlsGetValue@ 00000001800576a8     libvcruntime:winapi_downlevel.obj
 0002:000016c0       ??_C@_0M@JCPCPOEF@FlsSetValue@ 00000001800576c0     libvcruntime:winapi_downlevel.obj
 0002:000016d8       ??_C@_0BM@HCFOFFN@InitializeCriticalSectionEx@ 00000001800576d8     libvcruntime:winapi_downlevel.obj
 0002:00001700       standard_lookup_table      0000000180057700     libucrt:output.obj
 0002:00001760       ??_C@_1O@CEDCILHN@?$AA?$CI?$AAn?$AAu?$AAl?$AAl?$AA?$CJ@ 0000000180057760     libucrt:output.obj
 0002:00001770       ??_C@_06OJHGLDPL@?$CInull?$CJ@ 0000000180057770     libucrt:output.obj
 0002:000018f0       ??_C@_0EA@FCLIIPNN@Visual?5C?$CL?$CL?5CRT?3?5Not?5enough?5memo@ 00000001800578f0     libucrt:strerror.obj
 0002:00001980       ?large_power_data@?1??multiply_by_power_of_ten@__crt_strtox@@YA_NAEAUbig_integer@2@I@Z@4QBIB 0000000180057980     libucrt:input.obj
 0002:00002328       ?small_powers_of_ten@?1??multiply_by_power_of_ten@__crt_strtox@@YA_NAEAUbig_integer@2@I@Z@4QBIB 0000000180058328     libucrt:input.obj
 0002:00002350       ??_C@_1GE@DPGDJKLM@?$AAm?$AAi?$AAn?$AAk?$AAe?$AAr?$AAn?$AAe?$AAl?$AA?2?$AAc?$AAr?$AAt?$AAs?$AA?2@ 0000000180058350     libucrt:input.obj
 0002:000023c0       ??_C@_1FM@FELNCOBF@?$AA_?$AA_?$AAc?$AAr?$AAt?$AA_?$AAs?$AAt?$AAr?$AAt?$AAo?$AAx?$AA?3?$AA?3?$AAf@ 00000001800583c0     libucrt:input.obj
 0002:00002420       ??_C@_1BG@GEMHBGAF@?$AA_?$AAi?$AAs?$AA_?$AAd?$AAo?$AAu?$AAb?$AAl?$AAe@ 0000000180058420     libucrt:input.obj
 0002:00002440       ??_C@_1FK@JOJELFFO@?$AA_?$AA_?$AAc?$AAr?$AAt?$AA_?$AAs?$AAt?$AAr?$AAt?$AAo?$AAx?$AA?3?$AA?3?$AAf@ 0000000180058440     libucrt:input.obj
 0002:000024a0       ??_C@_1BI@BANMPGJI@?$AA?$CB?$AA_?$AAi?$AAs?$AA_?$AAd?$AAo?$AAu?$AAb?$AAl?$AAe@ 00000001800584a0     libucrt:input.obj
 0002:000024c0       ?constraints@?1??is_length_valid@__crt_stdio_input@@YA_NW4conversion_mode@2@W4length_modifier@2@@Z@4QAY0M@$$CBEA 00000001800584c0     libucrt:input.obj
 0002:00002538       ?inf_uppercase@?1???$parse_floating_point_possible_infinity@DV?$input_adapter_character_source@V?$stream_input_adapter@D@__crt_stdio_input@@@__crt_strtox@@_K@__crt_strtox@@YA?AW4floating_point_parse_result@1@AEADAEAV?$input_adapter_character_source@V?$stream_input_adapter@D@__crt_stdio_input@@@1@_K@Z@4QBDB 0000000180058538     libucrt:input.obj
 0002:0000253c       ?inf_lowercase@?1???$parse_floating_point_possible_infinity@DV?$input_adapter_character_source@V?$stream_input_adapter@D@__crt_stdio_input@@@__crt_strtox@@_K@__crt_strtox@@YA?AW4floating_point_parse_result@1@AEADAEAV?$input_adapter_character_source@V?$stream_input_adapter@D@__crt_stdio_input@@@1@_K@Z@4QBDB 000000018005853c     libucrt:input.obj
 0002:00002540       ?inity_uppercase@?1???$parse_floating_point_possible_infinity@DV?$input_adapter_character_source@V?$stream_input_adapter@D@__crt_stdio_input@@@__crt_strtox@@_K@__crt_strtox@@YA?AW4floating_point_parse_result@1@AEADAEAV?$input_adapter_character_source@V?$stream_input_adapter@D@__crt_stdio_input@@@1@_K@Z@4QBDB 0000000180058540     libucrt:input.obj
 0002:00002548       ?inity_lowercase@?1???$parse_floating_point_possible_infinity@DV?$input_adapter_character_source@V?$stream_input_adapter@D@__crt_stdio_input@@@__crt_strtox@@_K@__crt_strtox@@YA?AW4floating_point_parse_result@1@AEADAEAV?$input_adapter_character_source@V?$stream_input_adapter@D@__crt_stdio_input@@@1@_K@Z@4QBDB 0000000180058548     libucrt:input.obj
 0002:00002550       ?uppercase@?1???$parse_floating_point_possible_nan@DV?$input_adapter_character_source@V?$stream_input_adapter@D@__crt_stdio_input@@@__crt_strtox@@_K@__crt_strtox@@YA?AW4floating_point_parse_result@1@AEADAEAV?$input_adapter_character_source@V?$stream_input_adapter@D@__crt_stdio_input@@@1@_K@Z@4QBDB 0000000180058550     libucrt:input.obj
 0002:00002554       ?lowercase@?1???$parse_floating_point_possible_nan@DV?$input_adapter_character_source@V?$stream_input_adapter@D@__crt_stdio_input@@@__crt_strtox@@_K@__crt_strtox@@YA?AW4floating_point_parse_result@1@AEADAEAV?$input_adapter_character_source@V?$stream_input_adapter@D@__crt_stdio_input@@@1@_K@Z@4QBDB 0000000180058554     libucrt:input.obj
 0002:00002558       ?uppercase@?1???$parse_floating_point_possible_nan_is_snan@DV?$input_adapter_character_source@V?$stream_input_adapter@D@__crt_stdio_input@@@__crt_strtox@@@__crt_strtox@@YA_NAEADAEAV?$input_adapter_character_source@V?$stream_input_adapter@D@__crt_stdio_input@@@1@@Z@4QBDB 0000000180058558     libucrt:input.obj
 0002:00002560       ?lowercase@?1???$parse_floating_point_possible_nan_is_snan@DV?$input_adapter_character_source@V?$stream_input_adapter@D@__crt_stdio_input@@@__crt_strtox@@@__crt_strtox@@YA_NAEADAEAV?$input_adapter_character_source@V?$stream_input_adapter@D@__crt_stdio_input@@@1@@Z@4QBDB 0000000180058560     libucrt:input.obj
 0002:00002568       ?uppercase@?1???$parse_floating_point_possible_nan_is_ind@DV?$input_adapter_character_source@V?$stream_input_adapter@D@__crt_stdio_input@@@__crt_strtox@@@__crt_strtox@@YA_NAEADAEAV?$input_adapter_character_source@V?$stream_input_adapter@D@__crt_stdio_input@@@1@@Z@4QBDB 0000000180058568     libucrt:input.obj
 0002:0000256c       ?lowercase@?1???$parse_floating_point_possible_nan_is_ind@DV?$input_adapter_character_source@V?$stream_input_adapter@D@__crt_stdio_input@@@__crt_strtox@@@__crt_strtox@@YA_NAEADAEAV?$input_adapter_character_source@V?$stream_input_adapter@D@__crt_stdio_input@@@1@@Z@4QBDB 000000018005856c     libucrt:input.obj
 0002:000025a0       __acrt_exception_action_table 00000001800585a0     libucrt:exception_filter.obj
 0002:00002660       __acrt_signal_action_table_count 0000000180058660     libucrt:exception_filter.obj
 0002:00002668       __acrt_signal_action_first_fpe_index 0000000180058668     libucrt:exception_filter.obj
 0002:00002670       __acrt_signal_action_fpe_count 0000000180058670     libucrt:exception_filter.obj
 0002:00002678       ??_C@_1BI@BGOHAHKC@?$AAm?$AAs?$AAc?$AAo?$AAr?$AAe?$AAe?$AA?4?$AAd?$AAl?$AAl@ 0000000180058678     libucrt:exit.obj
 0002:00002690       ??_C@_0P@MIGLKIOC@CorExitProcess@ 0000000180058690     libucrt:exit.obj
 0002:00002820       ??_C@_03OEIAHPBN@INF@      0000000180058820     libucrt:cvt.obj
 0002:00002824       ??_C@_03OJHLLCGB@inf@      0000000180058824     libucrt:cvt.obj
 0002:00002828       ??_C@_03LKNCIKJB@NAN@      0000000180058828     libucrt:cvt.obj
 0002:0000282c       ??_C@_03LHCJEHON@nan@      000000018005882c     libucrt:cvt.obj
 0002:00002830       ??_C@_09OFJJIMPC@NAN?$CISNAN?$CJ@ 0000000180058830     libucrt:cvt.obj
 0002:00002840       ??_C@_09IPFBKMDL@nan?$CIsnan?$CJ@ 0000000180058840     libucrt:cvt.obj
 0002:00002850       ??_C@_08IKHNHAJ@NAN?$CIIND?$CJ@ 0000000180058850     libucrt:cvt.obj
 0002:00002860       ??_C@_08OFCDMILK@nan?$CIind?$CJ@ 0000000180058860     libucrt:cvt.obj
 0002:0000286c       ??_C@_05KLBDPFGC@e?$CL000@ 000000018005886c     libucrt:cvt.obj
 0002:00002880       __lc_time_c                0000000180058880     libucrt:nlsdata.obj
 0002:00002b40       ??_C@_03KOEHGMDN@Sun@      0000000180058b40     libucrt:nlsdata.obj
 0002:00002b44       ??_C@_03PDAGKDH@Mon@       0000000180058b44     libucrt:nlsdata.obj
 0002:00002b48       ??_C@_03NAGEINEP@Tue@      0000000180058b48     libucrt:nlsdata.obj
 0002:00002b4c       ??_C@_03MHOMLAJA@Wed@      0000000180058b4c     libucrt:nlsdata.obj
 0002:00002b50       ??_C@_03IOFIKPDN@Thu@      0000000180058b50     libucrt:nlsdata.obj
 0002:00002b54       ??_C@_03IDIOELNC@Fri@      0000000180058b54     libucrt:nlsdata.obj
 0002:00002b58       ??_C@_03FEFJNEK@Sat@       0000000180058b58     libucrt:nlsdata.obj
 0002:00002b5c       ??_C@_06OOPIFAJ@Sunday@    0000000180058b5c     libucrt:nlsdata.obj
 0002:00002b64       ??_C@_06JLEDEDGH@Monday@   0000000180058b64     libucrt:nlsdata.obj
 0002:00002b70       ??_C@_07BAAGCFCM@Tuesday@  0000000180058b70     libucrt:nlsdata.obj
 0002:00002b78       ??_C@_09DLIGFAKA@Wednesday@ 0000000180058b78     libucrt:nlsdata.obj
 0002:00002b88       ??_C@_08HACCIKIA@Thursday@ 0000000180058b88     libucrt:nlsdata.obj
 0002:00002b94       ??_C@_06JECMNKMI@Friday@   0000000180058b94     libucrt:nlsdata.obj
 0002:00002ba0       ??_C@_08INBOOONO@Saturday@ 0000000180058ba0     libucrt:nlsdata.obj
 0002:00002bac       ??_C@_03JIHJHPIE@Jan@      0000000180058bac     libucrt:nlsdata.obj
 0002:00002bb0       ??_C@_03HJBDCHOM@Feb@      0000000180058bb0     libucrt:nlsdata.obj
 0002:00002bb4       ??_C@_03ODNJBKGA@Mar@      0000000180058bb4     libucrt:nlsdata.obj
 0002:00002bb8       ??_C@_03LEOLGMJP@Apr@      0000000180058bb8     libucrt:nlsdata.obj
 0002:00002bbc       ??_C@_03CNMDKL@May@        0000000180058bbc     libucrt:nlsdata.obj
 0002:00002bc0       ??_C@_03IDFGHECI@Jun@      0000000180058bc0     libucrt:nlsdata.obj
 0002:00002bc4       ??_C@_03LBGABGKK@Jul@      0000000180058bc4     libucrt:nlsdata.obj
 0002:00002bc8       ??_C@_03IFJFEIGA@Aug@      0000000180058bc8     libucrt:nlsdata.obj
 0002:00002bcc       ??_C@_03GGCAPAJC@Sep@      0000000180058bcc     libucrt:nlsdata.obj
 0002:00002bd0       ??_C@_03BMAOKBAD@Oct@      0000000180058bd0     libucrt:nlsdata.obj
 0002:00002bd4       ??_C@_03JPJOFNIA@Nov@      0000000180058bd4     libucrt:nlsdata.obj
 0002:00002bd8       ??_C@_03MKABNOCG@Dec@      0000000180058bd8     libucrt:nlsdata.obj
 0002:00002be0       ??_C@_07CGJPFGJA@January@  0000000180058be0     libucrt:nlsdata.obj
 0002:00002be8       ??_C@_08GNJGEPFN@February@ 0000000180058be8     libucrt:nlsdata.obj
 0002:00002bf4       ??_C@_05HPCKOFNC@March@    0000000180058bf4     libucrt:nlsdata.obj
 0002:00002bfc       ??_C@_05DMJDNLEJ@April@    0000000180058bfc     libucrt:nlsdata.obj
 0002:00002c04       ??_C@_04CNLMGBGM@June@     0000000180058c04     libucrt:nlsdata.obj
 0002:00002c0c       ??_C@_04MIEPOIFP@July@     0000000180058c0c     libucrt:nlsdata.obj
 0002:00002c14       ??_C@_06LBBHFDDG@August@   0000000180058c14     libucrt:nlsdata.obj
 0002:00002c20       ??_C@_09BHHEALKD@September@ 0000000180058c20     libucrt:nlsdata.obj
 0002:00002c30       ??_C@_07JJNFCEND@October@  0000000180058c30     libucrt:nlsdata.obj
 0002:00002c38       ??_C@_08HCHEGEOA@November@ 0000000180058c38     libucrt:nlsdata.obj
 0002:00002c48       ??_C@_08EDHMEBNP@December@ 0000000180058c48     libucrt:nlsdata.obj
 0002:00002c54       ??_C@_02DEDBPAFC@AM@       0000000180058c54     libucrt:nlsdata.obj
 0002:00002c58       ??_C@_02CJNFDJBF@PM@       0000000180058c58     libucrt:nlsdata.obj
 0002:00002c60       ??_C@_08BPBNCDIB@MM?1dd?1yy@ 0000000180058c60     libucrt:nlsdata.obj
 0002:00002c70       ??_C@_0BE@CKGJFCPC@dddd?0?5MMMM?5dd?0?5yyyy@ 0000000180058c70     libucrt:nlsdata.obj
 0002:00002c88       ??_C@_08JCCMCCIL@HH?3mm?3ss@ 0000000180058c88     libucrt:nlsdata.obj
 0002:00002c98       ??_C@_17MBGCMIPB@?$AAS?$AAu?$AAn@ 0000000180058c98     libucrt:nlsdata.obj
 0002:00002ca0       ??_C@_17KBOMKBF@?$AAM?$AAo?$AAn@ 0000000180058ca0     libucrt:nlsdata.obj
 0002:00002ca8       ??_C@_17BMKGEGOJ@?$AAT?$AAu?$AAe@ 0000000180058ca8     libucrt:nlsdata.obj
 0002:00002cb0       ??_C@_17CJEDCEPE@?$AAW?$AAe?$AAd@ 0000000180058cb0     libucrt:nlsdata.obj
 0002:00002cb8       ??_C@_17PDPHAADD@?$AAT?$AAh?$AAu@ 0000000180058cb8     libucrt:nlsdata.obj
 0002:00002cc0       ??_C@_17HFOLPPLP@?$AAF?$AAr?$AAi@ 0000000180058cc0     libucrt:nlsdata.obj
 0002:00002cc8       ??_C@_17GGIBDPIH@?$AAS?$AAa?$AAt@ 0000000180058cc8     libucrt:nlsdata.obj
 0002:00002cd0       ??_C@_1O@IHNHDHPB@?$AAS?$AAu?$AAn?$AAd?$AAa?$AAy@ 0000000180058cd0     libucrt:nlsdata.obj
 0002:00002ce0       ??_C@_1O@MMNBFLIA@?$AAM?$AAo?$AAn?$AAd?$AAa?$AAy@ 0000000180058ce0     libucrt:nlsdata.obj
 0002:00002cf0       ??_C@_1BA@ENFBFFEK@?$AAT?$AAu?$AAe?$AAs?$AAd?$AAa?$AAy@ 0000000180058cf0     libucrt:nlsdata.obj
 0002:00002d00       ??_C@_1BE@EBOGMDOH@?$AAW?$AAe?$AAd?$AAn?$AAe?$AAs?$AAd?$AAa?$AAy@ 0000000180058d00     libucrt:nlsdata.obj
 0002:00002d18       ??_C@_1BC@HHMNLIHE@?$AAT?$AAh?$AAu?$AAr?$AAs?$AAd?$AAa?$AAy@ 0000000180058d18     libucrt:nlsdata.obj
 0002:00002d30       ??_C@_1O@PDICJHAG@?$AAF?$AAr?$AAi?$AAd?$AAa?$AAy@ 0000000180058d30     libucrt:nlsdata.obj
 0002:00002d40       ??_C@_1BC@ENMNNPAJ@?$AAS?$AAa?$AAt?$AAu?$AAr?$AAd?$AAa?$AAy@ 0000000180058d40     libucrt:nlsdata.obj
 0002:00002d58       ??_C@_17DKNBKCHM@?$AAJ?$AAa?$AAn@ 0000000180058d58     libucrt:nlsdata.obj
 0002:00002d60       ??_C@_17LMDJEKJN@?$AAF?$AAe?$AAb@ 0000000180058d60     libucrt:nlsdata.obj
 0002:00002d68       ??_C@_17CKNLEDEC@?$AAM?$AAa?$AAr@ 0000000180058d68     libucrt:nlsdata.obj
 0002:00002d70       ??_C@_17LFPOIHDD@?$AAA?$AAp?$AAr@ 0000000180058d70     libucrt:nlsdata.obj
 0002:00002d78       ??_C@_17PNNKMEED@?$AAM?$AAa?$AAy@ 0000000180058d78     libucrt:nlsdata.obj
 0002:00002d80       ??_C@_17KCJGOCPB@?$AAJ?$AAu?$AAn@ 0000000180058d80     libucrt:nlsdata.obj
 0002:00002d88       ??_C@_17IJPCKHK@?$AAJ?$AAu?$AAl@ 0000000180058d88     libucrt:nlsdata.obj
 0002:00002d90       ??_C@_17ICPELBCN@?$AAA?$AAu?$AAg@ 0000000180058d90     libucrt:nlsdata.obj
 0002:00002d98       ??_C@_17HCHCOKMG@?$AAS?$AAe?$AAp@ 0000000180058d98     libucrt:nlsdata.obj
 0002:00002da0       ??_C@_17FNLKOI@?$AAO?$AAc?$AAt@ 0000000180058da0     libucrt:nlsdata.obj
 0002:00002da8       ??_C@_17BBDMLCIG@?$AAN?$AAo?$AAv@ 0000000180058da8     libucrt:nlsdata.obj
 0002:00002db0       ??_C@_17EGKACKIF@?$AAD?$AAe?$AAc@ 0000000180058db0     libucrt:nlsdata.obj
 0002:00002db8       ??_C@_1BA@EFMEIEBA@?$AAJ?$AAa?$AAn?$AAu?$AAa?$AAr?$AAy@ 0000000180058db8     libucrt:nlsdata.obj
 0002:00002dc8       ??_C@_1BC@JGDDFFAM@?$AAF?$AAe?$AAb?$AAr?$AAu?$AAa?$AAr?$AAy@ 0000000180058dc8     libucrt:nlsdata.obj
 0002:00002de0       ??_C@_1M@IKEENEDF@?$AAM?$AAa?$AAr?$AAc?$AAh@ 0000000180058de0     libucrt:nlsdata.obj
 0002:00002df0       ??_C@_1M@GJNLMHFD@?$AAA?$AAp?$AAr?$AAi?$AAl@ 0000000180058df0     libucrt:nlsdata.obj
 0002:00002e00       ??_C@_19EPFLPGAP@?$AAJ?$AAu?$AAn?$AAe@ 0000000180058e00     libucrt:nlsdata.obj
 0002:00002e10       ??_C@_19BIFMLPCD@?$AAJ?$AAu?$AAl?$AAy@ 0000000180058e10     libucrt:nlsdata.obj
 0002:00002e20       ??_C@_1O@PAHLKOAC@?$AAA?$AAu?$AAg?$AAu?$AAs?$AAt@ 0000000180058e20     libucrt:nlsdata.obj
 0002:00002e30       ??_C@_1BE@DKAAMBJL@?$AAS?$AAe?$AAp?$AAt?$AAe?$AAm?$AAb?$AAe?$AAr@ 0000000180058e30     libucrt:nlsdata.obj
 0002:00002e48       ??_C@_1BA@EPANDLNG@?$AAO?$AAc?$AAt?$AAo?$AAb?$AAe?$AAr@ 0000000180058e48     libucrt:nlsdata.obj
 0002:00002e58       ??_C@_1BC@BGLIFPF@?$AAN?$AAo?$AAv?$AAe?$AAm?$AAb?$AAe?$AAr@ 0000000180058e58     libucrt:nlsdata.obj
 0002:00002e70       ??_C@_1BC@FEMKIFH@?$AAD?$AAe?$AAc?$AAe?$AAm?$AAb?$AAe?$AAr@ 0000000180058e70     libucrt:nlsdata.obj
 0002:00002e84       ??_C@_15ODEHAHHF@?$AAA?$AAM@ 0000000180058e84     libucrt:nlsdata.obj
 0002:00002e8c       ??_C@_15CLMNNGEL@?$AAP?$AAM@ 0000000180058e8c     libucrt:nlsdata.obj
 0002:00002e98       ??_C@_1BC@IEBCMHCM@?$AAM?$AAM?$AA?1?$AAd?$AAd?$AA?1?$AAy?$AAy@ 0000000180058e98     libucrt:nlsdata.obj
 0002:00002eb0       ??_C@_1CI@KNAKOEBC@?$AAd?$AAd?$AAd?$AAd?$AA?0?$AA?5?$AAM?$AAM?$AAM?$AAM?$AA?5?$AAd?$AAd?$AA?0?$AA?5@ 0000000180058eb0     libucrt:nlsdata.obj
 0002:00002ed8       ??_C@_1BC@GDGBMEMK@?$AAH?$AAH?$AA?3?$AAm?$AAm?$AA?3?$AAs?$AAs@ 0000000180058ed8     libucrt:nlsdata.obj
 0002:00002ef0       ??_C@_1M@BMHNFIME@?$AAe?$AAn?$AA?9?$AAU?$AAS@ 0000000180058ef0     libucrt:nlsdata.obj
 0002:00002f10       ?ccs@?1???$__acrt_stdio_parse_mode@_W@@YA?AU__acrt_stdio_stream_mode@@QEB_W@Z@4QB_WB 0000000180058f10     libucrt:openfile.obj
 0002:00002f18       ?utf8_encoding@?1???$__acrt_stdio_parse_mode@_W@@YA?AU__acrt_stdio_stream_mode@@QEB_W@Z@4QB_WB 0000000180058f18     libucrt:openfile.obj
 0002:00002f28       ?utf16_encoding@?1???$__acrt_stdio_parse_mode@_W@@YA?AU__acrt_stdio_stream_mode@@QEB_W@Z@4QB_WB 0000000180058f28     libucrt:openfile.obj
 0002:00002f38       ?unicode_encoding@?1???$__acrt_stdio_parse_mode@_W@@YA?AU__acrt_stdio_stream_mode@@QEB_W@Z@4QB_WB 0000000180058f38     libucrt:openfile.obj
 0002:00002ff0       ??_C@_1EA@JGEFHKEI@?$AAa?$AAp?$AAi?$AA?9?$AAm?$AAs?$AA?9?$AAw?$AAi?$AAn?$AA?9?$AAc?$AAo?$AAr?$AAe@ 0000000180058ff0     libucrt:winapi_thunks.obj
 0002:00003030       ??_C@_1DI@IJCEHOCB@?$AAa?$AAp?$AAi?$AA?9?$AAm?$AAs?$AA?9?$AAw?$AAi?$AAn?$AA?9?$AAc?$AAo?$AAr?$AAe@ 0000000180059030     libucrt:winapi_thunks.obj
 0002:00003070       ??_C@_1EI@MPIAOHOC@?$AAa?$AAp?$AAi?$AA?9?$AAm?$AAs?$AA?9?$AAw?$AAi?$AAn?$AA?9?$AAc?$AAo?$AAr?$AAe@ 0000000180059070     libucrt:winapi_thunks.obj
 0002:000030c0       ??_C@_1FK@FPHCKFIE@?$AAa?$AAp?$AAi?$AA?9?$AAm?$AAs?$AA?9?$AAw?$AAi?$AAn?$AA?9?$AAc?$AAo?$AAr?$AAe@ 00000001800590c0     libucrt:winapi_thunks.obj
 0002:00003120       ??_C@_1EM@DILCGIIO@?$AAa?$AAp?$AAi?$AA?9?$AAm?$AAs?$AA?9?$AAw?$AAi?$AAn?$AA?9?$AAc?$AAo?$AAr?$AAe@ 0000000180059120     libucrt:winapi_thunks.obj
 0002:00003170       ??_C@_1DM@LNCGDDPN@?$AAa?$AAp?$AAi?$AA?9?$AAm?$AAs?$AA?9?$AAw?$AAi?$AAn?$AA?9?$AAc?$AAo?$AAr?$AAe@ 0000000180059170     libucrt:winapi_thunks.obj
 0002:000031b0       ??_C@_1DO@FPAPJEMD@?$AAa?$AAp?$AAi?$AA?9?$AAm?$AAs?$AA?9?$AAw?$AAi?$AAn?$AA?9?$AAc?$AAo?$AAr?$AAe@ 00000001800591b0     libucrt:winapi_thunks.obj
 0002:000031f0       ??_C@_1DK@NDHNAHIO@?$AAa?$AAp?$AAi?$AA?9?$AAm?$AAs?$AA?9?$AAw?$AAi?$AAn?$AA?9?$AAc?$AAo?$AAr?$AAe@ 00000001800591f0     libucrt:winapi_thunks.obj
 0002:00003230       ??_C@_1DM@KGHDGBCM@?$AAa?$AAp?$AAi?$AA?9?$AAm?$AAs?$AA?9?$AAw?$AAi?$AAn?$AA?9?$AAc?$AAo?$AAr?$AAe@ 0000000180059230     libucrt:winapi_thunks.obj
 0002:00003270       ??_C@_1EO@IJIOEFOH@?$AAa?$AAp?$AAi?$AA?9?$AAm?$AAs?$AA?9?$AAw?$AAi?$AAn?$AA?9?$AAr?$AAt?$AAc?$AAo@ 0000000180059270     libucrt:winapi_thunks.obj
 0002:000032c0       ??_C@_1FG@HHGEKANL@?$AAa?$AAp?$AAi?$AA?9?$AAm?$AAs?$AA?9?$AAw?$AAi?$AAn?$AA?9?$AAs?$AAe?$AAc?$AAu@ 00000001800592c0     libucrt:winapi_thunks.obj
 0002:00003320       ??_C@_1EG@DBIOJECG@?$AAe?$AAx?$AAt?$AA?9?$AAm?$AAs?$AA?9?$AAw?$AAi?$AAn?$AA?9?$AAn?$AAt?$AAu?$AAs@ 0000000180059320     libucrt:winapi_thunks.obj
 0002:00003370       ??_C@_1EO@FIHMJCLF@?$AAe?$AAx?$AAt?$AA?9?$AAm?$AAs?$AA?9?$AAw?$AAi?$AAn?$AA?9?$AAn?$AAt?$AAu?$AAs@ 0000000180059370     libucrt:winapi_thunks.obj
 0002:000033c0       ??_C@_1BC@DNHGCMLG@?$AAa?$AAd?$AAv?$AAa?$AAp?$AAi?$AA3?$AA2@ 00000001800593c0     libucrt:winapi_thunks.obj
 0002:000033d8       ??_C@_1M@OAIMIKLP@?$AAn?$AAt?$AAd?$AAl?$AAl@ 00000001800593d8     libucrt:winapi_thunks.obj
 0002:000033f0       ??_C@_1EG@DPGNFKGC@?$AAa?$AAp?$AAi?$AA?9?$AAm?$AAs?$AA?9?$AAw?$AAi?$AAn?$AA?9?$AAa?$AAp?$AAp?$AAm@ 00000001800593f0     libucrt:winapi_thunks.obj
 0002:00003438       ??_C@_1O@BCCLBEOE@?$AAu?$AAs?$AAe?$AAr?$AA3?$AA2@ 0000000180059438     libucrt:winapi_thunks.obj
 0002:00003448       ??_C@_1BA@IAIFMGEF@?$AAe?$AAx?$AAt?$AA?9?$AAm?$AAs?$AA?9@ 0000000180059448     libucrt:winapi_thunks.obj
 0002:00003460       ??_C@_0BA@FHFNEAED@AreFileApisANSI@ 0000000180059460     libucrt:winapi_thunks.obj
 0002:00003478       ??_C@_0BA@IHGNDAEB@CompareStringEx@ 0000000180059478     libucrt:winapi_thunks.obj
 0002:000034b8       ??_C@_0O@KKBNKAPF@LCMapStringEx@ 00000001800594b8     libucrt:winapi_thunks.obj
 0002:000034d0       ??_C@_0BB@HBDEELFH@LocaleNameToLCID@ 00000001800594d0     libucrt:winapi_thunks.obj
 0002:000034e8       ??_C@_0CF@OJOFEIGO@AppPolicyGetProcessTerminationM@ 00000001800594e8     libucrt:winapi_thunks.obj
 0002:00003510       _sys_errlist               0000000180059510     libucrt:syserr.obj
 0002:00003670       ??_C@_08INEPGKHH@No?5error@ 0000000180059670     libucrt:syserr.obj
 0002:00003680       ??_C@_0BI@BJFCGOHL@Operation?5not?5permitted@ 0000000180059680     libucrt:syserr.obj
 0002:00003698       ??_C@_0BK@FMDHKPNF@No?5such?5file?5or?5directory@ 0000000180059698     libucrt:syserr.obj
 0002:000036b8       ??_C@_0BA@FKIAIBGA@No?5such?5process@ 00000001800596b8     libucrt:syserr.obj
 0002:000036c8       ??_C@_0BK@FJBOAFDK@Interrupted?5function?5call@ 00000001800596c8     libucrt:syserr.obj
 0002:000036e8       ??_C@_0BD@KKNFOBBD@Input?1output?5error@ 00000001800596e8     libucrt:syserr.obj
 0002:00003700       ??_C@_0BK@DPKMCKJ@No?5such?5device?5or?5address@ 0000000180059700     libucrt:syserr.obj
 0002:00003720       ??_C@_0BC@MFFGCDFL@Arg?5list?5too?5long@ 0000000180059720     libucrt:syserr.obj
 0002:00003738       ??_C@_0BC@HKPNECK@Exec?5format?5error@ 0000000180059738     libucrt:syserr.obj
 0002:00003750       ??_C@_0BE@NFGDDCEF@Bad?5file?5descriptor@ 0000000180059750     libucrt:syserr.obj
 0002:00003768       ??_C@_0BD@LOHELEP@No?5child?5processes@ 0000000180059768     libucrt:syserr.obj
 0002:00003780       ??_C@_0CB@EPFKGNAK@Resource?5temporarily?5unavailabl@ 0000000180059780     libucrt:syserr.obj
 0002:000037a8       ??_C@_0BB@IMDKMPFB@Not?5enough?5space@ 00000001800597a8     libucrt:syserr.obj
 0002:000037c0       ??_C@_0BC@HFNFNKAI@Permission?5denied@ 00000001800597c0     libucrt:syserr.obj
 0002:000037d8       ??_C@_0M@LOEHLCJD@Bad?5address@ 00000001800597d8     libucrt:syserr.obj
 0002:000037e8       ??_C@_0O@NIPGCINC@Unknown?5error@ 00000001800597e8     libucrt:syserr.obj
 0002:000037f8       ??_C@_0BA@BIBLIOEK@Resource?5device@ 00000001800597f8     libucrt:syserr.obj
 0002:00003808       ??_C@_0M@NAAJNNGH@File?5exists@ 0000000180059808     libucrt:syserr.obj
 0002:00003818       ??_C@_0O@OAMDNOCP@Improper?5link@ 0000000180059818     libucrt:syserr.obj
 0002:00003828       ??_C@_0P@NLEIANHE@No?5such?5device@ 0000000180059828     libucrt:syserr.obj
 0002:00003838       ??_C@_0BA@CJBACOOL@Not?5a?5directory@ 0000000180059838     libucrt:syserr.obj
 0002:00003848       ??_C@_0P@NDHGCGKE@Is?5a?5directory@ 0000000180059848     libucrt:syserr.obj
 0002:00003858       ??_C@_0BB@HMGGCEBG@Invalid?5argument@ 0000000180059858     libucrt:syserr.obj
 0002:00003870       ??_C@_0BO@IIFBODJE@Too?5many?5open?5files?5in?5system@ 0000000180059870     libucrt:syserr.obj
 0002:00003890       ??_C@_0BE@INBJMKGG@Too?5many?5open?5files@ 0000000180059890     libucrt:syserr.obj
 0002:000038a8       ??_C@_0CE@ONOKNLPF@Inappropriate?5I?1O?5control?5opera@ 00000001800598a8     libucrt:syserr.obj
 0002:000038d0       ??_C@_0P@LFMMIPAE@File?5too?5large@ 00000001800598d0     libucrt:syserr.obj
 0002:000038e0       ??_C@_0BI@FEALHKLD@No?5space?5left?5on?5device@ 00000001800598e0     libucrt:syserr.obj
 0002:000038f8       ??_C@_0N@FEHLOILP@Invalid?5seek@ 00000001800598f8     libucrt:syserr.obj
 0002:00003908       ??_C@_0BG@DDBFNKBH@Read?9only?5file?5system@ 0000000180059908     libucrt:syserr.obj
 0002:00003920       ??_C@_0P@PKCJJLLM@Too?5many?5links@ 0000000180059920     libucrt:syserr.obj
 0002:00003930       ??_C@_0M@LHEPIIOM@Broken?5pipe@ 0000000180059930     libucrt:syserr.obj
 0002:00003940       ??_C@_0N@MMJPGLJK@Domain?5error@ 0000000180059940     libucrt:syserr.obj
 0002:00003950       ??_C@_0BB@FCBJFCAJ@Result?5too?5large@ 0000000180059950     libucrt:syserr.obj
 0002:00003968       ??_C@_0BK@JAEBMJJM@Resource?5deadlock?5avoided@ 0000000180059968     libucrt:syserr.obj
 0002:00003988       ??_C@_0BC@BEDIHIDK@Filename?5too?5long@ 0000000180059988     libucrt:syserr.obj
 0002:000039a0       ??_C@_0BD@CLHBCGPB@No?5locks?5available@ 00000001800599a0     libucrt:syserr.obj
 0002:000039b8       ??_C@_0BJ@IHEHINLI@Function?5not?5implemented@ 00000001800599b8     libucrt:syserr.obj
 0002:000039d8       ??_C@_0BE@ICMCHPHH@Directory?5not?5empty@ 00000001800599d8     libucrt:syserr.obj
 0002:000039f0       ??_C@_0BG@KLEAJEFJ@Illegal?5byte?5sequence@ 00000001800599f0     libucrt:syserr.obj
 0002:00003a08       _sys_nerr                  0000000180059a08     libucrt:syserr.obj
 0002:00003a10       __newctype                 0000000180059a10     libucrt:ctype.obj
 0002:00003d10       __newclmap                 0000000180059d10     libucrt:ctype.obj
 0002:00003e90       __newcumap                 0000000180059e90     libucrt:ctype.obj
 0002:00004010       _wctype                    000000018005a010     libucrt:ctype.obj
 0002:00004268       ??_C@_1M@HPNHIDJI@?$AAj?$AAa?$AA?9?$AAJ?$AAP@ 000000018005a268     libucrt:mbctype.obj
 0002:00004278       ??_C@_1M@BIBDDEMK@?$AAz?$AAh?$AA?9?$AAC?$AAN@ 000000018005a278     libucrt:mbctype.obj
 0002:00004288       ??_C@_1M@JLOOOEGK@?$AAk?$AAo?$AA?9?$AAK?$AAR@ 000000018005a288     libucrt:mbctype.obj
 0002:00004298       ??_C@_1M@CLNBBOPM@?$AAz?$AAh?$AA?9?$AAT?$AAW@ 000000018005a298     libucrt:mbctype.obj
 0002:00004348       ??_C@_05DNEBIAHO@1?$CDINF@ 000000018005a348     libucrt:cfout.obj
 0002:00004350       ??_C@_06IMKFLFPG@1?$CDQNAN@ 000000018005a350     libucrt:cfout.obj
 0002:00004358       ??_C@_06PGGFOGJG@1?$CDSNAN@ 000000018005a358     libucrt:cfout.obj
 0002:00004360       ??_C@_05PHHOCPM@1?$CDIND@  000000018005a360     libucrt:cfout.obj
 0002:00004368       ??_C@_15PJPFLCCM@?$AAu?$AAk@ 000000018005a368     libucrt:get_qualified_locale.obj
 0002:000051b0       ??_C@_15EMKDOKLE@?$AAa?$AAr@ 000000018005b1b0     libucrt:lcidtoname_downlevel.obj
 0002:000051b8       ??_C@_15KNPADPLH@?$AAb?$AAg@ 000000018005b1b8     libucrt:lcidtoname_downlevel.obj
 0002:000051c0       ??_C@_15EDMHLDMO@?$AAc?$AAa@ 000000018005b1c0     libucrt:lcidtoname_downlevel.obj
 0002:000051c8       ??_C@_1O@BPEAJADD@?$AAz?$AAh?$AA?9?$AAC?$AAH?$AAS@ 000000018005b1c8     libucrt:lcidtoname_downlevel.obj
 0002:000051d8       ??_C@_15LJNHCMNK@?$AAc?$AAs@ 000000018005b1d8     libucrt:lcidtoname_downlevel.obj
 0002:000051e0       ??_C@_15FOMCIDHG@?$AAd?$AAa@ 000000018005b1e0     libucrt:lcidtoname_downlevel.obj
 0002:000051e8       ??_C@_15NBKABECB@?$AAd?$AAe@ 000000018005b1e8     libucrt:lcidtoname_downlevel.obj
 0002:000051f0       ??_C@_15GHPEIIAO@?$AAe?$AAl@ 000000018005b1f0     libucrt:lcidtoname_downlevel.obj
 0002:000051f8       ??_C@_15MNPNEAIF@?$AAe?$AAn@ 000000018005b1f8     libucrt:lcidtoname_downlevel.obj
 0002:00005200       ??_C@_15GPIOMPMH@?$AAe?$AAs@ 000000018005b200     libucrt:lcidtoname_downlevel.obj
 0002:00005208       ??_C@_15NGLOAKJC@?$AAf?$AAi@ 000000018005b208     libucrt:lcidtoname_downlevel.obj
 0002:00005210       ??_C@_15FBKGNKAM@?$AAf?$AAr@ 000000018005b210     libucrt:lcidtoname_downlevel.obj
 0002:00005218       ??_C@_15KGGCNEFK@?$AAh?$AAe@ 000000018005b218     libucrt:lcidtoname_downlevel.obj
 0002:00005220       ??_C@_15PGHLIDMF@?$AAh?$AAu@ 000000018005b220     libucrt:lcidtoname_downlevel.obj
 0002:00005228       ??_C@_15BIEMAPLM@?$AAi?$AAs@ 000000018005b228     libucrt:lcidtoname_downlevel.obj
 0002:00005230       ??_C@_15IFJLDHAF@?$AAi?$AAt@ 000000018005b230     libucrt:lcidtoname_downlevel.obj
 0002:00005238       ??_C@_15GEMIOCAG@?$AAj?$AAa@ 000000018005b238     libucrt:lcidtoname_downlevel.obj
 0002:00005240       ??_C@_15EPELEGJA@?$AAk?$AAo@ 000000018005b240     libucrt:lcidtoname_downlevel.obj
 0002:00005248       ??_C@_15NDDHIMN@?$AAn?$AAl@ 000000018005b248     libucrt:lcidtoname_downlevel.obj
 0002:00005250       ??_C@_15BPIGNHCD@?$AAn?$AAo@ 000000018005b250     libucrt:lcidtoname_downlevel.obj
 0002:00005258       ??_C@_15DEOPBLCG@?$AAp?$AAl@ 000000018005b258     libucrt:lcidtoname_downlevel.obj
 0002:00005260       ??_C@_15KBECGEFG@?$AAp?$AAt@ 000000018005b260     libucrt:lcidtoname_downlevel.obj
 0002:00005268       ??_C@_15GLJCBFMD@?$AAr?$AAo@ 000000018005b268     libucrt:lcidtoname_downlevel.obj
 0002:00005270       ??_C@_15FEDGKCDI@?$AAr?$AAu@ 000000018005b270     libucrt:lcidtoname_downlevel.obj
 0002:00005278       ??_C@_15GLKMLLHM@?$AAh?$AAr@ 000000018005b278     libucrt:lcidtoname_downlevel.obj
 0002:00005280       ??_C@_15CPKMFBDB@?$AAs?$AAk@ 000000018005b280     libucrt:lcidtoname_downlevel.obj
 0002:00005288       ??_C@_15BAAIOGMK@?$AAs?$AAq@ 000000018005b288     libucrt:lcidtoname_downlevel.obj
 0002:00005290       ??_C@_15INNPNOHD@?$AAs?$AAv@ 000000018005b290     libucrt:lcidtoname_downlevel.obj
 0002:00005298       ??_C@_15CABMMOGH@?$AAt?$AAh@ 000000018005b298     libucrt:lcidtoname_downlevel.obj
 0002:000052a0       ??_C@_15BPLIHJJM@?$AAt?$AAr@ 000000018005b2a0     libucrt:lcidtoname_downlevel.obj
 0002:000052a8       ??_C@_15NEOEKKDJ@?$AAu?$AAr@ 000000018005b2a8     libucrt:lcidtoname_downlevel.obj
 0002:000052b0       ??_C@_15NFICGAJK@?$AAi?$AAd@ 000000018005b2b0     libucrt:lcidtoname_downlevel.obj
 0002:000052b8       ??_C@_15HPJPHDM@?$AAb?$AAe@ 000000018005b2b8     libucrt:lcidtoname_downlevel.obj
 0002:000052c0       ??_C@_15LCHLGJII@?$AAs?$AAl@ 000000018005b2c0     libucrt:lcidtoname_downlevel.obj
 0002:000052c8       ??_C@_15PCFJPHHO@?$AAe?$AAt@ 000000018005b2c8     libucrt:lcidtoname_downlevel.obj
 0002:000052d0       ??_C@_15HPFPGODN@?$AAl?$AAv@ 000000018005b2d0     libucrt:lcidtoname_downlevel.obj
 0002:000052d8       ??_C@_15NFFGKGLG@?$AAl?$AAt@ 000000018005b2d8     libucrt:lcidtoname_downlevel.obj
 0002:000052e0       ??_C@_15BDAKCCHN@?$AAf?$AAa@ 000000018005b2e0     libucrt:lcidtoname_downlevel.obj
 0002:000052e8       ??_C@_15NFGIAIAJ@?$AAv?$AAi@ 000000018005b2e8     libucrt:lcidtoname_downlevel.obj
 0002:000052f0       ??_C@_15LMKNDMHN@?$AAh?$AAy@ 000000018005b2f0     libucrt:lcidtoname_downlevel.obj
 0002:000052f8       ??_C@_15IJBHMCFL@?$AAa?$AAz@ 000000018005b2f8     libucrt:lcidtoname_downlevel.obj
 0002:00005300       ??_C@_15EKOFJABL@?$AAe?$AAu@ 000000018005b300     libucrt:lcidtoname_downlevel.obj
 0002:00005308       ??_C@_15BGHADCNK@?$AAm?$AAk@ 000000018005b308     libucrt:lcidtoname_downlevel.obj
 0002:00005310       ??_C@_15JDNICKHM@?$AAa?$AAf@ 000000018005b310     libucrt:lcidtoname_downlevel.obj
 0002:00005318       ??_C@_15KPJEDBKD@?$AAk?$AAa@ 000000018005b318     libucrt:lcidtoname_downlevel.obj
 0002:00005320       ??_C@_15PDNFFFEO@?$AAf?$AAo@ 000000018005b320     libucrt:lcidtoname_downlevel.obj
 0002:00005328       ??_C@_15OMLEGLOC@?$AAh?$AAi@ 000000018005b328     libucrt:lcidtoname_downlevel.obj
 0002:00005330       ??_C@_15IDNNENKK@?$AAm?$AAs@ 000000018005b330     libucrt:lcidtoname_downlevel.obj
 0002:00005338       ??_C@_15MACJNBMH@?$AAk?$AAk@ 000000018005b338     libucrt:lcidtoname_downlevel.obj
 0002:00005340       ??_C@_15DKDJEOND@?$AAk?$AAy@ 000000018005b340     libucrt:lcidtoname_downlevel.obj
 0002:00005348       ??_C@_15DFGDLJBG@?$AAs?$AAw@ 000000018005b348     libucrt:lcidtoname_downlevel.obj
 0002:00005350       ??_C@_15BBFAICNG@?$AAu?$AAz@ 000000018005b350     libucrt:lcidtoname_downlevel.obj
 0002:00005358       ??_C@_15DKNDCGEA@?$AAt?$AAt@ 000000018005b358     libucrt:lcidtoname_downlevel.obj
 0002:00005360       ??_C@_15MGIFMDPL@?$AAp?$AAa@ 000000018005b360     libucrt:lcidtoname_downlevel.obj
 0002:00005368       ??_C@_15HCNDBBA@?$AAg?$AAu@ 000000018005b368     libucrt:lcidtoname_downlevel.obj
 0002:00005370       ??_C@_15FNBEIBON@?$AAt?$AAa@ 000000018005b370     libucrt:lcidtoname_downlevel.obj
 0002:00005378       ??_C@_15NCHGBGLK@?$AAt?$AAe@ 000000018005b378     libucrt:lcidtoname_downlevel.obj
 0002:00005380       ??_C@_15PHPHCBPF@?$AAk?$AAn@ 000000018005b380     libucrt:lcidtoname_downlevel.obj
 0002:00005388       ??_C@_15DLGBCKMP@?$AAm?$AAr@ 000000018005b388     libucrt:lcidtoname_downlevel.obj
 0002:00005390       ??_C@_15EABBLBFF@?$AAs?$AAa@ 000000018005b390     libucrt:lcidtoname_downlevel.obj
 0002:00005398       ??_C@_15CBKOMCOI@?$AAm?$AAn@ 000000018005b398     libucrt:lcidtoname_downlevel.obj
 0002:000053a0       ??_C@_15CKDMCJAF@?$AAg?$AAl@ 000000018005b3a0     libucrt:lcidtoname_downlevel.obj
 0002:000053a8       ??_C@_17CNJFBPG@?$AAk?$AAo?$AAk@ 000000018005b3a8     libucrt:lcidtoname_downlevel.obj
 0002:000053b0       ??_C@_17FFBJICPL@?$AAs?$AAy?$AAr@ 000000018005b3b0     libucrt:lcidtoname_downlevel.obj
 0002:000053b8       ??_C@_17KPNDCPAF@?$AAd?$AAi?$AAv@ 000000018005b3b8     libucrt:lcidtoname_downlevel.obj
 0002:000053c0       ??_C@_1M@OKAHONE@?$AAa?$AAr?$AA?9?$AAS?$AAA@ 000000018005b3c0     libucrt:lcidtoname_downlevel.obj
 0002:000053d0       ??_C@_1M@FFFIGIGK@?$AAb?$AAg?$AA?9?$AAB?$AAG@ 000000018005b3d0     libucrt:lcidtoname_downlevel.obj
 0002:000053e0       ??_C@_1M@BJNKEDC@?$AAc?$AAa?$AA?9?$AAE?$AAS@ 000000018005b3e0     libucrt:lcidtoname_downlevel.obj
 0002:000053f0       ??_C@_1M@IJJHFJHA@?$AAc?$AAs?$AA?9?$AAC?$AAZ@ 000000018005b3f0     libucrt:lcidtoname_downlevel.obj
 0002:00005400       ??_C@_1M@CLPEOBGI@?$AAd?$AAa?$AA?9?$AAD?$AAK@ 000000018005b400     libucrt:lcidtoname_downlevel.obj
 0002:00005410       ??_C@_1M@MCMADGCB@?$AAd?$AAe?$AA?9?$AAD?$AAE@ 000000018005b410     libucrt:lcidtoname_downlevel.obj
 0002:00005420       ??_C@_1M@OOCKEMAM@?$AAe?$AAl?$AA?9?$AAG?$AAR@ 000000018005b420     libucrt:lcidtoname_downlevel.obj
 0002:00005430       ??_C@_1M@DDNJFGID@?$AAf?$AAi?$AA?9?$AAF?$AAI@ 000000018005b430     libucrt:lcidtoname_downlevel.obj
 0002:00005440       ??_C@_1M@GLIPPMAC@?$AAf?$AAr?$AA?9?$AAF?$AAR@ 000000018005b440     libucrt:lcidtoname_downlevel.obj
 0002:00005450       ??_C@_1M@GFMCHPE@?$AAh?$AAe?$AA?9?$AAI?$AAL@ 000000018005b450     libucrt:lcidtoname_downlevel.obj
 0002:00005460       ??_C@_1M@MHLPGNKM@?$AAh?$AAu?$AA?9?$AAH?$AAU@ 000000018005b460     libucrt:lcidtoname_downlevel.obj
 0002:00005470       ??_C@_1M@LPDDNNPN@?$AAi?$AAs?$AA?9?$AAI?$AAS@ 000000018005b470     libucrt:lcidtoname_downlevel.obj
 0002:00005480       ??_C@_1M@MADIPODN@?$AAi?$AAt?$AA?9?$AAI?$AAT@ 000000018005b480     libucrt:lcidtoname_downlevel.obj
 0002:00005490       ??_C@_1M@IHBJJGG@?$AAn?$AAl?$AA?9?$AAN?$AAL@ 000000018005b490     libucrt:lcidtoname_downlevel.obj
 0002:000054a0       ??_C@_1M@EANAGDL@?$AAn?$AAb?$AA?9?$AAN?$AAO@ 000000018005b4a0     libucrt:lcidtoname_downlevel.obj
 0002:000054b0       ??_C@_1M@NEIEMEGP@?$AAp?$AAl?$AA?9?$AAP?$AAL@ 000000018005b4b0     libucrt:lcidtoname_downlevel.obj
 0002:000054c0       ??_C@_1M@BOCFIGEP@?$AAp?$AAt?$AA?9?$AAB?$AAR@ 000000018005b4c0     libucrt:lcidtoname_downlevel.obj
 0002:000054d0       ??_C@_1M@IMPFOPBG@?$AAr?$AAo?$AA?9?$AAR?$AAO@ 000000018005b4d0     libucrt:lcidtoname_downlevel.obj
 0002:000054e0       ??_C@_1M@IDNNEJMM@?$AAr?$AAu?$AA?9?$AAR?$AAU@ 000000018005b4e0     libucrt:lcidtoname_downlevel.obj
 0002:000054f0       ??_C@_1M@LILEEOGM@?$AAh?$AAr?$AA?9?$AAH?$AAR@ 000000018005b4f0     libucrt:lcidtoname_downlevel.obj
 0002:00005500       ??_C@_1M@FKIFEHPB@?$AAs?$AAk?$AA?9?$AAS?$AAK@ 000000018005b500     libucrt:lcidtoname_downlevel.obj
 0002:00005510       ??_C@_1M@LJMAMNPJ@?$AAs?$AAq?$AA?9?$AAA?$AAL@ 000000018005b510     libucrt:lcidtoname_downlevel.obj
 0002:00005520       ??_C@_1M@GIAKDKJK@?$AAs?$AAv?$AA?9?$AAS?$AAE@ 000000018005b520     libucrt:lcidtoname_downlevel.obj
 0002:00005530       ??_C@_1M@MKJKIKCL@?$AAt?$AAh?$AA?9?$AAT?$AAH@ 000000018005b530     libucrt:lcidtoname_downlevel.obj
 0002:00005540       ??_C@_1M@MFLCCMPB@?$AAt?$AAr?$AA?9?$AAT?$AAR@ 000000018005b540     libucrt:lcidtoname_downlevel.obj
 0002:00005550       ??_C@_1M@OIJHDKJN@?$AAu?$AAr?$AA?9?$AAP?$AAK@ 000000018005b550     libucrt:lcidtoname_downlevel.obj
 0002:00005560       ??_C@_1M@LHIPCIEK@?$AAi?$AAd?$AA?9?$AAI?$AAD@ 000000018005b560     libucrt:lcidtoname_downlevel.obj
 0002:00005570       ??_C@_1M@MFMOBGI@?$AAu?$AAk?$AA?9?$AAU?$AAA@ 000000018005b570     libucrt:lcidtoname_downlevel.obj
 0002:00005580       ??_C@_1M@OBGLJIPL@?$AAb?$AAe?$AA?9?$AAB?$AAY@ 000000018005b580     libucrt:lcidtoname_downlevel.obj
 0002:00005590       ??_C@_1M@BCFAJEAD@?$AAs?$AAl?$AA?9?$AAS?$AAI@ 000000018005b590     libucrt:lcidtoname_downlevel.obj
 0002:000055a0       ??_C@_1M@FKFFEDDN@?$AAe?$AAt?$AA?9?$AAE?$AAE@ 000000018005b5a0     libucrt:lcidtoname_downlevel.obj
 0002:000055b0       ??_C@_1M@KGKKAACI@?$AAl?$AAv?$AA?9?$AAL?$AAV@ 000000018005b5b0     libucrt:lcidtoname_downlevel.obj
 0002:000055c0       ??_C@_1M@IFGBIJO@?$AAl?$AAt?$AA?9?$AAL?$AAT@ 000000018005b5c0     libucrt:lcidtoname_downlevel.obj
 0002:000055d0       ??_C@_1M@FGEAHEDM@?$AAf?$AAa?$AA?9?$AAI?$AAR@ 000000018005b5d0     libucrt:lcidtoname_downlevel.obj
 0002:000055e0       ??_C@_1M@KBMAIBFN@?$AAv?$AAi?$AA?9?$AAV?$AAN@ 000000018005b5e0     libucrt:lcidtoname_downlevel.obj
 0002:000055f0       ??_C@_1M@GPCBKDJK@?$AAh?$AAy?$AA?9?$AAA?$AAM@ 000000018005b5f0     libucrt:lcidtoname_downlevel.obj
 0002:00005600       ??_C@_1BG@BECMDDJB@?$AAa?$AAz?$AA?9?$AAA?$AAZ?$AA?9?$AAL?$AAa?$AAt?$AAn@ 000000018005b600     libucrt:lcidtoname_downlevel.obj
 0002:00005618       ??_C@_1M@MAOFCAEA@?$AAe?$AAu?$AA?9?$AAE?$AAS@ 000000018005b618     libucrt:lcidtoname_downlevel.obj
 0002:00005628       ??_C@_1M@IGHABKPI@?$AAm?$AAk?$AA?9?$AAM?$AAK@ 000000018005b628     libucrt:lcidtoname_downlevel.obj
 0002:00005638       ??_C@_1M@IAIGNEJG@?$AAt?$AAn?$AA?9?$AAZ?$AAA@ 000000018005b638     libucrt:lcidtoname_downlevel.obj
 0002:00005648       ??_C@_1M@IIJCOJFA@?$AAx?$AAh?$AA?9?$AAZ?$AAA@ 000000018005b648     libucrt:lcidtoname_downlevel.obj
 0002:00005658       ??_C@_1M@LGPJHNJH@?$AAz?$AAu?$AA?9?$AAZ?$AAA@ 000000018005b658     libucrt:lcidtoname_downlevel.obj
 0002:00005668       ??_C@_1M@HOKAOIO@?$AAa?$AAf?$AA?9?$AAZ?$AAA@ 000000018005b668     libucrt:lcidtoname_downlevel.obj
 0002:00005678       ??_C@_1M@DPCLHLIE@?$AAk?$AAa?$AA?9?$AAG?$AAE@ 000000018005b678     libucrt:lcidtoname_downlevel.obj
 0002:00005688       ??_C@_1M@BLKMHJBI@?$AAf?$AAo?$AA?9?$AAF?$AAO@ 000000018005b688     libucrt:lcidtoname_downlevel.obj
 0002:00005698       ??_C@_1M@LGGJAPPB@?$AAh?$AAi?$AA?9?$AAI?$AAN@ 000000018005b698     libucrt:lcidtoname_downlevel.obj
 0002:000056a8       ??_C@_1M@FIKPIHFE@?$AAm?$AAt?$AA?9?$AAM?$AAT@ 000000018005b6a8     libucrt:lcidtoname_downlevel.obj
 0002:000056b8       ??_C@_1M@HEGGPBFA@?$AAs?$AAe?$AA?9?$AAN?$AAO@ 000000018005b6b8     libucrt:lcidtoname_downlevel.obj
 0002:000056c8       ??_C@_1M@EIBJEEPA@?$AAm?$AAs?$AA?9?$AAM?$AAY@ 000000018005b6c8     libucrt:lcidtoname_downlevel.obj
 0002:000056d8       ??_C@_1M@FHLBGMPP@?$AAk?$AAk?$AA?9?$AAK?$AAZ@ 000000018005b6d8     libucrt:lcidtoname_downlevel.obj
 0002:000056e8       ??_C@_1M@NGJJLCGI@?$AAk?$AAy?$AA?9?$AAK?$AAG@ 000000018005b6e8     libucrt:lcidtoname_downlevel.obj
 0002:000056f8       ??_C@_1M@GIENNBFC@?$AAs?$AAw?$AA?9?$AAK?$AAE@ 000000018005b6f8     libucrt:lcidtoname_downlevel.obj
 0002:00005708       ??_C@_1BG@NDGMJIMJ@?$AAu?$AAz?$AA?9?$AAU?$AAZ?$AA?9?$AAL?$AAa?$AAt?$AAn@ 000000018005b708     libucrt:lcidtoname_downlevel.obj
 0002:00005720       ??_C@_1M@IDCCIHBC@?$AAt?$AAt?$AA?9?$AAR?$AAU@ 000000018005b720     libucrt:lcidtoname_downlevel.obj
 0002:00005730       ??_C@_1M@LOICPMOJ@?$AAb?$AAn?$AA?9?$AAI?$AAN@ 000000018005b730     libucrt:lcidtoname_downlevel.obj
 0002:00005740       ??_C@_1M@KPKKNEAH@?$AAp?$AAa?$AA?9?$AAI?$AAN@ 000000018005b740     libucrt:lcidtoname_downlevel.obj
 0002:00005750       ??_C@_1M@PJGPPBOG@?$AAg?$AAu?$AA?9?$AAI?$AAN@ 000000018005b750     libucrt:lcidtoname_downlevel.obj
 0002:00005760       ??_C@_1M@KMKMOPHI@?$AAt?$AAa?$AA?9?$AAI?$AAN@ 000000018005b760     libucrt:lcidtoname_downlevel.obj
 0002:00005770       ??_C@_1M@KFEHEPAC@?$AAt?$AAe?$AA?9?$AAI?$AAN@ 000000018005b770     libucrt:lcidtoname_downlevel.obj
 0002:00005780       ??_C@_1M@CDCLMGHI@?$AAk?$AAn?$AA?9?$AAI?$AAN@ 000000018005b780     libucrt:lcidtoname_downlevel.obj
 0002:00005790       ??_C@_1M@MIODLDKF@?$AAm?$AAl?$AA?9?$AAI?$AAN@ 000000018005b790     libucrt:lcidtoname_downlevel.obj
 0002:000057a0       ??_C@_1M@PBIEACPO@?$AAm?$AAr?$AA?9?$AAI?$AAN@ 000000018005b7a0     libucrt:lcidtoname_downlevel.obj
 0002:000057b0       ??_C@_1M@NIDEAGPH@?$AAs?$AAa?$AA?9?$AAI?$AAN@ 000000018005b7b0     libucrt:lcidtoname_downlevel.obj
 0002:000057c0       ??_C@_1M@FHIHCBIO@?$AAm?$AAn?$AA?9?$AAM?$AAN@ 000000018005b7c0     libucrt:lcidtoname_downlevel.obj
 0002:000057d0       ??_C@_1M@JAIJPENP@?$AAc?$AAy?$AA?9?$AAG?$AAB@ 000000018005b7d0     libucrt:lcidtoname_downlevel.obj
 0002:000057e0       ??_C@_1M@PHGFBEPN@?$AAg?$AAl?$AA?9?$AAE?$AAS@ 000000018005b7e0     libucrt:lcidtoname_downlevel.obj
 0002:000057f0       ??_C@_1O@KPIPDNCP@?$AAk?$AAo?$AAk?$AA?9?$AAI?$AAN@ 000000018005b7f0     libucrt:lcidtoname_downlevel.obj
 0002:00005800       ??_C@_1O@KNHJLDJA@?$AAs?$AAy?$AAr?$AA?9?$AAS?$AAY@ 000000018005b800     libucrt:lcidtoname_downlevel.obj
 0002:00005810       ??_C@_1O@MKEKBLAH@?$AAd?$AAi?$AAv?$AA?9?$AAM?$AAV@ 000000018005b810     libucrt:lcidtoname_downlevel.obj
 0002:00005820       ??_C@_1O@OHDCKDDF@?$AAq?$AAu?$AAz?$AA?9?$AAB?$AAO@ 000000018005b820     libucrt:lcidtoname_downlevel.obj
 0002:00005830       ??_C@_1M@LEPJNLFD@?$AAn?$AAs?$AA?9?$AAZ?$AAA@ 000000018005b830     libucrt:lcidtoname_downlevel.obj
 0002:00005840       ??_C@_1M@OMLEIIJB@?$AAm?$AAi?$AA?9?$AAN?$AAZ@ 000000018005b840     libucrt:lcidtoname_downlevel.obj
 0002:00005850       ??_C@_1M@PMPEAILG@?$AAa?$AAr?$AA?9?$AAI?$AAQ@ 000000018005b850     libucrt:lcidtoname_downlevel.obj
 0002:00005860       ??_C@_1M@CNKPNOEE@?$AAd?$AAe?$AA?9?$AAC?$AAH@ 000000018005b860     libucrt:lcidtoname_downlevel.obj
 0002:00005870       ??_C@_1M@LKMGMLKO@?$AAe?$AAn?$AA?9?$AAG?$AAB@ 000000018005b870     libucrt:lcidtoname_downlevel.obj
 0002:00005880       ??_C@_1M@PGKJFFGL@?$AAe?$AAs?$AA?9?$AAM?$AAX@ 000000018005b880     libucrt:lcidtoname_downlevel.obj
 0002:00005890       ??_C@_1M@DNNANBDC@?$AAf?$AAr?$AA?9?$AAB?$AAE@ 000000018005b890     libucrt:lcidtoname_downlevel.obj
 0002:000058a0       ??_C@_1M@HLGMDFHM@?$AAi?$AAt?$AA?9?$AAC?$AAH@ 000000018005b8a0     libucrt:lcidtoname_downlevel.obj
 0002:000058b0       ??_C@_1M@CLLBGJH@?$AAn?$AAl?$AA?9?$AAB?$AAE@ 000000018005b8b0     libucrt:lcidtoname_downlevel.obj
 0002:000058c0       ??_C@_1M@BODBOGLF@?$AAn?$AAn?$AA?9?$AAN?$AAO@ 000000018005b8c0     libucrt:lcidtoname_downlevel.obj
 0002:000058d0       ??_C@_1M@HFFAHKAD@?$AAp?$AAt?$AA?9?$AAP?$AAT@ 000000018005b8d0     libucrt:lcidtoname_downlevel.obj
 0002:000058e0       ??_C@_1BG@LNOAKHIE@?$AAs?$AAr?$AA?9?$AAS?$AAP?$AA?9?$AAL?$AAa?$AAt?$AAn@ 000000018005b8e0     libucrt:lcidtoname_downlevel.obj
 0002:000058f8       ??_C@_1M@HBMHBGAK@?$AAs?$AAv?$AA?9?$AAF?$AAI@ 000000018005b8f8     libucrt:lcidtoname_downlevel.obj
 0002:00005908       ??_C@_1BG@DGCJGJBE@?$AAa?$AAz?$AA?9?$AAA?$AAZ?$AA?9?$AAC?$AAy?$AAr?$AAl@ 000000018005b908     libucrt:lcidtoname_downlevel.obj
 0002:00005920       ??_C@_1M@KEJDAAHB@?$AAs?$AAe?$AA?9?$AAS?$AAE@ 000000018005b920     libucrt:lcidtoname_downlevel.obj
 0002:00005930       ??_C@_1M@HEIBJJAD@?$AAm?$AAs?$AA?9?$AAB?$AAN@ 000000018005b930     libucrt:lcidtoname_downlevel.obj
 0002:00005940       ??_C@_1BG@PBGJMCEM@?$AAu?$AAz?$AA?9?$AAU?$AAZ?$AA?9?$AAC?$AAy?$AAr?$AAl@ 000000018005b940     libucrt:lcidtoname_downlevel.obj
 0002:00005958       ??_C@_1O@LAOBCMDF@?$AAq?$AAu?$AAz?$AA?9?$AAE?$AAC@ 000000018005b958     libucrt:lcidtoname_downlevel.obj
 0002:00005968       ??_C@_1M@POEEMAIO@?$AAa?$AAr?$AA?9?$AAE?$AAG@ 000000018005b968     libucrt:lcidtoname_downlevel.obj
 0002:00005978       ??_C@_1M@EFAKDEDL@?$AAz?$AAh?$AA?9?$AAH?$AAK@ 000000018005b978     libucrt:lcidtoname_downlevel.obj
 0002:00005988       ??_C@_1M@HKKIJHGI@?$AAd?$AAe?$AA?9?$AAA?$AAT@ 000000018005b988     libucrt:lcidtoname_downlevel.obj
 0002:00005998       ??_C@_1M@KBFBEHJF@?$AAe?$AAn?$AA?9?$AAA?$AAU@ 000000018005b998     libucrt:lcidtoname_downlevel.obj
 0002:000059a8       ??_C@_1M@MNPLFAAH@?$AAe?$AAs?$AA?9?$AAE?$AAS@ 000000018005b9a8     libucrt:lcidtoname_downlevel.obj
 0002:000059b8       ??_C@_1M@HJOOJFMA@?$AAf?$AAr?$AA?9?$AAC?$AAA@ 000000018005b9b8     libucrt:lcidtoname_downlevel.obj
 0002:000059c8       ??_C@_1BG@JPOFPNAB@?$AAs?$AAr?$AA?9?$AAS?$AAP?$AA?9?$AAC?$AAy?$AAr?$AAl@ 000000018005b9c8     libucrt:lcidtoname_downlevel.obj
 0002:000059e0       ??_C@_1M@LNFOCMOB@?$AAs?$AAe?$AA?9?$AAF?$AAI@ 000000018005b9e0     libucrt:lcidtoname_downlevel.obj
 0002:000059f0       ??_C@_1O@MGJBOAMB@?$AAq?$AAu?$AAz?$AA?9?$AAP?$AAE@ 000000018005b9f0     libucrt:lcidtoname_downlevel.obj
 0002:00005a00       ??_C@_1M@GJINLBOK@?$AAa?$AAr?$AA?9?$AAL?$AAY@ 000000018005ba00     libucrt:lcidtoname_downlevel.obj
 0002:00005a10       ??_C@_1M@GGMNHJNL@?$AAz?$AAh?$AA?9?$AAS?$AAG@ 000000018005ba10     libucrt:lcidtoname_downlevel.obj
 0002:00005a20       ??_C@_1M@HOIKODND@?$AAd?$AAe?$AA?9?$AAL?$AAU@ 000000018005ba20     libucrt:lcidtoname_downlevel.obj
 0002:00005a30       ??_C@_1M@DDOCCGFG@?$AAe?$AAn?$AA?9?$AAC?$AAA@ 000000018005ba30     libucrt:lcidtoname_downlevel.obj
 0002:00005a40       ??_C@_1M@BNOEMJLF@?$AAe?$AAs?$AA?9?$AAG?$AAT@ 000000018005ba40     libucrt:lcidtoname_downlevel.obj
 0002:00005a50       ??_C@_1M@EOGNKEK@?$AAf?$AAr?$AA?9?$AAC?$AAH@ 000000018005ba50     libucrt:lcidtoname_downlevel.obj
 0002:00005a60       ??_C@_1M@FLIDJFHL@?$AAh?$AAr?$AA?9?$AAB?$AAA@ 000000018005ba60     libucrt:lcidtoname_downlevel.obj
 0002:00005a70       ??_C@_1O@FMCELNAJ@?$AAs?$AAm?$AAj?$AA?9?$AAN?$AAO@ 000000018005ba70     libucrt:lcidtoname_downlevel.obj
 0002:00005a80       ??_C@_1M@JHGLJMGJ@?$AAa?$AAr?$AA?9?$AAD?$AAZ@ 000000018005ba80     libucrt:lcidtoname_downlevel.obj
 0002:00005a90       ??_C@_1M@JKKFDCNP@?$AAz?$AAh?$AA?9?$AAM?$AAO@ 000000018005ba90     libucrt:lcidtoname_downlevel.obj
 0002:00005aa0       ??_C@_1M@GEEFALPE@?$AAd?$AAe?$AA?9?$AAL?$AAI@ 000000018005baa0     libucrt:lcidtoname_downlevel.obj
 0002:00005ab0       ??_C@_1M@IGEOFBG@?$AAe?$AAn?$AA?9?$AAN?$AAZ@ 000000018005bab0     libucrt:lcidtoname_downlevel.obj
 0002:00005ac0       ??_C@_1M@KDBONEHP@?$AAe?$AAs?$AA?9?$AAC?$AAR@ 000000018005bac0     libucrt:lcidtoname_downlevel.obj
 0002:00005ad0       ??_C@_1M@FHMDOHNN@?$AAf?$AAr?$AA?9?$AAL?$AAU@ 000000018005bad0     libucrt:lcidtoname_downlevel.obj
 0002:00005ae0       ??_C@_1BG@NFKKMAFG@?$AAb?$AAs?$AA?9?$AAB?$AAA?$AA?9?$AAL?$AAa?$AAt?$AAn@ 000000018005bae0     libucrt:lcidtoname_downlevel.obj
 0002:00005af8       ??_C@_1O@IMNBEMCI@?$AAs?$AAm?$AAj?$AA?9?$AAS?$AAE@ 000000018005baf8     libucrt:lcidtoname_downlevel.obj
 0002:00005b08       ??_C@_1M@DHHMBNDP@?$AAa?$AAr?$AA?9?$AAM?$AAA@ 000000018005bb08     libucrt:lcidtoname_downlevel.obj
 0002:00005b18       ??_C@_1M@BNBLJCGH@?$AAe?$AAn?$AA?9?$AAI?$AAE@ 000000018005bb18     libucrt:lcidtoname_downlevel.obj
 0002:00005b28       ??_C@_1M@GEPAFMDL@?$AAe?$AAs?$AA?9?$AAP?$AAA@ 000000018005bb28     libucrt:lcidtoname_downlevel.obj
 0002:00005b38       ??_C@_1M@OJONDMDL@?$AAf?$AAr?$AA?9?$AAM?$AAC@ 000000018005bb38     libucrt:lcidtoname_downlevel.obj
 0002:00005b48       ??_C@_1BG@OBCNFJB@?$AAs?$AAr?$AA?9?$AAB?$AAA?$AA?9?$AAL?$AAa?$AAt?$AAn@ 000000018005bb48     libucrt:lcidtoname_downlevel.obj
 0002:00005b60       ??_C@_1O@KEMEEGPO@?$AAs?$AAm?$AAa?$AA?9?$AAN?$AAO@ 000000018005bb60     libucrt:lcidtoname_downlevel.obj
 0002:00005b70       ??_C@_1M@ELMGFODK@?$AAa?$AAr?$AA?9?$AAT?$AAN@ 000000018005bb70     libucrt:lcidtoname_downlevel.obj
 0002:00005b80       ??_C@_1M@BHDLHFAF@?$AAe?$AAn?$AA?9?$AAZ?$AAA@ 000000018005bb80     libucrt:lcidtoname_downlevel.obj
 0002:00005b90       ??_C@_1M@BMGIGLIF@?$AAe?$AAs?$AA?9?$AAD?$AAO@ 000000018005bb90     libucrt:lcidtoname_downlevel.obj
 0002:00005ba0       ??_C@_1BG@CMBHIPBE@?$AAs?$AAr?$AA?9?$AAB?$AAA?$AA?9?$AAC?$AAy?$AAr?$AAl@ 000000018005bba0     libucrt:lcidtoname_downlevel.obj
 0002:00005bb8       ??_C@_1O@HEDBLHNP@?$AAs?$AAm?$AAa?$AA?9?$AAS?$AAE@ 000000018005bbb8     libucrt:lcidtoname_downlevel.obj
 0002:00005bc8       ??_C@_1M@DAGCADIM@?$AAa?$AAr?$AA?9?$AAO?$AAM@ 000000018005bbc8     libucrt:lcidtoname_downlevel.obj
 0002:00005bd8       ??_C@_1M@FODLMICG@?$AAe?$AAn?$AA?9?$AAJ?$AAM@ 000000018005bbd8     libucrt:lcidtoname_downlevel.obj
 0002:00005be8       ??_C@_1M@DNMLCIHB@?$AAe?$AAs?$AA?9?$AAV?$AAE@ 000000018005bbe8     libucrt:lcidtoname_downlevel.obj
 0002:00005bf8       ??_C@_1O@EOKHMKJK@?$AAs?$AAm?$AAs?$AA?9?$AAF?$AAI@ 000000018005bbf8     libucrt:lcidtoname_downlevel.obj
 0002:00005c08       ??_C@_1M@CAFJMKOF@?$AAa?$AAr?$AA?9?$AAY?$AAE@ 000000018005bc08     libucrt:lcidtoname_downlevel.obj
 0002:00005c18       ??_C@_1M@CBFHIJLI@?$AAe?$AAn?$AA?9?$AAC?$AAB@ 000000018005bc18     libucrt:lcidtoname_downlevel.obj
 0002:00005c28       ??_C@_1M@BGNFLDN@?$AAe?$AAs?$AA?9?$AAC?$AAO@ 000000018005bc28     libucrt:lcidtoname_downlevel.obj
 0002:00005c38       ??_C@_1O@JMPHMAMC@?$AAs?$AAm?$AAn?$AA?9?$AAF?$AAI@ 000000018005bc38     libucrt:lcidtoname_downlevel.obj
 0002:00005c48       ??_C@_1M@JLANABKE@?$AAa?$AAr?$AA?9?$AAS?$AAY@ 000000018005bc48     libucrt:lcidtoname_downlevel.obj
 0002:00005c58       ??_C@_1M@HPKGCFGN@?$AAe?$AAn?$AA?9?$AAB?$AAZ@ 000000018005bc58     libucrt:lcidtoname_downlevel.obj
 0002:00005c68       ??_C@_1M@OLJCMLGM@?$AAe?$AAs?$AA?9?$AAP?$AAE@ 000000018005bc68     libucrt:lcidtoname_downlevel.obj
 0002:00005c78       ??_C@_1M@MKKGFKLE@?$AAa?$AAr?$AA?9?$AAJ?$AAO@ 000000018005bc78     libucrt:lcidtoname_downlevel.obj
 0002:00005c88       ??_C@_1M@EKPGLDNI@?$AAe?$AAn?$AA?9?$AAT?$AAT@ 000000018005bc88     libucrt:lcidtoname_downlevel.obj
 0002:00005c98       ??_C@_1M@OONGHFHE@?$AAe?$AAs?$AA?9?$AAA?$AAR@ 000000018005bc98     libucrt:lcidtoname_downlevel.obj
 0002:00005ca8       ??_C@_1M@OOJFGBHE@?$AAa?$AAr?$AA?9?$AAL?$AAB@ 000000018005bca8     libucrt:lcidtoname_downlevel.obj
 0002:00005cb8       ??_C@_1M@GCEJHNEG@?$AAe?$AAn?$AA?9?$AAZ?$AAW@ 000000018005bcb8     libucrt:lcidtoname_downlevel.obj
 0002:00005cc8       ??_C@_1M@JNOCAHJI@?$AAe?$AAs?$AA?9?$AAE?$AAC@ 000000018005bcc8     libucrt:lcidtoname_downlevel.obj
 0002:00005cd8       ??_C@_1M@JEFHPGGB@?$AAa?$AAr?$AA?9?$AAK?$AAW@ 000000018005bcd8     libucrt:lcidtoname_downlevel.obj
 0002:00005ce8       ??_C@_1M@MLKIBJOJ@?$AAe?$AAn?$AA?9?$AAP?$AAH@ 000000018005bce8     libucrt:lcidtoname_downlevel.obj
 0002:00005cf8       ??_C@_1M@BDNIPEND@?$AAe?$AAs?$AA?9?$AAC?$AAL@ 000000018005bcf8     libucrt:lcidtoname_downlevel.obj
 0002:00005d08       ??_C@_1M@MPNMEKBD@?$AAa?$AAr?$AA?9?$AAA?$AAE@ 000000018005bd08     libucrt:lcidtoname_downlevel.obj
 0002:00005d18       ??_C@_1M@KBJALCPI@?$AAe?$AAs?$AA?9?$AAU?$AAY@ 000000018005bd18     libucrt:lcidtoname_downlevel.obj
 0002:00005d28       ??_C@_1M@LLCCOAGA@?$AAa?$AAr?$AA?9?$AAB?$AAH@ 000000018005bd28     libucrt:lcidtoname_downlevel.obj
 0002:00005d38       ??_C@_1M@PBFNCDEL@?$AAe?$AAs?$AA?9?$AAP?$AAY@ 000000018005bd38     libucrt:lcidtoname_downlevel.obj
 0002:00005d48       ??_C@_1M@EDGINPNP@?$AAa?$AAr?$AA?9?$AAQ?$AAA@ 000000018005bd48     libucrt:lcidtoname_downlevel.obj
 0002:00005d58       ??_C@_1M@MKDBIIJI@?$AAe?$AAs?$AA?9?$AAB?$AAO@ 000000018005bd58     libucrt:lcidtoname_downlevel.obj
 0002:00005d68       ??_C@_1M@CPKKEBLD@?$AAe?$AAs?$AA?9?$AAS?$AAV@ 000000018005bd68     libucrt:lcidtoname_downlevel.obj
 0002:00005d78       ??_C@_1M@NDBGMMJL@?$AAe?$AAs?$AA?9?$AAH?$AAN@ 000000018005bd78     libucrt:lcidtoname_downlevel.obj
 0002:00005d88       ??_C@_1M@JIJIBHDP@?$AAe?$AAs?$AA?9?$AAN?$AAI@ 000000018005bd88     libucrt:lcidtoname_downlevel.obj
 0002:00005d98       ??_C@_1M@CGFMKEEK@?$AAe?$AAs?$AA?9?$AAP?$AAR@ 000000018005bd98     libucrt:lcidtoname_downlevel.obj
 0002:00005da8       ??_C@_1O@ICJHKIIK@?$AAz?$AAh?$AA?9?$AAC?$AAH?$AAT@ 000000018005bda8     libucrt:lcidtoname_downlevel.obj
 0002:00005db8       ??_C@_15CLNEJCE@?$AAs?$AAr@ 000000018005bdb8     libucrt:lcidtoname_downlevel.obj
 0002:00006c00       ??_C@_1M@KAHEKEIG@?$AAa?$AAf?$AA?9?$AAz?$AAa@ 000000018005cc00     libucrt:lcidtoname_downlevel.obj
 0002:00006c10       ??_C@_1M@GIECOABL@?$AAa?$AAr?$AA?9?$AAa?$AAe@ 000000018005cc10     libucrt:lcidtoname_downlevel.obj
 0002:00006c20       ??_C@_1M@BMLMEKGI@?$AAa?$AAr?$AA?9?$AAb?$AAh@ 000000018005cc20     libucrt:lcidtoname_downlevel.obj
 0002:00006c30       ??_C@_1M@DAPFDGGB@?$AAa?$AAr?$AA?9?$AAd?$AAz@ 000000018005cc30     libucrt:lcidtoname_downlevel.obj
 0002:00006c40       ??_C@_1M@FJNKGKIG@?$AAa?$AAr?$AA?9?$AAe?$AAg@ 000000018005cc40     libucrt:lcidtoname_downlevel.obj
 0002:00006c50       ??_C@_1M@FLGKKCLO@?$AAa?$AAr?$AA?9?$AAi?$AAq@ 000000018005cc50     libucrt:lcidtoname_downlevel.obj
 0002:00006c60       ??_C@_1M@GNDIPALM@?$AAa?$AAr?$AA?9?$AAj?$AAo@ 000000018005cc60     libucrt:lcidtoname_downlevel.obj
 0002:00006c70       ??_C@_1M@DDMJFMGJ@?$AAa?$AAr?$AA?9?$AAk?$AAw@ 000000018005cc70     libucrt:lcidtoname_downlevel.obj
 0002:00006c80       ??_C@_1M@EJALMLHM@?$AAa?$AAr?$AA?9?$AAl?$AAb@ 000000018005cc80     libucrt:lcidtoname_downlevel.obj
 0002:00006c90       ??_C@_1M@MOBDBLOC@?$AAa?$AAr?$AA?9?$AAl?$AAy@ 000000018005cc90     libucrt:lcidtoname_downlevel.obj
 0002:00006ca0       ??_C@_1M@JAOCLHDH@?$AAa?$AAr?$AA?9?$AAm?$AAa@ 000000018005cca0     libucrt:lcidtoname_downlevel.obj
 0002:00006cb0       ??_C@_1M@JHPMKJIE@?$AAa?$AAr?$AA?9?$AAo?$AAm@ 000000018005ccb0     libucrt:lcidtoname_downlevel.obj
 0002:00006cc0       ??_C@_1M@OEPGHFNH@?$AAa?$AAr?$AA?9?$AAq?$AAa@ 000000018005ccc0     libucrt:lcidtoname_downlevel.obj
 0002:00006cd0       ??_C@_1M@KJDONENM@?$AAa?$AAr?$AA?9?$AAs?$AAa@ 000000018005ccd0     libucrt:lcidtoname_downlevel.obj
 0002:00006ce0       ??_C@_1M@DMJDKLKM@?$AAa?$AAr?$AA?9?$AAs?$AAy@ 000000018005cce0     libucrt:lcidtoname_downlevel.obj
 0002:00006cf0       ??_C@_1M@OMFIPEDC@?$AAa?$AAr?$AA?9?$AAt?$AAn@ 000000018005ccf0     libucrt:lcidtoname_downlevel.obj
 0002:00006d00       ??_C@_1M@IHMHGAON@?$AAa?$AAr?$AA?9?$AAy?$AAe@ 000000018005cd00     libucrt:lcidtoname_downlevel.obj
 0002:00006d10       ??_C@_1BG@KDCPGJGB@?$AAa?$AAz?$AA?9?$AAa?$AAz?$AA?9?$AAc?$AAy?$AAr?$AAl@ 000000018005cd10     libucrt:lcidtoname_downlevel.obj
 0002:00006d28       ??_C@_1BG@IBCKDDOE@?$AAa?$AAz?$AA?9?$AAa?$AAz?$AA?9?$AAl?$AAa?$AAt?$AAn@ 000000018005cd28     libucrt:lcidtoname_downlevel.obj
 0002:00006d40       ??_C@_1M@EGPFDCPD@?$AAb?$AAe?$AA?9?$AAb?$AAy@ 000000018005cd40     libucrt:lcidtoname_downlevel.obj
 0002:00006d50       ??_C@_1M@PCMGMCGC@?$AAb?$AAg?$AA?9?$AAb?$AAg@ 000000018005cd50     libucrt:lcidtoname_downlevel.obj
 0002:00006d60       ??_C@_1M@BJBMFGOB@?$AAb?$AAn?$AA?9?$AAi?$AAn@ 000000018005cd60     libucrt:lcidtoname_downlevel.obj
 0002:00006d70       ??_C@_1BG@EAKMMACD@?$AAb?$AAs?$AA?9?$AAb?$AAa?$AA?9?$AAl?$AAa?$AAt?$AAn@ 000000018005cd70     libucrt:lcidtoname_downlevel.obj
 0002:00006d88       ??_C@_1M@KGADAODK@?$AAc?$AAa?$AA?9?$AAe?$AAs@ 000000018005cd88     libucrt:lcidtoname_downlevel.obj
 0002:00006d98       ??_C@_1M@COAJPDHI@?$AAc?$AAs?$AA?9?$AAc?$AAz@ 000000018005cd98     libucrt:lcidtoname_downlevel.obj
 0002:00006da8       ??_C@_1M@DHBHFONH@?$AAc?$AAy?$AA?9?$AAg?$AAb@ 000000018005cda8     libucrt:lcidtoname_downlevel.obj
 0002:00006db8       ??_C@_1M@IMGKELGA@?$AAd?$AAa?$AA?9?$AAd?$AAk@ 000000018005cdb8     libucrt:lcidtoname_downlevel.obj
 0002:00006dc8       ??_C@_1M@NNDGDNGA@?$AAd?$AAe?$AA?9?$AAa?$AAt@ 000000018005cdc8     libucrt:lcidtoname_downlevel.obj
 0002:00006dd8       ??_C@_1M@IKDBHEEM@?$AAd?$AAe?$AA?9?$AAc?$AAh@ 000000018005cdd8     libucrt:lcidtoname_downlevel.obj
 0002:00006de8       ??_C@_1M@GFFOJMCJ@?$AAd?$AAe?$AA?9?$AAd?$AAe@ 000000018005cde8     libucrt:lcidtoname_downlevel.obj
 0002:00006df8       ??_C@_1M@MDNLKBPM@?$AAd?$AAe?$AA?9?$AAl?$AAi@ 000000018005cdf8     libucrt:lcidtoname_downlevel.obj
 0002:00006e08       ??_C@_1M@NJBEEJNL@?$AAd?$AAe?$AA?9?$AAl?$AAu@ 000000018005ce08     libucrt:lcidtoname_downlevel.obj
 0002:00006e18       ??_C@_1O@GNNELBAP@?$AAd?$AAi?$AAv?$AA?9?$AAm?$AAv@ 000000018005ce18     libucrt:lcidtoname_downlevel.obj
 0002:00006e28       ??_C@_1M@EJLEOGAE@?$AAe?$AAl?$AA?9?$AAg?$AAr@ 000000018005ce28     libucrt:lcidtoname_downlevel.obj
 0002:00006e38       ??_C@_1M@GMPONJN@?$AAe?$AAn?$AA?9?$AAa?$AAu@ 000000018005ce38     libucrt:lcidtoname_downlevel.obj
 0002:00006e48       ??_C@_1M@NIDIIPGF@?$AAe?$AAn?$AA?9?$AAb?$AAz@ 000000018005ce48     libucrt:lcidtoname_downlevel.obj
 0002:00006e58       ??_C@_1M@JEHMIMFO@?$AAe?$AAn?$AA?9?$AAc?$AAa@ 000000018005ce58     libucrt:lcidtoname_downlevel.obj
 0002:00006e68       ??_C@_1M@IGMJCDLA@?$AAe?$AAn?$AA?9?$AAc?$AAb@ 000000018005ce68     libucrt:lcidtoname_downlevel.obj
 0002:00006e78       ??_C@_1M@BNFIGBKG@?$AAe?$AAn?$AA?9?$AAg?$AAb@ 000000018005ce78     libucrt:lcidtoname_downlevel.obj
 0002:00006e88       ??_C@_1M@LKIFDIGP@?$AAe?$AAn?$AA?9?$AAi?$AAe@ 000000018005ce88     libucrt:lcidtoname_downlevel.obj
 0002:00006e98       ??_C@_1M@PJKFGCCO@?$AAe?$AAn?$AA?9?$AAj?$AAm@ 000000018005ce98     libucrt:lcidtoname_downlevel.obj
 0002:00006ea8       ??_C@_1M@KPPKEPBO@?$AAe?$AAn?$AA?9?$AAn?$AAz@ 000000018005cea8     libucrt:lcidtoname_downlevel.obj
 0002:00006eb8       ??_C@_1M@GMDGLDOB@?$AAe?$AAn?$AA?9?$AAp?$AAh@ 000000018005ceb8     libucrt:lcidtoname_downlevel.obj
 0002:00006ec8       ??_C@_1M@ONGIBJNA@?$AAe?$AAn?$AA?9?$AAt?$AAt@ 000000018005cec8     libucrt:lcidtoname_downlevel.obj
 0002:00006ed8       ??_C@_1M@LLODPCMM@?$AAe?$AAn?$AA?9?$AAu?$AAs@ 000000018005ced8     libucrt:lcidtoname_downlevel.obj
 0002:00006ee8       ??_C@_1M@LAKFNPAN@?$AAe?$AAn?$AA?9?$AAz?$AAa@ 000000018005cee8     libucrt:lcidtoname_downlevel.obj
 0002:00006ef8       ??_C@_1M@MFNHNHEO@?$AAe?$AAn?$AA?9?$AAz?$AAw@ 000000018005cef8     libucrt:lcidtoname_downlevel.obj
 0002:00006f08       ??_C@_1M@EJEINPHM@?$AAe?$AAs?$AA?9?$AAa?$AAr@ 000000018005cf08     libucrt:lcidtoname_downlevel.obj
 0002:00006f18       ??_C@_1M@GNKPCCJA@?$AAe?$AAs?$AA?9?$AAb?$AAo@ 000000018005cf18     libucrt:lcidtoname_downlevel.obj
 0002:00006f28       ??_C@_1M@LEEGFONL@?$AAe?$AAs?$AA?9?$AAc?$AAl@ 000000018005cf28     libucrt:lcidtoname_downlevel.obj
 0002:00006f38       ??_C@_1M@KGPDPBDF@?$AAe?$AAs?$AA?9?$AAc?$AAo@ 000000018005cf38     libucrt:lcidtoname_downlevel.obj
 0002:00006f48       ??_C@_1M@EIAHOHH@?$AAe?$AAs?$AA?9?$AAc?$AAr@ 000000018005cf48     libucrt:lcidtoname_downlevel.obj
 0002:00006f58       ??_C@_1M@LLPGMBIN@?$AAe?$AAs?$AA?9?$AAd?$AAo@ 000000018005cf58     libucrt:lcidtoname_downlevel.obj
 0002:00006f68       ??_C@_1M@DKHMKNJA@?$AAe?$AAs?$AA?9?$AAe?$AAc@ 000000018005cf68     libucrt:lcidtoname_downlevel.obj
 0002:00006f78       ??_C@_1M@GKGFPKAP@?$AAe?$AAs?$AA?9?$AAe?$AAs@ 000000018005cf78     libucrt:lcidtoname_downlevel.obj
 0002:00006f88       ??_C@_1M@LKHKGDLN@?$AAe?$AAs?$AA?9?$AAg?$AAt@ 000000018005cf88     libucrt:lcidtoname_downlevel.obj
 0002:00006f98       ??_C@_1M@HEIIGGJD@?$AAe?$AAs?$AA?9?$AAh?$AAn@ 000000018005cf98     libucrt:lcidtoname_downlevel.obj
 0002:00006fa8       ??_C@_1M@FBDHPPGD@?$AAe?$AAs?$AA?9?$AAm?$AAx@ 000000018005cfa8     libucrt:lcidtoname_downlevel.obj
 0002:00006fb8       ??_C@_1M@DPAGLNDH@?$AAe?$AAs?$AA?9?$AAn?$AAi@ 000000018005cfb8     libucrt:lcidtoname_downlevel.obj
 0002:00006fc8       ??_C@_1M@MDGOPGDD@?$AAe?$AAs?$AA?9?$AAp?$AAa@ 000000018005cfc8     libucrt:lcidtoname_downlevel.obj
 0002:00006fd8       ??_C@_1M@EMAMGBGE@?$AAe?$AAs?$AA?9?$AAp?$AAe@ 000000018005cfd8     libucrt:lcidtoname_downlevel.obj
 0002:00006fe8       ??_C@_1M@IBMCAOEC@?$AAe?$AAs?$AA?9?$AAp?$AAr@ 000000018005cfe8     libucrt:lcidtoname_downlevel.obj
 0002:00006ff8       ??_C@_1M@FGMDIJED@?$AAe?$AAs?$AA?9?$AAp?$AAy@ 000000018005cff8     libucrt:lcidtoname_downlevel.obj
 0002:00007008       ??_C@_1M@IIDEOLLL@?$AAe?$AAs?$AA?9?$AAs?$AAv@ 000000018005d008     libucrt:lcidtoname_downlevel.obj
 0002:00007018       ??_C@_1M@GAOBIPA@?$AAe?$AAs?$AA?9?$AAu?$AAy@ 000000018005d018     libucrt:lcidtoname_downlevel.obj
 0002:00007028       ??_C@_1M@JKFFICHJ@?$AAe?$AAs?$AA?9?$AAv?$AAe@ 000000018005d028     libucrt:lcidtoname_downlevel.obj
 0002:00007038       ??_C@_1M@PNMLOJDF@?$AAe?$AAt?$AA?9?$AAe?$AAe@ 000000018005d038     libucrt:lcidtoname_downlevel.obj
 0002:00007048       ??_C@_1M@GHHLIKEI@?$AAe?$AAu?$AA?9?$AAe?$AAs@ 000000018005d048     libucrt:lcidtoname_downlevel.obj
 0002:00007058       ??_C@_1M@PBNONODE@?$AAf?$AAa?$AA?9?$AAi?$AAr@ 000000018005d058     libucrt:lcidtoname_downlevel.obj
 0002:00007068       ??_C@_1M@JEEHPMIL@?$AAf?$AAi?$AA?9?$AAf?$AAi@ 000000018005d068     libucrt:lcidtoname_downlevel.obj
 0002:00007078       ??_C@_1M@LMDCNDBA@?$AAf?$AAo?$AA?9?$AAf?$AAo@ 000000018005d078     libucrt:lcidtoname_downlevel.obj
 0002:00007088       ??_C@_1M@JKEOHLDK@?$AAf?$AAr?$AA?9?$AAb?$AAe@ 000000018005d088     libucrt:lcidtoname_downlevel.obj
 0002:00007098       ??_C@_1M@NOHADPMI@?$AAf?$AAr?$AA?9?$AAc?$AAa@ 000000018005d098     libucrt:lcidtoname_downlevel.obj
 0002:000070a8       ??_C@_1M@KDHIHAEC@?$AAf?$AAr?$AA?9?$AAc?$AAh@ 000000018005d0a8     libucrt:lcidtoname_downlevel.obj
 0002:000070b8       ??_C@_1M@MMBBFGAK@?$AAf?$AAr?$AA?9?$AAf?$AAr@ 000000018005d0b8     libucrt:lcidtoname_downlevel.obj
 0002:000070c8       ??_C@_1M@PAFNENNF@?$AAf?$AAr?$AA?9?$AAl?$AAu@ 000000018005d0c8     libucrt:lcidtoname_downlevel.obj
 0002:000070d8       ??_C@_1M@EOHDJGDD@?$AAf?$AAr?$AA?9?$AAm?$AAc@ 000000018005d0d8     libucrt:lcidtoname_downlevel.obj
 0002:000070e8       ??_C@_1M@FAPLLOPF@?$AAg?$AAl?$AA?9?$AAe?$AAs@ 000000018005d0e8     libucrt:lcidtoname_downlevel.obj
 0002:000070f8       ??_C@_1M@FOPBFLOO@?$AAg?$AAu?$AA?9?$AAi?$AAn@ 000000018005d0f8     libucrt:lcidtoname_downlevel.obj
 0002:00007108       ??_C@_1M@KBMCINPM@?$AAh?$AAe?$AA?9?$AAi?$AAl@ 000000018005d108     libucrt:lcidtoname_downlevel.obj
 0002:00007118       ??_C@_1M@BBPHKFPJ@?$AAh?$AAi?$AA?9?$AAi?$AAn@ 000000018005d118     libucrt:lcidtoname_downlevel.obj
 0002:00007128       ??_C@_1M@PMBNDPHD@?$AAh?$AAr?$AA?9?$AAb?$AAa@ 000000018005d128     libucrt:lcidtoname_downlevel.obj
 0002:00007138       ??_C@_1M@BPCKOEGE@?$AAh?$AAr?$AA?9?$AAh?$AAr@ 000000018005d138     libucrt:lcidtoname_downlevel.obj
 0002:00007148       ??_C@_1M@GACBMHKE@?$AAh?$AAu?$AA?9?$AAh?$AAu@ 000000018005d148     libucrt:lcidtoname_downlevel.obj
 0002:00007158       ??_C@_1M@MILPAJJC@?$AAh?$AAy?$AA?9?$AAa?$AAm@ 000000018005d158     libucrt:lcidtoname_downlevel.obj
 0002:00007168       ??_C@_1M@BABBICEC@?$AAi?$AAd?$AA?9?$AAi?$AAd@ 000000018005d168     libucrt:lcidtoname_downlevel.obj
 0002:00007178       ??_C@_1M@BIKNHHPF@?$AAi?$AAs?$AA?9?$AAi?$AAs@ 000000018005d178     libucrt:lcidtoname_downlevel.obj
 0002:00007188       ??_C@_1M@NMPCJPHE@?$AAi?$AAt?$AA?9?$AAc?$AAh@ 000000018005d188     libucrt:lcidtoname_downlevel.obj
 0002:00007198       ??_C@_1M@GHKGFEDF@?$AAi?$AAt?$AA?9?$AAi?$AAt@ 000000018005d198     libucrt:lcidtoname_downlevel.obj
 0002:000071a8       ??_C@_1M@NIEJCJJA@?$AAj?$AAa?$AA?9?$AAj?$AAp@ 000000018005d1a8     libucrt:lcidtoname_downlevel.obj
 0002:000071b8       ??_C@_1M@JILFNBIM@?$AAk?$AAa?$AA?9?$AAg?$AAe@ 000000018005d1b8     libucrt:lcidtoname_downlevel.obj
 0002:000071c8       ??_C@_1M@PACPMGPH@?$AAk?$AAk?$AA?9?$AAk?$AAz@ 000000018005d1c8     libucrt:lcidtoname_downlevel.obj
 0002:000071d8       ??_C@_1M@IELFGMHA@?$AAk?$AAn?$AA?9?$AAi?$AAn@ 000000018005d1d8     libucrt:lcidtoname_downlevel.obj
 0002:000071e8       ??_C@_1O@IBBJHCH@?$AAk?$AAo?$AAk?$AA?9?$AAi?$AAn@ 000000018005d1e8     libucrt:lcidtoname_downlevel.obj
 0002:000071f8       ??_C@_1M@DMHAEOGC@?$AAk?$AAo?$AA?9?$AAk?$AAr@ 000000018005d1f8     libucrt:lcidtoname_downlevel.obj
 0002:00007208       ??_C@_1M@HBAHBIGA@?$AAk?$AAy?$AA?9?$AAk?$AAg@ 000000018005d208     libucrt:lcidtoname_downlevel.obj
 0002:00007218       ??_C@_1M@KPMILCJG@?$AAl?$AAt?$AA?9?$AAl?$AAt@ 000000018005d218     libucrt:lcidtoname_downlevel.obj
 0002:00007228       ??_C@_1M@BDEKKCA@?$AAl?$AAv?$AA?9?$AAl?$AAv@ 000000018005d228     libucrt:lcidtoname_downlevel.obj
 0002:00007238       ??_C@_1M@ELCKCCJJ@?$AAm?$AAi?$AA?9?$AAn?$AAz@ 000000018005d238     libucrt:lcidtoname_downlevel.obj
 0002:00007248       ??_C@_1M@CBOOLAPA@?$AAm?$AAk?$AA?9?$AAm?$AAk@ 000000018005d248     libucrt:lcidtoname_downlevel.obj
 0002:00007258       ??_C@_1M@GPHNBJKN@?$AAm?$AAl?$AA?9?$AAi?$AAn@ 000000018005d258     libucrt:lcidtoname_downlevel.obj
 0002:00007268       ??_C@_1M@PABJILIG@?$AAm?$AAn?$AA?9?$AAm?$AAn@ 000000018005d268     libucrt:lcidtoname_downlevel.obj
 0002:00007278       ??_C@_1M@FGBKKIPG@?$AAm?$AAr?$AA?9?$AAi?$AAn@ 000000018005d278     libucrt:lcidtoname_downlevel.obj
 0002:00007288       ??_C@_1M@NDBPDDAL@?$AAm?$AAs?$AA?9?$AAb?$AAn@ 000000018005d288     libucrt:lcidtoname_downlevel.obj
 0002:00007298       ??_C@_1M@OPIHOOPI@?$AAm?$AAs?$AA?9?$AAm?$AAy@ 000000018005d298     libucrt:lcidtoname_downlevel.obj
 0002:000072a8       ??_C@_1M@PPDBCNFM@?$AAm?$AAt?$AA?9?$AAm?$AAt@ 000000018005d2a8     libucrt:lcidtoname_downlevel.obj
 0002:000072b8       ??_C@_1M@KDJDKMDD@?$AAn?$AAb?$AA?9?$AAn?$AAo@ 000000018005d2b8     libucrt:lcidtoname_downlevel.obj
 0002:000072c8       ??_C@_1M@KFCFLMJP@?$AAn?$AAl?$AA?9?$AAb?$AAe@ 000000018005d2c8     libucrt:lcidtoname_downlevel.obj
 0002:000072d8       ??_C@_1M@KPOPDDGO@?$AAn?$AAl?$AA?9?$AAn?$AAl@ 000000018005d2d8     libucrt:lcidtoname_downlevel.obj
 0002:000072e8       ??_C@_1M@LJKPEMLN@?$AAn?$AAn?$AA?9?$AAn?$AAo@ 000000018005d2e8     libucrt:lcidtoname_downlevel.obj
 0002:000072f8       ??_C@_1M@BDGHHBFL@?$AAn?$AAs?$AA?9?$AAz?$AAa@ 000000018005d2f8     libucrt:lcidtoname_downlevel.obj
 0002:00007308       ??_C@_1M@IDEHOAP@?$AAp?$AAa?$AA?9?$AAi?$AAn@ 000000018005d308     libucrt:lcidtoname_downlevel.obj
 0002:00007318       ??_C@_1M@HDBKGOGH@?$AAp?$AAl?$AA?9?$AAp?$AAl@ 000000018005d318     libucrt:lcidtoname_downlevel.obj
 0002:00007328       ??_C@_1M@LJLLCMEH@?$AAp?$AAt?$AA?9?$AAb?$AAr@ 000000018005d328     libucrt:lcidtoname_downlevel.obj
 0002:00007338       ??_C@_1M@NCMONAAL@?$AAp?$AAt?$AA?9?$AAp?$AAt@ 000000018005d338     libucrt:lcidtoname_downlevel.obj
 0002:00007348       ??_C@_1O@EAKMAJDN@?$AAq?$AAu?$AAz?$AA?9?$AAb?$AAo@ 000000018005d348     libucrt:lcidtoname_downlevel.obj
 0002:00007358       ??_C@_1O@BHHPIGDN@?$AAq?$AAu?$AAz?$AA?9?$AAe?$AAc@ 000000018005d358     libucrt:lcidtoname_downlevel.obj
 0002:00007368       ??_C@_1O@GBAPEKMJ@?$AAq?$AAu?$AAz?$AA?9?$AAp?$AAe@ 000000018005d368     libucrt:lcidtoname_downlevel.obj
 0002:00007378       ??_C@_1M@CLGLEFBO@?$AAr?$AAo?$AA?9?$AAr?$AAo@ 000000018005d378     libucrt:lcidtoname_downlevel.obj
 0002:00007388       ??_C@_1M@CEEDODME@?$AAr?$AAu?$AA?9?$AAr?$AAu@ 000000018005d388     libucrt:lcidtoname_downlevel.obj
 0002:00007398       ??_C@_1M@HPKKKMPP@?$AAs?$AAa?$AA?9?$AAi?$AAn@ 000000018005d398     libucrt:lcidtoname_downlevel.obj
 0002:000073a8       ??_C@_1M@BKMAIGOJ@?$AAs?$AAe?$AA?9?$AAf?$AAi@ 000000018005d3a8     libucrt:lcidtoname_downlevel.obj
 0002:000073b8       ??_C@_1M@NDPIFLFI@?$AAs?$AAe?$AA?9?$AAn?$AAo@ 000000018005d3b8     libucrt:lcidtoname_downlevel.obj
 0002:000073c8       ??_C@_1M@DANKKHJ@?$AAs?$AAe?$AA?9?$AAs?$AAe@ 000000018005d3c8     libucrt:lcidtoname_downlevel.obj
 0002:000073d8       ??_C@_1M@PNBLONPJ@?$AAs?$AAk?$AA?9?$AAs?$AAk@ 000000018005d3d8     libucrt:lcidtoname_downlevel.obj
 0002:000073e8       ??_C@_1M@LFMODOAL@?$AAs?$AAl?$AA?9?$AAs?$AAi@ 000000018005d3e8     libucrt:lcidtoname_downlevel.obj
 0002:000073f8       ??_C@_1O@DFKOMPG@?$AAs?$AAm?$AAa?$AA?9?$AAn?$AAo@ 000000018005d3f8     libucrt:lcidtoname_downlevel.obj
 0002:00007408       ??_C@_1O@NDKPBNNH@?$AAs?$AAm?$AAa?$AA?9?$AAs?$AAe@ 000000018005d408     libucrt:lcidtoname_downlevel.obj
 0002:00007418       ??_C@_1O@PLLKBHAB@?$AAs?$AAm?$AAj?$AA?9?$AAn?$AAo@ 000000018005d418     libucrt:lcidtoname_downlevel.obj
 0002:00007428       ??_C@_1O@CLEPOGCA@?$AAs?$AAm?$AAj?$AA?9?$AAs?$AAe@ 000000018005d428     libucrt:lcidtoname_downlevel.obj
 0002:00007438       ??_C@_1O@DLGJGKMK@?$AAs?$AAm?$AAn?$AA?9?$AAf?$AAi@ 000000018005d438     libucrt:lcidtoname_downlevel.obj
 0002:00007448       ??_C@_1O@OJDJGAJC@?$AAs?$AAm?$AAs?$AA?9?$AAf?$AAi@ 000000018005d448     libucrt:lcidtoname_downlevel.obj
 0002:00007458       ??_C@_1M@BOFOGHPB@?$AAs?$AAq?$AA?9?$AAa?$AAl@ 000000018005d458     libucrt:lcidtoname_downlevel.obj
 0002:00007468       ??_C@_1BG@LJBBIPGB@?$AAs?$AAr?$AA?9?$AAb?$AAa?$AA?9?$AAc?$AAy?$AAr?$AAl@ 000000018005d468     libucrt:lcidtoname_downlevel.obj
 0002:00007480       ??_C@_1BG@JLBENFOE@?$AAs?$AAr?$AA?9?$AAb?$AAa?$AA?9?$AAl?$AAa?$AAt?$AAn@ 000000018005d480     libucrt:lcidtoname_downlevel.obj
 0002:00007498       ??_C@_1BG@KODPNHE@?$AAs?$AAr?$AA?9?$AAs?$AAp?$AA?9?$AAc?$AAy?$AAr?$AAl@ 000000018005d498     libucrt:lcidtoname_downlevel.obj
 0002:000074b0       ??_C@_1BG@CIOGKHPB@?$AAs?$AAr?$AA?9?$AAs?$AAp?$AA?9?$AAl?$AAa?$AAt?$AAn@ 000000018005d4b0     libucrt:lcidtoname_downlevel.obj
 0002:000074c8       ??_C@_1M@NGFJLMAC@?$AAs?$AAv?$AA?9?$AAf?$AAi@ 000000018005d4c8     libucrt:lcidtoname_downlevel.obj
 0002:000074d8       ??_C@_1M@MPJEJAJC@?$AAs?$AAv?$AA?9?$AAs?$AAe@ 000000018005d4d8     libucrt:lcidtoname_downlevel.obj
 0002:000074e8       ??_C@_1M@MPNDHLFK@?$AAs?$AAw?$AA?9?$AAk?$AAe@ 000000018005d4e8     libucrt:lcidtoname_downlevel.obj
 0002:000074f8       ??_C@_1O@KOHBJJI@?$AAs?$AAy?$AAr?$AA?9?$AAs?$AAy@ 000000018005d4f8     libucrt:lcidtoname_downlevel.obj
 0002:00007508       ??_C@_1M@LDCEFHA@?$AAt?$AAa?$AA?9?$AAi?$AAn@ 000000018005d508     libucrt:lcidtoname_downlevel.obj
 0002:00007518       ??_C@_1M@CNJOFAK@?$AAt?$AAe?$AA?9?$AAi?$AAn@ 000000018005d518     libucrt:lcidtoname_downlevel.obj
 0002:00007528       ??_C@_1M@GNAECACD@?$AAt?$AAh?$AA?9?$AAt?$AAh@ 000000018005d528     libucrt:lcidtoname_downlevel.obj
 0002:00007538       ??_C@_1M@CHBIHOJO@?$AAt?$AAn?$AA?9?$AAz?$AAa@ 000000018005d538     libucrt:lcidtoname_downlevel.obj
 0002:00007548       ??_C@_1M@GCCMIGPJ@?$AAt?$AAr?$AA?9?$AAt?$AAr@ 000000018005d548     libucrt:lcidtoname_downlevel.obj
 0002:00007558       ??_C@_1M@CELMCNBK@?$AAt?$AAt?$AA?9?$AAr?$AAu@ 000000018005d558     libucrt:lcidtoname_downlevel.obj
 0002:00007568       ??_C@_1M@KLMCELGA@?$AAu?$AAk?$AA?9?$AAu?$AAa@ 000000018005d568     libucrt:lcidtoname_downlevel.obj
 0002:00007578       ??_C@_1M@EPAJJAJF@?$AAu?$AAr?$AA?9?$AAp?$AAk@ 000000018005d578     libucrt:lcidtoname_downlevel.obj
 0002:00007588       ??_C@_1BG@GEGPMCDJ@?$AAu?$AAz?$AA?9?$AAu?$AAz?$AA?9?$AAc?$AAy?$AAr?$AAl@ 000000018005d588     libucrt:lcidtoname_downlevel.obj
 0002:000075a0       ??_C@_1BG@EGGKJILM@?$AAu?$AAz?$AA?9?$AAu?$AAz?$AA?9?$AAl?$AAa?$AAt?$AAn@ 000000018005d5a0     libucrt:lcidtoname_downlevel.obj
 0002:000075b8       ??_C@_1M@GFOCLFF@?$AAv?$AAi?$AA?9?$AAv?$AAn@ 000000018005d5b8     libucrt:lcidtoname_downlevel.obj
 0002:000075c8       ??_C@_1M@CPAMEDFI@?$AAx?$AAh?$AA?9?$AAz?$AAa@ 000000018005d5c8     libucrt:lcidtoname_downlevel.obj
 0002:000075d8       ??_C@_1O@EBKIFIGN@?$AAz?$AAh?$AA?9?$AAc?$AAh?$AAs@ 000000018005d5d8     libucrt:lcidtoname_downlevel.obj
 0002:000075e8       ??_C@_1O@NMHPGANE@?$AAz?$AAh?$AA?9?$AAc?$AAh?$AAt@ 000000018005d5e8     libucrt:lcidtoname_downlevel.obj
 0002:000075f8       ??_C@_1M@LPINJOMC@?$AAz?$AAh?$AA?9?$AAc?$AAn@ 000000018005d5f8     libucrt:lcidtoname_downlevel.obj
 0002:00007608       ??_C@_1M@OCJEJODD@?$AAz?$AAh?$AA?9?$AAh?$AAk@ 000000018005d608     libucrt:lcidtoname_downlevel.obj
 0002:00007618       ??_C@_1M@DNDLJINH@?$AAz?$AAh?$AA?9?$AAm?$AAo@ 000000018005d618     libucrt:lcidtoname_downlevel.obj
 0002:00007628       ??_C@_1M@MBFDNDND@?$AAz?$AAh?$AA?9?$AAs?$AAg@ 000000018005d628     libucrt:lcidtoname_downlevel.obj
 0002:00007638       ??_C@_1M@IMEPLEPE@?$AAz?$AAh?$AA?9?$AAt?$AAw@ 000000018005d638     libucrt:lcidtoname_downlevel.obj
 0002:00007648       ??_C@_1M@BBGHNHJP@?$AAz?$AAu?$AA?9?$AAz?$AAa@ 000000018005d648     libucrt:lcidtoname_downlevel.obj
 0002:000078b0       ??_C@_1BA@BALFACEM@?$AAC?$AAO?$AAN?$AAO?$AAU?$AAT?$AA$@ 000000018005d8b0     libucrt:initcon.obj
 0002:000078c0       __log10_256_lead           000000018005d8c0     libucrt:log10_256_lead_tail_table.obj
 0002:000080d0       __log10_256_tail           000000018005e0d0     libucrt:log10_256_lead_tail_table.obj
 0002:000088e0       __log_F_inv_qword          000000018005e8e0     libucrt:log_f_inv_qword_table.obj
 0002:000090f0       ??_C@_05HGHHAHAP@log10@    000000018005f0f0     libucrt:log_special.obj
 0002:000090f8       ??_C@_09GPALILFO@bad?5int64@ 000000018005f0f8     bit64.obj
 0002:00009104       ??_C@_05LLAMLEHD@?$CFI64d@ 000000018005f104     bit64.obj
 0002:0000910c       ??_C@_04JAOJMBA@bnot@      000000018005f10c     bit64.obj
 0002:00009114       ??_C@_04BKGNPECA@band@     000000018005f114     bit64.obj
 0002:0000911c       ??_C@_03BBBGIIAC@bor@      000000018005f11c     bit64.obj
 0002:00009120       ??_C@_04CKCGDDNF@bxor@     000000018005f120     bit64.obj
 0002:00009128       ??_C@_06ELFGPGBK@lshift@   000000018005f128     bit64.obj
 0002:00009130       ??_C@_06HMLHBBIJ@rshift@   000000018005f130     bit64.obj
 0002:00009138       ??_C@_07JILILBLL@arshift@  000000018005f138     bit64.obj
 0002:00009140       ??_C@_03CLCAEGCJ@new@      000000018005f140     bit64.obj
 0002:00009144       ??_C@_03BDGOHNNK@add@      000000018005f144     bit64.obj
 0002:00009148       ??_C@_03KCMAIMAP@sub@      000000018005f148     bit64.obj
 0002:0000914c       ??_C@_03IMIFIBCN@mul@      000000018005f14c     bit64.obj
 0002:00009150       ??_C@_03FEJMGOGI@div@      000000018005f150     bit64.obj
 0002:00009154       ??_C@_03FFONCNID@mod@      000000018005f154     bit64.obj
 0002:00009158       ??_C@_02HIIGGHJB@eq@       000000018005f158     bit64.obj
 0002:0000915c       ??_C@_02KCAKIFL@lt@        000000018005f15c     bit64.obj
 0002:00009160       ??_C@_02FJPJILEL@le@       000000018005f160     bit64.obj
 0002:00009164       ??_C@_04GPMDFGEJ@type@     000000018005f164     bit64.obj
 0002:0000916c       ??_C@_05MEHDOBFN@__add@    000000018005f16c     bit64.obj
 0002:00009174       ??_C@_05HFNNBAII@__sub@    000000018005f174     bit64.obj
 0002:0000917c       ??_C@_05FLJIBNKK@__mul@    000000018005f17c     bit64.obj
 0002:00009184       ??_C@_05IDIBPCOP@__div@    000000018005f184     bit64.obj
 0002:0000918c       ??_C@_05ICPALBAE@__mod@    000000018005f18c     bit64.obj
 0002:00009194       ??_C@_05MHFNBPAK@__unm@    000000018005f194     bit64.obj
 0002:0000919c       ??_C@_04GIMIAOHA@__eq@     000000018005f19c     bit64.obj
 0002:000091a4       ??_C@_04BKGOMBLK@__lt@     000000018005f1a4     bit64.obj
 0002:000091ac       ??_C@_04EJLHOCKK@__le@     000000018005f1ac     bit64.obj
 0002:000091b8       ??_C@_0L@HDFPAPPH@__tostring@ 000000018005f1b8     bit64.obj
 0002:000091c8       ??_C@_08JOIMPOJO@tonumber@ 000000018005f1c8     bit64.obj
 0002:000091d8       ??_C@_07NHABFFHN@__index@  000000018005f1d8     bit64.obj
 0002:000091e0       ??_C@_05OALCLICP@bit64@    000000018005f1e0     bit64.obj
 0002:000091e8       metatable_name             000000018005f1e8     bit64.obj
 0002:000093e0       ??_C@_05GFCDIDHO@debug@    000000018005f3e0     exported.obj
 0002:000093e8       ??_C@_09GPFEECNC@traceback@ 000000018005f3e8     exported.obj
 0002:000093f4       ??_C@_06NKNNMLDJ@export@   000000018005f3f4     exported.obj
 0002:00009400       ??_C@_07PCNKBAGB@OnError@  000000018005f400     exported.obj
 0002:00009408       ??_C@_0N@NJMIGDDL@CreationTime@ 000000018005f408     exported.obj
 0002:00009418       ??_C@_0P@MFHPCDDH@LastAccessTime@ 000000018005f418     exported.obj
 0002:00009428       ??_C@_0O@FCFNCAHK@LastWriteTime@ 000000018005f428     exported.obj
 0002:00009438       ??_C@_0L@FCILKIIG@ChangeTime@ 000000018005f438     exported.obj
 0002:00009448       ??_C@_08BHIEONMC@FileSize@ 000000018005f448     exported.obj
 0002:00009458       ??_C@_0P@JBACEJLL@AllocationSize@ 000000018005f458     exported.obj
 0002:00009468       ??_C@_05BOOEKJH@Flags@     000000018005f468     exported.obj
 0002:00009470       ??_C@_0O@DLGJHFNH@NumberOfLinks@ 000000018005f470     exported.obj
 0002:00009480       ??_C@_05MHNOECFO@CRC32@    000000018005f480     exported.obj
 0002:00009488       ??_C@_08FDCJCDOL@FileName@ 000000018005f488     exported.obj
 0002:00009498       ??_C@_0BC@COCBGKAE@AlternateFileName@ 000000018005f498     exported.obj
 0002:000094b0       ??_C@_0M@OHKMKKDH@Description@ 000000018005f4b0     exported.obj
 0002:000094bc       ??_C@_05HDCNEILF@Owner@    000000018005f4bc     exported.obj
 0002:000094c8       ??_C@_0BB@OKGMKOG@CustomColumnData@ 000000018005f4c8     exported.obj
 0002:000094dc       ??_C@_01LOCGONAA@?$AA@     000000018005f4dc     service.obj
 0002:000094dc       ??_C@_11LOCGONAA@@         000000018005f4dc     exported.obj
 0002:000094e0       ??_C@_08JNHPECBG@UserData@ 000000018005f4e0     exported.obj
 0002:000094f0       ??_C@_0M@BDCAMGGD@ExtUserData@ 000000018005f4f0     exported.obj
 0002:00009500       ??_C@_0N@LHFGLEGJ@FreeUserData@ 000000018005f500     exported.obj
 0002:00009510       ??_C@_0M@DFMHDHBL@GetFindData@ 000000018005f510     exported.obj
 0002:00009520       ??_C@_08FFPEEIHA@GetFiles@ 000000018005f520     exported.obj
 0002:00009530       ??_C@_0BC@IECOKJFL@GetFiles?4DestPath@ 000000018005f530     exported.obj
 0002:00009544       ??_C@_05LFOKGKBN@?$DMboot@ 000000018005f544     exported.obj
 0002:0000954c       ??_C@_15CBMDENPJ@?$AA?4?$AA?9@ 000000018005f54c     exported.obj
 0002:00009558       ??_C@_07KNEGBPNO@package@  000000018005f558     exported.obj
 0002:00009560       ??_C@_07GCEAJMEA@preload@  000000018005f560     exported.obj
 0002:00009568       ??_C@_19BCNABNAK@?$AA?4?$AAl?$AAu?$AAa@ 000000018005f568     exported.obj
 0002:00009574       ??_C@_13BPINEIPE@?$AAr@    000000018005f574     exported.obj
 0002:00009578       ??_C@_1DC@PABHCCON@?$AAD?$AAe?$AAf?$AAa?$AAu?$AAl?$AAt?$AA?5?$AAs?$AAc?$AAr?$AAi?$AAp?$AAt?$AA?5@ 000000018005f578     exported.obj
 0002:000095ac       ??_C@_03JEOKDCFP@far@      000000018005f5ac     exported.obj
 0002:000095b0       ??_C@_0BE@HCPAIELH@ReloadDefaultScript@ 000000018005f5b0     exported.obj
 0002:000095c8       ??_C@_0L@OCPPMCCK@StructSize@ 000000018005f5c8     exported.obj
 0002:000095d4       ??_C@_06LBMCOACO@Buffer@   000000018005f5d4     exported.obj
 0002:000095dc       ??_C@_06EPIAKPGD@OpMode@   000000018005f5dc     exported.obj
 0002:000095e8       ??_C@_07GDADDFBD@Analyse@  000000018005f5e8     exported.obj
 0002:000095f0       ??_C@_0BB@CKIGBGLB@GetOpenPanelInfo@ 000000018005f5f0     exported.obj
 0002:00009608       ??_C@_08KDMNIFGM@FreeSize@ 000000018005f608     exported.obj
 0002:00009618       ??_C@_08PAJOMFPO@HostFile@ 000000018005f618     exported.obj
 0002:00009624       ??_C@_06IBPEEEAJ@CurDir@   000000018005f624     exported.obj
 0002:0000962c       ??_C@_06PEPCFMNJ@Format@   000000018005f62c     exported.obj
 0002:00009638       ??_C@_0L@CMHIOLLB@PanelTitle@ 000000018005f638     exported.obj
 0002:00009648       ??_C@_09PMEOAIAA@InfoLines@ 000000018005f648     exported.obj
 0002:00009658       ??_C@_0BA@BLCGOCOG@InfoLinesNumber@ 000000018005f658     exported.obj
 0002:00009668       ??_C@_04OJAHODMC@Text@     000000018005f668     exported.obj
 0002:00009670       ??_C@_04DICKPMGH@Data@     000000018005f670     exported.obj
 0002:00009678       ??_C@_0L@FPEHOFAI@DescrFiles@ 000000018005f678     exported.obj
 0002:00009688       ??_C@_0BA@BBOGKOKF@PanelModesArray@ 000000018005f688     exported.obj
 0002:00009698       ??_C@_0BB@LFNABPEF@PanelModesNumber@ 000000018005f698     exported.obj
 0002:000096b0       ??_C@_0M@KDJPJFOF@ColumnTypes@ 000000018005f6b0     exported.obj
 0002:000096c0       ??_C@_0N@ILFJPGHI@ColumnWidths@ 000000018005f6c0     exported.obj
 0002:000096d0       ??_C@_0BC@KELOOKNK@StatusColumnTypes@ 000000018005f6d0     exported.obj
 0002:000096e8       ??_C@_0BD@DNDIPKDK@StatusColumnWidths@ 000000018005f6e8     exported.obj
 0002:00009700       ??_C@_0N@EHCEJHEE@ColumnTitles@ 000000018005f700     exported.obj
 0002:00009710       ??_C@_0P@BEEDPJDK@StartPanelMode@ 000000018005f710     exported.obj
 0002:00009720       ??_C@_0O@NIFKFGBJ@StartSortMode@ 000000018005f720     exported.obj
 0002:00009730       ??_C@_0P@KMACBLNK@StartSortOrder@ 000000018005f730     exported.obj
 0002:00009740       ??_C@_06ONGFDHIA@KeyBar@   000000018005f740     exported.obj
 0002:00009748       ??_C@_0P@PKDBPEJI@VirtualKeyCode@ 000000018005f748     exported.obj
 0002:00009758       ??_C@_0BA@MFFHAKP@ControlKeyState@ 000000018005f758     exported.obj
 0002:00009768       ??_C@_08DGDJEKCP@LongText@ 000000018005f768     exported.obj
 0002:00009778       ??_C@_0BE@OPMKBLIP@_ModuleShortcutData@ 000000018005f778     exported.obj
 0002:00009790       ??_C@_0N@IHDKLODA@ShortcutData@ 000000018005f790     exported.obj
 0002:000097a0       ??_C@_05HIFJDKLD@array@    000000018005f7a0     exported.obj
 0002:000097a8       ??_C@_01EFFIKLCJ@n@        000000018005f7a8     exported.obj
 0002:000097aa       ??_C@_00CNPNBAHC@@         000000018005f7aa     exported.obj
 0002:000097ac       ??_C@_04DNCDCIAE@Open@     000000018005f7ac     exported.obj
 0002:000097b4       ??_C@_04OPJIDECA@hDlg@     000000018005f7b4     exported.obj
 0002:000097bc       ??_C@_06BNNOMDLO@Handle@   000000018005f7bc     exported.obj
 0002:000097c4       ??_C@_05LNOAKADA@panel@    000000018005f7c4     exported.obj
 0002:000097d0       ??_C@_0L@JMPDJFBN@ClosePanel@ 000000018005f7d0     exported.obj
 0002:000097e0       ??_C@_07MBOMJGGF@Compare@  000000018005f7e0     exported.obj
 0002:000097e8       ??_C@_09NANCCILE@Configure@ 000000018005f7e8     exported.obj
 0002:000097f8       ??_C@_0M@MMKKMEFA@DeleteFiles@ 000000018005f7f8     exported.obj
 0002:00009808       ??_C@_0O@GLLEDHJA@MakeDirectory@ 000000018005f808     exported.obj
 0002:00009818       ??_C@_0BD@PJNONGDB@MakeDirectory?4Name@ 000000018005f818     exported.obj
 0002:00009830       ??_C@_0BC@COPMJGBI@ProcessPanelEvent@ 000000018005f830     exported.obj
 0002:00009848       ??_C@_0BA@DPJAKFGC@ProcessHostFile@ 000000018005f848     exported.obj
 0002:00009858       ??_C@_0BC@HOBKGBBM@ProcessPanelInput@ 000000018005f858     exported.obj
 0002:00009870       ??_C@_08OBOOFGOD@PutFiles@ 000000018005f870     exported.obj
 0002:00009880       ??_C@_0N@KCFEBPAO@SetDirectory@ 000000018005f880     exported.obj
 0002:00009890       ??_C@_0M@PNOHHCCH@SetFindList@ 000000018005f890     exported.obj
 0002:000098a0       ??_C@_07EACELFAO@ExitFAR@  000000018005f8a0     exported.obj
 0002:000098a8       ??_C@_0O@OBCKADMD@GetPluginInfo@ 000000018005f8a8     exported.obj
 0002:000098b8       ??_C@_0O@GDMHGAFH@CommandPrefix@ 000000018005f8b8     exported.obj
 0002:000098c8       ??_C@_0O@PHBKMNMJ@DiskMenuGuids@ 000000018005f8c8     exported.obj
 0002:000098d8       ??_C@_0BA@NLBDFPEO@DiskMenuStrings@ 000000018005f8d8     exported.obj
 0002:000098e8       ??_C@_0BA@FOMPNLJF@PluginMenuGuids@ 000000018005f8e8     exported.obj
 0002:000098f8       ??_C@_0BC@DJMJFBJC@PluginMenuStrings@ 000000018005f8f8     exported.obj
 0002:00009910       ??_C@_0BC@ILBHAHCH@PluginConfigGuids@ 000000018005f910     exported.obj
 0002:00009928       ??_C@_0BE@GAFPNGIP@PluginConfigStrings@ 000000018005f928     exported.obj
 0002:00009940       ??_C@_0BD@DECJPBBK@ProcessEditorInput@ 000000018005f940     exported.obj
 0002:00009958       ??_C@_0BD@GEMPAGBO@ProcessEditorEvent@ 000000018005f958     exported.obj
 0002:0000996c       ??_C@_04KOACHJEN@Type@     000000018005f96c     exported.obj
 0002:00009978       ??_C@_0N@EKPHGDMI@StringNumber@ 000000018005f978     exported.obj
 0002:00009988       ??_C@_07MOCFLHCN@FileEOL@  000000018005f988     exported.obj
 0002:00009990       ??_C@_08DOHJINHB@CodePage@ 000000018005f990     exported.obj
 0002:000099a0       ??_C@_0BD@GGKMLEJG@ProcessViewerEvent@ 000000018005f9a0     exported.obj
 0002:000099b8       ??_C@_0BD@FNHBEIC@ProcessDialogEvent@ 000000018005f9b8     exported.obj
 0002:000099cc       ??_C@_06CPBJDKAC@Param2@   000000018005f9cc     exported.obj
 0002:000099d4       ??_C@_06EDEGJMB@Param1@    000000018005f9d4     exported.obj
 0002:000099dc       ??_C@_03MLMOILGK@Msg@      000000018005f9dc     exported.obj
 0002:000099e0       ??_C@_0BE@LHJGGGHN@ProcessSynchroEvent@ 000000018005f9e0     exported.obj
 0002:000099f8       ??_C@_0BB@PHIEFGHD@GetContentFields@ 000000018005f9f8     exported.obj
 0002:00009a10       ??_C@_0P@DPJDPMPI@GetContentData@ 000000018005fa10     exported.obj
 0002:00009a20       ??_C@_0N@DDJEHLKE@?$DM_globalinfo@ 000000018005fa20     exported.obj
 0002:00009a30       ??_C@_1CA@IBKDMBNJ@?$AA_?$AAg?$AAl?$AAo?$AAb?$AAa?$AAl?$AAi?$AAn?$AAf?$AAo?$AA?4?$AAl?$AAu?$AAa@ 000000018005fa30     exported.obj
 0002:00009a50       ??_C@_0O@GJMOPLGM@GetGlobalInfo@ 000000018005fa50     exported.obj
 0002:00009a60       ??_C@_0O@CALOEOI@MinFarVersion@ 000000018005fa60     exported.obj
 0002:00009a70       ??_C@_07NGFJPNPN@Version@  000000018005fa70     exported.obj
 0002:00009a78       ??_C@_04MJHIICBJ@Guid@     000000018005fa78     exported.obj
 0002:00009a80       ??_C@_05PABKJLOM@Title@    000000018005fa80     exported.obj
 0002:00009a88       ??_C@_06HHECMMLE@Author@   000000018005fa88     exported.obj
 0002:00009a90       ??_C@_0BE@DONMOPMJ@ProcessConsoleInput@ 000000018005fa90     exported.obj
 0002:00009aa8       KEY_OBJECT                 000000018005faa8     exported.obj
 0002:00009ab8       COLLECTOR_GI               000000018005fab8     exported.obj
 0002:00009ad0       COLLECTOR_OPI              000000018005fad0     exported.obj
 0002:00009ae8       COLLECTOR_PI               000000018005fae8     exported.obj
 0002:00009b00       ??_C@_0BI@IDKIJMME@FARMANAGERVERSION_MAJOR@ 000000018005fb00     flags.obj
 0002:00009b18       ??_C@_0BI@DMLKEAFC@FARMANAGERVERSION_MINOR@ 000000018005fb18     flags.obj
 0002:00009b30       ??_C@_0BL@NMALNAFP@FARMANAGERVERSION_REVISION@ 000000018005fb30     flags.obj
 0002:00009b50       ??_C@_0BI@OLPFLLDD@FARMANAGERVERSION_BUILD@ 000000018005fb50     flags.obj
 0002:00009b68       ??_C@_0BI@MOOFLFPC@FARMANAGERVERSION_STAGE@ 000000018005fb68     flags.obj
 0002:00009b80       ??_C@_0L@MIDBGFJO@CP_UNICODE@ 000000018005fb80     flags.obj
 0002:00009b90       ??_C@_0O@MNMCMEJH@CP_REVERSEBOM@ 000000018005fb90     flags.obj
 0002:00009ba0       ??_C@_0L@JDNPCEDH@CP_DEFAULT@ 000000018005fba0     flags.obj
 0002:00009bb0       ??_C@_0M@OMCMFJHA@CP_REDETECT@ 000000018005fbb0     flags.obj
 0002:00009bc0       ??_C@_09MNAPNKKC@INDEXMASK@ 000000018005fbc0     flags.obj
 0002:00009bd0       ??_C@_09BLFIDJLF@COLORMASK@ 000000018005fbd0     flags.obj
 0002:00009be0       ??_C@_09ENNBLPJC@ALPHAMASK@ 000000018005fbe0     flags.obj
 0002:00009bf0       ??_C@_0L@EHFOPLFD@PANEL_NONE@ 000000018005fbf0     flags.obj
 0002:00009c00       ??_C@_0N@LPMKALBG@PANEL_ACTIVE@ 000000018005fc00     flags.obj
 0002:00009c10       ??_C@_0O@HPKEABPN@PANEL_PASSIVE@ 000000018005fc10     flags.obj
 0002:00009c20       ??_C@_0L@GOEBPENN@PANEL_STOP@ 000000018005fc20     flags.obj
 0002:00009c30       ??_C@_0N@HLIFAAPJ@EEREDRAW_ALL@ 000000018005fc30     flags.obj
 0002:00009c40       ??_C@_0P@NHNDIKJ@CURRENT_EDITOR@ 000000018005fc40     flags.obj
 0002:00009c50       ??_C@_0BN@PPNDCHHA@EDITOR_COLOR_NORMAL_PRIORITY@ 000000018005fc50     flags.obj
 0002:00009c70       ??_C@_07MGGAEAFF@DI_TEXT@  000000018005fc70     flags.obj
 0002:00009c78       ??_C@_08HODBDEHE@DI_VTEXT@ 000000018005fc78     flags.obj
 0002:00009c88       ??_C@_0N@IGKKGFMF@DI_SINGLEBOX@ 000000018005fc88     flags.obj
 0002:00009c98       ??_C@_0N@EDCLIEAE@DI_DOUBLEBOX@ 000000018005fc98     flags.obj
 0002:00009ca8       ??_C@_07DOLIFAEF@DI_EDIT@  000000018005fca8     flags.obj
 0002:00009cb0       ??_C@_0L@EOMEIIFM@DI_PSWEDIT@ 000000018005fcb0     flags.obj
 0002:00009cc0       ??_C@_0L@MGOIMBKF@DI_FIXEDIT@ 000000018005fcc0     flags.obj
 0002:00009cd0       ??_C@_09GGAEMAPJ@DI_BUTTON@ 000000018005fcd0     flags.obj
 0002:00009ce0       ??_C@_0M@MHFHGPHJ@DI_CHECKBOX@ 000000018005fce0     flags.obj
 0002:00009cf0       ??_C@_0P@GIPCGMBE@DI_RADIOBUTTON@ 000000018005fcf0     flags.obj
 0002:00009d00       ??_C@_0M@MAKBFNGC@DI_COMBOBOX@ 000000018005fd00     flags.obj
 0002:00009d10       ??_C@_0L@ONDMPPPO@DI_LISTBOX@ 000000018005fd10     flags.obj
 0002:00009d20       ??_C@_0P@GDJDPEIK@DI_USERCONTROL@ 000000018005fd20     flags.obj
 0002:00009d30       ??_C@_08KAEGOLOB@DM_FIRST@ 000000018005fd30     flags.obj
 0002:00009d40       ??_C@_08MJMBFJHA@DM_CLOSE@ 000000018005fd40     flags.obj
 0002:00009d50       ??_C@_09KLJOCKAA@DM_ENABLE@ 000000018005fd50     flags.obj
 0002:00009d60       ??_C@_0BA@KAMJGFDG@DM_ENABLEREDRAW@ 000000018005fd60     flags.obj
 0002:00009d70       ??_C@_0O@FKGMMKLP@DM_GETDLGDATA@ 000000018005fd70     flags.obj
 0002:00009d80       ??_C@_0O@HEGKCPOI@DM_GETDLGITEM@ 000000018005fd80     flags.obj
 0002:00009d90       ??_C@_0O@BEHCGMCL@DM_GETDLGRECT@ 000000018005fd90     flags.obj
 0002:00009da0       ??_C@_0L@ELBDNLFO@DM_GETTEXT@ 000000018005fda0     flags.obj
 0002:00009dac       ??_C@_06IKGPEGEJ@DM_KEY@   000000018005fdac     flags.obj
 0002:00009db8       ??_C@_0O@DIPLLJEH@DM_MOVEDIALOG@ 000000018005fdb8     flags.obj
 0002:00009dc8       ??_C@_0O@EEEDHNPG@DM_SETDLGDATA@ 000000018005fdc8     flags.obj
 0002:00009dd8       ??_C@_0O@GKEFJIKB@DM_SETDLGITEM@ 000000018005fdd8     flags.obj
 0002:00009de8       ??_C@_0M@GOFGHDFK@DM_SETFOCUS@ 000000018005fde8     flags.obj
 0002:00009df8       ??_C@_09ILPFEDOM@DM_REDRAW@ 000000018005fdf8     flags.obj
 0002:00009e08       ??_C@_0L@LDOCOEIP@DM_SETTEXT@ 000000018005fe08     flags.obj
 0002:00009e18       ??_C@_0BE@LABEAIPD@DM_SETMAXTEXTLENGTH@ 000000018005fe18     flags.obj
 0002:00009e30       ??_C@_0O@BIFKIPIP@DM_SHOWDIALOG@ 000000018005fe30     flags.obj
 0002:00009e40       ??_C@_0M@JPHKGACH@DM_GETFOCUS@ 000000018005fe40     flags.obj
 0002:00009e50       ??_C@_0BA@NLMONBKJ@DM_GETCURSORPOS@ 000000018005fe50     flags.obj
 0002:00009e60       ??_C@_0BA@KPHABNOF@DM_SETCURSORPOS@ 000000018005fe60     flags.obj
 0002:00009e70       ??_C@_0O@LGEKFPKK@DM_SETTEXTPTR@ 000000018005fe70     flags.obj
 0002:00009e80       ??_C@_0M@NCOJHJKI@DM_SHOWITEM@ 000000018005fe80     flags.obj
 0002:00009e90       ??_C@_0O@GKKCFHIM@DM_ADDHISTORY@ 000000018005fe90     flags.obj
 0002:00009ea0       ??_C@_0M@MCEMDFMD@DM_GETCHECK@ 000000018005fea0     flags.obj
 0002:00009eb0       ??_C@_0M@DDGACGLO@DM_SETCHECK@ 000000018005feb0     flags.obj
 0002:00009ec0       ??_C@_0N@MEGOPFGK@DM_SET3STATE@ 000000018005fec0     flags.obj
 0002:00009ed0       ??_C@_0M@GEPBDDNC@DM_LISTSORT@ 000000018005fed0     flags.obj
 0002:00009ee0       ??_C@_0P@NFJNHAKH@DM_LISTGETITEM@ 000000018005fee0     flags.obj
 0002:00009ef0       ??_C@_0BB@EEIMACNO@DM_LISTGETCURPOS@ 000000018005fef0     flags.obj
 0002:00009f08       ??_C@_0BB@GKMJCDEM@DM_LISTSETCURPOS@ 000000018005ff08     flags.obj
 0002:00009f20       ??_C@_0O@NOPCAHGJ@DM_LISTDELETE@ 000000018005ff20     flags.obj
 0002:00009f30       ??_C@_0L@BMEAECNG@DM_LISTADD@ 000000018005ff30     flags.obj
 0002:00009f40       ??_C@_0O@HBHDMHP@DM_LISTADDSTR@ 000000018005ff40     flags.obj
 0002:00009f50       ??_C@_0O@PDFCNPKN@DM_LISTUPDATE@ 000000018005ff50     flags.obj
 0002:00009f60       ??_C@_0O@GAAGMJJL@DM_LISTINSERT@ 000000018005ff60     flags.obj
 0002:00009f70       ??_C@_0BC@MIFCLOBD@DM_LISTFINDSTRING@ 000000018005ff70     flags.obj
 0002:00009f88       ??_C@_0M@EEAEBLKC@DM_LISTINFO@ 000000018005ff88     flags.obj
 0002:00009f98       ??_C@_0P@PLJLJFPA@DM_LISTGETDATA@ 000000018005ff98     flags.obj
 0002:00009fa8       ??_C@_0P@DGKKKCB@DM_LISTSETDATA@ 000000018005ffa8     flags.obj
 0002:00009fb8       ??_C@_0BB@CELMNLLN@DM_LISTSETTITLES@ 000000018005ffb8     flags.obj
 0002:00009fd0       ??_C@_0BB@KPJPKCP@DM_LISTGETTITLES@ 000000018005ffd0     flags.obj
 0002:00009fe8       ??_C@_0BA@ICDJCFLE@DM_RESIZEDIALOG@ 000000018005ffe8     flags.obj
 0002:00009ff8       ??_C@_0BD@CNGGHGJF@DM_SETITEMPOSITION@ 000000018005fff8     flags.obj
 0002:0000a010       ??_C@_0BF@JMINBGBA@DM_GETDROPDOWNOPENED@ 0000000180060010     flags.obj
 0002:0000a028       ??_C@_0BF@LJIGJNAO@DM_SETDROPDOWNOPENED@ 0000000180060028     flags.obj
 0002:0000a040       ??_C@_0O@NPDKADMJ@DM_SETHISTORY@ 0000000180060040     flags.obj
 0002:0000a050       ??_C@_0BD@BPHAAEIM@DM_GETITEMPOSITION@ 0000000180060050     flags.obj
 0002:0000a068       ??_C@_0BC@BENFKLNH@DM_SETINPUTNOTIFY@ 0000000180060068     flags.obj
 0002:0000a080       ??_C@_0BH@CFMLLNNM@DM_SETMOUSEEVENTNOTIFY@ 0000000180060080     flags.obj
 0002:0000a098       ??_C@_0BF@IAGIACOD@DM_EDITUNCHANGEDFLAG@ 0000000180060098     flags.obj
 0002:0000a0b0       ??_C@_0P@OJKNHIPN@DM_GETITEMDATA@ 00000001800600b0     flags.obj
 0002:0000a0c0       ??_C@_0P@OGLDKOHO@DM_SETITEMDATA@ 00000001800600c0     flags.obj
 0002:0000a0d0       ??_C@_0L@KNFAKFKE@DM_LISTSET@ 00000001800600d0     flags.obj
 0002:0000a0e0       ??_C@_0BB@EPMFHAFO@DM_GETCURSORSIZE@ 00000001800600e0     flags.obj
 0002:0000a0f8       ??_C@_0BB@DANLMDCJ@DM_SETCURSORSIZE@ 00000001800600f8     flags.obj
 0002:0000a110       ??_C@_0BD@LAOOKGHD@DM_LISTGETDATASIZE@ 0000000180060110     flags.obj
 0002:0000a128       ??_C@_0BA@BHGANJAP@DM_GETSELECTION@ 0000000180060128     flags.obj
 0002:0000a138       ??_C@_0BA@GDNOBFED@DM_SETSELECTION@ 0000000180060138     flags.obj
 0002:0000a148       ??_C@_0BD@FIHDGIGO@DM_GETEDITPOSITION@ 0000000180060148     flags.obj
 0002:0000a160       ??_C@_0BD@GKGFBKHH@DM_SETEDITPOSITION@ 0000000180060160     flags.obj
 0002:0000a178       ??_C@_0BE@MCECGHBC@DM_SETCOMBOBOXEVENT@ 0000000180060178     flags.obj
 0002:0000a190       ??_C@_0BE@KGBLNJKA@DM_GETCOMBOBOXEVENT@ 0000000180060190     flags.obj
 0002:0000a1a8       ??_C@_0BD@CJEPBACF@DM_GETCONSTTEXTPTR@ 00000001800601a8     flags.obj
 0002:0000a1c0       ??_C@_0BD@HOOHICEG@DM_GETDLGITEMSHORT@ 00000001800601c0     flags.obj
 0002:0000a1d8       ??_C@_0BD@EMPBPAFP@DM_SETDLGITEMSHORT@ 00000001800601d8     flags.obj
 0002:0000a1f0       ??_C@_0BB@GAPFMPKE@DM_GETDIALOGINFO@ 00000001800601f0     flags.obj
 0002:0000a208       ??_C@_0BC@KJOLMFGG@DM_GETDIALOGTITLE@ 0000000180060208     flags.obj
 0002:0000a220       ??_C@_08COMJOMAC@DN_FIRST@ 0000000180060220     flags.obj
 0002:0000a230       ??_C@_0M@NNNAPNMA@DN_BTNCLICK@ 0000000180060230     flags.obj
 0002:0000a240       ??_C@_0BC@MJFJAANN@DN_CTLCOLORDIALOG@ 0000000180060240     flags.obj
 0002:0000a258       ??_C@_0BD@HFGBIBBL@DN_CTLCOLORDLGITEM@ 0000000180060258     flags.obj
 0002:0000a270       ??_C@_0BD@JMFJPHPD@DN_CTLCOLORDLGLIST@ 0000000180060270     flags.obj
 0002:0000a288       ??_C@_0O@NKBDPILK@DN_DRAWDIALOG@ 0000000180060288     flags.obj
 0002:0000a298       ??_C@_0P@KGKEDPBI@DN_DRAWDLGITEM@ 0000000180060298     flags.obj
 0002:0000a2a8       ??_C@_0O@JMKNGFLE@DN_EDITCHANGE@ 00000001800602a8     flags.obj
 0002:0000a2b8       ??_C@_0M@JHFIBKOO@DN_GOTFOCUS@ 00000001800602b8     flags.obj
 0002:0000a2c8       ??_C@_07NJJEMKPA@DN_HELP@  00000001800602c8     flags.obj
 0002:0000a2d0       ??_C@_09EDGJFAK@DN_HOTKEY@ 00000001800602d0     flags.obj
 0002:0000a2e0       ??_C@_0O@BJECHBCA@DN_INITDIALOG@ 00000001800602e0     flags.obj
 0002:0000a2f0       ??_C@_0N@CHLLLNBO@DN_KILLFOCUS@ 00000001800602f0     flags.obj
 0002:0000a300       ??_C@_0O@CLPABIGO@DN_LISTCHANGE@ 0000000180060300     flags.obj
 0002:0000a310       ??_C@_0L@MLMFBHN@DN_DRAGGED@ 0000000180060310     flags.obj
 0002:0000a320       ??_C@_0BB@BOOOCAEG@DN_RESIZECONSOLE@ 0000000180060320     flags.obj
 0002:0000a338       ??_C@_0BC@FHPPFLKG@DN_DRAWDIALOGDONE@ 0000000180060338     flags.obj
 0002:0000a350       ??_C@_0O@EONPBNNP@DN_LISTHOTKEY@ 0000000180060350     flags.obj
 0002:0000a360       ??_C@_08MDDLDGPO@DN_INPUT@ 0000000180060360     flags.obj
 0002:0000a370       ??_C@_0BA@FGOGLDBC@DN_CONTROLINPUT@ 0000000180060370     flags.obj
 0002:0000a380       ??_C@_08EHEOFOJD@DN_CLOSE@ 0000000180060380     flags.obj
 0002:0000a390       ??_C@_0M@POIFBPFN@DN_GETVALUE@ 0000000180060390     flags.obj
 0002:0000a3a0       ??_C@_0BC@MHCBFAAO@DN_DROPDOWNOPENED@ 00000001800603a0     flags.obj
 0002:0000a3b8       ??_C@_0BD@NGEKAPIF@DN_DRAWDLGITEMDONE@ 00000001800603b8     flags.obj
 0002:0000a3d0       ??_C@_07DIJJNCBA@DM_USER@  00000001800603d0     flags.obj
 0002:0000a3d8       ??_C@_0BB@HLBBGMAN@BSTATE_UNCHECKED@ 00000001800603d8     flags.obj
 0002:0000a3f0       ??_C@_0P@FALAMPGP@BSTATE_CHECKED@ 00000001800603f0     flags.obj
 0002:0000a400       ??_C@_0O@KBIFGGHO@BSTATE_3STATE@ 0000000180060400     flags.obj
 0002:0000a410       ??_C@_0O@ILJOJGLD@BSTATE_TOGGLE@ 0000000180060410     flags.obj
 0002:0000a420       ??_C@_08PPADCPCM@CBET_KEY@ 0000000180060420     flags.obj
 0002:0000a430       ??_C@_0L@KHCLMGFJ@CBET_MOUSE@ 0000000180060430     flags.obj
 0002:0000a440       ??_C@_0BA@KNHGEBNE@PTYPE_FILEPANEL@ 0000000180060440     flags.obj
 0002:0000a450       ??_C@_0BA@LPPHNHIG@PTYPE_TREEPANEL@ 0000000180060450     flags.obj
 0002:0000a460       ??_C@_0BB@JBINOKAI@PTYPE_QVIEWPANEL@ 0000000180060460     flags.obj
 0002:0000a478       ??_C@_0BA@NKMDEBG@PTYPE_INFOPANEL@ 0000000180060478     flags.obj
 0002:0000a488       ??_C@_0L@OPHJOKKE@SM_DEFAULT@ 0000000180060488     flags.obj
 0002:0000a498       ??_C@_0M@JGBFGGEA@SM_UNSORTED@ 0000000180060498     flags.obj
 0002:0000a4a8       ??_C@_07KIFHAGIL@SM_NAME@  00000001800604a8     flags.obj
 0002:0000a4b0       ??_C@_0M@OAFEBGNH@SM_FULLNAME@ 00000001800604b0     flags.obj
 0002:0000a4bc       ??_C@_06GJJJNNFE@SM_EXT@   00000001800604bc     flags.obj
 0002:0000a4c8       ??_C@_08FICJBKFN@SM_MTIME@ 00000001800604c8     flags.obj
 0002:0000a4d8       ??_C@_08GCCDHLCN@SM_CTIME@ 00000001800604d8     flags.obj
 0002:0000a4e8       ??_C@_08CPOLNKCG@SM_ATIME@ 00000001800604e8     flags.obj
 0002:0000a4f8       ??_C@_07OMPKMIKC@SM_SIZE@  00000001800604f8     flags.obj
 0002:0000a500       ??_C@_08BCBPOLMA@SM_DESCR@ 0000000180060500     flags.obj
 0002:0000a510       ??_C@_08MEAGCMBB@SM_OWNER@ 0000000180060510     flags.obj
 0002:0000a520       ??_C@_0BC@NKDBNAHD@SM_COMPRESSEDSIZE@ 0000000180060520     flags.obj
 0002:0000a538       ??_C@_0M@PKNLKFI@SM_NUMLINKS@ 0000000180060538     flags.obj
 0002:0000a548       ??_C@_0O@CCKEKPHL@SM_NUMSTREAMS@ 0000000180060548     flags.obj
 0002:0000a558       ??_C@_0P@PKGMDPMD@SM_STREAMSSIZE@ 0000000180060558     flags.obj
 0002:0000a568       ??_C@_0M@KALDNPOO@SM_NAMEONLY@ 0000000180060568     flags.obj
 0002:0000a578       ??_C@_09KFKGJDHC@SM_CHTIME@ 0000000180060578     flags.obj
 0002:0000a588       ??_C@_08DOEDKINA@SM_COUNT@ 0000000180060588     flags.obj
 0002:0000a598       ??_C@_07EOOHOKCC@SM_USER@  0000000180060598     flags.obj
 0002:0000a5a0       ??_C@_0P@FEMAMJLE@EEC_OPEN_ERROR@ 00000001800605a0     flags.obj
 0002:0000a5b0       ??_C@_0N@GLMELIKF@EEC_MODIFIED@ 00000001800605b0     flags.obj
 0002:0000a5c0       ??_C@_0BB@HALKEFOL@EEC_NOT_MODIFIED@ 00000001800605c0     flags.obj
 0002:0000a5d8       ??_C@_0BI@CNPFKHKO@EEC_LOADING_INTERRUPTED@ 00000001800605d8     flags.obj
 0002:0000a5f0       ??_C@_0BK@PHBCABMB@ACTL_GETFARMANAGERVERSION@ 00000001800605f0     flags.obj
 0002:0000a610       ??_C@_0N@DPABJDML@ACTL_WAITKEY@ 0000000180060610     flags.obj
 0002:0000a620       ??_C@_0O@CEHHJAFD@ACTL_GETCOLOR@ 0000000180060620     flags.obj
 0002:0000a630       ??_C@_0BD@OKPAACIK@ACTL_GETARRAYCOLOR@ 0000000180060630     flags.obj
 0002:0000a648       ??_C@_0BD@DIFEEKNN@ACTL_GETWINDOWINFO@ 0000000180060648     flags.obj
 0002:0000a660       ??_C@_0BE@PJBIPKOD@ACTL_GETWINDOWCOUNT@ 0000000180060660     flags.obj
 0002:0000a678       ??_C@_0BG@MNKPOEEN@ACTL_SETCURRENTWINDOW@ 0000000180060678     flags.obj
 0002:0000a690       ??_C@_0M@IHHFGPPA@ACTL_COMMIT@ 0000000180060690     flags.obj
 0002:0000a6a0       ??_C@_0BA@CLHFKJJP@ACTL_GETFARHWND@ 00000001800606a0     flags.obj
 0002:0000a6b0       ??_C@_0BD@JFOOLBPN@ACTL_SETARRAYCOLOR@ 00000001800606b0     flags.obj
 0002:0000a6c8       ??_C@_0P@JECKFIA@ACTL_REDRAWALL@ 00000001800606c8     flags.obj
 0002:0000a6d8       ??_C@_0N@DHPLJLHO@ACTL_SYNCHRO@ 00000001800606d8     flags.obj
 0002:0000a6e8       ??_C@_0BG@IJPADENB@ACTL_SETPROGRESSSTATE@ 00000001800606e8     flags.obj
 0002:0000a700       ??_C@_0BG@ICJFAPHK@ACTL_SETPROGRESSVALUE@ 0000000180060700     flags.obj
 0002:0000a718       ??_C@_09HNDBKLDC@ACTL_QUIT@ 0000000180060718     flags.obj
 0002:0000a728       ??_C@_0BA@LJCPDIKK@ACTL_GETFARRECT@ 0000000180060728     flags.obj
 0002:0000a738       ??_C@_0BC@FELBEIDG@ACTL_GETCURSORPOS@ 0000000180060738     flags.obj
 0002:0000a750       ??_C@_0BC@CAAPIEHK@ACTL_SETCURSORPOS@ 0000000180060750     flags.obj
 0002:0000a768       ??_C@_0BE@NPJGMDBM@ACTL_PROGRESSNOTIFY@ 0000000180060768     flags.obj
 0002:0000a780       ??_C@_0BD@IPKOEBIA@ACTL_GETWINDOWTYPE@ 0000000180060780     flags.obj
 0002:0000a798       ??_C@_09CEDFMINA@MSSC_POST@ 0000000180060798     flags.obj
 0002:0000a7a8       ??_C@_0L@MOADGAEB@MSSC_CHECK@ 00000001800607a8     flags.obj
 0002:0000a7b8       ??_C@_0BA@MMOAIEKP@MACROAREA_OTHER@ 00000001800607b8     flags.obj
 0002:0000a7c8       ??_C@_0BA@DEBOOAEB@MACROAREA_SHELL@ 00000001800607c8     flags.obj
 0002:0000a7d8       ??_C@_0BB@JIMPEHCD@MACROAREA_VIEWER@ 00000001800607d8     flags.obj
 0002:0000a7f0       ??_C@_0BB@KILFBFJH@MACROAREA_EDITOR@ 00000001800607f0     flags.obj
 0002:0000a808       ??_C@_0BB@CADENPFI@MACROAREA_DIALOG@ 0000000180060808     flags.obj
 0002:0000a820       ??_C@_0BB@MLMLHIGE@MACROAREA_SEARCH@ 0000000180060820     flags.obj
 0002:0000a838       ??_C@_0BA@KKMKOLIK@MACROAREA_DISKS@ 0000000180060838     flags.obj
 0002:0000a848       ??_C@_0BD@IGOOIJP@MACROAREA_MAINMENU@ 0000000180060848     flags.obj
 0002:0000a860       ??_C@_0P@LFLMAHBF@MACROAREA_MENU@ 0000000180060860     flags.obj
 0002:0000a870       ??_C@_0P@DKPKIEO@MACROAREA_HELP@ 0000000180060870     flags.obj
 0002:0000a880       ??_C@_0BE@MDJPICHC@MACROAREA_INFOPANEL@ 0000000180060880     flags.obj
 0002:0000a898       ??_C@_0BF@NLJMHMPP@MACROAREA_QVIEWPANEL@ 0000000180060898     flags.obj
 0002:0000a8b0       ??_C@_0BE@HBMEGBOC@MACROAREA_TREEPANEL@ 00000001800608b0     flags.obj
 0002:0000a8c8       ??_C@_0BF@FCHKCGLL@MACROAREA_FINDFOLDER@ 00000001800608c8     flags.obj
 0002:0000a8e0       ??_C@_0BD@JCFMJGDE@MACROAREA_USERMENU@ 00000001800608e0     flags.obj
 0002:0000a8f8       ??_C@_0BO@OMLEPJPM@MACROAREA_SHELLAUTOCOMPLETION@ 00000001800608f8     flags.obj
 0002:0000a918       ??_C@_0BP@OIHAIGBK@MACROAREA_DIALOGAUTOCOMPLETION@ 0000000180060918     flags.obj
 0002:0000a938       ??_C@_0BC@EIJFKPMK@MACROAREA_GRABBER@ 0000000180060938     flags.obj
 0002:0000a950       ??_C@_0BC@GNLOCEJP@MACROAREA_DESKTOP@ 0000000180060950     flags.obj
 0002:0000a968       ??_C@_0BB@JPEEDDOG@MACROAREA_COMMON@ 0000000180060968     flags.obj
 0002:0000a980       ??_C@_0BD@DIKEKAIJ@MACROSTATE_NOMACRO@ 0000000180060980     flags.obj
 0002:0000a998       ??_C@_0BF@PCDEFEGP@MACROSTATE_EXECUTING@ 0000000180060998     flags.obj
 0002:0000a9b0       ??_C@_0BM@EJOFDENO@MACROSTATE_EXECUTING_COMMON@ 00000001800609b0     flags.obj
 0002:0000a9d0       ??_C@_0BF@BGODKPBB@MACROSTATE_RECORDING@ 00000001800609d0     flags.obj
 0002:0000a9e8       ??_C@_0BM@OICPADFE@MACROSTATE_RECORDING_COMMON@ 00000001800609e8     flags.obj
 0002:0000aa08       ??_C@_0N@CGFFMLBC@MPEC_SUCCESS@ 0000000180060a08     flags.obj
 0002:0000aa18       ??_C@_0L@FJDDLDNN@MPEC_ERROR@ 0000000180060a18     flags.obj
 0002:0000aa28       ??_C@_0N@IBOAADDD@FMVT_UNKNOWN@ 0000000180060a28     flags.obj
 0002:0000aa38       ??_C@_0N@BDMFKEKE@FMVT_INTEGER@ 0000000180060a38     flags.obj
 0002:0000aa48       ??_C@_0M@LFMLDDKI@FMVT_STRING@ 0000000180060a48     flags.obj
 0002:0000aa58       ??_C@_0M@CKDAIOEN@FMVT_DOUBLE@ 0000000180060a58     flags.obj
 0002:0000aa68       ??_C@_0N@MHKOBOGF@FMVT_BOOLEAN@ 0000000180060a68     flags.obj
 0002:0000aa78       ??_C@_0M@GKPDICDA@FMVT_BINARY@ 0000000180060a78     flags.obj
 0002:0000aa88       ??_C@_0N@FMHCFNDF@FMVT_POINTER@ 0000000180060a88     flags.obj
 0002:0000aa98       ??_C@_08DDPDBBNO@FMVT_NIL@ 0000000180060a98     flags.obj
 0002:0000aaa8       ??_C@_0L@DJIKMOJA@FMVT_ARRAY@ 0000000180060aa8     flags.obj
 0002:0000aab8       ??_C@_0L@PMDDFEBD@FMVT_PANEL@ 0000000180060ab8     flags.obj
 0002:0000aac8       ??_C@_0L@ELHBHIEH@FMVT_ERROR@ 0000000180060ac8     flags.obj
 0002:0000aad8       ??_C@_0O@OGHFLIKM@WTYPE_UNKNOWN@ 0000000180060ad8     flags.obj
 0002:0000aae8       ??_C@_0O@DCGKMPOM@WTYPE_DESKTOP@ 0000000180060ae8     flags.obj
 0002:0000aaf8       ??_C@_0N@FNCFCPIG@WTYPE_PANELS@ 0000000180060af8     flags.obj
 0002:0000ab08       ??_C@_0N@EJKMDMBK@WTYPE_VIEWER@ 0000000180060b08     flags.obj
 0002:0000ab18       ??_C@_0N@HJNGGOKO@WTYPE_EDITOR@ 0000000180060b18     flags.obj
 0002:0000ab28       ??_C@_0N@PBFHKEGB@WTYPE_DIALOG@ 0000000180060b28     flags.obj
 0002:0000ab38       ??_C@_0M@OMKLELFA@WTYPE_VMENU@ 0000000180060b38     flags.obj
 0002:0000ab48       ??_C@_0L@BCEMNGOG@WTYPE_HELP@ 0000000180060b48     flags.obj
 0002:0000ab58       ??_C@_0P@MMIDEOJJ@WTYPE_COMBOBOX@ 0000000180060b58     flags.obj
 0002:0000ab68       ??_C@_0O@BHEBEELJ@WTYPE_GRABBER@ 0000000180060b68     flags.obj
 0002:0000ab78       ??_C@_0M@NFHHCILL@WTYPE_HMENU@ 0000000180060b78     flags.obj
 0002:0000ab88       ??_C@_0BA@IPEAOBGN@TBPS_NOPROGRESS@ 0000000180060b88     flags.obj
 0002:0000ab98       ??_C@_0BD@HMEHMDAL@TBPS_INDETERMINATE@ 0000000180060b98     flags.obj
 0002:0000abb0       ??_C@_0M@KHLNKPHE@TBPS_NORMAL@ 0000000180060bb0     flags.obj
 0002:0000abc0       ??_C@_0L@DFDPCOFD@TBPS_ERROR@ 0000000180060bc0     flags.obj
 0002:0000abd0       ??_C@_0M@GHGAPHPP@TBPS_PAUSED@ 0000000180060bd0     flags.obj
 0002:0000abe0       ??_C@_0O@MCNCFBLF@VSMT_VIEWMODE@ 0000000180060be0     flags.obj
 0002:0000abf0       ??_C@_09FLKONCNO@VSMT_WRAP@ 0000000180060bf0     flags.obj
 0002:0000ac00       ??_C@_0O@INKALKJK@VSMT_WORDWRAP@ 0000000180060c00     flags.obj
 0002:0000ac10       ??_C@_08FNEFFFEL@VMT_TEXT@ 0000000180060c10     flags.obj
 0002:0000ac20       ??_C@_07FLIHDEDA@VMT_HEX@  0000000180060c20     flags.obj
 0002:0000ac28       ??_C@_08BDDNDBMJ@VMT_DUMP@ 0000000180060c28     flags.obj
 0002:0000ac38       ??_C@_07OJCLGDHJ@VE_READ@  0000000180060c38     flags.obj
 0002:0000ac40       ??_C@_08JIBCCIDC@VE_CLOSE@ 0000000180060c40     flags.obj
 0002:0000ac50       ??_C@_0M@FEFKOOMJ@VE_GOTFOCUS@ 0000000180060c50     flags.obj
 0002:0000ac60       ??_C@_0N@ICHCAKIB@VE_KILLFOCUS@ 0000000180060c60     flags.obj
 0002:0000ac70       ??_C@_07BLBPFFLB@EE_READ@  0000000180060c70     flags.obj
 0002:0000ac78       ??_C@_07KJGPGPOC@EE_SAVE@  0000000180060c78     flags.obj
 0002:0000ac80       ??_C@_09NPOPIKMK@EE_REDRAW@ 0000000180060c80     flags.obj
 0002:0000ac90       ??_C@_08NFPFGIG@EE_CLOSE@  0000000180060c90     flags.obj
 0002:0000aca0       ??_C@_0M@CPNMNBMF@EE_GOTFOCUS@ 0000000180060ca0     flags.obj
 0002:0000acb0       ??_C@_0N@ILLPMAJF@EE_KILLFOCUS@ 0000000180060cb0     flags.obj
 0002:0000acc0       ??_C@_09MIOGFFI@EE_CHANGE@ 0000000180060cc0     flags.obj
 0002:0000acd0       ??_C@_0P@MBHAHBBG@DE_DLGPROCINIT@ 0000000180060cd0     flags.obj
 0002:0000ace0       ??_C@_0BC@BMFEJAMO@DE_DEFDLGPROCINIT@ 0000000180060ce0     flags.obj
 0002:0000acf8       ??_C@_0O@ICBCOJCG@DE_DLGPROCEND@ 0000000180060cf8     flags.obj
 0002:0000ad08       ??_C@_0BB@MNODJNPE@SE_COMMONSYNCHRO@ 0000000180060d08     flags.obj
 0002:0000ad20       ??_C@_0N@HKGMPMJE@ESPT_TABSIZE@ 0000000180060d20     flags.obj
 0002:0000ad30       ??_C@_0BA@GOKHPFCK@ESPT_EXPANDTABS@ 0000000180060d30     flags.obj
 0002:0000ad40       ??_C@_0BA@KOADDMLI@ESPT_AUTOINDENT@ 0000000180060d40     flags.obj
 0002:0000ad50       ??_C@_0BF@LPNONOMF@ESPT_CURSORBEYONDEOL@ 0000000180060d50     flags.obj
 0002:0000ad68       ??_C@_0BC@OECOCGLJ@ESPT_CHARCODEBASE@ 0000000180060d68     flags.obj
 0002:0000ad80       ??_C@_0O@PIAOJINE@ESPT_CODEPAGE@ 0000000180060d80     flags.obj
 0002:0000ad90       ??_C@_0BG@HAPABMJH@ESPT_SAVEFILEPOSITION@ 0000000180060d90     flags.obj
 0002:0000ada8       ??_C@_0O@KCPDJCKC@ESPT_LOCKMODE@ 0000000180060da8     flags.obj
 0002:0000adb8       ??_C@_0BA@EIGIAOHM@ESPT_SETWORDDIV@ 0000000180060db8     flags.obj
 0002:0000adc8       ??_C@_0BA@FGEHLJDF@ESPT_GETWORDDIV@ 0000000180060dc8     flags.obj
 0002:0000add8       ??_C@_0BE@MACJBCFP@ESPT_SHOWWHITESPACE@ 0000000180060dd8     flags.obj
 0002:0000adf0       ??_C@_0M@FICNFPPA@ESPT_SETBOM@ 0000000180060df0     flags.obj
 0002:0000ae00       ??_C@_09FLEMPKKP@EUR_BEGIN@ 0000000180060e00     flags.obj
 0002:0000ae10       ??_C@_07DDJDFJCN@EUR_END@  0000000180060e10     flags.obj
 0002:0000ae18       ??_C@_08FCONALGE@EUR_UNDO@ 0000000180060e18     flags.obj
 0002:0000ae28       ??_C@_08DHMMFAHF@EUR_REDO@ 0000000180060e28     flags.obj
 0002:0000ae38       ??_C@_0O@PKOIFEBO@EXPAND_NOTABS@ 0000000180060e38     flags.obj
 0002:0000ae48       ??_C@_0P@MLHPCNDM@EXPAND_ALLTABS@ 0000000180060e48     flags.obj
 0002:0000ae58       ??_C@_0P@OONGIIBL@EXPAND_NEWTABS@ 0000000180060e58     flags.obj
 0002:0000ae68       ??_C@_0BD@DKHPEOHH@EOPT_EXPANDALLTABS@ 0000000180060e68     flags.obj
 0002:0000ae80       ??_C@_0BG@BOINMDEK@EOPT_PERSISTENTBLOCKS@ 0000000180060e80     flags.obj
 0002:0000ae98       ??_C@_0BG@PIIHHCAN@EOPT_DELREMOVESBLOCKS@ 0000000180060e98     flags.obj
 0002:0000aeb0       ??_C@_0BA@KPJEAKBD@EOPT_AUTOINDENT@ 0000000180060eb0     flags.obj
 0002:0000aec0       ??_C@_0BG@MBPADLG@EOPT_SAVEFILEPOSITION@ 0000000180060ec0     flags.obj
 0002:0000aed8       ??_C@_0BI@PFHCGCAI@EOPT_AUTODETECTCODEPAGE@ 0000000180060ed8     flags.obj
 0002:0000aef0       ??_C@_0BF@IMCOEIAL@EOPT_CURSORBEYONDEOL@ 0000000180060ef0     flags.obj
 0002:0000af08       ??_C@_0BH@CJPAGGLC@EOPT_EXPANDONLYNEWTABS@ 0000000180060f08     flags.obj
 0002:0000af20       ??_C@_0BE@DDKCDJDC@EOPT_SHOWWHITESPACE@ 0000000180060f20     flags.obj
 0002:0000af38       ??_C@_08HMMLONBH@EOPT_BOM@ 0000000180060f38     flags.obj
 0002:0000af48       ??_C@_0BD@CLLAKGOA@EOPT_SHOWLINEBREAK@ 0000000180060f48     flags.obj
 0002:0000af60       ??_C@_0BC@JCJEPKEC@EOPT_SHOWTITLEBAR@ 0000000180060f60     flags.obj
 0002:0000af78       ??_C@_0BA@KPGMOBKI@EOPT_SHOWKEYBAR@ 0000000180060f78     flags.obj
 0002:0000af88       ??_C@_0BD@EFCFEAD@EOPT_SHOWSCROLLBAR@ 0000000180060f88     flags.obj
 0002:0000afa0       ??_C@_0L@BJCBJJNB@BTYPE_NONE@ 0000000180060fa0     flags.obj
 0002:0000afb0       ??_C@_0N@OPHHGFPF@BTYPE_STREAM@ 0000000180060fb0     flags.obj
 0002:0000afc0       ??_C@_0N@EMEGNPLI@BTYPE_COLUMN@ 0000000180060fc0     flags.obj
 0002:0000afd0       ??_C@_0BB@BNPDAPGB@ECSTATE_MODIFIED@ 0000000180060fd0     flags.obj
 0002:0000afe8       ??_C@_0O@GBBGHDFM@ECSTATE_SAVED@ 0000000180060fe8     flags.obj
 0002:0000aff8       ??_C@_0P@BECIAJAM@ECSTATE_LOCKED@ 0000000180060ff8     flags.obj
 0002:0000b008       ??_C@_0P@DOBJCNIG@ECTYPE_CHANGED@ 0000000180061008     flags.obj
 0002:0000b018       ??_C@_0N@MDEFMEEA@ECTYPE_ADDED@ 0000000180061018     flags.obj
 0002:0000b028       ??_C@_0P@NMOJJPOB@ECTYPE_DELETED@ 0000000180061028     flags.obj
 0002:0000b038       ??_C@_08HHHKLJPB@PLT_PATH@ 0000000180061038     flags.obj
 0002:0000b048       ??_C@_08KBAMIIFB@PFM_GUID@ 0000000180061048     flags.obj
 0002:0000b058       ??_C@_0P@KKEMMPNI@PFM_MODULENAME@ 0000000180061058     flags.obj
 0002:0000b068       ??_C@_09BOODOHKD@FFT_PANEL@ 0000000180061068     flags.obj
 0002:0000b078       ??_C@_0N@GMEDAGNH@FFT_FINDFILE@ 0000000180061078     flags.obj
 0002:0000b088       ??_C@_08KKCPIPGP@FFT_COPY@ 0000000180061088     flags.obj
 0002:0000b098       ??_C@_0L@EKPDMFDD@FFT_SELECT@ 0000000180061098     flags.obj
 0002:0000b0a8       ??_C@_0L@LGPEDLLD@FFT_CUSTOM@ 00000001800610a8     flags.obj
 0002:0000b0b8       ??_C@_0M@OIOMMFOE@FST_UNKNOWN@ 00000001800610b8     flags.obj
 0002:0000b0c8       ??_C@_0L@GGGOEGKJ@FST_SUBKEY@ 00000001800610c8     flags.obj
 0002:0000b0d8       ??_C@_09LFEEAJIC@FST_QWORD@ 00000001800610d8     flags.obj
 0002:0000b0e8       ??_C@_0L@LPMPBKDL@FST_STRING@ 00000001800610e8     flags.obj
 0002:0000b0f8       ??_C@_08EJJJCLIG@FST_DATA@ 00000001800610f8     flags.obj
 0002:0000b108       ??_C@_09OBBBBFPE@FSSF_ROOT@ 0000000180061108     flags.obj
 0002:0000b118       ??_C@_0BB@HDKCPBIO@FSSF_HISTORY_CMD@ 0000000180061118     flags.obj
 0002:0000b130       ??_C@_0BE@BLPOFODL@FSSF_HISTORY_FOLDER@ 0000000180061130     flags.obj
 0002:0000b148       ??_C@_0BC@NJCJCCNH@FSSF_HISTORY_VIEW@ 0000000180061148     flags.obj
 0002:0000b160       ??_C@_0BC@CODELNPP@FSSF_HISTORY_EDIT@ 0000000180061160     flags.obj
 0002:0000b178       ??_C@_0BG@IFGEMJIF@FSSF_HISTORY_EXTERNAL@ 0000000180061178     flags.obj
 0002:0000b190       ??_C@_0BG@DGAKDKFK@FSSF_FOLDERSHORTCUT_0@ 0000000180061190     flags.obj
 0002:0000b1a8       ??_C@_0BG@CPBBALBL@FSSF_FOLDERSHORTCUT_1@ 00000001800611a8     flags.obj
 0002:0000b1c0       ??_C@_0BG@EDMFINI@FSSF_FOLDERSHORTCUT_2@ 00000001800611c0     flags.obj
 0002:0000b1d8       ??_C@_0BG@BNCHGJJJ@FSSF_FOLDERSHORTCUT_3@ 00000001800611d8     flags.obj
 0002:0000b1f0       ??_C@_0BG@FCGGPPFO@FSSF_FOLDERSHORTCUT_4@ 00000001800611f0     flags.obj
 0002:0000b208       ??_C@_0BG@ELHNMOBP@FSSF_FOLDERSHORTCUT_5@ 0000000180061208     flags.obj
 0002:0000b220       ??_C@_0BG@GAFAJNNM@FSSF_FOLDERSHORTCUT_6@ 0000000180061220     flags.obj
 0002:0000b238       ??_C@_0BG@HJELKMJN@FSSF_FOLDERSHORTCUT_7@ 0000000180061238     flags.obj
 0002:0000b250       ??_C@_0BG@PONDLAFC@FSSF_FOLDERSHORTCUT_8@ 0000000180061250     flags.obj
 0002:0000b268       ??_C@_0BG@OHMIIBBD@FSSF_FOLDERSHORTCUT_9@ 0000000180061268     flags.obj
 0002:0000b280       ??_C@_0BD@PBIEGEHP@FSSF_CONFIRMATIONS@ 0000000180061280     flags.obj
 0002:0000b298       ??_C@_0M@PIGDMPJB@FSSF_SYSTEM@ 0000000180061298     flags.obj
 0002:0000b2a8       ??_C@_0L@LBFNJGFB@FSSF_PANEL@ 00000001800612a8     flags.obj
 0002:0000b2b8       ??_C@_0M@KJLIHDEL@FSSF_EDITOR@ 00000001800612b8     flags.obj
 0002:0000b2c8       ??_C@_0M@KEMGKEOF@FSSF_SCREEN@ 00000001800612c8     flags.obj
 0002:0000b2d8       ??_C@_0M@CBDJLJIE@FSSF_DIALOG@ 00000001800612d8     flags.obj
 0002:0000b2e8       ??_C@_0P@OCDADNBF@FSSF_INTERFACE@ 00000001800612e8     flags.obj
 0002:0000b2f8       ??_C@_0BB@GBBEBNKE@FSSF_PANELLAYOUT@ 00000001800612f8     flags.obj
 0002:0000b310       ??_C@_0M@JCGHGLJF@PSL_ROAMING@ 0000000180061310     flags.obj
 0002:0000b320       ??_C@_09EDBNDHCM@PSL_LOCAL@ 0000000180061320     flags.obj
 0002:0000b330       ??_C@_07BPEFOPGM@FCT_ANY@  0000000180061330     flags.obj
 0002:0000b338       ??_C@_0L@CDAEILNM@FCT_STREAM@ 0000000180061338     flags.obj
 0002:0000b348       ??_C@_0L@IADFDBJB@FCT_COLUMN@ 0000000180061348     flags.obj
 0002:0000b358       ??_C@_0O@KJFMBLFE@LINK_HARDLINK@ 0000000180061358     flags.obj
 0002:0000b368       ??_C@_0O@OOAFIIDA@LINK_JUNCTION@ 0000000180061368     flags.obj
 0002:0000b378       ??_C@_0O@FIAPLKLH@LINK_VOLMOUNT@ 0000000180061378     flags.obj
 0002:0000b388       ??_C@_0BB@JDBEPJDK@LINK_SYMLINKFILE@ 0000000180061388     flags.obj
 0002:0000b3a0       ??_C@_0BA@GFPIOFMG@LINK_SYMLINKDIR@ 00000001800613a0     flags.obj
 0002:0000b3b0       ??_C@_0N@PJENIJFN@LINK_SYMLINK@ 00000001800613b0     flags.obj
 0002:0000b3c0       ??_C@_08HNOHKPBK@CPM_FULL@ 00000001800613c0     flags.obj
 0002:0000b3d0       ??_C@_08LAEGFKJE@CPM_REAL@ 00000001800613d0     flags.obj
 0002:0000b3e0       ??_C@_0L@NPJNPCJM@CPM_NATIVE@ 00000001800613e0     flags.obj
 0002:0000b3f0       ??_C@_0L@NCFOENCC@VS_RELEASE@ 00000001800613f0     flags.obj
 0002:0000b400       ??_C@_08BDGLHPMJ@VS_ALPHA@ 0000000180061400     flags.obj
 0002:0000b410       ??_C@_07OKFPMINB@VS_BETA@  0000000180061410     flags.obj
 0002:0000b418       ??_C@_05MMFLPJEB@VS_RC@    0000000180061418     flags.obj
 0002:0000b420       ??_C@_0L@IIIJLOAF@VS_SPECIAL@ 0000000180061420     flags.obj
 0002:0000b430       ??_C@_0L@EAMAICHL@VS_PRIVATE@ 0000000180061430     flags.obj
 0002:0000b440       ??_C@_0BC@OOKLINPG@OPEN_LEFTDISKMENU@ 0000000180061440     flags.obj
 0002:0000b458       ??_C@_0BB@CEFDHHLF@OPEN_PLUGINSMENU@ 0000000180061458     flags.obj
 0002:0000b470       ??_C@_0O@IEJHJCNB@OPEN_FINDLIST@ 0000000180061470     flags.obj
 0002:0000b480       ??_C@_0O@OGDCDPNG@OPEN_SHORTCUT@ 0000000180061480     flags.obj
 0002:0000b490       ??_C@_0BB@JHCCMIPF@OPEN_COMMANDLINE@ 0000000180061490     flags.obj
 0002:0000b4a8       ??_C@_0M@DMJLHMGM@OPEN_EDITOR@ 00000001800614a8     flags.obj
 0002:0000b4b8       ??_C@_0M@MOBCONI@OPEN_VIEWER@ 00000001800614b8     flags.obj
 0002:0000b4c8       ??_C@_0P@LCDNLGDE@OPEN_FILEPANEL@ 00000001800614c8     flags.obj
 0002:0000b4d8       ??_C@_0M@LEBKLGKD@OPEN_DIALOG@ 00000001800614d8     flags.obj
 0002:0000b4e8       ??_C@_0N@CBHPGAKB@OPEN_ANALYSE@ 00000001800614e8     flags.obj
 0002:0000b4f8       ??_C@_0BD@NFNGGFHI@OPEN_RIGHTDISKMENU@ 00000001800614f8     flags.obj
 0002:0000b510       ??_C@_0P@FOKOAMLC@OPEN_FROMMACRO@ 0000000180061510     flags.obj
 0002:0000b520       ??_C@_0O@NEDDJIHC@OPEN_LUAMACRO@ 0000000180061520     flags.obj
 0002:0000b530       ??_C@_0P@GBMLNMMI@MCT_MACROPARSE@ 0000000180061530     flags.obj
 0002:0000b540       ??_C@_0P@GNPFPCF@MCT_LOADMACROS@ 0000000180061540     flags.obj
 0002:0000b550       ??_C@_0P@HMDDACMI@MCT_ENUMMACROS@ 0000000180061550     flags.obj
 0002:0000b560       ??_C@_0BA@MOCJHMJK@MCT_WRITEMACROS@ 0000000180061560     flags.obj
 0002:0000b570       ??_C@_0N@IGJGAHKE@MCT_GETMACRO@ 0000000180061570     flags.obj
 0002:0000b580       ??_C@_0BC@NFGGBILF@MCT_RECORDEDMACRO@ 0000000180061580     flags.obj
 0002:0000b598       ??_C@_0N@OLCKOJMI@MCT_DELMACRO@ 0000000180061598     flags.obj
 0002:0000b5a8       ??_C@_0BC@NALHIHJ@MCT_RUNSTARTMACRO@ 00000001800615a8     flags.obj
 0002:0000b5c0       ??_C@_0P@HOMHAEFB@MCT_EXECSTRING@ 00000001800615c0     flags.obj
 0002:0000b5d0       ??_C@_0O@CDBDPKIC@MCT_PANELSORT@ 00000001800615d0     flags.obj
 0002:0000b5e0       ??_C@_0BH@PKKJIOHM@MCT_GETCUSTOMSORTMODES@ 00000001800615e0     flags.obj
 0002:0000b5f8       ??_C@_0N@FOPIOCHO@MCT_ADDMACRO@ 00000001800615f8     flags.obj
 0002:0000b608       ??_C@_0N@BHFJFHA@MCT_KEYMACRO@ 0000000180061608     flags.obj
 0002:0000b618       ??_C@_0BB@LPDAOGB@MCT_CANPANELSORT@ 0000000180061618     flags.obj
 0002:0000b630       ??_C@_0BC@IOECJI@MPRT_NORMALFINISH@ 0000000180061630     flags.obj
 0002:0000b648       ??_C@_0BB@PMCBIGCA@MPRT_ERRORFINISH@ 0000000180061648     flags.obj
 0002:0000b660       ??_C@_0BA@BCBAEEOI@MPRT_ERRORPARSE@ 0000000180061660     flags.obj
 0002:0000b670       ??_C@_09EJDAADCN@MPRT_KEYS@ 0000000180061670     flags.obj
 0002:0000b680       ??_C@_0L@GEHHCKFA@MPRT_PRINT@ 0000000180061680     flags.obj
 0002:0000b690       ??_C@_0BA@OBIDLEIM@MPRT_PLUGINCALL@ 0000000180061690     flags.obj
 0002:0000b6a0       ??_C@_0BA@EJFFOAMM@MPRT_PLUGINMENU@ 00000001800616a0     flags.obj
 0002:0000b6b0       ??_C@_0BC@LEDOPMKI@MPRT_PLUGINCONFIG@ 00000001800616b0     flags.obj
 0002:0000b6c8       ??_C@_0BD@HHINMPPI@MPRT_PLUGINCOMMAND@ 00000001800616c8     flags.obj
 0002:0000b6e0       ??_C@_0O@IEMNLPAB@MPRT_USERMENU@ 00000001800616e0     flags.obj
 0002:0000b6f0       ??_C@_0BA@GEAFHJNF@MPRT_HASNOMACRO@ 00000001800616f0     flags.obj
 0002:0000b700       ??_C@_0BC@PNCKAHJO@FE_CHANGEVIEWMODE@ 0000000180061700     flags.obj
 0002:0000b718       ??_C@_09DENIDBMJ@FE_REDRAW@ 0000000180061718     flags.obj
 0002:0000b728       ??_C@_07CLNPDBLG@FE_IDLE@  0000000180061728     flags.obj
 0002:0000b730       ??_C@_08DENCGKED@FE_CLOSE@ 0000000180061730     flags.obj
 0002:0000b740       ??_C@_08MOMCCKPB@FE_BREAK@ 0000000180061740     flags.obj
 0002:0000b750       ??_C@_0L@LELAIPLL@FE_COMMAND@ 0000000180061750     flags.obj
 0002:0000b760       ??_C@_0M@FIECADDF@FE_GOTFOCUS@ 0000000180061760     flags.obj
 0002:0000b770       ??_C@_0N@DGHFKMFL@FE_KILLFOCUS@ 0000000180061770     flags.obj
 0002:0000b780       ??_C@_0BE@PONEECEM@FE_CHANGESORTPARAMS@ 0000000180061780     flags.obj
 0002:0000b798       ??_C@_0M@HNDHDHHO@FCF_FG_4BIT@ 0000000180061798     flags.obj
 0002:0000b7a8       ??_C@_0M@PJHNDJIE@FCF_BG_4BIT@ 00000001800617a8     flags.obj
 0002:0000b7b8       ??_C@_0N@HMKJBHOA@FCF_4BITMASK@ 00000001800617b8     flags.obj
 0002:0000b7c8       ??_C@_0BC@HCOAIAEK@FCF_INHERIT_STYLE@ 00000001800617c8     flags.obj
 0002:0000b7e0       ??_C@_0BB@PJFLJJLD@FCF_RAWATTR_MASK@ 00000001800617e0     flags.obj
 0002:0000b7f8       ??_C@_0M@LFMGCKHG@FCF_FG_BOLD@ 00000001800617f8     flags.obj
 0002:0000b808       ??_C@_0O@FAPDECBF@FCF_FG_ITALIC@ 0000000180061808     flags.obj
 0002:0000b818       ??_C@_0BB@NPEFGEGA@FCF_FG_UNDERLINE@ 0000000180061818     flags.obj
 0002:0000b830       ??_C@_0BC@KABNHAEN@FCF_FG_UNDERLINE2@ 0000000180061830     flags.obj
 0002:0000b848       ??_C@_0BA@DJMNLMK@FCF_FG_OVERLINE@ 0000000180061848     flags.obj
 0002:0000b858       ??_C@_0BB@NJMJIPGP@FCF_FG_STRIKEOUT@ 0000000180061858     flags.obj
 0002:0000b870       ??_C@_0N@HJOMADOA@FCF_FG_FAINT@ 0000000180061870     flags.obj
 0002:0000b880       ??_C@_0N@NHLHILNJ@FCF_FG_BLINK@ 0000000180061880     flags.obj
 0002:0000b890       ??_C@_0O@LGBGBIGB@FCF_STYLEMASK@ 0000000180061890     flags.obj
 0002:0000b8a0       ??_C@_08BKNBBLHK@FCF_NONE@ 00000001800618a0     flags.obj
 0002:0000b8b0       ??_C@_08FKIDFHCM@CDF_NONE@ 00000001800618b0     flags.obj
 0002:0000b8c0       ??_C@_0N@ELMEMNDH@FMSG_WARNING@ 00000001800618c0     flags.obj
 0002:0000b8d0       ??_C@_0P@HHIGLJAP@FMSG_ERRORTYPE@ 00000001800618d0     flags.obj
 0002:0000b8e0       ??_C@_0BE@FHOOILPH@FMSG_KEEPBACKGROUND@ 00000001800618e0     flags.obj
 0002:0000b8f8       ??_C@_0P@KBEMNNEP@FMSG_LEFTALIGN@ 00000001800618f8     flags.obj
 0002:0000b908       ??_C@_0O@FOIOKDHJ@FMSG_ALLINONE@ 0000000180061908     flags.obj
 0002:0000b918       ??_C@_0L@BGALGPOK@FMSG_MB_OK@ 0000000180061918     flags.obj
 0002:0000b928       ??_C@_0BB@JGAPGIEP@FMSG_MB_OKCANCEL@ 0000000180061928     flags.obj
 0002:0000b940       ??_C@_0BJ@BKJADAHA@FMSG_MB_ABORTRETRYIGNORE@ 0000000180061940     flags.obj
 0002:0000b960       ??_C@_0O@GPCAPHCL@FMSG_MB_YESNO@ 0000000180061960     flags.obj
 0002:0000b970       ??_C@_0BE@IBNOLCGP@FMSG_MB_YESNOCANCEL@ 0000000180061970     flags.obj
 0002:0000b988       ??_C@_0BE@OCLAIENB@FMSG_MB_RETRYCANCEL@ 0000000180061988     flags.obj
 0002:0000b9a0       ??_C@_09NEGPLEAH@FMSG_NONE@ 00000001800619a0     flags.obj
 0002:0000b9b0       ??_C@_0N@DHJCDIKM@DIF_BOXCOLOR@ 00000001800619b0     flags.obj
 0002:0000b9c0       ??_C@_09IAEPIICA@DIF_GROUP@ 00000001800619c0     flags.obj
 0002:0000b9d0       ??_C@_0N@GCKJNBCM@DIF_LEFTTEXT@ 00000001800619d0     flags.obj
 0002:0000b9e0       ??_C@_0P@BGPBEDHH@DIF_MOVESELECT@ 00000001800619e0     flags.obj
 0002:0000b9f0       ??_C@_0BC@PDKFKKEI@DIF_SHOWAMPERSAND@ 00000001800619f0     flags.obj
 0002:0000ba08       ??_C@_0BA@BLCOKAAO@DIF_CENTERGROUP@ 0000000180061a08     flags.obj
 0002:0000ba18       ??_C@_0P@MKFBJPOB@DIF_NOBRACKETS@ 0000000180061a18     flags.obj
 0002:0000ba28       ??_C@_0BF@JBCDBJCL@DIF_MANUALADDHISTORY@ 0000000180061a28     flags.obj
 0002:0000ba40       ??_C@_0O@JKNMBNLA@DIF_SEPARATOR@ 0000000180061a40     flags.obj
 0002:0000ba50       ??_C@_0P@CGILDLOA@DIF_SEPARATOR2@ 0000000180061a50     flags.obj
 0002:0000ba60       ??_C@_0L@NBPFNGLB@DIF_EDITOR@ 0000000180061a60     flags.obj
 0002:0000ba70       ??_C@_0BE@PFICAGJF@DIF_LISTNOAMPERSAND@ 0000000180061a70     flags.obj
 0002:0000ba88       ??_C@_0O@FFJNBMAD@DIF_LISTNOBOX@ 0000000180061a88     flags.obj
 0002:0000ba98       ??_C@_0M@IPFBMFDN@DIF_HISTORY@ 0000000180061a98     flags.obj
 0002:0000baa8       ??_C@_0P@EGFAEEDC@DIF_BTNNOCLOSE@ 0000000180061aa8     flags.obj
 0002:0000bab8       ??_C@_0P@KOJCCCGB@DIF_CENTERTEXT@ 0000000180061ab8     flags.obj
 0002:0000bac8       ??_C@_0BC@ODEMBOPK@DIF_SEPARATORUSER@ 0000000180061ac8     flags.obj
 0002:0000bae0       ??_C@_0O@IKJBMPOF@DIF_SETSHIELD@ 0000000180061ae0     flags.obj
 0002:0000baf0       ??_C@_0P@EEJEDBLH@DIF_EDITEXPAND@ 0000000180061af0     flags.obj
 0002:0000bb00       ??_C@_0BB@EIMEKEFP@DIF_DROPDOWNLIST@ 0000000180061b00     flags.obj
 0002:0000bb18       ??_C@_0BD@MNGIOLFF@DIF_USELASTHISTORY@ 0000000180061b18     flags.obj
 0002:0000bb30       ??_C@_0N@MOCGNIKC@DIF_MASKEDIT@ 0000000180061b30     flags.obj
 0002:0000bb40       ??_C@_0BD@LPDHCLJI@DIF_LISTTRACKMOUSE@ 0000000180061b40     flags.obj
 0002:0000bb58       ??_C@_0BK@LEFIBDOA@DIF_LISTTRACKMOUSEINFOCUS@ 0000000180061b58     flags.obj
 0002:0000bb78       ??_C@_0BC@JNLDMGBD@DIF_SELECTONENTRY@ 0000000180061b78     flags.obj
 0002:0000bb90       ??_C@_0L@KKNJDNBK@DIF_3STATE@ 0000000180061b90     flags.obj
 0002:0000bba0       ??_C@_0N@GBGHICKO@DIF_EDITPATH@ 0000000180061ba0     flags.obj
 0002:0000bbb0       ??_C@_0BB@NPNALIGO@DIF_LISTWRAPMODE@ 0000000180061bb0     flags.obj
 0002:0000bbc8       ??_C@_0BD@MFOKKGGF@DIF_NOAUTOCOMPLETE@ 0000000180061bc8     flags.obj
 0002:0000bbe0       ??_C@_0BG@MONEJILE@DIF_LISTAUTOHIGHLIGHT@ 0000000180061be0     flags.obj
 0002:0000bbf8       ??_C@_0BA@JNOKLHOL@DIF_LISTNOCLOSE@ 0000000180061bf8     flags.obj
 0002:0000bc08       ??_C@_0BB@GMKDKOOP@DIF_EDITPATHEXEC@ 0000000180061c08     flags.obj
 0002:0000bc20       ??_C@_0L@EPNFOPAK@DIF_HIDDEN@ 0000000180061c20     flags.obj
 0002:0000bc30       ??_C@_0N@KOGKCAKJ@DIF_READONLY@ 0000000180061c30     flags.obj
 0002:0000bc40       ??_C@_0M@NLLDINIM@DIF_NOFOCUS@ 0000000180061c40     flags.obj
 0002:0000bc50       ??_C@_0M@HCFLMDHK@DIF_DISABLE@ 0000000180061c50     flags.obj
 0002:0000bc60       ??_C@_0BC@CHAAKEJO@DIF_DEFAULTBUTTON@ 0000000180061c60     flags.obj
 0002:0000bc78       ??_C@_09LCJIOEMN@DIF_FOCUS@ 0000000180061c78     flags.obj
 0002:0000bc88       ??_C@_0O@KJADCBBN@DIF_RIGHTTEXT@ 0000000180061c88     flags.obj
 0002:0000bc98       ??_C@_0N@LAEOODAD@DIF_WORDWRAP@ 0000000180061c98     flags.obj
 0002:0000bca8       ??_C@_08KFOHCPDE@DIF_NONE@ 0000000180061ca8     flags.obj
 0002:0000bcb8       ??_C@_0N@EDHAFIIL@LIF_SELECTED@ 0000000180061cb8     flags.obj
 0002:0000bcc8       ??_C@_0M@BMGIEAIL@LIF_CHECKED@ 0000000180061cc8     flags.obj
 0002:0000bcd8       ??_C@_0O@KJIFADIG@LIF_SEPARATOR@ 0000000180061cd8     flags.obj
 0002:0000bce8       ??_C@_0M@HEFHLFIE@LIF_DISABLE@ 0000000180061ce8     flags.obj
 0002:0000bcf8       ??_C@_0L@PKDDGEEG@LIF_GRAYED@ 0000000180061cf8     flags.obj
 0002:0000bd08       ??_C@_0L@PFBGAOEP@LIF_HIDDEN@ 0000000180061d08     flags.obj
 0002:0000bd18       ??_C@_0BD@HEPCOIEH@LIF_DELETEUSERDATA@ 0000000180061d18     flags.obj
 0002:0000bd30       ??_C@_08BODPINCM@LIF_NONE@ 0000000180061d30     flags.obj
 0002:0000bd40       ??_C@_0BC@BGAENNBJ@LIFIND_EXACTMATCH@ 0000000180061d40     flags.obj
 0002:0000bd58       ??_C@_0M@FPOGKIGO@LIFIND_NONE@ 0000000180061d58     flags.obj
 0002:0000bd68       ??_C@_0BA@OOIEKCFB@LINFO_SHOWNOBOX@ 0000000180061d68     flags.obj
 0002:0000bd78       ??_C@_0BE@DECCEGNO@LINFO_AUTOHIGHLIGHT@ 0000000180061d78     flags.obj
 0002:0000bd90       ??_C@_0BH@BADLEILJ@LINFO_REVERSEHIGHLIGHT@ 0000000180061d90     flags.obj
 0002:0000bda8       ??_C@_0P@KLBMHNCG@LINFO_WRAPMODE@ 0000000180061da8     flags.obj
 0002:0000bdb8       ??_C@_0BE@OHJCOKAE@LINFO_SHOWAMPERSAND@ 0000000180061db8     flags.obj
 0002:0000bdd0       ??_C@_0L@EPACPANF@LINFO_NONE@ 0000000180061dd0     flags.obj
 0002:0000bde0       ??_C@_0N@OLGDMHKL@FDLG_WARNING@ 0000000180061de0     flags.obj
 0002:0000bdf0       ??_C@_0BB@DKMEBDJJ@FDLG_SMALLDIALOG@ 0000000180061df0     flags.obj
 0002:0000be08       ??_C@_0BC@ONGLDAJN@FDLG_NODRAWSHADOW@ 0000000180061e08     flags.obj
 0002:0000be20       ??_C@_0BB@NPLEEAKK@FDLG_NODRAWPANEL@ 0000000180061e20     flags.obj
 0002:0000be38       ??_C@_0BG@GHNOOENB@FDLG_KEEPCONSOLETITLE@ 0000000180061e38     flags.obj
 0002:0000be50       ??_C@_0O@MKFABCNE@FDLG_NONMODAL@ 0000000180061e50     flags.obj
 0002:0000be60       ??_C@_09NNFHCBNL@FDLG_NONE@ 0000000180061e60     flags.obj
 0002:0000be70       ??_C@_0N@JOOGIBAO@MIF_SELECTED@ 0000000180061e70     flags.obj
 0002:0000be80       ??_C@_0M@IHMNAMOE@MIF_CHECKED@ 0000000180061e80     flags.obj
 0002:0000be90       ??_C@_0O@DEIKOCPA@MIF_SEPARATOR@ 0000000180061e90     flags.obj
 0002:0000bea0       ??_C@_0M@OPPCPJOL@MIF_DISABLE@ 0000000180061ea0     flags.obj
 0002:0000beb0       ??_C@_0L@DLLNLLIG@MIF_GRAYED@ 0000000180061eb0     flags.obj
 0002:0000bec0       ??_C@_0L@DEJINBIP@MIF_HIDDEN@ 0000000180061ec0     flags.obj
 0002:0000bed0       ??_C@_08JEEJJGP@MIF_NONE@  0000000180061ed0     flags.obj
 0002:0000bee0       ??_C@_0BE@FALMPPJK@FMENU_SHOWAMPERSAND@ 0000000180061ee0     flags.obj
 0002:0000bef8       ??_C@_0P@HICDNKDJ@FMENU_WRAPMODE@ 0000000180061ef8     flags.obj
 0002:0000bf08       ??_C@_0BE@IDAMFDEA@FMENU_AUTOHIGHLIGHT@ 0000000180061f08     flags.obj
 0002:0000bf20       ??_C@_0BL@OKAIKPMN@FMENU_REVERSEAUTOHIGHLIGHT@ 0000000180061f20     flags.obj
 0002:0000bf40       ??_C@_0BJ@FCEONOJC@FMENU_CHANGECONSOLETITLE@ 0000000180061f40     flags.obj
 0002:0000bf60       ??_C@_0BA@GDFPJAAD@FMENU_SHOWNOBOX@ 0000000180061f60     flags.obj
 0002:0000bf70       ??_C@_0BD@PMEPMEOJ@FMENU_SHOWSHORTBOX@ 0000000180061f70     flags.obj
 0002:0000bf88       ??_C@_0BE@PDNJFEDO@FMENU_SHOWSINGLEBOX@ 0000000180061f88     flags.obj
 0002:0000bfa0       ??_C@_0BD@JBJJGCBE@FMENU_NODRAWSHADOW@ 0000000180061fa0     flags.obj
 0002:0000bfb8       ??_C@_0L@DGFIEOMD@FMENU_NONE@ 0000000180061fb8     flags.obj
 0002:0000bfc8       ??_C@_0O@JEAJLDHC@PPIF_SELECTED@ 0000000180061fc8     flags.obj
 0002:0000bfd8       ??_C@_0BC@LPBDBIOM@PPIF_PROCESSDESCR@ 0000000180061fd8     flags.obj
 0002:0000bff0       ??_C@_09OIFMMGNJ@PPIF_NONE@ 0000000180061ff0     flags.obj
 0002:0000c000       ??_C@_0BC@BONLDOOD@PFLAGS_SHOWHIDDEN@ 0000000180062000     flags.obj
 0002:0000c018       ??_C@_0BB@BCAJEJEH@PFLAGS_HIGHLIGHT@ 0000000180062018     flags.obj
 0002:0000c030       ??_C@_0BI@BFAFODJ@PFLAGS_REVERSESORTORDER@ 0000000180062030     flags.obj
 0002:0000c048       ??_C@_0BF@KJNCJPKN@PFLAGS_USESORTGROUPS@ 0000000180062048     flags.obj
 0002:0000c060       ??_C@_0BF@LBBAIOCD@PFLAGS_SELECTEDFIRST@ 0000000180062060     flags.obj
 0002:0000c078       ??_C@_0BB@KDANIJNM@PFLAGS_REALNAMES@ 0000000180062078     flags.obj
 0002:0000c090       ??_C@_0BB@ILEHDKFJ@PFLAGS_PANELLEFT@ 0000000180062090     flags.obj
 0002:0000c0a8       ??_C@_0BI@EHHAJLOH@PFLAGS_DIRECTORIESFIRST@ 00000001800620a8     flags.obj
 0002:0000c0c0       ??_C@_0BA@KJEPHDOM@PFLAGS_USECRC32@ 00000001800620c0     flags.obj
 0002:0000c0d0       ??_C@_0O@DBPJGING@PFLAGS_PLUGIN@ 00000001800620d0     flags.obj
 0002:0000c0e0       ??_C@_0P@MLDEBNPK@PFLAGS_VISIBLE@ 00000001800620e0     flags.obj
 0002:0000c0f0       ??_C@_0N@EOFAELOJ@PFLAGS_FOCUS@ 00000001800620f0     flags.obj
 0002:0000c100       ??_C@_0BI@EOCCAHFA@PFLAGS_ALTERNATIVENAMES@ 0000000180062100     flags.obj
 0002:0000c118       ??_C@_0BA@GHMDCHHI@PFLAGS_SHORTCUT@ 0000000180062118     flags.obj
 0002:0000c128       ??_C@_0M@NEMAHHGP@PFLAGS_NONE@ 0000000180062128     flags.obj
 0002:0000c138       ??_C@_0M@IDNADAFL@VF_NONMODAL@ 0000000180062138     flags.obj
 0002:0000c148       ??_C@_0BB@OCDDPIKL@VF_DELETEONCLOSE@ 0000000180062148     flags.obj
 0002:0000c160       ??_C@_0N@LDHALKKM@VF_ENABLE_F6@ 0000000180062160     flags.obj
 0002:0000c170       ??_C@_0BC@DLGKMECC@VF_DISABLEHISTORY@ 0000000180062170     flags.obj
 0002:0000c188       ??_C@_0BD@DHJCMLFI@VF_IMMEDIATERETURN@ 0000000180062188     flags.obj
 0002:0000c1a0       ??_C@_0BJ@OGNFHEJG@VF_DELETEONLYFILEONCLOSE@ 00000001800621a0     flags.obj
 0002:0000c1c0       ??_C@_07CJJFHP@VF_NONE@    00000001800621c0     flags.obj
 0002:0000c1c8       ??_C@_0M@PIFGAPFH@EF_NONMODAL@ 00000001800621c8     flags.obj
 0002:0000c1d8       ??_C@_0N@DBHFPBEO@EF_CREATENEW@ 00000001800621d8     flags.obj
 0002:0000c1e8       ??_C@_0N@LKLNHALI@EF_ENABLE_F6@ 00000001800621e8     flags.obj
 0002:0000c1f8       ??_C@_0BC@PPEPEFFI@EF_DISABLEHISTORY@ 00000001800621f8     flags.obj
 0002:0000c210       ??_C@_0BB@KGPIDKFC@EF_DELETEONCLOSE@ 0000000180062210     flags.obj
 0002:0000c228       ??_C@_0BD@IHIGHGPL@EF_IMMEDIATERETURN@ 0000000180062228     flags.obj
 0002:0000c240       ??_C@_0BJ@ILCPOFKL@EF_DELETEONLYFILEONCLOSE@ 0000000180062240     flags.obj
 0002:0000c260       ??_C@_09IJMPFPLB@EF_LOCKED@ 0000000180062260     flags.obj
 0002:0000c270       ??_C@_0BC@GFHJGKD@EF_DISABLESAVEPOS@ 0000000180062270     flags.obj
 0002:0000c288       ??_C@_0BB@NILAHAFO@EF_OPENMODE_MASK@ 0000000180062288     flags.obj
 0002:0000c2a0       ??_C@_0BC@GAIDEJIA@EF_OPENMODE_QUERY@ 00000001800622a0     flags.obj
 0002:0000c2b8       ??_C@_0BG@BFKJJBAG@EF_OPENMODE_NEWIFOPEN@ 00000001800622b8     flags.obj
 0002:0000c2d0       ??_C@_0BI@KGOKGPEI@EF_OPENMODE_USEEXISTING@ 00000001800622d0     flags.obj
 0002:0000c2e8       ??_C@_0BI@EJBKKDJ@EF_OPENMODE_BREAKIFOPEN@ 00000001800622e8     flags.obj
 0002:0000c300       ??_C@_0BJ@MOLGCBMH@EF_OPENMODE_RELOADIFOPEN@ 0000000180062300     flags.obj
 0002:0000c320       ??_C@_07MBPCONNA@EN_NONE@  0000000180062320     flags.obj
 0002:0000c328       ??_C@_0BC@HHNGCBAM@FHELP_NOSHOWERROR@ 0000000180062328     flags.obj
 0002:0000c340       ??_C@_0P@GANNLHEJ@FHELP_SELFHELP@ 0000000180062340     flags.obj
 0002:0000c350       ??_C@_0O@FLGGLFLC@FHELP_FARHELP@ 0000000180062350     flags.obj
 0002:0000c360       ??_C@_0BB@KNKDPNI@FHELP_CUSTOMFILE@ 0000000180062360     flags.obj
 0002:0000c378       ??_C@_0BB@IHFFPJJA@FHELP_CUSTOMPATH@ 0000000180062378     flags.obj
 0002:0000c390       ??_C@_0L@OOIMFPBD@FHELP_GUID@ 0000000180062390     flags.obj
 0002:0000c3a0       ??_C@_0BC@PNPOIHMG@FHELP_USECONTENTS@ 00000001800623a0     flags.obj
 0002:0000c3b8       ??_C@_0L@MAGMKNFN@FHELP_NONE@ 00000001800623b8     flags.obj
 0002:0000c3c8       ??_C@_0BE@GEGKIINM@KMFLAGS_SILENTCHECK@ 00000001800623c8     flags.obj
 0002:0000c3e0       ??_C@_0BM@BBOPLPKC@KMFLAGS_NOSENDKEYSTOPLUGINS@ 00000001800623e0     flags.obj
 0002:0000c400       ??_C@_0BF@PHHPAAOK@KMFLAGS_ENABLEOUTPUT@ 0000000180062400     flags.obj
 0002:0000c418       ??_C@_0BB@NCECNBPK@KMFLAGS_LANGMASK@ 0000000180062418     flags.obj
 0002:0000c430       ??_C@_0M@HFBACHCP@KMFLAGS_LUA@ 0000000180062430     flags.obj
 0002:0000c440       ??_C@_0BD@JHNPMIGP@KMFLAGS_MOONSCRIPT@ 0000000180062440     flags.obj
 0002:0000c458       ??_C@_0N@GIJCDFJI@KMFLAGS_NONE@ 0000000180062458     flags.obj
 0002:0000c468       ??_C@_0O@GKOLBMFK@AKMFLAGS_NONE@ 0000000180062468     flags.obj
 0002:0000c478       ??_C@_0P@LMBMJIMF@FSETCLR_REDRAW@ 0000000180062478     flags.obj
 0002:0000c488       ??_C@_0N@LCOHPDHN@FSETCLR_NONE@ 0000000180062488     flags.obj
 0002:0000c498       ??_C@_0N@MLMCEKPH@WIF_MODIFIED@ 0000000180062498     flags.obj
 0002:0000c4a8       ??_C@_0M@ICPAPCOF@WIF_CURRENT@ 00000001800624a8     flags.obj
 0002:0000c4b8       ??_C@_09FPGEBDGO@WIF_MODAL@ 00000001800624b8     flags.obj
 0002:0000c4c8       ??_C@_08DAKKFBIA@WIF_NONE@ 00000001800624c8     flags.obj
 0002:0000c4d8       ??_C@_0BG@JMJAOELH@VOPT_SAVEFILEPOSITION@ 00000001800624d8     flags.obj
 0002:0000c4f0       ??_C@_0BI@NCAHLEBN@VOPT_AUTODETECTCODEPAGE@ 00000001800624f0     flags.obj
 0002:0000c508       ??_C@_0BC@FGLBHLDI@VOPT_SHOWTITLEBAR@ 0000000180062508     flags.obj
 0002:0000c520       ??_C@_0BA@GAIDGLME@VOPT_SHOWKEYBAR@ 0000000180062520     flags.obj
 0002:0000c530       ??_C@_0BD@LEEGOJKA@VOPT_SHOWSCROLLBAR@ 0000000180062530     flags.obj
 0002:0000c548       ??_C@_0P@NEIKPMJJ@VOPT_QUICKVIEW@ 0000000180062548     flags.obj
 0002:0000c558       ??_C@_09FIOJMNJ@VOPT_NONE@ 0000000180062558     flags.obj
 0002:0000c568       ??_C@_0N@ILNDJNNO@VSMFL_REDRAW@ 0000000180062568     flags.obj
 0002:0000c578       ??_C@_0L@DLLCFLOD@VSMFL_NONE@ 0000000180062578     flags.obj
 0002:0000c588       ??_C@_0N@GHEHKHJN@VSP_NOREDRAW@ 0000000180062588     flags.obj
 0002:0000c598       ??_C@_0M@LHNGMHFO@VSP_PERCENT@ 0000000180062598     flags.obj
 0002:0000c5a8       ??_C@_0N@JGGGCNIP@VSP_RELATIVE@ 00000001800625a8     flags.obj
 0002:0000c5b8       ??_C@_0BA@JKDMJLJG@VSP_NORETNEWPOS@ 00000001800625b8     flags.obj
 0002:0000c5c8       ??_C@_08MOKEMBNE@VSP_NONE@ 00000001800625c8     flags.obj
 0002:0000c5d8       ??_C@_08FAPBJAKB@VMF_WRAP@ 00000001800625d8     flags.obj
 0002:0000c5e8       ??_C@_0N@GHBDMLON@VMF_WORDWRAP@ 00000001800625e8     flags.obj
 0002:0000c5f8       ??_C@_08KDJLELDJ@VMF_NONE@ 00000001800625f8     flags.obj
 0002:0000c608       ??_C@_0BB@EDGIEBDF@ECF_TABMARKFIRST@ 0000000180062608     flags.obj
 0002:0000c620       ??_C@_0BD@DKGCCJNG@ECF_TABMARKCURRENT@ 0000000180062620     flags.obj
 0002:0000c638       ??_C@_0P@BAFEMBAJ@ECF_AUTODELETE@ 0000000180062638     flags.obj
 0002:0000c648       ??_C@_08CDFMCHLP@ECF_NONE@ 0000000180062648     flags.obj
 0002:0000c658       ??_C@_0BA@KNNLMGCA@FIB_ENABLEEMPTY@ 0000000180062658     flags.obj
 0002:0000c668       ??_C@_0N@DLDJCGJI@FIB_PASSWORD@ 0000000180062668     flags.obj
 0002:0000c678       ??_C@_0O@DOHEGELC@FIB_EXPANDENV@ 0000000180062678     flags.obj
 0002:0000c688       ??_C@_0BF@CEMIHIOK@FIB_NOUSELASTHISTORY@ 0000000180062688     flags.obj
 0002:0000c6a0       ??_C@_0M@KJOJJDIM@FIB_BUTTONS@ 00000001800626a0     flags.obj
 0002:0000c6b0       ??_C@_0BA@COBBDHNL@FIB_NOAMPERSAND@ 00000001800626b0     flags.obj
 0002:0000c6c0       ??_C@_0N@LBOCEEGH@FIB_EDITPATH@ 00000001800626c0     flags.obj
 0002:0000c6d0       ??_C@_0BB@DCODFLEL@FIB_EDITPATHEXEC@ 00000001800626d0     flags.obj
 0002:0000c6e8       ??_C@_08HPFOCDKB@FIB_NONE@ 00000001800626e8     flags.obj
 0002:0000c6f8       ??_C@_0L@NMBLFMBN@FPF_LOADED@ 00000001800626f8     flags.obj
 0002:0000c708       ??_C@_08GKECKCCJ@FPF_ANSI@ 0000000180062708     flags.obj
 0002:0000c718       ??_C@_08OIOFCNLC@FPF_NONE@ 0000000180062718     flags.obj
 0002:0000c728       ??_C@_0L@HODJIPGA@PN_CMPNAME@ 0000000180062728     flags.obj
 0002:0000c738       ??_C@_0P@KDEENAHJ@PN_CMPNAMELIST@ 0000000180062738     flags.obj
 0002:0000c748       ??_C@_0BA@BJCCEIOI@PN_GENERATENAME@ 0000000180062748     flags.obj
 0002:0000c758       ??_C@_0N@FEGPCCPJ@PN_CHECKMASK@ 0000000180062758     flags.obj
 0002:0000c768       ??_C@_0M@NOOLKEBH@PN_SKIPPATH@ 0000000180062768     flags.obj
 0002:0000c778       ??_C@_0BE@OPDBOAAE@PN_SHOWERRORMESSAGE@ 0000000180062778     flags.obj
 0002:0000c790       ??_C@_07PFKJNCJP@PN_NONE@  0000000180062790     flags.obj
 0002:0000c798       ??_C@_0BG@GOMJDMCK@XLAT_SWITCHKEYBLAYOUT@ 0000000180062798     flags.obj
 0002:0000c7b0       ??_C@_0BE@KOIJDNLA@XLAT_SWITCHKEYBBEEP@ 00000001800627b0     flags.obj
 0002:0000c7c8       ??_C@_0BH@KBFAFPNA@XLAT_USEKEYBLAYOUTNAME@ 00000001800627c8     flags.obj
 0002:0000c7e0       ??_C@_0BH@IANKLOAC@XLAT_CONVERTALLCMDLINE@ 00000001800627e0     flags.obj
 0002:0000c7f8       ??_C@_09JCNLKBBK@XLAT_NONE@ 00000001800627f8     flags.obj
 0002:0000c808       ??_C@_0N@PJEDCNNJ@FRS_RETUPDIR@ 0000000180062808     flags.obj
 0002:0000c818       ??_C@_09GHEPLOHO@FRS_RECUR@ 0000000180062818     flags.obj
 0002:0000c828       ??_C@_0BA@JCPHOEAE@FRS_SCANSYMLINK@ 0000000180062828     flags.obj
 0002:0000c838       ??_C@_08JPCGJJKG@FRS_NONE@ 0000000180062838     flags.obj
 0002:0000c848       ??_C@_0P@LJPBHEIE@MLF_SHOWERRMSG@ 0000000180062848     flags.obj
 0002:0000c858       ??_C@_0BF@LMAGFLHF@MLF_DONOTUPDATEPANEL@ 0000000180062858     flags.obj
 0002:0000c870       ??_C@_0P@EPFBLPAE@MLF_HOLDTARGET@ 0000000180062870     flags.obj
 0002:0000c880       ??_C@_08EBKEJHAL@MLF_NONE@ 0000000180062880     flags.obj
 0002:0000c890       ??_C@_0M@JDMKDBDH@FFFS_COMMAS@ 0000000180062890     flags.obj
 0002:0000c8a0       ??_C@_0P@JPMLNBKL@FFFS_FLOATSIZE@ 00000001800628a0     flags.obj
 0002:0000c8b0       ??_C@_0BE@NPKCCEJ@FFFS_SHOWBYTESINDEX@ 00000001800628b0     flags.obj
 0002:0000c8c8       ??_C@_0O@FPIOAIMC@FFFS_ECONOMIC@ 00000001800628c8     flags.obj
 0002:0000c8d8       ??_C@_0O@HFIGPFIH@FFFS_THOUSAND@ 00000001800628d8     flags.obj
 0002:0000c8e8       ??_C@_0BC@LLLANJJO@FFFS_MINSIZEINDEX@ 00000001800628e8     flags.obj
 0002:0000c900       ??_C@_0BH@PEGBPJKE@FFFS_MINSIZEINDEX_MASK@ 0000000180062900     flags.obj
 0002:0000c918       ??_C@_09PBPAKNEI@FFFS_NONE@ 0000000180062918     flags.obj
 0002:0000c928       ??_C@_0L@NHEJGKCF@PF_PRELOAD@ 0000000180062928     flags.obj
 0002:0000c938       ??_C@_0BB@GCINAIGN@PF_DISABLEPANELS@ 0000000180062938     flags.obj
 0002:0000c950       ??_C@_09OENCMPGE@PF_EDITOR@ 0000000180062950     flags.obj
 0002:0000c960       ??_C@_09NEKIJNNA@PF_VIEWER@ 0000000180062960     flags.obj
 0002:0000c970       ??_C@_0P@MBLBBCNK@PF_FULLCMDLINE@ 0000000180062970     flags.obj
 0002:0000c980       ??_C@_09GMFDAFKL@PF_DIALOG@ 0000000180062980     flags.obj
 0002:0000c990       ??_C@_07MGEGJMPI@PF_NONE@  0000000180062990     flags.obj
 0002:0000c998       ??_C@_0BD@EGELEIIG@IPLFLAGS_SEPARATOR@ 0000000180062998     flags.obj
 0002:0000c9b0       ??_C@_0O@JBNJFHHK@IPLFLAGS_NONE@ 00000001800629b0     flags.obj
 0002:0000c9c0       ??_C@_0BD@KGHJOBGM@PMFLAGS_FULLSCREEN@ 00000001800629c0     flags.obj
 0002:0000c9d8       ??_C@_0BH@GDAAKEMH@PMFLAGS_DETAILEDSTATUS@ 00000001800629d8     flags.obj
 0002:0000c9f0       ??_C@_0BI@BMHIBDMH@PMFLAGS_ALIGNEXTENSIONS@ 00000001800629f0     flags.obj
 0002:0000ca08       ??_C@_0BH@KOFCBJBO@PMFLAGS_CASECONVERSION@ 0000000180062a08     flags.obj
 0002:0000ca20       ??_C@_0N@DLFMCMOB@PMFLAGS_NONE@ 0000000180062a20     flags.obj
 0002:0000ca30       ??_C@_0BD@PBMGDJEM@OPIF_DISABLEFILTER@ 0000000180062a30     flags.obj
 0002:0000ca48       ??_C@_0BH@FHBKALPD@OPIF_DISABLESORTGROUPS@ 0000000180062a48     flags.obj
 0002:0000ca60       ??_C@_0BJ@NGLIANCL@OPIF_DISABLEHIGHLIGHTING@ 0000000180062a60     flags.obj
 0002:0000ca80       ??_C@_0N@JANKJMLP@OPIF_ADDDOTS@ 0000000180062a80     flags.obj
 0002:0000ca90       ??_C@_0BC@HOFHNJIG@OPIF_RAWSELECTION@ 0000000180062a90     flags.obj
 0002:0000caa8       ??_C@_0P@OFEDJCO@OPIF_REALNAMES@ 0000000180062aa8     flags.obj
 0002:0000cab8       ??_C@_0BD@FPGMNAPD@OPIF_SHOWNAMESONLY@ 0000000180062ab8     flags.obj
 0002:0000cad0       ??_C@_0BJ@NMIFAPJD@OPIF_SHOWRIGHTALIGNNAMES@ 0000000180062ad0     flags.obj
 0002:0000caf0       ??_C@_0BG@HGPMKHIE@OPIF_SHOWPRESERVECASE@ 0000000180062af0     flags.obj
 0002:0000cb08       ??_C@_0BE@GJEJHNKJ@OPIF_COMPAREFATTIME@ 0000000180062b08     flags.obj
 0002:0000cb20       ??_C@_0BB@PELHBPAM@OPIF_EXTERNALGET@ 0000000180062b20     flags.obj
 0002:0000cb38       ??_C@_0BB@CFFPNDFK@OPIF_EXTERNALPUT@ 0000000180062b38     flags.obj
 0002:0000cb50       ??_C@_0BE@LKEMICNM@OPIF_EXTERNALDELETE@ 0000000180062b50     flags.obj
 0002:0000cb68       ??_C@_0BD@JIMJPFEP@OPIF_EXTERNALMKDIR@ 0000000180062b68     flags.obj
 0002:0000cb80       ??_C@_0BJ@CALDMPLF@OPIF_USEATTRHIGHLIGHTING@ 0000000180062b80     flags.obj
 0002:0000cba0       ??_C@_0O@JHHHMHIG@OPIF_USECRC32@ 0000000180062ba0     flags.obj
 0002:0000cbb0       ??_C@_0BB@PFDFAFHG@OPIF_USEFREESIZE@ 0000000180062bb0     flags.obj
 0002:0000cbc8       ??_C@_0O@FJPLJDBC@OPIF_SHORTCUT@ 0000000180062bc8     flags.obj
 0002:0000cbd8       ??_C@_09DOPJBMLM@OPIF_NONE@ 0000000180062bd8     flags.obj
 0002:0000cbe8       ??_C@_0L@GEHHKNBL@OPM_SILENT@ 0000000180062be8     flags.obj
 0002:0000cbf8       ??_C@_08EKEBOKEP@OPM_FIND@ 0000000180062bf8     flags.obj
 0002:0000cc08       ??_C@_08EHBLNDLO@OPM_VIEW@ 0000000180062c08     flags.obj
 0002:0000cc18       ??_C@_08LAAGEMJG@OPM_EDIT@ 0000000180062c18     flags.obj
 0002:0000cc28       ??_C@_0N@NDGKAFDM@OPM_TOPLEVEL@ 0000000180062c28     flags.obj
 0002:0000cc38       ??_C@_09EBKAPHPA@OPM_DESCR@ 0000000180062c38     flags.obj
 0002:0000cc48       ??_C@_0O@OPDAGBBE@OPM_QUICKVIEW@ 0000000180062c48     flags.obj
 0002:0000cc58       ??_C@_08LCEGJCAC@OPM_PGDN@ 0000000180062c58     flags.obj
 0002:0000cc68       ??_C@_0N@HKCLLJDG@OPM_COMMANDS@ 0000000180062c68     flags.obj
 0002:0000cc78       ??_C@_08EGEBMPBD@OPM_NONE@ 0000000180062c78     flags.obj
 0002:0000cc88       ??_C@_0M@MIGJPBPE@FOSF_ACTIVE@ 0000000180062c88     flags.obj
 0002:0000cc98       ??_C@_09FMOOJHDF@FOSF_NONE@ 0000000180062c98     flags.obj
 0002:0000cca8       ??_C@_09HNBBLIGN@PCIF_NONE@ 0000000180062ca8     flags.obj
 0002:0000ccb8       ??_C@_0BA@MAEBFMHC@FOREGROUND_BLUE@ 0000000180062cb8     flags.obj
 0002:0000ccc8       ??_C@_0BB@PDFNMAI@FOREGROUND_GREEN@ 0000000180062cc8     flags.obj
 0002:0000cce0       ??_C@_0P@PBJHCFGA@FOREGROUND_RED@ 0000000180062ce0     flags.obj
 0002:0000ccf0       ??_C@_0BF@OOGEJCC@FOREGROUND_INTENSITY@ 0000000180062cf0     flags.obj
 0002:0000cd08       ??_C@_0BA@PIFINJCK@BACKGROUND_BLUE@ 0000000180062d08     flags.obj
 0002:0000cd18       ??_C@_0BB@GKLNBMEL@BACKGROUND_GREEN@ 0000000180062d18     flags.obj
 0002:0000cd30       ??_C@_0P@DANALJMC@BACKGROUND_RED@ 0000000180062d30     flags.obj
 0002:0000cd40       ??_C@_0BF@NIGKKPCF@BACKGROUND_INTENSITY@ 0000000180062d40     flags.obj
 0002:0000cd58       ??_C@_0N@FEFOEFHG@CTRL_C_EVENT@ 0000000180062d58     flags.obj
 0002:0000cd68       ??_C@_0BB@ELEIIFAE@CTRL_BREAK_EVENT@ 0000000180062d68     flags.obj
 0002:0000cd80       ??_C@_0BB@KMPDMOKK@CTRL_CLOSE_EVENT@ 0000000180062d80     flags.obj
 0002:0000cd98       ??_C@_0BC@MCKCEPAL@CTRL_LOGOFF_EVENT@ 0000000180062d98     flags.obj
 0002:0000cdb0       ??_C@_0BE@BCNEFGKM@CTRL_SHUTDOWN_EVENT@ 0000000180062db0     flags.obj
 0002:0000cdc8       ??_C@_0BC@BBOPHMOM@ENABLE_LINE_INPUT@ 0000000180062dc8     flags.obj
 0002:0000cde0       ??_C@_0BC@JPFKLHOC@ENABLE_ECHO_INPUT@ 0000000180062de0     flags.obj
 0002:0000cdf8       ??_C@_0BH@EHINFMOF@ENABLE_PROCESSED_INPUT@ 0000000180062df8     flags.obj
 0002:0000ce10       ??_C@_0BE@BLAHACNB@ENABLE_WINDOW_INPUT@ 0000000180062e10     flags.obj
 0002:0000ce28       ??_C@_0BD@BJECBJPO@ENABLE_MOUSE_INPUT@ 0000000180062e28     flags.obj
 0002:0000ce40       ??_C@_0BD@KJBPOMPN@ENABLE_INSERT_MODE@ 0000000180062e40     flags.obj
 0002:0000ce58       ??_C@_0BH@BJKMFKAO@ENABLE_QUICK_EDIT_MODE@ 0000000180062e58     flags.obj
 0002:0000ce70       ??_C@_0BG@CBCHHIEH@ENABLE_EXTENDED_FLAGS@ 0000000180062e70     flags.obj
 0002:0000ce88       ??_C@_0BF@PEBFEBKN@ENABLE_AUTO_POSITION@ 0000000180062e88     flags.obj
 0002:0000cea0       ??_C@_0BI@MHKNPIFM@ENABLE_PROCESSED_OUTPUT@ 0000000180062ea0     flags.obj
 0002:0000ceb8       ??_C@_0BK@CDKLKCHJ@ENABLE_WRAP_AT_EOL_OUTPUT@ 0000000180062eb8     flags.obj
 0002:0000ced8       ??_C@_09JBABGNAE@KEY_EVENT@ 0000000180062ed8     flags.obj
 0002:0000cee8       ??_C@_0M@CPILDGOO@MOUSE_EVENT@ 0000000180062ee8     flags.obj
 0002:0000cef8       ??_C@_0BJ@OHDOHJKG@WINDOW_BUFFER_SIZE_EVENT@ 0000000180062ef8     flags.obj
 0002:0000cf18       ??_C@_0L@MPODFLFH@MENU_EVENT@ 0000000180062f18     flags.obj
 0002:0000cf28       ??_C@_0M@LNGHCCGJ@FOCUS_EVENT@ 0000000180062f28     flags.obj
 0002:0000cf38       ??_C@_0M@MKBGBFGO@CAPSLOCK_ON@ 0000000180062f38     flags.obj
 0002:0000cf48       ??_C@_0N@EMEOEKDA@ENHANCED_KEY@ 0000000180062f48     flags.obj
 0002:0000cf58       ??_C@_0BC@GDHABBAP@RIGHT_ALT_PRESSED@ 0000000180062f58     flags.obj
 0002:0000cf70       ??_C@_0BB@MCADLJJO@LEFT_ALT_PRESSED@ 0000000180062f70     flags.obj
 0002:0000cf88       ??_C@_0BD@NEHHNAHO@RIGHT_CTRL_PRESSED@ 0000000180062f88     flags.obj
 0002:0000cfa0       ??_C@_0BC@FDNOAAAE@LEFT_CTRL_PRESSED@ 0000000180062fa0     flags.obj
 0002:0000cfb8       ??_C@_0O@OGDFJMBK@SHIFT_PRESSED@ 0000000180062fb8     flags.obj
 0002:0000cfc8       ??_C@_0L@IMGKKBIM@NUMLOCK_ON@ 0000000180062fc8     flags.obj
 0002:0000cfd8       ??_C@_0O@LAHFNPLG@SCROLLLOCK_ON@ 0000000180062fd8     flags.obj
 0002:0000cfe8       ??_C@_0BN@HACKHGAB@FROM_LEFT_1ST_BUTTON_PRESSED@ 0000000180062fe8     flags.obj
 0002:0000d008       ??_C@_0BJ@JECFAJNJ@RIGHTMOST_BUTTON_PRESSED@ 0000000180063008     flags.obj
 0002:0000d028       ??_C@_0BN@BJCFPKCG@FROM_LEFT_2ND_BUTTON_PRESSED@ 0000000180063028     flags.obj
 0002:0000d048       ??_C@_0BN@PMJNFPGM@FROM_LEFT_3RD_BUTTON_PRESSED@ 0000000180063048     flags.obj
 0002:0000d068       ??_C@_0BN@CNMHAAPD@FROM_LEFT_4TH_BUTTON_PRESSED@ 0000000180063068     flags.obj
 0002:0000d088       ??_C@_0M@KKBDEELB@MOUSE_MOVED@ 0000000180063088     flags.obj
 0002:0000d098       ??_C@_0N@EDCKBGJE@DOUBLE_CLICK@ 0000000180063098     flags.obj
 0002:0000d0a8       ??_C@_0O@GABDOPO@MOUSE_WHEELED@ 00000001800630a8     flags.obj
 0002:0000d0b8       ??_C@_0BA@OOKCCMHH@KEY_WOW64_32KEY@ 00000001800630b8     flags.obj
 0002:0000d0c8       ??_C@_0BA@DBCPEIGE@KEY_WOW64_64KEY@ 00000001800630c8     flags.obj
 0002:0000d0e0       Keys                       00000001800630e0     flags.obj
 0002:0000e7a0       Vals                       00000001800647a0     flags.obj
 0002:0000fe58       ??_C@_06ICDCBJPI@Colors@   0000000180065e58     keysandcolors.obj
 0002:0000fe60       ??_C@_05GALAPKHH@Guids@    0000000180065e60     keysandcolors.obj
 0002:00012224       ??_C@_01EEMJAFIK@?6@       0000000180068224     lflua.obj
 0002:00012228       ??_C@_0BB@BJDGDOHH@cannot?5?$CFs?5?$CFs?3?5?$CFs@ 0000000180068228     lflua.obj
 0002:0001223c       ??_C@_03PKPBNCAL@?o?$LL?$LP@ 000000018006823c     lflua.obj
 0002:00012240       ??_C@_06CCPPALKB@?$DNstdin@ 0000000180068240     lflua.obj
 0002:00012248       ??_C@_01EOFPKCAF@?$EA@     0000000180068248     lflua.obj
 0002:0001224c       ??_C@_04PMOCAHAA@open@     000000018006824c     lflua.obj
 0002:00012254       ??_C@_15JJPIMNBO@?$AAr?$AAb@ 0000000180068254     lflua.obj
 0002:0001225c       ??_C@_06IEGCHAII@reopen@   000000018006825c     lflua.obj
 0002:00012264       ??_C@_04POLDLDMI@read@     0000000180068264     lflua.obj
 0002:0001226c       ??_C@_02LOCGON@?$AA?$AA@   000000018006826c     lflua.obj
 0002:00012270       ??_C@_09KIEPBIJC@far_regex@ 0000000180068270     lregex.obj
 0002:00012280       ??_C@_0BO@PBOFMCLL@attempt?5to?5access?5freed?5regex@ 0000000180068280     lregex.obj
 0002:000122a0       ??_C@_07IHINEPFG@?$CFs?5?$CI?$CFp?$CJ@ 00000001800682a0     lregex.obj
 0002:000122a8       ??_C@_01KMDKNFGN@?1@       00000001800682a8     lregex.obj
 0002:000122b0       ??_C@_0BE@BBBEAHLK@RECTL_CREATE?5failed@ 00000001800682b0     lregex.obj
 0002:000122c8       ??_C@_0BL@HEFMPIBG@invalid?5regular?5expression@ 00000001800682c8     lregex.obj
 0002:000122e8       ??_C@_0BK@JCLHPPNA@cannot?5add?5?$CFd?5stack?5slots@ 00000001800682e8     lregex.obj
 0002:00012308       ??_C@_0BM@MOHHGMBK@string?5or?5table?5or?5function@ 0000000180068308     lregex.obj
 0002:00012328       ??_C@_0CG@IDFLGMFM@replace?5string?3?5invalid?5capture@ 0000000180068328     lregex.obj
 0002:00012350       ??_C@_0BJ@IMAIDFKH@invalid?5replacement?5type@ 0000000180068350     lregex.obj
 0002:00012370       ??_C@_0BE@KPDOHKBE@invalid?5return?5type@ 0000000180068370     lregex.obj
 0002:00012384       ??_C@_04CKFJHKAP@find@     0000000180068384     lregex.obj
 0002:0001238c       ??_C@_04GOLEAPFD@gsub@     000000018006838c     lregex.obj
 0002:00012394       ??_C@_05FNONLPDI@match@    0000000180068394     lregex.obj
 0002:0001239c       ??_C@_04MGEIEJAD@exec@     000000018006839c     lregex.obj
 0002:000123a4       ??_C@_05GFGPIPHI@findW@    00000001800683a4     lregex.obj
 0002:000123ac       ??_C@_05HPGHPNC@gsubW@     00000001800683ac     lregex.obj
 0002:000123b4       ??_C@_06NNKFJOLC@matchW@   00000001800683b4     lregex.obj
 0002:000123bc       ??_C@_05GMDFNCGA@execW@    00000001800683bc     lregex.obj
 0002:000123c8       ??_C@_0O@OJAOCNID@bracketscount@ 00000001800683c8     lregex.obj
 0002:000123d8       ??_C@_04BDLIKKMN@__gc@     00000001800683d8     lregex.obj
 0002:000123e0       ??_C@_06DPFCLDIO@gmatch@   00000001800683e0     lregex.obj
 0002:000123e8       ??_C@_07PPMFDHAH@gmatchW@  00000001800683e8     lregex.obj
 0002:000123f0       ??_C@_05FGAODPCE@regex@    00000001800683f0     lregex.obj
 0002:00012400       regex_methods              0000000180068400     lregex.obj
 0002:000124c0       regex_functions            00000001800684c0     lregex.obj
 0002:00012580       ??_C@_0BC@PMGNICBE@MacroPluginReturn@ 0000000180068580     luamacro.obj
 0002:00012594       ??_C@_02JIEIHMJD@wl@       0000000180068594     luamacro.obj
 0002:00012598       ??_C@_15PMCGDJNJ@?$AAO?$AAK@ 0000000180068598     luamacro.obj
 0002:000125a0       ??_C@_1BC@GBFPAMBP@?$AAL?$AAu?$AAa?$AAM?$AAa?$AAc?$AAr?$AAo@ 00000001800685a0     luamacro.obj
 0002:000125c0       ??_C@_1FA@DAFHIDEP@?$AAt?$AAo?$AAo?$AA?5?$AAm?$AAa?$AAn?$AAy?$AA?5?$AAv?$AAa?$AAl?$AAu?$AAe?$AAs@ 00000001800685c0     luamacro.obj
 0002:00012610       ??_C@_0BN@ICDOMFBB@invalid?5argument?5?$CD?$CFd?5to?5?8?$CFs?8@ 0000000180068610     luamacro.obj
 0002:00012630       ??_C@_0BB@FCMFBGOM@invalid?5argument@ 0000000180068630     luamacro.obj
 0002:00012658       ??_C@_0BA@MDNLMOMP@far_usercontrol@ 0000000180068658     lusercontrol.obj
 0002:00012668       ??_C@_0BH@DOPNHMGD@bounds?5checking?5failed@ 0000000180068668     lusercontrol.obj
 0002:00012680       ??_C@_09LDLEBFOB@rawhandle@ 0000000180068680     lusercontrol.obj
 0002:0001268c       ??_C@_04IMAAEPPE@Char@     000000018006868c     lusercontrol.obj
 0002:00012698       ??_C@_0L@PLFFHFAH@Attributes@ 0000000180068698     lusercontrol.obj
 0002:000126a8       ??_C@_0BD@BPIMECDH@X?5must?5be?5positive@ 00000001800686a8     lusercontrol.obj
 0002:000126c0       ??_C@_0BD@MIGOMCGP@Y?5must?5be?5positive@ 00000001800686c0     lusercontrol.obj
 0002:000126d4       ??_C@_05MNDELLDN@__len@    00000001800686d4     lusercontrol.obj
 0002:000126e0       ??_C@_0L@GADKNKH@__newindex@ 00000001800686e0     lusercontrol.obj
 0002:000126f0       ??_C@_0BC@KFJDHEIC@CreateUserControl@ 00000001800686f0     lusercontrol.obj
 0002:00012710       usercontrol_methods        0000000180068710     lusercontrol.obj
 0002:00012760       usercontrol_functions      0000000180068760     lusercontrol.obj
 0002:00012780       ??_C@_07PHPIFDKI@LBUTTON@  0000000180068780     service.obj
 0002:00012788       ??_C@_07JOMJHALB@RBUTTON@  0000000180068788     service.obj
 0002:00012790       ??_C@_06JHILMIHF@CANCEL@   0000000180068790     service.obj
 0002:00012798       ??_C@_07DLFCFDDG@MBUTTON@  0000000180068798     service.obj
 0002:000127a0       ??_C@_08OPILMHEG@XBUTTON1@ 00000001800687a0     service.obj
 0002:000127b0       ??_C@_08MEKGJEIF@XBUTTON2@ 00000001800687b0     service.obj
 0002:000127bc       ??_C@_04FJBHJJME@BACK@     00000001800687bc     service.obj
 0002:000127c4       ??_C@_03CJMDHCGG@TAB@      00000001800687c4     service.obj
 0002:000127c8       ??_C@_05PONODPI@CLEAR@     00000001800687c8     service.obj
 0002:000127d0       ??_C@_06LJMOENAO@RETURN@   00000001800687d0     service.obj
 0002:000127d8       ??_C@_05OAHIEJBI@SHIFT@    00000001800687d8     service.obj
 0002:000127e0       ??_C@_07DBEDOPMC@CONTROL@  00000001800687e0     service.obj
 0002:000127e8       ??_C@_04IILMDFMO@MENU@     00000001800687e8     service.obj
 0002:000127f0       ??_C@_05DIAHPDGL@PAUSE@    00000001800687f0     service.obj
 0002:000127f8       ??_C@_07OPCFNGJB@CAPITAL@  00000001800687f8     service.obj
 0002:00012800       ??_C@_04KGDAIAGM@KANA@     0000000180068800     service.obj
 0002:00012808       ??_C@_05PPKJGOLB@JUNJA@    0000000180068808     service.obj
 0002:00012810       ??_C@_05JEIAEFOF@FINAL@    0000000180068810     service.obj
 0002:00012818       ??_C@_05CHABPOPI@HANJA@    0000000180068818     service.obj
 0002:00012820       ??_C@_06CDPDIIDH@ESCAPE@   0000000180068820     service.obj
 0002:00012828       ??_C@_0L@ODNCKDCK@NONCONVERT@ 0000000180068828     service.obj
 0002:00012834       ??_C@_06INBBKPI@ACCEPT@    0000000180068834     service.obj
 0002:00012840       ??_C@_0L@HEHNEBED@MODECHANGE@ 0000000180068840     service.obj
 0002:0001284c       ??_C@_05CAEOFMEP@SPACE@    000000018006884c     service.obj
 0002:00012854       ??_C@_05BFDHCIJM@PRIOR@    0000000180068854     service.obj
 0002:0001285c       ??_C@_04MOKMKBJN@NEXT@     000000018006885c     service.obj
 0002:00012864       ??_C@_03JMGAKCCH@END@      0000000180068864     service.obj
 0002:00012868       ??_C@_04GHGFPGNC@HOME@     0000000180068868     service.obj
 0002:00012870       ??_C@_04KCNEHMIH@LEFT@     0000000180068870     service.obj
 0002:00012878       ??_C@_02NAHCJHOC@UP@       0000000180068878     service.obj
 0002:0001287c       ??_C@_05PMAFOJDE@RIGHT@    000000018006887c     service.obj
 0002:00012884       ??_C@_04FANAOELO@DOWN@     0000000180068884     service.obj
 0002:0001288c       ??_C@_06LCPJPOPK@SELECT@   000000018006888c     service.obj
 0002:00012894       ??_C@_05ECKPOFCN@PRINT@    0000000180068894     service.obj
 0002:000128a0       ??_C@_07LBDEDADF@EXECUTE@  00000001800688a0     service.obj
 0002:000128a8       ??_C@_08EMOKHGD@SNAPSHOT@  00000001800688a8     service.obj
 0002:000128b4       ??_C@_06OEMEAEKN@INSERT@   00000001800688b4     service.obj
 0002:000128bc       ??_C@_06FKDAMKFP@DELETE@   00000001800688bc     service.obj
 0002:000128c4       ??_C@_04DOKPJKJF@HELP@     00000001800688c4     service.obj
 0002:000128cc       ??_C@_01GBGANLPD@0@        00000001800688cc     service.obj
 0002:000128d0       ??_C@_01HIHLOKLC@1@        00000001800688d0     service.obj
 0002:000128d4       ??_C@_01FDFGLJHB@2@        00000001800688d4     service.obj
 0002:000128d8       ??_C@_01EKENIIDA@3@        00000001800688d8     service.obj
 0002:000128dc       ??_C@_01FAMBOPH@4@         00000001800688dc     service.obj
 0002:000128e0       ??_C@_01BMBHCPLG@5@        00000001800688e0     service.obj
 0002:000128e4       ??_C@_01DHDKHMHF@6@        00000001800688e4     service.obj
 0002:000128e8       ??_C@_01COCBENDE@7@        00000001800688e8     service.obj
 0002:000128ec       ??_C@_01KJLJFBPL@8@        00000001800688ec     service.obj
 0002:000128f0       ??_C@_01LAKCGALK@9@        00000001800688f0     service.obj
 0002:000128f4       ??_C@_01FHEEJDEE@A@        00000001800688f4     service.obj
 0002:000128f8       ??_C@_01HMGJMAIH@B@        00000001800688f8     service.obj
 0002:000128fc       ??_C@_01GFHCPBMG@C@        00000001800688fc     service.obj
 0002:00012900       ??_C@_01CKDDGHAB@D@        0000000180068900     service.obj
 0002:00012904       ??_C@_01DDCIFGEA@E@        0000000180068904     service.obj
 0002:00012908       ??_C@_01BIAFAFID@F@        0000000180068908     service.obj
 0002:0001290c       ??_C@_01BBODEMC@G@         000000018006890c     service.obj
 0002:00012910       ??_C@_01IGIGCIAN@H@        0000000180068910     service.obj
 0002:00012914       ??_C@_01JPJNBJEM@I@        0000000180068914     service.obj
 0002:00012918       ??_C@_01LELAEKIP@J@        0000000180068918     service.obj
 0002:0001291c       ??_C@_01KNKLHLMO@K@        000000018006891c     service.obj
 0002:00012920       ??_C@_01OCOKONAJ@L@        0000000180068920     service.obj
 0002:00012924       ??_C@_01PLPBNMEI@M@        0000000180068924     service.obj
 0002:00012928       ??_C@_01NANMIPIL@N@        0000000180068928     service.obj
 0002:0001292c       ??_C@_01MJMHLOMK@O@        000000018006892c     service.obj
 0002:00012930       ??_C@_01EJNLAFE@P@         0000000180068930     service.obj
 0002:00012934       ??_C@_01BNIGIBBF@Q@        0000000180068934     service.obj
 0002:00012938       ??_C@_01DGKLNCNG@R@        0000000180068938     service.obj
 0002:0001293c       ??_C@_01CPLAODJH@S@        000000018006893c     service.obj
 0002:00012940       ??_C@_01GAPBHFFA@T@        0000000180068940     service.obj
 0002:00012944       ??_C@_01HJOKEEBB@U@        0000000180068944     service.obj
 0002:00012948       ??_C@_01FCMHBHNC@V@        0000000180068948     service.obj
 0002:0001294c       ??_C@_01ELNMCGJD@W@        000000018006894c     service.obj
 0002:00012950       ??_C@_01MMEEDKFM@X@        0000000180068950     service.obj
 0002:00012954       ??_C@_01NFFPALBN@Y@        0000000180068954     service.obj
 0002:00012958       ??_C@_01POHCFINO@Z@        0000000180068958     service.obj
 0002:0001295c       ??_C@_04ODLFFOHF@LWIN@     000000018006895c     service.obj
 0002:00012964       ??_C@_04DMGFHHJG@RWIN@     0000000180068964     service.obj
 0002:0001296c       ??_C@_04GKGJFGJO@APPS@     000000018006896c     service.obj
 0002:00012974       ??_C@_05DJAECLDN@SLEEP@    0000000180068974     service.obj
 0002:00012980       ??_C@_07NHIPMMJH@NUMPAD0@  0000000180068980     service.obj
 0002:00012988       ??_C@_07MOJEPNNG@NUMPAD1@  0000000180068988     service.obj
 0002:00012990       ??_C@_07OFLJKOBF@NUMPAD2@  0000000180068990     service.obj
 0002:00012998       ??_C@_07PMKCJPFE@NUMPAD3@  0000000180068998     service.obj
 0002:000129a0       ??_C@_07LDODAJJD@NUMPAD4@  00000001800689a0     service.obj
 0002:000129a8       ??_C@_07KKPIDINC@NUMPAD5@  00000001800689a8     service.obj
 0002:000129b0       ??_C@_07IBNFGLBB@NUMPAD6@  00000001800689b0     service.obj
 0002:000129b8       ??_C@_07JIMOFKFA@NUMPAD7@  00000001800689b8     service.obj
 0002:000129c0       ??_C@_07BPFGEGJP@NUMPAD8@  00000001800689c0     service.obj
 0002:000129c8       ??_C@_07GENHHNO@NUMPAD9@   00000001800689c8     service.obj
 0002:000129d0       ??_C@_08LDEOAAGM@MULTIPLY@ 00000001800689d0     service.obj
 0002:000129dc       ??_C@_03BOJFLAKG@ADD@      00000001800689dc     service.obj
 0002:000129e0       ??_C@_09POPINEFK@SEPARATOR@ 00000001800689e0     service.obj
 0002:000129f0       ??_C@_08MGBEENML@SUBTRACT@ 00000001800689f0     service.obj
 0002:00012a00       ??_C@_07LJPMJDLL@DECIMAL@  0000000180068a00     service.obj
 0002:00012a08       ??_C@_06FBFCJJMP@DIVIDE@   0000000180068a08     service.obj
 0002:00012a10       ??_C@_02LCPENACN@F1@       0000000180068a10     service.obj
 0002:00012a14       ??_C@_02JJNJIDOO@F2@       0000000180068a14     service.obj
 0002:00012a18       ??_C@_02IAMCLCKP@F3@       0000000180068a18     service.obj
 0002:00012a1c       ??_C@_02MPIDCEGI@F4@       0000000180068a1c     service.obj
 0002:00012a20       ??_C@_02NGJIBFCJ@F5@       0000000180068a20     service.obj
 0002:00012a24       ??_C@_02PNLFEGOK@F6@       0000000180068a24     service.obj
 0002:00012a28       ??_C@_02OEKOHHKL@F7@       0000000180068a28     service.obj
 0002:00012a2c       ??_C@_02GDDGGLGE@F8@       0000000180068a2c     service.obj
 0002:00012a30       ??_C@_02HKCNFKCF@F9@       0000000180068a30     service.obj
 0002:00012a34       ??_C@_03JKCLJOFG@F10@      0000000180068a34     service.obj
 0002:00012a38       ??_C@_03IDDAKPBH@F11@      0000000180068a38     service.obj
 0002:00012a3c       ??_C@_03KIBNPMNE@F12@      0000000180068a3c     service.obj
 0002:00012a40       ??_C@_03LBAGMNJF@F13@      0000000180068a40     service.obj
 0002:00012a44       ??_C@_03POEHFLFC@F14@      0000000180068a44     service.obj
 0002:00012a48       ??_C@_03OHFMGKBD@F15@      0000000180068a48     service.obj
 0002:00012a4c       ??_C@_03MMHBDJNA@F16@      0000000180068a4c     service.obj
 0002:00012a50       ??_C@_03NFGKAIJB@F17@      0000000180068a50     service.obj
 0002:00012a54       ??_C@_03FCPCBEFO@F18@      0000000180068a54     service.obj
 0002:00012a58       ??_C@_03ELOJCFBP@F19@      0000000180068a58     service.obj
 0002:00012a5c       ??_C@_03JIGNCAAP@F20@      0000000180068a5c     service.obj
 0002:00012a60       ??_C@_03IBHGBBEO@F21@      0000000180068a60     service.obj
 0002:00012a64       ??_C@_03KKFLECIN@F22@      0000000180068a64     service.obj
 0002:00012a68       ??_C@_03LDEAHDMM@F23@      0000000180068a68     service.obj
 0002:00012a6c       ??_C@_03PMABOFAL@F24@      0000000180068a6c     service.obj
 0002:00012a70       ??_C@_07FLMEHHJP@NUMLOCK@  0000000180068a70     service.obj
 0002:00012a78       ??_C@_06FNIKALAE@SCROLL@   0000000180068a78     service.obj
 0002:00012a80       ??_C@_0O@DBBJDALK@OEM_NEC_EQUAL@ 0000000180068a80     service.obj
 0002:00012a90       ??_C@_0P@JKGCFGCD@OEM_FJ_MASSHOU@ 0000000180068a90     service.obj
 0002:00012aa0       ??_C@_0P@NIEOFNLG@OEM_FJ_TOUROKU@ 0000000180068aa0     service.obj
 0002:00012ab0       ??_C@_0M@IBEHGLCM@OEM_FJ_LOYA@ 0000000180068ab0     service.obj
 0002:00012ac0       ??_C@_0M@FOJHECMP@OEM_FJ_ROYA@ 0000000180068ac0     service.obj
 0002:00012acc       ??_C@_06EPHNCIMI@LSHIFT@   0000000180068acc     service.obj
 0002:00012ad4       ??_C@_06HIJMMPFL@RSHIFT@   0000000180068ad4     service.obj
 0002:00012ae0       ??_C@_08IKMONEBG@LCONTROL@ 0000000180068ae0     service.obj
 0002:00012af0       ??_C@_08OOMMENPF@RCONTROL@ 0000000180068af0     service.obj
 0002:00012afc       ??_C@_05IHMGKJGH@LMENU@    0000000180068afc     service.obj
 0002:00012b04       ??_C@_05LOBKMKIM@RMENU@    0000000180068b04     service.obj
 0002:00012b10       ??_C@_0N@OAJIELLG@BROWSER_BACK@ 0000000180068b10     service.obj
 0002:00012b20       ??_C@_0BA@ENOAJOGH@BROWSER_FORWARD@ 0000000180068b20     service.obj
 0002:00012b30       ??_C@_0BA@GDNDIDGJ@BROWSER_REFRESH@ 0000000180068b30     service.obj
 0002:00012b40       ??_C@_0N@HKPDGANH@BROWSER_STOP@ 0000000180068b40     service.obj
 0002:00012b50       ??_C@_0P@BEAEBJDD@BROWSER_SEARCH@ 0000000180068b50     service.obj
 0002:00012b60       ??_C@_0BC@BOMJIH@BROWSER_FAVORITES@ 0000000180068b60     service.obj
 0002:00012b78       ??_C@_0N@NOOKCEKA@BROWSER_HOME@ 0000000180068b78     service.obj
 0002:00012b88       ??_C@_0M@ENOHKBMG@VOLUME_MUTE@ 0000000180068b88     service.obj
 0002:00012b98       ??_C@_0M@JOOBBDNO@VOLUME_DOWN@ 0000000180068b98     service.obj
 0002:00012ba8       ??_C@_09MGPMNMJC@VOLUME_UP@ 0000000180068ba8     service.obj
 0002:00012bb8       ??_C@_0BB@KLAENPA@MEDIA_NEXT_TRACK@ 0000000180068bb8     service.obj
 0002:00012bd0       ??_C@_0BB@CMOIJKPH@MEDIA_PREV_TRACK@ 0000000180068bd0     service.obj
 0002:00012be8       ??_C@_0L@KBJOCDHK@MEDIA_STOP@ 0000000180068be8     service.obj
 0002:00012bf8       ??_C@_0BB@HAEMIJHO@MEDIA_PLAY_PAUSE@ 0000000180068bf8     service.obj
 0002:00012c10       ??_C@_0M@GCIKMBID@LAUNCH_MAIL@ 0000000180068c10     service.obj
 0002:00012c20       ??_C@_0BE@FADJJAPM@LAUNCH_MEDIA_SELECT@ 0000000180068c20     service.obj
 0002:00012c38       ??_C@_0M@MGLJIDDM@LAUNCH_APP1@ 0000000180068c38     service.obj
 0002:00012c48       ??_C@_0M@ONJENAPP@LAUNCH_APP2@ 0000000180068c48     service.obj
 0002:00012c54       ??_C@_05OIODNPAD@OEM_1@    0000000180068c54     service.obj
 0002:00012c60       ??_C@_08LDJEIPBH@OEM_PLUS@ 0000000180068c60     service.obj
 0002:00012c70       ??_C@_09CLPFJEOD@OEM_COMMA@ 0000000180068c70     service.obj
 0002:00012c80       ??_C@_09OGMLCNMG@OEM_MINUS@ 0000000180068c80     service.obj
 0002:00012c90       ??_C@_0L@DNNMNDGM@OEM_PERIOD@ 0000000180068c90     service.obj
 0002:00012c9c       ??_C@_05MDMOIMMA@OEM_2@    0000000180068c9c     service.obj
 0002:00012ca4       ??_C@_05NKNFLNIB@OEM_3@    0000000180068ca4     service.obj
 0002:00012cac       ??_C@_05JFJECLEG@OEM_4@    0000000180068cac     service.obj
 0002:00012cb4       ??_C@_05IMIPBKAH@OEM_5@    0000000180068cb4     service.obj
 0002:00012cbc       ??_C@_05KHKCEJME@OEM_6@    0000000180068cbc     service.obj
 0002:00012cc4       ??_C@_05LOLJHIIF@OEM_7@    0000000180068cc4     service.obj
 0002:00012ccc       ??_C@_05DJCBGEEK@OEM_8@    0000000180068ccc     service.obj
 0002:00012cd8       ??_C@_07PEFKMFIE@OEM_102@  0000000180068cd8     service.obj
 0002:00012ce0       ??_C@_0L@EFLJCPAM@PROCESSKEY@ 0000000180068ce0     service.obj
 0002:00012cec       ??_C@_06HOICDKCB@PACKET@   0000000180068cec     service.obj
 0002:00012cf8       ??_C@_09CAKPMKHM@OEM_RESET@ 0000000180068cf8     service.obj
 0002:00012d08       ??_C@_08INMNLJCK@OEM_JUMP@ 0000000180068d08     service.obj
 0002:00012d18       ??_C@_07JNOAEEG@OEM_PA1@   0000000180068d18     service.obj
 0002:00012d20       ??_C@_07CCPDFHIF@OEM_PA2@  0000000180068d20     service.obj
 0002:00012d28       ??_C@_07DLOIGGME@OEM_PA3@  0000000180068d28     service.obj
 0002:00012d30       ??_C@_0L@OCAIHDP@OEM_WSCTRL@ 0000000180068d30     service.obj
 0002:00012d3c       ??_C@_04BNGOAFAJ@ATTN@     0000000180068d3c     service.obj
 0002:00012d44       ??_C@_05HGAHFFFL@CRSEL@    0000000180068d44     service.obj
 0002:00012d4c       ??_C@_05OKOOKOOH@EXSEL@    0000000180068d4c     service.obj
 0002:00012d54       ??_C@_05CCFENDFJ@EREOF@    0000000180068d54     service.obj
 0002:00012d5c       ??_C@_04MKCNCBEG@PLAY@     0000000180068d5c     service.obj
 0002:00012d64       ??_C@_04LGBIGMFG@ZOOM@     0000000180068d64     service.obj
 0002:00012d6c       ??_C@_06LJIOOKLP@NONAME@   0000000180068d6c     service.obj
 0002:00012d74       ??_C@_03KCLDMPAE@PA1@      0000000180068d74     service.obj
 0002:00012d78       ??_C@_09MBBEHOCK@OEM_CLEAR@ 0000000180068d78     service.obj
 0002:00012d88       ??_C@_09GJGOMOL@lua51?4dll@ 0000000180068d88     service.obj
 0002:00012d98       ??_C@_0M@PLOBHAKE@luaopen_bit@ 0000000180068d98     service.obj
 0002:00012da8       ??_C@_0M@IALDMMNC@luaopen_ffi@ 0000000180068da8     service.obj
 0002:00012db8       ??_C@_0M@DOFFFIEL@luaopen_jit@ 0000000180068db8     service.obj
 0002:00012dc8       ??_C@_0BK@FFJEICME@integer?5or?5light?5userdata@ 0000000180068dc8     service.obj
 0002:00012de8       ??_C@_0BD@PNJHLBDA@invalid?5flag?3?5?$CC?$CFs?$CC@ 0000000180068de8     service.obj
 0002:00012e00       ??_C@_0N@JJLBBDOC@invalid?5flag@ 0000000180068e00     service.obj
 0002:00012e10       ??_C@_0BJ@MIKGPOKL@invalid?5flag?5combination@ 0000000180068e10     service.obj
 0002:00012e30       ??_C@_08KJKIOMBF@3?40?40?4?$CFd@ 0000000180068e30     service.obj
 0002:00012e40       ??_C@_0P@EANMLDOP@MousePositionX@ 0000000180068e40     service.obj
 0002:00012e50       ??_C@_0P@FJMHICKO@MousePositionY@ 0000000180068e50     service.obj
 0002:00012e60       ??_C@_0M@BJAICPIE@ButtonState@ 0000000180068e60     service.obj
 0002:00012e70       ??_C@_0L@EMFBJIPA@EventFlags@ 0000000180068e70     service.obj
 0002:00012e80       ??_C@_07EEJLMCNH@CurLine@  0000000180068e80     service.obj
 0002:00012e88       ??_C@_06EDBJMJDC@CurPos@   0000000180068e88     service.obj
 0002:00012e90       ??_C@_09EGONKHKB@CurTabPos@ 0000000180068e90     service.obj
 0002:00012ea0       ??_C@_0O@OKGGHEJK@TopScreenLine@ 0000000180068ea0     service.obj
 0002:00012eb0       ??_C@_07GDAKJHLE@LeftPos@  0000000180068eb0     service.obj
 0002:00012eb8       ??_C@_08LLJICOLD@Overtype@ 0000000180068eb8     service.obj
 0002:00012ec8       ??_C@_0L@GEIEADPN@ModuleName@ 0000000180068ec8     service.obj
 0002:00012ed8       ??_C@_09HOIHBHIM@ModuleDir@ 0000000180068ed8     service.obj
 0002:00012ee8       ??_C@_0L@JLHCLFBG@PluginGuid@ 0000000180068ee8     service.obj
 0002:00012ef8       ??_C@_08GGMFPBHM@EditorID@ 0000000180068ef8     service.obj
 0002:00012f08       ??_C@_0M@CPDBGLHN@WindowSizeX@ 0000000180068f08     service.obj
 0002:00012f18       ??_C@_0M@DGCKFKDM@WindowSizeY@ 0000000180068f18     service.obj
 0002:00012f28       ??_C@_0L@PMKENHMA@TotalLines@ 0000000180068f28     service.obj
 0002:00012f38       ??_C@_09HKBEFIPN@BlockType@ 0000000180068f38     service.obj
 0002:00012f48       ??_C@_0P@GAEEHNHE@BlockStartLine@ 0000000180068f48     service.obj
 0002:00012f58       ??_C@_07KHIHFBFN@Options@  0000000180068f58     service.obj
 0002:00012f60       ??_C@_07FLDNELFM@TabSize@  0000000180068f60     service.obj
 0002:00012f68       ??_C@_0O@EBLDFOPH@BookmarkCount@ 0000000180068f68     service.obj
 0002:00012f78       ??_C@_0BF@ODFKBFAK@SessionBookmarkCount@ 0000000180068f78     service.obj
 0002:00012f90       ??_C@_08CPAOHJDL@CurState@ 0000000180068f90     service.obj
 0002:00012fa0       ??_C@_0N@DAJMJAE@StringLength@ 0000000180068fa0     service.obj
 0002:00012fb0       ??_C@_08JPMALCFA@SelStart@ 0000000180068fb0     service.obj
 0002:00012fbc       ??_C@_06JLEHDHII@SelEnd@   0000000180068fbc     service.obj
 0002:00012fc8       ??_C@_0L@IFNFGDGN@StringText@ 0000000180068fc8     service.obj
 0002:00012fd8       ??_C@_09IBGOAAEM@StringEOL@ 0000000180068fd8     service.obj
 0002:00012fe4       ??_C@_06MFLCIING@redraw@   0000000180068fe4     service.obj
 0002:00012ff0       ??_C@_07HICINA@restore@    0000000180068ff0     service.obj
 0002:00012ff8       ??_C@_0CG@LAKEGANL@must?5be?5?8redraw?8?0?5?8restore?8?0?5or@ 0000000180068ff8     service.obj
 0002:00013020       ??_C@_04LIDDHMOL@Line@     0000000180069020     service.obj
 0002:00013028       ??_C@_06OIIFPIKD@Cursor@   0000000180069028     service.obj
 0002:00013030       ??_C@_0L@GDDEHGKI@ScreenLine@ 0000000180069030     service.obj
 0002:00013040       ??_C@_0O@CIAFMMMB@BlockStartPos@ 0000000180069040     service.obj
 0002:00013050       ??_C@_0L@EKLJJHPF@BlockWidth@ 0000000180069050     service.obj
 0002:00013060       ??_C@_0M@NKKGBDGK@BlockHeight@ 0000000180069060     service.obj
 0002:00013070       ??_C@_09JFPCGCOC@StartLine@ 0000000180069070     service.obj
 0002:00013080       ??_C@_08JBNOANJG@StartPos@ 0000000180069080     service.obj
 0002:00013090       ??_C@_07DCKCOCOC@EndLine@  0000000180069090     service.obj
 0002:00013098       ??_C@_06KGHIGMHC@EndPos@   0000000180069098     service.obj
 0002:000130a0       ??_C@_0BA@HNIJJEO@ForegroundColor@ 00000001800690a0     service.obj
 0002:000130b0       ??_C@_0BA@DPMBBMBG@BackgroundColor@ 00000001800690b0     service.obj
 0002:000130c0       ??_C@_0O@NHKEGDJF@GUID?5required@ 00000001800690c0     service.obj
 0002:000130d0       ??_C@_0BJ@BMOGHFAN@table?5or?5number?5expected@ 00000001800690d0     service.obj
 0002:000130f0       ??_C@_08KGEIBGG@Priority@  00000001800690f0     service.obj
 0002:000130fc       ??_C@_05PDOBBJNA@Color@    00000001800690fc     service.obj
 0002:00013108       ??_C@_09KDLBEGCN@EventType@ 0000000180069108     service.obj
 0002:00013118       ??_C@_07HPHPOAEG@KeyDown@  0000000180069118     service.obj
 0002:00013120       ??_C@_0M@FGGHEADP@RepeatCount@ 0000000180069120     service.obj
 0002:00013130       ??_C@_0BA@KCCLHPM@VirtualScanCode@ 0000000180069130     service.obj
 0002:00013140       ??_C@_0M@PBJKDIHH@UnicodeChar@ 0000000180069140     service.obj
 0002:0001314c       ??_C@_05GIPJKPFG@SizeX@    000000018006914c     service.obj
 0002:00013154       ??_C@_05HBOCJOBH@SizeY@    0000000180069154     service.obj
 0002:00013160       ??_C@_09GEJJJAHL@CommandId@ 0000000180069160     service.obj
 0002:00013170       ??_C@_08GPNNBNIL@SetFocus@ 0000000180069170     service.obj
 0002:00013180       ??_C@_0M@BEDENHPD@invalid?5key@ 0000000180069180     service.obj
 0002:00013190       ??_C@_19IBCFILMC@?$AAM?$AAe?$AAn?$AAu@ 0000000180069190     service.obj
 0002:000131a0       ??_C@_0BN@JBAMKCCJ@must?5be?5table?0?5string?5or?5nil@ 00000001800691a0     service.obj
 0002:000131c0       ??_C@_09FDAFFNEA@MaxHeight@ 00000001800691c0     service.obj
 0002:000131cc       ??_C@_06DDHCBBGN@Bottom@   00000001800691cc     service.obj
 0002:000131d8       ??_C@_09CFELDMD@HelpTopic@ 00000001800691d8     service.obj
 0002:000131e8       ??_C@_0M@GGMLPAIK@SelectIndex@ 00000001800691e8     service.obj
 0002:000131f4       ??_C@_02HOGEDOAB@Id@       00000001800691f4     service.obj
 0002:000131f8       ??_C@_05LCLENNFI@table@    00000001800691f8     service.obj
 0002:00013200       ??_C@_06ICGJLFIM@string@   0000000180069200     service.obj
 0002:00013208       ??_C@_07FJOBMBFC@checked@  0000000180069208     service.obj
 0002:00013210       ??_C@_09MOAJOJKN@separator@ 0000000180069210     service.obj
 0002:00013220       ??_C@_07DBNODEFN@disable@  0000000180069220     service.obj
 0002:00013228       ??_C@_06JHIAOIKD@grayed@   0000000180069228     service.obj
 0002:00013230       ??_C@_06JIKFICKK@hidden@   0000000180069230     service.obj
 0002:00013238       ??_C@_08CJLOJPNI@selected@ 0000000180069238     service.obj
 0002:00013248       ??_C@_08MMCKBNNI@AccelKey@ 0000000180069248     service.obj
 0002:00013258       ??_C@_08PNHLLJE@BreakKey@  0000000180069258     service.obj
 0002:00013264       ??_C@_15FMBEJGOH@?$AAO?$AAk@ 0000000180069264     service.obj
 0002:00013270       ??_C@_1BC@IBCAPFAE@?$AAO?$AAk?$AAC?$AAa?$AAn?$AAc?$AAe?$AAl@ 0000000180069270     service.obj
 0002:00013288       ??_C@_1CC@HODOHOHB@?$AAA?$AAb?$AAo?$AAr?$AAt?$AAR?$AAe?$AAt?$AAr?$AAy?$AAI?$AAg?$AAn?$AAo?$AAr@ 0000000180069288     service.obj
 0002:000132b0       ??_C@_1M@GGPOIMAD@?$AAY?$AAe?$AAs?$AAN?$AAo@ 00000001800692b0     service.obj
 0002:000132c0       ??_C@_1BI@BNDFIGCI@?$AAY?$AAe?$AAs?$AAN?$AAo?$AAC?$AAa?$AAn?$AAc?$AAe?$AAl@ 00000001800692c0     service.obj
 0002:000132d8       ??_C@_1BI@KMMIHPHF@?$AAR?$AAe?$AAt?$AAr?$AAy?$AAC?$AAa?$AAn?$AAc?$AAe?$AAl@ 00000001800692d8     service.obj
 0002:000132f0       ??_C@_1DG@LMKDDADI@?$AA?$DM?$AAn?$AAo?$AAn?$AA?9?$AAs?$AAt?$AAr?$AAi?$AAn?$AAg?$AA?5?$AAe?$AAr?$AAr@ 00000001800692f0     service.obj
 0002:00013328       ??_C@_15IEGBJKPD@?$AA?3?$AA?6@ 0000000180069328     service.obj
 0002:00013330       ??_C@_19FFLPMPBO@?$AA?6?$AA?5?$AA?5?$AA?5@ 0000000180069330     service.obj
 0002:0001333c       ??_C@_15JCKODCLA@?$AA?6?$AA?7@ 000000018006933c     service.obj
 0002:00013348       ??_C@_1M@ILHOPKA@?$AAE?$AAr?$AAr?$AAo?$AAr@ 0000000180069348     service.obj
 0002:00013358       ??_C@_08FNIIFOJC@tostring@ 0000000180069358     service.obj
 0002:00013368       ??_C@_0BJ@JOELOGM@cannot?5convert?5to?5string@ 0000000180069368     service.obj
 0002:00013388       ??_C@_1BA@HHOMBECE@?$AAM?$AAe?$AAs?$AAs?$AAa?$AAg?$AAe@ 0000000180069388     service.obj
 0002:00013398       ??_C@_17PAGBAIDI@?$AA?$DL?$AAO?$AAK@ 0000000180069398     service.obj
 0002:000133a0       ??_C@_09ENKGJCEC@OwnerGuid@ 00000001800693a0     service.obj
 0002:000133b0       ??_C@_0N@CCPLCIHE@PluginHandle@ 00000001800693b0     service.obj
 0002:000133c0       ??_C@_0N@HEHBMBNM@PluginObject@ 00000001800693c0     service.obj
 0002:000133d0       ??_C@_09BKHPOLGD@PanelType@ 00000001800693d0     service.obj
 0002:000133dc       ??_C@_04GOOOJOPP@left@     00000001800693dc     service.obj
 0002:000133e4       ??_C@_03FGFCOCMD@top@      00000001800693e4     service.obj
 0002:000133e8       ??_C@_05DHJDAOHK@right@    00000001800693e8     service.obj
 0002:000133f0       ??_C@_06PMMPCIPB@bottom@   00000001800693f0     service.obj
 0002:000133f8       ??_C@_09MCEJMINN@PanelRect@ 00000001800693f8     service.obj
 0002:00013408       ??_C@_0M@DDGFKGKJ@ItemsNumber@ 0000000180069408     service.obj
 0002:00013418       ??_C@_0BE@EOBAHHNK@SelectedItemsNumber@ 0000000180069418     service.obj
 0002:00013430       ??_C@_0M@JMILNLLF@CurrentItem@ 0000000180069430     service.obj
 0002:00013440       ??_C@_0N@CDHIFJIH@TopPanelItem@ 0000000180069440     service.obj
 0002:00013450       ??_C@_08IMMBLBLF@ViewMode@ 0000000180069450     service.obj
 0002:00013460       ??_C@_08CENECNJD@SortMode@ 0000000180069460     service.obj
 0002:0001346c       ??_C@_04FABLJDN@Name@      000000018006946c     service.obj
 0002:00013474       ??_C@_05LOJBNELM@Param@    0000000180069474     service.obj
 0002:0001347c       ??_C@_04PBAHLACE@File@     000000018006947c     service.obj
 0002:00013488       ??_C@_08HGEAFCFN@PluginId@ 0000000180069488     service.obj
 0002:00013498       ??_C@_0BA@MLHECKCE@table?5or?5string@ 0000000180069498     service.obj
 0002:000134a8       ??_C@_0BD@CKJHMJBG@non?9positive?5index@ 00000001800694a8     service.obj
 0002:000134c0       ??_C@_0BA@GNKNKKDM@number?5or?5table@ 00000001800694c0     service.obj
 0002:000134d0       ??_C@_0CI@DDAJHJKO@?$CFs?5?9?5unsupported?5type?5in?5dialog@ 00000001800694d0     service.obj
 0002:000134f8       ??_C@_0CD@JIANOKII@unsupported?5flag?5in?5dialog?5item@ 00000001800694f8     service.obj
 0002:00013520       ??_C@_0CB@EOGFCCCC@value?5at?5index?5?$CFd?5is?5not?5a?5tabl@ 0000000180069520     service.obj
 0002:00013548       ??_C@_0O@FEBHKEHB@closed?5dialog@ 0000000180069548     service.obj
 0002:00013558       ??_C@_0BK@NEMPGLFN@operation?5not?5implemented@ 0000000180069558     service.obj
 0002:00013574       ??_C@_04KPCPLBPL@Left@     0000000180069574     service.obj
 0002:0001357c       ??_C@_03PGGAENPN@Top@      000000018006957c     service.obj
 0002:00013580       ??_C@_05DADPALEM@Right@    0000000180069580     service.obj
 0002:00013588       ??_C@_0CK@JHNDGJBB@element?5?$CD?$CFd?5in?5argument?5?$CD4?5is?5n@ 0000000180069588     service.obj
 0002:000135b8       ??_C@_0L@CECHCPAP@StartIndex@ 00000001800695b8     service.obj
 0002:000135c4       ??_C@_05IJGIMMHE@Count@    00000001800695c4     service.obj
 0002:000135d0       ??_C@_07NOCIGAPP@Pattern@  00000001800695d0     service.obj
 0002:000135d8       ??_C@_09IMOCKOO@SelectPos@ 00000001800695d8     service.obj
 0002:000135e4       ??_C@_06DJONBJOP@TopPos@   00000001800695e4     service.obj
 0002:000135f0       ??_C@_09OGCBKCAK@MaxLength@ 00000001800695f0     service.obj
 0002:000135fc       ??_C@_05FNNGFGLF@Index@    00000001800695fc     service.obj
 0002:00013608       ??_C@_07GHGHLGFI@GetType@  0000000180069608     service.obj
 0002:00013610       ??_C@_07MMLMCDAI@ValType@  0000000180069610     service.obj
 0002:00013618       ??_C@_05LPIJGKJ@Value@     0000000180069618     service.obj
 0002:00013620       ??_C@_0L@LPFMIAHH@helpstring@ 0000000180069620     service.obj
 0002:00013630       ??_C@_0P@NABDHFON@getvaluestring@ 0000000180069630     service.obj
 0002:00013640       ??_C@_0BJ@IINAPFDG@Items?$FL?$CFd?$FN?5is?5not?5a?5table@ 0000000180069640     service.obj
 0002:00013660       ??_C@_0CC@GBOJFNBI@error?5occured?5in?5dialog?5procedu@ 0000000180069660     service.obj
 0002:00013688       ??_C@_0M@EHMONPJO@?$CFs?5?$CIclosed?$CJ@ 0000000180069688     service.obj
 0002:00013698       ??_C@_08GDAJJKGC@ViewerID@ 0000000180069698     service.obj
 0002:000136a8       ??_C@_07MJHBHMFM@FilePos@  00000001800696a8     service.obj
 0002:000136b0       ??_C@_07FBAHDBGN@CurMode@  00000001800696b0     service.obj
 0002:000136b8       ??_C@_06IMBBKDFH@iParam@   00000001800696b8     service.obj
 0002:000136c0       ??_C@_1BE@CGKCNEEP@?$AAI?$AAn?$AAp?$AAu?$AAt?$AA?5?$AAB?$AAo?$AAx@ 00000001800696c0     service.obj
 0002:000136d8       ??_C@_1CA@PCDNIBFH@?$AAE?$AAn?$AAt?$AAe?$AAr?$AA?5?$AAt?$AAh?$AAe?$AA?5?$AAt?$AAe?$AAx?$AAt?$AA?3@ 00000001800696d8     service.obj
 0002:000136f8       ??_C@_15GALJLHBD@?$AA?$DO?$AA?$DO@ 00000001800696f8     service.obj
 0002:00013700       ??_C@_0BG@GAFLOAPP@command?5not?5supported@ 0000000180069700     service.obj
 0002:00013718       ??_C@_09MIJAKHKB@Completed@ 0000000180069718     service.obj
 0002:00013724       ??_C@_05KGEAEGFG@Total@    0000000180069724     service.obj
 0002:00013730       ??_C@_0P@DJOANNIK@?$CFd?4?$CFd?4?$CFd?4?$CFd?4?$CFd@ 0000000180069730     service.obj
 0002:00013740       ??_C@_03FCCPIJGJ@Pos@      0000000180069740     service.obj
 0002:00013748       ??_C@_08NNKIOIN@TypeName@  0000000180069748     service.obj
 0002:00013758       ??_C@_07ONPPLIAF@ErrCode@  0000000180069758     service.obj
 0002:00013760       ??_C@_07LJDOKIBM@ErrPosX@  0000000180069760     service.obj
 0002:00013768       ??_C@_07KACFJJFN@ErrPosY@  0000000180069768     service.obj
 0002:00013770       ??_C@_06HBEFEBCM@ErrSrc@   0000000180069770     service.obj
 0002:00013778       ??_C@_06LDIMCHFC@?$CF?$CKs?$CFs?5@ 0000000180069778     service.obj
 0002:00013780       ??_C@_09HNJDNMKK@?$CF?$CF?$CFdd?$CF?$CFs?5@ 0000000180069780     service.obj
 0002:00013790       ??_C@_0CC@JIGPFMKG@global?5?$GAtostring?8?5is?5not?5functi@ 0000000180069790     service.obj
 0002:000137b8       ??_C@_0CH@OINAPBOJ@tostring?$CI?$CJ?5returned?5a?5non?9strin@ 00000001800697b8     service.obj
 0002:000137e0       ??_C@_04CIMGMMMG@text@     00000001800697e0     service.obj
 0002:000137e8       ??_C@_03CAOIPBNL@arg@      00000001800697e8     service.obj
 0002:000137f0       ??_C@_0ME@JDKAEDFJ@local?5items?0n?$DN?4?4?4?6local?5bottom?$DN@ 00000001800697f0     service.obj
 0002:000138b8       ??_C@_0CG@FGNNCNLL@attempt?5to?5access?5invalid?5file?5@ 00000001800698b8     service.obj
 0002:000138e0       ??_C@_07BJOIOONN@Strings@  00000001800698e0     service.obj
 0002:000138e8       ??_C@_08FGAFMHLF@DiskMenu@ 00000001800698e8     service.obj
 0002:000138f8       ??_C@_0L@NHENMPLN@PluginMenu@ 00000001800698f8     service.obj
 0002:00013908       ??_C@_0N@IEACHFBM@PluginConfig@ 0000000180069908     service.obj
 0002:00013918       ??_C@_05GCJGCMFJ@PInfo@    0000000180069918     service.obj
 0002:00013920       ??_C@_05HMEFBOHK@GInfo@    0000000180069920     service.obj
 0002:00013928       ??_C@_0N@GAMEMCEE@invalid?5GUID@ 0000000180069928     service.obj
 0002:00013938       ??_C@_0BP@NJEEOHDB@attempt?5to?5access?5closed?5timer@ 0000000180069938     service.obj
 0002:00013958       ??_C@_05LGELBCGM@Close@    0000000180069958     service.obj
 0002:00013960       ??_C@_07DOAOMMKG@Enabled@  0000000180069960     service.obj
 0002:00013968       ??_C@_08KDKDEPAG@Interval@ 0000000180069968     service.obj
 0002:00013978       ??_C@_07CIINKFND@OnTimer@  0000000180069978     service.obj
 0002:00013980       ??_C@_06EFCDMIMC@Closed@   0000000180069980     service.obj
 0002:00013988       ??_C@_0CE@LHJCBGGH@attempt?5to?5call?5non?9existent?5me@ 0000000180069988     service.obj
 0002:000139b0       ??_C@_0BO@PNFLEJKN@attempt?5to?5access?5a?5closed?5?$CFs@ 00000001800699b0     service.obj
 0002:000139d0       ??_C@_04OKOFBOPB@Time@     00000001800699d0     service.obj
 0002:000139d8       ??_C@_04LADJNOK@Lock@      00000001800699d8     service.obj
 0002:000139e0       ??_C@_09KFKKEOOH@GetFilesW@ 00000001800699e0     service.obj
 0002:000139f0       ??_C@_0BE@OGGJBMCE@insufficient?5memory@ 00000001800699f0     service.obj
 0002:00013a08       ??_C@_09MMBIJGAH@PutFilesW@ 0000000180069a08     service.obj
 0002:00013a18       ??_C@_0N@HPKKMFEI@GetFindDataW@ 0000000180069a18     service.obj
 0002:00013a28       ??_C@_0O@GNDAADHN@FreeFindDataW@ 0000000180069a28     service.obj
 0002:00013a38       ??_C@_0O@BCOALCIL@SetDirectoryW@ 0000000180069a38     service.obj
 0002:00013a48       ??_C@_0P@LKPINHLK@FreeFileFilter@ 0000000180069a48     service.obj
 0002:00013a58       ??_C@_0BA@JGEOEAE@OpenFiltersMenu@ 0000000180069a58     service.obj
 0002:00013a68       ??_C@_0BB@OPPOFOAK@StartingToFilter@ 0000000180069a68     service.obj
 0002:00013a80       ??_C@_0P@JDMCHDIM@IsFileInFilter@ 0000000180069a80     service.obj
 0002:00013a90       ??_C@_04MIIPNNEF@send@     0000000180069a90     service.obj
 0002:00013a98       ??_C@_06JBKGCNBB@Delete@   0000000180069a98     service.obj
 0002:00013aa0       ??_C@_04PAFOOALK@Enum@     0000000180069aa0     service.obj
 0002:00013aa8       ??_C@_04HJMOFLDF@Free@     0000000180069aa8     service.obj
 0002:00013ab0       ??_C@_03NNDHPFFO@Get@      0000000180069ab0     service.obj
 0002:00013ab4       ??_C@_03CEMDFJG@Set@       0000000180069ab4     service.obj
 0002:00013ab8       ??_C@_0N@OELJMCEC@CreateSubkey@ 0000000180069ab8     service.obj
 0002:00013ac8       ??_C@_0L@CPCKAMD@OpenSubkey@ 0000000180069ac8     service.obj
 0002:00013ad8       ??_C@_08EGJLHNCO@AddColor@ 0000000180069ad8     service.obj
 0002:00013ae8       ??_C@_0BD@DOFEEDDC@AddSessionBookmark@ 0000000180069ae8     service.obj
 0002:00013b00       ??_C@_0BG@IGFHDIIN@ClearSessionBookmarks@ 0000000180069b00     service.obj
 0002:00013b18       ??_C@_08PDEJHGJI@DelColor@ 0000000180069b18     service.obj
 0002:00013b28       ??_C@_0M@LPIECDD@DeleteBlock@ 0000000180069b28     service.obj
 0002:00013b38       ??_C@_0L@BCLIBKOC@DeleteChar@ 0000000180069b38     service.obj
 0002:00013b48       ??_C@_0BG@KOELEFCN@DeleteSessionBookmark@ 0000000180069b48     service.obj
 0002:00013b60       ??_C@_0N@EKENACAE@DeleteString@ 0000000180069b60     service.obj
 0002:00013b70       ??_C@_06MJDIICIN@Editor@   0000000180069b70     service.obj
 0002:00013b78       ??_C@_0L@HDLPOLMA@ExpandTabs@ 0000000180069b78     service.obj
 0002:00013b88       ??_C@_0N@MGAOADJN@GetBookmarks@ 0000000180069b88     service.obj
 0002:00013b98       ??_C@_08JOPFJIPE@GetColor@ 0000000180069b98     service.obj
 0002:00013ba8       ??_C@_0M@FECPLAMN@GetFileName@ 0000000180069ba8     service.obj
 0002:00013bb8       ??_C@_07NAJNLNAF@GetInfo@  0000000180069bb8     service.obj
 0002:00013bc0       ??_C@_0N@KIILHCLH@GetSelection@ 0000000180069bc0     service.obj
 0002:00013bd0       ??_C@_0BE@LBJJGOGD@GetSessionBookmarks@ 0000000180069bd0     service.obj
 0002:00013be8       ??_C@_09HBLKHMEA@GetString@ 0000000180069be8     service.obj
 0002:00013bf8       ??_C@_0L@IDFHDAHP@GetStringW@ 0000000180069bf8     service.obj
 0002:00013c08       ??_C@_0N@ICPGLOEG@InsertString@ 0000000180069c08     service.obj
 0002:00013c18       ??_C@_0L@JMOIGJIA@InsertText@ 0000000180069c18     service.obj
 0002:00013c28       ??_C@_0M@BINOKANK@InsertTextW@ 0000000180069c28     service.obj
 0002:00013c38       ??_C@_0BE@CNGODNDI@NextSessionBookmark@ 0000000180069c38     service.obj
 0002:00013c50       ??_C@_0BE@IEBIGOAP@PrevSessionBookmark@ 0000000180069c50     service.obj
 0002:00013c68       ??_C@_0N@FNCEPAJJ@ProcessInput@ 0000000180069c68     service.obj
 0002:00013c78       ??_C@_04GMBKPCGK@Quit@     0000000180069c78     service.obj
 0002:00013c80       ??_C@_09KINLOJJJ@ReadInput@ 0000000180069c80     service.obj
 0002:00013c90       ??_C@_09DBPLBJBJ@RealToTab@ 0000000180069c90     service.obj
 0002:00013c9c       ??_C@_06KAPLBEK@Redraw@    0000000180069c9c     service.obj
 0002:00013ca8       ??_C@_08FBDDPFPJ@SaveFile@ 0000000180069ca8     service.obj
 0002:00013cb4       ??_C@_06HJGPBJLE@Select@   0000000180069cb4     service.obj
 0002:00013cc0       ??_C@_09PPEOOGEC@SetKeyBar@ 0000000180069cc0     service.obj
 0002:00013cd0       ??_C@_08CCKJEGOF@SetParam@ 0000000180069cd0     service.obj
 0002:00013ce0       ??_C@_0M@GKIFPNAD@SetPosition@ 0000000180069ce0     service.obj
 0002:00013cf0       ??_C@_09FPPPFNNC@SetString@ 0000000180069cf0     service.obj
 0002:00013d00       ??_C@_0L@JNHIIHDG@SetStringW@ 0000000180069d00     service.obj
 0002:00013d10       ??_C@_08GMCCAJLF@SetTitle@ 0000000180069d10     service.obj
 0002:00013d20       ??_C@_08JNAOBKMI@GetTitle@ 0000000180069d20     service.obj
 0002:00013d30       ??_C@_0BF@LIMPGNED@SubscribeChangeEvent@ 0000000180069d30     service.obj
 0002:00013d48       ??_C@_09JFBCONJH@TabToReal@ 0000000180069d48     service.obj
 0002:00013d58       ??_C@_08IBJJAHJG@UndoRedo@ 0000000180069d58     service.obj
 0002:00013d68       ??_C@_07JMDLHPJF@SetMode@  0000000180069d68     service.obj
 0002:00013d70       ??_C@_06PJECNADJ@Viewer@   0000000180069d70     service.obj
 0002:00013d78       ??_C@_0P@OAACIGEB@BeginSelection@ 0000000180069d78     service.obj
 0002:00013d88       ??_C@_0BB@PJGDGIKA@CheckPanelsExist@ 0000000180069d88     service.obj
 0002:00013da0       ??_C@_0P@DFBDDHFA@ClearSelection@ 0000000180069da0     service.obj
 0002:00013db0       ??_C@_0N@BHLDKHDJ@EndSelection@ 0000000180069db0     service.obj
 0002:00013dc0       ??_C@_0L@KOHCMOPM@GetCmdLine@ 0000000180069dc0     service.obj
 0002:00013dd0       ??_C@_0O@NLDIMJEA@GetCmdLinePos@ 0000000180069dd0     service.obj
 0002:00013de0       ??_C@_0BE@CBPLLCEH@GetCmdLineSelection@ 0000000180069de0     service.obj
 0002:00013df8       ??_C@_0P@CMFANDFM@GetColumnTypes@ 0000000180069df8     service.obj
 0002:00013e08       ??_C@_0BA@DJGLDCBG@GetColumnWidths@ 0000000180069e08     service.obj
 0002:00013e18       ??_C@_0BE@JPAIJBCI@GetCurrentPanelItem@ 0000000180069e18     service.obj
 0002:00013e30       ??_C@_0BC@NGKPIKGL@GetPanelDirectory@ 0000000180069e30     service.obj
 0002:00013e48       ??_C@_0P@GODLFFFJ@GetPanelFormat@ 0000000180069e48     service.obj
 0002:00013e58       ??_C@_0BB@LCMBHPNI@GetPanelHostFile@ 0000000180069e58     service.obj
 0002:00013e70       ??_C@_0N@HPIPGDFA@GetPanelInfo@ 0000000180069e70     service.obj
 0002:00013e80       ??_C@_0N@HAFLAIHA@GetPanelItem@ 0000000180069e80     service.obj
 0002:00013e90       ??_C@_0P@HCBKDPMP@GetPanelPrefix@ 0000000180069e90     service.obj
 0002:00013ea0       ??_C@_0BF@MEMFMMGB@GetSelectedPanelItem@ 0000000180069ea0     service.obj
 0002:00013eb8       ??_C@_0O@HEGDGAJG@GetUserScreen@ 0000000180069eb8     service.obj
 0002:00013ec8       ??_C@_0O@EHOCCHAL@InsertCmdLine@ 0000000180069ec8     service.obj
 0002:00013ed8       ??_C@_0O@OMMHIHHH@IsActivePanel@ 0000000180069ed8     service.obj
 0002:00013ee8       ??_C@_0M@LCEPDNPK@RedrawPanel@ 0000000180069ee8     service.obj
 0002:00013ef8       ??_C@_0P@OPKJJMLB@SetActivePanel@ 0000000180069ef8     service.obj
 0002:00013f08       ??_C@_0L@LAFNHJLF@SetCmdLine@ 0000000180069f08     service.obj
 0002:00013f18       ??_C@_0O@KECGHKDH@SetCmdLinePos@ 0000000180069f18     service.obj
 0002:00013f28       ??_C@_0BE@IPNAPCDL@SetCmdLineSelection@ 0000000180069f28     service.obj
 0002:00013f40       ??_C@_0BE@PAPEKLCP@SetDirectoriesFirst@ 0000000180069f40     service.obj
 0002:00013f58       ??_C@_0BC@PDKEABHF@SetPanelDirectory@ 0000000180069f58     service.obj
 0002:00013f70       ??_C@_0N@NMDFLOPL@SetSelection@ 0000000180069f70     service.obj
 0002:00013f80       ??_C@_0M@CMMMGIDG@SetSortMode@ 0000000180069f80     service.obj
 0002:00013f90       ??_C@_0N@HCHLALN@SetSortOrder@ 0000000180069f90     service.obj
 0002:00013fa0       ??_C@_0O@LHNNDOB@SetUserScreen@ 0000000180069fa0     service.obj
 0002:00013fb0       ??_C@_0M@IENJPEBA@SetViewMode@ 0000000180069fb0     service.obj
 0002:00013fc0       ??_C@_0M@EICBHAOA@UpdatePanel@ 0000000180069fc0     service.obj
 0002:00013fd0       ??_C@_0BC@BIIKJLKB@PluginStartupInfo@ 0000000180069fd0     service.obj
 0002:00013fe8       ??_C@_0L@PJAHNOGM@DialogInit@ 0000000180069fe8     service.obj
 0002:00013ff8       ??_C@_09DBEDLMHB@DialogRun@ 0000000180069ff8     service.obj
 0002:00014008       ??_C@_0L@DLFLHLOO@DialogFree@ 000000018006a008     service.obj
 0002:00014018       ??_C@_0P@HLOFPDFP@SendDlgMessage@ 000000018006a018     service.obj
 0002:00014028       ??_C@_0L@CKELNLCE@GetDlgItem@ 000000018006a028     service.obj
 0002:00014038       ??_C@_0L@DEGEGMGN@SetDlgItem@ 000000018006a038     service.obj
 0002:00014048       ??_C@_0BK@EBIPEKDH@SubscribeDialogDrawEvents@ 000000018006a048     service.obj
 0002:00014068       ??_C@_0L@MCFABBED@GetDirList@ 000000018006a068     service.obj
 0002:00014074       ??_C@_06KCCBBIBJ@GetMsg@   000000018006a074     service.obj
 0002:00014080       ??_C@_0BB@HIDBFOJJ@GetPluginDirList@ 000000018006a080     service.obj
 0002:00014094       ??_C@_04IFEHPILC@Menu@     000000018006a094     service.obj
 0002:000140a0       ??_C@_07BEIHKDLJ@Message@  000000018006a0a0     service.obj
 0002:000140a8       ??_C@_0O@CGLFPNOD@RestoreScreen@ 000000018006a0a8     service.obj
 0002:000140b8       ??_C@_0L@PGGGPLFK@SaveScreen@ 000000018006a0b8     service.obj
 0002:000140c8       ??_C@_0L@HABDNHIM@FreeScreen@ 000000018006a0c8     service.obj
 0002:000140d8       ??_C@_08DAHHHDJC@ShowHelp@ 000000018006a0d8     service.obj
 0002:000140e8       ??_C@_08IAADAJIH@InputBox@ 000000018006a0e8     service.obj
 0002:000140f8       ??_C@_0L@HHLOIHOP@AdvControl@ 000000018006a0f8     service.obj
 0002:00014108       ??_C@_0N@GHGEMEN@MacroLoadAll@ 000000018006a108     service.obj
 0002:00014118       ??_C@_0N@NAGBAPAE@MacroSaveAll@ 000000018006a118     service.obj
 0002:00014128       ??_C@_0O@KGHDMPAJ@MacroGetState@ 000000018006a128     service.obj
 0002:00014138       ??_C@_0N@PNLHCOIE@MacroGetArea@ 000000018006a138     service.obj
 0002:00014148       ??_C@_09KGKKBHMO@MacroPost@ 000000018006a148     service.obj
 0002:00014158       ??_C@_0L@KBAKOGFP@MacroCheck@ 000000018006a158     service.obj
 0002:00014168       ??_C@_08KAFLEHAN@MacroAdd@ 000000018006a168     service.obj
 0002:00014178       ??_C@_0M@KFMHCNNB@MacroDelete@ 000000018006a178     service.obj
 0002:00014188       ??_C@_0BC@MJDKBAPF@MacroGetLastError@ 000000018006a188     service.obj
 0002:000141a0       ??_C@_0N@COEPENFH@MacroExecute@ 000000018006a1a0     service.obj
 0002:000141b0       ??_C@_0BB@BICELPOF@CreateFileFilter@ 000000018006a1b0     service.obj
 0002:000141c8       ??_C@_0L@CHJBHF@LoadPlugin@ 000000018006a1c8     service.obj
 0002:000141d8       ??_C@_0N@DHIONCLI@UnloadPlugin@ 000000018006a1d8     service.obj
 0002:000141e8       ??_C@_0BB@IJHIBGJA@ForcedLoadPlugin@ 000000018006a1e8     service.obj
 0002:00014200       ??_C@_0L@DACPHGGH@FindPlugin@ 000000018006a200     service.obj
 0002:00014210       ??_C@_0BF@KLOGLFMF@GetPluginInformation@ 000000018006a210     service.obj
 0002:00014228       ??_C@_0L@JIDCIJHM@GetPlugins@ 000000018006a228     service.obj
 0002:00014238       ??_C@_0P@IKAEEPOB@IsPluginLoaded@ 000000018006a238     service.obj
 0002:00014248       ??_C@_0P@HMKEDHIE@CreateSettings@ 000000018006a248     service.obj
 0002:00014258       ??_C@_0N@GOMOBHDB@FreeSettings@ 000000018006a258     service.obj
 0002:00014268       ??_C@_0M@IFKFGKML@ColorDialog@ 000000018006a268     service.obj
 0002:00014278       ??_C@_0BA@EOCNNPOG@CopyToClipboard@ 000000018006a278     service.obj
 0002:00014288       ??_C@_0BD@PLIHDKFC@PasteFromClipboard@ 000000018006a288     service.obj
 0002:000142a0       ??_C@_0BC@FJDIKOMH@InputRecordToName@ 000000018006a2a0     service.obj
 0002:000142b8       ??_C@_0BC@FFNOIDFI@NameToInputRecord@ 000000018006a2b8     service.obj
 0002:000142d0       ??_C@_08HGLFNLMB@LStricmp@ 000000018006a2d0     service.obj
 0002:000142e0       ??_C@_09GALOFBAC@LStrnicmp@ 000000018006a2e0     service.obj
 0002:000142f0       ??_C@_0M@KPPMMAOL@ProcessName@ 000000018006a2f0     service.obj
 0002:00014300       ??_C@_0M@KFCNKLDK@GetPathRoot@ 000000018006a300     service.obj
 0002:00014310       ??_C@_0BE@EPGHGPJC@GetReparsePointInfo@ 000000018006a310     service.obj
 0002:00014328       ??_C@_08DNJCLFF@LIsAlpha@  000000018006a328     service.obj
 0002:00014338       ??_C@_0M@LKJIEECA@LIsAlphanum@ 000000018006a338     service.obj
 0002:00014348       ??_C@_08MAHKICD@LIsLower@  000000018006a348     service.obj
 0002:00014358       ??_C@_08FHLJMDJK@LIsUpper@ 000000018006a358     service.obj
 0002:00014368       ??_C@_09LPKAHGM@LLowerBuf@ 000000018006a368     service.obj
 0002:00014378       ??_C@_09GLKFOOEP@LUpperBuf@ 000000018006a378     service.obj
 0002:00014384       ??_C@_06ILCHIEBO@MkTemp@   000000018006a384     service.obj
 0002:0001438c       ??_C@_06DKBBJCCG@MkLink@   000000018006a38c     service.obj
 0002:00014398       ??_C@_0N@CCDDAJK@TruncPathStr@ 000000018006a398     service.obj
 0002:000143a8       ??_C@_08BNEIIKEJ@TruncStr@ 000000018006a3a8     service.obj
 0002:000143b8       ??_C@_0BA@CLEHBIPM@RecursiveSearch@ 000000018006a3b8     service.obj
 0002:000143c8       ??_C@_0M@HKHGOOHG@ConvertPath@ 000000018006a3c8     service.obj
 0002:000143d4       ??_C@_04OCDKHGII@XLat@     000000018006a3d4     service.obj
 0002:000143e0       ??_C@_0P@BGLLKGOI@FormatFileSize@ 000000018006a3e0     service.obj
 0002:000143f0       ??_C@_08KJBLDCDF@FarClock@ 000000018006a3f0     service.obj
 0002:00014400       ??_C@_0BD@ELMHPHAC@CPluginStartupInfo@ 000000018006a400     service.obj
 0002:00014418       ??_C@_0BE@DJLJEKBK@GetCurrentDirectory@ 000000018006a418     service.obj
 0002:00014430       ??_C@_0N@MOMBJEKA@GetFileOwner@ 000000018006a430     service.obj
 0002:00014440       ??_C@_0BB@JBNBALEM@GetNumberOfLinks@ 000000018006a440     service.obj
 0002:00014458       ??_C@_0BB@OPAJHEIC@GetLuafarVersion@ 000000018006a458     service.obj
 0002:00014470       ??_C@_0O@BJEAJNBH@MakeMenuItems@ 000000018006a470     service.obj
 0002:00014480       ??_C@_0BB@HLFLDCHO@RunDefaultScript@ 000000018006a480     service.obj
 0002:00014494       ??_C@_04JLAJABDJ@Show@     000000018006a494     service.obj
 0002:0001449c       ??_C@_05NHFJDMOA@Timer@    000000018006a49c     service.obj
 0002:000144a8       ??_C@_0BD@KCMHFGFP@FileTimeResolution@ 000000018006a4a8     service.obj
 0002:000144bc       ??_C@_04CPPPJGME@Host@     000000018006a4bc     service.obj
 0002:000144c8       ??_C@_0N@ECMJOJJG@MacroCallFar@ 000000018006a4c8     service.obj
 0002:000144d8       ??_C@_0BC@JJHHFNMP@FarMacroCallToLua@ 000000018006a4d8     service.obj
 0002:000144ec       ??_C@_06GIFLLBB@editor@    000000018006a4ec     service.obj
 0002:000144f4       ??_C@_06DGPPOJKF@viewer@   000000018006a4f4     service.obj
 0002:000144fc       ??_C@_01DICPFPGM@k@        000000018006a4fc     service.obj
 0002:00014500       ??_C@_06BPGFKLEK@__mode@   000000018006a500     service.obj
 0002:00014508       ??_C@_1CC@OPOAGCKN@?$AA?2?$AAl?$AAu?$AAa?$AAf?$AAa?$AAr?$AA_?$AAi?$AAn?$AAi?$AAt?$AA?4?$AAl?$AAu@ 000000018006a508     service.obj
 0002:00014530       ??_C@_1BG@BDOBMIBP@?$AAF?$AAA?$AAR?$AAP?$AAR?$AAO?$AAF?$AAI?$AAL?$AAE@ 000000018006a530     service.obj
 0002:00014548       ??_C@_02KFNNKBCK@io@       000000018006a548     service.obj
 0002:0001454c       ??_C@_02EHCHIAMF@os@       000000018006a54c     service.obj
 0002:00014550       ??_C@_04CFDJAKFL@math@     000000018006a550     service.obj
 0002:00014558       ??_C@_07GAJMMAJO@unicode@  000000018006a558     service.obj
 0002:00014560       ??_C@_04LHHHFLPP@utf8@     000000018006a560     service.obj
 0002:00014568       ??_C@_03JECLAOEA@win@      000000018006a568     service.obj
 0002:0001456c       ??_C@_05NDNJFBEF@cfind@    000000018006a56c     service.obj
 0002:00014574       ??_C@_03EDMBFDDG@bit@      000000018006a574     service.obj
 0002:00014578       ??_C@_03IGHFHLNJ@jit@      000000018006a578     service.obj
 0002:00014580       ??_C@_08LBNNGFKE@_PRELOAD@ 000000018006a580     service.obj
 0002:0001458c       ??_C@_03DIJDOPEA@ffi@      000000018006a58c     service.obj
 0002:00014590       ??_C@_06ONNDGCDK@dofile@   000000018006a590     service.obj
 0002:00014598       ??_C@_08BNNFLGCJ@loadfile@ 000000018006a598     service.obj
 0002:000145a4       ??_C@_06JLGJNGCD@luafar@   000000018006a5a4     service.obj
 0002:000145ac       ??_C@_03OFAPEBGM@?$CFs?6@  000000018006a5ac     service.obj
 0002:000145b0       filefilter_methods         000000018006a5b0     service.obj
 0002:00014620       SettingsType               000000018006a620     service.obj
 0002:00014630       VirtualKeyStrings          000000018006a630     service.obj
 0002:00014e30       FAR_FLAGSTABLE             000000018006ae30     service.obj
 0002:00014e40       SettingsHandles            000000018006ae40     service.obj
 0002:00014e60       FAKE_PLUGIN_DATA_KEY       000000018006ae60     service.obj
 0002:00014e70       SavedScreenType            000000018006ae70     service.obj
 0002:00014e80       editor_funcs               000000018006ae80     service.obj
 0002:00015110       panel_funcs                000000018006b110     service.obj
 0002:00015340       far_Dialog                 000000018006b340     service.obj
 0002:00015570       FarTimerType               000000018006b570     service.obj
 0002:00015580       FarTimerQueueKey           000000018006b580     service.obj
 0002:000155b0       api_functions              000000018006b5b0     service.obj
 0002:00015690       far_host_funcs             000000018006b690     service.obj
 0002:000156f0       far_funcs                  000000018006b6f0     service.obj
 0002:00015c00       FAR_DN_STORAGE             000000018006bc00     service.obj
 0002:00015ce0       timer_methods              000000018006bce0     service.obj
 0002:00015d30       dialog_methods             000000018006bd30     service.obj
 0002:00015d80       FarFileFilterType          000000018006bd80     service.obj
 0002:00015d90       viewer_funcs               000000018006bd90     service.obj
 0002:00015e30       Settings_methods           000000018006be30     service.obj
 0002:00015ed0       FAR_VIRTUALKEYS            000000018006bed0     service.obj
 0002:00015ee8       FarDialogType              000000018006bee8     service.obj
 0002:00015ef8       AddMacroDataType           000000018006bef8     service.obj
 0002:00015f10       PluginHandleType           000000018006bf10     service.obj
 0002:00015f20       ??_C@_0BO@BNLBHKJN@unable?5to?5dump?5given?5function@ 000000018006bf20     slnunico.obj
 0002:00015f40       ??_C@_02HIBBOKEN@?2r@      000000018006bf40     slnunico.obj
 0002:00015f44       ??_C@_04MPDIABOK@?2000@    000000018006bf44     slnunico.obj
 0002:00015f4c       ??_C@_05GGBDHNF@?9?$CL?5?$CD0@ 000000018006bf4c     slnunico.obj
 0002:00015f58       ??_C@_0CA@COOMGCAO@invalid?5format?5?$CIrepeated?5flags?$CJ@ 000000018006bf58     slnunico.obj
 0002:00015f78       ??_C@_0CN@KALFEKPN@invalid?5format?5?$CIwidth?5or?5precis@ 000000018006bf78     slnunico.obj
 0002:00015fa8       ??_C@_0CC@KIPBEOBI@invalid?5option?5?8?$CF?$CF?$CFc?8?5to?5?8forma@ 000000018006bfa8     slnunico.obj
 0002:00015fcc       ??_C@_04GGLOKIEE@dump@     000000018006bfcc     slnunico.obj
 0002:00015fd4       ??_C@_06DLEPGFEF@format@   000000018006bfd4     slnunico.obj
 0002:00015fdc       ??_C@_03HOKODIMJ@rep@      000000018006bfdc     slnunico.obj
 0002:00015fe0       ??_C@_09GCBMKPBD@utf8valid@ 000000018006bfe0     slnunico.obj
 0002:00016040       ??_C@_0BE@LDJANOJE@?$CFs?5expected?0?5got?5?$CFs@ 000000018006c040     lutf8lib.obj
 0002:00016058       ??_C@_0BD@MJACNLBA@invalid?5UTF?98?5code@ 000000018006c058     lutf8lib.obj
 0002:00016070       ??_C@_0BP@MEEJFMAG@initial?5position?5out?5of?5string@ 000000018006c070     lutf8lib.obj
 0002:00016090       ??_C@_0BN@IINPNO@final?5position?5out?5of?5string@ 000000018006c090     lutf8lib.obj
 0002:000160b0       ??_C@_0N@FCPHIMMG@out?5of?5range@ 000000018006c0b0     lutf8lib.obj
 0002:000160c0       ??_C@_0BG@DFAIEAEC@string?5slice?5too?5long@ 000000018006c0c0     lutf8lib.obj
 0002:000160d8       ??_C@_0BD@JFBPAFFP@value?5out?5of?5range@ 000000018006c0d8     lutf8lib.obj
 0002:000160f0       ??_C@_0O@FJKLBAIJ@number?1string@ 000000018006c0f0     lutf8lib.obj
 0002:00016100       ??_C@_0BE@MHMGJPCL@invalid?5escape?5?8?$CFc?8@ 000000018006c100     lutf8lib.obj
 0002:00016118       ??_C@_0O@BGLHAEFA@invalid?5index@ 000000018006c118     lutf8lib.obj
 0002:00016128       ??_C@_0BG@OBAFCJJL@position?5out?5of?5range@ 000000018006c128     lutf8lib.obj
 0002:00016140       ??_C@_0CI@HDBIKOFJ@initial?5position?5is?5a?5continuat@ 000000018006c140     lutf8lib.obj
 0002:00016168       ??_C@_0BL@JNACDPC@invalid?5capture?5index?5?$CF?$CF?$CFd@ 000000018006c168     lutf8lib.obj
 0002:00016188       ??_C@_0BI@ECNPHIBF@invalid?5pattern?5capture@ 000000018006c188     lutf8lib.obj
 0002:000161a0       ??_C@_0CD@PLJBIEHA@malformed?5pattern?5?$CIends?5with?5?8?$CF@ 000000018006c1a0     lutf8lib.obj
 0002:000161c8       ??_C@_0CA@CFGACOGB@malformed?5pattern?5?$CImissing?5?8?$FN?8?$CJ@ 000000018006c1c8     lutf8lib.obj
 0002:000161e8       ??_C@_0CP@FCNHBCLO@malformed?5pattern?5?$CImissing?5argu@ 000000018006c1e8     lutf8lib.obj
 0002:00016218       ??_C@_0BC@IMEAEJPD@too?5many?5captures@ 000000018006c218     lutf8lib.obj
 0002:00016230       ??_C@_0BE@LPFFPFJG@pattern?5too?5complex@ 000000018006c230     lutf8lib.obj
 0002:00016248       ??_C@_0CD@LOJJMDBH@missing?5?8?$FL?8?5after?5?8?$CF?$CFf?8?5in?5patt@ 000000018006c248     lutf8lib.obj
 0002:00016270       ??_C@_0BG@LEHNKOGD@invalid?5capture?5index@ 000000018006c270     lutf8lib.obj
 0002:00016288       ??_C@_0BD@BFKNEALP@unfinished?5capture@ 000000018006c288     lutf8lib.obj
 0002:000162a0       ??_C@_0L@NLFJOONJ@?$FO$?$CK?$CL?$DP?4?$CI?$FL?$CF?9@ 000000018006c2a0     lutf8lib.obj
 0002:000162b0       ??_C@_0CK@KLCOLAN@invalid?5use?5of?5?8?$CFc?8?5in?5replacem@ 000000018006c2b0     lutf8lib.obj
 0002:000162e0       ??_C@_0CB@LPDIHGGA@invalid?5replacement?5value?5?$CIa?5?$CFs@ 000000018006c2e0     lutf8lib.obj
 0002:00016308       ??_C@_0BP@PPPOBACA@string?1function?1table?5expected@ 000000018006c308     lutf8lib.obj
 0002:00016328       ??_C@_06KLHHMIGM@offset@   000000018006c328     lutf8lib.obj
 0002:00016330       ??_C@_05CFHFIAJO@codes@    000000018006c330     lutf8lib.obj
 0002:00016338       ??_C@_09HHCEKEIA@codepoint@ 000000018006c338     lutf8lib.obj
 0002:00016344       ??_C@_03BKCJCHLK@len@      000000018006c344     lutf8lib.obj
 0002:00016348       ??_C@_07KOIEOCCE@reverse@  000000018006c348     lutf8lib.obj
 0002:00016350       ??_C@_05IPJEPLHL@lower@    000000018006c350     lutf8lib.obj
 0002:00016358       ??_C@_05NECKJAMC@upper@    000000018006c358     lutf8lib.obj
 0002:00016360       ??_C@_05PHLGJONK@title@    000000018006c360     lutf8lib.obj
 0002:00016368       ??_C@_04MLGPBLN@fold@      000000018006c368     lutf8lib.obj
 0002:00016370       ??_C@_04IHGKJMLH@byte@     000000018006c370     lutf8lib.obj
 0002:00016378       ??_C@_04ENMBGAPA@char@     000000018006c378     lutf8lib.obj
 0002:00016380       ??_C@_06CHNIFGOF@escape@   000000018006c380     lutf8lib.obj
 0002:00016388       ??_C@_06OAOPNKHP@insert@   000000018006c388     lutf8lib.obj
 0002:00016390       ??_C@_06LEMKAMD@remove@    000000018006c390     lutf8lib.obj
 0002:00016398       ??_C@_07BAPMOMKI@charpos@  000000018006c398     lutf8lib.obj
 0002:000163a0       ??_C@_04CJGEDOF@next@      000000018006c3a0     lutf8lib.obj
 0002:000163a8       ??_C@_05IGKADHGO@width@    000000018006c3a8     lutf8lib.obj
 0002:000163b0       ??_C@_0L@OLBIGGEG@widthindex@ 000000018006c3b0     lutf8lib.obj
 0002:000163c0       ??_C@_08GEDFKPFE@ncasecmp@ 000000018006c3c0     lutf8lib.obj
 0002:000163d0       ??_C@_0M@GMACFGDH@charpattern@ 000000018006c3d0     lutf8lib.obj
 0002:0001640c       ??_C@_05DFJCHPDH@input@    000000018006c40c     uliolib51.obj
 0002:00016414       ??_C@_06DKIGHACF@output@   000000018006c414     uliolib51.obj
 0002:0001641c       ??_C@_06DJHOIPC@?$CFs?3?5?$CFs@ 000000018006c41c     uliolib51.obj
 0002:00016424       ??_C@_02DKCKIIND@?$CFs@    000000018006c424     uliolib51.obj
 0002:00016428       ??_C@_05KCHOJJD@FILE?$CK@  000000018006c428     uliolib51.obj
 0002:00016430       ??_C@_0M@IBKPHHKH@closed?5file@ 000000018006c430     uliolib51.obj
 0002:0001643c       ??_C@_04DAMGJPCA@file@     000000018006c43c     uliolib51.obj
 0002:00016448       ??_C@_0BN@LPOOHAOM@attempt?5to?5use?5a?5closed?5file@ 000000018006c448     uliolib51.obj
 0002:00016468       ??_C@_0BL@PEFGCPAG@cannot?5close?5standard?5file@ 000000018006c468     uliolib51.obj
 0002:00016488       ??_C@_07DMJMBBKE@__close@  000000018006c488     uliolib51.obj
 0002:00016490       ??_C@_0O@PLFAPHPG@file?5?$CIclosed?$CJ@ 000000018006c490     uliolib51.obj
 0002:000164a0       ??_C@_09BPMAMLLD@file?5?$CI?$CFp?$CJ@ 000000018006c4a0     uliolib51.obj
 0002:000164b0       ??_C@_17OBBFBLGE@?$AAr?$AAw?$AAa@ 000000018006c4b0     uliolib51.obj
 0002:000164b8       ??_C@_0CP@DHGANCPP@invalid?5mode?5?8?$CFs?8?5?$CIshould?5match@ 000000018006c4b8     uliolib51.obj
 0002:000164e8       ??_C@_0BL@JMNLNGCA@standard?5?$CFs?5file?5is?5closed@ 000000018006c4e8     uliolib51.obj
 0002:00016504       ??_C@_13CIFDLIMG@?$AAw@    000000018006c504     uliolib51.obj
 0002:00016508       ??_C@_03DLDNIBIK@?$CFlf@   000000018006c508     uliolib51.obj
 0002:00016510       ??_C@_0BD@IOJAAODF@too?5many?5arguments@ 000000018006c510     uliolib51.obj
 0002:00016528       ??_C@_0P@PJFAGLMH@invalid?5option@ 000000018006c528     uliolib51.obj
 0002:00016538       ??_C@_0P@CENJCLHM@invalid?5format@ 000000018006c538     uliolib51.obj
 0002:00016548       ??_C@_0BH@PBGIDLEF@file?5is?5already?5closed@ 000000018006c548     uliolib51.obj
 0002:00016560       ??_C@_05CGOEHEFE@?$CF?414g@ 000000018006c560     uliolib51.obj
 0002:00016568       ??_C@_03KCHOJKKI@set@      000000018006c568     uliolib51.obj
 0002:0001656c       ??_C@_03LIBLMJMB@cur@      000000018006c56c     uliolib51.obj
 0002:00016570       ??_C@_03JBJLGPFL@end@      000000018006c570     uliolib51.obj
 0002:00016578       ??_C@_0BP@MGCOJADF@not?5an?5integer?5in?5proper?5range@ 000000018006c578     uliolib51.obj
 0002:00016598       ??_C@_02KAJCLHKP@no@       000000018006c598     uliolib51.obj
 0002:0001659c       ??_C@_04PLMLMMEO@full@     000000018006c59c     uliolib51.obj
 0002:000165a4       ??_C@_04HJPCFDOP@line@     000000018006c5a4     uliolib51.obj
 0002:000165b0       ??_C@_0DB@KKADAMFH@rawhandle?5is?5only?5available?5in?5@ 000000018006c5b0     uliolib51.obj
 0002:000165e4       ??_C@_05LBOHBHFK@close@    000000018006c5e4     uliolib51.obj
 0002:000165ec       ??_C@_05GLCAEPFP@flush@    000000018006c5ec     uliolib51.obj
 0002:000165f4       ??_C@_05DENOCHIP@lines@    000000018006c5f4     uliolib51.obj
 0002:000165fc       ??_C@_05IACAFMHP@popen@    000000018006c5fc     uliolib51.obj
 0002:00016608       ??_C@_07FKJPAINK@tmpfile@  000000018006c608     uliolib51.obj
 0002:00016610       ??_C@_05NGFEDHGN@write@    000000018006c610     uliolib51.obj
 0002:00016618       ??_C@_04EDECCOGL@seek@     000000018006c618     uliolib51.obj
 0002:00016620       ??_C@_07HHBPNGAN@setvbuf@  000000018006c620     uliolib51.obj
 0002:00016628       ??_C@_05MHOFLBOO@stdin@    000000018006c628     uliolib51.obj
 0002:00016630       ??_C@_06DJDOIFHB@stdout@   000000018006c630     uliolib51.obj
 0002:00016638       ??_C@_06FJGNEBG@stderr@    000000018006c638     uliolib51.obj
 0002:00016810       ??_C@_0BN@GMPFCLAN@unable?5to?5get?5ModuleFileName@ 000000018006c810     uloadlib51.obj
 0002:00016830       ??_C@_13MGDFOILI@?$AA?$CB@ 000000018006c830     uloadlib51.obj
 0002:00016838       ??_C@_09GMLHALBF@LOADLIB?3?5@ 000000018006c838     uloadlib51.obj
 0002:00016844       ??_C@_04HDOCAJNK@?$CFs?$CFs@ 000000018006c844     uloadlib51.obj
 0002:00016850       ??_C@_08HNNNOMMJ@_LOADLIB@ 000000018006c850     uloadlib51.obj
 0002:0001685c       ??_C@_04HKFDNBLD@init@     000000018006c85c     uloadlib51.obj
 0002:00016864       ??_C@_13FPGAJAPJ@?$AA?2@   000000018006c864     uloadlib51.obj
 0002:00016868       ??_C@_13JOFGPIOO@?$AA?4@   000000018006c868     uloadlib51.obj
 0002:00016870       ??_C@_0BO@COFCKCAL@?8package?4?$CFs?8?5must?5be?5a?5string@ 000000018006c870     uloadlib51.obj
 0002:00016890       ??_C@_0CE@EPEHLLIH@?8package?4?$CFs?8?5contains?5invalid?5U@ 000000018006c890     uloadlib51.obj
 0002:000168b4       ??_C@_13HGPDMIBE@?$AA?$DP@ 000000018006c8b4     uloadlib51.obj
 0002:000168b8       ??_C@_0P@NEBKIMDC@?6?7no?5file?5?8?$CFs?8@ 000000018006c8b8     uloadlib51.obj
 0002:000168c8       ??_C@_0CO@KHMIPLKM@error?5loading?5module?5?8?$CFs?8?5from?5@ 000000018006c8c8     uloadlib51.obj
 0002:000168f8       ??_C@_04LNEJFJGI@path@     000000018006c8f8     uloadlib51.obj
 0002:00016900       ??_C@_01IDAFKMJL@_@        000000018006c900     uloadlib51.obj
 0002:00016904       ??_C@_01LFCBOECM@?4@       000000018006c904     uloadlib51.obj
 0002:00016908       ??_C@_0L@KHKMBFOE@luaopen_?$CFs@ 000000018006c908     uloadlib51.obj
 0002:00016914       ??_C@_05EEMJHCCC@cpath@    000000018006c914     uloadlib51.obj
 0002:00016920       ??_C@_0BO@KOILFIGK@?6?7no?5module?5?8?$CFs?8?5in?5file?5?8?$CFs?8@ 000000018006c920     uloadlib51.obj
 0002:00016940       ??_C@_0CC@CCJHFBLH@?8package?4preload?8?5must?5be?5a?5tab@ 000000018006c940     uloadlib51.obj
 0002:00016968       ??_C@_0CB@NPNABMBF@?6?7no?5field?5package?4preload?$FL?8?$CFs?8@ 000000018006c968     uloadlib51.obj
 0002:00016990       ??_C@_07PINPBNPB@_LOADED@  000000018006c990     uloadlib51.obj
 0002:00016998       ??_C@_0CL@DIEJCPFH@loop?5or?5previous?5error?5loading?5@ 000000018006c998     uloadlib51.obj
 0002:000169c8       ??_C@_07JAOCDFCG@loaders@  000000018006c9c8     uloadlib51.obj
 0002:000169d0       ??_C@_0CC@IGEJMOFI@?8package?4loaders?8?5must?5be?5a?5tab@ 000000018006c9d0     uloadlib51.obj
 0002:000169f8       ??_C@_0BJ@HFHHABH@module?5?8?$CFs?8?5not?5found?3?$CFs@ 000000018006c9f8     uloadlib51.obj
 0002:00016a14       ??_C@_01INIBCBCB@f@        000000018006ca14     uloadlib51.obj
 0002:00016a18       ??_C@_0CI@GKOMOAFD@?8module?8?5not?5called?5from?5a?5Lua?5@ 000000018006ca18     uloadlib51.obj
 0002:00016a40       ??_C@_02CCIJHOCI@_M@       000000018006ca40     uloadlib51.obj
 0002:00016a44       ??_C@_05ICMCJINN@_NAME@    000000018006ca44     uloadlib51.obj
 0002:00016a50       ??_C@_08HONLOGDK@_PACKAGE@ 000000018006ca50     uloadlib51.obj
 0002:00016a60       ??_C@_0BO@CBJIAGLF@name?5conflict?5for?5module?5?8?$CFs?8@ 000000018006ca60     uloadlib51.obj
 0002:00016a80       ??_C@_17KOAMMDLI@?$AA?$DL?$AA?$AB?$AA?$DL@ 000000018006ca80     uloadlib51.obj
 0002:00016a88       ??_C@_15HKKNGJC@?$AA?$DL?$AA?$DL@ 000000018006ca88     uloadlib51.obj
 0002:00016a90       ??_C@_13GGAHEHIG@?$AA?$AB@ 000000018006ca90     uloadlib51.obj
 0002:00016a98       ??_C@_07KOEABFCN@loadlib@  000000018006ca98     uloadlib51.obj
 0002:00016aa0       ??_C@_06LNOHAKGK@seeall@   000000018006caa0     uloadlib51.obj
 0002:00016aa8       ??_C@_06BIEEJMKO@module@   000000018006caa8     uloadlib51.obj
 0002:00016ab0       ??_C@_07FFLLPPLH@require@  000000018006cab0     uloadlib51.obj
 0002:00016ac0       ??_C@_1HE@JLDBNBHO@?$AA?4?$AA?2?$AA?$DP?$AA?4?$AAl?$AAu?$AAa?$AA?$DL?$AA?$CB?$AA?2?$AAl?$AAu?$AAa?$AA?2?$AA?$DP@ 000000018006cac0     uloadlib51.obj
 0002:00016b38       ??_C@_1BC@ILFFIBFI@?$AAL?$AAU?$AAA?$AA_?$AAP?$AAA?$AAT?$AAH@ 000000018006cb38     uloadlib51.obj
 0002:00016b50       ??_C@_1DM@FGPGEDD@?$AA?4?$AA?2?$AA?$DP?$AA?4?$AAd?$AAl?$AAl?$AA?$DL?$AA?$CB?$AA?2?$AA?$DP?$AA?4?$AAd?$AAl?$AAl@ 000000018006cb50     uloadlib51.obj
 0002:00016b90       ??_C@_1BE@EFNILHBI@?$AAL?$AAU?$AAA?$AA_?$AAC?$AAP?$AAA?$AAT?$AAH@ 000000018006cb90     uloadlib51.obj
 0002:00016ba8       ??_C@_1BE@CKNDCMBB@?$AA?2?$AA?6?$AA?$DL?$AA?6?$AA?$DP?$AA?6?$AA?$CB?$AA?6?$AA?9@ 000000018006cba8     uloadlib51.obj
 0002:00016bbc       ??_C@_06HEJKKHEK@config@   000000018006cbbc     uloadlib51.obj
 0002:00016bc4       ??_C@_06IILMCCFO@loaded@   000000018006cbc4     uloadlib51.obj
 0002:00016c68       ??_C@_0BB@BLJKPILH@system?5error?5?$CFd?6@ 000000018006cc68     ustring.obj
 0002:00016c80       ??_C@_0BJ@MEAJDMDL@invalid?5multibyte?5string@ 000000018006cc80     ustring.obj
 0002:00016ca0       ??_C@_0BG@ELIKBHAO@invalid?5UTF?916?5string@ 000000018006cca0     ustring.obj
 0002:00016cb8       ??_C@_0M@KJGJBDLL@MaxCharSize@ 000000018006ccb8     ustring.obj
 0002:00016cc8       ??_C@_0M@IMOFNPBB@DefaultChar@ 000000018006ccc8     ustring.obj
 0002:00016cd8       ??_C@_08HIIJAENB@LeadByte@ 000000018006ccd8     ustring.obj
 0002:00016ce8       ??_C@_0BD@CBNPFFPH@UnicodeDefaultChar@ 000000018006cce8     ustring.obj
 0002:00016d00       ??_C@_0N@DJCOCBOB@CodePageName@ 000000018006cd00     ustring.obj
 0002:00016d10       ??_C@_0N@IFJMFGJK@unknown?5type@ 000000018006cd10     ustring.obj
 0002:00016d20       ??_C@_0BC@GPFCFLGN@no?5root?5directory@ 000000018006cd20     ustring.obj
 0002:00016d38       ??_C@_09HPGMKNKO@removable@ 000000018006cd38     ustring.obj
 0002:00016d44       ??_C@_05OFLEIIDM@fixed@    000000018006cd44     ustring.obj
 0002:00016d4c       ??_C@_06IMIHEKN@remote@    000000018006cd4c     ustring.obj
 0002:00016d54       ??_C@_05POABADMF@cdrom@    000000018006cd54     ustring.obj
 0002:00016d60       ??_C@_07BHCBOAMP@ramdisk@  000000018006cd60     ustring.obj
 0002:00016d68       ??_C@_0L@PLJFMBIJ@MemoryLoad@ 000000018006cd68     ustring.obj
 0002:00016d78       ??_C@_09MMAOIBBJ@TotalPhys@ 000000018006cd78     ustring.obj
 0002:00016d88       ??_C@_09KFOEOLH@AvailPhys@ 000000018006cd88     ustring.obj
 0002:00016d98       ??_C@_0O@PEEMGPEP@TotalPageFile@ 000000018006cd98     ustring.obj
 0002:00016da8       ??_C@_0O@LLHOKNF@AvailPageFile@ 000000018006cda8     ustring.obj
 0002:00016db8       ??_C@_0N@LCJEOHMM@TotalVirtual@ 000000018006cdb8     ustring.obj
 0002:00016dc8       ??_C@_0N@EGHLANBF@AvailVirtual@ 000000018006cdc8     ustring.obj
 0002:00016dd8       ??_C@_0BF@KKNLCGDE@AvailExtendedVirtual@ 000000018006cdd8     ustring.obj
 0002:00016df0       ??_C@_0P@KJDDGAFH@FileAttributes@ 000000018006cdf0     ustring.obj
 0002:00016e00       ??_C@_0BE@DEHGONAH@EnumSystemCodePages@ 000000018006ce00     ustring.obj
 0002:00016e14       ??_C@_06FMJLOCAF@GetACP@   000000018006ce14     ustring.obj
 0002:00016e20       ??_C@_09HLFMNDA@GetCPInfo@ 000000018006ce20     ustring.obj
 0002:00016e30       ??_C@_0O@PIBBCLJF@GetCurrentDir@ 000000018006ce30     ustring.obj
 0002:00016e40       ??_C@_0N@IIBOJKJ@GetDriveType@ 000000018006ce40     ustring.obj
 0002:00016e50       ??_C@_0M@KHMMJMNI@GetFileAttr@ 000000018006ce50     ustring.obj
 0002:00016e60       ??_C@_0M@ONGMCNNE@GetKeyState@ 000000018006ce60     ustring.obj
 0002:00016e70       ??_C@_0BH@KKAFOIJJ@GetLogicalDriveStrings@ 000000018006ce70     ustring.obj
 0002:00016e88       ??_C@_08OMCNFONF@GetOEMCP@ 000000018006ce88     ustring.obj
 0002:00016e98       ??_C@_0N@EBDGNADB@GetConsoleCP@ 000000018006ce98     ustring.obj
 0002:00016ea8       ??_C@_0N@DFIIBMHN@SetConsoleCP@ 000000018006cea8     ustring.obj
 0002:00016eb8       ??_C@_0BD@LLGELLLN@GetConsoleOutputCP@ 000000018006ceb8     ustring.obj
 0002:00016ed0       ??_C@_0BD@EBEOINFF@SetConsoleOutputCP@ 000000018006ced0     ustring.obj
 0002:00016ee8       ??_C@_0BD@IHIHPGDL@GlobalMemoryStatus@ 000000018006cee8     ustring.obj
 0002:00016f00       ??_C@_0BE@HCIKGJGE@MultiByteToWideChar@ 000000018006cf00     ustring.obj
 0002:00016f18       ??_C@_09EPINLGBH@OemToUtf8@ 000000018006cf18     ustring.obj
 0002:00016f28       ??_C@_0BC@NFCPMJFM@OutputDebugString@ 000000018006cf28     ustring.obj
 0002:00016f40       ??_C@_0BA@MNJFBAJH@SHGetFolderPath@ 000000018006cf40     ustring.obj
 0002:00016f50       ??_C@_0L@PMCLJMMJ@SearchPath@ 000000018006cf50     ustring.obj
 0002:00016f60       ??_C@_0O@IHAPJIOC@SetCurrentDir@ 000000018006cf60     ustring.obj
 0002:00016f70       ??_C@_0M@KINCEKFL@SetFileAttr@ 000000018006cf70     ustring.obj
 0002:00016f7c       ??_C@_05PFDOMJEF@Sleep@    000000018006cf7c     ustring.obj
 0002:00016f88       ??_C@_0M@KJELMDJD@Utf16ToUtf8@ 000000018006cf88     ustring.obj
 0002:00016f98       ??_C@_09LCEKPEGC@Utf8ToOem@ 000000018006cf98     ustring.obj
 0002:00016fa8       ??_C@_0M@GJGCILHG@Utf8ToUtf16@ 000000018006cfa8     ustring.obj
 0002:00016fb4       ??_C@_04NDFIEGPL@Uuid@     000000018006cfb4     ustring.obj
 0002:00016fc0       ??_C@_0BE@LJADKLBD@WideCharToMultiByte@ 000000018006cfc0     ustring.obj
 0002:00016fd4       ??_C@_04GFOHBGIO@subW@     000000018006cfd4     ustring.obj
 0002:00016fdc       ??_C@_06FHFOAHML@system@   000000018006cfdc     ustring.obj
 0002:00016fe4       ??_C@_04NOFELICG@lenW@     000000018006cfe4     ustring.obj
 0002:00016ff0       ??_C@_07JOJHCKGP@ustring@  000000018006cff0     ustring.obj
 0002:00017000       ustring_funcs              000000018006d000     ustring.obj
 0002:000171f0       ??_C@_0DJ@KKHMCMAP@bad?5field?5?$FL?$CFd?$FN?5in?5table?5stackpo@ 000000018006d1f0     util.obj
 0002:00017230       ??_C@_0DJ@PFHHGAMM@bad?5field?5?8?$CFs?8?5in?5table?5stackpo@ 000000018006d230     util.obj
 0002:0001726c       ??_C@_06EBGNBFIA@number@   000000018006d26c     util.obj
 0002:00017274       ??_C@_04CBBMIBLK@HKLM@     000000018006d274     win.obj
 0002:0001727c       ??_C@_04LEMDOLAJ@HKCC@     000000018006d27c     win.obj
 0002:00017284       ??_C@_04OHBKMIBJ@HKCR@     000000018006d284     win.obj
 0002:0001728c       ??_C@_04KIFLFONO@HKCU@     000000018006d28c     win.obj
 0002:00017294       ??_C@_03DLBIJLAB@HKU@      000000018006d294     win.obj
 0002:00017298       ??_C@_0DA@DKALLFDI@must?5be?5?8HKLM?8?0?5?8HKCC?8?0?5?8HKCR?8?0@ 000000018006d298     win.obj
 0002:000172c8       ??_C@_05KDALNKAH@dword@    000000018006d2c8     win.obj
 0002:000172d0       ??_C@_06FNFBAEBE@binary@   000000018006d2d0     win.obj
 0002:000172d8       ??_C@_0N@CBOMHLPN@expandstring@ 000000018006d2d8     win.obj
 0002:000172e8       ??_C@_0M@PEGIPCHN@multistring@ 000000018006d2e8     win.obj
 0002:000172f8       ??_C@_0BH@NOJOGNJM@unsupported?5value?5type@ 000000018006d2f8     win.obj
 0002:00017310       ??_C@_0BD@MJODDCFG@OpenRegKey?5failed?4@ 000000018006d310     win.obj
 0002:00017328       ??_C@_0BI@COLHBIIE@RegQueryValueEx?5failed?4@ 000000018006d328     win.obj
 0002:00017340       ??_C@_1BK@BIGILECK@?$AAA?$AAd?$AAv?$AAa?$AAp?$AAi?$AA3?$AA2?$AA?4?$AAd?$AAl?$AAl@ 000000018006d340     win.obj
 0002:00017360       ??_C@_0BA@LILAPHGE@RegDeleteKeyExW@ 000000018006d360     win.obj
 0002:00017370       ??_C@_0BG@HHFHBIKG@RegOpenKeyExW?5failed?4@ 000000018006d370     win.obj
 0002:00017388       ??_C@_05DFPNHDMN@wYear@    000000018006d388     win.obj
 0002:00017390       ??_C@_06MGNNJGBJ@wMonth@   000000018006d390     win.obj
 0002:00017398       ??_C@_0L@OAHPHHP@wDayOfWeek@ 000000018006d398     win.obj
 0002:000173a4       ??_C@_04NBLBJIPP@wDay@     000000018006d3a4     win.obj
 0002:000173ac       ??_C@_05BMOPCGDH@wHour@    000000018006d3ac     win.obj
 0002:000173b8       ??_C@_07HPODENI@wMinute@   000000018006d3b8     win.obj
 0002:000173c0       ??_C@_07IIEDHHJN@wSecond@  000000018006d3c0     win.obj
 0002:000173c8       ??_C@_0O@HBAPEOKP@wMilliseconds@ 000000018006d3c8     win.obj
 0002:000173d8       ??_C@_0BA@IAFODGNM@CursorPositionX@ 000000018006d3d8     win.obj
 0002:000173e8       ??_C@_0BA@JJEFAHJN@CursorPositionY@ 000000018006d3e8     win.obj
 0002:000173f8       ??_C@_0L@NFCEOFBF@WindowLeft@ 000000018006d3f8     win.obj
 0002:00017408       ??_C@_09JHGOALHG@WindowTop@ 000000018006d408     win.obj
 0002:00017418       ??_C@_0M@HHPHMPGH@WindowRight@ 000000018006d418     win.obj
 0002:00017428       ??_C@_0N@JPIJCAOJ@WindowBottom@ 000000018006d428     win.obj
 0002:00017438       ??_C@_0BD@DOLDEII@MaximumWindowSizeX@ 000000018006d438     win.obj
 0002:00017450       ??_C@_0BD@BKPAAFMJ@MaximumWindowSizeY@ 000000018006d450     win.obj
 0002:00017464       ??_C@_01PFHFFBPC@t@        000000018006d464     win.obj
 0002:00017468       ??_C@_0BJ@LPJMBJJL@directory?5already?5exists@ 000000018006d468     win.obj
 0002:00017484       ??_C@_02NIKKAELB@XP@       000000018006d484     win.obj
 0002:00017488       ??_C@_05OFKKJCED@XPSP1@    000000018006d488     win.obj
 0002:00017490       ??_C@_05MOIHMBIA@XPSP2@    000000018006d490     win.obj
 0002:00017498       ??_C@_05NHJMPAMB@XPSP3@    000000018006d498     win.obj
 0002:000174a0       ??_C@_05FGFMDFJC@Vista@    000000018006d4a0     win.obj
 0002:000174a8       ??_C@_08ENCCDKOP@VistaSP1@ 000000018006d4a8     win.obj
 0002:000174b8       ??_C@_08GGAPGJCM@VistaSP2@ 000000018006d4b8     win.obj
 0002:000174c4       ??_C@_02PJEKLOOM@W7@       000000018006d4c4     win.obj
 0002:000174c8       ??_C@_05DPOOILML@W7SP1@    000000018006d4c8     win.obj
 0002:000174d0       ??_C@_02HONCKCCD@W8@       000000018006d4d0     win.obj
 0002:000174d4       ??_C@_04HCPPKHCP@W8?41@    000000018006d4d4     win.obj
 0002:000174dc       ??_C@_03HCIOKOKM@W10@      000000018006d4dc     win.obj
 0002:000174e0       ??_C@_06LGMEBDBC@Server@   000000018006d4e0     win.obj
 0002:000174e8       ??_C@_0BH@CNFJKJGO@invalid?5argument?5value@ 000000018006d4e8     win.obj
 0002:00017500       ??_C@_0BK@LNHOAEDA@must?5be?5string?5or?5integer@ 000000018006d500     win.obj
 0002:00017520       ??_C@_0BK@JGAEKFII@invalid?5value?5at?5key?5?8?$CFs?8@ 000000018006d520     win.obj
 0002:00017540       ??_C@_0O@CFPMOCDP@CompareString@ 000000018006d540     win.obj
 0002:00017550       ??_C@_08PPLNFCGA@CopyFile@ 000000018006d550     win.obj
 0002:00017560       ??_C@_09INHPLKKM@CreateDir@ 000000018006d560     win.obj
 0002:00017570       ??_C@_0L@GPLPOFDC@DeleteFile@ 000000018006d570     win.obj
 0002:00017580       ??_C@_0N@FOJPHHPH@DeleteRegKey@ 000000018006d580     win.obj
 0002:00017590       ??_C@_0P@PCCDOIAL@DeleteRegValue@ 000000018006d590     win.obj
 0002:000175a0       ??_C@_0L@DGAGCFOP@EnumRegKey@ 000000018006d5a0     win.obj
 0002:000175b0       ??_C@_0N@PFFNCIBD@EnumRegValue@ 000000018006d5b0     win.obj
 0002:000175c0       ??_C@_0L@MGMEFCAE@ExtractKey@ 000000018006d5c0     win.obj
 0002:000175d0       ??_C@_0N@HALOIPMN@ExtractKeyEx@ 000000018006d5d0     win.obj
 0002:000175e0       ??_C@_0N@DNBFBBHK@IsWinVersion@ 000000018006d5e0     win.obj
 0002:000175f0       ??_C@_0BI@EKFDIGHI@FileTimeToLocalFileTime@ 000000018006d5f0     win.obj
 0002:00017608       ??_C@_0BF@KPJNHALE@FileTimeToSystemTime@ 000000018006d608     win.obj
 0002:00017620       ??_C@_0BL@NAIJNMLL@GetConsoleScreenBufferInfo@ 000000018006d620     win.obj
 0002:0001763c       ??_C@_06CALCCDMF@GetEnv@   000000018006d63c     win.obj
 0002:00017648       ??_C@_0M@EINGHLOA@GetFileInfo@ 000000018006d648     win.obj
 0002:00017658       ??_C@_0N@HDKONBLE@GetFileTimes@ 000000018006d658     win.obj
 0002:00017668       ??_C@_09GFGIAJLD@GetRegKey@ 000000018006d668     win.obj
 0002:00017678       ??_C@_0BI@ENMDHCMK@GetSystemTimeAsFileTime@ 000000018006d678     win.obj
 0002:00017690       ??_C@_0P@GGGHOPAD@GetVirtualKeys@ 000000018006d690     win.obj
 0002:000176a0       ??_C@_0P@MIPPOCAO@IsProcess64bit@ 000000018006d6a0     win.obj
 0002:000176b0       ??_C@_08CALLHOCI@MoveFile@ 000000018006d6b0     win.obj
 0002:000176c0       ??_C@_09EDKALOCB@RemoveDir@ 000000018006d6c0     win.obj
 0002:000176d0       ??_C@_0L@HBAGBENL@RenameFile@ 000000018006d6d0     win.obj
 0002:000176dc       ??_C@_06LDCDJLBI@SetEnv@   000000018006d6dc     win.obj
 0002:000176e8       ??_C@_0N@HBABNPI@SetFileTimes@ 000000018006d6e8     win.obj
 0002:000176f8       ??_C@_09ELCNCICB@SetRegKey@ 000000018006d6f8     win.obj
 0002:00017708       ??_C@_0N@BFFIJKHB@ShellExecute@ 000000018006d708     win.obj
 0002:00017718       ??_C@_0BF@HBHGIPOG@SystemTimeToFileTime@ 000000018006d718     win.obj
 0002:00017730       ??_C@_06DNONFAKH@wcscmp@   000000018006d730     win.obj
 0002:00017738       ??_C@_0N@OCKOJJEP@WriteConsole@ 000000018006d738     win.obj
 0002:00017750       win_funcs                  000000018006d750     win.obj
 0002:00017950       __real@3ff0000000000000    000000018006d950     service.obj
 0002:00017958       __real@4059000000000000    000000018006d958     service.obj
 0002:00017960       __real@41e0000000000000    000000018006d960     service.obj
 0002:00017968       __real@41f0000000000000    000000018006d968     win.obj
 0002:00017970       __real@43e0000000000000    000000018006d970     util.obj
 0002:00017978       __real@bff0000000000000    000000018006d978     exported.obj
 0002:00017980       __xmm@80000000000000008000000000000000 000000018006d980     bit64.obj
 0002:00017990       __xmm@ffffffffffffffffffffffffffffffff 000000018006d990     service.obj
 0002:00017a00       _load_config_used          000000018006da00     LIBCMT:loadcfg.obj
 0002:00017b80       __volatile_metadata        000000018006db80     <linker-defined>
 0002:00017e98       __rtc_iaa                  000000018006de98     LIBCMT:initsect.obj
 0002:00017ea0       __rtc_izz                  000000018006dea0     LIBCMT:initsect.obj
 0002:00017ea8       __rtc_taa                  000000018006dea8     LIBCMT:initsect.obj
 0002:00017eb0       __rtc_tzz                  000000018006deb0     LIBCMT:initsect.obj
 0002:0001cd4c       __IMPORT_DESCRIPTOR_KERNEL32 0000000180072d4c     kernel32:KERNEL32.dll
 0002:0001cd60       __IMPORT_DESCRIPTOR_ADVAPI32 0000000180072d60     advapi32:ADVAPI32.dll
 0002:0001cd74       __IMPORT_DESCRIPTOR_USER32 0000000180072d74     user32:USER32.dll
 0002:0001cd88       __IMPORT_DESCRIPTOR_SHELL32 0000000180072d88     shell32:SHELL32.dll
 0002:0001cd9c       __IMPORT_DESCRIPTOR_RPCRT4 0000000180072d9c     rpcrt4:RPCRT4.dll
 0002:0001cdb0       __IMPORT_DESCRIPTOR_lua51  0000000180072db0     lua51:lua51.dll
 0002:0001cdc4       __NULL_IMPORT_DESCRIPTOR   0000000180072dc4     kernel32:KERNEL32.dll
 0003:00000000       __security_cookie_complement 0000000180075000     LIBCMT:gs_cookie.obj
 0003:00000008       __security_cookie          0000000180075008     LIBCMT:gs_cookie.obj
 0003:00000010       __scrt_native_dllmain_reason 0000000180075010     LIBCMT:utility.obj
 0003:00000018       __isa_available            0000000180075018     LIBCMT:cpu_disp.obj
 0003:0000001c       __isa_enabled              000000018007501c     LIBCMT:cpu_disp.obj
 0003:00000020       __memcpy_nt_iters          0000000180075020     LIBCMT:cpu_disp.obj
 0003:00000028       __memset_nt_iters          0000000180075028     LIBCMT:cpu_disp.obj
 0003:00000050       _iob                       0000000180075050     libucrt:_file.obj
 0003:00000160       __abort_behavior           0000000180075160     libucrt:abort.obj
 0003:00000170       __acrt_initial_locale_data 0000000180075170     libucrt:nlsdata.obj
 0003:000002c8       __acrt_initial_locale_pointers 00000001800752c8     libucrt:nlsdata.obj
 0003:000002d8       __acrt_wide_c_locale_string 00000001800752d8     libucrt:nlsdata.obj
 0003:000002e0       __badioinfo                00000001800752e0     libucrt:ioinit.obj
 0003:00000330       _lookuptrailbytes          0000000180075330     libucrt:read.obj
 0003:00000430       _pwctype                   0000000180075430     libucrt:ctype.obj
 0003:00000440       __acrt_initial_multibyte_data 0000000180075440     libucrt:mbctype.obj
 0003:00000980       __globallocalestatus       0000000180075980     libucrt:glstatus.obj
 0003:00000990       __acrt_lconv_c             0000000180075990     libucrt:localeconv.obj
 0003:00000a28       __acrt_lconv_static_decimal 0000000180075a28     libucrt:localeconv.obj
 0003:00000a2c       __acrt_lconv_static_W_decimal 0000000180075a2c     libucrt:localeconv.obj
 0003:00000a44       _fltused                   0000000180075a44     LIBCMT:fltused.obj
 0003:00000a50       GetPluginData              0000000180075a50     service.obj
 0003:0000c120       ?__type_info_root_node@@3U__type_info_node@@A 0000000180081120     LIBCMT:tncleanup.obj
 0003:0000c130       __scrt_current_native_startup_state 0000000180081130     LIBCMT:utility.obj
 0003:0000c138       __scrt_native_startup_lock 0000000180081138     LIBCMT:utility.obj
 0003:0000c178       __scrt_debugger_hook_flag  0000000180081178     LIBCMT:utility_desktop.obj
 0003:0000c180       __castguard_check_failure_os_handled_fptr 0000000180081180     LIBCMT:guard_support.obj
 0003:0000c188       __favor                    0000000180081188     LIBCMT:cpu_disp.obj
 0003:0000c190       ?__WinRTOutOfMemoryExceptionCallback@@3P6APEAXXZEA 0000000180081190     libvcruntime:ehhelpers.obj
 0003:0000c198       ?pArgList@UnDecorator@@0PEAVReplicator@@EA 0000000180081198     libvcruntime:undname.obj
 0003:0000c1a0       ?pZNameList@UnDecorator@@0PEAVReplicator@@EA 00000001800811a0     libvcruntime:undname.obj
 0003:0000c1a8       ?pTemplateArgList@UnDecorator@@0PEAVReplicator@@EA 00000001800811a8     libvcruntime:undname.obj
 0003:0000c1b0       ?gName@UnDecorator@@0PEBDEB 00000001800811b0     libvcruntime:undname.obj
 0003:0000c1b8       ?name@UnDecorator@@0PEBDEB 00000001800811b8     libvcruntime:undname.obj
 0003:0000c1c0       ?disableFlags@UnDecorator@@0KA 00000001800811c0     libvcruntime:undname.obj
 0003:0000c1c4       ?fExplicitTemplateParams@UnDecorator@@0_NA 00000001800811c4     libvcruntime:undname.obj
 0003:0000c1c5       ?fGetTemplateArgumentList@UnDecorator@@0_NA 00000001800811c5     libvcruntime:undname.obj
 0003:0000c1c8       ?m_pGetParameter@UnDecorator@@0P6APEADJ@ZEA 00000001800811c8     libvcruntime:undname.obj
 0003:0000c1d0       ?m_CHPENameOffset@UnDecorator@@0KA 00000001800811d0     libvcruntime:undname.obj
 0003:0000c1d4       ?m_recursionLevel@UnDecorator@@0KA 00000001800811d4     libvcruntime:undname.obj
 0003:0000c2f0       __pPurecall                00000001800812f0     libvcruntime:purevirt_data.obj
 0003:0000c2f8       _nstream                   00000001800812f8     libucrt:_file.obj
 0003:0000c300       __piob                     0000000180081300     libucrt:_file.obj
 0003:0000c308       _cflush                    0000000180081308     libucrt:_file.obj
 0003:0000c360       ?c_exit_complete@?1???R<lambda_6e4b09c48022b2350581041d5f6b0c4c>@@QEBA@XZ@4_NA 0000000180081360     libucrt:exit.obj
 0003:0000c478       _environ_table             0000000180081478     libucrt:environment_initialization.obj
 0003:0000c480       _wenviron_table            0000000180081480     libucrt:environment_initialization.obj
 0003:0000c488       __dcrt_initial_wide_environment 0000000180081488     libucrt:environment_initialization.obj
 0003:0000c490       __dcrt_initial_narrow_environment 0000000180081490     libucrt:environment_initialization.obj
 0003:0000c498       __acrt_atexit_table        0000000180081498     libucrt:onexit.obj
 0003:0000c4b0       __acrt_at_quick_exit_table 00000001800814b0     libucrt:onexit.obj
 0003:0000c4e0       __acrt_stdout_buffer       00000001800814e0     libucrt:_sftbuf.obj
 0003:0000c4e8       __acrt_stderr_buffer       00000001800814e8     libucrt:_sftbuf.obj
 0003:0000c4f0       __acrt_locale_changed_data 00000001800814f0     libucrt:wsetlocale.obj
 0003:0000c4f8       __acrt_current_locale_data 00000001800814f8     libucrt:nlsdata.obj
 0003:0000c500       __pioinfo                  0000000180081500     libucrt:ioinit.obj
 0003:0000c900       _nhandle                   0000000180081900     libucrt:ioinit.obj
 0003:0000ccf4       _commode                   0000000180081cf4     libucrt:ncommode.obj
 0003:0000ccf8       _mbctype                   0000000180081cf8     libucrt:mbctype.obj
 0003:0000cd00       _mbcasemap                 0000000180081d00     libucrt:mbctype.obj
 0003:0000cd08       __acrt_current_multibyte_data 0000000180081d08     libucrt:mbctype.obj
 0003:0000cd18       _pgmptr                    0000000180081d18     libucrt:argv_data.obj
 0003:0000cd20       __argc                     0000000180081d20     libucrt:argv_data.obj
 0003:0000cd28       __argv                     0000000180081d28     libucrt:argv_data.obj
 0003:0000cd30       __wargv                    0000000180081d30     libucrt:argv_data.obj
 0003:0000cd38       _acmdln                    0000000180081d38     libucrt:argv_data.obj
 0003:0000cd40       _wcmdln                    0000000180081d40     libucrt:argv_data.obj
 0003:0000cd48       __acrt_heap                0000000180081d48     libucrt:heap_handle.obj
 0003:0000cd84       __acrt_lconv_static_null   0000000180081d84     libucrt:localeconv.obj
 0003:0000cd88       __acrt_lconv_static_W_null 0000000180081d88     libucrt:localeconv.obj
 0003:0000cd8c       _umaskval                  0000000180081d8c     libucrt:umask.obj
 0003:0000cd9c       _fmode                     0000000180081d9c     libucrt:txtmode.obj
 0003:0000cda0       __fma3_is_available        0000000180081da0     libucrt:fma3_available.obj
 0003:0000cda4       __use_fma3_lib             0000000180081da4     libucrt:fma3_available.obj
 0003:0000cdc0       __scrt_ucrt_dll_is_in_use  0000000180081dc0     <common>
 0003:0000cdc8       __dyn_tls_init_callback    0000000180081dc8     <common>
 0003:0000cdd0       EnumCP                     0000000180081dd0     <common>
 0003:0000cde0       ?_OptionsStorage@?1??__local_stdio_printf_options@@9@9 0000000180081de0     <common>
 0003:0000cde8       ?_OptionsStorage@?1??__local_stdio_scanf_options@@9@9 0000000180081de8     <common>

 entry point at        0001:000354fc

 Static symbols

 0000:fff75000       .debug$S                   0000000180000000     luafar3.exp
 0000:fff75000       .debug$S                   0000000180000000     advapi32:ADVAPI32.dll
 0000:fff75000       .debug$S                   0000000180000000     advapi32:ADVAPI32.dll
 0000:fff75000       .debug$S                   0000000180000000     advapi32:ADVAPI32.dll
 0000:fff75000       .debug$S                   0000000180000000     advapi32:ADVAPI32.dll
 0000:fff75000       .debug$S                   0000000180000000     advapi32:ADVAPI32.dll
 0000:fff75000       .debug$S                   0000000180000000     advapi32:ADVAPI32.dll
 0000:fff75000       .debug$S                   0000000180000000     advapi32:ADVAPI32.dll
 0000:fff75000       .debug$S                   0000000180000000     advapi32:ADVAPI32.dll
 0000:fff75000       .debug$S                   0000000180000000     advapi32:ADVAPI32.dll
 0000:fff75000       .debug$S                   0000000180000000     kernel32:KERNEL32.dll
 0000:fff75000       .debug$S                   0000000180000000     kernel32:KERNEL32.dll
 0000:fff75000       .debug$S                   0000000180000000     kernel32:KERNEL32.dll
 0000:fff75000       .debug$S                   0000000180000000     kernel32:KERNEL32.dll
 0000:fff75000       .debug$S                   0000000180000000     kernel32:KERNEL32.dll
 0000:fff75000       .debug$S                   0000000180000000     kernel32:KERNEL32.dll
 0000:fff75000       .debug$S                   0000000180000000     kernel32:KERNEL32.dll
 0000:fff75000       .debug$S                   0000000180000000     kernel32:KERNEL32.dll
 0000:fff75000       .debug$S                   0000000180000000     kernel32:KERNEL32.dll
 0000:fff75000       .debug$S                   0000000180000000     kernel32:KERNEL32.dll
 0000:fff75000       .debug$S                   0000000180000000     kernel32:KERNEL32.dll
 0000:fff75000       .debug$S                   0000000180000000     kernel32:KERNEL32.dll
 0000:fff75000       .debug$S                   0000000180000000     kernel32:KERNEL32.dll
 0000:fff75000       .debug$S                   0000000180000000     kernel32:KERNEL32.dll
 0000:fff75000       .debug$S                   0000000180000000     kernel32:KERNEL32.dll
 0000:fff75000       .debug$S                   0000000180000000     kernel32:KERNEL32.dll
 0000:fff75000       .debug$S                   0000000180000000     kernel32:KERNEL32.dll
 0000:fff75000       .debug$S                   0000000180000000     kernel32:KERNEL32.dll
 0000:fff75000       .debug$S                   0000000180000000     kernel32:KERNEL32.dll
 0000:fff75000       .debug$S                   0000000180000000     kernel32:KERNEL32.dll
 0000:fff75000       .debug$S                   0000000180000000     kernel32:KERNEL32.dll
 0000:fff75000       .debug$S                   0000000180000000     kernel32:KERNEL32.dll
 0000:fff75000       .debug$S                   0000000180000000     kernel32:KERNEL32.dll
 0000:fff75000       .debug$S                   0000000180000000     kernel32:KERNEL32.dll
 0000:fff75000       .debug$S                   0000000180000000     kernel32:KERNEL32.dll
 0000:fff75000       .debug$S                   0000000180000000     kernel32:KERNEL32.dll
 0000:fff75000       .debug$S                   0000000180000000     kernel32:KERNEL32.dll
 0000:fff75000       .debug$S                   0000000180000000     kernel32:KERNEL32.dll
 0000:fff75000       .debug$S                   0000000180000000     kernel32:KERNEL32.dll
 0000:fff75000       .debug$S                   0000000180000000     kernel32:KERNEL32.dll
 0000:fff75000       .debug$S                   0000000180000000     kernel32:KERNEL32.dll
 0000:fff75000       .debug$S                   0000000180000000     kernel32:KERNEL32.dll
 0000:fff75000       .debug$S                   0000000180000000     kernel32:KERNEL32.dll
 0000:fff75000       .debug$S                   0000000180000000     kernel32:KERNEL32.dll
 0000:fff75000       .debug$S                   0000000180000000     kernel32:KERNEL32.dll
 0000:fff75000       .debug$S                   0000000180000000     kernel32:KERNEL32.dll
 0000:fff75000       .debug$S                   0000000180000000     kernel32:KERNEL32.dll
 0000:fff75000       .debug$S                   0000000180000000     kernel32:KERNEL32.dll
 0000:fff75000       .debug$S                   0000000180000000     kernel32:KERNEL32.dll
 0000:fff75000       .debug$S                   0000000180000000     kernel32:KERNEL32.dll
 0000:fff75000       .debug$S                   0000000180000000     kernel32:KERNEL32.dll
 0000:fff75000       .debug$S                   0000000180000000     kernel32:KERNEL32.dll
 0000:fff75000       .debug$S                   0000000180000000     kernel32:KERNEL32.dll
 0000:fff75000       .debug$S                   0000000180000000     kernel32:KERNEL32.dll
 0000:fff75000       .debug$S                   0000000180000000     kernel32:KERNEL32.dll
 0000:fff75000       .debug$S                   0000000180000000     kernel32:KERNEL32.dll
 0000:fff75000       .debug$S                   0000000180000000     kernel32:KERNEL32.dll
 0000:fff75000       .debug$S                   0000000180000000     kernel32:KERNEL32.dll
 0000:fff75000       .debug$S                   0000000180000000     kernel32:KERNEL32.dll
 0000:fff75000       .debug$S                   0000000180000000     kernel32:KERNEL32.dll
 0000:fff75000       .debug$S                   0000000180000000     kernel32:KERNEL32.dll
 0000:fff75000       .debug$S                   0000000180000000     kernel32:KERNEL32.dll
 0000:fff75000       .debug$S                   0000000180000000     kernel32:KERNEL32.dll
 0000:fff75000       .debug$S                   0000000180000000     kernel32:KERNEL32.dll
 0000:fff75000       .debug$S                   0000000180000000     kernel32:KERNEL32.dll
 0000:fff75000       .debug$S                   0000000180000000     kernel32:KERNEL32.dll
 0000:fff75000       .debug$S                   0000000180000000     kernel32:KERNEL32.dll
 0000:fff75000       .debug$S                   0000000180000000     kernel32:KERNEL32.dll
 0000:fff75000       .debug$S                   0000000180000000     kernel32:KERNEL32.dll
 0000:fff75000       .debug$S                   0000000180000000     kernel32:KERNEL32.dll
 0000:fff75000       .debug$S                   0000000180000000     kernel32:KERNEL32.dll
 0000:fff75000       .debug$S                   0000000180000000     kernel32:KERNEL32.dll
 0000:fff75000       .debug$S                   0000000180000000     kernel32:KERNEL32.dll
 0000:fff75000       .debug$S                   0000000180000000     kernel32:KERNEL32.dll
 0000:fff75000       .debug$S                   0000000180000000     kernel32:KERNEL32.dll
 0000:fff75000       .debug$S                   0000000180000000     kernel32:KERNEL32.dll
 0000:fff75000       .debug$S                   0000000180000000     kernel32:KERNEL32.dll
 0000:fff75000       .debug$S                   0000000180000000     kernel32:KERNEL32.dll
 0000:fff75000       .debug$S                   0000000180000000     kernel32:KERNEL32.dll
 0000:fff75000       .debug$S                   0000000180000000     kernel32:KERNEL32.dll
 0000:fff75000       .debug$S                   0000000180000000     kernel32:KERNEL32.dll
 0000:fff75000       .debug$S                   0000000180000000     kernel32:KERNEL32.dll
 0000:fff75000       .debug$S                   0000000180000000     kernel32:KERNEL32.dll
 0000:fff75000       .debug$S                   0000000180000000     kernel32:KERNEL32.dll
 0000:fff75000       .debug$S                   0000000180000000     kernel32:KERNEL32.dll
 0000:fff75000       .debug$S                   0000000180000000     kernel32:KERNEL32.dll
 0000:fff75000       .debug$S                   0000000180000000     kernel32:KERNEL32.dll
 0000:fff75000       .debug$S                   0000000180000000     kernel32:KERNEL32.dll
 0000:fff75000       .debug$S                   0000000180000000     kernel32:KERNEL32.dll
 0000:fff75000       .debug$S                   0000000180000000     kernel32:KERNEL32.dll
 0000:fff75000       .debug$S                   0000000180000000     kernel32:KERNEL32.dll
 0000:fff75000       .debug$S                   0000000180000000     kernel32:KERNEL32.dll
 0000:fff75000       .debug$S                   0000000180000000     kernel32:KERNEL32.dll
 0000:fff75000       .debug$S                   0000000180000000     kernel32:KERNEL32.dll
 0000:fff75000       .debug$S                   0000000180000000     kernel32:KERNEL32.dll
 0000:fff75000       .debug$S                   0000000180000000     kernel32:KERNEL32.dll
 0000:fff75000       .debug$S                   0000000180000000     kernel32:KERNEL32.dll
 0000:fff75000       .debug$S                   0000000180000000     kernel32:KERNEL32.dll
 0000:fff75000       .debug$S                   0000000180000000     kernel32:KERNEL32.dll
 0000:fff75000       .debug$S                   0000000180000000     kernel32:KERNEL32.dll
 0000:fff75000       .debug$S                   0000000180000000     kernel32:KERNEL32.dll
 0000:fff75000       .debug$S                   0000000180000000     kernel32:KERNEL32.dll
 0000:fff75000       .debug$S                   0000000180000000     kernel32:KERNEL32.dll
 0000:fff75000       .debug$S                   0000000180000000     kernel32:KERNEL32.dll
 0000:fff75000       .debug$S                   0000000180000000     kernel32:KERNEL32.dll
 0000:fff75000       .debug$S                   0000000180000000     kernel32:KERNEL32.dll
 0000:fff75000       .debug$S                   0000000180000000     kernel32:KERNEL32.dll
 0000:fff75000       .debug$S                   0000000180000000     kernel32:KERNEL32.dll
 0000:fff75000       .debug$S                   0000000180000000     kernel32:KERNEL32.dll
 0000:fff75000       .debug$S                   0000000180000000     kernel32:KERNEL32.dll
 0000:fff75000       .debug$S                   0000000180000000     kernel32:KERNEL32.dll
 0000:fff75000       .debug$S                   0000000180000000     kernel32:KERNEL32.dll
 0000:fff75000       .debug$S                   0000000180000000     kernel32:KERNEL32.dll
 0000:fff75000       .debug$S                   0000000180000000     kernel32:KERNEL32.dll
 0000:fff75000       .debug$S                   0000000180000000     kernel32:KERNEL32.dll
 0000:fff75000       .debug$S                   0000000180000000     kernel32:KERNEL32.dll
 0000:fff75000       .debug$S                   0000000180000000     kernel32:KERNEL32.dll
 0000:fff75000       .debug$S                   0000000180000000     kernel32:KERNEL32.dll
 0000:fff75000       .debug$S                   0000000180000000     kernel32:KERNEL32.dll
 0000:fff75000       .debug$S                   0000000180000000     kernel32:KERNEL32.dll
 0000:fff75000       .debug$S                   0000000180000000     kernel32:KERNEL32.dll
 0000:fff75000       .debug$S                   0000000180000000     kernel32:KERNEL32.dll
 0000:fff75000       .debug$S                   0000000180000000     kernel32:KERNEL32.dll
 0000:fff75000       .debug$S                   0000000180000000     kernel32:KERNEL32.dll
 0000:fff75000       .debug$S                   0000000180000000     kernel32:KERNEL32.dll
 0000:fff75000       .debug$S                   0000000180000000     kernel32:KERNEL32.dll
 0000:fff75000       .debug$S                   0000000180000000     kernel32:KERNEL32.dll
 0000:fff75000       .debug$S                   0000000180000000     kernel32:KERNEL32.dll
 0000:fff75000       .debug$S                   0000000180000000     kernel32:KERNEL32.dll
 0000:fff75000       .debug$S                   0000000180000000     kernel32:KERNEL32.dll
 0000:fff75000       .debug$S                   0000000180000000     kernel32:KERNEL32.dll
 0000:fff75000       .debug$S                   0000000180000000     kernel32:KERNEL32.dll
 0000:fff75000       .debug$S                   0000000180000000     kernel32:KERNEL32.dll
 0000:fff75000       .debug$S                   0000000180000000     kernel32:KERNEL32.dll
 0000:fff75000       .debug$S                   0000000180000000     kernel32:KERNEL32.dll
 0000:fff75000       .debug$S                   0000000180000000     kernel32:KERNEL32.dll
 0000:fff75000       .debug$S                   0000000180000000     kernel32:KERNEL32.dll
 0000:fff75000       .debug$S                   0000000180000000     kernel32:KERNEL32.dll
 0000:fff75000       .debug$S                   0000000180000000     kernel32:KERNEL32.dll
 0000:fff75000       .debug$S                   0000000180000000     kernel32:KERNEL32.dll
 0000:fff75000       .debug$S                   0000000180000000     kernel32:KERNEL32.dll
 0000:fff75000       .debug$S                   0000000180000000     kernel32:KERNEL32.dll
 0000:fff75000       .debug$S                   0000000180000000     rpcrt4:RPCRT4.dll
 0000:fff75000       .debug$S                   0000000180000000     rpcrt4:RPCRT4.dll
 0000:fff75000       .debug$S                   0000000180000000     rpcrt4:RPCRT4.dll
 0000:fff75000       .debug$S                   0000000180000000     rpcrt4:RPCRT4.dll
 0000:fff75000       .debug$S                   0000000180000000     shell32:SHELL32.dll
 0000:fff75000       .debug$S                   0000000180000000     shell32:SHELL32.dll
 0000:fff75000       .debug$S                   0000000180000000     user32:USER32.dll
 0000:fff75000       .debug$S                   0000000180000000     lua51:lua51.dll
 0000:fff75000       .debug$S                   0000000180000000     lua51:lua51.dll
 0000:fff75000       .debug$S                   0000000180000000     lua51:lua51.dll
 0000:fff75000       .debug$S                   0000000180000000     lua51:lua51.dll
 0000:fff75000       .debug$S                   0000000180000000     lua51:lua51.dll
 0000:fff75000       .debug$S                   0000000180000000     lua51:lua51.dll
 0000:fff75000       .debug$S                   0000000180000000     lua51:lua51.dll
 0000:fff75000       .debug$S                   0000000180000000     lua51:lua51.dll
 0000:fff75000       .debug$S                   0000000180000000     lua51:lua51.dll
 0000:fff75000       .debug$S                   0000000180000000     lua51:lua51.dll
 0000:fff75000       .debug$S                   0000000180000000     lua51:lua51.dll
 0000:fff75000       .debug$S                   0000000180000000     lua51:lua51.dll
 0000:fff75000       .debug$S                   0000000180000000     lua51:lua51.dll
 0000:fff75000       .debug$S                   0000000180000000     lua51:lua51.dll
 0000:fff75000       .debug$S                   0000000180000000     lua51:lua51.dll
 0000:fff75000       .debug$S                   0000000180000000     lua51:lua51.dll
 0000:fff75000       .debug$S                   0000000180000000     lua51:lua51.dll
 0000:fff75000       .debug$S                   0000000180000000     lua51:lua51.dll
 0000:fff75000       .debug$S                   0000000180000000     lua51:lua51.dll
 0000:fff75000       .debug$S                   0000000180000000     lua51:lua51.dll
 0000:fff75000       .debug$S                   0000000180000000     lua51:lua51.dll
 0000:fff75000       .debug$S                   0000000180000000     lua51:lua51.dll
 0000:fff75000       .debug$S                   0000000180000000     lua51:lua51.dll
 0000:fff75000       .debug$S                   0000000180000000     lua51:lua51.dll
 0000:fff75000       .debug$S                   0000000180000000     lua51:lua51.dll
 0000:fff75000       .debug$S                   0000000180000000     lua51:lua51.dll
 0000:fff75000       .debug$S                   0000000180000000     lua51:lua51.dll
 0000:fff75000       .debug$S                   0000000180000000     lua51:lua51.dll
 0000:fff75000       .debug$S                   0000000180000000     lua51:lua51.dll
 0000:fff75000       .debug$S                   0000000180000000     lua51:lua51.dll
 0000:fff75000       .debug$S                   0000000180000000     lua51:lua51.dll
 0000:fff75000       .debug$S                   0000000180000000     lua51:lua51.dll
 0000:fff75000       .debug$S                   0000000180000000     lua51:lua51.dll
 0000:fff75000       .debug$S                   0000000180000000     lua51:lua51.dll
 0000:fff75000       .debug$S                   0000000180000000     lua51:lua51.dll
 0000:fff75000       .debug$S                   0000000180000000     lua51:lua51.dll
 0000:fff75000       .debug$S                   0000000180000000     lua51:lua51.dll
 0000:fff75000       .debug$S                   0000000180000000     lua51:lua51.dll
 0000:fff75000       .debug$S                   0000000180000000     lua51:lua51.dll
 0000:fff75000       .debug$S                   0000000180000000     lua51:lua51.dll
 0000:fff75000       .debug$S                   0000000180000000     lua51:lua51.dll
 0000:fff75000       .debug$S                   0000000180000000     lua51:lua51.dll
 0000:fff75000       .debug$S                   0000000180000000     lua51:lua51.dll
 0000:fff75000       .debug$S                   0000000180000000     lua51:lua51.dll
 0000:fff75000       .debug$S                   0000000180000000     lua51:lua51.dll
 0000:fff75000       .debug$S                   0000000180000000     lua51:lua51.dll
 0000:fff75000       .debug$S                   0000000180000000     lua51:lua51.dll
 0000:fff75000       .debug$S                   0000000180000000     lua51:lua51.dll
 0000:fff75000       .debug$S                   0000000180000000     lua51:lua51.dll
 0000:fff75000       .debug$S                   0000000180000000     lua51:lua51.dll
 0000:fff75000       .debug$S                   0000000180000000     lua51:lua51.dll
 0000:fff75000       .debug$S                   0000000180000000     lua51:lua51.dll
 0000:fff75000       .debug$S                   0000000180000000     lua51:lua51.dll
 0000:fff75000       .debug$S                   0000000180000000     lua51:lua51.dll
 0000:fff75000       .debug$S                   0000000180000000     lua51:lua51.dll
 0000:fff75000       .debug$S                   0000000180000000     lua51:lua51.dll
 0000:fff75000       .debug$S                   0000000180000000     lua51:lua51.dll
 0000:fff75000       .debug$S                   0000000180000000     lua51:lua51.dll
 0000:fff75000       .debug$S                   0000000180000000     lua51:lua51.dll
 0000:fff75000       .debug$S                   0000000180000000     lua51:lua51.dll
 0000:fff75000       .debug$S                   0000000180000000     lua51:lua51.dll
 0000:fff75000       .debug$S                   0000000180000000     lua51:lua51.dll
 0000:fff75000       .debug$S                   0000000180000000     lua51:lua51.dll
 0000:fff75000       .debug$S                   0000000180000000     lua51:lua51.dll
 0000:fff75000       .debug$S                   0000000180000000     lua51:lua51.dll
 0000:fff75000       .debug$S                   0000000180000000     lua51:lua51.dll
 0000:fff75000       .debug$S                   0000000180000000     lua51:lua51.dll
 0000:fff75000       .debug$S                   0000000180000000     lua51:lua51.dll
 0000:fff75000       .debug$S                   0000000180000000     lua51:lua51.dll
 0000:fff75000       .debug$S                   0000000180000000     lua51:lua51.dll
 0000:fff75000       .debug$S                   0000000180000000     lua51:lua51.dll
 0000:fff75000       .debug$S                   0000000180000000     lua51:lua51.dll
 0000:fff75000       .debug$S                   0000000180000000     lua51:lua51.dll
 0000:fff75000       .debug$S                   0000000180000000     lua51:lua51.dll
 0000:fff75000       .debug$S                   0000000180000000     lua51:lua51.dll
 0000:fff75000       .debug$S                   0000000180000000     lua51:lua51.dll
 0000:fff75000       .debug$S                   0000000180000000     lua51:lua51.dll
 0000:fff75000       .debug$S                   0000000180000000     lua51:lua51.dll
 0000:fff75000       .debug$S                   0000000180000000     lua51:lua51.dll
 0000:fff75000       .debug$S                   0000000180000000     lua51:lua51.dll
 0000:fff75000       .debug$S                   0000000180000000     lua51:lua51.dll
 0000:fff75000       .debug$S                   0000000180000000     lua51:lua51.dll
 0000:fff75000       .debug$S                   0000000180000000     lua51:lua51.dll
 0000:fff75000       .debug$S                   0000000180000000     lua51:lua51.dll
 0000:fff75000       .debug$S                   0000000180000000     lua51:lua51.dll
 0000:fff75000       .debug$S                   0000000180000000     lua51:lua51.dll
 0000:fff75000       .debug$S                   0000000180000000     lua51:lua51.dll
 0000:fff75000       .debug$S                   0000000180000000     lua51:lua51.dll
 0000:fff75000       .debug$S                   0000000180000000     lua51:lua51.dll
 0001:00000390       band                       0000000180001390 f   bit64.obj
 0001:00000460       bor                        0000000180001460 f   bit64.obj
 0001:00000530       bxor                       0000000180001530 f   bit64.obj
 0001:00000600       bnot                       0000000180001600 f   bit64.obj
 0001:00000630       lshift                     0000000180001630 f   bit64.obj
 0001:00000680       rshift                     0000000180001680 f   bit64.obj
 0001:000006d0       arshift                    00000001800016d0 f   bit64.obj
 0001:00000730       f_new                      0000000180001730 f   bit64.obj
 0001:000009a0       f_tostring                 00000001800019a0 f   bit64.obj
 0001:00000a00       f_type                     0000000180001a00 f   bit64.obj
 0001:00000aa0       f_add                      0000000180001aa0 f   bit64.obj
 0001:00000b70       f_sub                      0000000180001b70 f   bit64.obj
 0001:00000bc0       f_mul                      0000000180001bc0 f   bit64.obj
 0001:00000ca0       f_div                      0000000180001ca0 f   bit64.obj
 0001:00000d20       f_mod                      0000000180001d20 f   bit64.obj
 0001:00000d80       f_unm                      0000000180001d80 f   bit64.obj
 0001:00000db0       f_eq                       0000000180001db0 f   bit64.obj
 0001:00000e00       f_lt                       0000000180001e00 f   bit64.obj
 0001:00000e50       f_le                       0000000180001e50 f   bit64.obj
 0001:00000ea0       f_tonumber                 0000000180001ea0 f   bit64.obj
 0001:00002830       RegisterObject             0000000180003830 f   exported.obj
 0001:000028c0       PushAnalyseInfo            00000001800038c0 f   exported.obj
 0001:00003928       $LN22                      0000000180004928     exported.obj
 0001:000039e0       FillFarMacroCall_Callback  00000001800049e0 f   exported.obj
 0001:00003a50       FillFarMacroCall           0000000180004a50 f   exported.obj
 0001:00005800       $LN61                      0000000180006800     exported.obj
 0001:0000580c       $LN60                      000000018000680c     exported.obj
 0001:000065d0       getF                       00000001800075d0 f   lflua.obj
 0001:00006660       errfile                    0000000180007660 f   lflua.obj
 0001:00008b10       FL_PushParams              0000000180009b10 f   luamacro.obj
 0001:00008d84       $LN33                      0000000180009d84     luamacro.obj
 0001:00008db0       InitMPR                    0000000180009db0 f   luamacro.obj
 0001:000093e0       MacroCallFarCallback       000000018000a3e0 f   luamacro.obj
 0001:00009700       CheckFarUserControlIndex   000000018000a700 f   lusercontrol.obj
 0001:00009770       uc_tostring                000000018000a770 f   lusercontrol.obj
 0001:000097f0       uc_index                   000000018000a7f0 f   lusercontrol.obj
 0001:00009970       uc_newindex                000000018000a970 f   lusercontrol.obj
 0001:00009b60       uc_New                     000000018000ab60 f   lusercontrol.obj
 0001:00009dc0       OptHandle                  000000018000adc0 f   service.obj
 0001:00009e30       get_env_flag               000000018000ae30 f   service.obj
 0001:00009fb0       check_env_flag             000000018000afb0 f   service.obj
 0001:0000a3c0       CheckFlagsFromTable        000000018000b3c0 f   service.obj
 0001:0000a440       GetRealPluginData          000000018000b440 f   service.obj
 0001:0000a460       GetFakePluginData          000000018000b460 f   service.obj
 0001:0000a4b0       PluginHandle_rawhandle     000000018000b4b0 f   service.obj
 0001:0000a630       far_GetFileOwner           000000018000b630 f   service.obj
 0001:0000a8e0       far_GetNumberOfLinks       000000018000b8e0 f   service.obj
 0001:0000a9e0       far_GetLuafarVersion       000000018000b9e0 f   service.obj
 0001:0000ab70       FillEditorSetPosition      000000018000bb70 f   service.obj
 0001:0000b510       far_PluginStartupInfo      000000018000c510 f   service.obj
 0001:0000b6e0       far_GetCurrentDirectory    000000018000c6e0 f   service.obj
 0001:0000b810       push_ev_filename           000000018000c810 f   service.obj
 0001:0000b9a0       editor_GetFileName         000000018000c9a0 f   service.obj
 0001:0000b9f0       editor_GetInfo             000000018000c9f0 f   service.obj
 0001:0000be70       _EditorGetString           000000018000ce70 f   service.obj
 0001:0000c330       editor_GetString           000000018000d330 f   service.obj
 0001:0000c340       editor_GetStringW          000000018000d340 f   service.obj
 0001:0000c350       _EditorSetString           000000018000d350 f   service.obj
 0001:0000c620       editor_SetString           000000018000d620 f   service.obj
 0001:0000c630       editor_SetStringW          000000018000d630 f   service.obj
 0001:0000c640       editor_InsertString        000000018000d640 f   service.obj
 0001:0000c6c0       editor_DeleteString        000000018000d6c0 f   service.obj
 0001:0000c720       _EditorInsertText          000000018000d720 f   service.obj
 0001:0000c8f0       editor_InsertText          000000018000d8f0 f   service.obj
 0001:0000c900       editor_InsertTextW         000000018000d900 f   service.obj
 0001:0000c910       editor_DeleteChar          000000018000d910 f   service.obj
 0001:0000c970       editor_DeleteBlock         000000018000d970 f   service.obj
 0001:0000c9d0       editor_UndoRedo            000000018000d9d0 f   service.obj
 0001:0000ca80       FillKeyBarTitles           000000018000da80 f   service.obj
 0001:0000ccc0       SetKeyBar                  000000018000dcc0 f   service.obj
 0001:0000ce10       editor_SetKeyBar           000000018000de10 f   service.obj
 0001:0000ce20       viewer_SetKeyBar           000000018000de20 f   service.obj
 0001:0000ce30       editor_SetParam            000000018000de30 f   service.obj
 0001:0000d110       editor_SetPosition         000000018000e110 f   service.obj
 0001:0000d260       editor_Redraw              000000018000e260 f   service.obj
 0001:0000d2c0       editor_ExpandTabs          000000018000e2c0 f   service.obj
 0001:0000d340       PushBookmarks              000000018000e340 f   service.obj
 0001:0000d540       editor_GetBookmarks        000000018000e540 f   service.obj
 0001:0000d550       editor_GetSessionBookmarks 000000018000e550 f   service.obj
 0001:0000d560       editor_AddSessionBookmark  000000018000e560 f   service.obj
 0001:0000d5c0       editor_ClearSessionBookmarks 000000018000e5c0 f   service.obj
 0001:0000d620       editor_DeleteSessionBookmark 000000018000e620 f   service.obj
 0001:0000d6a0       editor_NextSessionBookmark 000000018000e6a0 f   service.obj
 0001:0000d700       editor_PrevSessionBookmark 000000018000e700 f   service.obj
 0001:0000d760       editor_SetTitle            000000018000e760 f   service.obj
 0001:0000d8a0       editor_GetTitle            000000018000e8a0 f   service.obj
 0001:0000da00       editor_Quit                000000018000ea00 f   service.obj
 0001:0000da60       FillEditorSelect           000000018000ea60 f   service.obj
 0001:0000dc10       editor_Select              000000018000ec10 f   service.obj
 0001:0000dd50       editor_GetSelection        000000018000ed50 f   service.obj
 0001:0000e160       _EditorTabConvert          000000018000f160 f   service.obj
 0001:0000e230       editor_TabToReal           000000018000f230 f   service.obj
 0001:0000e240       editor_RealToTab           000000018000f240 f   service.obj
 0001:0000e4f0       editor_AddColor            000000018000f4f0 f   service.obj
 0001:0000e730       editor_DelColor            000000018000f730 f   service.obj
 0001:0000e880       editor_GetColor            000000018000f880 f   service.obj
 0001:0000eb00       editor_SaveFile            000000018000fb00 f   service.obj
 0001:0000f0f0       editor_ReadInput           00000001800100f0 f   service.obj
 0001:0000f750       OptInputRecord             0000000180010750 f   service.obj
 0001:0000f800       editor_ProcessInput        0000000180010800 f   service.obj
 0001:0000f8b0       editor_SubscribeChangeEvent 00000001800108b0 f   service.obj
 0001:0000f970       far_Menu                   0000000180010970 f   service.obj
 0001:00010fd0       far_Message                0000000180011fd0 f   service.obj
 0001:000114d0       panel_CheckPanelsExist     00000001800124d0 f   service.obj
 0001:00011520       panel_ClosePanel           0000000180012520 f   service.obj
 0001:00011650       panel_GetPanelInfo         0000000180012650 f   service.obj
 0001:000119d0       get_panel_item             00000001800129d0 f   service.obj
 0001:00011ae0       panel_GetPanelItem         0000000180012ae0 f   service.obj
 0001:00011af0       panel_GetSelectedPanelItem 0000000180012af0 f   service.obj
 0001:00011b00       panel_GetCurrentPanelItem  0000000180012b00 f   service.obj
 0001:00011b10       get_string_info            0000000180012b10 f   service.obj
 0001:00011ca0       panel_GetPanelFormat       0000000180012ca0 f   service.obj
 0001:00011cb0       panel_GetPanelHostFile     0000000180012cb0 f   service.obj
 0001:00011cc0       panel_GetColumnTypes       0000000180012cc0 f   service.obj
 0001:00011cd0       panel_GetColumnWidths      0000000180012cd0 f   service.obj
 0001:00011ce0       panel_GetPanelPrefix       0000000180012ce0 f   service.obj
 0001:00011cf0       panel_RedrawPanel          0000000180012cf0 f   service.obj
 0001:00011e20       SetPanelBooleanProperty    0000000180012e20 f   service.obj
 0001:00011ee0       SetPanelIntegerProperty    0000000180012ee0 f   service.obj
 0001:00011fa0       panel_SetSortOrder         0000000180012fa0 f   service.obj
 0001:00011fb0       panel_SetDirectoriesFirst  0000000180012fb0 f   service.obj
 0001:00011fc0       panel_UpdatePanel          0000000180012fc0 f   service.obj
 0001:00011fd0       panel_SetSortMode          0000000180012fd0 f   service.obj
 0001:00011fe0       panel_SetViewMode          0000000180012fe0 f   service.obj
 0001:00011ff0       panel_GetPanelDirectory    0000000180012ff0 f   service.obj
 0001:00012390       panel_SetPanelDirectory    0000000180013390 f   service.obj
 0001:00012870       panel_GetCmdLine           0000000180013870 f   service.obj
 0001:000129b0       panel_SetCmdLine           00000001800139b0 f   service.obj
 0001:00012ad0       panel_GetCmdLinePos        0000000180013ad0 f   service.obj
 0001:00012b40       panel_SetCmdLinePos        0000000180013b40 f   service.obj
 0001:00012bb0       panel_InsertCmdLine        0000000180013bb0 f   service.obj
 0001:00012cd0       panel_GetCmdLineSelection  0000000180013cd0 f   service.obj
 0001:00012d90       panel_SetCmdLineSelection  0000000180013d90 f   service.obj
 0001:00012e60       ChangePanelSelection       0000000180013e60 f   service.obj
 0001:000130d0       panel_SetSelection         00000001800140d0 f   service.obj
 0001:000130e0       panel_ClearSelection       00000001800140e0 f   service.obj
 0001:000130f0       panel_BeginSelection       00000001800140f0 f   service.obj
 0001:00013180       panel_EndSelection         0000000180014180 f   service.obj
 0001:00013210       panel_SetUserScreen        0000000180014210 f   service.obj
 0001:00013280       panel_GetUserScreen        0000000180014280 f   service.obj
 0001:000132f0       panel_IsActivePanel        00000001800142f0 f   service.obj
 0001:00013340       panel_SetActivePanel       0000000180014340 f   service.obj
 0001:000133d0       far_GetDirList             00000001800143d0 f   service.obj
 0001:00013530       far_GetPluginDirList       0000000180014530 f   service.obj
 0001:000136b0       far_RestoreScreen          00000001800146b0 f   service.obj
 0001:00013730       far_FreeScreen             0000000180014730 f   service.obj
 0001:00013790       far_SaveScreen             0000000180014790 f   service.obj
 0001:00013b80       PushList                   0000000180014b80 f   service.obj
 0001:00013dd0       SetFarDialogItem           0000000180014dd0 f   service.obj
 0001:00014470       PushDlgItem                0000000180015470 f   service.obj
 0001:00014930       PushDlgItemNum             0000000180015930 f   service.obj
 0001:00014a10       SetDlgItem                 0000000180015a10 f   service.obj
 0001:00014c00       far_SendDlgMessage         0000000180015c00 f   service.obj
 0001:000164bc       $LN309                     00000001800174bc     service.obj
 0001:000164c8       $LN308                     00000001800174c8     service.obj
 0001:0001650c       $LN307                     000000018001750c     service.obj
 0001:00016594       $LN306                     0000000180017594     service.obj
 0001:0001693c       $LN72                      000000018001793c     service.obj
 0001:0001694c       $LN71                      000000018001794c     service.obj
 0001:00016964       $LN70                      0000000180017964     service.obj
 0001:00016c54       $LN31                      0000000180017c54     service.obj
 0001:00016c6c       $LN30                      0000000180017c6c     service.obj
 0001:00016e90       far_DialogInit             0000000180017e90 f   service.obj
 0001:000173b0       free_dialog                00000001800183b0 f   service.obj
 0001:00017420       far_DialogRun              0000000180018420 f   service.obj
 0001:000174c0       far_DialogFree             00000001800184c0 f   service.obj
 0001:00017540       dialog_tostring            0000000180018540 f   service.obj
 0001:000175a0       dialog_rawhandle           00000001800185a0 f   service.obj
 0001:000175f0       far_GetDlgItem             00000001800185f0 f   service.obj
 0001:00017690       far_SetDlgItem             0000000180018690 f   service.obj
 0001:00017730       far_SubscribeDialogDrawEvents 0000000180018730 f   service.obj
 0001:00017750       editor_Editor              0000000180018750 f   service.obj
 0001:00017a70       viewer_Viewer              0000000180018a70 f   service.obj
 0001:00017d60       viewer_GetFileName         0000000180018d60 f   service.obj
 0001:00017da0       viewer_GetInfo             0000000180018da0 f   service.obj
 0001:00018090       viewer_Quit                0000000180019090 f   service.obj
 0001:000180e0       viewer_Redraw              00000001800190e0 f   service.obj
 0001:00018130       viewer_Select              0000000180019130 f   service.obj
 0001:00018200       viewer_SetPosition         0000000180019200 f   service.obj
 0001:000184a0       viewer_SetMode             00000001800194a0 f   service.obj
 0001:000185c0       far_ShowHelp               00000001800195c0 f   service.obj
 0001:00018830       far_InputBox               0000000180019830 f   service.obj
 0001:00018e40       far_GetMsg                 0000000180019e40 f   service.obj
 0001:00019010       far_Text                   000000018001a010 f   service.obj
 0001:000191b0       far_CopyToClipboard        000000018001a1b0 f   service.obj
 0001:00019340       far_PasteFromClipboard     000000018001a340 f   service.obj
 0001:00019440       far_InputRecordToName      000000018001a440 f   service.obj
 0001:00019760       far_NameToInputRecord      000000018001a760 f   service.obj
 0001:000198a0       far_LStricmp               000000018001a8a0 f   service.obj
 0001:00019a50       far_LStrnicmp              000000018001aa50 f   service.obj
 0001:00019c20       far_ProcessName            000000018001ac20 f   service.obj
 0001:0001a070       far_GetReparsePointInfo    000000018001b070 f   service.obj
 0001:0001a250       far_LIsAlpha               000000018001b250 f   service.obj
 0001:0001a350       far_LIsAlphanum            000000018001b350 f   service.obj
 0001:0001a450       far_LIsLower               000000018001b450 f   service.obj
 0001:0001a550       far_LIsUpper               000000018001b550 f   service.obj
 0001:0001a650       convert_buf                000000018001b650 f   service.obj
 0001:0001a770       far_LLowerBuf              000000018001b770 f   service.obj
 0001:0001a780       far_LUpperBuf              000000018001b780 f   service.obj
 0001:0001a790       far_MkTemp                 000000018001b790 f   service.obj
 0001:0001a980       far_MkLink                 000000018001b980 f   service.obj
 0001:0001abd0       far_GetPathRoot            000000018001bbd0 f   service.obj
 0001:0001ada0       truncstring                000000018001bda0 f   service.obj
 0001:0001afe0       far_TruncPathStr           000000018001bfe0 f   service.obj
 0001:0001aff0       far_TruncStr               000000018001bff0 f   service.obj
 0001:0001b000       FrsUserFunc                000000018001c000 f   service.obj
 0001:0001b1d0       far_RecursiveSearch        000000018001c1d0 f   service.obj
 0001:0001b540       far_ConvertPath            000000018001c540 f   service.obj
 0001:0001b750       far_AdvControl             000000018001c750 f   service.obj
 0001:0001c1a8       $LN101                     000000018001d1a8     service.obj
 0001:0001c220       far_MacroLoadAll           000000018001d220 f   service.obj
 0001:0001c3d0       far_MacroSaveAll           000000018001d3d0 f   service.obj
 0001:0001c420       far_MacroGetState          000000018001d420 f   service.obj
 0001:0001c460       far_MacroGetArea           000000018001d460 f   service.obj
 0001:0001c4a0       MacroSendString            000000018001d4a0 f   service.obj
 0001:0001c780       far_MacroPost              000000018001d780 f   service.obj
 0001:0001c790       far_MacroCheck             000000018001d790 f   service.obj
 0001:0001c7a0       far_MacroGetLastError      000000018001d7a0 f   service.obj
 0001:0001ca70       far_MacroAdd               000000018001da70 f   service.obj
 0001:0001cf80       far_MacroDelete            000000018001df80 f   service.obj
 0001:0001d040       AddMacroData_gc            000000018001e040 f   service.obj
 0001:0001d100       far_MacroExecute           000000018001e100 f   service.obj
 0001:0001d330       far_CPluginStartupInfo     000000018001e330 f   service.obj
 0001:0001d400       far_MakeMenuItems          000000018001e400 f   service.obj
 0001:0001d7b0       far_Show                   000000018001e7b0 f   service.obj
 0001:0001d870       far_CreateFileFilter       000000018001e870 f   service.obj
 0001:0001d930       filefilter_Free            000000018001e930 f   service.obj
 0001:0001d9c0       filefilter_gc              000000018001e9c0 f   service.obj
 0001:0001da50       filefilter_tostring        000000018001ea50 f   service.obj
 0001:0001dab0       filefilter_OpenMenu        000000018001eab0 f   service.obj
 0001:0001db30       filefilter_Starting        000000018001eb30 f   service.obj
 0001:0001dbb0       filefilter_IsFileInFilter  000000018001ebb0 f   service.obj
 0001:0001dca0       plugin_load                000000018001eca0 f   service.obj
 0001:0001de10       far_LoadPlugin             000000018001ee10 f   service.obj
 0001:0001de20       far_ForcedLoadPlugin       000000018001ee20 f   service.obj
 0001:0001de30       far_UnloadPlugin           000000018001ee30 f   service.obj
 0001:0001de90       far_FindPlugin             000000018001ee90 f   service.obj
 0001:0001e030       PutPluginMenuItemToTable   000000018001f030 f   service.obj
 0001:0001e230       PutVersionInfoToTable      000000018001f230 f   service.obj
 0001:0001e370       far_GetPluginInformation   000000018001f370 f   service.obj
 0001:0001e9d0       far_GetPlugins             000000018001f9d0 f   service.obj
 0001:0001eaf0       far_IsPluginLoaded         000000018001faf0 f   service.obj
 0001:0001ec20       far_XLat                   000000018001fc20 f   service.obj
 0001:0001ee90       far_FormatFileSize         000000018001fe90 f   service.obj
 0001:0001f080       far_FarClock               0000000180020080 f   service.obj
 0001:0001f130       far_Timer                  0000000180020130 f   service.obj
 0001:0001f330       timer_Close                0000000180020330 f   service.obj
 0001:0001f3f0       timer_gc                   00000001800203f0 f   service.obj
 0001:0001f490       timer_tostring             0000000180020490 f   service.obj
 0001:0001f4f0       timer_index                00000001800204f0 f   service.obj
 0001:0001f660       timer_newindex             0000000180020660 f   service.obj
 0001:0001f810       far_CreateSettings         0000000180020810 f   service.obj
 0001:0001fa00       Settings_set               0000000180020a00 f   service.obj
 0001:0001fce0       Settings_get               0000000180020ce0 f   service.obj
 0001:0001ff70       Settings_delete            0000000180020f70 f   service.obj
 0001:00020120       Settings_createsubkey      0000000180021120 f   service.obj
 0001:000203d0       Settings_opensubkey        00000001800213d0 f   service.obj
 0001:00020570       Settings_enum              0000000180021570 f   service.obj
 0001:00020ba0       Settings_free              0000000180021ba0 f   service.obj
 0001:00020c40       far_FreeSettings           0000000180021c40 f   service.obj
 0001:00020cf0       Settings_tostring          0000000180021cf0 f   service.obj
 0001:00020d50       far_ColorDialog            0000000180021d50 f   service.obj
 0001:00020f10       far_RunDefaultScript       0000000180021f10 f   service.obj
 0001:00020f40       far_FileTimeResolution     0000000180021f40 f   service.obj
 0001:00020fc0       GetPluginModuleHandle      0000000180021fc0 f   service.obj
 0001:00021090       far_host_GetFiles          0000000180022090 f   service.obj
 0001:000213a0       far_host_PutFiles          00000001800223a0 f   service.obj
 0001:000216b0       far_host_GetFindData       00000001800226b0 f   service.obj
 0001:00021850       far_host_FreeUserData      0000000180022850 f   service.obj
 0001:000219b0       far_host_SetDirectory      00000001800229b0 f   service.obj
 0001:00021be0       luaopen_far                0000000180022be0 f   service.obj
 0001:00022560       CustomAllocator            0000000180023560 f   service.obj
 0001:00022ac0       str_rep                    0000000180023ac0 f   slnunico.obj
 0001:00022b70       writer                     0000000180023b70 f   slnunico.obj
 0001:00022b90       str_dump                   0000000180023b90 f   slnunico.obj
 0001:00022c30       str_format                 0000000180023c30 f   slnunico.obj
 0001:000233cc       $LN115                     00000001800243cc     slnunico.obj
 0001:000233e8       $LN114                     00000001800243e8     slnunico.obj
 0001:00023420       utf8_valid                 0000000180024420 f   slnunico.obj
 0001:00023540       utf8_offset                0000000180024540 f   lutf8lib.obj
 0001:000235e0       utf8_range                 00000001800245e0 f   lutf8lib.obj
 0001:000236e0       utf8_isdigit               00000001800246e0 f   lutf8lib.obj
 0001:00023760       utf8_islower               0000000180024760 f   lutf8lib.obj
 0001:000237e0       utf8_iscompose             00000001800247e0 f   lutf8lib.obj
 0001:00023860       utf8_isgraph               0000000180024860 f   lutf8lib.obj
 0001:00023980       utf8_width                 0000000180024980 f   lutf8lib.obj
 0001:00023b30       utf8_safe_decode           0000000180024b30 f   lutf8lib.obj
 0001:00023c00       Lutf8_len                  0000000180024c00 f   lutf8lib.obj
 0001:00023e50       Lutf8_sub                  0000000180024e50 f   lutf8lib.obj
 0001:00023ef0       Lutf8_reverse              0000000180024ef0 f   lutf8lib.obj
 0001:00024140       Lutf8_byte                 0000000180025140 f   lutf8lib.obj
 0001:000242c0       Lutf8_codepoint            00000001800252c0 f   lutf8lib.obj
 0001:00024500       Lutf8_char                 0000000180025500 f   lutf8lib.obj
 0001:00024640       Lutf8_lower                0000000180025640 f   lutf8lib.obj
 0001:00024980       Lutf8_upper                0000000180025980 f   lutf8lib.obj
 0001:00024cc0       Lutf8_title                0000000180025cc0 f   lutf8lib.obj
 0001:00025000       Lutf8_fold                 0000000180026000 f   lutf8lib.obj
 0001:00025340       Lutf8_escape               0000000180026340 f   lutf8lib.obj
 0001:000256b8       $LN113                     00000001800266b8     lutf8lib.obj
 0001:000256c8       $LN112                     00000001800266c8     lutf8lib.obj
 0001:00025720       Lutf8_insert               0000000180026720 f   lutf8lib.obj
 0001:00025860       Lutf8_remove               0000000180026860 f   lutf8lib.obj
 0001:00025970       push_offset                0000000180026970 f   lutf8lib.obj
 0001:00025ad0       Lutf8_charpos              0000000180026ad0 f   lutf8lib.obj
 0001:00025bd0       Lutf8_offset               0000000180026bd0 f   lutf8lib.obj
 0001:00025d50       Lutf8_next                 0000000180026d50 f   lutf8lib.obj
 0001:00025e10       iter_aux                   0000000180026e10 f   lutf8lib.obj
 0001:00025fa0       iter_auxstrict             0000000180026fa0 f   lutf8lib.obj
 0001:00025fb0       iter_auxlax                0000000180026fb0 f   lutf8lib.obj
 0001:00025fc0       Lutf8_codes                0000000180026fc0 f   lutf8lib.obj
 0001:00026040       Lutf8_width                0000000180027040 f   lutf8lib.obj
 0001:00026220       Lutf8_widthindex           0000000180027220 f   lutf8lib.obj
 0001:000263e0       Lutf8_ncasecmp             00000001800273e0 f   lutf8lib.obj
 0001:000266b0       classend                   00000001800276b0 f   lutf8lib.obj
 0001:00026830       match_class                0000000180027830 f   lutf8lib.obj
 0001:00026ca8       $LN152                     0000000180027ca8     lutf8lib.obj
 0001:00026d10       matchbracketclass          0000000180027d10 f   lutf8lib.obj
 0001:00027070       singlematch                0000000180028070 f   lutf8lib.obj
 0001:00027260       matchbalance               0000000180028260 f   lutf8lib.obj
 0001:00027570       start_capture              0000000180028570 f   lutf8lib.obj
 0001:00027600       match                      0000000180028600 f   lutf8lib.obj
 0001:00027d90       $LN261                     0000000180028d90     lutf8lib.obj
 0001:00027da0       $LN260                     0000000180028da0     lutf8lib.obj
 0001:00027de0       push_onecapture            0000000180028de0 f   lutf8lib.obj
 0001:00027f10       push_captures              0000000180028f10 f   lutf8lib.obj
 0001:00028080       find_aux                   0000000180029080 f   lutf8lib.obj
 0001:00028510       Lutf8_find                 0000000180029510 f   lutf8lib.obj
 0001:00028520       Lutf8_match                0000000180029520 f   lutf8lib.obj
 0001:00028530       gmatch_aux                 0000000180029530 f   lutf8lib.obj
 0001:00028690       Lutf8_gmatch               0000000180029690 f   lutf8lib.obj
 0001:000286f0       add_s                      00000001800296f0 f   lutf8lib.obj
 0001:00028a50       Lutf8_gsub                 0000000180029a50 f   lutf8lib.obj
 0001:00029220       pushresult                 000000018002a220 f   uliolib51.obj
 0001:00029390       fileerror                  000000018002a390 f   uliolib51.obj
 0001:000294d0       io_type                    000000018002a4d0 f   uliolib51.obj
 0001:000295b0       newfile                    000000018002a5b0 f   uliolib51.obj
 0001:00029610       io_noclose                 000000018002a610 f   uliolib51.obj
 0001:00029640       io_pclose                  000000018002a640 f   uliolib51.obj
 0001:000296f0       io_fclose                  000000018002a6f0 f   uliolib51.obj
 0001:000297a0       aux_close                  000000018002a7a0 f   uliolib51.obj
 0001:000297f0       io_close                   000000018002a7f0 f   uliolib51.obj
 0001:00029890       io_gc                      000000018002a890 f   uliolib51.obj
 0001:000298f0       io_tostring                000000018002a8f0 f   uliolib51.obj
 0001:00029950       io_open                    000000018002a950 f   uliolib51.obj
 0001:00029c70       io_popen                   000000018002ac70 f   uliolib51.obj
 0001:00029e90       io_tmpfile                 000000018002ae90 f   uliolib51.obj
 0001:00029f40       g_iofile                   000000018002af40 f   uliolib51.obj
 0001:0002a100       io_input                   000000018002b100 f   uliolib51.obj
 0001:0002a120       io_output                  000000018002b120 f   uliolib51.obj
 0001:0002a140       f_lines                    000000018002b140 f   uliolib51.obj
 0001:0002a1b0       io_lines                   000000018002b1b0 f   uliolib51.obj
 0001:0002a3c0       read_line                  000000018002b3c0 f   uliolib51.obj
 0001:0002a4d0       read_chars                 000000018002b4d0 f   uliolib51.obj
 0001:0002a5a0       g_read                     000000018002b5a0 f   uliolib51.obj
 0001:0002a8d0       io_read                    000000018002b8d0 f   uliolib51.obj
 0001:0002a940       f_read                     000000018002b940 f   uliolib51.obj
 0001:0002a9a0       io_readline                000000018002b9a0 f   uliolib51.obj
 0001:0002aa80       g_write                    000000018002ba80 f   uliolib51.obj
 0001:0002ab90       io_write                   000000018002bb90 f   uliolib51.obj
 0001:0002ac00       f_write                    000000018002bc00 f   uliolib51.obj
 0001:0002ac60       f_seek                     000000018002bc60 f   uliolib51.obj
 0001:0002ad90       f_setvbuf                  000000018002bd90 f   uliolib51.obj
 0001:0002ae90       io_flush                   000000018002be90 f   uliolib51.obj
 0001:0002af60       f_flush                    000000018002bf60 f   uliolib51.obj
 0001:0002b020       f_rawhandle                000000018002c020 f   uliolib51.obj
 0001:0002b360       gctm                       000000018002c360 f   uloadlib51.obj
 0001:0002b3b0       ll_loadfunc                000000018002c3b0 f   uloadlib51.obj
 0001:0002b5e0       ll_loadlib                 000000018002c5e0 f   uloadlib51.obj
 0001:0002b720       findfile                   000000018002c720 f   uloadlib51.obj
 0001:0002bc40       loaderror                  000000018002cc40 f   uloadlib51.obj
 0001:0002bd70       loader_Lua                 000000018002cd70 f   uloadlib51.obj
 0001:0002bdd0       mkfuncname                 000000018002cdd0 f   uloadlib51.obj
 0001:0002be50       loader_C                   000000018002ce50 f   uloadlib51.obj
 0001:0002bed0       loader_Croot               000000018002ced0 f   uloadlib51.obj
 0001:0002bfb0       loader_preload             000000018002cfb0 f   uloadlib51.obj
 0001:0002c050       ll_require                 000000018002d050 f   uloadlib51.obj
 0001:0002c2c0       ll_module                  000000018002d2c0 f   uloadlib51.obj
 0001:0002c550       ll_seeall                  000000018002d550 f   uloadlib51.obj
 0001:0002c5d0       setpath                    000000018002d5d0 f   uloadlib51.obj
 0001:0002e548       $LN27                      000000018002f548     ustring.obj
 0001:0002f690       ustring_OutputDebugString  0000000180030690 f   ustring.obj
 0001:0002f820       ustring_system             0000000180030820 f   ustring.obj
 0001:00030070       win_GetEnv                 0000000180031070 f   win.obj
 0001:00030320       win_SetEnv                 0000000180031320 f   win.obj
 0001:000304d0       CheckHKey                  00000001800314d0 f   win.obj
 0001:00030600       win_SetRegKey              0000000180031600 f   win.obj
 0001:00030ce0       win_GetRegKey              0000000180031ce0 f   win.obj
 0001:000311e0       win_DeleteRegKey           00000001800321e0 f   win.obj
 0001:00031370       win_DeleteRegValue         0000000180032370 f   win.obj
 0001:00031610       win_EnumRegKey             0000000180032610 f   win.obj
 0001:000318c0       win_EnumRegValue           00000001800328c0 f   win.obj
 0001:00031b70       win_ExtractKey             0000000180032b70 f   win.obj
 0001:00031c40       win_ExtractKeyEx           0000000180032c40 f   win.obj
 0001:00031ce0       PushWinFindData            0000000180032ce0 f   win.obj
 0001:00031f60       win_GetFileInfo            0000000180032f60 f   win.obj
 0001:000320b0       win_GetSystemTimeAsFileTime 00000001800330b0 f   win.obj
 0001:00032170       win_FileTimeToSystemTime   0000000180033170 f   win.obj
 0001:00032380       win_SystemTimeToFileTime   0000000180033380 f   win.obj
 0001:00032710       win_FileTimeToLocalFileTime 0000000180033710 f   win.obj
 0001:00032830       win_CompareString          0000000180033830 f   win.obj
 0001:00032af0       win_wcscmp                 0000000180033af0 f   win.obj
 0001:00032cb0       win_GetVirtualKeys         0000000180033cb0 f   win.obj
 0001:00032d70       win_GetConsoleScreenBufferInfo 0000000180033d70 f   win.obj
 0001:00032ff0       win_CopyFile               0000000180033ff0 f   win.obj
 0001:000331e0       win_MoveFile               00000001800341e0 f   win.obj
 0001:00033420       win_DeleteFile             0000000180034420 f   win.obj
 0001:00033540       mkdir                      0000000180034540 f   win.obj
 0001:00033750       win_CreateDir              0000000180034750 f   win.obj
 0001:00033960       win_RemoveDir              0000000180034960 f   win.obj
 0001:00033a80       win_ShellExecute           0000000180034a80 f   win.obj
 0001:00033e40       win_IsProcess64bit         0000000180034e40 f   win.obj
 0001:00034900       win_GetFileTimes           0000000180035900 f   win.obj
 0001:00034b90       ExtractFileTime            0000000180035b90 f   win.obj
 0001:00034c60       win_SetFileTimes           0000000180035c60 f   win.obj
 0001:00034f10       $$000000                   0000000180035f10     LIBCMT:amdsecgs.obj
 0001:000350f8       capture_current_context    00000001800360f8 f   LIBCMT:gs_report.obj
 0001:00035168       capture_previous_context   0000000180036168 f   LIBCMT:gs_report.obj
 0001:000351dc       ?dllmain_crt_dispatch@@YAHQEAUHINSTANCE__@@KQEAX@Z 00000001800361dc f   LIBCMT:dll_dllmain.obj
 0001:0003522c       ?dllmain_crt_process_attach@@YAHQEAUHINSTANCE__@@QEAX@Z 000000018003622c f   LIBCMT:dll_dllmain.obj
 0001:00035344       ?dllmain_crt_process_detach@@YAH_N@Z 0000000180036344 f   LIBCMT:dll_dllmain.obj
 0001:000353c8       ?dllmain_dispatch@@YAHQEAUHINSTANCE__@@KQEAX@Z 00000001800363c8 f   LIBCMT:dll_dllmain.obj
 0001:00036500       $$000000                   0000000180037500     libvcruntime:memset.obj
 0001:000366c0       $$000000                   00000001800376c0     libvcruntime:notify.obj
 0001:00036960       $$000000                   0000000180037960     libvcruntime:memcpy.obj
 0001:00037008       ?try_get_function@@YAPEAXW4function_id@?A0x3064ecbf@@QEBDQEBW4module_id@2@2@Z 0000000180038008 f   libvcruntime:winapi_downlevel.obj
 0001:000372f0       $$000000                   00000001800382f0     libvcruntime:handlers.obj
 0001:000373f8       ??$?RV<lambda_fe5404e9642edbb7c8ae71e1dcfa4018>@@AEAV<lambda_36eeb330e99a4f0bf8a7da86d0894cb9>@@V<lambda_2fa474834de80dc12f7a3c6eddd7a366>@@@?$__crt_seh_guarded_call@H@@QEAAH$$QEAV<lambda_fe5404e9642edbb7c8ae71e1dcfa4018>@@AEAV<lambda_36eeb330e99a4f0bf8a7da86d0894cb9>@@$$QEAV<lambda_2fa474834de80dc12f7a3c6eddd7a366>@@@Z 00000001800383f8 f   libucrt:output.obj
 0001:00037438       ??$common_vsprintf@Vstandard_base@__crt_stdio_output@@D@@YAH_KQEAD0QEBDQEAU__crt_locale_pointers@@1@Z 0000000180038438 f   libucrt:output.obj
 0001:00037604       ??$common_vsprintf@Vstandard_base@__crt_stdio_output@@_W@@YAH_KQEA_W0QEB_WQEAU__crt_locale_pointers@@QEAD@Z 0000000180038604 f   libucrt:output.obj
 0001:00037de8       ??R<lambda_36eeb330e99a4f0bf8a7da86d0894cb9>@@QEBAHXZ 0000000180038de8 f   libucrt:output.obj
 0001:0003aa94       common_control87           000000018003ba94 f   libucrt:ieee.obj
 0001:0003ad54       ??$common_fsopen@_W@@YAPEAU_iobuf@@QEB_W0H@Z 000000018003bd54 f   libucrt:fopen.obj
 0001:0003b1a4       ??$common_freopen@_W@@YAHQEAPEAU_iobuf@@QEB_W1V__crt_stdio_stream@@H@Z 000000018003c1a4 f   libucrt:freopen.obj
 0001:0003bc60       $$000000                   000000018003cc60     libucrt:strncmp.obj
 0001:0003be40       $$000000                   000000018003ce40     libucrt:strncpy.obj
 0001:0003bfb4       fallbackMethod             000000018003cfb4 f   libucrt:strpbrk.obj
 0001:0003c384       $LN78                      000000018003d384     libucrt:strpbrk.obj
 0001:0003c3c0       $LN77                      000000018003d3c0     libucrt:strpbrk.obj
 0001:0003c400       $LN76                      000000018003d400     libucrt:strpbrk.obj
 0001:0003c440       ??$common_popen@_W@@YAPEAU_iobuf@@QEB_W0@Z 000000018003d440 f   libucrt:popen.obj
 0001:0003c60c       ??$common_popen_nolock@_W@@YAPEAU_iobuf@@QEB_W0HAEAY01H@Z 000000018003d60c f   libucrt:popen.obj
 0001:0003c92c       ??$get_executable_path@_W@@YAPEB_WQEB_W@Z 000000018003d92c f   libucrt:popen.obj
 0001:0003cac4       ?idtab@@YAPEAUprocess_handle_pair@?A0xe43b7539@@QEAU_iobuf@@@Z 000000018003dac4 f   libucrt:popen.obj
 0001:0003cc2c       ??$?RV<lambda_842d9ff0dc9ef11c61343bbaebe7f885>@@AEAV<lambda_c5860995281e5c4ce005b3de8f5874ee>@@V<lambda_d90129c13df834fdcbf8d2b88dafcf2d>@@@?$__crt_seh_guarded_call@X@@QEAAX$$QEAV<lambda_842d9ff0dc9ef11c61343bbaebe7f885>@@AEAV<lambda_c5860995281e5c4ce005b3de8f5874ee>@@$$QEAV<lambda_d90129c13df834fdcbf8d2b88dafcf2d>@@@Z 000000018003dc2c f   libucrt:fflush.obj
 0001:0003ccc8       ??$?RV<lambda_886d6c58226a84441f68b9f2b8217b83>@@AEAV<lambda_ab61a845afdef5b7c387490eaf3616ee>@@V<lambda_f7f22ab5edc0698d5f6905b0d3f44752>@@@?$__crt_seh_guarded_call@X@@QEAAX$$QEAV<lambda_886d6c58226a84441f68b9f2b8217b83>@@AEAV<lambda_ab61a845afdef5b7c387490eaf3616ee>@@$$QEAV<lambda_f7f22ab5edc0698d5f6905b0d3f44752>@@@Z 000000018003dcc8 f   libucrt:fflush.obj
 0001:0003cda8       ??$?RV<lambda_c376a267cfb53b6959b3b692ec76b120>@@AEAV<lambda_9a32fed5bf61b6b509b2d3f6003082a1>@@V<lambda_572fbb9fa0ab338edf41edfd4b5fcc8d>@@@?$__crt_seh_guarded_call@H@@QEAAH$$QEAV<lambda_c376a267cfb53b6959b3b692ec76b120>@@AEAV<lambda_9a32fed5bf61b6b509b2d3f6003082a1>@@$$QEAV<lambda_572fbb9fa0ab338edf41edfd4b5fcc8d>@@@Z 000000018003dda8 f   libucrt:fflush.obj
 0001:0003cde8       ?common_flush_all@@YAH_N@Z 000000018003dde8 f   libucrt:fflush.obj
 0001:0003d030       ??$common_fgets@D@@YAPEADQEADHV__crt_stdio_stream@@@Z 000000018003e030 f   libucrt:fgets.obj
 0001:0003d104       ??$generate_tmpfile_file_name@D@@YA_NQEAD_K@Z 000000018003e104 f   libucrt:tmpfile.obj
 0001:0003d1a0       ??$get_tmpfile_buffer_nolock@D@@YAPEADW4buffer_id@?A0x5b9a7937@@@Z 000000018003e1a0 f   libucrt:tmpfile.obj
 0001:0003d1e4       ??$initialize_tmpfile_buffer_nolock@D@@YA_NW4buffer_id@?A0x5b9a7937@@@Z 000000018003e1e4 f   libucrt:tmpfile.obj
 0001:0003d2d0       ?common_tmpfile@@YAHQEAPEAU_iobuf@@H@Z 000000018003e2d0 f   libucrt:tmpfile.obj
 0001:0003d334       ?common_tmpfile_nolock@@YAHQEAPEAU_iobuf@@H@Z 000000018003e334 f   libucrt:tmpfile.obj
 0001:0003d560       ??$?RV<lambda_2831f20263db5b546e098b45503eb778>@@AEAV<lambda_5856287d7ecd2be6c9197bb4007c3f6e>@@V<lambda_0838d7e100fbcbd261b69cfea6abb102>@@@?$__crt_seh_guarded_call@_K@@QEAA_K$$QEAV<lambda_2831f20263db5b546e098b45503eb778>@@AEAV<lambda_5856287d7ecd2be6c9197bb4007c3f6e>@@$$QEAV<lambda_0838d7e100fbcbd261b69cfea6abb102>@@@Z 000000018003e560 f   libucrt:fwrite.obj
 0001:0003d5a0       ??R<lambda_5856287d7ecd2be6c9197bb4007c3f6e>@@QEBA_KXZ 000000018003e5a0 f   libucrt:fwrite.obj
 0001:0003d834       ??$?RV<lambda_84ec643ea9557e2f7dc01bb0e9624395>@@AEAV<lambda_ca71763b3c0644891230e4f79ea54fa6>@@V<lambda_439a761618c59b0600e24586724d733b>@@@?$__crt_seh_guarded_call@H@@QEAAH$$QEAV<lambda_84ec643ea9557e2f7dc01bb0e9624395>@@AEAV<lambda_ca71763b3c0644891230e4f79ea54fa6>@@$$QEAV<lambda_439a761618c59b0600e24586724d733b>@@@Z 000000018003e834 f   libucrt:setvbuf.obj
 0001:0003d874       ??R<lambda_ca71763b3c0644891230e4f79ea54fa6>@@QEBAHXZ 000000018003e874 f   libucrt:setvbuf.obj
 0001:0003d9f0       ??$?RV<lambda_082dd7c0feb7dbdaf245f261e54a6583>@@AEAV<lambda_f3caf1ecae5fe01a9a1a6239afa44510>@@V<lambda_c640b76c0755ae85b317b35c67c61e6b>@@@?$__crt_seh_guarded_call@H@@QEAAH$$QEAV<lambda_082dd7c0feb7dbdaf245f261e54a6583>@@AEAV<lambda_f3caf1ecae5fe01a9a1a6239afa44510>@@$$QEAV<lambda_c640b76c0755ae85b317b35c67c61e6b>@@@Z 000000018003e9f0 f   libucrt:input.obj
 0001:0003f710       ??R<lambda_156378f40168adef48d7ddfcff3a1264>@@QEBA_NXZ 0000000180040710 f   libucrt:input.obj
 0001:0003f78c       ??R<lambda_f3caf1ecae5fe01a9a1a6239afa44510>@@QEBAHXZ 000000018004078c f   libucrt:input.obj
 0001:00042e30       memcpy_s                   0000000180043e30 f   libucrt:cfout.obj
 0001:00042e30       memcpy_s                   0000000180043e30 f   libucrt:input.obj
 0001:00042eb8       ??$common_ftell@_J@@YA_JV__crt_stdio_stream@@@Z 0000000180043eb8 f   libucrt:ftell.obj
 0001:00042f0c       ??$common_ftell_nolock@_J@@YA_JV__crt_stdio_stream@@@Z 0000000180043f0c f   libucrt:ftell.obj
 0001:0004303c       ?common_ftell_read_mode_nolock@@YA_JV__crt_stdio_stream@@_J1@Z 000000018004403c f   libucrt:ftell.obj
 0001:00043188       ?common_ftell_translated_utf8_nolock@@YA_JV__crt_stdio_stream@@_J@Z 0000000180044188 f   libucrt:ftell.obj
 0001:00043304       ?count_newline_bytes@@YA_JQEBD0W4__crt_lowio_text_mode@@@Z 0000000180044304 f   libucrt:ftell.obj
 0001:00043398       ?common_fseek@@YAHV__crt_stdio_stream@@_JH@Z 0000000180044398 f   libucrt:fseek.obj
 0001:00043404       ?common_fseek_binary_mode_read_only_fast_track_nolock@@YA_NV__crt_stdio_stream@@_JH@Z 0000000180044404 f   libucrt:fseek.obj
 0001:000434e8       ?common_fseek_nolock@@YAHV__crt_stdio_stream@@_JH@Z 00000001800444e8 f   libucrt:fseek.obj
 0001:000435a8       ??$common_dupenv_s@_W@@YAHQEAPEA_WQEA_KQEB_WHQEBDH@Z 00000001800445a8 f   libucrt:getenv.obj
 0001:0004369c       ??$common_getenv@_W@@YAPEA_WQEB_W@Z 000000018004469c f   libucrt:getenv.obj
 0001:000436fc       ??$common_getenv_nolock@_W@@YAPEA_WQEB_W@Z 00000001800446fc f   libucrt:getenv.obj
 0001:00043b68       ??$?RV<lambda_d80eeec6fff315bfe5c115232f3240e3>@@AEAV<lambda_6e4b09c48022b2350581041d5f6b0c4c>@@V<lambda_2358e3775559c9db80273638284d5e45>@@@?$__crt_seh_guarded_call@X@@QEAAX$$QEAV<lambda_d80eeec6fff315bfe5c115232f3240e3>@@AEAV<lambda_6e4b09c48022b2350581041d5f6b0c4c>@@$$QEAV<lambda_2358e3775559c9db80273638284d5e45>@@@Z 0000000180044b68 f   libucrt:exit.obj
 0001:00043ba0       ??R<lambda_6e4b09c48022b2350581041d5f6b0c4c>@@QEBA@XZ 0000000180044ba0 f   libucrt:exit.obj
 0001:00043c64       ?atexit_exception_filter@@YAHK@Z 0000000180044c64 f   libucrt:exit.obj
 0001:00043c70       ?common_exit@@YAXHW4_crt_exit_cleanup_mode@@W4_crt_exit_return_mode@@@Z 0000000180044c70 f   libucrt:exit.obj
 0001:00043d2c       ?exit_or_terminate_process@@YAXI@Z 0000000180044d2c f   libucrt:exit.obj
 0001:00043d78       ?try_cor_exit_process@@YAXI@Z 0000000180044d78 f   libucrt:exit.obj
 0001:00043e00       ??$parse_command_line@D@@YAXPEADPEAPEAD0PEA_K2@Z 0000000180044e00 f   libucrt:argv_parsing.obj
 0001:000441ac       ??$common_initialize_environment_nolock@D@@YAHXZ 00000001800451ac f   libucrt:environment_initialization.obj
 0001:00044218       ??$common_initialize_environment_nolock@_W@@YAHXZ 0000000180045218 f   libucrt:environment_initialization.obj
 0001:00044280       ??$create_environment@D@@YAQEAPEADQEAD@Z 0000000180045280 f   libucrt:environment_initialization.obj
 0001:00044388       ??$create_environment@_W@@YAQEAPEA_WQEA_W@Z 0000000180045388 f   libucrt:environment_initialization.obj
 0001:0004449c       ??$free_environment@D@@YAXQEAPEAD@Z 000000018004549c f   libucrt:environment_initialization.obj
 0001:0004449c       ??$free_environment@_W@@YAXQEAPEA_W@Z 000000018004549c f   libucrt:environment_initialization.obj
 0001:000444e0       ??$initialize_environment_by_cloning_nolock@_W@@YAHXZ 00000001800454e0 f   libucrt:environment_initialization.obj
 0001:00044594       ??$uninitialize_environment_internal@D@@YAXAEAPEAPEAD@Z 0000000180045594 f   libucrt:environment_initialization.obj
 0001:000445b0       ??$uninitialize_environment_internal@_W@@YAXAEAPEAPEA_W@Z 00000001800455b0 f   libucrt:environment_initialization.obj
 0001:00044648       ??$?RV<lambda_7777bce6b2f8c936911f934f8298dc43>@@AEAV<lambda_f03950bc5685219e0bcd2087efbe011e>@@V<lambda_3883c3dff614d5e0c5f61bb1ac94921c>@@@?$__crt_seh_guarded_call@H@@QEAAH$$QEAV<lambda_7777bce6b2f8c936911f934f8298dc43>@@AEAV<lambda_f03950bc5685219e0bcd2087efbe011e>@@$$QEAV<lambda_3883c3dff614d5e0c5f61bb1ac94921c>@@@Z 0000000180045648 f   libucrt:onexit.obj
 0001:00044684       ??R<lambda_f03950bc5685219e0bcd2087efbe011e>@@QEBAHXZ 0000000180045684 f   libucrt:onexit.obj
 0001:00044800       initialize_global_variables 0000000180045800 f   libucrt:initialization.obj
 0001:00044814       initialize_c               0000000180045814 f   libucrt:initialization.obj
 0001:00044838       initialize_environment     0000000180045838 f   libucrt:initialization.obj
 0001:00044838       initialize_global_state_isolation 0000000180045838 f   libucrt:initialization.obj
 0001:00044838       report_memory_leaks        0000000180045838 f   libucrt:initialization.obj
 0001:00044838       uninitialize_c             0000000180045838 f   libucrt:initialization.obj
 0001:00044838       uninitialize_global_state_isolation 0000000180045838 f   libucrt:initialization.obj
 0001:0004483c       uninitialize_environment   000000018004583c f   libucrt:initialization.obj
 0001:0004484c       initialize_pointers        000000018004584c f   libucrt:initialization.obj
 0001:0004488c       uninitialize_vcruntime     000000018004588c f   libucrt:initialization.obj
 0001:00044894       uninitialize_allocated_memory 0000000180045894 f   libucrt:initialization.obj
 0001:000448d4       uninitialize_allocated_io_buffers 00000001800458d4 f   libucrt:initialization.obj
 0001:000449d0       ?_strupr_s_l_stat@@YAHQEAD_KQEAU__crt_locale_pointers@@@Z 00000001800459d0 f   libucrt:strupr.obj
 0001:00046518       ??$?RV<lambda_0ae27a3a962d80f24befdcbee591983d>@@AEAV<lambda_8d0ee55de4b1038c4002e0adecdf1839>@@V<lambda_dc504788e8f1664fe9b84e20bfb512f2>@@@?$__crt_seh_guarded_call@X@@QEAAX$$QEAV<lambda_0ae27a3a962d80f24befdcbee591983d>@@AEAV<lambda_8d0ee55de4b1038c4002e0adecdf1839>@@$$QEAV<lambda_dc504788e8f1664fe9b84e20bfb512f2>@@@Z 0000000180047518 f   libucrt:per_thread_data.obj
 0001:00046558       ??$?RV<lambda_2d41944a1d46af3157314b8a01080d33>@@AEAV<lambda_8f455de75cd7d7f24b4096f044d8b9e6>@@V<lambda_aa500f224e6afead328df44964fe2772>@@@?$__crt_seh_guarded_call@X@@QEAAX$$QEAV<lambda_2d41944a1d46af3157314b8a01080d33>@@AEAV<lambda_8f455de75cd7d7f24b4096f044d8b9e6>@@$$QEAV<lambda_aa500f224e6afead328df44964fe2772>@@@Z 0000000180047558 f   libucrt:per_thread_data.obj
 0001:00046598       ??$?RV<lambda_aa87e3671a710a21b5dc78c0bdf72e11>@@AEAV<lambda_92619d2358a28f41a33ba319515a20b9>@@V<lambda_6992ecaafeb10aed2b74cb1fae11a551>@@@?$__crt_seh_guarded_call@X@@QEAAX$$QEAV<lambda_aa87e3671a710a21b5dc78c0bdf72e11>@@AEAV<lambda_92619d2358a28f41a33ba319515a20b9>@@$$QEAV<lambda_6992ecaafeb10aed2b74cb1fae11a551>@@@Z 0000000180047598 f   libucrt:per_thread_data.obj
 0001:000465e0       ??$?RV<lambda_f2e299630e499de9f9a165e60fcd3db5>@@AEAV<lambda_2ae9d31cdba2644fcbeaf08da7c24588>@@V<lambda_40d01ff24d0e7b3814fdbdcee8eab3c7>@@@?$__crt_seh_guarded_call@X@@QEAAX$$QEAV<lambda_f2e299630e499de9f9a165e60fcd3db5>@@AEAV<lambda_2ae9d31cdba2644fcbeaf08da7c24588>@@$$QEAV<lambda_40d01ff24d0e7b3814fdbdcee8eab3c7>@@@Z 00000001800475e0 f   libucrt:per_thread_data.obj
 0001:00046640       ?construct_ptd_array@@YAXQEAU__acrt_ptd@@@Z 0000000180047640 f   libucrt:per_thread_data.obj
 0001:00046710       ?destroy_fls@@YAXPEAX@Z    0000000180047710 f   libucrt:per_thread_data.obj
 0001:00046730       ?destroy_ptd_array@@YAXQEAU__acrt_ptd@@@Z 0000000180047730 f   libucrt:per_thread_data.obj
 0001:00046828       ?replace_current_thread_locale_nolock@@YAXQEAU__acrt_ptd@@QEAU__crt_locale_data@@@Z 0000000180047828 f   libucrt:per_thread_data.obj
 0001:00046be4       ?fp_format_a@@YAHQEBNPEAD_KQEAD2H_NIQEAU__crt_locale_pointers@@@Z 0000000180047be4 f   libucrt:cvt.obj
 0001:00046f54       ?fp_format_e@@YAHQEBNQEAD_K12H_NIQEAU__crt_locale_pointers@@@Z 0000000180047f54 f   libucrt:cvt.obj
 0001:00047030       ?fp_format_e_internal@@YAHQEAD_KH_NIQEAU_strflt@@2QEAU__crt_locale_pointers@@@Z 0000000180048030 f   libucrt:cvt.obj
 0001:00047204       ?fp_format_f_internal@@YAHQEAD_KHQEAU_strflt@@_NQEAU__crt_locale_pointers@@@Z 0000000180048204 f   libucrt:cvt.obj
 0001:00047348       ?fp_format_g@@YAHQEBNQEAD_K12H_NIQEAU__crt_locale_pointers@@@Z 0000000180048348 f   libucrt:cvt.obj
 0001:000478e4       ??$?RV<lambda_410d79af7f07d98d83a3f525b3859a53>@@AEAV<lambda_3e16ef9562a7dcce91392c22ab16ea36>@@V<lambda_38119f0e861e05405d8a144b9b982f0a>@@@?$__crt_seh_guarded_call@X@@QEAAX$$QEAV<lambda_410d79af7f07d98d83a3f525b3859a53>@@AEAV<lambda_3e16ef9562a7dcce91392c22ab16ea36>@@$$QEAV<lambda_38119f0e861e05405d8a144b9b982f0a>@@@Z 00000001800488e4 f   libucrt:wsetlocale.obj
 0001:00047990       ?initialize_inherited_file_handles_nolock@@YAXXZ 0000000180048990 f   libucrt:ioinit.obj
 0001:00047a80       ?initialize_stdio_handles_nolock@@YAXXZ 0000000180048a80 f   libucrt:ioinit.obj
 0001:00047c08       ??$?RV<lambda_751a882b2c74d4b022dec766aa51a29a>@@AEAV<lambda_628dfdc04ba53c8bfc02c9951375f3f5>@@V<lambda_f6c7be5f7998530c34de24c7437d6b54>@@@?$__crt_seh_guarded_call@H@@QEAAH$$QEAV<lambda_751a882b2c74d4b022dec766aa51a29a>@@AEAV<lambda_628dfdc04ba53c8bfc02c9951375f3f5>@@$$QEAV<lambda_f6c7be5f7998530c34de24c7437d6b54>@@@Z 0000000180048c08 f   libucrt:close.obj
 0001:00047e54       ?find_or_allocate_unused_stream_nolock@@YA?AV__crt_stdio_stream@@XZ 0000000180048e54 f   libucrt:stream.obj
 0001:00047ff0       $$000000                   0000000180048ff0     libucrt:fpsr.obj
 0001:00048464       ?try_get_function@@YAPEAXW4function_id@?A0x391cf84c@@QEBDQEBW4module_id@2@2@Z 0000000180049464 f   libucrt:winapi_thunks.obj
 0001:00048cf8       ??$common_lseek@J@@YAJHJH@Z 0000000180049cf8 f   libucrt:lseek.obj
 0001:00048de4       ??$common_lseek@_J@@YA_JH_JH@Z 0000000180049de4 f   libucrt:lseek.obj
 0001:00048ed4       ??$common_lseek_nolock@J@@YAJHJH@Z 0000000180049ed4 f   libucrt:lseek.obj
 0001:00048fc8       ??$common_lseek_nolock@_J@@YA_JH_JH@Z 0000000180049fc8 f   libucrt:lseek.obj
 0001:000490e4       ??$translate_text_mode_nolock@D@@YAHHQEAD_K@Z 000000018004a0e4 f   libucrt:read.obj
 0001:000492a4       ??$translate_text_mode_nolock@_W@@YAHHQEA_W_K@Z 000000018004a2a4 f   libucrt:read.obj
 0001:00049520       ?translate_ansi_or_utf8_nolock@@YAHHQEAD_KQEA_W1@Z 000000018004a520 f   libucrt:read.obj
 0001:0004a754       ??$common_fdopen@_W@@YAPEAU_iobuf@@HQEB_W@Z 000000018004b754 f   libucrt:fdopen.obj
 0001:0004a848       ??$?RV<lambda_a37b2b86f63e897a80ea819b0eb08c01>@@AEAV<lambda_38ce7e780aa69e748d6df282ebc68efe>@@V<lambda_99fb1378e971ab6e7edea83e3a7a83a2>@@@?$__crt_seh_guarded_call@H@@QEAAH$$QEAV<lambda_a37b2b86f63e897a80ea819b0eb08c01>@@AEAV<lambda_38ce7e780aa69e748d6df282ebc68efe>@@$$QEAV<lambda_99fb1378e971ab6e7edea83e3a7a83a2>@@@Z 000000018004b848 f   libucrt:commit.obj
 0001:0004a968       ?write_double_translated_ansi_nolock@@YA?AUwrite_result@?A0x17268360@@HQEBDI@Z 000000018004b968 f   libucrt:write.obj
 0001:0004ae38       ?write_text_ansi_nolock@@YA?AUwrite_result@?A0x17268360@@HQEBDI@Z 000000018004be38 f   libucrt:write.obj
 0001:0004af3c       ?write_text_utf16le_nolock@@YA?AUwrite_result@?A0x17268360@@HQEBDI@Z 000000018004bf3c f   libucrt:write.obj
 0001:0004b058       ?write_text_utf8_nolock@@YA?AUwrite_result@?A0x17268360@@HQEBDI@Z 000000018004c058 f   libucrt:write.obj
 0001:0004b590       ??$common_xtox@_KD@@YAH_KQEAD0I_N@Z 000000018004c590 f   libucrt:xtoa.obj
 0001:0004b65c       ??$common_xtox_s@_KD@@YAH_KQEAD0I_N@Z 000000018004c65c f   libucrt:xtoa.obj
 0001:0004b7f8       ??$common_sopen_dispatch@D@@YAHQEBDHHHQEAHH@Z 000000018004c7f8 f   libucrt:open.obj
 0001:0004b8bc       ??$common_sopen_dispatch@_W@@YAHQEB_WHHHQEAHH@Z 000000018004c8bc f   libucrt:open.obj
 0001:0004b980       ?configure_text_mode@@YAHHUfile_options@?A0xa9d50aae@@HAEAW4__crt_lowio_text_mode@@@Z 000000018004c980 f   libucrt:open.obj
 0001:0004bc14       ?decode_options@@YA?AUfile_options@?A0xa9d50aae@@HHH@Z 000000018004cc14 f   libucrt:open.obj
 0001:0004be20       ?truncate_ctrl_z_if_present@@YAHH@Z 000000018004ce20 f   libucrt:open.obj
 0001:0004c4f4       ??$write_buffer_nolock@D@@YA_NDV__crt_stdio_stream@@@Z 000000018004d4f4 f   libucrt:_flsbuf.obj
 0001:0004c5d8       ?stream_is_at_end_of_file_nolock@@YA_NV__crt_stdio_stream@@@Z 000000018004d5d8 f   libucrt:_flsbuf.obj
 0001:0004c894       ??$?RV<lambda_24016bbcb8f60cbe41e899a2382ed12a>@@AEAV<lambda_f9f2d660215b636168e2032e31cf969c>@@V<lambda_7fbd5cec917a4378cbcd803f78c7a734>@@@?$__crt_seh_guarded_call@_N@@QEAA_N$$QEAV<lambda_24016bbcb8f60cbe41e899a2382ed12a>@@AEAV<lambda_f9f2d660215b636168e2032e31cf969c>@@$$QEAV<lambda_7fbd5cec917a4378cbcd803f78c7a734>@@@Z 000000018004d894 f   libucrt:spawnv.obj
 0001:0004c8d4       ??$common_spawnv@_W@@YA_JHQEB_WQEBQEB_W1@Z 000000018004d8d4 f   libucrt:spawnv.obj
 0001:0004cb24       ??$execute_command@_W@@YA_JHQEB_WQEBQEB_W1@Z 000000018004db24 f   libucrt:spawnv.obj
 0001:0004cd84       ??R<lambda_f9f2d660215b636168e2032e31cf969c>@@QEBA_NXZ 000000018004dd84 f   libucrt:spawnv.obj
 0001:0004cf80       ?accumulate_inheritable_handles@@YA_NQEAPEAEQEA_K_N@Z 000000018004df80 f   libucrt:spawnv.obj
 0001:0004cfe0       ??$common_spawnvp@_W@@YA_JHQEB_WQEBQEB_W1@Z 000000018004dfe0 f   libucrt:spawnvp.obj
 0001:0004d34c       ?<lambda_invoker_cdecl>@<lambda_a1ce4c8ae42411fd470c77163914f50e>@@CAHPEBX0@Z 000000018004e34c f   libucrt:argv_wildcards.obj
 0001:0004d4ec       ??$common_expand_argv_wildcards@D@@YAHQEAPEADQEAPEAPEAD@Z 000000018004e4ec f   libucrt:argv_wildcards.obj
 0001:0004d6f8       ??$copy_and_add_argument_to_buffer@D@@YAHQEBD0_KAEAV?$argument_list@D@?A0x5f5c8891@@@Z 000000018004e6f8 f   libucrt:argv_wildcards.obj
 0001:0004d880       ??$expand_argument_wildcards@D@@YAHQEAD0AEAV?$argument_list@D@?A0x5f5c8891@@@Z 000000018004e880 f   libucrt:argv_wildcards.obj
 0001:0004ddcc       ??$?RV<lambda_efdfa57d1f175319df784efa44bb7b81>@@AEAV<lambda_5f0a4c1567f8adc6734073e5d1e1b35c>@@V<lambda_2e8a7d3640ea6ccb4c2413664c2db6fd>@@@?$__crt_seh_guarded_call@X@@QEAAX$$QEAV<lambda_efdfa57d1f175319df784efa44bb7b81>@@AEAV<lambda_5f0a4c1567f8adc6734073e5d1e1b35c>@@$$QEAV<lambda_2e8a7d3640ea6ccb4c2413664c2db6fd>@@@Z 000000018004edcc f   libucrt:mbctype.obj
 0001:0004df88       ?getSystemCP@@YAHH@Z       000000018004ef88 f   libucrt:mbctype.obj
 0001:0004e008       ?setSBCS@@YAXPEAU__crt_multibyte_data@@@Z 000000018004f008 f   libucrt:mbctype.obj
 0001:0004e098       ?setSBUpLow@@YAXPEAU__crt_multibyte_data@@@Z 000000018004f098 f   libucrt:mbctype.obj
 0001:0004e27c       ?setmbcp_internal@@YAHH_NQEAU__acrt_ptd@@QEAPEAU__crt_multibyte_data@@@Z 000000018004f27c f   libucrt:mbctype.obj
 0001:0004e440       ?update_thread_multibyte_data_internal@@YAPEAU__crt_multibyte_data@@QEAU__acrt_ptd@@QEAPEAU1@@Z 000000018004f440 f   libucrt:mbctype.obj
 0001:0004e830       ?x_ismbbtype_l@@YAHPEAU__crt_locale_pointers@@IHH@Z 000000018004f830 f   libucrt:ismbbyte.obj
 0001:0004eb7c       ??$common_set_variable_in_environment_nolock@_W@@YAHQEA_WH@Z 000000018004fb7c f   libucrt:setenv.obj
 0001:0004eea0       ??$copy_environment@_W@@YAPEAPEA_WQEAPEA_W@Z 000000018004fea0 f   libucrt:setenv.obj
 0001:0004f0e8       ??$?RV<lambda_450d765d439847d4c735a33c368b5fc0>@@AEAV<lambda_44731a7d0e6d81c3e6aa82d741081786>@@V<lambda_601a2a7da3b7a96e9554ac7215c4b07c>@@@?$__crt_seh_guarded_call@P6AXH@Z@@QEAAP6AXH@Z$$QEAV<lambda_450d765d439847d4c735a33c368b5fc0>@@AEAV<lambda_44731a7d0e6d81c3e6aa82d741081786>@@$$QEAV<lambda_601a2a7da3b7a96e9554ac7215c4b07c>@@@Z 00000001800500e8 f   libucrt:signal.obj
 0001:0004f444       ?__acrt_LCMapStringA_stat@@YAHPEAU__crt_locale_pointers@@PEB_WKPEBDHPEADHHH@Z 0000000180050444 f   libucrt:lcmapstringa.obj
 0001:000513a8       ?free_crt_array_internal@@YAXQEAPEBX_K@Z 00000001800523a8 f   libucrt:inittime.obj
 0001:00052628       ??$construct_environment_block@_W@@YAHQEBQEB_WQEAPEA_W@Z 0000000180053628 f   libucrt:cenvarg.obj
 0001:00052f1c       ?initialize_multibyte@@YAHXZ 0000000180053f1c f   libucrt:multibyte_initializer.obj
 0001:000532b0       $$000000                   00000001800542b0     libucrt:log10.obj
 0001:00053994       _call_matherr              0000000180054994 f   libucrt:libm_error.obj
 0001:000539fc       _exception_enabled         00000001800549fc f   libucrt:libm_error.obj
 0001:00053c90       _log_special_common        0000000180054c90 f   libucrt:log_special.obj
 0001:00054340       $$000000                   0000000180055340     LIBCMT:chkstk.obj
 0001:000543d0       $$000000                   00000001800553d0     libvcruntime:memcmp.obj
 0001:000544b0       $$000000                   00000001800554b0     libvcruntime:memchr.obj
 0001:00054530       $$000000                   0000000180055530     libucrt:strcmp.obj
 0001:000545b0       $$000000                   00000001800555b0     LIBCMT:guard_dispatch.obj
 0001:000545d0       $$000000                   00000001800555d0     LIBCMT:guard_xfg_dispatch.obj
 0001:000545f0       ?fin$0@?0??dllmain_crt_process_attach@@YAHQEAUHINSTANCE__@@QEAX@Z@4HA 00000001800555f0 f   LIBCMT:dll_dllmain.obj
 0001:00054607       ?fin$0@?0??dllmain_crt_process_detach@@YAH_N@Z@4HA 0000000180055607 f   LIBCMT:dll_dllmain.obj
 0001:00054620       ?fin$1@?0??dllmain_crt_process_detach@@YAH_N@Z@4HA 0000000180055620 f   LIBCMT:dll_dllmain.obj
 0001:00054634       ?filt$0@?0??dllmain_dispatch@@YAHQEAUHINSTANCE__@@KQEAX@Z@4HA 0000000180055634 f   LIBCMT:dll_dllmain.obj
 0001:0005466a       __scrt_is_nonwritable_in_current_image$filt$0 000000018005566a f   LIBCMT:utility.obj
 0001:00054682       __DestructExceptionObject$filt$0 0000000180055682 f   libvcruntime:ehhelpers.obj
 0001:00054718       ?fin$0@?0???$?RV<lambda_842d9ff0dc9ef11c61343bbaebe7f885>@@AEAV<lambda_c5860995281e5c4ce005b3de8f5874ee>@@V<lambda_d90129c13df834fdcbf8d2b88dafcf2d>@@@?$__crt_seh_guarded_call@X@@QEAAX$$QEAV<lambda_842d9ff0dc9ef11c61343bbaebe7f885>@@AEAV<lambda_c5860995281e5c4ce005b3de8f5874ee>@@$$QEAV<lambda_d90129c13df834fdcbf8d2b88dafcf2d>@@@Z@4HA 0000000180055718 f   libucrt:fflush.obj
 0001:00054718       ?fin$0@?0???$?RV<lambda_c376a267cfb53b6959b3b692ec76b120>@@AEAV<lambda_9a32fed5bf61b6b509b2d3f6003082a1>@@V<lambda_572fbb9fa0ab338edf41edfd4b5fcc8d>@@@?$__crt_seh_guarded_call@H@@QEAAH$$QEAV<lambda_c376a267cfb53b6959b3b692ec76b120>@@AEAV<lambda_9a32fed5bf61b6b509b2d3f6003082a1>@@$$QEAV<lambda_572fbb9fa0ab338edf41edfd4b5fcc8d>@@@Z@4HA 0000000180055718 f   libucrt:fflush.obj
 0001:00054718       ?fin$0@?0???$?RV<lambda_2831f20263db5b546e098b45503eb778>@@AEAV<lambda_5856287d7ecd2be6c9197bb4007c3f6e>@@V<lambda_0838d7e100fbcbd261b69cfea6abb102>@@@?$__crt_seh_guarded_call@_K@@QEAA_K$$QEAV<lambda_2831f20263db5b546e098b45503eb778>@@AEAV<lambda_5856287d7ecd2be6c9197bb4007c3f6e>@@$$QEAV<lambda_0838d7e100fbcbd261b69cfea6abb102>@@@Z@4HA 0000000180055718 f   libucrt:fwrite.obj
 0001:00054718       ?fin$0@?0???$?RV<lambda_082dd7c0feb7dbdaf245f261e54a6583>@@AEAV<lambda_f3caf1ecae5fe01a9a1a6239afa44510>@@V<lambda_c640b76c0755ae85b317b35c67c61e6b>@@@?$__crt_seh_guarded_call@H@@QEAAH$$QEAV<lambda_082dd7c0feb7dbdaf245f261e54a6583>@@AEAV<lambda_f3caf1ecae5fe01a9a1a6239afa44510>@@$$QEAV<lambda_c640b76c0755ae85b317b35c67c61e6b>@@@Z@4HA 0000000180055718 f   libucrt:input.obj
 0001:00054718       ?fin$0@?0???$?RV<lambda_fe5404e9642edbb7c8ae71e1dcfa4018>@@AEAV<lambda_36eeb330e99a4f0bf8a7da86d0894cb9>@@V<lambda_2fa474834de80dc12f7a3c6eddd7a366>@@@?$__crt_seh_guarded_call@H@@QEAAH$$QEAV<lambda_fe5404e9642edbb7c8ae71e1dcfa4018>@@AEAV<lambda_36eeb330e99a4f0bf8a7da86d0894cb9>@@$$QEAV<lambda_2fa474834de80dc12f7a3c6eddd7a366>@@@Z@4HA 0000000180055718 f   libucrt:output.obj
 0001:00054718       ?fin$0@?0???$?RV<lambda_84ec643ea9557e2f7dc01bb0e9624395>@@AEAV<lambda_ca71763b3c0644891230e4f79ea54fa6>@@V<lambda_439a761618c59b0600e24586724d733b>@@@?$__crt_seh_guarded_call@H@@QEAAH$$QEAV<lambda_84ec643ea9557e2f7dc01bb0e9624395>@@AEAV<lambda_ca71763b3c0644891230e4f79ea54fa6>@@$$QEAV<lambda_439a761618c59b0600e24586724d733b>@@@Z@4HA 0000000180055718 f   libucrt:setvbuf.obj
 0001:00054733       clearerr_s$fin$0           0000000180055733 f   libucrt:clearerr.obj
 0001:00054733       fclose$fin$0               0000000180055733 f   libucrt:fclose.obj
 0001:00054733       ?fin$0@?0??common_fseek@@YAHV__crt_stdio_stream@@_JH@Z@4HA 0000000180055733 f   libucrt:fseek.obj
 0001:00054733       ?fin$0@?0???$common_ftell@_J@@YA_JV__crt_stdio_stream@@@Z@4HA 0000000180055733 f   libucrt:ftell.obj
 0001:00054733       rewind$fin$0               0000000180055733 f   libucrt:rewind.obj
 0001:0005474b       _ctrlfp$filt$0             000000018005574b f   libucrt:fpctrl.obj
 0001:0005474b       common_control87$filt$0    000000018005574b f   libucrt:ieee.obj
 0001:00054777       ?fin$0@?0???$common_fsopen@_W@@YAPEAU_iobuf@@QEB_W0H@Z@4HA 0000000180055777 f   libucrt:fopen.obj
 0001:000547a2       fgetc$fin$0                00000001800557a2 f   libucrt:fgetc.obj
 0001:000547bc       ?fin$0@?0???$common_freopen@_W@@YAHQEAPEAU_iobuf@@QEB_W1V__crt_stdio_stream@@H@Z@4HA 00000001800557bc f   libucrt:freopen.obj
 0001:000547d4       ungetc$fin$0               00000001800557d4 f   libucrt:ungetc.obj
 0001:000547ec       fread_s$fin$0              00000001800557ec f   libucrt:fread.obj
 0001:00054804       ?fin$0@?0???$common_popen@_W@@YAPEAU_iobuf@@QEB_W0@Z@4HA 0000000180055804 f   libucrt:popen.obj
 0001:0005481f       _pclose$fin$0              000000018005581f f   libucrt:popen.obj
 0001:00054838       ?fin$0@?0???$?RV<lambda_886d6c58226a84441f68b9f2b8217b83>@@AEAV<lambda_ab61a845afdef5b7c387490eaf3616ee>@@V<lambda_f7f22ab5edc0698d5f6905b0d3f44752>@@@?$__crt_seh_guarded_call@X@@QEAAX$$QEAV<lambda_886d6c58226a84441f68b9f2b8217b83>@@AEAV<lambda_ab61a845afdef5b7c387490eaf3616ee>@@$$QEAV<lambda_f7f22ab5edc0698d5f6905b0d3f44752>@@@Z@4HA 0000000180055838 f   libucrt:fflush.obj
 0001:00054855       ?fin$0@?0???$common_fgets@D@@YAPEADQEADHV__crt_stdio_stream@@@Z@4HA 0000000180055855 f   libucrt:fgets.obj
 0001:0005486d       ?fin$0@?0??common_tmpfile@@YAHQEAPEAU_iobuf@@H@Z@4HA 000000018005586d f   libucrt:tmpfile.obj
 0001:00054886       ?fin$0@?0??common_tmpfile_nolock@@YAHQEAPEAU_iobuf@@H@Z@4HA 0000000180055886 f   libucrt:tmpfile.obj
 0001:000548af       ?fin$0@?0???$common_dupenv_s@_W@@YAHQEAPEA_WQEA_KQEB_WHQEBDH@Z@4HA 00000001800558af f   libucrt:getenv.obj
 0001:000548c8       ?fin$0@?0???$common_getenv@_W@@YAPEA_WQEB_W@Z@4HA 00000001800558c8 f   libucrt:getenv.obj
 0001:000548e1       ?fin$0@?0???$?RV<lambda_24016bbcb8f60cbe41e899a2382ed12a>@@AEAV<lambda_f9f2d660215b636168e2032e31cf969c>@@V<lambda_7fbd5cec917a4378cbcd803f78c7a734>@@@?$__crt_seh_guarded_call@_N@@QEAA_N$$QEAV<lambda_24016bbcb8f60cbe41e899a2382ed12a>@@AEAV<lambda_f9f2d660215b636168e2032e31cf969c>@@$$QEAV<lambda_7fbd5cec917a4378cbcd803f78c7a734>@@@Z@4HA 00000001800558e1 f   libucrt:spawnv.obj
 0001:000548e1       ?fin$0@?0???$?RV<lambda_0ae27a3a962d80f24befdcbee591983d>@@AEAV<lambda_8d0ee55de4b1038c4002e0adecdf1839>@@V<lambda_dc504788e8f1664fe9b84e20bfb512f2>@@@?$__crt_seh_guarded_call@X@@QEAAX$$QEAV<lambda_0ae27a3a962d80f24befdcbee591983d>@@AEAV<lambda_8d0ee55de4b1038c4002e0adecdf1839>@@$$QEAV<lambda_dc504788e8f1664fe9b84e20bfb512f2>@@@Z@4HA 00000001800558e1 f   libucrt:per_thread_data.obj
 0001:000548e1       ?fin$0@?0???$?RV<lambda_2d41944a1d46af3157314b8a01080d33>@@AEAV<lambda_8f455de75cd7d7f24b4096f044d8b9e6>@@V<lambda_aa500f224e6afead328df44964fe2772>@@@?$__crt_seh_guarded_call@X@@QEAAX$$QEAV<lambda_2d41944a1d46af3157314b8a01080d33>@@AEAV<lambda_8f455de75cd7d7f24b4096f044d8b9e6>@@$$QEAV<lambda_aa500f224e6afead328df44964fe2772>@@@Z@4HA 00000001800558e1 f   libucrt:per_thread_data.obj
 0001:000548e1       ?fin$0@?0???$?RV<lambda_aa87e3671a710a21b5dc78c0bdf72e11>@@AEAV<lambda_92619d2358a28f41a33ba319515a20b9>@@V<lambda_6992ecaafeb10aed2b74cb1fae11a551>@@@?$__crt_seh_guarded_call@X@@QEAAX$$QEAV<lambda_aa87e3671a710a21b5dc78c0bdf72e11>@@AEAV<lambda_92619d2358a28f41a33ba319515a20b9>@@$$QEAV<lambda_6992ecaafeb10aed2b74cb1fae11a551>@@@Z@4HA 00000001800558e1 f   libucrt:per_thread_data.obj
 0001:000548e1       ?fin$0@?0???$?RV<lambda_f2e299630e499de9f9a165e60fcd3db5>@@AEAV<lambda_2ae9d31cdba2644fcbeaf08da7c24588>@@V<lambda_40d01ff24d0e7b3814fdbdcee8eab3c7>@@@?$__crt_seh_guarded_call@X@@QEAAX$$QEAV<lambda_f2e299630e499de9f9a165e60fcd3db5>@@AEAV<lambda_2ae9d31cdba2644fcbeaf08da7c24588>@@$$QEAV<lambda_40d01ff24d0e7b3814fdbdcee8eab3c7>@@@Z@4HA 00000001800558e1 f   libucrt:per_thread_data.obj
 0001:000548e1       ?fin$0@?0???$?RV<lambda_efdfa57d1f175319df784efa44bb7b81>@@AEAV<lambda_5f0a4c1567f8adc6734073e5d1e1b35c>@@V<lambda_2e8a7d3640ea6ccb4c2413664c2db6fd>@@@?$__crt_seh_guarded_call@X@@QEAAX$$QEAV<lambda_efdfa57d1f175319df784efa44bb7b81>@@AEAV<lambda_5f0a4c1567f8adc6734073e5d1e1b35c>@@$$QEAV<lambda_2e8a7d3640ea6ccb4c2413664c2db6fd>@@@Z@4HA 00000001800558e1 f   libucrt:mbctype.obj
 0001:000548e1       ?fin$0@?0???$?RV<lambda_450d765d439847d4c735a33c368b5fc0>@@AEAV<lambda_44731a7d0e6d81c3e6aa82d741081786>@@V<lambda_601a2a7da3b7a96e9554ac7215c4b07c>@@@?$__crt_seh_guarded_call@P6AXH@Z@@QEAAP6AXH@Z$$QEAV<lambda_450d765d439847d4c735a33c368b5fc0>@@AEAV<lambda_44731a7d0e6d81c3e6aa82d741081786>@@$$QEAV<lambda_601a2a7da3b7a96e9554ac7215c4b07c>@@@Z@4HA 00000001800558e1 f   libucrt:signal.obj
 0001:000548e1       ?fin$0@?0???$?RV<lambda_d80eeec6fff315bfe5c115232f3240e3>@@AEAV<lambda_6e4b09c48022b2350581041d5f6b0c4c>@@V<lambda_2358e3775559c9db80273638284d5e45>@@@?$__crt_seh_guarded_call@X@@QEAAX$$QEAV<lambda_d80eeec6fff315bfe5c115232f3240e3>@@AEAV<lambda_6e4b09c48022b2350581041d5f6b0c4c>@@$$QEAV<lambda_2358e3775559c9db80273638284d5e45>@@@Z@4HA 00000001800558e1 f   libucrt:exit.obj
 0001:000548e1       ?fin$0@?0???$?RV<lambda_7777bce6b2f8c936911f934f8298dc43>@@AEAV<lambda_f03950bc5685219e0bcd2087efbe011e>@@V<lambda_3883c3dff614d5e0c5f61bb1ac94921c>@@@?$__crt_seh_guarded_call@H@@QEAAH$$QEAV<lambda_7777bce6b2f8c936911f934f8298dc43>@@AEAV<lambda_f03950bc5685219e0bcd2087efbe011e>@@$$QEAV<lambda_3883c3dff614d5e0c5f61bb1ac94921c>@@@Z@4HA 00000001800558e1 f   libucrt:onexit.obj
 0001:000548fb       ?filt$0@?0???R<lambda_6e4b09c48022b2350581041d5f6b0c4c>@@QEBA@XZ@4HA 00000001800558fb f   libucrt:exit.obj
 0001:00054916       ?fin$0@?0???$?RV<lambda_410d79af7f07d98d83a3f525b3859a53>@@AEAV<lambda_3e16ef9562a7dcce91392c22ab16ea36>@@V<lambda_38119f0e861e05405d8a144b9b982f0a>@@@?$__crt_seh_guarded_call@X@@QEAAX$$QEAV<lambda_410d79af7f07d98d83a3f525b3859a53>@@AEAV<lambda_3e16ef9562a7dcce91392c22ab16ea36>@@$$QEAV<lambda_38119f0e861e05405d8a144b9b982f0a>@@@Z@4HA 0000000180055916 f   libucrt:wsetlocale.obj
 0001:00054930       __acrt_initialize_lowio$fin$0 0000000180055930 f   libucrt:ioinit.obj
 0001:00054930       __acrt_lowio_ensure_fh_exists$fin$0 0000000180055930 f   libucrt:osfinfo.obj
 0001:00054930       _alloc_osfhnd$fin$0        0000000180055930 f   libucrt:osfinfo.obj
 0001:00054949       ?fin$0@?0???$?RV<lambda_751a882b2c74d4b022dec766aa51a29a>@@AEAV<lambda_628dfdc04ba53c8bfc02c9951375f3f5>@@V<lambda_f6c7be5f7998530c34de24c7437d6b54>@@@?$__crt_seh_guarded_call@H@@QEAAH$$QEAV<lambda_751a882b2c74d4b022dec766aa51a29a>@@AEAV<lambda_628dfdc04ba53c8bfc02c9951375f3f5>@@$$QEAV<lambda_f6c7be5f7998530c34de24c7437d6b54>@@@Z@4HA 0000000180055949 f   libucrt:close.obj
 0001:00054949       ?fin$0@?0???$?RV<lambda_a37b2b86f63e897a80ea819b0eb08c01>@@AEAV<lambda_38ce7e780aa69e748d6df282ebc68efe>@@V<lambda_99fb1378e971ab6e7edea83e3a7a83a2>@@@?$__crt_seh_guarded_call@H@@QEAAH$$QEAV<lambda_a37b2b86f63e897a80ea819b0eb08c01>@@AEAV<lambda_38ce7e780aa69e748d6df282ebc68efe>@@$$QEAV<lambda_99fb1378e971ab6e7edea83e3a7a83a2>@@@Z@4HA 0000000180055949 f   libucrt:commit.obj
 0001:00054963       _fcloseall$fin$0           0000000180055963 f   libucrt:closeall.obj
 0001:00054963       ?fin$0@?0??__acrt_stdio_allocate_stream@@YA?AV__crt_stdio_stream@@XZ@4HA 0000000180055963 f   libucrt:stream.obj
 0001:0005497c       ?fin$0@?0???$common_lseek@J@@YAJHJH@Z@4HA 000000018005597c f   libucrt:lseek.obj
 0001:0005497c       ?fin$0@?0???$common_lseek@_J@@YA_JH_JH@Z@4HA 000000018005597c f   libucrt:lseek.obj
 0001:0005497c       _write$fin$0               000000018005597c f   libucrt:write.obj
 0001:00054993       _read$fin$0                0000000180055993 f   libucrt:read.obj
 0001:000549aa       _pipe$fin$1                00000001800559aa f   libucrt:pipe.obj
 0001:000549c6       _pipe$fin$0                00000001800559c6 f   libucrt:pipe.obj
 0001:000549e2       ?fin$0@?0???$common_fdopen@_W@@YAPEAU_iobuf@@HQEB_W@Z@4HA 00000001800559e2 f   libucrt:fdopen.obj
 0001:000549fc       ?fin$0@?0???$common_sopen_dispatch@D@@YAHQEBDHHHQEAHH@Z@4HA 00000001800559fc f   libucrt:open.obj
 0001:000549fc       ?fin$0@?0???$common_sopen_dispatch@_W@@YAHQEB_WHHHQEAHH@Z@4HA 00000001800559fc f   libucrt:open.obj
 0001:00054a4f       _rmtmp$fin$0               0000000180055a4f f   libucrt:rmtmp.obj
 0001:00054a69       _rmtmp$fin$1               0000000180055a69 f   libucrt:rmtmp.obj
 0001:00054a82       ?fin$0@?0??update_thread_multibyte_data_internal@@YAPEAU__crt_multibyte_data@@QEAU__acrt_ptd@@QEAPEAU1@@Z@4HA 0000000180055a82 f   libucrt:mbctype.obj
 0001:00054a9b       _query_new_handler$fin$0   0000000180055a9b f   libucrt:new_handler.obj
 0001:00054ab1       raise$fin$0                0000000180055ab1 f   libucrt:signal.obj
 0001:00054ad2       __acrt_update_thread_locale_data$fin$0 0000000180055ad2 f   libucrt:locale_refcounting.obj
 0001:00054af0       _IsNonwritableInCurrentImage$filt$0 0000000180055af0 f   LIBCMT:pesect.obj
 0002:000007e0       GS_ExceptionPointers       00000001800567e0     LIBCMT:gs_report.obj
 0002:00000800       ?tokenTable@@3QBUStringLiteral@@B 0000000180056800     libvcruntime:undname.obj
 0002:00000900       ?nameTable@@3QBUStringLiteral@@B 0000000180056900     libvcruntime:undname.obj
 0002:00000e30       ?rttiTable@@3QBUStringLiteral@@B 0000000180056e30     libvcruntime:undname.obj
 0002:00000e80       ?IndirectionName@@3QBUStringLiteral@@B 0000000180056e80     libvcruntime:undname.obj
 0002:00000ee0       ?PrefixName@@3QBUStringLiteral@@B 0000000180056ee0     libvcruntime:undname.obj
 0002:000015b8       ?module_names@?A0x3064ecbf@@3QBQEB_WB 00000001800575b8     libvcruntime:winapi_downlevel.obj
 0002:00001678       ?candidate_modules@?1??try_get_FlsAlloc@@YAP6AKP6AXPEAX@Z@ZXZ@4QBW4module_id@?A0x3064ecbf@@B 0000000180057678     libvcruntime:winapi_downlevel.obj
 0002:00001690       ?candidate_modules@?1??try_get_FlsFree@@YAP6AHK@ZXZ@4QBW4module_id@?A0x3064ecbf@@B 0000000180057690     libvcruntime:winapi_downlevel.obj
 0002:000016a0       ?candidate_modules@?1??try_get_FlsGetValue@@YAP6APEAXK@ZXZ@4QBW4module_id@?A0x3064ecbf@@B 00000001800576a0     libvcruntime:winapi_downlevel.obj
 0002:000016b8       ?candidate_modules@?1??try_get_FlsSetValue@@YAP6AHKPEAX@ZXZ@4QBW4module_id@?A0x3064ecbf@@B 00000001800576b8     libvcruntime:winapi_downlevel.obj
 0002:000016d0       ?candidate_modules@?1??try_get_InitializeCriticalSectionEx@@YAP6AHPEAU_RTL_CRITICAL_SECTION@@KK@ZXZ@4QBW4module_id@?A0x3064ecbf@@B 00000001800576d0     libvcruntime:winapi_downlevel.obj
 0002:00001780       ?errtable@@3QBUerrentry@?A0x31fdb9ec@@B 0000000180057780     libucrt:errno.obj
 0002:00001930       ?default_cmd_exe@?1???$common_popen_nolock@_W@@YAPEAU_iobuf@@QEB_W0HAEAY01H@Z@4QB_WB 0000000180057930     libucrt:popen.obj
 0002:00001940       ?slash_c@?1???$common_popen_nolock@_W@@YAPEAU_iobuf@@QEB_W0HAEAY01H@Z@4QB_WB 0000000180057940     libucrt:popen.obj
 0002:00001950       ?comspec_name@?1???$get_comspec@_W@@YAPEB_WXZ@4QB_WB 0000000180057950     libucrt:popen.obj
 0002:00001960       ?backslash@?L@???$get_executable_path@_W@@YAPEB_WQEB_W@Z@4QB_WB 0000000180057960     libucrt:popen.obj
 0002:00001968       ?path_name@?1???$get_path@_W@@YAPEB_WXZ@4QB_WB 0000000180057968     libucrt:popen.obj
 0002:00002290       ?large_power_indices@?1??multiply_by_power_of_ten@__crt_strtox@@YA_NAEAUbig_integer@2@I@Z@4QBUunpack_index@?1??12@YA_N0I@Z@B 0000000180058290     libucrt:input.obj
 0002:00002570       ?comspec_name@?1???$common_system@_W@@YAHQEB_W@Z@4QB_WB 0000000180058570     libucrt:system.obj
 0002:00002580       ?cmd_exe@?1???$common_system@_W@@YAHQEB_W@Z@4QB_WB 0000000180058580     libucrt:system.obj
 0002:00002590       ?slash_c@?1???$common_system@_W@@YAHQEB_W@Z@4QB_WB 0000000180058590     libucrt:system.obj
 0002:000026a0       __acrt_initializers        00000001800586a0     libucrt:initialization.obj
 0002:000027a0       ?strings@?1??fp_format_nan_or_infinity@@YAHW4__acrt_fp_class@@_NPEAD_K1@Z@4QAY03QEBDA 00000001800587a0     libucrt:cvt.obj
 0002:00002f00       __real@433fffffffffffff    0000000180058f00     libucrt:fpsr.obj
 0002:00002f08       __real@c33fffffffffffff    0000000180058f08     libucrt:fpsr.obj
 0002:00002f50       ?module_names@?A0x391cf84c@@3QBQEB_WB 0000000180058f50     libucrt:winapi_thunks.obj
 0002:00003458       ?candidate_modules@?1??try_get_AreFileApisANSI@@YAP6AHXZXZ@4QBW4module_id@?A0x391cf84c@@B 0000000180059458     libucrt:winapi_thunks.obj
 0002:00003470       ?candidate_modules@?1??try_get_CompareStringEx@@YAP6AHPEB_WK0H0HPEAU_nlsversioninfo@@PEAX_J@ZXZ@4QBW4module_id@?A0x391cf84c@@B 0000000180059470     libucrt:winapi_thunks.obj
 0002:00003488       ?candidate_modules@?1??try_get_FlsAlloc@@YAP6AKP6AXPEAX@Z@ZXZ@4QBW4module_id@?A0x391cf84c@@B 0000000180059488     libucrt:winapi_thunks.obj
 0002:00003490       ?candidate_modules@?1??try_get_FlsFree@@YAP6AHK@ZXZ@4QBW4module_id@?A0x391cf84c@@B 0000000180059490     libucrt:winapi_thunks.obj
 0002:00003498       ?candidate_modules@?1??try_get_FlsGetValue@@YAP6APEAXK@ZXZ@4QBW4module_id@?A0x391cf84c@@B 0000000180059498     libucrt:winapi_thunks.obj
 0002:000034a0       ?candidate_modules@?1??try_get_FlsSetValue@@YAP6AHKPEAX@ZXZ@4QBW4module_id@?A0x391cf84c@@B 00000001800594a0     libucrt:winapi_thunks.obj
 0002:000034a8       ?candidate_modules@?1??try_get_InitializeCriticalSectionEx@@YAP6AHPEAU_RTL_CRITICAL_SECTION@@KK@ZXZ@4QBW4module_id@?A0x391cf84c@@B 00000001800594a8     libucrt:winapi_thunks.obj
 0002:000034b0       ?candidate_modules@?1??try_get_LCMapStringEx@@YAP6AHPEB_WK0HPEA_WHPEAU_nlsversioninfo@@PEAX_J@ZXZ@4QBW4module_id@?A0x391cf84c@@B 00000001800594b0     libucrt:winapi_thunks.obj
 0002:000034c8       ?candidate_modules@?1??try_get_LocaleNameToLCID@@YAP6AKPEB_WK@ZXZ@4QBW4module_id@?A0x391cf84c@@B 00000001800594c8     libucrt:winapi_thunks.obj
 0002:000034e4       ?candidate_modules@?1??try_get_AppPolicyGetProcessTerminationMethod@@YAP6AJPEAXPEAW4AppPolicyProcessTerminationMethod@@@ZXZ@4QBW4module_id@?A0x391cf84c@@B 00000001800594e4     libucrt:winapi_thunks.obj
 0002:00004214       ?dot_slash@?CB@???$common_spawnv@_W@@YA_JHQEB_WQEBQEB_W1@Z@4QB_WB 000000018005a214     libucrt:spawnv.obj
 0002:00004220       ?extensions@?CP@???$common_spawnv@_W@@YA_JHQEB_WQEBQEB_W1@Z@4QAY04$$CB_WA 000000018005a220     libucrt:spawnv.obj
 0002:00004248       ?_mb_locale_names@@3QBQEB_WB 000000018005a248     libucrt:mbctype.obj
 0002:000042b0       ?large_power_indices@?1??multiply_by_power_of_ten@__crt_strtox@@YA_NAEAUbig_integer@2@I@Z@4QBUunpack_index@?1??12@YA_N0I@Z@B 000000018005a2b0     libucrt:cfout.obj
 0002:00004370       ?LcidToLocaleNameTable@?A0x881e4c05@@3QBULcidToLocaleName@1@B 000000018005a370     libucrt:lcidtoname_downlevel.obj
 0002:00005dc0       ?LocaleNameToIndexTable@?A0x881e4c05@@3QBULocaleNameIndex@1@B 000000018005bdc0     libucrt:lcidtoname_downlevel.obj
 0002:00007654       ?equal_sign@?BD@???$construct_environment_block@_W@@YAHQEBQEB_WQEAPEA_W@Z@4QB_WB 000000018005d654     libucrt:cenvarg.obj
 0002:00007660       __real_ninf                000000018005d660     libucrt:log10.obj
 0002:00007670       __real_inf                 000000018005d670     libucrt:log10.obj
 0002:00007680       __real_neg_qnan            000000018005d680     libucrt:log10.obj
 0002:00007690       __real_qnanbit             000000018005d690     libucrt:log10.obj
 0002:000076a0       __int_1023                 000000018005d6a0     libucrt:log10.obj
 0002:000076b0       __mask_001                 000000018005d6b0     libucrt:log10.obj
 0002:000076c0       __mask_mant                000000018005d6c0     libucrt:log10.obj
 0002:000076d0       __mask_mant_top8           000000018005d6d0     libucrt:log10.obj
 0002:000076e0       __mask_mant9               000000018005d6e0     libucrt:log10.obj
 0002:000076f0       __real_log10_e             000000018005d6f0     libucrt:log10.obj
 0002:00007700       __real_log10_e_lead        000000018005d700     libucrt:log10.obj
 0002:00007710       __real_log10_e_tail        000000018005d710     libucrt:log10.obj
 0002:00007720       __real_log10_2_lead        000000018005d720     libucrt:log10.obj
 0002:00007730       __real_log10_2_tail        000000018005d730     libucrt:log10.obj
 0002:00007740       __real_two                 000000018005d740     libucrt:log10.obj
 0002:00007750       __real_one                 000000018005d750     libucrt:log10.obj
 0002:00007760       __real_half                000000018005d760     libucrt:log10.obj
 0002:00007770       __mask_100                 000000018005d770     libucrt:log10.obj
 0002:00007780       __real_1_over_512          000000018005d780     libucrt:log10.obj
 0002:00007790       __real_1_over_2            000000018005d790     libucrt:log10.obj
 0002:000077a0       __real_1_over_3            000000018005d7a0     libucrt:log10.obj
 0002:000077b0       __real_1_over_4            000000018005d7b0     libucrt:log10.obj
 0002:000077c0       __real_1_over_5            000000018005d7c0     libucrt:log10.obj
 0002:000077d0       __real_1_over_6            000000018005d7d0     libucrt:log10.obj
 0002:000077e0       __real_neg_1023            000000018005d7e0     libucrt:log10.obj
 0002:000077f0       __mask_2045                000000018005d7f0     libucrt:log10.obj
 0002:00007800       __real_threshold           000000018005d800     libucrt:log10.obj
 0002:00007810       __real_near_one_lt         000000018005d810     libucrt:log10.obj
 0002:00007820       __real_near_one_gt         000000018005d820     libucrt:log10.obj
 0002:00007830       __real_min_norm            000000018005d830     libucrt:log10.obj
 0002:00007840       __real_notsign             000000018005d840     libucrt:log10.obj
 0002:00007850       __real_ca1                 000000018005d850     libucrt:log10.obj
 0002:00007860       __real_ca2                 000000018005d860     libucrt:log10.obj
 0002:00007870       __real_ca3                 000000018005d870     libucrt:log10.obj
 0002:00007880       __real_ca4                 000000018005d880     libucrt:log10.obj
 0002:00007890       __mask_lower               000000018005d890     libucrt:log10.obj
 0002:000078a0       __flag_x_zero              000000018005d8a0     libucrt:log10.obj
 0002:000078a4       __flag_x_neg               000000018005d8a4     libucrt:log10.obj
 0002:000078a8       __flag_x_nan               000000018005d8a8     libucrt:log10.obj
 0002:00009200       metamethods                000000018005f200     bit64.obj
 0002:000092c0       funcs                      000000018005f2c0     bit64.obj
 0002:0000fe70       colors                     0000000180065e70     keysandcolors.obj
 0002:00010dd0       guids                      0000000180066dd0     keysandcolors.obj
 0002:00012648       LuamacroGuid               0000000180068648     luamacro.obj
 0002:00014e54       ?key@?3??far_Menu@@9@9     000000018006ae54     service.obj
 0002:00015590       ?C@?3??far_InputRecordToName@@9@9 000000018006b590     service.obj
 0002:00015598       ?FarGuid@?1??far_CreateSettings@@9@9 000000018006b598     service.obj
 0002:00015bb0       lualibs_extra              000000018006bbb0     service.obj
 0002:00015c10       lualibs                    000000018006bc10     service.obj
 0002:00015ee0       ?A@?3??far_InputRecordToName@@9@9 000000018006bee0     service.obj
 0002:00015f08       ?S@?3??far_InputRecordToName@@9@9 000000018006bf08     service.obj
 0002:00015ff0       uniclib                    000000018006bff0     slnunico.obj
 0002:000163e0       ?limits@?1??utf8_decode@@9@9 000000018006c3e0     lutf8lib.obj
 0002:000163f8       UTF8PATT                   000000018006c3f8     lutf8lib.obj
 0002:00016640       flib                       000000018006c640     uliolib51.obj
 0002:000166f0       iolib                      000000018006c6f0     uliolib51.obj
 0002:000167b0       ?mode@?1??f_seek@@9@9      000000018006c7b0     uliolib51.obj
 0002:000167c0       ?modenames@?1??f_seek@@9@9 000000018006c7c0     uliolib51.obj
 0002:000167e0       ?modenames@?1??f_setvbuf@@9@9 000000018006c7e0     uliolib51.obj
 0002:00016800       ?mode@?1??f_setvbuf@@9@9   000000018006c800     uliolib51.obj
 0002:00016bd0       pk_funcs                   000000018006cbd0     uloadlib51.obj
 0002:00016c00       sentinel_                  000000018006cc00     uloadlib51.obj
 0002:00016c08       ll_funcs                   000000018006cc08     uloadlib51.obj
 0002:00016c40       loaders                    000000018006cc40     uloadlib51.obj
 0002:00017eb8       $unwind$sprintf            000000018006deb8     bit64.obj
 0002:00017eb8       $unwind$fprintf            000000018006deb8     service.obj
 0002:00017eb8       $unwind$fscanf             000000018006deb8     uliolib51.obj
 0002:00017ec4       $unwind$arshift            000000018006dec4     bit64.obj
 0002:00017ec4       $unwind$bit64_push         000000018006dec4     bit64.obj
 0002:00017ec4       $unwind$bit64_pushuserdata 000000018006dec4     bit64.obj
 0002:00017ec4       $unwind$f_div              000000018006dec4     bit64.obj
 0002:00017ec4       $unwind$f_eq               000000018006dec4     bit64.obj
 0002:00017ec4       $unwind$f_le               000000018006dec4     bit64.obj
 0002:00017ec4       $unwind$f_lt               000000018006dec4     bit64.obj
 0002:00017ec4       $unwind$f_sub              000000018006dec4     bit64.obj
 0002:00017ec4       $unwind$lshift             000000018006dec4     bit64.obj
 0002:00017ec4       $unwind$rshift             000000018006dec4     bit64.obj
 0002:00017ec4       $unwind$GetExportFunction  000000018006dec4     exported.obj
 0002:00017ec4       $unwind$LF_Analyse         000000018006dec4     exported.obj
 0002:00017ec4       $unwind$LF_ClosePanel      000000018006dec4     exported.obj
 0002:00017ec4       $unwind$LF_Compare         000000018006dec4     exported.obj
 0002:00017ec4       $unwind$LF_ExitFAR         000000018006dec4     exported.obj
 0002:00017ec4       $unwind$LF_FreeContentData 000000018006dec4     exported.obj
 0002:00017ec4       $unwind$LF_ProcessEditorInput 000000018006dec4     exported.obj
 0002:00017ec4       $unwind$LF_ProcessPanelInput 000000018006dec4     exported.obj
 0002:00017ec4       $unwind$LF_SetFindList     000000018006dec4     exported.obj
 0002:00017ec4       $unwind$PushPluginPair     000000018006dec4     exported.obj
 0002:00017ec4       $unwind$RegisterObject     000000018006dec4     exported.obj
 0002:00017ec4       $unwind$func_New           000000018006dec4     lregex.obj
 0002:00017ec4       $unwind$method_bracketscount 000000018006dec4     lregex.obj
 0002:00017ec4       $unwind$method_gc          000000018006dec4     lregex.obj
 0002:00017ec4       $unwind$method_tostring    000000018006dec4     lregex.obj
 0002:00017ec4       $unwind$Lutf8_codes        000000018006dec4     lutf8lib.obj
 0002:00017ec4       $unwind$CheckFlagsFromTable 000000018006dec4     service.obj
 0002:00017ec4       $unwind$DialogHandleEqual  000000018006dec4     service.obj
 0002:00017ec4       $unwind$GetFakePluginData  000000018006dec4     service.obj
 0002:00017ec4       $unwind$LF_GetLuafarAPI    000000018006dec4     service.obj
 0002:00017ec4       $unwind$LF_InitLuaState2   000000018006dec4     service.obj
 0002:00017ec4       $unwind$PushFarColor       000000018006dec4     service.obj
 0002:00017ec4       $unwind$Settings_free      000000018006dec4     service.obj
 0002:00017ec4       $unwind$editor_AddSessionBookmark 000000018006dec4     service.obj
 0002:00017ec4       $unwind$editor_ClearSessionBookmarks 000000018006dec4     service.obj
 0002:00017ec4       $unwind$editor_DeleteBlock 000000018006dec4     service.obj
 0002:00017ec4       $unwind$editor_DeleteChar  000000018006dec4     service.obj
 0002:00017ec4       $unwind$editor_DeleteString 000000018006dec4     service.obj
 0002:00017ec4       $unwind$editor_NextSessionBookmark 000000018006dec4     service.obj
 0002:00017ec4       $unwind$editor_PrevSessionBookmark 000000018006dec4     service.obj
 0002:00017ec4       $unwind$editor_Quit        000000018006dec4     service.obj
 0002:00017ec4       $unwind$editor_Redraw      000000018006dec4     service.obj
 0002:00017ec4       $unwind$far_DialogFree     000000018006dec4     service.obj
 0002:00017ec4       $unwind$far_FileTimeResolution 000000018006dec4     service.obj
 0002:00017ec4       $unwind$far_FreeScreen     000000018006dec4     service.obj
 0002:00017ec4       $unwind$far_Show           000000018006dec4     service.obj
 0002:00017ec4       $unwind$far_UnloadPlugin   000000018006dec4     service.obj
 0002:00017ec4       $unwind$filefilter_Free    000000018006dec4     service.obj
 0002:00017ec4       $unwind$filefilter_OpenMenu 000000018006dec4     service.obj
 0002:00017ec4       $unwind$filefilter_Starting 000000018006dec4     service.obj
 0002:00017ec4       $unwind$filefilter_gc      000000018006dec4     service.obj
 0002:00017ec4       $unwind$free_dialog        000000018006dec4     service.obj
 0002:00017ec4       $unwind$panel_BeginSelection 000000018006dec4     service.obj
 0002:00017ec4       $unwind$panel_CheckPanelsExist 000000018006dec4     service.obj
 0002:00017ec4       $unwind$panel_EndSelection 000000018006dec4     service.obj
 0002:00017ec4       $unwind$panel_GetCmdLinePos 000000018006dec4     service.obj
 0002:00017ec4       $unwind$panel_IsActivePanel 000000018006dec4     service.obj
 0002:00017ec4       $unwind$pushFileTime       000000018006dec4     service.obj
 0002:00017ec4       $unwind$viewer_Quit        000000018006dec4     service.obj
 0002:00017ec4       $unwind$viewer_Redraw      000000018006dec4     service.obj
 0002:00017ec4       $unwind$f_read             000000018006dec4     uliolib51.obj
 0002:00017ec4       $unwind$f_write            000000018006dec4     uliolib51.obj
 0002:00017ec4       $unwind$io_read            000000018006dec4     uliolib51.obj
 0002:00017ec4       $unwind$io_tmpfile         000000018006dec4     uliolib51.obj
 0002:00017ec4       $unwind$io_type            000000018006dec4     uliolib51.obj
 0002:00017ec4       $unwind$io_write           000000018006dec4     uliolib51.obj
 0002:00017ec4       $unwind$newfile            000000018006dec4     uliolib51.obj
 0002:00017ec4       $unwind$loader_Lua         000000018006dec4     uloadlib51.obj
 0002:00017ec4       $unwind$loader_preload     000000018006dec4     uloadlib51.obj
 0002:00017ec4       $unwind$mkfuncname         000000018006dec4     uloadlib51.obj
 0002:00017ec4       $unwind$GetBoolFromTable   000000018006dec4     ustring.obj
 0002:00017ec4       $unwind$GetOptBoolFromTable 000000018006dec4     ustring.obj
 0002:00017ec4       $unwind$GetOptIntFromArray 000000018006dec4     ustring.obj
 0002:00017ec4       $unwind$GetOptIntFromTable 000000018006dec4     ustring.obj
 0002:00017ec4       $unwind$PutBoolToTable     000000018006dec4     ustring.obj
 0002:00017ec4       $unwind$PutIntToArray      000000018006dec4     ustring.obj
 0002:00017ec4       $unwind$PutIntToTable      000000018006dec4     ustring.obj
 0002:00017ec4       $unwind$PutLStrToTable     000000018006dec4     ustring.obj
 0002:00017ec4       $unwind$PutNumToTable      000000018006dec4     ustring.obj
 0002:00017ec4       $unwind$PutStrToArray      000000018006dec4     ustring.obj
 0002:00017ec4       $unwind$PutStrToTable      000000018006dec4     ustring.obj
 0002:00017ec4       $unwind$SysErrorReturn     000000018006dec4     ustring.obj
 0002:00017ec4       $unwind$ustring_EnumSystemCodePages 000000018006dec4     ustring.obj
 0002:00017ec4       $unwind$ustring_GetKeyState 000000018006dec4     ustring.obj
 0002:00017ec4       $unwind$win_FileTimeToLocalFileTime 000000018006dec4     win.obj
 0002:00017ec4       $unwind$win_GetSystemTimeAsFileTime 000000018006dec4     win.obj
 0002:00017ec4       $unwind$_RTC_Initialize    000000018006dec4     LIBCMT:initsect.obj
 0002:00017ec4       $unwind$_RTC_Terminate     000000018006dec4     LIBCMT:initsect.obj
 0002:00017ec4       $unwind$__vcrt_FlsSetValue 000000018006dec4     libvcruntime:winapi_downlevel.obj
 0002:00017ec4       $unwind$??$common_initialize_environment_nolock@D@@YAHXZ 000000018006dec4     libucrt:environment_initialization.obj
 0002:00017ec4       $unwind$??$common_initialize_environment_nolock@_W@@YAHXZ 000000018006dec4     libucrt:environment_initialization.obj
 0002:00017ec4       $unwind$__acrt_wgetpath    000000018006dec4     libucrt:getpath.obj
 0002:00017ec4       $unwind$__acrt_fp_strflt_to_string 000000018006dec4     libucrt:_fptostr.obj
 0002:00017ec4       $unwind$_realloc_base      000000018006dec4     libucrt:realloc_base.obj
 0002:00017ec4       $unwind$?replace_current_thread_locale_nolock@@YAXQEAU__acrt_ptd@@QEAU__crt_locale_data@@@Z 000000018006dec4     libucrt:per_thread_data.obj
 0002:00017ec4       $unwind$__acrt_execute_uninitializers 000000018006dec4     libucrt:shared_initialization.obj
 0002:00017ec4       $unwind$__acrt_FlsSetValue 000000018006dec4     libucrt:winapi_thunks.obj
 0002:00017ec4       $unwind$__acrt_LocaleNameToLCID 000000018006dec4     libucrt:winapi_thunks.obj
 0002:00017ec4       $unwind$_updatetlocinfoEx_nolock 000000018006dec4     libucrt:locale_refcounting.obj
 0002:00017ec4       $unwind$_close_nolock      000000018006dec4     libucrt:close.obj
 0002:00017ec4       $unwind$__acrt_uninitialize_lowio 000000018006dec4     libucrt:ioinit.obj
 0002:00017ec4       $unwind$__acrt_errno_map_os_error 000000018006dec4     libucrt:errno.obj
 0002:00017ec4       $unwind$_initterm_e        000000018006dec4     libucrt:initterm.obj
 0002:00017ec4       $unwind$__acrt_stdio_allocate_buffer_nolock 000000018006dec4     libucrt:_getbuf.obj
 0002:00017ec4       $unwind$__acrt_stdio_begin_temporary_buffering_nolock 000000018006dec4     libucrt:_sftbuf.obj
 0002:00017ec4       $unwind$_fclose_nolock     000000018006dec4     libucrt:fclose.obj
 0002:00017ec4       $unwind$?common_fseek_binary_mode_read_only_fast_track_nolock@@YA_NV__crt_stdio_stream@@_JH@Z 000000018006dec4     libucrt:fseek.obj
 0002:00017ec4       $unwind$??R<lambda_156378f40168adef48d7ddfcff3a1264>@@QEBA_NXZ 000000018006dec4     libucrt:input.obj
 0002:00017ec4       $unwind$?process@?$input_processor@DV?$stream_input_adapter@D@__crt_stdio_input@@@__crt_stdio_input@@QEAAHXZ 000000018006dec4     libucrt:input.obj
 0002:00017ec4       $unwind$?process_conversion_specifier@?$input_processor@DV?$stream_input_adapter@D@__crt_stdio_input@@@__crt_stdio_input@@AEAA_NXZ 000000018006dec4     libucrt:input.obj
 0002:00017ec4       $unwind$?process_floating_point_specifier@?$input_processor@DV?$stream_input_adapter@D@__crt_stdio_input@@@__crt_stdio_input@@AEAA_NXZ 000000018006dec4     libucrt:input.obj
 0002:00017ec4       $unwind$?process_literal_character_tchar@?$input_processor@DV?$stream_input_adapter@D@__crt_stdio_input@@@__crt_stdio_input@@AEAA_ND@Z 000000018006dec4     libucrt:input.obj
 0002:00017ec4       $unwind$?process_state@?$input_processor@DV?$stream_input_adapter@D@__crt_stdio_input@@@__crt_stdio_input@@AEAA_NXZ 000000018006dec4     libucrt:input.obj
 0002:00017ec4       $unwind$?write_integer@?$input_processor@DV?$stream_input_adapter@D@__crt_stdio_input@@@__crt_stdio_input@@AEAA_N_K@Z 000000018006dec4     libucrt:input.obj
 0002:00017ec4       $unwind$??$get_tmpfile_buffer_nolock@D@@YAPEADW4buffer_id@?A0x5b9a7937@@@Z 000000018006dec4     libucrt:tmpfile.obj
 0002:00017ec4       $unwind$_ungetc_nolock     000000018006dec4     libucrt:ungetc.obj
 0002:00017ec4       $unwind$strncpy_s          000000018006dec4     libucrt:strncpy_s.obj
 0002:00017ed0       $unwind$bit64_getvalue     000000018006ded0     bit64.obj
 0002:00017ed0       $unwind$LF_ProcessConsoleInput 000000018006ded0     exported.obj
 0002:00017ed0       $unwind$check_regex_pattern 000000018006ded0     lregex.obj
 0002:00017ed0       $unwind$_cwait             000000018006ded0     libucrt:wait.obj
 0002:00017ed0       $unwind$?type_case_c_tchar@?$output_processor@_WV?$string_output_adapter@_W@__crt_stdio_output@@V?$standard_base@_WV?$string_output_adapter@_W@__crt_stdio_output@@@2@@__crt_stdio_output@@AEAA_N_W@Z 000000018006ded0     libucrt:output.obj
 0002:00017ee0       $chain$0$bit64_getvalue    000000018006dee0     bit64.obj
 0002:00017ef4       $chain$1$bit64_getvalue    000000018006def4     bit64.obj
 0002:00017f04       $unwind$check64            000000018006df04     bit64.obj
 0002:00017f04       $unwind$AddMacroData_gc    000000018006df04     service.obj
 0002:00017f04       $unwind$far_MacroDelete    000000018006df04     service.obj
 0002:00017f04       $unwind$_free_osfhnd       000000018006df04     libucrt:osfinfo.obj
 0002:00017f04       $unwind$__acrt_stdio_refill_and_read_narrow_nolock 000000018006df04     libucrt:_filbuf.obj
 0002:00017f18       $unwind$band               000000018006df18     bit64.obj
 0002:00017f18       $unwind$bor                000000018006df18     bit64.obj
 0002:00017f18       $unwind$bxor               000000018006df18     bit64.obj
 0002:00017f18       $unwind$f_add              000000018006df18     bit64.obj
 0002:00017f18       $unwind$f_mul              000000018006df18     bit64.obj
 0002:00017f18       $unwind$PackMacroValues    000000018006df18     exported.obj
 0002:00017f18       $unwind$push_far_regex     000000018006df18     lregex.obj
 0002:00017f18       $unwind$InitMPR            000000018006df18     luamacro.obj
 0002:00017f18       $unwind$uc_New             000000018006df18     lusercontrol.obj
 0002:00017f18       $unwind$classend           000000018006df18     lutf8lib.obj
 0002:00017f18       $unwind$push_offset        000000018006df18     lutf8lib.obj
 0002:00017f18       $unwind$OptInputRecord     000000018006df18     service.obj
 0002:00017f18       $unwind$PutVersionInfoToTable 000000018006df18     service.obj
 0002:00017f18       $unwind$far_CreateFileFilter 000000018006df18     service.obj
 0002:00017f18       $unwind$timer_index        000000018006df18     service.obj
 0002:00017f18       $unwind$f_seek             000000018006df18     uliolib51.obj
 0002:00017f18       $unwind$__scrt_dllmain_exception_filter 000000018006df18     LIBCMT:utility.obj
 0002:00017f18       $unwind$__dcrt_get_wide_environment_from_os 000000018006df18     libucrt:get_environment_from_os.obj
 0002:00017f18       $unwind$??$common_getenv_nolock@_W@@YAPEA_WQEB_W@Z 000000018006df18     libucrt:getenv.obj
 0002:00017f18       $unwind$_ischartype_l      000000018006df18     libucrt:_ctype.obj
 0002:00017f18       $unwind$_recalloc_base     000000018006df18     libucrt:recalloc.obj
 0002:00017f18       $unwind$__acrt_free_locale 000000018006df18     libucrt:locale_refcounting.obj
 0002:00017f18       $unwind$__acrt_lowio_create_handle_array 000000018006df18     libucrt:osfinfo.obj
 0002:00017f18       $unwind$?setSBCS@@YAXPEAU__crt_multibyte_data@@@Z 000000018006df18     libucrt:mbctype.obj
 0002:00017f18       $unwind$_seh_filter_exe    000000018006df18     libucrt:exception_filter.obj
 0002:00017f18       $unwind$_initterm          000000018006df18     libucrt:initterm.obj
 0002:00017f18       $unwind$?scan_scanset_range@?$format_string_parser@D@__crt_stdio_input@@AEAA_NXZ 000000018006df18     libucrt:input.obj
 0002:00017f18       $unwind$??$ensure_buffer_is_big_enough@D@formatting_buffer@__crt_stdio_output@@QEAA_N_K@Z 000000018006df18     libucrt:output.obj
 0002:00017f18       $unwind$??$ensure_buffer_is_big_enough@_W@formatting_buffer@__crt_stdio_output@@QEAA_N_K@Z 000000018006df18     libucrt:output.obj
 0002:00017f18       $unwind$?find_or_allocate_unused_stream_nolock@@YA?AV__crt_stdio_stream@@XZ 000000018006df18     libucrt:stream.obj
 0002:00017f2c       $unwind$bnot               000000018006df2c     bit64.obj
 0002:00017f2c       $unwind$f_tonumber         000000018006df2c     bit64.obj
 0002:00017f2c       $unwind$f_unm              000000018006df2c     bit64.obj
 0002:00017f2c       $unwind$luaopen_bit64      000000018006df2c     bit64.obj
 0002:00017f2c       $unwind$FarPanelItemFreeCallback 000000018006df2c     exported.obj
 0002:00017f2c       $unwind$PushPluginObject   000000018006df2c     exported.obj
 0002:00017f2c       $unwind$traceback          000000018006df2c     exported.obj
 0002:00017f2c       $unwind$luaopen_regex      000000018006df2c     lregex.obj
 0002:00017f2c       $unwind$luaopen_usercontrol 000000018006df2c     lusercontrol.obj
 0002:00017f2c       $unwind$uc_len             000000018006df2c     lusercontrol.obj
 0002:00017f2c       $unwind$uc_tostring        000000018006df2c     lusercontrol.obj
 0002:00017f2c       $unwind$Lutf8_gmatch       000000018006df2c     lutf8lib.obj
 0002:00017f2c       $unwind$push_onecapture    000000018006df2c     lutf8lib.obj
 0002:00017f2c       $unwind$OptHandle          000000018006df2c     service.obj
 0002:00017f2c       $unwind$PluginHandle_rawhandle 000000018006df2c     service.obj
 0002:00017f2c       $unwind$Settings_tostring  000000018006df2c     service.obj
 0002:00017f2c       $unwind$TimerCallback      000000018006df2c     service.obj
 0002:00017f2c       $unwind$dialog_rawhandle   000000018006df2c     service.obj
 0002:00017f2c       $unwind$dialog_tostring    000000018006df2c     service.obj
 0002:00017f2c       $unwind$editor_GetFileName 000000018006df2c     service.obj
 0002:00017f2c       $unwind$far_CPluginStartupInfo 000000018006df2c     service.obj
 0002:00017f2c       $unwind$far_FarClock       000000018006df2c     service.obj
 0002:00017f2c       $unwind$far_FreeSettings   000000018006df2c     service.obj
 0002:00017f2c       $unwind$far_GetLuafarVersion 000000018006df2c     service.obj
 0002:00017f2c       $unwind$far_MacroGetArea   000000018006df2c     service.obj
 0002:00017f2c       $unwind$far_MacroGetState  000000018006df2c     service.obj
 0002:00017f2c       $unwind$far_MacroSaveAll   000000018006df2c     service.obj
 0002:00017f2c       $unwind$far_RunDefaultScript 000000018006df2c     service.obj
 0002:00017f2c       $unwind$filefilter_tostring 000000018006df2c     service.obj
 0002:00017f2c       $unwind$timer_tostring     000000018006df2c     service.obj
 0002:00017f2c       $unwind$viewer_GetFileName 000000018006df2c     service.obj
 0002:00017f2c       $unwind$aux_close          000000018006df2c     uliolib51.obj
 0002:00017f2c       $unwind$f_lines            000000018006df2c     uliolib51.obj
 0002:00017f2c       $unwind$io_close           000000018006df2c     uliolib51.obj
 0002:00017f2c       $unwind$io_gc              000000018006df2c     uliolib51.obj
 0002:00017f2c       $unwind$io_noclose         000000018006df2c     uliolib51.obj
 0002:00017f2c       $unwind$io_tostring        000000018006df2c     uliolib51.obj
 0002:00017f2c       $unwind$gctm               000000018006df2c     uloadlib51.obj
 0002:00017f2c       $unwind$ll_seeall          000000018006df2c     uloadlib51.obj
 0002:00017f2c       $unwind$check_utf16_string 000000018006df2c     ustring.obj
 0002:00017f2c       $unwind$luaopen_ustring    000000018006df2c     ustring.obj
 0002:00017f2c       $unwind$ustring_GetACP     000000018006df2c     ustring.obj
 0002:00017f2c       $unwind$ustring_GetConsoleCP 000000018006df2c     ustring.obj
 0002:00017f2c       $unwind$ustring_GetConsoleOutputCP 000000018006df2c     ustring.obj
 0002:00017f2c       $unwind$ustring_GetOEMCP   000000018006df2c     ustring.obj
 0002:00017f2c       $unwind$ustring_len        000000018006df2c     ustring.obj
 0002:00017f2c       $unwind$CheckHKey          000000018006df2c     win.obj
 0002:00017f2c       $unwind$luaopen_win        000000018006df2c     win.obj
 0002:00017f2c       $unwind$__raise_securityfailure 000000018006df2c     LIBCMT:gs_report.obj
 0002:00017f2c       $unwind$__scrt_initialize_crt 000000018006df2c     LIBCMT:utility.obj
 0002:00017f2c       $unwind$__scrt_initialize_onexit_tables 000000018006df2c     LIBCMT:utility.obj
 0002:00017f2c       $unwind$__scrt_release_startup_lock 000000018006df2c     LIBCMT:utility.obj
 0002:00017f2c       $unwind$__scrt_uninitialize_crt 000000018006df2c     LIBCMT:utility.obj
 0002:00017f2c       $unwind$__vcrt_uninitialize_locks 000000018006df2c     libvcruntime:locks.obj
 0002:00017f2c       $unwind$__vcrt_freeptd     000000018006df2c     libvcruntime:per_thread_data.obj
 0002:00017f2c       $unwind$__std_type_info_destroy_list 000000018006df2c     libvcruntime:std_type_info.obj
 0002:00017f2c       $unwind$__vcrt_FlsAlloc    000000018006df2c     libvcruntime:winapi_downlevel.obj
 0002:00017f2c       $unwind$__vcrt_FlsFree     000000018006df2c     libvcruntime:winapi_downlevel.obj
 0002:00017f2c       $unwind$__vcrt_FlsGetValue 000000018006df2c     libvcruntime:winapi_downlevel.obj
 0002:00017f2c       $unwind$?idtab@@YAPEAUprocess_handle_pair@?A0xe43b7539@@QEAU_iobuf@@@Z 000000018006df2c     libucrt:popen.obj
 0002:00017f2c       $unwind$_calloc_base       000000018006df2c     libucrt:calloc_base.obj
 0002:00017f2c       $unwind$_malloc_base       000000018006df2c     libucrt:malloc_base.obj
 0002:00017f2c       $unwind$_callnewh          000000018006df2c     libucrt:new_handler.obj
 0002:00017f2c       $unwind$initialize_pointers 000000018006df2c     libucrt:initialization.obj
 0002:00017f2c       $unwind$uninitialize_allocated_memory 000000018006df2c     libucrt:initialization.obj
 0002:00017f2c       $unwind$__acrt_initialize_locks 000000018006df2c     libucrt:locks.obj
 0002:00017f2c       $unwind$__acrt_uninitialize_locks 000000018006df2c     libucrt:locks.obj
 0002:00017f2c       $unwind$__acrt_freeptd     000000018006df2c     libucrt:per_thread_data.obj
 0002:00017f2c       $unwind$__acrt_getptd_head 000000018006df2c     libucrt:per_thread_data.obj
 0002:00017f2c       $unwind$__acrt_get_process_end_policy 000000018006df2c     libucrt:win_policies.obj
 0002:00017f2c       $unwind$__acrt_AppPolicyGetProcessTerminationMethodInternal 000000018006df2c     libucrt:winapi_thunks.obj
 0002:00017f2c       $unwind$__acrt_FlsAlloc    000000018006df2c     libucrt:winapi_thunks.obj
 0002:00017f2c       $unwind$__acrt_FlsFree     000000018006df2c     libucrt:winapi_thunks.obj
 0002:00017f2c       $unwind$__acrt_FlsGetValue 000000018006df2c     libucrt:winapi_thunks.obj
 0002:00017f2c       $unwind$__acrt_uninitialize_winapi_thunks 000000018006df2c     libucrt:winapi_thunks.obj
 0002:00017f2c       $unwind$__acrt_update_locale_info 000000018006df2c     libucrt:locale_update.obj
 0002:00017f2c       $unwind$__acrt_update_multibyte_info 000000018006df2c     libucrt:locale_update.obj
 0002:00017f2c       $unwind$__acrt_allocate_buffer_for_argv 000000018006df2c     libucrt:argv_parsing.obj
 0002:00017f2c       $unwind$?exit_or_terminate_process@@YAXI@Z 000000018006df2c     libucrt:exit.obj
 0002:00017f2c       $unwind$?try_cor_exit_process@@YAXI@Z 000000018006df2c     libucrt:exit.obj
 0002:00017f2c       $unwind$__acrt_uninitialize_stdio 000000018006df2c     libucrt:_file.obj
 0002:00017f2c       $unwind$?stream_is_at_end_of_file_nolock@@YA_NV__crt_stdio_stream@@@Z 000000018006df2c     libucrt:_flsbuf.obj
 0002:00017f2c       $unwind$__acrt_stdio_free_buffer_nolock 000000018006df2c     libucrt:_freebuf.obj
 0002:00017f2c       $unwind$_fflush_nolock     000000018006df2c     libucrt:fflush.obj
 0002:00017f2c       $unwind$?scan_optional_field_width@?$format_string_parser@D@__crt_stdio_input@@AEAA_NXZ 000000018006df2c     libucrt:input.obj
 0002:00017f2c       $unwind$?state_case_normal@?$output_processor@DV?$stream_output_adapter@D@__crt_stdio_output@@V?$standard_base@DV?$stream_output_adapter@D@__crt_stdio_output@@@2@@__crt_stdio_output@@AEAA_NXZ 000000018006df2c     libucrt:output.obj
 0002:00017f2c       $unwind$?state_case_normal@?$output_processor@DV?$string_output_adapter@D@__crt_stdio_output@@V?$standard_base@DV?$string_output_adapter@D@__crt_stdio_output@@@2@@__crt_stdio_output@@AEAA_NXZ 000000018006df2c     libucrt:output.obj
 0002:00017f2c       $unwind$?state_case_normal_tchar@?$output_processor@DV?$stream_output_adapter@D@__crt_stdio_output@@V?$standard_base@DV?$stream_output_adapter@D@__crt_stdio_output@@@2@@__crt_stdio_output@@AEAA_ND@Z 000000018006df2c     libucrt:output.obj
 0002:00017f2c       $unwind$?type_case_c_tchar@?$output_processor@DV?$stream_output_adapter@D@__crt_stdio_output@@V?$standard_base@DV?$stream_output_adapter@D@__crt_stdio_output@@@2@@__crt_stdio_output@@AEAA_ND@Z 000000018006df2c     libucrt:output.obj
 0002:00017f2c       $unwind$?type_case_c_tchar@?$output_processor@DV?$string_output_adapter@D@__crt_stdio_output@@V?$standard_base@DV?$string_output_adapter@D@__crt_stdio_output@@@2@@__crt_stdio_output@@AEAA_ND@Z 000000018006df2c     libucrt:output.obj
 0002:00017f2c       $unwind$?type_case_s@?$output_processor@DV?$stream_output_adapter@D@__crt_stdio_output@@V?$standard_base@DV?$stream_output_adapter@D@__crt_stdio_output@@@2@@__crt_stdio_output@@AEAA_NXZ 000000018006df2c     libucrt:output.obj
 0002:00017f2c       $unwind$?type_case_s@?$output_processor@DV?$string_output_adapter@D@__crt_stdio_output@@V?$standard_base@DV?$string_output_adapter@D@__crt_stdio_output@@@2@@__crt_stdio_output@@AEAA_NXZ 000000018006df2c     libucrt:output.obj
 0002:00017f2c       $unwind$strcpy_s           000000018006df2c     libucrt:strcpy_s.obj
 0002:00017f2c       $unwind$_strupr            000000018006df2c     libucrt:strupr.obj
 0002:00017f2c       $unwind$wcscat_s           000000018006df2c     libucrt:wcscat_s.obj
 0002:00017f2c       $unwind$wcscpy_s           000000018006df2c     libucrt:wcscpy_s.obj
 0002:00017f2c       $unwind$_clrfp             000000018006df2c     libucrt:fpctrl.obj
 0002:00017f2c       $unwind$_set_statfp        000000018006df2c     libucrt:fpctrl.obj
 0002:00017f2c       $unwind$_clearfp           000000018006df2c     libucrt:ieee.obj
 0002:00017f2c       $unwind$fegetenv           000000018006df2c     libucrt:fegetenv.obj
 0002:00017f2c       $unwind$feholdexcept       000000018006df2c     libucrt:feholdexcept.obj
 0002:00017f2c       $unwind$fesetenv           000000018006df2c     libucrt:fesetenv.obj
 0002:00017f34       $unwind$f_new              000000018006df34     bit64.obj
 0002:00017f44       $chain$0$f_new             000000018006df44     bit64.obj
 0002:00017f58       $chain$1$f_new             000000018006df58     bit64.obj
 0002:00017f68       $unwind$f_tostring         000000018006df68     bit64.obj
 0002:00017f68       $unwind$ustring_Uuid       000000018006df68     ustring.obj
 0002:00017f78       $unwind$f_type             000000018006df78     bit64.obj
 0002:00017f78       $unwind$LF_FreeFindData    000000018006df78     exported.obj
 0002:00017f78       $unwind$GetFileTimeFromTable 000000018006df78     util.obj
 0002:00017f80       $chain$0$f_type            000000018006df80     bit64.obj
 0002:00017f94       $chain$1$f_type            000000018006df94     bit64.obj
 0002:00017fa4       $unwind$f_mod              000000018006dfa4     bit64.obj
 0002:00017fa4       $unwind$LF_Configure       000000018006dfa4     exported.obj
 0002:00017fa4       $unwind$LF_DeleteFiles     000000018006dfa4     exported.obj
 0002:00017fa4       $unwind$LF_ProcessViewerEvent 000000018006dfa4     exported.obj
 0002:00017fa4       $unwind$CheckFarUserControlIndex 000000018006dfa4     lusercontrol.obj
 0002:00017fa4       $unwind$match_class        000000018006dfa4     lutf8lib.obj
 0002:00017fa4       $unwind$utf8_safe_decode   000000018006dfa4     lutf8lib.obj
 0002:00017fa4       $unwind$LF_InitLuaState1   000000018006dfa4     service.obj
 0002:00017fa4       $unwind$OptFlags           000000018006dfa4     service.obj
 0002:00017fa4       $unwind$check_env_flag     000000018006dfa4     service.obj
 0002:00017fa4       $unwind$editor_DeleteSessionBookmark 000000018006dfa4     service.obj
 0002:00017fa4       $unwind$far_DialogRun      000000018006dfa4     service.obj
 0002:00017fa4       $unwind$luaopen_luafar3    000000018006dfa4     service.obj
 0002:00017fa4       $unwind$panel_GetUserScreen 000000018006dfa4     service.obj
 0002:00017fa4       $unwind$panel_SetActivePanel 000000018006dfa4     service.obj
 0002:00017fa4       $unwind$panel_SetCmdLinePos 000000018006dfa4     service.obj
 0002:00017fa4       $unwind$panel_SetUserScreen 000000018006dfa4     service.obj
 0002:00017fa4       $unwind$f_flush            000000018006dfa4     uliolib51.obj
 0002:00017fa4       $unwind$f_setvbuf          000000018006dfa4     uliolib51.obj
 0002:00017fa4       $unwind$io_fclose          000000018006dfa4     uliolib51.obj
 0002:00017fa4       $unwind$io_flush           000000018006dfa4     uliolib51.obj
 0002:00017fa4       $unwind$io_pclose          000000018006dfa4     uliolib51.obj
 0002:00017fa4       $unwind$io_readline        000000018006dfa4     uliolib51.obj
 0002:00017fa4       $unwind$luaopen_uio        000000018006dfa4     uliolib51.obj
 0002:00017fa4       $unwind$ll_require         000000018006dfa4     uloadlib51.obj
 0002:00017fa4       $unwind$loader_C           000000018006dfa4     uloadlib51.obj
 0002:00017fa4       $unwind$opt_utf8_string    000000018006dfa4     ustring.obj
 0002:00017fa4       $unwind$_DllMainCRTStartup 000000018006dfa4     LIBCMT:dll_dllmain.obj
 0002:00017fa4       $unwind$__vcrt_getptd_noexit 000000018006dfa4     libvcruntime:per_thread_data.obj
 0002:00017fa4       $unwind$__vcrt_InitializeCriticalSectionEx 000000018006dfa4     libvcruntime:winapi_downlevel.obj
 0002:00017fa4       $unwind$memcpy_s           000000018006dfa4     libucrt:cfout.obj
 0002:00017fa4       $unwind$__acrt_getptd      000000018006dfa4     libucrt:per_thread_data.obj
 0002:00017fa4       $unwind$__acrt_getptd_noexit 000000018006dfa4     libucrt:per_thread_data.obj
 0002:00017fa4       $unwind$__acrt_execute_initializers 000000018006dfa4     libucrt:shared_initialization.obj
 0002:00017fa4       $unwind$__acrt_InitializeCriticalSectionEx 000000018006dfa4     libucrt:winapi_thunks.obj
 0002:00017fa4       $unwind$?free_crt_array_internal@@YAXQEAPEBX_K@Z 000000018006dfa4     libucrt:inittime.obj
 0002:00017fa4       $unwind$??$common_lseek_nolock@_J@@YA_JH_JH@Z 000000018006dfa4     libucrt:lseek.obj
 0002:00017fa4       $unwind$__acrt_stdio_flush_and_write_narrow_nolock 000000018006dfa4     libucrt:_flsbuf.obj
 0002:00017fa4       $unwind$__acrt_stdio_flush_nolock 000000018006dfa4     libucrt:fflush.obj
 0002:00017fa4       $unwind$?common_fseek_nolock@@YAHV__crt_stdio_stream@@_JH@Z 000000018006dfa4     libucrt:fseek.obj
 0002:00017fa4       $unwind$??$common_ftell_nolock@_J@@YA_JV__crt_stdio_stream@@@Z 000000018006dfa4     libucrt:ftell.obj
 0002:00017fa4       $unwind$??R<lambda_5856287d7ecd2be6c9197bb4007c3f6e>@@QEBA_KXZ 000000018006dfa4     libucrt:fwrite.obj
 0002:00017fa4       $unwind$??$skip_whitespace@Vstream_input_adapter@__crt_stdio_input@@D@__crt_stdio_input@@YAHAEAV?$stream_input_adapter@D@0@QEAU__crt_locale_pointers@@@Z 000000018006dfa4     libucrt:input.obj
 0002:00017fa4       $unwind$?advance@?$format_string_parser@D@__crt_stdio_input@@QEAA_NXZ 000000018006dfa4     libucrt:input.obj
 0002:00017fa4       $unwind$?process_string_specifier@?$input_processor@DV?$stream_input_adapter@D@__crt_stdio_input@@@__crt_stdio_input@@AEAA_NW4conversion_mode@2@@Z 000000018006dfa4     libucrt:input.obj
 0002:00017fa4       $unwind$memcpy_s           000000018006dfa4     libucrt:input.obj
 0002:00017fa4       $unwind$??0_LocaleUpdate@@QEAA@QEAU__crt_locale_pointers@@@Z 000000018006dfa4     libucrt:output.obj
 0002:00017fa4       $unwind$?type_case_Z@?$output_processor@_WV?$string_output_adapter@_W@__crt_stdio_output@@V?$standard_base@_WV?$string_output_adapter@_W@__crt_stdio_output@@@2@@__crt_stdio_output@@AEAA_NXZ 000000018006dfa4     libucrt:output.obj
 0002:00017fa4       $unwind$?type_case_n@?$output_processor@DV?$stream_output_adapter@D@__crt_stdio_output@@V?$standard_base@DV?$stream_output_adapter@D@__crt_stdio_output@@@2@@__crt_stdio_output@@AEAA_NXZ 000000018006dfa4     libucrt:output.obj
 0002:00017fa4       $unwind$?type_case_n@?$output_processor@DV?$string_output_adapter@D@__crt_stdio_output@@V?$standard_base@DV?$string_output_adapter@D@__crt_stdio_output@@@2@@__crt_stdio_output@@AEAA_NXZ 000000018006dfa4     libucrt:output.obj
 0002:00017fa4       $unwind$?type_case_n@?$output_processor@_WV?$string_output_adapter@_W@__crt_stdio_output@@V?$standard_base@_WV?$string_output_adapter@_W@__crt_stdio_output@@@2@@__crt_stdio_output@@AEAA_NXZ 000000018006dfa4     libucrt:output.obj
 0002:00017fa4       $unwind$?type_case_s@?$output_processor@_WV?$string_output_adapter@_W@__crt_stdio_output@@V?$standard_base@_WV?$string_output_adapter@_W@__crt_stdio_output@@@2@@__crt_stdio_output@@AEAA_NXZ 000000018006dfa4     libucrt:output.obj
 0002:00017fa4       $unwind$??R<lambda_ca71763b3c0644891230e4f79ea54fa6>@@QEBAHXZ 000000018006dfa4     libucrt:setvbuf.obj
 0002:00017fa4       $unwind$__acrt_stdio_free_tmpfile_name_buffers_nolock 000000018006dfa4     libucrt:tmpfile.obj
 0002:00017fa4       $unwind$_exception_enabled 000000018006dfa4     libucrt:libm_error.obj
 0002:00017fb4       $unwind$pcall_msg          000000018006dfb4     exported.obj
 0002:00017fb4       $unwind$FillInputRecord    000000018006dfb4     service.obj
 0002:00017fc4       $chain$3$pcall_msg         000000018006dfc4     exported.obj
 0002:00017fe4       $chain$4$pcall_msg         000000018006dfe4     exported.obj
 0002:00017ff4       $unwind$LF_GetFiles        000000018006dff4     exported.obj
 0002:00017ff4       $unwind$_AddStringToCollector 000000018006dff4     exported.obj
 0002:00018000       $chain$3$_AddStringToCollector 000000018006e000     exported.obj
 0002:00018020       $chain$4$_AddStringToCollector 000000018006e020     exported.obj
 0002:00018034       $chain$5$_AddStringToCollector 000000018006e034     exported.obj
 0002:00018044       $chain$6$_AddStringToCollector 000000018006e044     exported.obj
 0002:00018054       $unwind$AddBufToCollector  000000018006e054     exported.obj
 0002:00018054       $unwind$start_capture      000000018006e054     lutf8lib.obj
 0002:00018054       $unwind$FillEditorSetPosition 000000018006e054     service.obj
 0002:00018054       $unwind$NewDialogData      000000018006e054     service.obj
 0002:00018054       $unwind$PushPanelItems     000000018006e054     service.obj
 0002:00018054       $unwind$SetPanelBooleanProperty 000000018006e054     service.obj
 0002:00018054       $unwind$SetPanelIntegerProperty 000000018006e054     service.obj
 0002:00018054       $unwind$timer_newindex     000000018006e054     service.obj
 0002:00018054       $unwind$win_GetVirtualKeys 000000018006e054     win.obj
 0002:0001806c       $unwind$CreateStringsArray 000000018006e06c     exported.obj
 0002:0001806c       $unwind$LF_DlgProc         000000018006e06c     service.obj
 0002:00018080       $chain$1$CreateStringsArray 000000018006e080     exported.obj
 0002:00018098       $chain$2$CreateStringsArray 000000018006e098     exported.obj
 0002:000180a8       $unwind$FillPluginPanelItem 000000018006e0a8     exported.obj
 0002:000180b8       $chain$2$FillPluginPanelItem 000000018006e0b8     exported.obj
 0002:000180d4       $chain$3$FillPluginPanelItem 000000018006e0d4     exported.obj
 0002:000180e8       $chain$4$FillPluginPanelItem 000000018006e0e8     exported.obj
 0002:000180f8       $chain$5$FillPluginPanelItem 000000018006e0f8     exported.obj
 0002:0001810c       $chain$6$FillPluginPanelItem 000000018006e10c     exported.obj
 0002:0001811c       $chain$7$FillPluginPanelItem 000000018006e11c     exported.obj
 0002:0001812c       $unwind$LF_GetFindData     000000018006e12c     exported.obj
 0002:00018138       $chain$3$LF_GetFindData    000000018006e138     exported.obj
 0002:00018158       $chain$4$LF_GetFindData    000000018006e158     exported.obj
 0002:0001816c       $chain$5$LF_GetFindData    000000018006e16c     exported.obj
 0002:0001817c       $chain$6$LF_GetFindData    000000018006e17c     exported.obj
 0002:0001818c       $chain$0$LF_FreeFindData   000000018006e18c     exported.obj
 0002:000181a0       $chain$1$LF_FreeFindData   000000018006e1a0     exported.obj
 0002:000181b0       $unwind$UpdateFileSelection 000000018006e1b0     exported.obj
 0002:000181c0       $chain$3$UpdateFileSelection 000000018006e1c0     exported.obj
 0002:000181e0       $chain$4$UpdateFileSelection 000000018006e1e0     exported.obj
 0002:000181f0       $chain$0$LF_GetFiles       000000018006e1f0     exported.obj
 0002:00018204       $chain$1$LF_GetFiles       000000018006e204     exported.obj
 0002:00018218       $chain$3$LF_GetFiles       000000018006e218     exported.obj
 0002:00018230       $chain$4$LF_GetFiles       000000018006e230     exported.obj
 0002:00018240       $chain$5$LF_GetFiles       000000018006e240     exported.obj
 0002:00018250       $chain$7$LF_GetFiles       000000018006e250     exported.obj
 0002:00018264       $chain$8$LF_GetFiles       000000018006e264     exported.obj
 0002:00018274       $unwind$RunDefaultScript   000000018006e274     exported.obj
 0002:00018274       $unwind$_setmbcp_nolock    000000018006e274     libucrt:mbctype.obj
 0002:00018294       $unwind$PushAnalyseInfo    000000018006e294     exported.obj
 0002:00018294       $unwind$uc_newindex        000000018006e294     lusercontrol.obj
 0002:000182a0       $chain$2$PushAnalyseInfo   000000018006e2a0     exported.obj
 0002:000182bc       $chain$3$PushAnalyseInfo   000000018006e2bc     exported.obj
 0002:000182cc       $unwind$LF_GetOpenPanelInfo 000000018006e2cc     exported.obj
 0002:000182d8       $chain$0$LF_GetOpenPanelInfo 000000018006e2d8     exported.obj
 0002:000182ec       $chain$2$LF_GetOpenPanelInfo 000000018006e2ec     exported.obj
 0002:00018300       $chain$3$LF_GetOpenPanelInfo 000000018006e300     exported.obj
 0002:00018314       $chain$7$LF_GetOpenPanelInfo 000000018006e314     exported.obj
 0002:00018334       $chain$8$LF_GetOpenPanelInfo 000000018006e334     exported.obj
 0002:00018348       $chain$9$LF_GetOpenPanelInfo 000000018006e348     exported.obj
 0002:00018358       $chain$10$LF_GetOpenPanelInfo 000000018006e358     exported.obj
 0002:0001836c       $chain$11$LF_GetOpenPanelInfo 000000018006e36c     exported.obj
 0002:0001837c       $chain$12$LF_GetOpenPanelInfo 000000018006e37c     exported.obj
 0002:0001838c       $unwind$PushFarMacroValue  000000018006e38c     exported.obj
 0002:0001838c       $unwind$capture_current_context 000000018006e38c     LIBCMT:gs_report.obj
 0002:00018398       $chain$0$PushFarMacroValue 000000018006e398     exported.obj
 0002:000183ac       $chain$4$PushFarMacroValue 000000018006e3ac     exported.obj
 0002:000183c8       $chain$5$PushFarMacroValue 000000018006e3c8     exported.obj
 0002:000183d8       $unwind$FillFarMacroCall_Callback 000000018006e3d8     exported.obj
 0002:000183e4       $chain$0$FillFarMacroCall_Callback 000000018006e3e4     exported.obj
 0002:000183f8       $chain$1$FillFarMacroCall_Callback 000000018006e3f8     exported.obj
 0002:00018408       $unwind$FillFarMacroCall   000000018006e408     exported.obj
 0002:00018418       $chain$3$FillFarMacroCall  000000018006e418     exported.obj
 0002:00018438       $chain$4$FillFarMacroCall  000000018006e438     exported.obj
 0002:00018448       $unwind$LF_Open            000000018006e448     exported.obj
 0002:0001845c       $chain$1$LF_Open           000000018006e45c     exported.obj
 0002:00018470       $chain$2$LF_Open           000000018006e470     exported.obj
 0002:00018484       $chain$3$LF_Open           000000018006e484     exported.obj
 0002:00018494       $chain$4$LF_Open           000000018006e494     exported.obj
 0002:000184a4       $unwind$LF_MakeDirectory   000000018006e4a4     exported.obj
 0002:000184a4       $unwind$timer_Close        000000018006e4a4     service.obj
 0002:000184a4       $unwind$timer_gc           000000018006e4a4     service.obj
 0002:000184a4       $unwind$iswctype           000000018006e4a4     libucrt:iswctype.obj
 0002:000184b0       $chain$0$LF_MakeDirectory  000000018006e4b0     exported.obj
 0002:000184c4       $chain$1$LF_MakeDirectory  000000018006e4c4     exported.obj
 0002:000184d4       $unwind$LF_ProcessPanelEvent 000000018006e4d4     exported.obj
 0002:000184e4       $chain$0$LF_ProcessPanelEvent 000000018006e4e4     exported.obj
 0002:000184f8       $chain$1$LF_ProcessPanelEvent 000000018006e4f8     exported.obj
 0002:0001850c       $chain$2$LF_ProcessPanelEvent 000000018006e50c     exported.obj
 0002:0001851c       $chain$3$LF_ProcessPanelEvent 000000018006e51c     exported.obj
 0002:0001852c       $unwind$LF_ProcessHostFile 000000018006e52c     exported.obj
 0002:00018538       $chain$0$LF_ProcessHostFile 000000018006e538     exported.obj
 0002:0001854c       $chain$1$LF_ProcessHostFile 000000018006e54c     exported.obj
 0002:0001855c       $unwind$LF_ProcessEditorEvent 000000018006e55c     exported.obj
 0002:0001855c       $unwind$LF_ProcessSynchroEvent 000000018006e55c     exported.obj
 0002:0001855c       $unwind$LF_PutFiles        000000018006e55c     exported.obj
 0002:0001855c       $unwind$LF_SetDirectory    000000018006e55c     exported.obj
 0002:0001855c       $unwind$ustring_GetLogicalDriveStrings 000000018006e55c     ustring.obj
 0002:0001855c       $unwind$capture_previous_context 000000018006e55c     LIBCMT:gs_report.obj
 0002:00018568       $chain$0$LF_PutFiles       000000018006e568     exported.obj
 0002:0001857c       $chain$2$LF_PutFiles       000000018006e57c     exported.obj
 0002:00018594       $chain$3$LF_PutFiles       000000018006e594     exported.obj
 0002:000185a4       $chain$4$LF_PutFiles       000000018006e5a4     exported.obj
 0002:000185b4       $chain$0$LF_SetDirectory   000000018006e5b4     exported.obj
 0002:000185c8       $chain$2$LF_SetDirectory   000000018006e5c8     exported.obj
 0002:000185e0       $chain$3$LF_SetDirectory   000000018006e5e0     exported.obj
 0002:000185f0       $chain$4$LF_SetDirectory   000000018006e5f0     exported.obj
 0002:00018600       $unwind$getPluginMenuItems 000000018006e600     exported.obj
 0002:00018618       $unwind$LF_GetPluginInfo   000000018006e618     exported.obj
 0002:00018624       $chain$1$LF_GetPluginInfo  000000018006e624     exported.obj
 0002:0001863c       $chain$2$LF_GetPluginInfo  000000018006e63c     exported.obj
 0002:0001864c       $chain$0$LF_ProcessEditorEvent 000000018006e64c     exported.obj
 0002:00018660       $chain$2$LF_ProcessEditorEvent 000000018006e660     exported.obj
 0002:00018678       $chain$3$LF_ProcessEditorEvent 000000018006e678     exported.obj
 0002:00018688       $chain$4$LF_ProcessEditorEvent 000000018006e688     exported.obj
 0002:00018698       $unwind$LF_ProcessDialogEvent 000000018006e698     exported.obj
 0002:000186ac       $chain$0$LF_ProcessDialogEvent 000000018006e6ac     exported.obj
 0002:000186c0       $chain$1$LF_ProcessDialogEvent 000000018006e6c0     exported.obj
 0002:000186d0       $chain$1$LF_ProcessSynchroEvent 000000018006e6d0     exported.obj
 0002:000186e8       $chain$2$LF_ProcessSynchroEvent 000000018006e6e8     exported.obj
 0002:000186fc       $chain$3$LF_ProcessSynchroEvent 000000018006e6fc     exported.obj
 0002:0001870c       $chain$5$LF_ProcessSynchroEvent 000000018006e70c     exported.obj
 0002:00018720       $chain$6$LF_ProcessSynchroEvent 000000018006e720     exported.obj
 0002:00018730       $unwind$LF_GetContentFields 000000018006e730     exported.obj
 0002:00018740       $chain$0$LF_GetContentFields 000000018006e740     exported.obj
 0002:00018754       $chain$3$LF_GetContentFields 000000018006e754     exported.obj
 0002:00018770       $chain$4$LF_GetContentFields 000000018006e770     exported.obj
 0002:00018780       $chain$5$LF_GetContentFields 000000018006e780     exported.obj
 0002:00018790       $unwind$LF_GetContentData  000000018006e790     exported.obj
 0002:000187ac       $unwind$LF_GetGlobalInfo   000000018006e7ac     exported.obj
 0002:000187c0       $chain$2$LF_GetGlobalInfo  000000018006e7c0     exported.obj
 0002:000187d8       $chain$3$LF_GetGlobalInfo  000000018006e7d8     exported.obj
 0002:000187ec       $chain$4$LF_GetGlobalInfo  000000018006e7ec     exported.obj
 0002:000187fc       $chain$0$LF_ProcessConsoleInput 000000018006e7fc     exported.obj
 0002:00018810       $chain$1$LF_ProcessConsoleInput 000000018006e810     exported.obj
 0002:00018820       $unwind$getF               000000018006e820     lflua.obj
 0002:00018830       $unwind$errfile            000000018006e830     lflua.obj
 0002:00018830       $unwind$far_GetDlgItem     000000018006e830     service.obj
 0002:00018830       $unwind$far_SetDlgItem     000000018006e830     service.obj
 0002:00018830       $unwind$??$common_lseek_nolock@J@@YAJHJH@Z 000000018006e830     libucrt:lseek.obj
 0002:00018830       $unwind$_invalid_parameter 000000018006e830     libucrt:invalid_parameter.obj
 0002:00018830       $unwind$_wcsdup            000000018006e830     libucrt:wcsdup.obj
 0002:00018844       $unwind$LF_LoadFile        000000018006e844     lflua.obj
 0002:00018864       $unwind$luaB_loadfileW     000000018006e864     lflua.obj
 0002:00018864       $unwind$io_lines           000000018006e864     uliolib51.obj
 0002:00018864       $unwind$ustring_OutputDebugString 000000018006e864     ustring.obj
 0002:0001886c       $chain$0$luaB_loadfileW    000000018006e86c     lflua.obj
 0002:00018880       $chain$2$luaB_loadfileW    000000018006e880     lflua.obj
 0002:00018898       $chain$3$luaB_loadfileW    000000018006e898     lflua.obj
 0002:000188ac       $chain$4$luaB_loadfileW    000000018006e8ac     lflua.obj
 0002:000188bc       $chain$5$luaB_loadfileW    000000018006e8bc     lflua.obj
 0002:000188cc       $chain$6$luaB_loadfileW    000000018006e8cc     lflua.obj
 0002:000188dc       $unwind$luaB_dofileW       000000018006e8dc     lflua.obj
 0002:000188dc       $unwind$ustring_GetFileAttr 000000018006e8dc     ustring.obj
 0002:000188dc       $unwind$ustring_SetCurrentDir 000000018006e8dc     ustring.obj
 0002:000188dc       $unwind$ustring_SetFileAttr 000000018006e8dc     ustring.obj
 0002:000188dc       $unwind$win_DeleteFile     000000018006e8dc     win.obj
 0002:000188dc       $unwind$win_RemoveDir      000000018006e8dc     win.obj
 0002:000188e8       $chain$0$luaB_dofileW      000000018006e8e8     lflua.obj
 0002:000188fc       $chain$2$luaB_dofileW      000000018006e8fc     lflua.obj
 0002:00018914       $chain$3$luaB_dofileW      000000018006e914     lflua.obj
 0002:00018924       $chain$4$luaB_dofileW      000000018006e924     lflua.obj
 0002:00018934       $unwind$LF_Gsub            000000018006e934     lflua.obj
 0002:00018954       $chain$0$check_regex_pattern 000000018006e954     lregex.obj
 0002:00018968       $chain$1$check_regex_pattern 000000018006e968     lregex.obj
 0002:00018978       $unwind$_regex_gmatch_closure 000000018006e978     lregex.obj
 0002:00018988       $chain$2$_regex_gmatch_closure 000000018006e988     lregex.obj
 0002:000189a4       $chain$3$_regex_gmatch_closure 000000018006e9a4     lregex.obj
 0002:000189b4       $unwind$_Gmatch            000000018006e9b4     lregex.obj
 0002:000189b4       $unwind$plugin_load        000000018006e9b4     service.obj
 0002:000189d0       $unwind$rx_find_match      000000018006e9d0     lregex.obj
 0002:000189ec       $unwind$rx_gsub            000000018006e9ec     lregex.obj
 0002:00018a14       $unwind$method_matchW      000000018006ea14     lregex.obj
 0002:00018a28       $unwind$func_matchW        000000018006ea28     lregex.obj
 0002:00018a3c       $unwind$FL_PushParams      000000018006ea3c     luamacro.obj
 0002:00018a48       $chain$0$FL_PushParams     000000018006ea48     luamacro.obj
 0002:00018a5c       $chain$1$FL_PushParams     000000018006ea5c     luamacro.obj
 0002:00018a70       $chain$5$FL_PushParams     000000018006ea70     luamacro.obj
 0002:00018a90       $chain$6$FL_PushParams     000000018006ea90     luamacro.obj
 0002:00018aa0       $chain$7$FL_PushParams     000000018006eaa0     luamacro.obj
 0002:00018ab0       $chain$8$FL_PushParams     000000018006eab0     luamacro.obj
 0002:00018ac0       $unwind$Open_Luamacro      000000018006eac0     luamacro.obj
 0002:00018ad4       $chain$1$Open_Luamacro     000000018006ead4     luamacro.obj
 0002:00018aec       $chain$2$Open_Luamacro     000000018006eaec     luamacro.obj
 0002:00018afc       $unwind$far_MacroCallFar   000000018006eafc     luamacro.obj
 0002:00018b14       $chain$1$far_MacroCallFar  000000018006eb14     luamacro.obj
 0002:00018b2c       $chain$3$far_MacroCallFar  000000018006eb2c     luamacro.obj
 0002:00018b44       $chain$4$far_MacroCallFar  000000018006eb44     luamacro.obj
 0002:00018b54       $chain$5$far_MacroCallFar  000000018006eb54     luamacro.obj
 0002:00018b64       $unwind$far_FarMacroCallToLua 000000018006eb64     luamacro.obj
 0002:00018b64       $unwind$far_CopyToClipboard 000000018006eb64     service.obj
 0002:00018b64       $unwind$__dcrt_lowio_ensure_console_output_initialized 000000018006eb64     libucrt:initcon.obj
 0002:00018b64       $unwind$_isleadbyte_l      000000018006eb64     libucrt:_wctype.obj
 0002:00018b64       $unwind$?getSystemCP@@YAHH@Z 000000018006eb64     libucrt:mbctype.obj
 0002:00018b6c       $chain$0$far_FarMacroCallToLua 000000018006eb6c     luamacro.obj
 0002:00018b80       $chain$1$far_FarMacroCallToLua 000000018006eb80     luamacro.obj
 0002:00018b90       $unwind$uc_index           000000018006eb90     lusercontrol.obj
 0002:00018ba8       $chain$3$uc_index          000000018006eba8     lusercontrol.obj
 0002:00018bbc       $chain$4$uc_index          000000018006ebbc     lusercontrol.obj
 0002:00018bcc       $chain$3$uc_newindex       000000018006ebcc     lusercontrol.obj
 0002:00018bec       $chain$4$uc_newindex       000000018006ebec     lusercontrol.obj
 0002:00018c00       $chain$5$uc_newindex       000000018006ec00     lusercontrol.obj
 0002:00018c10       $chain$6$uc_newindex       000000018006ec10     lusercontrol.obj
 0002:00018c20       $unwind$CreateRegKey       000000018006ec20     reg.obj
 0002:00018c28       $unwind$DllMain            000000018006ec28     service.obj
 0002:00018c28       $unwind$GetRealPluginData  000000018006ec28     service.obj
 0002:00018c28       $unwind$far_SubscribeDialogDrawEvents 000000018006ec28     service.obj
 0002:00018c28       $unwind$luaopen_unicode    000000018006ec28     slnunico.obj
 0002:00018c28       $unwind$writer             000000018006ec28     slnunico.obj
 0002:00018c28       $unwind$ustring_Sleep      000000018006ec28     ustring.obj
 0002:00018c28       $unwind$win_IsProcess64bit 000000018006ec28     win.obj
 0002:00018c28       $unwind$__scrt_initialize_default_local_stdio_options 000000018006ec28     LIBCMT:default_local_stdio_options.obj
 0002:00018c28       $unwind$?dllmain_crt_dispatch@@YAHQEAUHINSTANCE__@@KQEAX@Z 000000018006ec28     LIBCMT:dll_dllmain.obj
 0002:00018c28       $unwind$__report_rangecheckfailure 000000018006ec28     LIBCMT:gs_report.obj
 0002:00018c28       $unwind$__GSHandlerCheck   000000018006ec28     LIBCMT:gshandler.obj
 0002:00018c28       $unwind$__scrt_acquire_startup_lock 000000018006ec28     LIBCMT:utility.obj
 0002:00018c28       $unwind$__scrt_dllmain_after_initialize_c 000000018006ec28     LIBCMT:utility.obj
 0002:00018c28       $unwind$__scrt_dllmain_before_initialize_c 000000018006ec28     LIBCMT:utility.obj
 0002:00018c28       $unwind$__scrt_dllmain_crt_thread_attach 000000018006ec28     LIBCMT:utility.obj
 0002:00018c28       $unwind$__scrt_dllmain_crt_thread_detach 000000018006ec28     LIBCMT:utility.obj
 0002:00018c28       $unwind$__scrt_dllmain_uninitialize_c 000000018006ec28     LIBCMT:utility.obj
 0002:00018c28       $unwind$__scrt_dllmain_uninitialize_critical 000000018006ec28     LIBCMT:utility.obj
 0002:00018c28       $unwind$__vcrt_initialize  000000018006ec28     libvcruntime:initialization.obj
 0002:00018c28       $unwind$__vcrt_thread_attach 000000018006ec28     libvcruntime:initialization.obj
 0002:00018c28       $unwind$__vcrt_thread_detach 000000018006ec28     libvcruntime:initialization.obj
 0002:00018c28       $unwind$__vcrt_uninitialize 000000018006ec28     libvcruntime:initialization.obj
 0002:00018c28       $unwind$__vcrt_uninitialize_critical 000000018006ec28     libvcruntime:initialization.obj
 0002:00018c28       $unwind$__vcrt_initialize_locks 000000018006ec28     libvcruntime:locks.obj
 0002:00018c28       $unwind$__vcrt_freefls     000000018006ec28     libvcruntime:per_thread_data.obj
 0002:00018c28       $unwind$__vcrt_getptd      000000018006ec28     libvcruntime:per_thread_data.obj
 0002:00018c28       $unwind$__vcrt_initialize_ptd 000000018006ec28     libvcruntime:per_thread_data.obj
 0002:00018c28       $unwind$__vcrt_uninitialize_ptd 000000018006ec28     libvcruntime:per_thread_data.obj
 0002:00018c28       $unwind$__dcrt_terminate_console_output 000000018006ec28     libucrt:initcon.obj
 0002:00018c28       $unwind$??$uninitialize_environment_internal@D@@YAXAEAPEAPEAD@Z 000000018006ec28     libucrt:environment_initialization.obj
 0002:00018c28       $unwind$??$uninitialize_environment_internal@_W@@YAXAEAPEAPEA_W@Z 000000018006ec28     libucrt:environment_initialization.obj
 0002:00018c28       $unwind$__dcrt_get_or_create_wide_environment_nolock 000000018006ec28     libucrt:environment_initialization.obj
 0002:00018c28       $unwind$__dcrt_uninitialize_environments_nolock 000000018006ec28     libucrt:environment_initialization.obj
 0002:00018c28       $unwind$?__c32rtomb_utf8@__crt_mbstring@@YA_KPEAD_UPEAU_Mbstatet@@@Z 000000018006ec28     libucrt:c32rtomb.obj
 0002:00018c28       $unwind$__acrt_initialize_heap 000000018006ec28     libucrt:heap_handle.obj
 0002:00018c28       $unwind$_msize_base        000000018006ec28     libucrt:msize.obj
 0002:00018c28       $unwind$?initialize_multibyte@@YAHXZ 000000018006ec28     libucrt:multibyte_initializer.obj
 0002:00018c28       $unwind$__acrt_thread_attach 000000018006ec28     libucrt:initialization.obj
 0002:00018c28       $unwind$__acrt_thread_detach 000000018006ec28     libucrt:initialization.obj
 0002:00018c28       $unwind$__acrt_uninitialize 000000018006ec28     libucrt:initialization.obj
 0002:00018c28       $unwind$__acrt_uninitialize_critical 000000018006ec28     libucrt:initialization.obj
 0002:00018c28       $unwind$initialize_c       000000018006ec28     libucrt:initialization.obj
 0002:00018c28       $unwind$uninitialize_allocated_io_buffers 000000018006ec28     libucrt:initialization.obj
 0002:00018c28       $unwind$uninitialize_environment 000000018006ec28     libucrt:initialization.obj
 0002:00018c28       $unwind$__acrt_initialize_ptd 000000018006ec28     libucrt:per_thread_data.obj
 0002:00018c28       $unwind$__acrt_uninitialize_ptd 000000018006ec28     libucrt:per_thread_data.obj
 0002:00018c28       $unwind$__acrt_AreFileApisANSI 000000018006ec28     libucrt:winapi_thunks.obj
 0002:00018c28       $unwind$__pctype_func      000000018006ec28     libucrt:ctype.obj
 0002:00018c28       $unwind$__acrt_release_locale_ref 000000018006ec28     libucrt:locale_refcounting.obj
 0002:00018c28       $unwind$_isatty            000000018006ec28     libucrt:isatty.obj
 0002:00018c28       $unwind$_get_osfhandle     000000018006ec28     libucrt:osfinfo.obj
 0002:00018c28       $unwind$_get_fmode         000000018006ec28     libucrt:setmode.obj
 0002:00018c28       $unwind$__acrt_initialize_multibyte 000000018006ec28     libucrt:mbctype.obj
 0002:00018c28       $unwind$__acrt_update_thread_multibyte_data 000000018006ec28     libucrt:mbctype.obj
 0002:00018c28       $unwind$__doserrno         000000018006ec28     libucrt:errno.obj
 0002:00018c28       $unwind$_errno             000000018006ec28     libucrt:errno.obj
 0002:00018c28       $unwind$_invoke_watson     000000018006ec28     libucrt:invalid_parameter.obj
 0002:00018c28       $unwind$abort              000000018006ec28     libucrt:abort.obj
 0002:00018c28       $unwind$__acrt_initialize_command_line 000000018006ec28     libucrt:argv_data.obj
 0002:00018c28       $unwind$feof               000000018006ec28     libucrt:feoferr.obj
 0002:00018c28       $unwind$ferror             000000018006ec28     libucrt:feoferr.obj
 0002:00018c28       $unwind$_fgetc_nolock      000000018006ec28     libucrt:fgetc.obj
 0002:00018c28       $unwind$_fileno            000000018006ec28     libucrt:fileno.obj
 0002:00018c28       $unwind$?state_case_normal_tchar@?$output_processor@DV?$string_output_adapter@D@__crt_stdio_output@@V?$standard_base@DV?$string_output_adapter@D@__crt_stdio_output@@@2@@__crt_stdio_output@@AEAA_ND@Z 000000018006ec28     libucrt:output.obj
 0002:00018c28       $unwind$?state_case_size@?$output_processor@DV?$stream_output_adapter@D@__crt_stdio_output@@V?$standard_base@DV?$stream_output_adapter@D@__crt_stdio_output@@@2@@__crt_stdio_output@@AEAA_NXZ 000000018006ec28     libucrt:output.obj
 0002:00018c28       $unwind$?state_case_size@?$output_processor@DV?$string_output_adapter@D@__crt_stdio_output@@V?$standard_base@DV?$string_output_adapter@D@__crt_stdio_output@@@2@@__crt_stdio_output@@AEAA_NXZ 000000018006ec28     libucrt:output.obj
 0002:00018c28       $unwind$?state_case_size@?$output_processor@_WV?$string_output_adapter@_W@__crt_stdio_output@@V?$standard_base@_WV?$string_output_adapter@_W@__crt_stdio_output@@@2@@__crt_stdio_output@@AEAA_NXZ 000000018006ec28     libucrt:output.obj
 0002:00018c28       $unwind$?validate_stream_is_ansi_if_required@?$__acrt_stdio_char_traits@D@@SA_NQEAU_iobuf@@@Z 000000018006ec28     libucrt:output.obj
 0002:00018c28       $unwind$__acrt_uninitialize_tmpfile 000000018006ec28     libucrt:rmtmp.obj
 0002:00018c28       $unwind$tmpfile            000000018006ec28     libucrt:tmpfile.obj
 0002:00018c28       $unwind$_stricmp           000000018006ec28     libucrt:stricmp.obj
 0002:00018c28       $unwind$_wcsicmp           000000018006ec28     libucrt:wcsicmp.obj
 0002:00018c28       $unwind$_wcsnicmp          000000018006ec28     libucrt:wcsnicmp.obj
 0002:00018c28       $unwind$_wcsnicoll         000000018006ec28     libucrt:wcsnicol.obj
 0002:00018c28       $unwind$_statfp            000000018006ec28     libucrt:fpctrl.obj
 0002:00018c28       $unwind$fegetround         000000018006ec28     libucrt:fegetround.obj
 0002:00018c28       $unwind$_set_errno_from_matherr 000000018006ec28     libucrt:fpexcept.obj
 0002:00018c30       $chain$0$DllMain           000000018006ec30     service.obj
 0002:00018c44       $chain$1$DllMain           000000018006ec44     service.obj
 0002:00018c54       $unwind$get_env_flag       000000018006ec54     service.obj
 0002:00018c64       $unwind$matchbalance       000000018006ec64     lutf8lib.obj
 0002:00018c64       $unwind$GetFlagCombination 000000018006ec64     service.obj
 0002:00018c64       $unwind$?try_get_function@@YAPEAXW4function_id@?A0x3064ecbf@@QEBDQEBW4module_id@2@2@Z 000000018006ec64     libvcruntime:winapi_downlevel.obj
 0002:00018c64       $unwind$?try_get_function@@YAPEAXW4function_id@?A0x391cf84c@@QEBDQEBW4module_id@2@2@Z 000000018006ec64     libucrt:winapi_thunks.obj
 0002:00018c64       $unwind$??$process_string_specifier_tchar@D@?$input_processor@DV?$stream_input_adapter@D@__crt_stdio_input@@@__crt_stdio_input@@AEAA_NW4conversion_mode@1@D@Z 000000018006ec64     libucrt:input.obj
 0002:00018c80       $unwind$ConvertLuaValue    000000018006ec80     service.obj
 0002:00018c94       $unwind$far_GetFileOwner   000000018006ec94     service.obj
 0002:00018cb8       $unwind$far_GetNumberOfLinks 000000018006ecb8     service.obj
 0002:00018cc8       $chain$0$far_GetNumberOfLinks 000000018006ecc8     service.obj
 0002:00018cdc       $chain$1$far_GetNumberOfLinks 000000018006ecdc     service.obj
 0002:00018cec       $unwind$StoreTempString    000000018006ecec     service.obj
 0002:00018d04       $chain$0$StoreTempString   000000018006ed04     service.obj
 0002:00018d18       $chain$1$StoreTempString   000000018006ed18     service.obj
 0002:00018d28       $unwind$PushPanelItem      000000018006ed28     service.obj
 0002:00018d38       $chain$2$PushPanelItem     000000018006ed38     service.obj
 0002:00018d54       $chain$3$PushPanelItem     000000018006ed54     service.obj
 0002:00018d68       $chain$4$PushPanelItem     000000018006ed68     service.obj
 0002:00018d78       $chain$5$PushPanelItem     000000018006ed78     service.obj
 0002:00018d8c       $unwind$far_PluginStartupInfo 000000018006ed8c     service.obj
 0002:00018d9c       $chain$0$far_PluginStartupInfo 000000018006ed9c     service.obj
 0002:00018db0       $chain$2$far_PluginStartupInfo 000000018006edb0     service.obj
 0002:00018dc8       $chain$3$far_PluginStartupInfo 000000018006edc8     service.obj
 0002:00018dd8       $chain$4$far_PluginStartupInfo 000000018006edd8     service.obj
 0002:00018de8       $unwind$far_GetCurrentDirectory 000000018006ede8     service.obj
 0002:00018de8       $unwind$loaderror          000000018006ede8     uloadlib51.obj
 0002:00018de8       $unwind$?process_integer_specifier@?$input_processor@DV?$stream_input_adapter@D@__crt_stdio_input@@@__crt_stdio_input@@AEAA_NI_N@Z 000000018006ede8     libucrt:input.obj
 0002:00018dfc       $chain$0$far_GetCurrentDirectory 000000018006edfc     service.obj
 0002:00018e10       $chain$1$far_GetCurrentDirectory 000000018006ee10     service.obj
 0002:00018e20       $unwind$push_ev_filename   000000018006ee20     service.obj
 0002:00018e34       $chain$0$push_ev_filename  000000018006ee34     service.obj
 0002:00018e48       $chain$1$push_ev_filename  000000018006ee48     service.obj
 0002:00018e58       $unwind$editor_GetInfo     000000018006ee58     service.obj
 0002:00018e70       $chain$0$editor_GetInfo    000000018006ee70     service.obj
 0002:00018e84       $chain$1$editor_GetInfo    000000018006ee84     service.obj
 0002:00018e94       $unwind$_EditorGetString   000000018006ee94     service.obj
 0002:00018ebc       $unwind$_EditorSetString   000000018006eebc     service.obj
 0002:00018ed0       $chain$0$_EditorSetString  000000018006eed0     service.obj
 0002:00018ee4       $chain$1$_EditorSetString  000000018006eee4     service.obj
 0002:00018ef8       $chain$2$_EditorSetString  000000018006eef8     service.obj
 0002:00018f08       $chain$3$_EditorSetString  000000018006ef08     service.obj
 0002:00018f18       $unwind$editor_ExpandTabs  000000018006ef18     service.obj
 0002:00018f18       $unwind$editor_InsertString 000000018006ef18     service.obj
 0002:00018f18       $unwind$utf8_valid         000000018006ef18     slnunico.obj
 0002:00018f18       $unwind$ustring_sub        000000018006ef18     ustring.obj
 0002:00018f28       $unwind$_EditorInsertText  000000018006ef28     service.obj
 0002:00018f38       $chain$1$_EditorInsertText 000000018006ef38     service.obj
 0002:00018f50       $chain$2$_EditorInsertText 000000018006ef50     service.obj
 0002:00018f60       $unwind$editor_UndoRedo    000000018006ef60     service.obj
 0002:00018f78       $unwind$FillKeyBarTitles   000000018006ef78     service.obj
 0002:00018f88       $chain$1$FillKeyBarTitles  000000018006ef88     service.obj
 0002:00018fa0       $chain$2$FillKeyBarTitles  000000018006efa0     service.obj
 0002:00018fb0       $unwind$PushDlgItemNum     000000018006efb0     service.obj
 0002:00018fb0       $unwind$SetKeyBar          000000018006efb0     service.obj
 0002:00018fb0       $unwind$far_Timer          000000018006efb0     service.obj
 0002:00018fb0       $unwind$ll_loadfunc        000000018006efb0     uloadlib51.obj
 0002:00018fb0       $unwind$??$parse_integer@_KV?$c_string_character_source@D@__crt_strtox@@@__crt_strtox@@YA_KQEAU__crt_locale_pointers@@V?$c_string_character_source@D@0@H_N@Z 000000018006efb0     libucrt:atox.obj
 0002:00018fb0       $unwind$_wcsicmp_l         000000018006efb0     libucrt:wcsicmp.obj
 0002:00018fc8       $unwind$editor_SetParam    000000018006efc8     service.obj
 0002:00018fe0       $chain$1$editor_SetParam   000000018006efe0     service.obj
 0002:00018ff8       $chain$2$editor_SetParam   000000018006eff8     service.obj
 0002:0001900c       $chain$3$editor_SetParam   000000018006f00c     service.obj
 0002:0001901c       $chain$4$editor_SetParam   000000018006f01c     service.obj
 0002:0001902c       $unwind$editor_SetPosition 000000018006f02c     service.obj
 0002:00019044       $unwind$PushBookmarks      000000018006f044     service.obj
 0002:00019044       $unwind$ExtractFileTime    000000018006f044     win.obj
 0002:0001905c       $chain$0$PushBookmarks     000000018006f05c     service.obj
 0002:00019070       $chain$1$PushBookmarks     000000018006f070     service.obj
 0002:00019080       $unwind$editor_SetTitle    000000018006f080     service.obj
 0002:00019080       $unwind$panel_ClosePanel   000000018006f080     service.obj
 0002:00019090       $chain$1$editor_SetTitle   000000018006f090     service.obj
 0002:000190a8       $chain$2$editor_SetTitle   000000018006f0a8     service.obj
 0002:000190bc       $chain$3$editor_SetTitle   000000018006f0bc     service.obj
 0002:000190cc       $chain$4$editor_SetTitle   000000018006f0cc     service.obj
 0002:000190dc       $unwind$PushDNParams       000000018006f0dc     service.obj
 0002:000190dc       $unwind$editor_GetTitle    000000018006f0dc     service.obj
 0002:000190dc       $unwind$panel_GetCmdLine   000000018006f0dc     service.obj
 0002:000190dc       $unwind$luaopen_upackage   000000018006f0dc     uloadlib51.obj
 0002:000190f4       $unwind$FillEditorSelect   000000018006f0f4     service.obj
 0002:00019104       $chain$0$FillEditorSelect  000000018006f104     service.obj
 0002:00019118       $chain$1$FillEditorSelect  000000018006f118     service.obj
 0002:00019128       $unwind$editor_Select      000000018006f128     service.obj
 0002:00019140       $unwind$editor_GetSelection 000000018006f140     service.obj
 0002:00019164       $unwind$_EditorTabConvert  000000018006f164     service.obj
 0002:0001917c       $unwind$GetFarColor        000000018006f17c     service.obj
 0002:0001918c       $chain$2$GetFarColor       000000018006f18c     service.obj
 0002:000191a8       $chain$3$GetFarColor       000000018006f1a8     service.obj
 0002:000191c0       $chain$4$GetFarColor       000000018006f1c0     service.obj
 0002:000191d4       $chain$5$GetFarColor       000000018006f1d4     service.obj
 0002:000191e4       $unwind$editor_AddColor    000000018006f1e4     service.obj
 0002:00019204       $unwind$editor_DelColor    000000018006f204     service.obj
 0002:00019220       $unwind$editor_GetColor    000000018006f220     service.obj
 0002:0001923c       $unwind$editor_SaveFile    000000018006f23c     service.obj
 0002:00019254       $unwind$PushInputRecord    000000018006f254     service.obj
 0002:00019260       $chain$0$PushInputRecord   000000018006f260     service.obj
 0002:00019274       $chain$3$PushInputRecord   000000018006f274     service.obj
 0002:00019290       $chain$4$PushInputRecord   000000018006f290     service.obj
 0002:000192a0       $chain$5$PushInputRecord   000000018006f2a0     service.obj
 0002:000192b0       $unwind$editor_ProcessInput 000000018006f2b0     service.obj
 0002:000192b0       $unwind$editor_ReadInput   000000018006f2b0     service.obj
 0002:000192b0       $unwind$panel_GetCmdLineSelection 000000018006f2b0     service.obj
 0002:000192b0       $unwind$win_FileTimeToSystemTime 000000018006f2b0     win.obj
 0002:000192c4       $chain$0$FillInputRecord   000000018006f2c4     service.obj
 0002:000192d8       $chain$2$FillInputRecord   000000018006f2d8     service.obj
 0002:000192f0       $chain$3$FillInputRecord   000000018006f2f0     service.obj
 0002:00019300       $chain$4$FillInputRecord   000000018006f300     service.obj
 0002:00019310       $unwind$editor_SubscribeChangeEvent 000000018006f310     service.obj
 0002:00019310       $unwind$panel_SetCmdLineSelection 000000018006f310     service.obj
 0002:00019310       $unwind$viewer_Select      000000018006f310     service.obj
 0002:00019310       $unwind$win_SystemTimeToFileTime 000000018006f310     win.obj
 0002:00019328       $unwind$far_Menu           000000018006f328     service.obj
 0002:00019348       $chain$1$far_Menu          000000018006f348     service.obj
 0002:00019360       $chain$2$far_Menu          000000018006f360     service.obj
 0002:00019370       $unwind$LF_Message         000000018006f370     service.obj
 0002:00019394       $unwind$LF_Error           000000018006f394     service.obj
 0002:000193ac       $chain$0$LF_Error          000000018006f3ac     service.obj
 0002:000193c0       $chain$1$LF_Error          000000018006f3c0     service.obj
 0002:000193d0       $unwind$far_Message        000000018006f3d0     service.obj
 0002:000193e8       $chain$1$panel_ClosePanel  000000018006f3e8     service.obj
 0002:00019400       $chain$2$panel_ClosePanel  000000018006f400     service.obj
 0002:00019414       $chain$3$panel_ClosePanel  000000018006f414     service.obj
 0002:00019424       $chain$4$panel_ClosePanel  000000018006f424     service.obj
 0002:00019434       $unwind$panel_GetPanelInfo 000000018006f434     service.obj
 0002:0001944c       $unwind$get_panel_item     000000018006f44c     service.obj
 0002:0001944c       $unwind$__dcrt_get_narrow_environment_from_os 000000018006f44c     libucrt:get_environment_from_os.obj
 0002:0001944c       $unwind$?fp_format_f_internal@@YAHQEAD_KHQEAU_strflt@@_NQEAU__crt_locale_pointers@@@Z 000000018006f44c     libucrt:cvt.obj
 0002:0001944c       $unwind$??$__acrt_wcs_to_mbs_cp@U__crt_win32_buffer_internal_dynamic_resizing@@@@YAHQEB_WAEAV?$__crt_win32_buffer@DU__crt_win32_buffer_internal_dynamic_resizing@@@@I@Z 000000018006f44c     libucrt:argv_wildcards.obj
 0002:00019464       $unwind$get_string_info    000000018006f464     service.obj
 0002:00019480       $unwind$panel_RedrawPanel  000000018006f480     service.obj
 0002:0001949c       $unwind$panel_GetPanelDirectory 000000018006f49c     service.obj
 0002:000194b4       $unwind$panel_SetPanelDirectory 000000018006f4b4     service.obj
 0002:000194dc       $unwind$panel_InsertCmdLine 000000018006f4dc     service.obj
 0002:000194dc       $unwind$panel_SetCmdLine   000000018006f4dc     service.obj
 0002:000194dc       $unwind$??$get_executable_path@_W@@YAPEB_WQEB_W@Z 000000018006f4dc     libucrt:popen.obj
 0002:000194f4       $unwind$ChangePanelSelection 000000018006f4f4     service.obj
 0002:00019510       $chain$0$ChangePanelSelection 000000018006f510     service.obj
 0002:00019524       $chain$1$ChangePanelSelection 000000018006f524     service.obj
 0002:00019538       $chain$2$ChangePanelSelection 000000018006f538     service.obj
 0002:00019548       $chain$3$ChangePanelSelection 000000018006f548     service.obj
 0002:00019558       $unwind$far_GetDirList     000000018006f558     service.obj
 0002:00019558       $unwind$far_LStricmp       000000018006f558     service.obj
 0002:00019558       $unwind$far_LStrnicmp      000000018006f558     service.obj
 0002:00019558       $unwind$far_MkLink         000000018006f558     service.obj
 0002:00019558       $unwind$ustring_system     000000018006f558     ustring.obj
 0002:00019558       $unwind$win_CopyFile       000000018006f558     win.obj
 0002:00019558       $unwind$win_wcscmp         000000018006f558     win.obj
 0002:0001956c       $unwind$far_GetPluginDirList 000000018006f56c     service.obj
 0002:00019578       $chain$2$far_GetPluginDirList 000000018006f578     service.obj
 0002:00019594       $chain$3$far_GetPluginDirList 000000018006f594     service.obj
 0002:000195a8       $chain$4$far_GetPluginDirList 000000018006f5a8     service.obj
 0002:000195b8       $chain$5$far_GetPluginDirList 000000018006f5b8     service.obj
 0002:000195c8       $unwind$far_RestoreScreen  000000018006f5c8     service.obj
 0002:000195d4       $unwind$utf8_range         000000018006f5d4     lutf8lib.obj
 0002:000195d4       $unwind$far_SaveScreen     000000018006f5d4     service.obj
 0002:000195f0       $unwind$CreateList         000000018006f5f0     service.obj
 0002:00019600       $chain$3$CreateList        000000018006f600     service.obj
 0002:00019620       $chain$4$CreateList        000000018006f620     service.obj
 0002:00019630       $unwind$PushList           000000018006f630     service.obj
 0002:0001963c       $chain$5$PushList          000000018006f63c     service.obj
 0002:00019664       $chain$6$PushList          000000018006f664     service.obj
 0002:00019674       $unwind$SetFarDialogItem   000000018006f674     service.obj
 0002:00019684       $chain$2$SetFarDialogItem  000000018006f684     service.obj
 0002:000196a0       $unwind$ProcessDNResult    000000018006f6a0     service.obj
 0002:000196a0       $unwind$PushDlgItem        000000018006f6a0     service.obj
 0002:000196a0       $unwind$PushWinFindData    000000018006f6a0     win.obj
 0002:000196b4       $chain$0$PushDlgItem       000000018006f6b4     service.obj
 0002:000196c8       $unwind$SetDlgItem         000000018006f6c8     service.obj
 0002:000196e4       $unwind$far_SendDlgMessage 000000018006f6e4     service.obj
 0002:0001970c       $chain$0$ProcessDNResult   000000018006f70c     service.obj
 0002:00019720       $chain$1$ProcessDNResult   000000018006f720     service.obj
 0002:00019730       $chain$1$LF_DlgProc        000000018006f730     service.obj
 0002:00019748       $chain$2$LF_DlgProc        000000018006f748     service.obj
 0002:00019758       $unwind$far_DialogInit     000000018006f758     service.obj
 0002:0001977c       $chain$0$far_DialogInit    000000018006f77c     service.obj
 0002:00019790       $unwind$editor_Editor      000000018006f790     service.obj
 0002:000197a8       $unwind$viewer_Viewer      000000018006f7a8     service.obj
 0002:000197c0       $unwind$viewer_GetInfo     000000018006f7c0     service.obj
 0002:000197d8       $unwind$viewer_SetPosition 000000018006f7d8     service.obj
 0002:000197e8       $chain$2$viewer_SetPosition 000000018006f7e8     service.obj
 0002:00019804       $chain$3$viewer_SetPosition 000000018006f804     service.obj
 0002:00019818       $chain$4$viewer_SetPosition 000000018006f818     service.obj
 0002:00019828       $chain$5$viewer_SetPosition 000000018006f828     service.obj
 0002:00019838       $unwind$viewer_SetMode     000000018006f838     service.obj
 0002:00019848       $unwind$far_ShowHelp       000000018006f848     service.obj
 0002:0001985c       $chain$1$far_ShowHelp      000000018006f85c     service.obj
 0002:00019874       $chain$2$far_ShowHelp      000000018006f874     service.obj
 0002:00019884       $unwind$far_InputBox       000000018006f884     service.obj
 0002:000198a0       $unwind$far_GetMsg         000000018006f8a0     service.obj
 0002:000198b4       $chain$1$far_GetMsg        000000018006f8b4     service.obj
 0002:000198cc       $chain$2$far_GetMsg        000000018006f8cc     service.obj
 0002:000198e0       $chain$3$far_GetMsg        000000018006f8e0     service.obj
 0002:000198f0       $chain$4$far_GetMsg        000000018006f8f0     service.obj
 0002:000198f0       $chain$6$far_GetMsg        000000018006f8f0     service.obj
 0002:00019900       $chain$5$far_GetMsg        000000018006f900     service.obj
 0002:00019918       $unwind$far_Text           000000018006f918     service.obj
 0002:00019930       $chain$1$far_Text          000000018006f930     service.obj
 0002:00019948       $chain$2$far_Text          000000018006f948     service.obj
 0002:0001995c       $chain$3$far_Text          000000018006f95c     service.obj
 0002:0001996c       $chain$4$far_Text          000000018006f96c     service.obj
 0002:0001997c       $chain$3$far_CopyToClipboard 000000018006f97c     service.obj
 0002:0001999c       $chain$4$far_CopyToClipboard 000000018006f99c     service.obj
 0002:000199b4       $chain$5$far_CopyToClipboard 000000018006f9b4     service.obj
 0002:000199c4       $unwind$far_PasteFromClipboard 000000018006f9c4     service.obj
 0002:000199d8       $unwind$far_InputRecordToName 000000018006f9d8     service.obj
 0002:000199f8       $unwind$far_NameToInputRecord 000000018006f9f8     service.obj
 0002:00019a08       $chain$2$far_NameToInputRecord 000000018006fa08     service.obj
 0002:00019a24       $chain$3$far_NameToInputRecord 000000018006fa24     service.obj
 0002:00019a38       $chain$4$far_NameToInputRecord 000000018006fa38     service.obj
 0002:00019a48       $chain$5$far_NameToInputRecord 000000018006fa48     service.obj
 0002:00019a58       $unwind$far_ProcessName    000000018006fa58     service.obj
 0002:00019a6c       $chain$2$far_ProcessName   000000018006fa6c     service.obj
 0002:00019a84       $unwind$far_GetPathRoot    000000018006fa84     service.obj
 0002:00019a84       $unwind$far_GetReparsePointInfo 000000018006fa84     service.obj
 0002:00019a9c       $unwind$far_LIsAlpha       000000018006fa9c     service.obj
 0002:00019a9c       $unwind$far_LIsAlphanum    000000018006fa9c     service.obj
 0002:00019a9c       $unwind$far_LIsLower       000000018006fa9c     service.obj
 0002:00019a9c       $unwind$far_LIsUpper       000000018006fa9c     service.obj
 0002:00019a9c       $unwind$ll_loadlib         000000018006fa9c     uloadlib51.obj
 0002:00019a9c       $unwind$ustring_Utf8ToUtf16 000000018006fa9c     ustring.obj
 0002:00019a9c       $unwind$?decode_options@@YA?AUfile_options@?A0xa9d50aae@@HHH@Z 000000018006fa9c     libucrt:open.obj
 0002:00019ab0       $unwind$convert_buf        000000018006fab0     service.obj
 0002:00019ac8       $unwind$far_MkTemp         000000018006fac8     service.obj
 0002:00019adc       $unwind$truncstring        000000018006fadc     service.obj
 0002:00019af4       $unwind$FrsUserFunc        000000018006faf4     service.obj
 0002:00019b08       $chain$1$FrsUserFunc       000000018006fb08     service.obj
 0002:00019b20       $chain$2$FrsUserFunc       000000018006fb20     service.obj
 0002:00019b30       $unwind$far_RecursiveSearch 000000018006fb30     service.obj
 0002:00019b44       $unwind$far_ConvertPath    000000018006fb44     service.obj
 0002:00019b44       $unwind$??$parse_integer@KV?$c_string_character_source@_W@__crt_strtox@@@__crt_strtox@@YAKQEAU__crt_locale_pointers@@V?$c_string_character_source@_W@0@H_N@Z 000000018006fb44     libucrt:atox.obj
 0002:00019b5c       $unwind$far_AdvControl     000000018006fb5c     service.obj
 0002:00019b84       $chain$0$far_AdvControl    000000018006fb84     service.obj
 0002:00019b98       $chain$1$far_AdvControl    000000018006fb98     service.obj
 0002:00019ba8       $unwind$far_MacroLoadAll   000000018006fba8     service.obj
 0002:00019bb8       $chain$1$far_MacroLoadAll  000000018006fbb8     service.obj
 0002:00019bd0       $chain$2$far_MacroLoadAll  000000018006fbd0     service.obj
 0002:00019be0       $unwind$MacroSendString    000000018006fbe0     service.obj
 0002:00019c00       $unwind$far_MacroGetLastError 000000018006fc00     service.obj
 0002:00019c00       $unwind$fileerror          000000018006fc00     uliolib51.obj
 0002:00019c10       $chain$0$far_MacroGetLastError 000000018006fc10     service.obj
 0002:00019c24       $chain$1$far_MacroGetLastError 000000018006fc24     service.obj
 0002:00019c38       $chain$2$far_MacroGetLastError 000000018006fc38     service.obj
 0002:00019c48       $chain$3$far_MacroGetLastError 000000018006fc48     service.obj
 0002:00019c58       $unwind$MacroAddCallback   000000018006fc58     service.obj
 0002:00019c6c       $unwind$far_MacroAdd       000000018006fc6c     service.obj
 0002:00019c94       $unwind$far_MacroExecute   000000018006fc94     service.obj
 0002:00019cac       $unwind$far_MakeMenuItems  000000018006fcac     service.obj
 0002:00019cc0       $chain$5$far_MakeMenuItems 000000018006fcc0     service.obj
 0002:00019ce8       $chain$6$far_MakeMenuItems 000000018006fce8     service.obj
 0002:00019cf8       $unwind$filefilter_IsFileInFilter 000000018006fcf8     service.obj
 0002:00019d14       $unwind$far_FindPlugin     000000018006fd14     service.obj
 0002:00019d24       $chain$1$far_FindPlugin    000000018006fd24     service.obj
 0002:00019d3c       $chain$3$far_FindPlugin    000000018006fd3c     service.obj
 0002:00019d54       $chain$4$far_FindPlugin    000000018006fd54     service.obj
 0002:00019d64       $unwind$PutPluginMenuItemToTable 000000018006fd64     service.obj
 0002:00019d74       $chain$2$PutPluginMenuItemToTable 000000018006fd74     service.obj
 0002:00019d90       $chain$3$PutPluginMenuItemToTable 000000018006fd90     service.obj
 0002:00019da0       $unwind$far_GetPluginInformation 000000018006fda0     service.obj
 0002:00019db4       $chain$0$far_GetPluginInformation 000000018006fdb4     service.obj
 0002:00019dc8       $chain$1$far_GetPluginInformation 000000018006fdc8     service.obj
 0002:00019dd8       $unwind$Lutf8_sub          000000018006fdd8     lutf8lib.obj
 0002:00019dd8       $unwind$far_GetPlugins     000000018006fdd8     service.obj
 0002:00019de4       $chain$1$far_GetPlugins    000000018006fde4     service.obj
 0002:00019dfc       $chain$2$far_GetPlugins    000000018006fdfc     service.obj
 0002:00019e10       $chain$3$far_GetPlugins    000000018006fe10     service.obj
 0002:00019e20       $chain$4$far_GetPlugins    000000018006fe20     service.obj
 0002:00019e30       $unwind$far_IsPluginLoaded 000000018006fe30     service.obj
 0002:00019e4c       $chain$0$far_IsPluginLoaded 000000018006fe4c     service.obj
 0002:00019e60       $chain$1$far_IsPluginLoaded 000000018006fe60     service.obj
 0002:00019e70       $unwind$far_XLat           000000018006fe70     service.obj
 0002:00019e70       $unwind$io_open            000000018006fe70     uliolib51.obj
 0002:00019e88       $unwind$Lutf8_insert       000000018006fe88     lutf8lib.obj
 0002:00019e88       $unwind$far_FormatFileSize 000000018006fe88     service.obj
 0002:00019e88       $unwind$win_GetEnv         000000018006fe88     win.obj
 0002:00019ea8       $chain$0$timer_Close       000000018006fea8     service.obj
 0002:00019ebc       $chain$1$timer_Close       000000018006febc     service.obj
 0002:00019ecc       $chain$0$timer_gc          000000018006fecc     service.obj
 0002:00019ee0       $chain$1$timer_gc          000000018006fee0     service.obj
 0002:00019ef0       $unwind$far_CreateSettings 000000018006fef0     service.obj
 0002:00019f0c       $unwind$Settings_set       000000018006ff0c     service.obj
 0002:00019f28       $unwind$Settings_get       000000018006ff28     service.obj
 0002:00019f40       $unwind$Settings_delete    000000018006ff40     service.obj
 0002:00019f4c       $chain$2$Settings_delete   000000018006ff4c     service.obj
 0002:00019f68       $chain$3$Settings_delete   000000018006ff68     service.obj
 0002:00019f78       $unwind$Settings_createsubkey 000000018006ff78     service.obj
 0002:00019f90       $unwind$Settings_opensubkey 000000018006ff90     service.obj
 0002:00019f98       $chain$3$Settings_opensubkey 000000018006ff98     service.obj
 0002:00019fb8       $chain$4$Settings_opensubkey 000000018006ffb8     service.obj
 0002:00019fcc       $chain$5$Settings_opensubkey 000000018006ffcc     service.obj
 0002:00019fdc       $chain$6$Settings_opensubkey 000000018006ffdc     service.obj
 0002:00019fec       $unwind$Settings_enum      000000018006ffec     service.obj
 0002:00019ffc       $chain$1$Settings_enum     000000018006fffc     service.obj
 0002:0001a014       $chain$2$Settings_enum     0000000180070014     service.obj
 0002:0001a028       $chain$3$Settings_enum     0000000180070028     service.obj
 0002:0001a038       $chain$5$Settings_enum     0000000180070038     service.obj
 0002:0001a050       $chain$6$Settings_enum     0000000180070050     service.obj
 0002:0001a060       $unwind$far_ColorDialog    0000000180070060     service.obj
 0002:0001a07c       $unwind$GetPluginModuleHandle 000000018007007c     service.obj
 0002:0001a08c       $chain$0$GetPluginModuleHandle 000000018007008c     service.obj
 0002:0001a0a0       $chain$1$GetPluginModuleHandle 00000001800700a0     service.obj
 0002:0001a0b4       $chain$2$GetPluginModuleHandle 00000001800700b4     service.obj
 0002:0001a0c4       $chain$4$GetPluginModuleHandle 00000001800700c4     service.obj
 0002:0001a0d8       $chain$5$GetPluginModuleHandle 00000001800700d8     service.obj
 0002:0001a0e8       $unwind$far_host_GetFiles  00000001800700e8     service.obj
 0002:0001a0e8       $unwind$far_host_PutFiles  00000001800700e8     service.obj
 0002:0001a10c       $chain$0$far_host_GetFiles 000000018007010c     service.obj
 0002:0001a120       $chain$1$far_host_GetFiles 0000000180070120     service.obj
 0002:0001a130       $chain$0$far_host_PutFiles 0000000180070130     service.obj
 0002:0001a144       $chain$1$far_host_PutFiles 0000000180070144     service.obj
 0002:0001a154       $unwind$far_host_GetFindData 0000000180070154     service.obj
 0002:0001a170       $unwind$far_host_FreeUserData 0000000180070170     service.obj
 0002:0001a180       $chain$1$far_host_FreeUserData 0000000180070180     service.obj
 0002:0001a198       $chain$2$far_host_FreeUserData 0000000180070198     service.obj
 0002:0001a1a8       $unwind$far_host_SetDirectory 00000001800701a8     service.obj
 0002:0001a1c8       $chain$1$far_host_SetDirectory 00000001800701c8     service.obj
 0002:0001a1e0       $chain$2$far_host_SetDirectory 00000001800701e0     service.obj
 0002:0001a1f0       $unwind$luaopen_far        00000001800701f0     service.obj
 0002:0001a1f0       $unwind$__acrt_DownlevelLocaleNameToLCID 00000001800701f0     libucrt:lcidtoname_downlevel.obj
 0002:0001a1f0       $unwind$??R<lambda_f03950bc5685219e0bcd2087efbe011e>@@QEBAHXZ 00000001800701f0     libucrt:onexit.obj
 0002:0001a1f0       $unwind$??$parse_floating_point_possible_infinity@DV?$input_adapter_character_source@V?$stream_input_adapter@D@__crt_stdio_input@@@__crt_strtox@@_K@__crt_strtox@@YA?AW4floating_point_parse_result@0@AEADAEAV?$input_adapter_character_source@V?$stream_input_adapter@D@__crt_stdio_input@@@0@_K@Z 00000001800701f0     libucrt:input.obj
 0002:0001a1f0       $unwind$??$parse_floating_point_possible_nan_is_ind@DV?$input_adapter_character_source@V?$stream_input_adapter@D@__crt_stdio_input@@@__crt_strtox@@@__crt_strtox@@YA_NAEADAEAV?$input_adapter_character_source@V?$stream_input_adapter@D@__crt_stdio_input@@@0@@Z 00000001800701f0     libucrt:input.obj
 0002:0001a1f0       $unwind$??$parse_floating_point_possible_nan_is_snan@DV?$input_adapter_character_source@V?$stream_input_adapter@D@__crt_stdio_input@@@__crt_strtox@@@__crt_strtox@@YA_NAEADAEAV?$input_adapter_character_source@V?$stream_input_adapter@D@__crt_stdio_input@@@0@@Z 00000001800701f0     libucrt:input.obj
 0002:0001a1f0       $unwind$?type_case_integer@?$output_processor@DV?$stream_output_adapter@D@__crt_stdio_output@@V?$standard_base@DV?$stream_output_adapter@D@__crt_stdio_output@@@2@@__crt_stdio_output@@AEAA_NI_N@Z 00000001800701f0     libucrt:output.obj
 0002:0001a1f0       $unwind$?type_case_integer@?$output_processor@DV?$string_output_adapter@D@__crt_stdio_output@@V?$standard_base@DV?$string_output_adapter@D@__crt_stdio_output@@@2@@__crt_stdio_output@@AEAA_NI_N@Z 00000001800701f0     libucrt:output.obj
 0002:0001a1f0       $unwind$?type_case_integer@?$output_processor@_WV?$string_output_adapter@_W@__crt_stdio_output@@V?$standard_base@_WV?$string_output_adapter@_W@__crt_stdio_output@@@2@@__crt_stdio_output@@AEAA_NI_N@Z 00000001800701f0     libucrt:output.obj
 0002:0001a208       $unwind$LF_RunLuafarInit   0000000180070208     service.obj
 0002:0001a21c       $unwind$LF_DoFile          000000018007021c     service.obj
 0002:0001a22c       $chain$0$LF_DoFile         000000018007022c     service.obj
 0002:0001a240       $chain$2$LF_DoFile         0000000180070240     service.obj
 0002:0001a258       $chain$3$LF_DoFile         0000000180070258     service.obj
 0002:0001a268       $chain$4$LF_DoFile         0000000180070268     service.obj
 0002:0001a278       $unwind$_snwprintf         0000000180070278     slnunico.obj
 0002:0001a288       $unwind$str_rep            0000000180070288     slnunico.obj
 0002:0001a2a4       $unwind$str_dump           00000001800702a4     slnunico.obj
 0002:0001a2b8       $unwind$str_format         00000001800702b8     slnunico.obj
 0002:0001a2e0       $unwind$utf8_iscompose     00000001800702e0     lutf8lib.obj
 0002:0001a2e0       $unwind$utf8_isdigit       00000001800702e0     lutf8lib.obj
 0002:0001a2e0       $unwind$utf8_isgraph       00000001800702e0     lutf8lib.obj
 0002:0001a2e0       $unwind$utf8_islower       00000001800702e0     lutf8lib.obj
 0002:0001a2e0       $unwind$??$type_case_integer_parse_into_buffer@I@?$output_processor@DV?$stream_output_adapter@D@__crt_stdio_output@@V?$standard_base@DV?$stream_output_adapter@D@__crt_stdio_output@@@2@@__crt_stdio_output@@AEAAXII_N@Z 00000001800702e0     libucrt:output.obj
 0002:0001a2e0       $unwind$??$type_case_integer_parse_into_buffer@I@?$output_processor@DV?$string_output_adapter@D@__crt_stdio_output@@V?$standard_base@DV?$string_output_adapter@D@__crt_stdio_output@@@2@@__crt_stdio_output@@AEAAXII_N@Z 00000001800702e0     libucrt:output.obj
 0002:0001a2e0       $unwind$??$type_case_integer_parse_into_buffer@I@?$output_processor@_WV?$string_output_adapter@_W@__crt_stdio_output@@V?$standard_base@_WV?$string_output_adapter@_W@__crt_stdio_output@@@2@@__crt_stdio_output@@AEAAXII_N@Z 00000001800702e0     libucrt:output.obj
 0002:0001a2e0       $unwind$??$type_case_integer_parse_into_buffer@_K@?$output_processor@DV?$stream_output_adapter@D@__crt_stdio_output@@V?$standard_base@DV?$stream_output_adapter@D@__crt_stdio_output@@@2@@__crt_stdio_output@@AEAAX_KI_N@Z 00000001800702e0     libucrt:output.obj
 0002:0001a2e0       $unwind$??$type_case_integer_parse_into_buffer@_K@?$output_processor@DV?$string_output_adapter@D@__crt_stdio_output@@V?$standard_base@DV?$string_output_adapter@D@__crt_stdio_output@@@2@@__crt_stdio_output@@AEAAX_KI_N@Z 00000001800702e0     libucrt:output.obj
 0002:0001a2e0       $unwind$??$type_case_integer_parse_into_buffer@_K@?$output_processor@_WV?$string_output_adapter@_W@__crt_stdio_output@@V?$standard_base@_WV?$string_output_adapter@_W@__crt_stdio_output@@@2@@__crt_stdio_output@@AEAAX_KI_N@Z 00000001800702e0     libucrt:output.obj
 0002:0001a2e8       $unwind$utf8_width         00000001800702e8     lutf8lib.obj
 0002:0001a2f4       $unwind$Lutf8_len          00000001800702f4     lutf8lib.obj
 0002:0001a30c       $unwind$Lutf8_reverse      000000018007030c     lutf8lib.obj
 0002:0001a330       $unwind$Lutf8_byte         0000000180070330     lutf8lib.obj
 0002:0001a340       $chain$1$Lutf8_byte        0000000180070340     lutf8lib.obj
 0002:0001a358       $chain$3$Lutf8_byte        0000000180070358     lutf8lib.obj
 0002:0001a36c       $chain$4$Lutf8_byte        000000018007036c     lutf8lib.obj
 0002:0001a37c       $unwind$Lutf8_codepoint    000000018007037c     lutf8lib.obj
 0002:0001a390       $chain$0$Lutf8_codepoint   0000000180070390     lutf8lib.obj
 0002:0001a3a4       $chain$2$Lutf8_codepoint   00000001800703a4     lutf8lib.obj
 0002:0001a3b8       $unwind$Lutf8_char         00000001800703b8     lutf8lib.obj
 0002:0001a3d4       $chain$0$Lutf8_char        00000001800703d4     lutf8lib.obj
 0002:0001a3e8       $chain$1$Lutf8_char        00000001800703e8     lutf8lib.obj
 0002:0001a3f8       $unwind$Lutf8_fold         00000001800703f8     lutf8lib.obj
 0002:0001a3f8       $unwind$Lutf8_lower        00000001800703f8     lutf8lib.obj
 0002:0001a3f8       $unwind$Lutf8_title        00000001800703f8     lutf8lib.obj
 0002:0001a3f8       $unwind$Lutf8_upper        00000001800703f8     lutf8lib.obj
 0002:0001a410       $chain$1$Lutf8_lower       0000000180070410     lutf8lib.obj
 0002:0001a428       $chain$2$Lutf8_lower       0000000180070428     lutf8lib.obj
 0002:0001a43c       $chain$3$Lutf8_lower       000000018007043c     lutf8lib.obj
 0002:0001a44c       $chain$4$Lutf8_lower       000000018007044c     lutf8lib.obj
 0002:0001a45c       $chain$1$Lutf8_upper       000000018007045c     lutf8lib.obj
 0002:0001a474       $chain$2$Lutf8_upper       0000000180070474     lutf8lib.obj
 0002:0001a488       $chain$3$Lutf8_upper       0000000180070488     lutf8lib.obj
 0002:0001a498       $chain$4$Lutf8_upper       0000000180070498     lutf8lib.obj
 0002:0001a4a8       $chain$1$Lutf8_title       00000001800704a8     lutf8lib.obj
 0002:0001a4c0       $chain$2$Lutf8_title       00000001800704c0     lutf8lib.obj
 0002:0001a4d4       $chain$3$Lutf8_title       00000001800704d4     lutf8lib.obj
 0002:0001a4e4       $chain$4$Lutf8_title       00000001800704e4     lutf8lib.obj
 0002:0001a4f4       $chain$1$Lutf8_fold        00000001800704f4     lutf8lib.obj
 0002:0001a50c       $chain$2$Lutf8_fold        000000018007050c     lutf8lib.obj
 0002:0001a520       $chain$3$Lutf8_fold        0000000180070520     lutf8lib.obj
 0002:0001a530       $chain$4$Lutf8_fold        0000000180070530     lutf8lib.obj
 0002:0001a540       $unwind$Lutf8_escape       0000000180070540     lutf8lib.obj
 0002:0001a558       $chain$4$Lutf8_escape      0000000180070558     lutf8lib.obj
 0002:0001a57c       $chain$5$Lutf8_escape      000000018007057c     lutf8lib.obj
 0002:0001a58c       $unwind$Lutf8_remove       000000018007058c     lutf8lib.obj
 0002:0001a5a8       $unwind$Lutf8_charpos      00000001800705a8     lutf8lib.obj
 0002:0001a5c0       $unwind$Lutf8_offset       00000001800705c0     lutf8lib.obj
 0002:0001a5d4       $unwind$Lutf8_next         00000001800705d4     lutf8lib.obj
 0002:0001a5d4       $unwind$win_CreateDir      00000001800705d4     win.obj
 0002:0001a5ec       $unwind$iter_aux           00000001800705ec     lutf8lib.obj
 0002:0001a5ec       $unwind$g_write            00000001800705ec     uliolib51.obj
 0002:0001a600       $unwind$Lutf8_width        0000000180070600     lutf8lib.obj
 0002:0001a618       $chain$3$Lutf8_width       0000000180070618     lutf8lib.obj
 0002:0001a630       $chain$4$Lutf8_width       0000000180070630     lutf8lib.obj
 0002:0001a640       $unwind$Lutf8_widthindex   0000000180070640     lutf8lib.obj
 0002:0001a640       $unwind$_fwrite_nolock     0000000180070640     libucrt:fwrite.obj
 0002:0001a65c       $unwind$Lutf8_ncasecmp     000000018007065c     lutf8lib.obj
 0002:0001a65c       $unwind$matchbracketclass  000000018007065c     lutf8lib.obj
 0002:0001a674       $unwind$singlematch        0000000180070674     lutf8lib.obj
 0002:0001a688       $chain$3$singlematch       0000000180070688     lutf8lib.obj
 0002:0001a6a0       $chain$4$singlematch       00000001800706a0     lutf8lib.obj
 0002:0001a6b4       $unwind$match              00000001800706b4     lutf8lib.obj
 0002:0001a6c0       $chain$4$match             00000001800706c0     lutf8lib.obj
 0002:0001a6e4       $chain$5$match             00000001800706e4     lutf8lib.obj
 0002:0001a6f4       $chain$1$push_onecapture   00000001800706f4     lutf8lib.obj
 0002:0001a70c       $chain$3$push_onecapture   000000018007070c     lutf8lib.obj
 0002:0001a724       $unwind$push_captures      0000000180070724     lutf8lib.obj
 0002:0001a738       $chain$1$push_captures     0000000180070738     lutf8lib.obj
 0002:0001a750       $chain$2$push_captures     0000000180070750     lutf8lib.obj
 0002:0001a760       $chain$3$push_captures     0000000180070760     lutf8lib.obj
 0002:0001a778       $unwind$find_aux           0000000180070778     lutf8lib.obj
 0002:0001a7a0       $unwind$gmatch_aux         00000001800707a0     lutf8lib.obj
 0002:0001a7c4       $unwind$add_s              00000001800707c4     lutf8lib.obj
 0002:0001a7e0       $chain$1$add_s             00000001800707e0     lutf8lib.obj
 0002:0001a7f8       $chain$2$add_s             00000001800707f8     lutf8lib.obj
 0002:0001a808       $unwind$Lutf8_gsub         0000000180070808     lutf8lib.obj
 0002:0001a830       $unwind$luaopen_utf8       0000000180070830     lutf8lib.obj
 0002:0001a848       $unwind$pushresult         0000000180070848     uliolib51.obj
 0002:0001a858       $chain$1$pushresult        0000000180070858     uliolib51.obj
 0002:0001a870       $chain$2$pushresult        0000000180070870     uliolib51.obj
 0002:0001a880       $chain$1$fileerror         0000000180070880     uliolib51.obj
 0002:0001a898       $chain$2$fileerror         0000000180070898     uliolib51.obj
 0002:0001a8a8       $unwind$io_popen           00000001800708a8     uliolib51.obj
 0002:0001a8b4       $chain$2$io_popen          00000001800708b4     uliolib51.obj
 0002:0001a8d0       $chain$3$io_popen          00000001800708d0     uliolib51.obj
 0002:0001a8e4       $chain$4$io_popen          00000001800708e4     uliolib51.obj
 0002:0001a8f4       $chain$5$io_popen          00000001800708f4     uliolib51.obj
 0002:0001a904       $unwind$g_iofile           0000000180070904     uliolib51.obj
 0002:0001a910       $chain$3$g_iofile          0000000180070910     uliolib51.obj
 0002:0001a930       $chain$4$g_iofile          0000000180070930     uliolib51.obj
 0002:0001a940       $chain$5$g_iofile          0000000180070940     uliolib51.obj
 0002:0001a960       $chain$3$io_lines          0000000180070960     uliolib51.obj
 0002:0001a980       $chain$4$io_lines          0000000180070980     uliolib51.obj
 0002:0001a994       $unwind$read_line          0000000180070994     uliolib51.obj
 0002:0001a9b0       $unwind$read_chars         00000001800709b0     uliolib51.obj
 0002:0001a9b0       $unwind$ustring_GetCurrentDir 00000001800709b0     ustring.obj
 0002:0001a9cc       $unwind$g_read             00000001800709cc     uliolib51.obj
 0002:0001a9ec       $unwind$findfile           00000001800709ec     uloadlib51.obj
 0002:0001aa0c       $chain$0$findfile          0000000180070a0c     uloadlib51.obj
 0002:0001aa20       $chain$1$findfile          0000000180070a20     uloadlib51.obj
 0002:0001aa30       $chain$0$loaderror         0000000180070a30     uloadlib51.obj
 0002:0001aa44       $chain$1$loaderror         0000000180070a44     uloadlib51.obj
 0002:0001aa54       $unwind$loader_Croot       0000000180070a54     uloadlib51.obj
 0002:0001aa64       $unwind$ll_module          0000000180070a64     uloadlib51.obj
 0002:0001aa80       $unwind$setpath            0000000180070a80     uloadlib51.obj
 0002:0001aa9c       $unwind$pusherrorcode      0000000180070a9c     ustring.obj
 0002:0001aab4       $chain$0$pusherrorcode     0000000180070ab4     ustring.obj
 0002:0001aac8       $chain$1$pusherrorcode     0000000180070ac8     ustring.obj
 0002:0001aadc       $chain$2$pusherrorcode     0000000180070adc     ustring.obj
 0002:0001aaec       $chain$3$pusherrorcode     0000000180070aec     ustring.obj
 0002:0001aafc       $unwind$PutWStrToTable     0000000180070afc     ustring.obj
 0002:0001aafc       $unwind$strerror           0000000180070afc     libucrt:strerror.obj
 0002:0001aafc       $unwind$?convert_hexadecimal_string_to_floating_type_common@__crt_strtox@@YA?AW4SLD_STATUS@@AEBUfloating_point_string@1@AEBVfloating_point_value@1@@Z 0000000180070afc     libucrt:input.obj
 0002:0001ab08       $unwind$PutWStrToArray     0000000180070b08     ustring.obj
 0002:0001ab08       $unwind$GetIntFromArray    0000000180070b08     util.obj
 0002:0001ab08       $unwind$??$initialize_environment_by_cloning_nolock@_W@@YAHXZ 0000000180070b08     libucrt:environment_initialization.obj
 0002:0001ab08       $unwind$??$generate_tmpfile_file_name@D@@YA_NQEAD_K@Z 0000000180070b08     libucrt:tmpfile.obj
 0002:0001ab08       $unwind$_strdup            0000000180070b08     libucrt:strdup.obj
 0002:0001ab08       $unwind$strpbrk            0000000180070b08     libucrt:strpbrk.obj
 0002:0001ab18       $unwind$GetOptNumFromTable 0000000180070b18     ustring.obj
 0002:0001ab24       $unwind$check_utf8_string  0000000180070b24     ustring.obj
 0002:0001ab3c       $unwind$utf8_to_utf16      0000000180070b3c     ustring.obj
 0002:0001ab54       $chain$3$utf8_to_utf16     0000000180070b54     ustring.obj
 0002:0001ab68       $chain$4$utf8_to_utf16     0000000180070b68     ustring.obj
 0002:0001ab78       $unwind$push_multibyte_string 0000000180070b78     ustring.obj
 0002:0001ab8c       $chain$2$push_multibyte_string 0000000180070b8c     ustring.obj
 0002:0001aba4       $chain$3$push_multibyte_string 0000000180070ba4     ustring.obj
 0002:0001abb8       $unwind$push_utf8_string   0000000180070bb8     ustring.obj
 0002:0001abb8       $unwind$_wdupenv_s         0000000180070bb8     libucrt:getenv.obj
 0002:0001abb8       $unwind$strtol             0000000180070bb8     libucrt:strtox.obj
 0002:0001abb8       $unwind$strtoull           0000000180070bb8     libucrt:strtox.obj
 0002:0001abb8       $unwind$wcstol             0000000180070bb8     libucrt:strtox.obj
 0002:0001abb8       $unwind$wctomb_s           0000000180070bb8     libucrt:wctomb.obj
 0002:0001abb8       $unwind$_ui64toa_s         0000000180070bb8     libucrt:xtoa.obj
 0002:0001abb8       $unwind$_sopen_s           0000000180070bb8     libucrt:open.obj
 0002:0001abb8       $unwind$_wsopen_s          0000000180070bb8     libucrt:open.obj
 0002:0001abb8       $unwind$_invalid_parameter_noinfo 0000000180070bb8     libucrt:invalid_parameter.obj
 0002:0001abb8       $unwind$fflush             0000000180070bb8     libucrt:fflush.obj
 0002:0001abb8       $unwind$fread              0000000180070bb8     libucrt:fread.obj
 0002:0001abb8       $unwind$_wfreopen          0000000180070bb8     libucrt:freopen.obj
 0002:0001abb8       $unwind$??$parse_floating_point_write_result@M@__crt_strtox@@YA?AW4SLD_STATUS@@W4floating_point_parse_result@0@AEBUfloating_point_string@0@QEAM@Z 0000000180070bb8     libucrt:input.obj
 0002:0001abb8       $unwind$??$parse_floating_point_write_result@N@__crt_strtox@@YA?AW4SLD_STATUS@@W4floating_point_parse_result@0@AEBUfloating_point_string@0@QEAN@Z 0000000180070bb8     libucrt:input.obj
 0002:0001abb8       $unwind$?as_double@floating_point_value@__crt_strtox@@QEBAAEANXZ 0000000180070bb8     libucrt:input.obj
 0002:0001abb8       $unwind$?as_float@floating_point_value@__crt_strtox@@QEBAAEAMXZ 0000000180070bb8     libucrt:input.obj
 0002:0001abb8       $unwind$_log10_special     0000000180070bb8     libucrt:log_special.obj
 0002:0001abc0       $unwind$ustring_WideCharToMultiByte 0000000180070bc0     ustring.obj
 0002:0001abd4       $chain$1$ustring_WideCharToMultiByte 0000000180070bd4     ustring.obj
 0002:0001abec       $chain$2$ustring_WideCharToMultiByte 0000000180070bec     ustring.obj
 0002:0001abfc       $unwind$ustring_MultiByteToWideChar 0000000180070bfc     ustring.obj
 0002:0001ac18       $unwind$ustring_OemToUtf8  0000000180070c18     ustring.obj
 0002:0001ac24       $chain$1$ustring_OemToUtf8 0000000180070c24     ustring.obj
 0002:0001ac3c       $chain$2$ustring_OemToUtf8 0000000180070c3c     ustring.obj
 0002:0001ac4c       $unwind$ustring_Utf8ToOem  0000000180070c4c     ustring.obj
 0002:0001ac60       $chain$0$ustring_Utf8ToOem 0000000180070c60     ustring.obj
 0002:0001ac74       $chain$1$ustring_Utf8ToOem 0000000180070c74     ustring.obj
 0002:0001ac84       $unwind$ustring_Utf16ToUtf8 0000000180070c84     ustring.obj
 0002:0001ac84       $unwind$?__mbrtowc_utf8@__crt_mbstring@@YA_KPEA_WPEBD_KPEAU_Mbstatet@@@Z 0000000180070c84     libucrt:mbrtowc.obj
 0002:0001ac84       $unwind$??$common_xtox_s@_KD@@YAH_KQEAD0I_N@Z 0000000180070c84     libucrt:xtoa.obj
 0002:0001ac8c       $unwind$ustring_SetConsoleCP 0000000180070c8c     ustring.obj
 0002:0001ac8c       $unwind$ustring_SetConsoleOutputCP 0000000180070c8c     ustring.obj
 0002:0001ac98       $unwind$EnumCodePagesProc  0000000180070c98     ustring.obj
 0002:0001aca4       $chain$2$EnumCodePagesProc 0000000180070ca4     ustring.obj
 0002:0001acc0       $chain$3$EnumCodePagesProc 0000000180070cc0     ustring.obj
 0002:0001acd0       $unwind$ustring_GetCPInfo  0000000180070cd0     ustring.obj
 0002:0001ace8       $chain$1$ustring_GetCPInfo 0000000180070ce8     ustring.obj
 0002:0001ad00       $chain$2$ustring_GetCPInfo 0000000180070d00     ustring.obj
 0002:0001ad10       $chain$0$ustring_GetLogicalDriveStrings 0000000180070d10     ustring.obj
 0002:0001ad24       $chain$2$ustring_GetLogicalDriveStrings 0000000180070d24     ustring.obj
 0002:0001ad3c       $chain$3$ustring_GetLogicalDriveStrings 0000000180070d3c     ustring.obj
 0002:0001ad4c       $chain$4$ustring_GetLogicalDriveStrings 0000000180070d4c     ustring.obj
 0002:0001ad5c       $unwind$ustring_GetDriveType 0000000180070d5c     ustring.obj
 0002:0001ad64       $chain$0$ustring_GetDriveType 0000000180070d64     ustring.obj
 0002:0001ad78       $chain$2$ustring_GetDriveType 0000000180070d78     ustring.obj
 0002:0001ad90       $chain$3$ustring_GetDriveType 0000000180070d90     ustring.obj
 0002:0001ada4       $chain$4$ustring_GetDriveType 0000000180070da4     ustring.obj
 0002:0001adb4       $chain$5$ustring_GetDriveType 0000000180070db4     ustring.obj
 0002:0001adc4       $chain$6$ustring_GetDriveType 0000000180070dc4     ustring.obj
 0002:0001add4       $unwind$ustring_SearchPath 0000000180070dd4     ustring.obj
 0002:0001adf0       $chain$0$ustring_SearchPath 0000000180070df0     ustring.obj
 0002:0001ae04       $chain$1$ustring_SearchPath 0000000180070e04     ustring.obj
 0002:0001ae18       $chain$2$ustring_SearchPath 0000000180070e18     ustring.obj
 0002:0001ae28       $chain$3$ustring_SearchPath 0000000180070e28     ustring.obj
 0002:0001ae38       $unwind$ustring_GlobalMemoryStatus 0000000180070e38     ustring.obj
 0002:0001ae48       $chain$0$ustring_GlobalMemoryStatus 0000000180070e48     ustring.obj
 0002:0001ae5c       $chain$1$ustring_GlobalMemoryStatus 0000000180070e5c     ustring.obj
 0002:0001ae6c       $unwind$PushAttrString     0000000180070e6c     ustring.obj
 0002:0001ae6c       $unwind$fallbackMethod     0000000180070e6c     libucrt:strpbrk.obj
 0002:0001ae7c       $chain$2$ustring_SetFileAttr 0000000180070e7c     ustring.obj
 0002:0001ae98       $chain$3$ustring_SetFileAttr 0000000180070e98     ustring.obj
 0002:0001aea8       $chain$2$ustring_GetFileAttr 0000000180070ea8     ustring.obj
 0002:0001aec4       $chain$3$ustring_GetFileAttr 0000000180070ec4     ustring.obj
 0002:0001aed4       $unwind$ustring_SHGetFolderPath 0000000180070ed4     ustring.obj
 0002:0001aeec       $chain$1$ustring_SHGetFolderPath 0000000180070eec     ustring.obj
 0002:0001af04       $chain$2$ustring_SHGetFolderPath 0000000180070f04     ustring.obj
 0002:0001af14       $chain$2$ustring_OutputDebugString 0000000180070f14     ustring.obj
 0002:0001af30       $chain$3$ustring_OutputDebugString 0000000180070f30     ustring.obj
 0002:0001af44       $chain$4$ustring_OutputDebugString 0000000180070f44     ustring.obj
 0002:0001af54       $chain$5$ustring_OutputDebugString 0000000180070f54     ustring.obj
 0002:0001af64       $chain$0$ustring_GetCurrentDir 0000000180070f64     ustring.obj
 0002:0001af78       $chain$1$ustring_GetCurrentDir 0000000180070f78     ustring.obj
 0002:0001af8c       $chain$2$ustring_GetCurrentDir 0000000180070f8c     ustring.obj
 0002:0001af9c       $chain$3$ustring_GetCurrentDir 0000000180070f9c     ustring.obj
 0002:0001afac       $chain$2$ustring_SetCurrentDir 0000000180070fac     ustring.obj
 0002:0001afc8       $chain$3$ustring_SetCurrentDir 0000000180070fc8     ustring.obj
 0002:0001afd8       $chain$0$GetFileTimeFromTable 0000000180070fd8     util.obj
 0002:0001afec       $chain$1$GetFileTimeFromTable 0000000180070fec     util.obj
 0002:0001affc       $unwind$PutFileTimeToTable 0000000180070ffc     util.obj
 0002:0001affc       $unwind$__acrt_lowio_destroy_handle_array 0000000180070ffc     libucrt:osfinfo.obj
 0002:0001b00c       $unwind$win_DeleteRegKey   000000018007100c     win.obj
 0002:0001b00c       $unwind$win_SetEnv         000000018007100c     win.obj
 0002:0001b01c       $chain$0$win_SetEnv        000000018007101c     win.obj
 0002:0001b030       $chain$1$win_SetEnv        0000000180071030     win.obj
 0002:0001b040       $unwind$win_SetRegKey      0000000180071040     win.obj
 0002:0001b058       $chain$1$win_SetRegKey     0000000180071058     win.obj
 0002:0001b06c       $unwind$win_GetRegKey      000000018007106c     win.obj
 0002:0001b07c       $chain$1$win_GetRegKey     000000018007107c     win.obj
 0002:0001b094       $chain$2$win_GetRegKey     0000000180071094     win.obj
 0002:0001b0a8       $chain$0$win_DeleteRegKey  00000001800710a8     win.obj
 0002:0001b0bc       $chain$1$win_DeleteRegKey  00000001800710bc     win.obj
 0002:0001b0cc       $unwind$win_DeleteRegValue 00000001800710cc     win.obj
 0002:0001b0d8       $chain$4$win_DeleteRegValue 00000001800710d8     win.obj
 0002:0001b0fc       $chain$5$win_DeleteRegValue 00000001800710fc     win.obj
 0002:0001b11c       $chain$6$win_DeleteRegValue 000000018007111c     win.obj
 0002:0001b130       $unwind$win_EnumRegKey     0000000180071130     win.obj
 0002:0001b130       $unwind$win_EnumRegValue   0000000180071130     win.obj
 0002:0001b154       $unwind$win_ExtractKey     0000000180071154     win.obj
 0002:0001b154       $unwind$win_ExtractKeyEx   0000000180071154     win.obj
 0002:0001b168       $chain$0$PushWinFindData   0000000180071168     win.obj
 0002:0001b17c       $chain$1$PushWinFindData   000000018007117c     win.obj
 0002:0001b18c       $unwind$win_GetFileInfo    000000018007118c     win.obj
 0002:0001b1ac       $unwind$win_CompareString  00000001800711ac     win.obj
 0002:0001b1c4       $unwind$win_GetConsoleScreenBufferInfo 00000001800711c4     win.obj
 0002:0001b1d4       $chain$0$win_GetConsoleScreenBufferInfo 00000001800711d4     win.obj
 0002:0001b1e8       $chain$1$win_GetConsoleScreenBufferInfo 00000001800711e8     win.obj
 0002:0001b1f8       $unwind$win_MoveFile       00000001800711f8     win.obj
 0002:0001b210       $chain$2$win_DeleteFile    0000000180071210     win.obj
 0002:0001b22c       $chain$3$win_DeleteFile    000000018007122c     win.obj
 0002:0001b23c       $unwind$mkdir              000000018007123c     win.obj
 0002:0001b254       $chain$0$mkdir             0000000180071254     win.obj
 0002:0001b268       $chain$2$win_RemoveDir     0000000180071268     win.obj
 0002:0001b284       $chain$3$win_RemoveDir     0000000180071284     win.obj
 0002:0001b294       $unwind$win_ShellExecute   0000000180071294     win.obj
 0002:0001b2a8       $chain$0$win_ShellExecute  00000001800712a8     win.obj
 0002:0001b2bc       $chain$1$win_ShellExecute  00000001800712bc     win.obj
 0002:0001b2cc       $unwind$win_WriteConsole   00000001800712cc     win.obj
 0002:0001b2ec       $unwind$win_IsWinVersion   00000001800712ec     win.obj
 0002:0001b30c       $chain$1$win_IsWinVersion  000000018007130c     win.obj
 0002:0001b324       $chain$2$win_IsWinVersion  0000000180071324     win.obj
 0002:0001b334       $unwind$win_GetFileTimes   0000000180071334     win.obj
 0002:0001b334       $unwind$win_SetFileTimes   0000000180071334     win.obj
 0002:0001b348       $xdatasym                  0000000180071348     LIBCMT:amdsecgs.obj
 0002:0001b34c       $unwind$__report_securityfailure 000000018007134c     LIBCMT:gs_report.obj
 0002:0001b354       $unwind$__report_gsfailure 0000000180071354     LIBCMT:gs_report.obj
 0002:0001b35c       $unwind$?dllmain_crt_process_attach@@YAHQEAUHINSTANCE__@@QEAX@Z 000000018007135c     LIBCMT:dll_dllmain.obj
 0002:0001b398       $unwind$?fin$0@?0??dllmain_crt_process_attach@@YAHQEAUHINSTANCE__@@QEAX@Z@4HA 0000000180071398     LIBCMT:dll_dllmain.obj
 0002:0001b398       $unwind$?fin$0@?0??dllmain_crt_process_detach@@YAH_N@Z@4HA 0000000180071398     LIBCMT:dll_dllmain.obj
 0002:0001b398       $unwind$?fin$1@?0??dllmain_crt_process_detach@@YAH_N@Z@4HA 0000000180071398     LIBCMT:dll_dllmain.obj
 0002:0001b398       $unwind$_IsNonwritableInCurrentImage$filt$0 0000000180071398     LIBCMT:pesect.obj
 0002:0001b398       $unwind$?fin$0@?0???$common_popen@_W@@YAPEAU_iobuf@@QEB_W0@Z@4HA 0000000180071398     libucrt:popen.obj
 0002:0001b398       $unwind$_pclose$fin$0      0000000180071398     libucrt:popen.obj
 0002:0001b398       $unwind$?fin$0@?0???$common_getenv@_W@@YAPEA_WQEB_W@Z@4HA 0000000180071398     libucrt:getenv.obj
 0002:0001b398       $unwind$?fin$0@?0???$?RV<lambda_24016bbcb8f60cbe41e899a2382ed12a>@@AEAV<lambda_f9f2d660215b636168e2032e31cf969c>@@V<lambda_7fbd5cec917a4378cbcd803f78c7a734>@@@?$__crt_seh_guarded_call@_N@@QEAA_N$$QEAV<lambda_24016bbcb8f60cbe41e899a2382ed12a>@@AEAV<lambda_f9f2d660215b636168e2032e31cf969c>@@$$QEAV<lambda_7fbd5cec917a4378cbcd803f78c7a734>@@@Z@4HA 0000000180071398     libucrt:spawnv.obj
 0002:0001b398       $unwind$_query_new_handler$fin$0 0000000180071398     libucrt:new_handler.obj
 0002:0001b398       $unwind$?fin$0@?0???$?RV<lambda_0ae27a3a962d80f24befdcbee591983d>@@AEAV<lambda_8d0ee55de4b1038c4002e0adecdf1839>@@V<lambda_dc504788e8f1664fe9b84e20bfb512f2>@@@?$__crt_seh_guarded_call@X@@QEAAX$$QEAV<lambda_0ae27a3a962d80f24befdcbee591983d>@@AEAV<lambda_8d0ee55de4b1038c4002e0adecdf1839>@@$$QEAV<lambda_dc504788e8f1664fe9b84e20bfb512f2>@@@Z@4HA 0000000180071398     libucrt:per_thread_data.obj
 0002:0001b398       $unwind$?fin$0@?0???$?RV<lambda_2d41944a1d46af3157314b8a01080d33>@@AEAV<lambda_8f455de75cd7d7f24b4096f044d8b9e6>@@V<lambda_aa500f224e6afead328df44964fe2772>@@@?$__crt_seh_guarded_call@X@@QEAAX$$QEAV<lambda_2d41944a1d46af3157314b8a01080d33>@@AEAV<lambda_8f455de75cd7d7f24b4096f044d8b9e6>@@$$QEAV<lambda_aa500f224e6afead328df44964fe2772>@@@Z@4HA 0000000180071398     libucrt:per_thread_data.obj
 0002:0001b398       $unwind$?fin$0@?0???$?RV<lambda_aa87e3671a710a21b5dc78c0bdf72e11>@@AEAV<lambda_92619d2358a28f41a33ba319515a20b9>@@V<lambda_6992ecaafeb10aed2b74cb1fae11a551>@@@?$__crt_seh_guarded_call@X@@QEAAX$$QEAV<lambda_aa87e3671a710a21b5dc78c0bdf72e11>@@AEAV<lambda_92619d2358a28f41a33ba319515a20b9>@@$$QEAV<lambda_6992ecaafeb10aed2b74cb1fae11a551>@@@Z@4HA 0000000180071398     libucrt:per_thread_data.obj
 0002:0001b398       $unwind$?fin$0@?0???$?RV<lambda_f2e299630e499de9f9a165e60fcd3db5>@@AEAV<lambda_2ae9d31cdba2644fcbeaf08da7c24588>@@V<lambda_40d01ff24d0e7b3814fdbdcee8eab3c7>@@@?$__crt_seh_guarded_call@X@@QEAAX$$QEAV<lambda_f2e299630e499de9f9a165e60fcd3db5>@@AEAV<lambda_2ae9d31cdba2644fcbeaf08da7c24588>@@$$QEAV<lambda_40d01ff24d0e7b3814fdbdcee8eab3c7>@@@Z@4HA 0000000180071398     libucrt:per_thread_data.obj
 0002:0001b398       $unwind$__acrt_update_thread_locale_data$fin$0 0000000180071398     libucrt:locale_refcounting.obj
 0002:0001b398       $unwind$?fin$0@?0???$?RV<lambda_410d79af7f07d98d83a3f525b3859a53>@@AEAV<lambda_3e16ef9562a7dcce91392c22ab16ea36>@@V<lambda_38119f0e861e05405d8a144b9b982f0a>@@@?$__crt_seh_guarded_call@X@@QEAAX$$QEAV<lambda_410d79af7f07d98d83a3f525b3859a53>@@AEAV<lambda_3e16ef9562a7dcce91392c22ab16ea36>@@$$QEAV<lambda_38119f0e861e05405d8a144b9b982f0a>@@@Z@4HA 0000000180071398     libucrt:wsetlocale.obj
 0002:0001b398       $unwind$?fin$0@?0???$?RV<lambda_751a882b2c74d4b022dec766aa51a29a>@@AEAV<lambda_628dfdc04ba53c8bfc02c9951375f3f5>@@V<lambda_f6c7be5f7998530c34de24c7437d6b54>@@@?$__crt_seh_guarded_call@H@@QEAAH$$QEAV<lambda_751a882b2c74d4b022dec766aa51a29a>@@AEAV<lambda_628dfdc04ba53c8bfc02c9951375f3f5>@@$$QEAV<lambda_f6c7be5f7998530c34de24c7437d6b54>@@@Z@4HA 0000000180071398     libucrt:close.obj
 0002:0001b398       $unwind$?fin$0@?0???$?RV<lambda_a37b2b86f63e897a80ea819b0eb08c01>@@AEAV<lambda_38ce7e780aa69e748d6df282ebc68efe>@@V<lambda_99fb1378e971ab6e7edea83e3a7a83a2>@@@?$__crt_seh_guarded_call@H@@QEAAH$$QEAV<lambda_a37b2b86f63e897a80ea819b0eb08c01>@@AEAV<lambda_38ce7e780aa69e748d6df282ebc68efe>@@$$QEAV<lambda_99fb1378e971ab6e7edea83e3a7a83a2>@@@Z@4HA 0000000180071398     libucrt:commit.obj
 0002:0001b398       $unwind$__acrt_initialize_lowio$fin$0 0000000180071398     libucrt:ioinit.obj
 0002:0001b398       $unwind$?fin$0@?0???$common_lseek@J@@YAJHJH@Z@4HA 0000000180071398     libucrt:lseek.obj
 0002:0001b398       $unwind$?fin$0@?0???$common_lseek@_J@@YA_JH_JH@Z@4HA 0000000180071398     libucrt:lseek.obj
 0002:0001b398       $unwind$__acrt_lowio_ensure_fh_exists$fin$0 0000000180071398     libucrt:osfinfo.obj
 0002:0001b398       $unwind$_alloc_osfhnd$fin$0 0000000180071398     libucrt:osfinfo.obj
 0002:0001b398       $unwind$_read$fin$0        0000000180071398     libucrt:read.obj
 0002:0001b398       $unwind$_write$fin$0       0000000180071398     libucrt:write.obj
 0002:0001b398       $unwind$?fin$0@?0???$?RV<lambda_efdfa57d1f175319df784efa44bb7b81>@@AEAV<lambda_5f0a4c1567f8adc6734073e5d1e1b35c>@@V<lambda_2e8a7d3640ea6ccb4c2413664c2db6fd>@@@?$__crt_seh_guarded_call@X@@QEAAX$$QEAV<lambda_efdfa57d1f175319df784efa44bb7b81>@@AEAV<lambda_5f0a4c1567f8adc6734073e5d1e1b35c>@@$$QEAV<lambda_2e8a7d3640ea6ccb4c2413664c2db6fd>@@@Z@4HA 0000000180071398     libucrt:mbctype.obj
 0002:0001b398       $unwind$?fin$0@?0??update_thread_multibyte_data_internal@@YAPEAU__crt_multibyte_data@@QEAU__acrt_ptd@@QEAPEAU1@@Z@4HA 0000000180071398     libucrt:mbctype.obj
 0002:0001b398       $unwind$?fin$0@?0???$?RV<lambda_450d765d439847d4c735a33c368b5fc0>@@AEAV<lambda_44731a7d0e6d81c3e6aa82d741081786>@@V<lambda_601a2a7da3b7a96e9554ac7215c4b07c>@@@?$__crt_seh_guarded_call@P6AXH@Z@@QEAAP6AXH@Z$$QEAV<lambda_450d765d439847d4c735a33c368b5fc0>@@AEAV<lambda_44731a7d0e6d81c3e6aa82d741081786>@@$$QEAV<lambda_601a2a7da3b7a96e9554ac7215c4b07c>@@@Z@4HA 0000000180071398     libucrt:signal.obj
 0002:0001b398       $unwind$raise$fin$0        0000000180071398     libucrt:signal.obj
 0002:0001b398       $unwind$?filt$0@?0???R<lambda_6e4b09c48022b2350581041d5f6b0c4c>@@QEBA@XZ@4HA 0000000180071398     libucrt:exit.obj
 0002:0001b398       $unwind$?fin$0@?0???$?RV<lambda_d80eeec6fff315bfe5c115232f3240e3>@@AEAV<lambda_6e4b09c48022b2350581041d5f6b0c4c>@@V<lambda_2358e3775559c9db80273638284d5e45>@@@?$__crt_seh_guarded_call@X@@QEAAX$$QEAV<lambda_d80eeec6fff315bfe5c115232f3240e3>@@AEAV<lambda_6e4b09c48022b2350581041d5f6b0c4c>@@$$QEAV<lambda_2358e3775559c9db80273638284d5e45>@@@Z@4HA 0000000180071398     libucrt:exit.obj
 0002:0001b398       $unwind$?fin$0@?0???$?RV<lambda_7777bce6b2f8c936911f934f8298dc43>@@AEAV<lambda_f03950bc5685219e0bcd2087efbe011e>@@V<lambda_3883c3dff614d5e0c5f61bb1ac94921c>@@@?$__crt_seh_guarded_call@H@@QEAAH$$QEAV<lambda_7777bce6b2f8c936911f934f8298dc43>@@AEAV<lambda_f03950bc5685219e0bcd2087efbe011e>@@$$QEAV<lambda_3883c3dff614d5e0c5f61bb1ac94921c>@@@Z@4HA 0000000180071398     libucrt:onexit.obj
 0002:0001b398       $unwind$clearerr_s$fin$0   0000000180071398     libucrt:clearerr.obj
 0002:0001b398       $unwind$_fcloseall$fin$0   0000000180071398     libucrt:closeall.obj
 0002:0001b398       $unwind$fclose$fin$0       0000000180071398     libucrt:fclose.obj
 0002:0001b398       $unwind$?fin$0@?0???$common_fdopen@_W@@YAPEAU_iobuf@@HQEB_W@Z@4HA 0000000180071398     libucrt:fdopen.obj
 0002:0001b398       $unwind$?fin$0@?0???$?RV<lambda_842d9ff0dc9ef11c61343bbaebe7f885>@@AEAV<lambda_c5860995281e5c4ce005b3de8f5874ee>@@V<lambda_d90129c13df834fdcbf8d2b88dafcf2d>@@@?$__crt_seh_guarded_call@X@@QEAAX$$QEAV<lambda_842d9ff0dc9ef11c61343bbaebe7f885>@@AEAV<lambda_c5860995281e5c4ce005b3de8f5874ee>@@$$QEAV<lambda_d90129c13df834fdcbf8d2b88dafcf2d>@@@Z@4HA 0000000180071398     libucrt:fflush.obj
 0002:0001b398       $unwind$?fin$0@?0???$?RV<lambda_886d6c58226a84441f68b9f2b8217b83>@@AEAV<lambda_ab61a845afdef5b7c387490eaf3616ee>@@V<lambda_f7f22ab5edc0698d5f6905b0d3f44752>@@@?$__crt_seh_guarded_call@X@@QEAAX$$QEAV<lambda_886d6c58226a84441f68b9f2b8217b83>@@AEAV<lambda_ab61a845afdef5b7c387490eaf3616ee>@@$$QEAV<lambda_f7f22ab5edc0698d5f6905b0d3f44752>@@@Z@4HA 0000000180071398     libucrt:fflush.obj
 0002:0001b398       $unwind$?fin$0@?0???$?RV<lambda_c376a267cfb53b6959b3b692ec76b120>@@AEAV<lambda_9a32fed5bf61b6b509b2d3f6003082a1>@@V<lambda_572fbb9fa0ab338edf41edfd4b5fcc8d>@@@?$__crt_seh_guarded_call@H@@QEAAH$$QEAV<lambda_c376a267cfb53b6959b3b692ec76b120>@@AEAV<lambda_9a32fed5bf61b6b509b2d3f6003082a1>@@$$QEAV<lambda_572fbb9fa0ab338edf41edfd4b5fcc8d>@@@Z@4HA 0000000180071398     libucrt:fflush.obj
 0002:0001b398       $unwind$fgetc$fin$0        0000000180071398     libucrt:fgetc.obj
 0002:0001b398       $unwind$?fin$0@?0???$common_fgets@D@@YAPEADQEADHV__crt_stdio_stream@@@Z@4HA 0000000180071398     libucrt:fgets.obj
 0002:0001b398       $unwind$?fin$0@?0???$common_fsopen@_W@@YAPEAU_iobuf@@QEB_W0H@Z@4HA 0000000180071398     libucrt:fopen.obj
 0002:0001b398       $unwind$?fin$0@?0???$common_freopen@_W@@YAHQEAPEAU_iobuf@@QEB_W1V__crt_stdio_stream@@H@Z@4HA 0000000180071398     libucrt:freopen.obj
 0002:0001b398       $unwind$?fin$0@?0??common_fseek@@YAHV__crt_stdio_stream@@_JH@Z@4HA 0000000180071398     libucrt:fseek.obj
 0002:0001b398       $unwind$?fin$0@?0???$common_ftell@_J@@YA_JV__crt_stdio_stream@@@Z@4HA 0000000180071398     libucrt:ftell.obj
 0002:0001b398       $unwind$?fin$0@?0???$?RV<lambda_2831f20263db5b546e098b45503eb778>@@AEAV<lambda_5856287d7ecd2be6c9197bb4007c3f6e>@@V<lambda_0838d7e100fbcbd261b69cfea6abb102>@@@?$__crt_seh_guarded_call@_K@@QEAA_K$$QEAV<lambda_2831f20263db5b546e098b45503eb778>@@AEAV<lambda_5856287d7ecd2be6c9197bb4007c3f6e>@@$$QEAV<lambda_0838d7e100fbcbd261b69cfea6abb102>@@@Z@4HA 0000000180071398     libucrt:fwrite.obj
 0002:0001b398       $unwind$?fin$0@?0???$?RV<lambda_082dd7c0feb7dbdaf245f261e54a6583>@@AEAV<lambda_f3caf1ecae5fe01a9a1a6239afa44510>@@V<lambda_c640b76c0755ae85b317b35c67c61e6b>@@@?$__crt_seh_guarded_call@H@@QEAAH$$QEAV<lambda_082dd7c0feb7dbdaf245f261e54a6583>@@AEAV<lambda_f3caf1ecae5fe01a9a1a6239afa44510>@@$$QEAV<lambda_c640b76c0755ae85b317b35c67c61e6b>@@@Z@4HA 0000000180071398     libucrt:input.obj
 0002:0001b398       $unwind$?fin$0@?0???$?RV<lambda_fe5404e9642edbb7c8ae71e1dcfa4018>@@AEAV<lambda_36eeb330e99a4f0bf8a7da86d0894cb9>@@V<lambda_2fa474834de80dc12f7a3c6eddd7a366>@@@?$__crt_seh_guarded_call@H@@QEAAH$$QEAV<lambda_fe5404e9642edbb7c8ae71e1dcfa4018>@@AEAV<lambda_36eeb330e99a4f0bf8a7da86d0894cb9>@@$$QEAV<lambda_2fa474834de80dc12f7a3c6eddd7a366>@@@Z@4HA 0000000180071398     libucrt:output.obj
 0002:0001b398       $unwind$rewind$fin$0       0000000180071398     libucrt:rewind.obj
 0002:0001b398       $unwind$_rmtmp$fin$0       0000000180071398     libucrt:rmtmp.obj
 0002:0001b398       $unwind$_rmtmp$fin$1       0000000180071398     libucrt:rmtmp.obj
 0002:0001b398       $unwind$?fin$0@?0???$?RV<lambda_84ec643ea9557e2f7dc01bb0e9624395>@@AEAV<lambda_ca71763b3c0644891230e4f79ea54fa6>@@V<lambda_439a761618c59b0600e24586724d733b>@@@?$__crt_seh_guarded_call@H@@QEAAH$$QEAV<lambda_84ec643ea9557e2f7dc01bb0e9624395>@@AEAV<lambda_ca71763b3c0644891230e4f79ea54fa6>@@$$QEAV<lambda_439a761618c59b0600e24586724d733b>@@@Z@4HA 0000000180071398     libucrt:setvbuf.obj
 0002:0001b398       $unwind$?fin$0@?0??__acrt_stdio_allocate_stream@@YA?AV__crt_stdio_stream@@XZ@4HA 0000000180071398     libucrt:stream.obj
 0002:0001b398       $unwind$?fin$0@?0??common_tmpfile@@YAHQEAPEAU_iobuf@@H@Z@4HA 0000000180071398     libucrt:tmpfile.obj
 0002:0001b398       $unwind$ungetc$fin$0       0000000180071398     libucrt:ungetc.obj
 0002:0001b398       $unwind$_ctrlfp$filt$0     0000000180071398     libucrt:fpctrl.obj
 0002:0001b398       $unwind$common_control87$filt$0 0000000180071398     libucrt:ieee.obj
 0002:0001b3a0       $unwind$?dllmain_crt_process_detach@@YAH_N@Z 00000001800713a0     LIBCMT:dll_dllmain.obj
 0002:0001b3f4       $unwind$?dllmain_dispatch@@YAHQEAUHINSTANCE__@@KQEAX@Z 00000001800713f4     LIBCMT:dll_dllmain.obj
 0002:0001b41c       $unwind$?filt$0@?0??dllmain_dispatch@@YAHQEAUHINSTANCE__@@KQEAX@Z@4HA 000000018007141c     LIBCMT:dll_dllmain.obj
 0002:0001b41c       $unwind$_pipe$fin$0        000000018007141c     libucrt:pipe.obj
 0002:0001b41c       $unwind$_pipe$fin$1        000000018007141c     libucrt:pipe.obj
 0002:0001b41c       $unwind$?fin$0@?0???$common_dupenv_s@_W@@YAHQEAPEA_WQEA_KQEB_WHQEBDH@Z@4HA 000000018007141c     libucrt:getenv.obj
 0002:0001b41c       $unwind$fread_s$fin$0      000000018007141c     libucrt:fread.obj
 0002:0001b41c       $unwind$?fin$0@?0??common_tmpfile_nolock@@YAHQEAPEAU_iobuf@@H@Z@4HA 000000018007141c     libucrt:tmpfile.obj
 0002:0001b424       $unwind$__security_init_cookie 0000000180071424     LIBCMT:gs_support.obj
 0002:0001b430       $unwind$__scrt_is_nonwritable_in_current_image 0000000180071430     LIBCMT:utility.obj
 0002:0001b450       $unwind$__scrt_is_nonwritable_in_current_image$filt$0 0000000180071450     LIBCMT:utility.obj
 0002:0001b458       $unwind$__scrt_fastfail    0000000180071458     LIBCMT:utility_desktop.obj
 0002:0001b468       $unwind$__isa_available_init 0000000180071468     LIBCMT:cpu_disp.obj
 0002:0001b478       $xdatasym                  0000000180071478     LIBCMT:guard_dispatch.obj
 0002:0001b480       $xdatasym                  0000000180071480     LIBCMT:guard_xfg_dispatch.obj
 0002:0001b484       $unwind$wcsstr             0000000180071484     libvcruntime:wcsstr.obj
 0002:0001b498       $unwind$__C_specific_handler 0000000180071498     libvcruntime:riscchandler.obj
 0002:0001b4b4       $unwind$__DestructExceptionObject 00000001800714b4     libvcruntime:ehhelpers.obj
 0002:0001b4d4       $unwind$__DestructExceptionObject$filt$0 00000001800714d4     libvcruntime:ehhelpers.obj
 0002:0001b4e0       $xdatasym                  00000001800714e0     libvcruntime:memset.obj
 0002:0001b4f0       $xdatasym                  00000001800714f0     libvcruntime:notify.obj
 0002:0001b500       $xdatasym                  0000000180071500     libvcruntime:memcpy.obj
 0002:0001b510       $xdatasym                  0000000180071510     libvcruntime:handlers.obj
 0002:0001b530       $unwind$__stdio_common_vfscanf 0000000180071530     libucrt:input.obj
 0002:0001b530       $unwind$__stdio_common_vfprintf 0000000180071530     libucrt:output.obj
 0002:0001b538       $unwind$??$common_vsprintf@Vstandard_base@__crt_stdio_output@@D@@YAH_KQEAD0QEBDQEAU__crt_locale_pointers@@1@Z 0000000180071538     libucrt:output.obj
 0002:0001b538       $unwind$??$common_vsprintf@Vstandard_base@__crt_stdio_output@@_W@@YAH_KQEA_W0QEB_WQEAU__crt_locale_pointers@@QEAD@Z 0000000180071538     libucrt:output.obj
 0002:0001b558       $unwind$_chsize_nolock     0000000180071558     libucrt:chsize.obj
 0002:0001b558       $unwind$??$parse_command_line@D@@YAXPEADPEAPEAD0PEA_K2@Z 0000000180071558     libucrt:argv_parsing.obj
 0002:0001b558       $unwind$?write_string_impl@?$output_adapter_common@DV?$stream_output_adapter@D@__crt_stdio_output@@@__crt_stdio_output@@IEBAXQEBDHQEAHAEAV__crt_deferred_errno_cache@@@Z 0000000180071558     libucrt:output.obj
 0002:0001b574       $unwind$?truncate_ctrl_z_if_present@@YAHH@Z 0000000180071574     libucrt:open.obj
 0002:0001b574       $unwind$?process@?$output_processor@DV?$stream_output_adapter@D@__crt_stdio_output@@V?$standard_base@DV?$stream_output_adapter@D@__crt_stdio_output@@@2@@__crt_stdio_output@@QEAAHXZ 0000000180071574     libucrt:output.obj
 0002:0001b574       $unwind$?process@?$output_processor@DV?$string_output_adapter@D@__crt_stdio_output@@V?$standard_base@DV?$string_output_adapter@D@__crt_stdio_output@@@2@@__crt_stdio_output@@QEAAHXZ 0000000180071574     libucrt:output.obj
 0002:0001b584       $unwind$?parse_int_from_format_string@?$output_processor@DV?$stream_output_adapter@D@__crt_stdio_output@@V?$standard_base@DV?$stream_output_adapter@D@__crt_stdio_output@@@2@@__crt_stdio_output@@AEAA_NQEAH@Z 0000000180071584     libucrt:output.obj
 0002:0001b584       $unwind$?parse_int_from_format_string@?$output_processor@DV?$string_output_adapter@D@__crt_stdio_output@@V?$standard_base@DV?$string_output_adapter@D@__crt_stdio_output@@@2@@__crt_stdio_output@@AEAA_NQEAH@Z 0000000180071584     libucrt:output.obj
 0002:0001b584       $unwind$?process@?$output_processor@_WV?$string_output_adapter@_W@__crt_stdio_output@@V?$standard_base@_WV?$string_output_adapter@_W@__crt_stdio_output@@@2@@__crt_stdio_output@@QEAAHXZ 0000000180071584     libucrt:output.obj
 0002:0001b598       $unwind$?configure_text_mode@@YAHHUfile_options@?A0xa9d50aae@@HAEAW4__crt_lowio_text_mode@@@Z 0000000180071598     libucrt:open.obj
 0002:0001b598       $unwind$?state_case_type@?$output_processor@DV?$stream_output_adapter@D@__crt_stdio_output@@V?$standard_base@DV?$stream_output_adapter@D@__crt_stdio_output@@@2@@__crt_stdio_output@@AEAA_NXZ 0000000180071598     libucrt:output.obj
 0002:0001b598       $unwind$?state_case_type@?$output_processor@DV?$string_output_adapter@D@__crt_stdio_output@@V?$standard_base@DV?$string_output_adapter@D@__crt_stdio_output@@@2@@__crt_stdio_output@@AEAA_NXZ 0000000180071598     libucrt:output.obj
 0002:0001b5b0       $unwind$?type_case_a@?$output_processor@DV?$stream_output_adapter@D@__crt_stdio_output@@V?$standard_base@DV?$stream_output_adapter@D@__crt_stdio_output@@@2@@__crt_stdio_output@@AEAA_NXZ 00000001800715b0     libucrt:output.obj
 0002:0001b5b0       $unwind$?type_case_a@?$output_processor@DV?$string_output_adapter@D@__crt_stdio_output@@V?$standard_base@DV?$string_output_adapter@D@__crt_stdio_output@@@2@@__crt_stdio_output@@AEAA_NXZ 00000001800715b0     libucrt:output.obj
 0002:0001b5bc       $unwind$?write_stored_string_tchar@?$output_processor@DV?$stream_output_adapter@D@__crt_stdio_output@@V?$standard_base@DV?$stream_output_adapter@D@__crt_stdio_output@@@2@@__crt_stdio_output@@AEAA_ND@Z 00000001800715bc     libucrt:output.obj
 0002:0001b5bc       $unwind$?write_stored_string_tchar@?$output_processor@DV?$string_output_adapter@D@__crt_stdio_output@@V?$standard_base@DV?$string_output_adapter@D@__crt_stdio_output@@@2@@__crt_stdio_output@@AEAA_ND@Z 00000001800715bc     libucrt:output.obj
 0002:0001b5d4       $unwind$??R<lambda_36eeb330e99a4f0bf8a7da86d0894cb9>@@QEBAHXZ 00000001800715d4     libucrt:output.obj
 0002:0001b5f4       $unwind$??$write_multiple_characters@V?$stream_output_adapter@D@__crt_stdio_output@@D@__crt_stdio_output@@YAXAEBV?$stream_output_adapter@D@0@DHQEAH@Z 00000001800715f4     libucrt:output.obj
 0002:0001b5f4       $unwind$?write_string@?$string_output_adapter@D@__crt_stdio_output@@QEBAXQEBDHQEAHAEAV__crt_deferred_errno_cache@@@Z 00000001800715f4     libucrt:output.obj
 0002:0001b60c       $unwind$?write_string@?$string_output_adapter@_W@__crt_stdio_output@@QEBAXQEB_WHQEAHAEAV__crt_deferred_errno_cache@@@Z 000000018007160c     libucrt:output.obj
 0002:0001b624       $unwind$?parse_int_from_format_string@?$output_processor@_WV?$string_output_adapter@_W@__crt_stdio_output@@V?$standard_base@_WV?$string_output_adapter@_W@__crt_stdio_output@@@2@@__crt_stdio_output@@AEAA_NQEAH@Z 0000000180071624     libucrt:output.obj
 0002:0001b638       $unwind$?state_case_type@?$output_processor@_WV?$string_output_adapter@_W@__crt_stdio_output@@V?$standard_base@_WV?$string_output_adapter@_W@__crt_stdio_output@@@2@@__crt_stdio_output@@AEAA_NXZ 0000000180071638     libucrt:output.obj
 0002:0001b65c       $unwind$?type_case_a@?$output_processor@_WV?$string_output_adapter@_W@__crt_stdio_output@@V?$standard_base@_WV?$string_output_adapter@_W@__crt_stdio_output@@@2@@__crt_stdio_output@@AEAA_NXZ 000000018007165c     libucrt:output.obj
 0002:0001b66c       $unwind$?write_stored_string_tchar@?$output_processor@_WV?$string_output_adapter@_W@__crt_stdio_output@@V?$standard_base@_WV?$string_output_adapter@_W@__crt_stdio_output@@@2@@__crt_stdio_output@@AEAA_N_W@Z 000000018007166c     libucrt:output.obj
 0002:0001b680       $unwind$??$write_multiple_characters@V?$string_output_adapter@D@__crt_stdio_output@@D@__crt_stdio_output@@YAXAEBV?$string_output_adapter@D@0@DHQEAH@Z 0000000180071680     libucrt:output.obj
 0002:0001b680       $unwind$??$write_multiple_characters@V?$string_output_adapter@_W@__crt_stdio_output@@D@__crt_stdio_output@@YAXAEBV?$string_output_adapter@_W@0@DHQEAH@Z 0000000180071680     libucrt:output.obj
 0002:0001b68c       $unwind$??$?RV<lambda_fe5404e9642edbb7c8ae71e1dcfa4018>@@AEAV<lambda_36eeb330e99a4f0bf8a7da86d0894cb9>@@V<lambda_2fa474834de80dc12f7a3c6eddd7a366>@@@?$__crt_seh_guarded_call@H@@QEAAH$$QEAV<lambda_fe5404e9642edbb7c8ae71e1dcfa4018>@@AEAV<lambda_36eeb330e99a4f0bf8a7da86d0894cb9>@@$$QEAV<lambda_2fa474834de80dc12f7a3c6eddd7a366>@@@Z 000000018007168c     libucrt:output.obj
 0002:0001b6b0       $unwind$fclose             00000001800716b0     libucrt:fclose.obj
 0002:0001b6d4       $unwind$common_control87   00000001800716d4     libucrt:ieee.obj
 0002:0001b700       $unwind$??$common_fsopen@_W@@YAPEAU_iobuf@@QEB_W0H@Z 0000000180071700     libucrt:fopen.obj
 0002:0001b72c       $unwind$__GSHandlerCheck_SEH 000000018007172c     LIBCMT:gshandlerseh.obj
 0002:0001b72c       $unwind$??$common_xtox@_KD@@YAH_KQEAD0I_N@Z 000000018007172c     libucrt:xtoa.obj
 0002:0001b72c       $unwind$?initialize_stdio_handles_nolock@@YAXXZ 000000018007172c     libucrt:ioinit.obj
 0002:0001b72c       $unwind$__acrt_lowio_set_os_handle 000000018007172c     libucrt:osfinfo.obj
 0002:0001b72c       $unwind$__acrt_initialize_stdio 000000018007172c     libucrt:_file.obj
 0002:0001b72c       $unwind$??$__acrt_stdio_parse_mode@_W@@YA?AU__acrt_stdio_stream_mode@@QEB_W@Z 000000018007172c     libucrt:openfile.obj
 0002:0001b744       $unwind$fgetc              0000000180071744     libucrt:fgetc.obj
 0002:0001b778       $unwind$??$common_freopen@_W@@YAHQEAPEAU_iobuf@@QEB_W1V__crt_stdio_stream@@H@Z 0000000180071778     libucrt:freopen.obj
 0002:0001b7a4       $unwind$rewind             00000001800717a4     libucrt:rewind.obj
 0002:0001b7c8       $unwind$ungetc             00000001800717c8     libucrt:ungetc.obj
 0002:0001b7ec       $unwind$fread_s            00000001800717ec     libucrt:fread.obj
 0002:0001b81c       $unwind$_fread_nolock_s    000000018007181c     libucrt:fread.obj
 0002:0001b834       $unwind$__acrt_initialize_winapi_thunks 0000000180071834     libucrt:winapi_thunks.obj
 0002:0001b834       $unwind$wcsncpy            0000000180071834     libucrt:wcsncpy.obj
 0002:0001b840       $xdatasym                  0000000180071840     libucrt:strncmp.obj
 0002:0001b844       $unwind$_mbsdec_l          0000000180071844     libucrt:mbsdec.obj
 0002:0001b844       $unwind$isdigit            0000000180071844     libucrt:_ctype.obj
 0002:0001b844       $unwind$isspace            0000000180071844     libucrt:_ctype.obj
 0002:0001b844       $unwind$_stricmp_l         0000000180071844     libucrt:stricmp.obj
 0002:0001b844       $unwind$_strupr_s_l        0000000180071844     libucrt:strupr.obj
 0002:0001b850       $xdatasym                  0000000180071850     libucrt:strncpy.obj
 0002:0001b854       $unwind$_pclose            0000000180071854     libucrt:popen.obj
 0002:0001b87c       $unwind$??$common_popen@_W@@YAPEAU_iobuf@@QEB_W0@Z 000000018007187c     libucrt:popen.obj
 0002:0001b8ac       $unwind$??$common_popen_nolock@_W@@YAPEAU_iobuf@@QEB_W0HAEAY01H@Z 00000001800718ac     libucrt:popen.obj
 0002:0001b8cc       $unwind$?common_flush_all@@YAH_N@Z 00000001800718cc     libucrt:fflush.obj
 0002:0001b8d4       $unwind$??$?RV<lambda_842d9ff0dc9ef11c61343bbaebe7f885>@@AEAV<lambda_c5860995281e5c4ce005b3de8f5874ee>@@V<lambda_d90129c13df834fdcbf8d2b88dafcf2d>@@@?$__crt_seh_guarded_call@X@@QEAAX$$QEAV<lambda_842d9ff0dc9ef11c61343bbaebe7f885>@@AEAV<lambda_c5860995281e5c4ce005b3de8f5874ee>@@$$QEAV<lambda_d90129c13df834fdcbf8d2b88dafcf2d>@@@Z 00000001800718d4     libucrt:fflush.obj
 0002:0001b8f8       $unwind$??$?RV<lambda_886d6c58226a84441f68b9f2b8217b83>@@AEAV<lambda_ab61a845afdef5b7c387490eaf3616ee>@@V<lambda_f7f22ab5edc0698d5f6905b0d3f44752>@@@?$__crt_seh_guarded_call@X@@QEAAX$$QEAV<lambda_886d6c58226a84441f68b9f2b8217b83>@@AEAV<lambda_ab61a845afdef5b7c387490eaf3616ee>@@$$QEAV<lambda_f7f22ab5edc0698d5f6905b0d3f44752>@@@Z 00000001800718f8     libucrt:fflush.obj
 0002:0001b920       $unwind$??$?RV<lambda_c376a267cfb53b6959b3b692ec76b120>@@AEAV<lambda_9a32fed5bf61b6b509b2d3f6003082a1>@@V<lambda_572fbb9fa0ab338edf41edfd4b5fcc8d>@@@?$__crt_seh_guarded_call@H@@QEAAH$$QEAV<lambda_c376a267cfb53b6959b3b692ec76b120>@@AEAV<lambda_9a32fed5bf61b6b509b2d3f6003082a1>@@$$QEAV<lambda_572fbb9fa0ab338edf41edfd4b5fcc8d>@@@Z 0000000180071920     libucrt:fflush.obj
 0002:0001b944       $unwind$clearerr_s         0000000180071944     libucrt:clearerr.obj
 0002:0001b96c       $unwind$??$common_fgets@D@@YAPEADQEADHV__crt_stdio_stream@@@Z 000000018007196c     libucrt:fgets.obj
 0002:0001b998       $unwind$?common_tmpfile_nolock@@YAHQEAPEAU_iobuf@@H@Z 0000000180071998     libucrt:tmpfile.obj
 0002:0001b9c4       $unwind$??$copy_environment@_W@@YAPEAPEA_WQEAPEA_W@Z 00000001800719c4     libucrt:setenv.obj
 0002:0001b9c4       $unwind$??$__acrt_mbs_to_wcs_cp@U__crt_win32_buffer_internal_dynamic_resizing@@@@YAHQEBDAEAV?$__crt_win32_buffer@_WU__crt_win32_buffer_internal_dynamic_resizing@@@@I@Z 00000001800719c4     libucrt:createprocessa.obj
 0002:0001b9c4       $unwind$??$initialize_tmpfile_buffer_nolock@D@@YA_NW4buffer_id@?A0x5b9a7937@@@Z 00000001800719c4     libucrt:tmpfile.obj
 0002:0001b9dc       $unwind$?common_tmpfile@@YAHQEAPEAU_iobuf@@H@Z 00000001800719dc     libucrt:tmpfile.obj
 0002:0001ba00       $unwind$fwrite             0000000180071a00     libucrt:fwrite.obj
 0002:0001ba08       $unwind$??$?RV<lambda_2831f20263db5b546e098b45503eb778>@@AEAV<lambda_5856287d7ecd2be6c9197bb4007c3f6e>@@V<lambda_0838d7e100fbcbd261b69cfea6abb102>@@@?$__crt_seh_guarded_call@_K@@QEAA_K$$QEAV<lambda_2831f20263db5b546e098b45503eb778>@@AEAV<lambda_5856287d7ecd2be6c9197bb4007c3f6e>@@$$QEAV<lambda_0838d7e100fbcbd261b69cfea6abb102>@@@Z 0000000180071a08     libucrt:fwrite.obj
 0002:0001ba2c       $unwind$setvbuf            0000000180071a2c     libucrt:setvbuf.obj
 0002:0001ba34       $unwind$??$?RV<lambda_84ec643ea9557e2f7dc01bb0e9624395>@@AEAV<lambda_ca71763b3c0644891230e4f79ea54fa6>@@V<lambda_439a761618c59b0600e24586724d733b>@@@?$__crt_seh_guarded_call@H@@QEAAH$$QEAV<lambda_84ec643ea9557e2f7dc01bb0e9624395>@@AEAV<lambda_ca71763b3c0644891230e4f79ea54fa6>@@$$QEAV<lambda_439a761618c59b0600e24586724d733b>@@@Z 0000000180071a34     libucrt:setvbuf.obj
 0002:0001ba58       $unwind$?divide@__crt_strtox@@YA_KAEAUbig_integer@1@AEBU21@@Z 0000000180071a58     libucrt:input.obj
 0002:0001ba70       $chain$0$?divide@__crt_strtox@@YA_KAEAUbig_integer@1@AEBU21@@Z 0000000180071a70     libucrt:input.obj
 0002:0001ba84       $chain$1$?divide@__crt_strtox@@YA_KAEAUbig_integer@1@AEBU21@@Z 0000000180071a84     libucrt:input.obj
 0002:0001ba94       $unwind$?assemble_floating_point_value@__crt_strtox@@YA?AW4SLD_STATUS@@_KH_N1AEBVfloating_point_value@1@@Z 0000000180071a94     libucrt:input.obj
 0002:0001baac       $unwind$?assemble_floating_point_value_from_big_integer@__crt_strtox@@YA?AW4SLD_STATUS@@AEBUbig_integer@1@I_N1AEBVfloating_point_value@1@@Z 0000000180071aac     libucrt:input.obj
 0002:0001bac8       $unwind$?convert_decimal_string_to_floating_type_common@__crt_strtox@@YA?AW4SLD_STATUS@@AEBUfloating_point_string@1@AEBVfloating_point_value@1@@Z 0000000180071ac8     libucrt:input.obj
 0002:0001baec       $unwind$?write_character@?$input_processor@DV?$stream_input_adapter@D@__crt_stdio_input@@@__crt_stdio_input@@AEAA_NQEFA_W_KAEAPEFA_WAEA_KD@Z 0000000180071aec     libucrt:input.obj
 0002:0001bafc       $unwind$??R<lambda_f3caf1ecae5fe01a9a1a6239afa44510>@@QEBAHXZ 0000000180071afc     libucrt:input.obj
 0002:0001bb1c       $unwind$??$process_floating_point_specifier_t@M@?$input_processor@DV?$stream_input_adapter@D@__crt_stdio_input@@@__crt_stdio_input@@AEAA_NXZ 0000000180071b1c     libucrt:input.obj
 0002:0001bb1c       $unwind$??$process_floating_point_specifier_t@N@?$input_processor@DV?$stream_input_adapter@D@__crt_stdio_input@@@__crt_stdio_input@@AEAA_NXZ 0000000180071b1c     libucrt:input.obj
 0002:0001bb28       $unwind$??$parse_integer@_KV?$input_adapter_character_source@V?$stream_input_adapter@D@__crt_stdio_input@@@__crt_strtox@@@__crt_strtox@@YA_KQEAU__crt_locale_pointers@@V?$input_adapter_character_source@V?$stream_input_adapter@D@__crt_stdio_input@@@0@H_N@Z 0000000180071b28     libucrt:input.obj
 0002:0001bb44       $unwind$??$process_string_specifier_tchar@_W@?$input_processor@DV?$stream_input_adapter@D@__crt_stdio_input@@@__crt_stdio_input@@AEAA_NW4conversion_mode@1@_W@Z 0000000180071b44     libucrt:input.obj
 0002:0001bb5c       $unwind$??$?RV<lambda_082dd7c0feb7dbdaf245f261e54a6583>@@AEAV<lambda_f3caf1ecae5fe01a9a1a6239afa44510>@@V<lambda_c640b76c0755ae85b317b35c67c61e6b>@@@?$__crt_seh_guarded_call@H@@QEAAH$$QEAV<lambda_082dd7c0feb7dbdaf245f261e54a6583>@@AEAV<lambda_f3caf1ecae5fe01a9a1a6239afa44510>@@$$QEAV<lambda_c640b76c0755ae85b317b35c67c61e6b>@@@Z 0000000180071b5c     libucrt:input.obj
 0002:0001bb80       $unwind$??$parse_floating_point@V?$input_adapter_character_source@V?$stream_input_adapter@D@__crt_stdio_input@@@__crt_strtox@@M@__crt_strtox@@YA?AW4SLD_STATUS@@QEAU__crt_locale_pointers@@V?$input_adapter_character_source@V?$stream_input_adapter@D@__crt_stdio_input@@@0@QEAM@Z 0000000180071b80     libucrt:input.obj
 0002:0001bb80       $unwind$??$parse_floating_point@V?$input_adapter_character_source@V?$stream_input_adapter@D@__crt_stdio_input@@@__crt_strtox@@N@__crt_strtox@@YA?AW4SLD_STATUS@@QEAU__crt_locale_pointers@@V?$input_adapter_character_source@V?$stream_input_adapter@D@__crt_stdio_input@@@0@QEAN@Z 0000000180071b80     libucrt:input.obj
 0002:0001bb98       $unwind$??$parse_floating_point_from_source@V?$input_adapter_character_source@V?$stream_input_adapter@D@__crt_stdio_input@@@__crt_strtox@@@__crt_strtox@@YA?AW4floating_point_parse_result@0@QEAU__crt_locale_pointers@@AEAV?$input_adapter_character_source@V?$stream_input_adapter@D@__crt_stdio_input@@@0@AEAUfloating_point_string@0@@Z 0000000180071b98     libucrt:input.obj
 0002:0001bbb0       $unwind$??$parse_floating_point_possible_nan@DV?$input_adapter_character_source@V?$stream_input_adapter@D@__crt_stdio_input@@@__crt_strtox@@_K@__crt_strtox@@YA?AW4floating_point_parse_result@0@AEADAEAV?$input_adapter_character_source@V?$stream_input_adapter@D@__crt_stdio_input@@@0@_K@Z 0000000180071bb0     libucrt:input.obj
 0002:0001bbc4       $unwind$?common_ftell_translated_utf8_nolock@@YA_JV__crt_stdio_stream@@_J@Z 0000000180071bc4     libucrt:ftell.obj
 0002:0001bbec       $unwind$?common_ftell_read_mode_nolock@@YA_JV__crt_stdio_stream@@_J1@Z 0000000180071bec     libucrt:ftell.obj
 0002:0001bc04       $unwind$??$common_ftell@_J@@YA_JV__crt_stdio_stream@@@Z 0000000180071c04     libucrt:ftell.obj
 0002:0001bc28       $unwind$?common_fseek@@YAHV__crt_stdio_stream@@_JH@Z 0000000180071c28     libucrt:fseek.obj
 0002:0001bc50       $unwind$??$common_getenv@_W@@YAPEA_WQEB_W@Z 0000000180071c50     libucrt:getenv.obj
 0002:0001bc70       $unwind$??$common_dupenv_s@_W@@YAHQEAPEA_WQEA_KQEB_WHQEBDH@Z 0000000180071c70     libucrt:getenv.obj
 0002:0001bcb0       $unwind$_wsystem           0000000180071cb0     libucrt:system.obj
 0002:0001bcc8       $unwind$?common_exit@@YAXHW4_crt_exit_cleanup_mode@@W4_crt_exit_return_mode@@@Z 0000000180071cc8     libucrt:exit.obj
 0002:0001bcd4       $unwind$??R<lambda_6e4b09c48022b2350581041d5f6b0c4c>@@QEBA@XZ 0000000180071cd4     libucrt:exit.obj
 0002:0001bcf4       $unwind$??$?RV<lambda_d80eeec6fff315bfe5c115232f3240e3>@@AEAV<lambda_6e4b09c48022b2350581041d5f6b0c4c>@@V<lambda_2358e3775559c9db80273638284d5e45>@@@?$__crt_seh_guarded_call@X@@QEAAX$$QEAV<lambda_d80eeec6fff315bfe5c115232f3240e3>@@AEAV<lambda_6e4b09c48022b2350581041d5f6b0c4c>@@$$QEAV<lambda_2358e3775559c9db80273638284d5e45>@@@Z 0000000180071cf4     libucrt:exit.obj
 0002:0001bd18       $unwind$_configure_narrow_argv 0000000180071d18     libucrt:argv_parsing.obj
 0002:0001bd2c       $unwind$??$free_environment@D@@YAXQEAPEAD@Z 0000000180071d2c     libucrt:environment_initialization.obj
 0002:0001bd2c       $unwind$??$free_environment@_W@@YAXQEAPEA_W@Z 0000000180071d2c     libucrt:environment_initialization.obj
 0002:0001bd38       $unwind$??$create_environment@D@@YAQEAPEADQEAD@Z 0000000180071d38     libucrt:environment_initialization.obj
 0002:0001bd38       $unwind$??$create_environment@_W@@YAQEAPEA_WQEA_W@Z 0000000180071d38     libucrt:environment_initialization.obj
 0002:0001bd50       $unwind$_execute_onexit_table 0000000180071d50     libucrt:onexit.obj
 0002:0001bd58       $unwind$??$?RV<lambda_7777bce6b2f8c936911f934f8298dc43>@@AEAV<lambda_f03950bc5685219e0bcd2087efbe011e>@@V<lambda_3883c3dff614d5e0c5f61bb1ac94921c>@@@?$__crt_seh_guarded_call@H@@QEAAH$$QEAV<lambda_7777bce6b2f8c936911f934f8298dc43>@@AEAV<lambda_f03950bc5685219e0bcd2087efbe011e>@@$$QEAV<lambda_3883c3dff614d5e0c5f61bb1ac94921c>@@@Z 0000000180071d58     libucrt:onexit.obj
 0002:0001bd7c       $unwind$terminate          0000000180071d7c     libucrt:terminate.obj
 0002:0001bd9c       $unwind$?_strupr_s_l_stat@@YAHQEAD_KQEAU__crt_locale_pointers@@@Z 0000000180071d9c     libucrt:strupr.obj
 0002:0001bdc0       $unwind$??$parse_integer@KV?$c_string_character_source@D@__crt_strtox@@@__crt_strtox@@YAKQEAU__crt_locale_pointers@@V?$c_string_character_source@D@0@H_N@Z 0000000180071dc0     libucrt:atox.obj
 0002:0001bddc       $unwind$__acrt_call_reportfault 0000000180071ddc     libucrt:invalid_parameter.obj
 0002:0001bdfc       $unwind$_free_base         0000000180071dfc     libucrt:free_base.obj
 0002:0001bdfc       $unwind$?destroy_fls@@YAXPEAX@Z 0000000180071dfc     libucrt:per_thread_data.obj
 0002:0001bdfc       $unwind$__acrt_locale_free_numeric 0000000180071dfc     libucrt:initnum.obj
 0002:0001bdfc       $unwind$__acrt_locale_free_lc_time_if_unreferenced 0000000180071dfc     libucrt:locale_refcounting.obj
 0002:0001be04       $unwind$?fp_format_e@@YAHQEBNQEAD_K12H_NIQEAU__crt_locale_pointers@@@Z 0000000180071e04     libucrt:cvt.obj
 0002:0001be04       $unwind$_mbtowc_l          0000000180071e04     libucrt:mbtowc.obj
 0002:0001be04       $unwind$__acrt_CompareStringEx 0000000180071e04     libucrt:winapi_thunks.obj
 0002:0001be04       $unwind$__acrt_LCMapStringEx 0000000180071e04     libucrt:winapi_thunks.obj
 0002:0001be04       $unwind$__acrt_LCMapStringW 0000000180071e04     libucrt:lcmapstringw.obj
 0002:0001be04       $unwind$_wcsnicoll_l       0000000180071e04     libucrt:wcsnicol.obj
 0002:0001be18       $unwind$_wctomb_s_l        0000000180071e18     libucrt:wctomb.obj
 0002:0001be28       $unwind$?construct_ptd_array@@YAXQEAU__acrt_ptd@@@Z 0000000180071e28     libucrt:per_thread_data.obj
 0002:0001be30       $unwind$?destroy_ptd_array@@YAXQEAU__acrt_ptd@@@Z 0000000180071e30     libucrt:per_thread_data.obj
 0002:0001be38       $unwind$??$?RV<lambda_0ae27a3a962d80f24befdcbee591983d>@@AEAV<lambda_8d0ee55de4b1038c4002e0adecdf1839>@@V<lambda_dc504788e8f1664fe9b84e20bfb512f2>@@@?$__crt_seh_guarded_call@X@@QEAAX$$QEAV<lambda_0ae27a3a962d80f24befdcbee591983d>@@AEAV<lambda_8d0ee55de4b1038c4002e0adecdf1839>@@$$QEAV<lambda_dc504788e8f1664fe9b84e20bfb512f2>@@@Z 0000000180071e38     libucrt:per_thread_data.obj
 0002:0001be5c       $unwind$??$?RV<lambda_aa87e3671a710a21b5dc78c0bdf72e11>@@AEAV<lambda_92619d2358a28f41a33ba319515a20b9>@@V<lambda_6992ecaafeb10aed2b74cb1fae11a551>@@@?$__crt_seh_guarded_call@X@@QEAAX$$QEAV<lambda_aa87e3671a710a21b5dc78c0bdf72e11>@@AEAV<lambda_92619d2358a28f41a33ba319515a20b9>@@$$QEAV<lambda_6992ecaafeb10aed2b74cb1fae11a551>@@@Z 0000000180071e5c     libucrt:per_thread_data.obj
 0002:0001be80       $unwind$??$?RV<lambda_f2e299630e499de9f9a165e60fcd3db5>@@AEAV<lambda_2ae9d31cdba2644fcbeaf08da7c24588>@@V<lambda_40d01ff24d0e7b3814fdbdcee8eab3c7>@@@?$__crt_seh_guarded_call@X@@QEAAX$$QEAV<lambda_f2e299630e499de9f9a165e60fcd3db5>@@AEAV<lambda_2ae9d31cdba2644fcbeaf08da7c24588>@@$$QEAV<lambda_40d01ff24d0e7b3814fdbdcee8eab3c7>@@@Z 0000000180071e80     libucrt:per_thread_data.obj
 0002:0001bea4       $unwind$??$?RV<lambda_2d41944a1d46af3157314b8a01080d33>@@AEAV<lambda_8f455de75cd7d7f24b4096f044d8b9e6>@@V<lambda_aa500f224e6afead328df44964fe2772>@@@?$__crt_seh_guarded_call@X@@QEAAX$$QEAV<lambda_2d41944a1d46af3157314b8a01080d33>@@AEAV<lambda_8f455de75cd7d7f24b4096f044d8b9e6>@@$$QEAV<lambda_aa500f224e6afead328df44964fe2772>@@@Z 0000000180071ea4     libucrt:per_thread_data.obj
 0002:0001bec8       $unwind$__acrt_fp_format   0000000180071ec8     libucrt:cvt.obj
 0002:0001bedc       $unwind$?fp_format_e_internal@@YAHQEAD_KH_NIQEAU_strflt@@2QEAU__crt_locale_pointers@@@Z 0000000180071edc     libucrt:cvt.obj
 0002:0001bef4       $unwind$?fp_format_a@@YAHQEBNPEAD_KQEAD2H_NIQEAU__crt_locale_pointers@@@Z 0000000180071ef4     libucrt:cvt.obj
 0002:0001bf10       $unwind$?fp_format_g@@YAHQEBNQEAD_K12H_NIQEAU__crt_locale_pointers@@@Z 0000000180071f10     libucrt:cvt.obj
 0002:0001bf24       $unwind$__acrt_stdio_end_temporary_buffering_nolock 0000000180071f24     libucrt:_sftbuf.obj
 0002:0001bf2c       $unwind$__acrt_uninitialize_locale 0000000180071f2c     libucrt:wsetlocale.obj
 0002:0001bf2c       $unwind$__acrt_get_sigabrt_handler 0000000180071f2c     libucrt:signal.obj
 0002:0001bf34       $unwind$??$?RV<lambda_410d79af7f07d98d83a3f525b3859a53>@@AEAV<lambda_3e16ef9562a7dcce91392c22ab16ea36>@@V<lambda_38119f0e861e05405d8a144b9b982f0a>@@@?$__crt_seh_guarded_call@X@@QEAAX$$QEAV<lambda_410d79af7f07d98d83a3f525b3859a53>@@AEAV<lambda_3e16ef9562a7dcce91392c22ab16ea36>@@$$QEAV<lambda_38119f0e861e05405d8a144b9b982f0a>@@@Z 0000000180071f34     libucrt:wsetlocale.obj
 0002:0001bf5c       $unwind$__acrt_initialize_lowio 0000000180071f5c     libucrt:ioinit.obj
 0002:0001bf7c       $unwind$?initialize_inherited_file_handles_nolock@@YAXXZ 0000000180071f7c     libucrt:ioinit.obj
 0002:0001bf98       $unwind$_close             0000000180071f98     libucrt:close.obj
 0002:0001bf98       $unwind$_commit            0000000180071f98     libucrt:commit.obj
 0002:0001bfa0       $unwind$??$?RV<lambda_751a882b2c74d4b022dec766aa51a29a>@@AEAV<lambda_628dfdc04ba53c8bfc02c9951375f3f5>@@V<lambda_f6c7be5f7998530c34de24c7437d6b54>@@@?$__crt_seh_guarded_call@H@@QEAAH$$QEAV<lambda_751a882b2c74d4b022dec766aa51a29a>@@AEAV<lambda_628dfdc04ba53c8bfc02c9951375f3f5>@@$$QEAV<lambda_f6c7be5f7998530c34de24c7437d6b54>@@@Z 0000000180071fa0     libucrt:close.obj
 0002:0001bfc4       $unwind$?__acrt_stdio_allocate_stream@@YA?AV__crt_stdio_stream@@XZ 0000000180071fc4     libucrt:stream.obj
 0002:0001bfe8       $xdatasym                  0000000180071fe8     libucrt:fpsr.obj
 0002:0001bff0       $unwind$_wopenfile         0000000180071ff0     libucrt:openfile.obj
 0002:0001c004       $unwind$_fcloseall         0000000180072004     libucrt:closeall.obj
 0002:0001c028       $unwind$??$common_lseek@J@@YAJHJH@Z 0000000180072028     libucrt:lseek.obj
 0002:0001c058       $unwind$??$common_lseek@_J@@YA_JH_JH@Z 0000000180072058     libucrt:lseek.obj
 0002:0001c088       $unwind$_read              0000000180072088     libucrt:read.obj
 0002:0001c0b8       $unwind$_read_nolock       00000001800720b8     libucrt:read.obj
 0002:0001c0d0       $unwind$?translate_ansi_or_utf8_nolock@@YAHHQEAD_KQEA_W1@Z 00000001800720d0     libucrt:read.obj
 0002:0001c0ec       $unwind$??$translate_text_mode_nolock@D@@YAHHQEAD_K@Z 00000001800720ec     libucrt:read.obj
 0002:0001c104       $unwind$??$translate_text_mode_nolock@_W@@YAHHQEA_W_K@Z 0000000180072104     libucrt:read.obj
 0002:0001c11c       $unwind$_towlower_l        000000018007211c     libucrt:towlower.obj
 0002:0001c124       $unwind$_isctype_l         0000000180072124     libucrt:isctype.obj
 0002:0001c140       $unwind$_waccess_s         0000000180072140     libucrt:waccess.obj
 0002:0001c150       $unwind$_pipe              0000000180072150     libucrt:pipe.obj
 0002:0001c190       $unwind$??$common_fdopen@_W@@YAPEAU_iobuf@@HQEB_W@Z 0000000180072190     libucrt:fdopen.obj
 0002:0001c1b0       $unwind$??$?RV<lambda_a37b2b86f63e897a80ea819b0eb08c01>@@AEAV<lambda_38ce7e780aa69e748d6df282ebc68efe>@@V<lambda_99fb1378e971ab6e7edea83e3a7a83a2>@@@?$__crt_seh_guarded_call@H@@QEAAH$$QEAV<lambda_a37b2b86f63e897a80ea819b0eb08c01>@@AEAV<lambda_38ce7e780aa69e748d6df282ebc68efe>@@$$QEAV<lambda_99fb1378e971ab6e7edea83e3a7a83a2>@@@Z 00000001800721b0     libucrt:commit.obj
 0002:0001c1d4       $unwind$_write             00000001800721d4     libucrt:write.obj
 0002:0001c204       $unwind$_write_nolock      0000000180072204     libucrt:write.obj
 0002:0001c21c       $unwind$?write_double_translated_ansi_nolock@@YA?AUwrite_result@?A0x17268360@@HQEBDI@Z 000000018007221c     libucrt:write.obj
 0002:0001c240       $unwind$?write_text_ansi_nolock@@YA?AUwrite_result@?A0x17268360@@HQEBDI@Z 0000000180072240     libucrt:write.obj
 0002:0001c240       $unwind$?write_text_utf16le_nolock@@YA?AUwrite_result@?A0x17268360@@HQEBDI@Z 0000000180072240     libucrt:write.obj
 0002:0001c260       $unwind$?write_text_utf8_nolock@@YA?AUwrite_result@?A0x17268360@@HQEBDI@Z 0000000180072260     libucrt:write.obj
 0002:0001c284       $unwind$__acrt_GetTempPathA 0000000180072284     libucrt:gettemppath.obj
 0002:0001c29c       $unwind$_sopen_nolock      000000018007229c     libucrt:open.obj
 0002:0001c2b8       $unwind$_wsopen_nolock     00000001800722b8     libucrt:open.obj
 0002:0001c2d8       $unwind$??$common_sopen_dispatch@D@@YAHQEBDHHHQEAHH@Z 00000001800722d8     libucrt:open.obj
 0002:0001c2fc       $unwind$?fin$0@?0???$common_sopen_dispatch@D@@YAHQEBDHHHQEAHH@Z@4HA 00000001800722fc     libucrt:open.obj
 0002:0001c2fc       $unwind$?fin$0@?0???$common_sopen_dispatch@_W@@YAHQEB_WHHHQEAHH@Z@4HA 00000001800722fc     libucrt:open.obj
 0002:0001c304       $unwind$??$common_sopen_dispatch@_W@@YAHQEB_WHHHQEAHH@Z 0000000180072304     libucrt:open.obj
 0002:0001c328       $unwind$_rmtmp             0000000180072328     libucrt:rmtmp.obj
 0002:0001c35c       $unwind$??$write_buffer_nolock@D@@YA_NDV__crt_stdio_stream@@@Z 000000018007235c     libucrt:_flsbuf.obj
 0002:0001c36c       $unwind$?accumulate_inheritable_handles@@YA_NQEAPEAEQEA_K_N@Z 000000018007236c     libucrt:spawnv.obj
 0002:0001c374       $unwind$??R<lambda_f9f2d660215b636168e2032e31cf969c>@@QEBA_NXZ 0000000180072374     libucrt:spawnv.obj
 0002:0001c390       $unwind$??$common_spawnv@_W@@YA_JHQEB_WQEBQEB_W1@Z 0000000180072390     libucrt:spawnv.obj
 0002:0001c3ac       $unwind$??$?RV<lambda_24016bbcb8f60cbe41e899a2382ed12a>@@AEAV<lambda_f9f2d660215b636168e2032e31cf969c>@@V<lambda_7fbd5cec917a4378cbcd803f78c7a734>@@@?$__crt_seh_guarded_call@_N@@QEAA_N$$QEAV<lambda_24016bbcb8f60cbe41e899a2382ed12a>@@AEAV<lambda_f9f2d660215b636168e2032e31cf969c>@@$$QEAV<lambda_7fbd5cec917a4378cbcd803f78c7a734>@@@Z 00000001800723ac     libucrt:spawnv.obj
 0002:0001c3d0       $unwind$??$execute_command@_W@@YA_JHQEB_WQEBQEB_W1@Z 00000001800723d0     libucrt:spawnv.obj
 0002:0001c3ec       $unwind$??$common_spawnvp@_W@@YA_JHQEB_WQEBQEB_W1@Z 00000001800723ec     libucrt:spawnvp.obj
 0002:0001c40c       $unwind$??$common_expand_argv_wildcards@D@@YAHQEAPEADQEAPEAPEAD@Z 000000018007240c     libucrt:argv_wildcards.obj
 0002:0001c424       $unwind$??$common_set_variable_in_environment_nolock@_W@@YAHQEA_WH@Z 0000000180072424     libucrt:setenv.obj
 0002:0001c424       $unwind$??$copy_and_add_argument_to_buffer@D@@YAHQEBD0_KAEAV?$argument_list@D@?A0x5f5c8891@@@Z 0000000180072424     libucrt:argv_wildcards.obj
 0002:0001c440       $unwind$??$expand_argument_wildcards@D@@YAHQEAD0AEAV?$argument_list@D@?A0x5f5c8891@@@Z 0000000180072440     libucrt:argv_wildcards.obj
 0002:0001c464       $unwind$__acrt_GetModuleFileNameA 0000000180072464     libucrt:getmodulefilenamea.obj
 0002:0001c480       $unwind$__dcrt_write_console 0000000180072480     libucrt:initcon.obj
 0002:0001c480       $unwind$??$__acrt_wcs_to_mbs_cp@U__crt_win32_buffer_no_resizing@@@@YAHQEB_WAEAV?$__crt_win32_buffer@DU__crt_win32_buffer_no_resizing@@@@I@Z 0000000180072480     libucrt:getmodulefilenamea.obj
 0002:0001c494       $unwind$?update_thread_multibyte_data_internal@@YAPEAU__crt_multibyte_data@@QEAU__acrt_ptd@@QEAPEAU1@@Z 0000000180072494     libucrt:mbctype.obj
 0002:0001c4bc       $unwind$?setmbcp_internal@@YAHH_NQEAU__acrt_ptd@@QEAPEAU__crt_multibyte_data@@@Z 00000001800724bc     libucrt:mbctype.obj
 0002:0001c4cc       $unwind$?setSBUpLow@@YAXPEAU__crt_multibyte_data@@@Z 00000001800724cc     libucrt:mbctype.obj
 0002:0001c4e8       $unwind$??$?RV<lambda_efdfa57d1f175319df784efa44bb7b81>@@AEAV<lambda_5f0a4c1567f8adc6734073e5d1e1b35c>@@V<lambda_2e8a7d3640ea6ccb4c2413664c2db6fd>@@@?$__crt_seh_guarded_call@X@@QEAAX$$QEAV<lambda_efdfa57d1f175319df784efa44bb7b81>@@AEAV<lambda_5f0a4c1567f8adc6734073e5d1e1b35c>@@$$QEAV<lambda_2e8a7d3640ea6ccb4c2413664c2db6fd>@@@Z 00000001800724e8     libucrt:mbctype.obj
 0002:0001c50c       $unwind$?x_ismbbtype_l@@YAHPEAU__crt_locale_pointers@@IHH@Z 000000018007250c     libucrt:ismbbyte.obj
 0002:0001c51c       $unwind$__GSHandlerCheckCommon 000000018007251c     LIBCMT:gshandler.obj
 0002:0001c51c       $unwind$__acrt_WideCharToMultiByte 000000018007251c     libucrt:widechartomultibyte.obj
 0002:0001c524       $unwind$_query_new_handler 0000000180072524     libucrt:new_handler.obj
 0002:0001c544       $unwind$raise              0000000180072544     libucrt:signal.obj
 0002:0001c580       $unwind$??$?RV<lambda_450d765d439847d4c735a33c368b5fc0>@@AEAV<lambda_44731a7d0e6d81c3e6aa82d741081786>@@V<lambda_601a2a7da3b7a96e9554ac7215c4b07c>@@@?$__crt_seh_guarded_call@P6AXH@Z@@QEAAP6AXH@Z$$QEAV<lambda_450d765d439847d4c735a33c368b5fc0>@@AEAV<lambda_44731a7d0e6d81c3e6aa82d741081786>@@$$QEAV<lambda_601a2a7da3b7a96e9554ac7215c4b07c>@@@Z 0000000180072580     libucrt:signal.obj
 0002:0001c5a4       $unwind$__acrt_LCMapStringA 00000001800725a4     libucrt:lcmapstringa.obj
 0002:0001c5b4       $unwind$?__acrt_LCMapStringA_stat@@YAHPEAU__crt_locale_pointers@@PEB_WKPEBDHPEADHHH@Z 00000001800725b4     libucrt:lcmapstringa.obj
 0002:0001c5dc       $unwind$?__mbsrtowcs_utf8@__crt_mbstring@@YA_KPEA_WPEAPEBD_KPEAU_Mbstatet@@@Z 00000001800725dc     libucrt:mbrtowc.obj
 0002:0001c5f4       $unwind$__acrt_update_thread_locale_data 00000001800725f4     libucrt:locale_refcounting.obj
 0002:0001c618       $unwind$__acrt_fltout      0000000180072618     libucrt:cfout.obj
 0002:0001c638       $unwind$__acrt_locale_free_monetary 0000000180072638     libucrt:initmon.obj
 0002:0001c640       $unwind$__acrt_locale_free_time 0000000180072640     libucrt:inittime.obj
 0002:0001c650       $unwind$__acrt_GetStringTypeA 0000000180072650     libucrt:getstringtypea.obj
 0002:0001c678       $unwind$_alloc_osfhnd      0000000180072678     libucrt:osfinfo.obj
 0002:0001c6a8       $unwind$__acrt_lowio_ensure_fh_exists 00000001800726a8     libucrt:osfinfo.obj
 0002:0001c6d4       $unwind$_wcsnicmp_l        00000001800726d4     libucrt:wcsnicmp.obj
 0002:0001c6f0       $unwind$_setmode_nolock    00000001800726f0     libucrt:setmode.obj
 0002:0001c700       $unwind$_putwch_nolock     0000000180072700     libucrt:putwch.obj
 0002:0001c708       $unwind$__acrt_fenv_set_control 0000000180072708     libucrt:_fenvutils.obj
 0002:0001c718       $unwind$__acrt_CompareStringW 0000000180072718     libucrt:comparestringw.obj
 0002:0001c730       $unwind$__acrt_pack_wide_command_line_and_environment 0000000180072730     libucrt:cenvarg.obj
 0002:0001c74c       $unwind$??$construct_environment_block@_W@@YAHQEBQEB_WQEAPEA_W@Z 000000018007274c     libucrt:cenvarg.obj
 0002:0001c76c       $unwind$qsort              000000018007276c     libucrt:qsort.obj
 0002:0001c784       $chain$4$qsort             0000000180072784     libucrt:qsort.obj
 0002:0001c7a8       $chain$5$qsort             00000001800727a8     libucrt:qsort.obj
 0002:0001c7b8       $unwind$?__mbrtoc32_utf8@__crt_mbstring@@YA_KPEA_UPEBD_KPEAU_Mbstatet@@@Z 00000001800727b8     libucrt:mbrtoc32.obj
 0002:0001c7d8       $xdatasym                  00000001800727d8     libucrt:log10.obj
 0002:0001c7e4       $unwind$_call_matherr      00000001800727e4     libucrt:libm_error.obj
 0002:0001c7ec       $unwind$_handle_error      00000001800727ec     libucrt:libm_error.obj
 0002:0001c80c       $unwind$__acrt_initialize_fma3 000000018007280c     libucrt:fma3_available.obj
 0002:0001c814       $unwind$_log_special_common 0000000180072814     libucrt:log_special.obj
 0002:0001c820       $unwind$_raise_exc         0000000180072820     libucrt:fpexcept.obj
 0002:0001c828       $unwind$_raise_exc_ex      0000000180072828     libucrt:fpexcept.obj
 0002:0001c83c       $unwind$_ctrlfp            000000018007283c     libucrt:fpctrl.obj
 0002:0001c864       $unwind$_IsNonwritableInCurrentImage 0000000180072864     LIBCMT:pesect.obj
 0002:0001c888       $xdatasym                  0000000180072888     LIBCMT:chkstk.obj
 0002:0001c890       $unwind$_local_unwind      0000000180072890     libvcruntime:jmpuwind.obj
 0002:0001c898       $xdatasym                  0000000180072898     libvcruntime:memcmp.obj
 0002:0001c8a0       $xdatasym                  00000001800728a0     libvcruntime:memchr.obj
 0002:0001c8a8       $xdatasym                  00000001800728a8     libucrt:strcmp.obj
 0002:0001c8b0       .edata                     00000001800728b0     luafar3.exp
 0002:0001c8d8       rgpv                       00000001800728d8     luafar3.exp
 0002:0001c984       rgszName                   0000000180072984     luafar3.exp
 0002:0001ca30       rgwOrd                     0000000180072a30     luafar3.exp
 0002:0001ca86       szName                     0000000180072a86     luafar3.exp
 0002:0001ca92       $N00001                    0000000180072a92     luafar3.exp
 0002:0001ca9d       $N00002                    0000000180072a9d     luafar3.exp
 0002:0001caad       $N00003                    0000000180072aad     luafar3.exp
 0002:0001cabb       $N00004                    0000000180072abb     luafar3.exp
 0002:0001cac6       $N00005                    0000000180072ac6     luafar3.exp
 0002:0001cad3       $N00006                    0000000180072ad3     luafar3.exp
 0002:0001cae2       $N00007                    0000000180072ae2     luafar3.exp
 0002:0001caed       $N00008                    0000000180072aed     luafar3.exp
 0002:0001caf7       $N00009                    0000000180072af7     luafar3.exp
 0002:0001cb02       $N00010                    0000000180072b02     luafar3.exp
 0002:0001cb15       $N00011                    0000000180072b15     luafar3.exp
 0002:0001cb25       $N00012                    0000000180072b25     luafar3.exp
 0002:0001cb37       $N00013                    0000000180072b37     luafar3.exp
 0002:0001cb4b       $N00014                    0000000180072b4b     luafar3.exp
 0002:0001cb57       $N00015                    0000000180072b57     luafar3.exp
 0002:0001cb66       $N00016                    0000000180072b66     luafar3.exp
 0002:0001cb77       $N00017                    0000000180072b77     luafar3.exp
 0002:0001cb87       $N00018                    0000000180072b87     luafar3.exp
 0002:0001cb9b       $N00019                    0000000180072b9b     luafar3.exp
 0002:0001cbac       $N00020                    0000000180072bac     luafar3.exp
 0002:0001cbb4       $N00021                    0000000180072bb4     luafar3.exp
 0002:0001cbc5       $N00022                    0000000180072bc5     luafar3.exp
 0002:0001cbd6       $N00023                    0000000180072bd6     luafar3.exp
 0002:0001cbe2       $N00024                    0000000180072be2     luafar3.exp
 0002:0001cbf3       $N00025                    0000000180072bf3     luafar3.exp
 0002:0001cc04       $N00026                    0000000180072c04     luafar3.exp
 0002:0001cc0f       $N00027                    0000000180072c0f     luafar3.exp
 0002:0001cc17       $N00028                    0000000180072c17     luafar3.exp
 0002:0001cc2e       $N00029                    0000000180072c2e     luafar3.exp
 0002:0001cc44       $N00030                    0000000180072c44     luafar3.exp
 0002:0001cc5a       $N00031                    0000000180072c5a     luafar3.exp
 0002:0001cc70       $N00032                    0000000180072c70     luafar3.exp
 0002:0001cc82       $N00033                    0000000180072c82     luafar3.exp
 0002:0001cc95       $N00034                    0000000180072c95     luafar3.exp
 0002:0001ccaa       $N00035                    0000000180072caa     luafar3.exp
 0002:0001ccbf       $N00036                    0000000180072cbf     luafar3.exp
 0002:0001ccd6       $N00037                    0000000180072cd6     luafar3.exp
 0002:0001ccec       $N00038                    0000000180072cec     luafar3.exp
 0002:0001ccf8       $N00039                    0000000180072cf8     luafar3.exp
 0002:0001cd0c       $N00040                    0000000180072d0c     luafar3.exp
 0002:0001cd1d       $N00041                    0000000180072d1d     luafar3.exp
 0002:0001cd2d       $N00042                    0000000180072d2d     luafar3.exp
 0002:0001cd3c       $N00043                    0000000180072d3c     luafar3.exp
 0002:0001d9a0       .idata$6                   00000001800739a0     kernel32:KERNEL32.dll
 0002:0001da46       .idata$6                   0000000180073a46     advapi32:ADVAPI32.dll
 0002:0001da62       .idata$6                   0000000180073a62     user32:USER32.dll
 0002:0001da92       .idata$6                   0000000180073a92     shell32:SHELL32.dll
 0002:0001dae0       .idata$6                   0000000180073ae0     rpcrt4:RPCRT4.dll
 0002:0001e088       .idata$6                   0000000180074088     lua51:lua51.dll
 0003:00000030       ?__vcrt_flsindex@@3KA      0000000180075030     libvcruntime:per_thread_data.obj
 0003:00000040       ?dazSupported@?1??common_control87@@9@9 0000000180075040     libucrt:ieee.obj
 0003:00000158       ?errno_no_memory@@3HA      0000000180075158     libucrt:errno.obj
 0003:0000015c       ?doserrno_no_memory@@3KA   000000018007515c     libucrt:errno.obj
 0003:00000164       ?__acrt_flsindex@@3KA      0000000180075164     libucrt:per_thread_data.obj
 0003:00000670       _mbctypes                  0000000180075670     libucrt:mbctype.obj
 0003:00000780       _mbcasemaps                0000000180075780     libucrt:mbctype.obj
 0003:00000880       ?__rgctypeflag@@3PADA      0000000180075880     libucrt:mbctype.obj
 0003:00000890       ?__rgcode_page_info@@3PAUcode_page_info@@A 0000000180075890     libucrt:mbctype.obj
 0003:00000a30       ?__dcrt_lowio_console_output_handle@@3PEAXEA 0000000180075a30     libucrt:initcon.obj
 0003:00000a40       ?dazSupported@?1??_ctrlfp@@9@9 0000000180075a40     libucrt:fpctrl.obj
 0003:00000a60       unprintable_table          0000000180075a60     lutf8lib.obj
 0003:00000b20       tolower_table              0000000180075b20     lutf8lib.obj
 0003:00001600       alpha_table                0000000180076600     lutf8lib.obj
 0003:00003520       doublewidth_table          0000000180078520     lutf8lib.obj
 0003:00003a10       toupper_table              0000000180078a10     lutf8lib.obj
 0003:000045d0       xdigit_table               00000001800795d0     lutf8lib.obj
 0003:00004620       upper_table                0000000180079620     lutf8lib.obj
 0003:00004d30       digit_table                0000000180079d30     lutf8lib.obj
 0003:00005010       cntrl_table                000000018007a010     lutf8lib.obj
 0003:00005140       compose_table              000000018007a140     lutf8lib.obj
 0003:00005f80       totitle_table              000000018007af80     lutf8lib.obj
 0003:00006b60       alnum_extend_table         000000018007bb60     lutf8lib.obj
 0003:00007190       graph_table                000000018007c190     lutf8lib.obj
 0003:00009710       lower_table                000000018007e710     lutf8lib.obj
 0003:00009ec0       tofold_table               000000018007eec0     lutf8lib.obj
 0003:0000aae0       punct_table                000000018007fae0     lutf8lib.obj
 0003:0000b4a0       space_table                00000001800804a0     lutf8lib.obj
 0003:0000b500       ambiwidth_table            0000000180080500     lutf8lib.obj
 0003:0000bba0       GS_ExceptionRecord         0000000180080ba0     LIBCMT:gs_report.obj
 0003:0000bc40       GS_ContextRecord           0000000180080c40     LIBCMT:gs_report.obj
 0003:0000c110       ?__proc_attached@@3HA      0000000180081110     LIBCMT:dll_dllmain.obj
 0003:0000c140       ?is_initialized_as_dll@@3_NA 0000000180081140     LIBCMT:utility.obj
 0003:0000c141       ?module_local_atexit_table_initialized@@3_NA 0000000180081141     LIBCMT:utility.obj
 0003:0000c148       ?module_local_atexit_table@@3U_onexit_table_t@@A 0000000180081148     LIBCMT:utility.obj
 0003:0000c160       ?module_local_at_quick_exit_table@@3U_onexit_table_t@@A 0000000180081160     LIBCMT:utility.obj
 0003:0000c1d8       ?heap@@3V_HeapManager@@A   00000001800811d8     libvcruntime:undname.obj
 0003:0000c200       ?__vcrt_startup_thread_ptd@@3U__vcrt_ptd@@A 0000000180081200     libvcruntime:per_thread_data.obj
 0003:0000c280       __vcrt_lock_table          0000000180081280     libvcruntime:locks.obj
 0003:0000c2a8       __vcrt_locks_initialized   00000001800812a8     libvcruntime:locks.obj
 0003:0000c2b0       ?module_handles@@3PAPEAUHINSTANCE__@@A 00000001800812b0     libvcruntime:winapi_downlevel.obj
 0003:0000c2c8       ?function_pointers@@3PAPEAXA 00000001800812c8     libvcruntime:winapi_downlevel.obj
 0003:0000c310       ?__idtabsiz@@3IA           0000000180081310     libucrt:popen.obj
 0003:0000c318       ?__idpairs@@3PEAUprocess_handle_pair@?A0xe43b7539@@EA 0000000180081318     libucrt:popen.obj
 0003:0000c320       ?narrow_tmpfile_buffer_pointers@@3PAPEADA 0000000180081320     libucrt:tmpfile.obj
 0003:0000c338       ?wide_tmpfile_buffer_pointers@@3PAPEA_WA 0000000180081338     libucrt:tmpfile.obj
 0003:0000c350       ?c_termination_complete@@3JA 0000000180081350     libucrt:exit.obj
 0003:0000c358       ?thread_local_exit_callback_func@@3P6AXPEAXK0@ZEA 0000000180081358     libucrt:exit.obj
 0003:0000c370       ?program_name@?1???$common_configure_argv@D@@YAHW4_crt_argv_mode@@@Z@4PADA 0000000180081370     libucrt:argv_parsing.obj
 0003:0000c4c8       ?__acrt_invalid_parameter_handler@@3V?$dual_state_global@P6AXPEB_W00I_K@Z@__crt_state_management@@A 00000001800814c8     libucrt:invalid_parameter.obj
 0003:0000c4d0       ?internal_state@?1??_mbtowc_l@@9@4U_Mbstatet@@A 00000001800814d0     libucrt:mbtowc.obj
 0003:0000c4d8       ?enable_percent_n@@3_KA    00000001800814d8     libucrt:printf_count_output.obj
 0003:0000c910       ?module_handles@@3PAPEAUHINSTANCE__@@A 0000000180081910     libucrt:winapi_thunks.obj
 0003:0000c9b0       ?encoded_function_pointers@@3PAPEAXA 00000001800819b0     libucrt:winapi_thunks.obj
 0003:0000cac0       ?__acrt_lock_table@@3PAU_RTL_CRITICAL_SECTION@@A 0000000180081ac0     libucrt:locks.obj
 0003:0000ccf0       ?__acrt_locks_initialized@@3IA 0000000180081cf0     libucrt:locks.obj
 0003:0000cd10       ?fSystemSet@@3HA           0000000180081d10     libucrt:mbctype.obj
 0003:0000cd14       ?initialized@?1??__acrt_initialize_multibyte@@9@4_NA 0000000180081d14     libucrt:mbctype.obj
 0003:0000cd50       ?__acrt_new_handler@@3V?$dual_state_global@P6AH_K@Z@__crt_state_management@@A 0000000180081d50     libucrt:new_handler.obj
 0003:0000cd58       ?ctrlc_action@@3V?$dual_state_global@P6AXH@Z@__crt_state_management@@A 0000000180081d58     libucrt:signal.obj
 0003:0000cd60       ?ctrlbreak_action@@3V?$dual_state_global@P6AXH@Z@__crt_state_management@@A 0000000180081d60     libucrt:signal.obj
 0003:0000cd68       ?abort_action@@3V?$dual_state_global@P6AXH@Z@__crt_state_management@@A 0000000180081d68     libucrt:signal.obj
 0003:0000cd70       ?term_action@@3V?$dual_state_global@P6AXH@Z@__crt_state_management@@A 0000000180081d70     libucrt:signal.obj
 0003:0000cd78       ?user_matherr@@3V?$dual_state_global@P6AHPEAU_exception@@@Z@__crt_state_management@@A 0000000180081d78     libucrt:matherr.obj
 0003:0000cd80       ?__acrt_global_new_mode@@3V?$dual_state_global@J@__crt_state_management@@A 0000000180081d80     libucrt:new_mode.obj
 0003:0000cd90       ?internal_pst@?1??__mbrtoc32_utf8@__crt_mbstring@@YA_KPEA_UPEBD_KPEAU_Mbstatet@@@Z@4U3@A 0000000180081d90     libucrt:mbrtoc32.obj
 0003:0000cd98       ?__acrt_app_type@@3W4_crt_app_type@@A 0000000180081d98     libucrt:report_runtime_error.obj
 0003:0000cda8       luaopen_bit                0000000180081da8     service.obj
 0003:0000cdb0       luaopen_ffi                0000000180081db0     service.obj
 0003:0000cdb8       luaopen_jit                0000000180081db8     service.obj
 0005:00000000       MsetTab                    0000000180087000     libvcruntime:memset.obj
 0005:00000050       MoveSmall                  0000000180087050     libvcruntime:memcpy.obj
 0005:00000090       MoveSmallYmm               0000000180087090     libvcruntime:memcpy.obj
 0005:000000b4       MoveSmallYmmNT             00000001800870b4     libvcruntime:memcpy.obj
 0005:000000d8       MoveSmallXmm               00000001800870d8     libvcruntime:memcpy.obj
 0006:00000060       $R000000                   0000000180088060     luafar3.res
